 luafar3

 Timestamp is 5dd49439 (Wed Nov 20 04:17:45 2019)

 Preferred load address is 0000000180000000

 Start         Length     Name                   Class
 0001:00000000 00000008H .CRT$XCA                CODE
 0001:00000008 00000008H .CRT$XCZ                CODE
 0001:00000010 00000008H .CRT$XIA                CODE
 0001:00000018 00000018H .CRT$XIC                CODE
 0001:00000030 00000008H .CRT$XIZ                CODE
 0001:00000038 00000008H .CRT$XPA                CODE
 0001:00000040 00000018H .CRT$XPX                CODE
 0001:00000058 00000008H .CRT$XPXA               CODE
 0001:00000060 00000008H .CRT$XPZ                CODE
 0001:00000068 00000008H .CRT$XTA                CODE
 0001:00000070 00000010H .CRT$XTZ                CODE
 0001:00000078 00000000H .gfids$y                CODE
 0001:00000080 00019ac0H .rdata                  CODE
 0001:00019b40 00000000H .rdata$r                CODE
 0001:00019b40 00000280H .rdata$zzzdbg           CODE
 0001:00019dc0 00000008H .rtc$IAA                CODE
 0001:00019dc8 00000008H .rtc$IZZ                CODE
 0001:00019dd0 00000008H .rtc$TAA                CODE
 0001:00019dd8 00000008H .rtc$TZZ                CODE
 0001:00019de0 00043b30H .text$mn                CODE
 0001:0005d910 00000020H .text$mn$00             CODE
 0001:0005d930 00000490H .text$x                 CODE
 0001:0005ddc0 00003580H .xdata                  CODE
 0001:00061340 00000000H .xdata$x                CODE
 0001:00061340 0000049cH .edata                  CODE
 0002:00000000 0000bf90H .data                   DATA
 0002:0000bf90 00000000H .data$r                 DATA
 0002:0000bf90 00001250H .bss                    DATA
 0003:00000000 00003d44H .pdata                  DATA
 0004:00000000 00000728H .idata$5                DATA
 0004:00000728 00000010H .00cfg                  DATA
 0004:00000738 00000078H .idata$2                DATA
 0004:000007b0 00000018H .idata$3                DATA
 0004:000007c8 00000728H .idata$4                DATA
 0004:00000ef0 00000fceH .idata$6                DATA
 0005:00000000 00000060H .rsrc$01                DATA
 0005:00000060 00000358H .rsrc$02                DATA

  Address         Publics by Value              Rva+Base               Lib:Object

 0000:00000000       __guard_longjmp_count      0000000000000000     <absolute>
 0000:00000000       __guard_iat_table          0000000000000000     <absolute>
 0000:00000000       __guard_fids_count         0000000000000000     <absolute>
 0000:00000000       __hybrid_code_map_count    0000000000000000     <absolute>
 0000:00000000       __hybrid_code_map          0000000000000000     <absolute>
 0000:00000000       __guard_iat_count          0000000000000000     <absolute>
 0000:00000000       __guard_longjmp_table      0000000000000000     <absolute>
 0000:00000000       __volatile_metadata        0000000000000000     <absolute>
 0000:00000000       __enclave_config           0000000000000000     <absolute>
 0000:00000000       ___safe_se_handler_table   0000000000000000     <absolute>
 0000:00000000       ___safe_se_handler_count   0000000000000000     <absolute>
 0000:00000000       __guard_fids_table         0000000000000000     <absolute>
 0000:00000000       __hybrid_auxiliary_iat     0000000000000000     <absolute>
 0000:00000000       __dynamic_value_reloc_table 0000000000000000     <absolute>
 0000:00000100       __guard_flags              0000000000000100     <absolute>
 0000:00000000       __ImageBase                0000000180000000     <linker-defined>
 0001:00000000       __xc_a                     0000000180001000     LIBCMT:initializers.obj
 0001:00000008       __xc_z                     0000000180001008     LIBCMT:initializers.obj
 0001:00000010       __xi_a                     0000000180001010     LIBCMT:initializers.obj
 0001:00000018       __acrt_stdio_initializer   0000000180001018     libucrt:stdio_initializer.obj
 0001:00000020       __acrt_multibyte_initializer 0000000180001020     libucrt:multibyte_initializer.obj
 0001:00000028       __acrt_tran_fma3_initializer 0000000180001028     libucrt:fma3_initializer.obj
 0001:00000030       __xi_z                     0000000180001030     LIBCMT:initializers.obj
 0001:00000038       __xp_a                     0000000180001038     LIBCMT:initializers.obj
 0001:00000040       __acrt_locale_terminator   0000000180001040     libucrt:locale_initializer.obj
 0001:00000048       __acrt_tmpfile_terminator  0000000180001048     libucrt:tmpfile_initializer.obj
 0001:00000050       __dcrt_console_output_terminator 0000000180001050     libucrt:console_output_initializer.obj
 0001:00000058       __acrt_stdio_terminator    0000000180001058     libucrt:stdio_initializer.obj
 0001:00000060       __xp_z                     0000000180001060     LIBCMT:initializers.obj
 0001:00000068       __xt_a                     0000000180001068     LIBCMT:initializers.obj
 0001:00000070       __xt_z                     0000000180001070     LIBCMT:initializers.obj
 0001:00000250       metatable_name             0000000180001250     bit64.obj
 0001:00000260       ??_C@_04JAOJMBA@bnot@      0000000180001260     bit64.obj
 0001:00000268       ??_C@_04BKGNPECA@band@     0000000180001268     bit64.obj
 0001:00000270       ??_C@_03BBBGIIAC@bor@      0000000180001270     bit64.obj
 0001:00000274       ??_C@_04CKCGDDNF@bxor@     0000000180001274     bit64.obj
 0001:0000027c       ??_C@_06ELFGPGBK@lshift@   000000018000127c     bit64.obj
 0001:00000284       ??_C@_06HMLHBBIJ@rshift@   0000000180001284     bit64.obj
 0001:00000290       ??_C@_07JILILBLL@arshift@  0000000180001290     bit64.obj
 0001:00000298       ??_C@_03CLCAEGCJ@new@      0000000180001298     bit64.obj
 0001:0000029c       ??_C@_03BDGOHNNK@add@      000000018000129c     bit64.obj
 0001:000002a0       ??_C@_03KCMAIMAP@sub@      00000001800012a0     bit64.obj
 0001:000002a4       ??_C@_03IMIFIBCN@mul@      00000001800012a4     bit64.obj
 0001:000002a8       ??_C@_03FEJMGOGI@div@      00000001800012a8     bit64.obj
 0001:000002ac       ??_C@_03FFONCNID@mod@      00000001800012ac     bit64.obj
 0001:000002b0       ??_C@_02HIIGGHJB@eq@       00000001800012b0     bit64.obj
 0001:000002b4       ??_C@_02KCAKIFL@lt@        00000001800012b4     bit64.obj
 0001:000002b8       ??_C@_02FJPJILEL@le@       00000001800012b8     bit64.obj
 0001:000002bc       ??_C@_04GPMDFGEJ@type@     00000001800012bc     bit64.obj
 0001:000002c4       ??_C@_05MEHDOBFN@__add@    00000001800012c4     bit64.obj
 0001:000002cc       ??_C@_05HFNNBAII@__sub@    00000001800012cc     bit64.obj
 0001:000002d4       ??_C@_05FLJIBNKK@__mul@    00000001800012d4     bit64.obj
 0001:000002dc       ??_C@_05IDIBPCOP@__div@    00000001800012dc     bit64.obj
 0001:000002e4       ??_C@_05ICPALBAE@__mod@    00000001800012e4     bit64.obj
 0001:000002ec       ??_C@_05MHFNBPAK@__unm@    00000001800012ec     bit64.obj
 0001:000002f4       ??_C@_04GIMIAOHA@__eq@     00000001800012f4     bit64.obj
 0001:000002fc       ??_C@_04BKGOMBLK@__lt@     00000001800012fc     bit64.obj
 0001:00000304       ??_C@_04EJLHOCKK@__le@     0000000180001304     bit64.obj
 0001:00000310       ??_C@_0L@HDFPAPPH@__tostring@ 0000000180001310     bit64.obj
 0001:00000320       ??_C@_09GPALILFO@bad?5int64@ 0000000180001320     bit64.obj
 0001:0000032c       ??_C@_05LLAMLEHD@?$CFI64d@ 000000018000132c     bit64.obj
 0001:00000334       ??_C@_05OALCLICP@bit64@    0000000180001334     bit64.obj
 0001:00000340       __real@433fffffffffffff    0000000180001340     bit64.obj
 0001:00000350       __xmm@80000000000000008000000000000000 0000000180001350     bit64.obj
 0001:00000360       COLLECTOR_FD               0000000180001360     exported.obj
 0001:00000378       COLLECTOR_OPI              0000000180001378     exported.obj
 0001:00000390       COLLECTOR_PI               0000000180001390     exported.obj
 0001:000003a8       KEY_OBJECT                 00000001800013a8     exported.obj
 0001:00000c68       ??_C@_05GFCDIDHO@debug@    0000000180001c68     exported.obj
 0001:00000c70       ??_C@_09GPFEECNC@traceback@ 0000000180001c70     exported.obj
 0001:00000c7c       ??_C@_06NKNNMLDJ@export@   0000000180001c7c     exported.obj
 0001:00000c88       ??_C@_07PCNKBAGB@OnError@  0000000180001c88     exported.obj
 0001:00000c90       ??_C@_0N@NJMIGDDL@CreationTime@ 0000000180001c90     exported.obj
 0001:00000ca0       ??_C@_0P@MFHPCDDH@LastAccessTime@ 0000000180001ca0     exported.obj
 0001:00000cb0       ??_C@_0O@FCFNCAHK@LastWriteTime@ 0000000180001cb0     exported.obj
 0001:00000cc0       ??_C@_0L@FCILKIIG@ChangeTime@ 0000000180001cc0     exported.obj
 0001:00000cd0       ??_C@_08BHIEONMC@FileSize@ 0000000180001cd0     exported.obj
 0001:00000ce0       ??_C@_0P@JBACEJLL@AllocationSize@ 0000000180001ce0     exported.obj
 0001:00000cf0       ??_C@_05BOOEKJH@Flags@     0000000180001cf0     exported.obj
 0001:00000cf8       ??_C@_0O@DLGJHFNH@NumberOfLinks@ 0000000180001cf8     exported.obj
 0001:00000d08       ??_C@_05MHNOECFO@CRC32@    0000000180001d08     exported.obj
 0001:00000d10       ??_C@_08FDCJCDOL@FileName@ 0000000180001d10     exported.obj
 0001:00000d20       ??_C@_0BC@COCBGKAE@AlternateFileName@ 0000000180001d20     exported.obj
 0001:00000d38       ??_C@_0M@OHKMKKDH@Description@ 0000000180001d38     exported.obj
 0001:00000d44       ??_C@_05HDCNEILF@Owner@    0000000180001d44     exported.obj
 0001:00000d50       ??_C@_0BB@OKGMKOG@CustomColumnData@ 0000000180001d50     exported.obj
 0001:00000d64       ??_C@_11LOCGONAA@@         0000000180001d64     exported.obj
 0001:00000d68       ??_C@_08JNHPECBG@UserData@ 0000000180001d68     exported.obj
 0001:00000d78       ??_C@_0M@DFMHDHBL@GetFindData@ 0000000180001d78     exported.obj
 0001:00000d88       ??_C@_08FFPEEIHA@GetFiles@ 0000000180001d88     exported.obj
 0001:00000d98       ??_C@_0BC@IECOKJFL@GetFiles?4DestPath@ 0000000180001d98     exported.obj
 0001:00000dac       ??_C@_05LFOKGKBN@?$DMboot@ 0000000180001dac     exported.obj
 0001:00000db4       ??_C@_15CBMDENPJ@?$AA?4?$AA?9@ 0000000180001db4     exported.obj
 0001:00000dc0       ??_C@_07KNEGBPNO@package@  0000000180001dc0     exported.obj
 0001:00000dc8       ??_C@_07GCEAJMEA@preload@  0000000180001dc8     exported.obj
 0001:00000dd0       ??_C@_19BCNABNAK@?$AA?4?$AAl?$AAu?$AAa@ 0000000180001dd0     exported.obj
 0001:00000ddc       ??_C@_13BPINEIPE@?$AAr@    0000000180001ddc     exported.obj
 0001:00000de0       ??_C@_1DC@PABHCCON@?$AAD?$AAe?$AAf?$AAa?$AAu?$AAl?$AAt?$AA?5?$AAs?$AAc?$AAr?$AAi?$AAp?$AAt?$AA?5@ 0000000180001de0     exported.obj
 0001:00000e14       ??_C@_03JEOKDCFP@far@      0000000180001e14     exported.obj
 0001:00000e18       ??_C@_0BE@HCPAIELH@ReloadDefaultScript@ 0000000180001e18     exported.obj
 0001:00000e30       ??_C@_0L@OCPPMCCK@StructSize@ 0000000180001e30     exported.obj
 0001:00000e3c       ??_C@_06LBMCOACO@Buffer@   0000000180001e3c     exported.obj
 0001:00000e44       ??_C@_06EPIAKPGD@OpMode@   0000000180001e44     exported.obj
 0001:00000e50       ??_C@_07GDADDFBD@Analyse@  0000000180001e50     exported.obj
 0001:00000e58       ??_C@_0BB@CKIGBGLB@GetOpenPanelInfo@ 0000000180001e58     exported.obj
 0001:00000e70       ??_C@_08KDMNIFGM@FreeSize@ 0000000180001e70     exported.obj
 0001:00000e80       ??_C@_08PAJOMFPO@HostFile@ 0000000180001e80     exported.obj
 0001:00000e8c       ??_C@_06IBPEEEAJ@CurDir@   0000000180001e8c     exported.obj
 0001:00000e94       ??_C@_06PEPCFMNJ@Format@   0000000180001e94     exported.obj
 0001:00000ea0       ??_C@_0L@CMHIOLLB@PanelTitle@ 0000000180001ea0     exported.obj
 0001:00000eb0       ??_C@_09PMEOAIAA@InfoLines@ 0000000180001eb0     exported.obj
 0001:00000ec0       ??_C@_0BA@BLCGOCOG@InfoLinesNumber@ 0000000180001ec0     exported.obj
 0001:00000ed0       ??_C@_04OJAHODMC@Text@     0000000180001ed0     exported.obj
 0001:00000ed8       ??_C@_04DICKPMGH@Data@     0000000180001ed8     exported.obj
 0001:00000ee0       ??_C@_0L@FPEHOFAI@DescrFiles@ 0000000180001ee0     exported.obj
 0001:00000ef0       ??_C@_0BA@BBOGKOKF@PanelModesArray@ 0000000180001ef0     exported.obj
 0001:00000f00       ??_C@_0BB@LFNABPEF@PanelModesNumber@ 0000000180001f00     exported.obj
 0001:00000f18       ??_C@_0M@KDJPJFOF@ColumnTypes@ 0000000180001f18     exported.obj
 0001:00000f28       ??_C@_0N@ILFJPGHI@ColumnWidths@ 0000000180001f28     exported.obj
 0001:00000f38       ??_C@_0BC@KELOOKNK@StatusColumnTypes@ 0000000180001f38     exported.obj
 0001:00000f50       ??_C@_0BD@DNDIPKDK@StatusColumnWidths@ 0000000180001f50     exported.obj
 0001:00000f68       ??_C@_0N@EHCEJHEE@ColumnTitles@ 0000000180001f68     exported.obj
 0001:00000f78       ??_C@_0P@BEEDPJDK@StartPanelMode@ 0000000180001f78     exported.obj
 0001:00000f88       ??_C@_0O@NIFKFGBJ@StartSortMode@ 0000000180001f88     exported.obj
 0001:00000f98       ??_C@_0P@KMACBLNK@StartSortOrder@ 0000000180001f98     exported.obj
 0001:00000fa8       ??_C@_06ONGFDHIA@KeyBar@   0000000180001fa8     exported.obj
 0001:00000fb0       ??_C@_0P@PKDBPEJI@VirtualKeyCode@ 0000000180001fb0     exported.obj
 0001:00000fc0       ??_C@_0BA@MFFHAKP@ControlKeyState@ 0000000180001fc0     exported.obj
 0001:00000fd0       ??_C@_08DGDJEKCP@LongText@ 0000000180001fd0     exported.obj
 0001:00000fe0       ??_C@_0N@IHDKLODA@ShortcutData@ 0000000180001fe0     exported.obj
 0001:00000ff0       ??_C@_05HIFJDKLD@array@    0000000180001ff0     exported.obj
 0001:00000ff8       ??_C@_01EFFIKLCJ@n@        0000000180001ff8     exported.obj
 0001:00000ffa       ??_C@_00CNPNBAHC@@         0000000180001ffa     exported.obj
 0001:00000ffc       ??_C@_04DNCDCIAE@Open@     0000000180001ffc     exported.obj
 0001:00001004       ??_C@_04OPJIDECA@hDlg@     0000000180002004     exported.obj
 0001:0000100c       ??_C@_06BNNOMDLO@Handle@   000000018000200c     exported.obj
 0001:00001014       ??_C@_05LNOAKADA@panel@    0000000180002014     exported.obj
 0001:00001020       ??_C@_0L@JMPDJFBN@ClosePanel@ 0000000180002020     exported.obj
 0001:00001030       ??_C@_07MBOMJGGF@Compare@  0000000180002030     exported.obj
 0001:00001038       ??_C@_09NANCCILE@Configure@ 0000000180002038     exported.obj
 0001:00001048       ??_C@_0M@MMKKMEFA@DeleteFiles@ 0000000180002048     exported.obj
 0001:00001058       ??_C@_0O@GLLEDHJA@MakeDirectory@ 0000000180002058     exported.obj
 0001:00001068       ??_C@_0BD@PJNONGDB@MakeDirectory?4Name@ 0000000180002068     exported.obj
 0001:00001080       ??_C@_0BC@COPMJGBI@ProcessPanelEvent@ 0000000180002080     exported.obj
 0001:00001098       ??_C@_0BA@DPJAKFGC@ProcessHostFile@ 0000000180002098     exported.obj
 0001:000010a8       ??_C@_0BC@HOBKGBBM@ProcessPanelInput@ 00000001800020a8     exported.obj
 0001:000010c0       ??_C@_08OBOOFGOD@PutFiles@ 00000001800020c0     exported.obj
 0001:000010d0       ??_C@_0N@KCFEBPAO@SetDirectory@ 00000001800020d0     exported.obj
 0001:000010e0       ??_C@_0M@PNOHHCCH@SetFindList@ 00000001800020e0     exported.obj
 0001:000010f0       ??_C@_07EACELFAO@ExitFAR@  00000001800020f0     exported.obj
 0001:000010f8       ??_C@_0O@OBCKADMD@GetPluginInfo@ 00000001800020f8     exported.obj
 0001:00001108       ??_C@_0O@GDMHGAFH@CommandPrefix@ 0000000180002108     exported.obj
 0001:00001118       ??_C@_0O@PHBKMNMJ@DiskMenuGuids@ 0000000180002118     exported.obj
 0001:00001128       ??_C@_0BA@NLBDFPEO@DiskMenuStrings@ 0000000180002128     exported.obj
 0001:00001138       ??_C@_0BA@FOMPNLJF@PluginMenuGuids@ 0000000180002138     exported.obj
 0001:00001148       ??_C@_0BC@DJMJFBJC@PluginMenuStrings@ 0000000180002148     exported.obj
 0001:00001160       ??_C@_0BC@ILBHAHCH@PluginConfigGuids@ 0000000180002160     exported.obj
 0001:00001178       ??_C@_0BE@GAFPNGIP@PluginConfigStrings@ 0000000180002178     exported.obj
 0001:00001190       ??_C@_0BD@DECJPBBK@ProcessEditorInput@ 0000000180002190     exported.obj
 0001:000011a8       ??_C@_0BD@GEMPAGBO@ProcessEditorEvent@ 00000001800021a8     exported.obj
 0001:000011bc       ??_C@_04KOACHJEN@Type@     00000001800021bc     exported.obj
 0001:000011c8       ??_C@_0N@EKPHGDMI@StringNumber@ 00000001800021c8     exported.obj
 0001:000011d8       ??_C@_07MOCFLHCN@FileEOL@  00000001800021d8     exported.obj
 0001:000011e0       ??_C@_08DOHJINHB@CodePage@ 00000001800021e0     exported.obj
 0001:000011f0       ??_C@_0BD@GGKMLEJG@ProcessViewerEvent@ 00000001800021f0     exported.obj
 0001:00001208       ??_C@_0BD@FNHBEIC@ProcessDialogEvent@ 0000000180002208     exported.obj
 0001:0000121c       ??_C@_06CPBJDKAC@Param2@   000000018000221c     exported.obj
 0001:00001224       ??_C@_06EDEGJMB@Param1@    0000000180002224     exported.obj
 0001:0000122c       ??_C@_03MLMOILGK@Msg@      000000018000222c     exported.obj
 0001:00001230       ??_C@_0BE@LHJGGGHN@ProcessSynchroEvent@ 0000000180002230     exported.obj
 0001:00001248       ??_C@_0BB@PHIEFGHD@GetContentFields@ 0000000180002248     exported.obj
 0001:00001260       ??_C@_0P@DPJDPMPI@GetContentData@ 0000000180002260     exported.obj
 0001:00001270       ??_C@_0N@DDJEHLKE@?$DM_globalinfo@ 0000000180002270     exported.obj
 0001:00001280       ??_C@_1CA@IBKDMBNJ@?$AA_?$AAg?$AAl?$AAo?$AAb?$AAa?$AAl?$AAi?$AAn?$AAf?$AAo?$AA?4?$AAl?$AAu?$AAa@ 0000000180002280     exported.obj
 0001:000012a0       ??_C@_0O@GJMOPLGM@GetGlobalInfo@ 00000001800022a0     exported.obj
 0001:000012b0       ??_C@_0O@CALOEOI@MinFarVersion@ 00000001800022b0     exported.obj
 0001:000012c0       ??_C@_07NGFJPNPN@Version@  00000001800022c0     exported.obj
 0001:000012c8       ??_C@_04MJHIICBJ@Guid@     00000001800022c8     exported.obj
 0001:000012d0       ??_C@_05PABKJLOM@Title@    00000001800022d0     exported.obj
 0001:000012d8       ??_C@_06HHECMMLE@Author@   00000001800022d8     exported.obj
 0001:000012e0       ??_C@_0BE@DONMOPMJ@ProcessConsoleInput@ 00000001800022e0     exported.obj
 0001:000012f8       __real@43e0000000000000    00000001800022f8     exported.obj
 0001:00001300       __real@bff0000000000000    0000000180002300     exported.obj
 0001:00001bb0       Vals                       0000000180002bb0     flags.obj
 0001:00003230       ??_C@_0BI@IDKIJMME@FARMANAGERVERSION_MAJOR@ 0000000180004230     flags.obj
 0001:00003248       ??_C@_0BI@DMLKEAFC@FARMANAGERVERSION_MINOR@ 0000000180004248     flags.obj
 0001:00003260       ??_C@_0BL@NMALNAFP@FARMANAGERVERSION_REVISION@ 0000000180004260     flags.obj
 0001:00003280       ??_C@_0BI@OLPFLLDD@FARMANAGERVERSION_BUILD@ 0000000180004280     flags.obj
 0001:00003298       ??_C@_0BI@MOOFLFPC@FARMANAGERVERSION_STAGE@ 0000000180004298     flags.obj
 0001:000032b0       ??_C@_0L@MIDBGFJO@CP_UNICODE@ 00000001800042b0     flags.obj
 0001:000032c0       ??_C@_0O@MNMCMEJH@CP_REVERSEBOM@ 00000001800042c0     flags.obj
 0001:000032d0       ??_C@_0L@JDNPCEDH@CP_DEFAULT@ 00000001800042d0     flags.obj
 0001:000032e0       ??_C@_0M@OMCMFJHA@CP_REDETECT@ 00000001800042e0     flags.obj
 0001:000032f0       ??_C@_09MNAPNKKC@INDEXMASK@ 00000001800042f0     flags.obj
 0001:00003300       ??_C@_09BLFIDJLF@COLORMASK@ 0000000180004300     flags.obj
 0001:00003310       ??_C@_09ENNBLPJC@ALPHAMASK@ 0000000180004310     flags.obj
 0001:00003320       ??_C@_0L@EHFOPLFD@PANEL_NONE@ 0000000180004320     flags.obj
 0001:00003330       ??_C@_0N@LPMKALBG@PANEL_ACTIVE@ 0000000180004330     flags.obj
 0001:00003340       ??_C@_0O@HPKEABPN@PANEL_PASSIVE@ 0000000180004340     flags.obj
 0001:00003350       ??_C@_0L@GOEBPENN@PANEL_STOP@ 0000000180004350     flags.obj
 0001:00003360       ??_C@_0N@HLIFAAPJ@EEREDRAW_ALL@ 0000000180004360     flags.obj
 0001:00003370       ??_C@_0P@NHNDIKJ@CURRENT_EDITOR@ 0000000180004370     flags.obj
 0001:00003380       ??_C@_0BN@PPNDCHHA@EDITOR_COLOR_NORMAL_PRIORITY@ 0000000180004380     flags.obj
 0001:000033a0       ??_C@_07MGGAEAFF@DI_TEXT@  00000001800043a0     flags.obj
 0001:000033a8       ??_C@_08HODBDEHE@DI_VTEXT@ 00000001800043a8     flags.obj
 0001:000033b8       ??_C@_0N@IGKKGFMF@DI_SINGLEBOX@ 00000001800043b8     flags.obj
 0001:000033c8       ??_C@_0N@EDCLIEAE@DI_DOUBLEBOX@ 00000001800043c8     flags.obj
 0001:000033d8       ??_C@_07DOLIFAEF@DI_EDIT@  00000001800043d8     flags.obj
 0001:000033e0       ??_C@_0L@EOMEIIFM@DI_PSWEDIT@ 00000001800043e0     flags.obj
 0001:000033f0       ??_C@_0L@MGOIMBKF@DI_FIXEDIT@ 00000001800043f0     flags.obj
 0001:00003400       ??_C@_09GGAEMAPJ@DI_BUTTON@ 0000000180004400     flags.obj
 0001:00003410       ??_C@_0M@MHFHGPHJ@DI_CHECKBOX@ 0000000180004410     flags.obj
 0001:00003420       ??_C@_0P@GIPCGMBE@DI_RADIOBUTTON@ 0000000180004420     flags.obj
 0001:00003430       ??_C@_0M@MAKBFNGC@DI_COMBOBOX@ 0000000180004430     flags.obj
 0001:00003440       ??_C@_0L@ONDMPPPO@DI_LISTBOX@ 0000000180004440     flags.obj
 0001:00003450       ??_C@_0P@GDJDPEIK@DI_USERCONTROL@ 0000000180004450     flags.obj
 0001:00003460       ??_C@_08KAEGOLOB@DM_FIRST@ 0000000180004460     flags.obj
 0001:00003470       ??_C@_08MJMBFJHA@DM_CLOSE@ 0000000180004470     flags.obj
 0001:00003480       ??_C@_09KLJOCKAA@DM_ENABLE@ 0000000180004480     flags.obj
 0001:00003490       ??_C@_0BA@KAMJGFDG@DM_ENABLEREDRAW@ 0000000180004490     flags.obj
 0001:000034a0       ??_C@_0O@FKGMMKLP@DM_GETDLGDATA@ 00000001800044a0     flags.obj
 0001:000034b0       ??_C@_0O@HEGKCPOI@DM_GETDLGITEM@ 00000001800044b0     flags.obj
 0001:000034c0       ??_C@_0O@BEHCGMCL@DM_GETDLGRECT@ 00000001800044c0     flags.obj
 0001:000034d0       ??_C@_0L@ELBDNLFO@DM_GETTEXT@ 00000001800044d0     flags.obj
 0001:000034dc       ??_C@_06IKGPEGEJ@DM_KEY@   00000001800044dc     flags.obj
 0001:000034e8       ??_C@_0O@DIPLLJEH@DM_MOVEDIALOG@ 00000001800044e8     flags.obj
 0001:000034f8       ??_C@_0O@EEEDHNPG@DM_SETDLGDATA@ 00000001800044f8     flags.obj
 0001:00003508       ??_C@_0O@GKEFJIKB@DM_SETDLGITEM@ 0000000180004508     flags.obj
 0001:00003518       ??_C@_0M@GOFGHDFK@DM_SETFOCUS@ 0000000180004518     flags.obj
 0001:00003528       ??_C@_09ILPFEDOM@DM_REDRAW@ 0000000180004528     flags.obj
 0001:00003538       ??_C@_0L@LDOCOEIP@DM_SETTEXT@ 0000000180004538     flags.obj
 0001:00003548       ??_C@_0BE@LABEAIPD@DM_SETMAXTEXTLENGTH@ 0000000180004548     flags.obj
 0001:00003560       ??_C@_0O@BIFKIPIP@DM_SHOWDIALOG@ 0000000180004560     flags.obj
 0001:00003570       ??_C@_0M@JPHKGACH@DM_GETFOCUS@ 0000000180004570     flags.obj
 0001:00003580       ??_C@_0BA@NLMONBKJ@DM_GETCURSORPOS@ 0000000180004580     flags.obj
 0001:00003590       ??_C@_0BA@KPHABNOF@DM_SETCURSORPOS@ 0000000180004590     flags.obj
 0001:000035a0       ??_C@_0O@LGEKFPKK@DM_SETTEXTPTR@ 00000001800045a0     flags.obj
 0001:000035b0       ??_C@_0M@NCOJHJKI@DM_SHOWITEM@ 00000001800045b0     flags.obj
 0001:000035c0       ??_C@_0O@GKKCFHIM@DM_ADDHISTORY@ 00000001800045c0     flags.obj
 0001:000035d0       ??_C@_0M@MCEMDFMD@DM_GETCHECK@ 00000001800045d0     flags.obj
 0001:000035e0       ??_C@_0M@DDGACGLO@DM_SETCHECK@ 00000001800045e0     flags.obj
 0001:000035f0       ??_C@_0N@MEGOPFGK@DM_SET3STATE@ 00000001800045f0     flags.obj
 0001:00003600       ??_C@_0M@GEPBDDNC@DM_LISTSORT@ 0000000180004600     flags.obj
 0001:00003610       ??_C@_0P@NFJNHAKH@DM_LISTGETITEM@ 0000000180004610     flags.obj
 0001:00003620       ??_C@_0BB@EEIMACNO@DM_LISTGETCURPOS@ 0000000180004620     flags.obj
 0001:00003638       ??_C@_0BB@GKMJCDEM@DM_LISTSETCURPOS@ 0000000180004638     flags.obj
 0001:00003650       ??_C@_0O@NOPCAHGJ@DM_LISTDELETE@ 0000000180004650     flags.obj
 0001:00003660       ??_C@_0L@BMEAECNG@DM_LISTADD@ 0000000180004660     flags.obj
 0001:00003670       ??_C@_0O@HBHDMHP@DM_LISTADDSTR@ 0000000180004670     flags.obj
 0001:00003680       ??_C@_0O@PDFCNPKN@DM_LISTUPDATE@ 0000000180004680     flags.obj
 0001:00003690       ??_C@_0O@GAAGMJJL@DM_LISTINSERT@ 0000000180004690     flags.obj
 0001:000036a0       ??_C@_0BC@MIFCLOBD@DM_LISTFINDSTRING@ 00000001800046a0     flags.obj
 0001:000036b8       ??_C@_0M@EEAEBLKC@DM_LISTINFO@ 00000001800046b8     flags.obj
 0001:000036c8       ??_C@_0P@PLJLJFPA@DM_LISTGETDATA@ 00000001800046c8     flags.obj
 0001:000036d8       ??_C@_0P@DGKKKCB@DM_LISTSETDATA@ 00000001800046d8     flags.obj
 0001:000036e8       ??_C@_0BB@CELMNLLN@DM_LISTSETTITLES@ 00000001800046e8     flags.obj
 0001:00003700       ??_C@_0BB@KPJPKCP@DM_LISTGETTITLES@ 0000000180004700     flags.obj
 0001:00003718       ??_C@_0BA@ICDJCFLE@DM_RESIZEDIALOG@ 0000000180004718     flags.obj
 0001:00003728       ??_C@_0BD@CNGGHGJF@DM_SETITEMPOSITION@ 0000000180004728     flags.obj
 0001:00003740       ??_C@_0BF@JMINBGBA@DM_GETDROPDOWNOPENED@ 0000000180004740     flags.obj
 0001:00003758       ??_C@_0BF@LJIGJNAO@DM_SETDROPDOWNOPENED@ 0000000180004758     flags.obj
 0001:00003770       ??_C@_0O@NPDKADMJ@DM_SETHISTORY@ 0000000180004770     flags.obj
 0001:00003780       ??_C@_0BD@BPHAAEIM@DM_GETITEMPOSITION@ 0000000180004780     flags.obj
 0001:00003798       ??_C@_0BC@BENFKLNH@DM_SETINPUTNOTIFY@ 0000000180004798     flags.obj
 0001:000037b0       ??_C@_0BH@CFMLLNNM@DM_SETMOUSEEVENTNOTIFY@ 00000001800047b0     flags.obj
 0001:000037c8       ??_C@_0BF@IAGIACOD@DM_EDITUNCHANGEDFLAG@ 00000001800047c8     flags.obj
 0001:000037e0       ??_C@_0P@OJKNHIPN@DM_GETITEMDATA@ 00000001800047e0     flags.obj
 0001:000037f0       ??_C@_0P@OGLDKOHO@DM_SETITEMDATA@ 00000001800047f0     flags.obj
 0001:00003800       ??_C@_0L@KNFAKFKE@DM_LISTSET@ 0000000180004800     flags.obj
 0001:00003810       ??_C@_0BB@EPMFHAFO@DM_GETCURSORSIZE@ 0000000180004810     flags.obj
 0001:00003828       ??_C@_0BB@DANLMDCJ@DM_SETCURSORSIZE@ 0000000180004828     flags.obj
 0001:00003840       ??_C@_0BD@LAOOKGHD@DM_LISTGETDATASIZE@ 0000000180004840     flags.obj
 0001:00003858       ??_C@_0BA@BHGANJAP@DM_GETSELECTION@ 0000000180004858     flags.obj
 0001:00003868       ??_C@_0BA@GDNOBFED@DM_SETSELECTION@ 0000000180004868     flags.obj
 0001:00003878       ??_C@_0BD@FIHDGIGO@DM_GETEDITPOSITION@ 0000000180004878     flags.obj
 0001:00003890       ??_C@_0BD@GKGFBKHH@DM_SETEDITPOSITION@ 0000000180004890     flags.obj
 0001:000038a8       ??_C@_0BE@MCECGHBC@DM_SETCOMBOBOXEVENT@ 00000001800048a8     flags.obj
 0001:000038c0       ??_C@_0BE@KGBLNJKA@DM_GETCOMBOBOXEVENT@ 00000001800048c0     flags.obj
 0001:000038d8       ??_C@_0BD@CJEPBACF@DM_GETCONSTTEXTPTR@ 00000001800048d8     flags.obj
 0001:000038f0       ??_C@_0BD@HOOHICEG@DM_GETDLGITEMSHORT@ 00000001800048f0     flags.obj
 0001:00003908       ??_C@_0BD@EMPBPAFP@DM_SETDLGITEMSHORT@ 0000000180004908     flags.obj
 0001:00003920       ??_C@_0BB@GAPFMPKE@DM_GETDIALOGINFO@ 0000000180004920     flags.obj
 0001:00003938       ??_C@_0BC@KJOLMFGG@DM_GETDIALOGTITLE@ 0000000180004938     flags.obj
 0001:00003950       ??_C@_08COMJOMAC@DN_FIRST@ 0000000180004950     flags.obj
 0001:00003960       ??_C@_0M@NNNAPNMA@DN_BTNCLICK@ 0000000180004960     flags.obj
 0001:00003970       ??_C@_0BC@MJFJAANN@DN_CTLCOLORDIALOG@ 0000000180004970     flags.obj
 0001:00003988       ??_C@_0BD@HFGBIBBL@DN_CTLCOLORDLGITEM@ 0000000180004988     flags.obj
 0001:000039a0       ??_C@_0BD@JMFJPHPD@DN_CTLCOLORDLGLIST@ 00000001800049a0     flags.obj
 0001:000039b8       ??_C@_0O@NKBDPILK@DN_DRAWDIALOG@ 00000001800049b8     flags.obj
 0001:000039c8       ??_C@_0P@KGKEDPBI@DN_DRAWDLGITEM@ 00000001800049c8     flags.obj
 0001:000039d8       ??_C@_0O@JMKNGFLE@DN_EDITCHANGE@ 00000001800049d8     flags.obj
 0001:000039e8       ??_C@_0N@OCGKCPJF@DN_ENTERIDLE@ 00000001800049e8     flags.obj
 0001:000039f8       ??_C@_0M@JHFIBKOO@DN_GOTFOCUS@ 00000001800049f8     flags.obj
 0001:00003a08       ??_C@_07NJJEMKPA@DN_HELP@  0000000180004a08     flags.obj
 0001:00003a10       ??_C@_09EDGJFAK@DN_HOTKEY@ 0000000180004a10     flags.obj
 0001:00003a20       ??_C@_0O@BJECHBCA@DN_INITDIALOG@ 0000000180004a20     flags.obj
 0001:00003a30       ??_C@_0N@CHLLLNBO@DN_KILLFOCUS@ 0000000180004a30     flags.obj
 0001:00003a40       ??_C@_0O@CLPABIGO@DN_LISTCHANGE@ 0000000180004a40     flags.obj
 0001:00003a50       ??_C@_0L@MLMFBHN@DN_DRAGGED@ 0000000180004a50     flags.obj
 0001:00003a60       ??_C@_0BB@BOOOCAEG@DN_RESIZECONSOLE@ 0000000180004a60     flags.obj
 0001:00003a78       ??_C@_0BC@FHPPFLKG@DN_DRAWDIALOGDONE@ 0000000180004a78     flags.obj
 0001:00003a90       ??_C@_0O@EONPBNNP@DN_LISTHOTKEY@ 0000000180004a90     flags.obj
 0001:00003aa0       ??_C@_08MDDLDGPO@DN_INPUT@ 0000000180004aa0     flags.obj
 0001:00003ab0       ??_C@_0BA@FGOGLDBC@DN_CONTROLINPUT@ 0000000180004ab0     flags.obj
 0001:00003ac0       ??_C@_08EHEOFOJD@DN_CLOSE@ 0000000180004ac0     flags.obj
 0001:00003ad0       ??_C@_0M@POIFBPFN@DN_GETVALUE@ 0000000180004ad0     flags.obj
 0001:00003ae0       ??_C@_0BC@MHCBFAAO@DN_DROPDOWNOPENED@ 0000000180004ae0     flags.obj
 0001:00003af8       ??_C@_0BD@NGEKAPIF@DN_DRAWDLGITEMDONE@ 0000000180004af8     flags.obj
 0001:00003b10       ??_C@_07DIJJNCBA@DM_USER@  0000000180004b10     flags.obj
 0001:00003b18       ??_C@_0BB@HLBBGMAN@BSTATE_UNCHECKED@ 0000000180004b18     flags.obj
 0001:00003b30       ??_C@_0P@FALAMPGP@BSTATE_CHECKED@ 0000000180004b30     flags.obj
 0001:00003b40       ??_C@_0O@KBIFGGHO@BSTATE_3STATE@ 0000000180004b40     flags.obj
 0001:00003b50       ??_C@_0O@ILJOJGLD@BSTATE_TOGGLE@ 0000000180004b50     flags.obj
 0001:00003b60       ??_C@_08PPADCPCM@CBET_KEY@ 0000000180004b60     flags.obj
 0001:00003b70       ??_C@_0L@KHCLMGFJ@CBET_MOUSE@ 0000000180004b70     flags.obj
 0001:00003b80       ??_C@_0BA@KNHGEBNE@PTYPE_FILEPANEL@ 0000000180004b80     flags.obj
 0001:00003b90       ??_C@_0BA@LPPHNHIG@PTYPE_TREEPANEL@ 0000000180004b90     flags.obj
 0001:00003ba0       ??_C@_0BB@JBINOKAI@PTYPE_QVIEWPANEL@ 0000000180004ba0     flags.obj
 0001:00003bb8       ??_C@_0BA@NKMDEBG@PTYPE_INFOPANEL@ 0000000180004bb8     flags.obj
 0001:00003bc8       ??_C@_0L@OPHJOKKE@SM_DEFAULT@ 0000000180004bc8     flags.obj
 0001:00003bd8       ??_C@_0M@JGBFGGEA@SM_UNSORTED@ 0000000180004bd8     flags.obj
 0001:00003be8       ??_C@_07KIFHAGIL@SM_NAME@  0000000180004be8     flags.obj
 0001:00003bf0       ??_C@_06GJJJNNFE@SM_EXT@   0000000180004bf0     flags.obj
 0001:00003bf8       ??_C@_08FICJBKFN@SM_MTIME@ 0000000180004bf8     flags.obj
 0001:00003c08       ??_C@_08GCCDHLCN@SM_CTIME@ 0000000180004c08     flags.obj
 0001:00003c18       ??_C@_08CPOLNKCG@SM_ATIME@ 0000000180004c18     flags.obj
 0001:00003c28       ??_C@_07OMPKMIKC@SM_SIZE@  0000000180004c28     flags.obj
 0001:00003c30       ??_C@_08BCBPOLMA@SM_DESCR@ 0000000180004c30     flags.obj
 0001:00003c40       ??_C@_08MEAGCMBB@SM_OWNER@ 0000000180004c40     flags.obj
 0001:00003c50       ??_C@_0BC@NKDBNAHD@SM_COMPRESSEDSIZE@ 0000000180004c50     flags.obj
 0001:00003c68       ??_C@_0M@PKNLKFI@SM_NUMLINKS@ 0000000180004c68     flags.obj
 0001:00003c78       ??_C@_0O@CCKEKPHL@SM_NUMSTREAMS@ 0000000180004c78     flags.obj
 0001:00003c88       ??_C@_0P@PKGMDPMD@SM_STREAMSSIZE@ 0000000180004c88     flags.obj
 0001:00003c98       ??_C@_0M@OAFEBGNH@SM_FULLNAME@ 0000000180004c98     flags.obj
 0001:00003ca8       ??_C@_09KFKGJDHC@SM_CHTIME@ 0000000180004ca8     flags.obj
 0001:00003cb8       ??_C@_08DOEDKINA@SM_COUNT@ 0000000180004cb8     flags.obj
 0001:00003cc8       ??_C@_0P@FEMAMJLE@EEC_OPEN_ERROR@ 0000000180004cc8     flags.obj
 0001:00003cd8       ??_C@_0N@GLMELIKF@EEC_MODIFIED@ 0000000180004cd8     flags.obj
 0001:00003ce8       ??_C@_0BB@HALKEFOL@EEC_NOT_MODIFIED@ 0000000180004ce8     flags.obj
 0001:00003d00       ??_C@_0BI@CNPFKHKO@EEC_LOADING_INTERRUPTED@ 0000000180004d00     flags.obj
 0001:00003d18       ??_C@_0BK@PHBCABMB@ACTL_GETFARMANAGERVERSION@ 0000000180004d18     flags.obj
 0001:00003d38       ??_C@_0N@DPABJDML@ACTL_WAITKEY@ 0000000180004d38     flags.obj
 0001:00003d48       ??_C@_0O@CEHHJAFD@ACTL_GETCOLOR@ 0000000180004d48     flags.obj
 0001:00003d58       ??_C@_0BD@OKPAACIK@ACTL_GETARRAYCOLOR@ 0000000180004d58     flags.obj
 0001:00003d70       ??_C@_0BD@DIFEEKNN@ACTL_GETWINDOWINFO@ 0000000180004d70     flags.obj
 0001:00003d88       ??_C@_0BE@PJBIPKOD@ACTL_GETWINDOWCOUNT@ 0000000180004d88     flags.obj
 0001:00003da0       ??_C@_0BG@MNKPOEEN@ACTL_SETCURRENTWINDOW@ 0000000180004da0     flags.obj
 0001:00003db8       ??_C@_0M@IHHFGPPA@ACTL_COMMIT@ 0000000180004db8     flags.obj
 0001:00003dc8       ??_C@_0BA@CLHFKJJP@ACTL_GETFARHWND@ 0000000180004dc8     flags.obj
 0001:00003dd8       ??_C@_0BD@JFOOLBPN@ACTL_SETARRAYCOLOR@ 0000000180004dd8     flags.obj
 0001:00003df0       ??_C@_0P@JECKFIA@ACTL_REDRAWALL@ 0000000180004df0     flags.obj
 0001:00003e00       ??_C@_0N@DHPLJLHO@ACTL_SYNCHRO@ 0000000180004e00     flags.obj
 0001:00003e10       ??_C@_0BG@IJPADENB@ACTL_SETPROGRESSSTATE@ 0000000180004e10     flags.obj
 0001:00003e28       ??_C@_0BG@ICJFAPHK@ACTL_SETPROGRESSVALUE@ 0000000180004e28     flags.obj
 0001:00003e40       ??_C@_09HNDBKLDC@ACTL_QUIT@ 0000000180004e40     flags.obj
 0001:00003e50       ??_C@_0BA@LJCPDIKK@ACTL_GETFARRECT@ 0000000180004e50     flags.obj
 0001:00003e60       ??_C@_0BC@FELBEIDG@ACTL_GETCURSORPOS@ 0000000180004e60     flags.obj
 0001:00003e78       ??_C@_0BC@CAAPIEHK@ACTL_SETCURSORPOS@ 0000000180004e78     flags.obj
 0001:00003e90       ??_C@_0BE@NPJGMDBM@ACTL_PROGRESSNOTIFY@ 0000000180004e90     flags.obj
 0001:00003ea8       ??_C@_0BD@IPKOEBIA@ACTL_GETWINDOWTYPE@ 0000000180004ea8     flags.obj
 0001:00003ec0       ??_C@_09CEDFMINA@MSSC_POST@ 0000000180004ec0     flags.obj
 0001:00003ed0       ??_C@_0L@MOADGAEB@MSSC_CHECK@ 0000000180004ed0     flags.obj
 0001:00003ee0       ??_C@_0BA@MMOAIEKP@MACROAREA_OTHER@ 0000000180004ee0     flags.obj
 0001:00003ef0       ??_C@_0BA@DEBOOAEB@MACROAREA_SHELL@ 0000000180004ef0     flags.obj
 0001:00003f00       ??_C@_0BB@JIMPEHCD@MACROAREA_VIEWER@ 0000000180004f00     flags.obj
 0001:00003f18       ??_C@_0BB@KILFBFJH@MACROAREA_EDITOR@ 0000000180004f18     flags.obj
 0001:00003f30       ??_C@_0BB@CADENPFI@MACROAREA_DIALOG@ 0000000180004f30     flags.obj
 0001:00003f48       ??_C@_0BB@MLMLHIGE@MACROAREA_SEARCH@ 0000000180004f48     flags.obj
 0001:00003f60       ??_C@_0BA@KKMKOLIK@MACROAREA_DISKS@ 0000000180004f60     flags.obj
 0001:00003f70       ??_C@_0BD@IGOOIJP@MACROAREA_MAINMENU@ 0000000180004f70     flags.obj
 0001:00003f88       ??_C@_0P@LFLMAHBF@MACROAREA_MENU@ 0000000180004f88     flags.obj
 0001:00003f98       ??_C@_0P@DKPKIEO@MACROAREA_HELP@ 0000000180004f98     flags.obj
 0001:00003fa8       ??_C@_0BE@MDJPICHC@MACROAREA_INFOPANEL@ 0000000180004fa8     flags.obj
 0001:00003fc0       ??_C@_0BF@NLJMHMPP@MACROAREA_QVIEWPANEL@ 0000000180004fc0     flags.obj
 0001:00003fd8       ??_C@_0BE@HBMEGBOC@MACROAREA_TREEPANEL@ 0000000180004fd8     flags.obj
 0001:00003ff0       ??_C@_0BF@FCHKCGLL@MACROAREA_FINDFOLDER@ 0000000180004ff0     flags.obj
 0001:00004008       ??_C@_0BD@JCFMJGDE@MACROAREA_USERMENU@ 0000000180005008     flags.obj
 0001:00004020       ??_C@_0BO@OMLEPJPM@MACROAREA_SHELLAUTOCOMPLETION@ 0000000180005020     flags.obj
 0001:00004040       ??_C@_0BP@OIHAIGBK@MACROAREA_DIALOGAUTOCOMPLETION@ 0000000180005040     flags.obj
 0001:00004060       ??_C@_0BC@EIJFKPMK@MACROAREA_GRABBER@ 0000000180005060     flags.obj
 0001:00004078       ??_C@_0BC@GNLOCEJP@MACROAREA_DESKTOP@ 0000000180005078     flags.obj
 0001:00004090       ??_C@_0BB@JPEEDDOG@MACROAREA_COMMON@ 0000000180005090     flags.obj
 0001:000040a8       ??_C@_0BD@DIKEKAIJ@MACROSTATE_NOMACRO@ 00000001800050a8     flags.obj
 0001:000040c0       ??_C@_0BF@PCDEFEGP@MACROSTATE_EXECUTING@ 00000001800050c0     flags.obj
 0001:000040d8       ??_C@_0BM@EJOFDENO@MACROSTATE_EXECUTING_COMMON@ 00000001800050d8     flags.obj
 0001:000040f8       ??_C@_0BF@BGODKPBB@MACROSTATE_RECORDING@ 00000001800050f8     flags.obj
 0001:00004110       ??_C@_0BM@OICPADFE@MACROSTATE_RECORDING_COMMON@ 0000000180005110     flags.obj
 0001:00004130       ??_C@_0N@CGFFMLBC@MPEC_SUCCESS@ 0000000180005130     flags.obj
 0001:00004140       ??_C@_0L@FJDDLDNN@MPEC_ERROR@ 0000000180005140     flags.obj
 0001:00004150       ??_C@_0N@IBOAADDD@FMVT_UNKNOWN@ 0000000180005150     flags.obj
 0001:00004160       ??_C@_0N@BDMFKEKE@FMVT_INTEGER@ 0000000180005160     flags.obj
 0001:00004170       ??_C@_0M@LFMLDDKI@FMVT_STRING@ 0000000180005170     flags.obj
 0001:00004180       ??_C@_0M@CKDAIOEN@FMVT_DOUBLE@ 0000000180005180     flags.obj
 0001:00004190       ??_C@_0N@MHKOBOGF@FMVT_BOOLEAN@ 0000000180005190     flags.obj
 0001:000041a0       ??_C@_0M@GKPDICDA@FMVT_BINARY@ 00000001800051a0     flags.obj
 0001:000041b0       ??_C@_0N@FMHCFNDF@FMVT_POINTER@ 00000001800051b0     flags.obj
 0001:000041c0       ??_C@_08DDPDBBNO@FMVT_NIL@ 00000001800051c0     flags.obj
 0001:000041d0       ??_C@_0L@DJIKMOJA@FMVT_ARRAY@ 00000001800051d0     flags.obj
 0001:000041e0       ??_C@_0L@PMDDFEBD@FMVT_PANEL@ 00000001800051e0     flags.obj
 0001:000041f0       ??_C@_0L@ELHBHIEH@FMVT_ERROR@ 00000001800051f0     flags.obj
 0001:00004200       ??_C@_0O@DCGKMPOM@WTYPE_DESKTOP@ 0000000180005200     flags.obj
 0001:00004210       ??_C@_0N@FNCFCPIG@WTYPE_PANELS@ 0000000180005210     flags.obj
 0001:00004220       ??_C@_0N@EJKMDMBK@WTYPE_VIEWER@ 0000000180005220     flags.obj
 0001:00004230       ??_C@_0N@HJNGGOKO@WTYPE_EDITOR@ 0000000180005230     flags.obj
 0001:00004240       ??_C@_0N@PBFHKEGB@WTYPE_DIALOG@ 0000000180005240     flags.obj
 0001:00004250       ??_C@_0M@OMKLELFA@WTYPE_VMENU@ 0000000180005250     flags.obj
 0001:00004260       ??_C@_0L@BCEMNGOG@WTYPE_HELP@ 0000000180005260     flags.obj
 0001:00004270       ??_C@_0P@MMIDEOJJ@WTYPE_COMBOBOX@ 0000000180005270     flags.obj
 0001:00004280       ??_C@_0O@BHEBEELJ@WTYPE_GRABBER@ 0000000180005280     flags.obj
 0001:00004290       ??_C@_0M@NFHHCILL@WTYPE_HMENU@ 0000000180005290     flags.obj
 0001:000042a0       ??_C@_0BA@IPEAOBGN@TBPS_NOPROGRESS@ 00000001800052a0     flags.obj
 0001:000042b0       ??_C@_0BD@HMEHMDAL@TBPS_INDETERMINATE@ 00000001800052b0     flags.obj
 0001:000042c8       ??_C@_0M@KHLNKPHE@TBPS_NORMAL@ 00000001800052c8     flags.obj
 0001:000042d8       ??_C@_0L@DFDPCOFD@TBPS_ERROR@ 00000001800052d8     flags.obj
 0001:000042e8       ??_C@_0M@GHGAPHPP@TBPS_PAUSED@ 00000001800052e8     flags.obj
 0001:000042f8       ??_C@_0O@MCNCFBLF@VSMT_VIEWMODE@ 00000001800052f8     flags.obj
 0001:00004308       ??_C@_09FLKONCNO@VSMT_WRAP@ 0000000180005308     flags.obj
 0001:00004318       ??_C@_0O@INKALKJK@VSMT_WORDWRAP@ 0000000180005318     flags.obj
 0001:00004328       ??_C@_08FNEFFFEL@VMT_TEXT@ 0000000180005328     flags.obj
 0001:00004338       ??_C@_07FLIHDEDA@VMT_HEX@  0000000180005338     flags.obj
 0001:00004340       ??_C@_08BDDNDBMJ@VMT_DUMP@ 0000000180005340     flags.obj
 0001:00004350       ??_C@_07OJCLGDHJ@VE_READ@  0000000180005350     flags.obj
 0001:00004358       ??_C@_08JIBCCIDC@VE_CLOSE@ 0000000180005358     flags.obj
 0001:00004368       ??_C@_0M@FEFKOOMJ@VE_GOTFOCUS@ 0000000180005368     flags.obj
 0001:00004378       ??_C@_0N@ICHCAKIB@VE_KILLFOCUS@ 0000000180005378     flags.obj
 0001:00004388       ??_C@_07BLBPFFLB@EE_READ@  0000000180005388     flags.obj
 0001:00004390       ??_C@_07KJGPGPOC@EE_SAVE@  0000000180005390     flags.obj
 0001:00004398       ??_C@_09NPOPIKMK@EE_REDRAW@ 0000000180005398     flags.obj
 0001:000043a8       ??_C@_08NFPFGIG@EE_CLOSE@  00000001800053a8     flags.obj
 0001:000043b8       ??_C@_0M@CPNMNBMF@EE_GOTFOCUS@ 00000001800053b8     flags.obj
 0001:000043c8       ??_C@_0N@ILLPMAJF@EE_KILLFOCUS@ 00000001800053c8     flags.obj
 0001:000043d8       ??_C@_09MIOGFFI@EE_CHANGE@ 00000001800053d8     flags.obj
 0001:000043e8       ??_C@_0P@MBHAHBBG@DE_DLGPROCINIT@ 00000001800053e8     flags.obj
 0001:000043f8       ??_C@_0BC@BMFEJAMO@DE_DEFDLGPROCINIT@ 00000001800053f8     flags.obj
 0001:00004410       ??_C@_0O@ICBCOJCG@DE_DLGPROCEND@ 0000000180005410     flags.obj
 0001:00004420       ??_C@_0BB@MNODJNPE@SE_COMMONSYNCHRO@ 0000000180005420     flags.obj
 0001:00004438       ??_C@_0N@HKGMPMJE@ESPT_TABSIZE@ 0000000180005438     flags.obj
 0001:00004448       ??_C@_0BA@GOKHPFCK@ESPT_EXPANDTABS@ 0000000180005448     flags.obj
 0001:00004458       ??_C@_0BA@KOADDMLI@ESPT_AUTOINDENT@ 0000000180005458     flags.obj
 0001:00004468       ??_C@_0BF@LPNONOMF@ESPT_CURSORBEYONDEOL@ 0000000180005468     flags.obj
 0001:00004480       ??_C@_0BC@OECOCGLJ@ESPT_CHARCODEBASE@ 0000000180005480     flags.obj
 0001:00004498       ??_C@_0O@PIAOJINE@ESPT_CODEPAGE@ 0000000180005498     flags.obj
 0001:000044a8       ??_C@_0BG@HAPABMJH@ESPT_SAVEFILEPOSITION@ 00000001800054a8     flags.obj
 0001:000044c0       ??_C@_0O@KCPDJCKC@ESPT_LOCKMODE@ 00000001800054c0     flags.obj
 0001:000044d0       ??_C@_0BA@EIGIAOHM@ESPT_SETWORDDIV@ 00000001800054d0     flags.obj
 0001:000044e0       ??_C@_0BA@FGEHLJDF@ESPT_GETWORDDIV@ 00000001800054e0     flags.obj
 0001:000044f0       ??_C@_0BE@MACJBCFP@ESPT_SHOWWHITESPACE@ 00000001800054f0     flags.obj
 0001:00004508       ??_C@_0M@FICNFPPA@ESPT_SETBOM@ 0000000180005508     flags.obj
 0001:00004518       ??_C@_09FLEMPKKP@EUR_BEGIN@ 0000000180005518     flags.obj
 0001:00004528       ??_C@_07DDJDFJCN@EUR_END@  0000000180005528     flags.obj
 0001:00004530       ??_C@_08FCONALGE@EUR_UNDO@ 0000000180005530     flags.obj
 0001:00004540       ??_C@_08DHMMFAHF@EUR_REDO@ 0000000180005540     flags.obj
 0001:00004550       ??_C@_0O@PKOIFEBO@EXPAND_NOTABS@ 0000000180005550     flags.obj
 0001:00004560       ??_C@_0P@MLHPCNDM@EXPAND_ALLTABS@ 0000000180005560     flags.obj
 0001:00004570       ??_C@_0P@OONGIIBL@EXPAND_NEWTABS@ 0000000180005570     flags.obj
 0001:00004580       ??_C@_0BD@DKHPEOHH@EOPT_EXPANDALLTABS@ 0000000180005580     flags.obj
 0001:00004598       ??_C@_0BG@BOINMDEK@EOPT_PERSISTENTBLOCKS@ 0000000180005598     flags.obj
 0001:000045b0       ??_C@_0BG@PIIHHCAN@EOPT_DELREMOVESBLOCKS@ 00000001800055b0     flags.obj
 0001:000045c8       ??_C@_0BA@KPJEAKBD@EOPT_AUTOINDENT@ 00000001800055c8     flags.obj
 0001:000045d8       ??_C@_0BG@MBPADLG@EOPT_SAVEFILEPOSITION@ 00000001800055d8     flags.obj
 0001:000045f0       ??_C@_0BI@PFHCGCAI@EOPT_AUTODETECTCODEPAGE@ 00000001800055f0     flags.obj
 0001:00004608       ??_C@_0BF@IMCOEIAL@EOPT_CURSORBEYONDEOL@ 0000000180005608     flags.obj
 0001:00004620       ??_C@_0BH@CJPAGGLC@EOPT_EXPANDONLYNEWTABS@ 0000000180005620     flags.obj
 0001:00004638       ??_C@_0BE@DDKCDJDC@EOPT_SHOWWHITESPACE@ 0000000180005638     flags.obj
 0001:00004650       ??_C@_08HMMLONBH@EOPT_BOM@ 0000000180005650     flags.obj
 0001:00004660       ??_C@_0BD@CLLAKGOA@EOPT_SHOWLINEBREAK@ 0000000180005660     flags.obj
 0001:00004678       ??_C@_0BC@JCJEPKEC@EOPT_SHOWTITLEBAR@ 0000000180005678     flags.obj
 0001:00004690       ??_C@_0BA@KPGMOBKI@EOPT_SHOWKEYBAR@ 0000000180005690     flags.obj
 0001:000046a0       ??_C@_0BD@EFCFEAD@EOPT_SHOWSCROLLBAR@ 00000001800056a0     flags.obj
 0001:000046b8       ??_C@_0L@BJCBJJNB@BTYPE_NONE@ 00000001800056b8     flags.obj
 0001:000046c8       ??_C@_0N@OPHHGFPF@BTYPE_STREAM@ 00000001800056c8     flags.obj
 0001:000046d8       ??_C@_0N@EMEGNPLI@BTYPE_COLUMN@ 00000001800056d8     flags.obj
 0001:000046e8       ??_C@_0BB@BNPDAPGB@ECSTATE_MODIFIED@ 00000001800056e8     flags.obj
 0001:00004700       ??_C@_0O@GBBGHDFM@ECSTATE_SAVED@ 0000000180005700     flags.obj
 0001:00004710       ??_C@_0P@BECIAJAM@ECSTATE_LOCKED@ 0000000180005710     flags.obj
 0001:00004720       ??_C@_0P@DOBJCNIG@ECTYPE_CHANGED@ 0000000180005720     flags.obj
 0001:00004730       ??_C@_0N@MDEFMEEA@ECTYPE_ADDED@ 0000000180005730     flags.obj
 0001:00004740       ??_C@_0P@NMOJJPOB@ECTYPE_DELETED@ 0000000180005740     flags.obj
 0001:00004750       ??_C@_08HHHKLJPB@PLT_PATH@ 0000000180005750     flags.obj
 0001:00004760       ??_C@_08KBAMIIFB@PFM_GUID@ 0000000180005760     flags.obj
 0001:00004770       ??_C@_0P@KKEMMPNI@PFM_MODULENAME@ 0000000180005770     flags.obj
 0001:00004780       ??_C@_09BOODOHKD@FFT_PANEL@ 0000000180005780     flags.obj
 0001:00004790       ??_C@_0N@GMEDAGNH@FFT_FINDFILE@ 0000000180005790     flags.obj
 0001:000047a0       ??_C@_08KKCPIPGP@FFT_COPY@ 00000001800057a0     flags.obj
 0001:000047b0       ??_C@_0L@EKPDMFDD@FFT_SELECT@ 00000001800057b0     flags.obj
 0001:000047c0       ??_C@_0L@LGPEDLLD@FFT_CUSTOM@ 00000001800057c0     flags.obj
 0001:000047d0       ??_C@_0M@OIOMMFOE@FST_UNKNOWN@ 00000001800057d0     flags.obj
 0001:000047e0       ??_C@_0L@GGGOEGKJ@FST_SUBKEY@ 00000001800057e0     flags.obj
 0001:000047f0       ??_C@_09LFEEAJIC@FST_QWORD@ 00000001800057f0     flags.obj
 0001:00004800       ??_C@_0L@LPMPBKDL@FST_STRING@ 0000000180005800     flags.obj
 0001:00004810       ??_C@_08EJJJCLIG@FST_DATA@ 0000000180005810     flags.obj
 0001:00004820       ??_C@_09OBBBBFPE@FSSF_ROOT@ 0000000180005820     flags.obj
 0001:00004830       ??_C@_0BB@HDKCPBIO@FSSF_HISTORY_CMD@ 0000000180005830     flags.obj
 0001:00004848       ??_C@_0BE@BLPOFODL@FSSF_HISTORY_FOLDER@ 0000000180005848     flags.obj
 0001:00004860       ??_C@_0BC@NJCJCCNH@FSSF_HISTORY_VIEW@ 0000000180005860     flags.obj
 0001:00004878       ??_C@_0BC@CODELNPP@FSSF_HISTORY_EDIT@ 0000000180005878     flags.obj
 0001:00004890       ??_C@_0BG@IFGEMJIF@FSSF_HISTORY_EXTERNAL@ 0000000180005890     flags.obj
 0001:000048a8       ??_C@_0BG@DGAKDKFK@FSSF_FOLDERSHORTCUT_0@ 00000001800058a8     flags.obj
 0001:000048c0       ??_C@_0BG@CPBBALBL@FSSF_FOLDERSHORTCUT_1@ 00000001800058c0     flags.obj
 0001:000048d8       ??_C@_0BG@EDMFINI@FSSF_FOLDERSHORTCUT_2@ 00000001800058d8     flags.obj
 0001:000048f0       ??_C@_0BG@BNCHGJJJ@FSSF_FOLDERSHORTCUT_3@ 00000001800058f0     flags.obj
 0001:00004908       ??_C@_0BG@FCGGPPFO@FSSF_FOLDERSHORTCUT_4@ 0000000180005908     flags.obj
 0001:00004920       ??_C@_0BG@ELHNMOBP@FSSF_FOLDERSHORTCUT_5@ 0000000180005920     flags.obj
 0001:00004938       ??_C@_0BG@GAFAJNNM@FSSF_FOLDERSHORTCUT_6@ 0000000180005938     flags.obj
 0001:00004950       ??_C@_0BG@HJELKMJN@FSSF_FOLDERSHORTCUT_7@ 0000000180005950     flags.obj
 0001:00004968       ??_C@_0BG@PONDLAFC@FSSF_FOLDERSHORTCUT_8@ 0000000180005968     flags.obj
 0001:00004980       ??_C@_0BG@OHMIIBBD@FSSF_FOLDERSHORTCUT_9@ 0000000180005980     flags.obj
 0001:00004998       ??_C@_0BD@PBIEGEHP@FSSF_CONFIRMATIONS@ 0000000180005998     flags.obj
 0001:000049b0       ??_C@_0M@PIGDMPJB@FSSF_SYSTEM@ 00000001800059b0     flags.obj
 0001:000049c0       ??_C@_0L@LBFNJGFB@FSSF_PANEL@ 00000001800059c0     flags.obj
 0001:000049d0       ??_C@_0M@KJLIHDEL@FSSF_EDITOR@ 00000001800059d0     flags.obj
 0001:000049e0       ??_C@_0M@KEMGKEOF@FSSF_SCREEN@ 00000001800059e0     flags.obj
 0001:000049f0       ??_C@_0M@CBDJLJIE@FSSF_DIALOG@ 00000001800059f0     flags.obj
 0001:00004a00       ??_C@_0P@OCDADNBF@FSSF_INTERFACE@ 0000000180005a00     flags.obj
 0001:00004a10       ??_C@_0BB@GBBEBNKE@FSSF_PANELLAYOUT@ 0000000180005a10     flags.obj
 0001:00004a28       ??_C@_0M@JCGHGLJF@PSL_ROAMING@ 0000000180005a28     flags.obj
 0001:00004a38       ??_C@_09EDBNDHCM@PSL_LOCAL@ 0000000180005a38     flags.obj
 0001:00004a48       ??_C@_07BPEFOPGM@FCT_ANY@  0000000180005a48     flags.obj
 0001:00004a50       ??_C@_0L@CDAEILNM@FCT_STREAM@ 0000000180005a50     flags.obj
 0001:00004a60       ??_C@_0L@IADFDBJB@FCT_COLUMN@ 0000000180005a60     flags.obj
 0001:00004a70       ??_C@_0O@KJFMBLFE@LINK_HARDLINK@ 0000000180005a70     flags.obj
 0001:00004a80       ??_C@_0O@OOAFIIDA@LINK_JUNCTION@ 0000000180005a80     flags.obj
 0001:00004a90       ??_C@_0O@FIAPLKLH@LINK_VOLMOUNT@ 0000000180005a90     flags.obj
 0001:00004aa0       ??_C@_0BB@JDBEPJDK@LINK_SYMLINKFILE@ 0000000180005aa0     flags.obj
 0001:00004ab8       ??_C@_0BA@GFPIOFMG@LINK_SYMLINKDIR@ 0000000180005ab8     flags.obj
 0001:00004ac8       ??_C@_0N@PJENIJFN@LINK_SYMLINK@ 0000000180005ac8     flags.obj
 0001:00004ad8       ??_C@_08HNOHKPBK@CPM_FULL@ 0000000180005ad8     flags.obj
 0001:00004ae8       ??_C@_08LAEGFKJE@CPM_REAL@ 0000000180005ae8     flags.obj
 0001:00004af8       ??_C@_0L@NPJNPCJM@CPM_NATIVE@ 0000000180005af8     flags.obj
 0001:00004b08       ??_C@_0L@NCFOENCC@VS_RELEASE@ 0000000180005b08     flags.obj
 0001:00004b18       ??_C@_08BDGLHPMJ@VS_ALPHA@ 0000000180005b18     flags.obj
 0001:00004b28       ??_C@_07OKFPMINB@VS_BETA@  0000000180005b28     flags.obj
 0001:00004b30       ??_C@_05MMFLPJEB@VS_RC@    0000000180005b30     flags.obj
 0001:00004b38       ??_C@_0L@IIIJLOAF@VS_SPECIAL@ 0000000180005b38     flags.obj
 0001:00004b48       ??_C@_0L@EAMAICHL@VS_PRIVATE@ 0000000180005b48     flags.obj
 0001:00004b58       ??_C@_0BC@OOKLINPG@OPEN_LEFTDISKMENU@ 0000000180005b58     flags.obj
 0001:00004b70       ??_C@_0BB@CEFDHHLF@OPEN_PLUGINSMENU@ 0000000180005b70     flags.obj
 0001:00004b88       ??_C@_0O@IEJHJCNB@OPEN_FINDLIST@ 0000000180005b88     flags.obj
 0001:00004b98       ??_C@_0O@OGDCDPNG@OPEN_SHORTCUT@ 0000000180005b98     flags.obj
 0001:00004ba8       ??_C@_0BB@JHCCMIPF@OPEN_COMMANDLINE@ 0000000180005ba8     flags.obj
 0001:00004bc0       ??_C@_0M@DMJLHMGM@OPEN_EDITOR@ 0000000180005bc0     flags.obj
 0001:00004bd0       ??_C@_0M@MOBCONI@OPEN_VIEWER@ 0000000180005bd0     flags.obj
 0001:00004be0       ??_C@_0P@LCDNLGDE@OPEN_FILEPANEL@ 0000000180005be0     flags.obj
 0001:00004bf0       ??_C@_0M@LEBKLGKD@OPEN_DIALOG@ 0000000180005bf0     flags.obj
 0001:00004c00       ??_C@_0N@CBHPGAKB@OPEN_ANALYSE@ 0000000180005c00     flags.obj
 0001:00004c10       ??_C@_0BD@NFNGGFHI@OPEN_RIGHTDISKMENU@ 0000000180005c10     flags.obj
 0001:00004c28       ??_C@_0P@FOKOAMLC@OPEN_FROMMACRO@ 0000000180005c28     flags.obj
 0001:00004c38       ??_C@_0O@NEDDJIHC@OPEN_LUAMACRO@ 0000000180005c38     flags.obj
 0001:00004c48       ??_C@_0P@GBMLNMMI@MCT_MACROPARSE@ 0000000180005c48     flags.obj
 0001:00004c58       ??_C@_0P@GNPFPCF@MCT_LOADMACROS@ 0000000180005c58     flags.obj
 0001:00004c68       ??_C@_0P@HMDDACMI@MCT_ENUMMACROS@ 0000000180005c68     flags.obj
 0001:00004c78       ??_C@_0BA@MOCJHMJK@MCT_WRITEMACROS@ 0000000180005c78     flags.obj
 0001:00004c88       ??_C@_0N@IGJGAHKE@MCT_GETMACRO@ 0000000180005c88     flags.obj
 0001:00004c98       ??_C@_0BC@NFGGBILF@MCT_RECORDEDMACRO@ 0000000180005c98     flags.obj
 0001:00004cb0       ??_C@_0N@OLCKOJMI@MCT_DELMACRO@ 0000000180005cb0     flags.obj
 0001:00004cc0       ??_C@_0BC@NALHIHJ@MCT_RUNSTARTMACRO@ 0000000180005cc0     flags.obj
 0001:00004cd8       ??_C@_0P@HOMHAEFB@MCT_EXECSTRING@ 0000000180005cd8     flags.obj
 0001:00004ce8       ??_C@_0O@CDBDPKIC@MCT_PANELSORT@ 0000000180005ce8     flags.obj
 0001:00004cf8       ??_C@_0BH@PKKJIOHM@MCT_GETCUSTOMSORTMODES@ 0000000180005cf8     flags.obj
 0001:00004d10       ??_C@_0N@FOPIOCHO@MCT_ADDMACRO@ 0000000180005d10     flags.obj
 0001:00004d20       ??_C@_0N@BHFJFHA@MCT_KEYMACRO@ 0000000180005d20     flags.obj
 0001:00004d30       ??_C@_0BB@LPDAOGB@MCT_CANPANELSORT@ 0000000180005d30     flags.obj
 0001:00004d48       ??_C@_0BC@IOECJI@MPRT_NORMALFINISH@ 0000000180005d48     flags.obj
 0001:00004d60       ??_C@_0BB@PMCBIGCA@MPRT_ERRORFINISH@ 0000000180005d60     flags.obj
 0001:00004d78       ??_C@_0BA@BCBAEEOI@MPRT_ERRORPARSE@ 0000000180005d78     flags.obj
 0001:00004d88       ??_C@_09EJDAADCN@MPRT_KEYS@ 0000000180005d88     flags.obj
 0001:00004d98       ??_C@_0L@GEHHCKFA@MPRT_PRINT@ 0000000180005d98     flags.obj
 0001:00004da8       ??_C@_0BA@OBIDLEIM@MPRT_PLUGINCALL@ 0000000180005da8     flags.obj
 0001:00004db8       ??_C@_0BA@EJFFOAMM@MPRT_PLUGINMENU@ 0000000180005db8     flags.obj
 0001:00004dc8       ??_C@_0BC@LEDOPMKI@MPRT_PLUGINCONFIG@ 0000000180005dc8     flags.obj
 0001:00004de0       ??_C@_0BD@HHINMPPI@MPRT_PLUGINCOMMAND@ 0000000180005de0     flags.obj
 0001:00004df8       ??_C@_0O@IEMNLPAB@MPRT_USERMENU@ 0000000180005df8     flags.obj
 0001:00004e08       ??_C@_0BA@GEAFHJNF@MPRT_HASNOMACRO@ 0000000180005e08     flags.obj
 0001:00004e18       ??_C@_0BC@PNCKAHJO@FE_CHANGEVIEWMODE@ 0000000180005e18     flags.obj
 0001:00004e30       ??_C@_09DENIDBMJ@FE_REDRAW@ 0000000180005e30     flags.obj
 0001:00004e40       ??_C@_07CLNPDBLG@FE_IDLE@  0000000180005e40     flags.obj
 0001:00004e48       ??_C@_08DENCGKED@FE_CLOSE@ 0000000180005e48     flags.obj
 0001:00004e58       ??_C@_08MOMCCKPB@FE_BREAK@ 0000000180005e58     flags.obj
 0001:00004e68       ??_C@_0L@LELAIPLL@FE_COMMAND@ 0000000180005e68     flags.obj
 0001:00004e78       ??_C@_0M@FIECADDF@FE_GOTFOCUS@ 0000000180005e78     flags.obj
 0001:00004e88       ??_C@_0N@DGHFKMFL@FE_KILLFOCUS@ 0000000180005e88     flags.obj
 0001:00004e98       ??_C@_0BE@PONEECEM@FE_CHANGESORTPARAMS@ 0000000180005e98     flags.obj
 0001:00004eb0       ??_C@_0M@HNDHDHHO@FCF_FG_4BIT@ 0000000180005eb0     flags.obj
 0001:00004ec0       ??_C@_0M@PJHNDJIE@FCF_BG_4BIT@ 0000000180005ec0     flags.obj
 0001:00004ed0       ??_C@_0N@HMKJBHOA@FCF_4BITMASK@ 0000000180005ed0     flags.obj
 0001:00004ee0       ??_C@_0BB@PJFLJJLD@FCF_RAWATTR_MASK@ 0000000180005ee0     flags.obj
 0001:00004ef8       ??_C@_0BC@NKBLNNIA@FCF_EXTENDEDFLAGS@ 0000000180005ef8     flags.obj
 0001:00004f10       ??_C@_0M@LFMGCKHG@FCF_FG_BOLD@ 0000000180005f10     flags.obj
 0001:00004f20       ??_C@_0O@FAPDECBF@FCF_FG_ITALIC@ 0000000180005f20     flags.obj
 0001:00004f30       ??_C@_0BB@NPEFGEGA@FCF_FG_UNDERLINE@ 0000000180005f30     flags.obj
 0001:00004f48       ??_C@_0O@LGBGBIGB@FCF_STYLEMASK@ 0000000180005f48     flags.obj
 0001:00004f58       ??_C@_08BKNBBLHK@FCF_NONE@ 0000000180005f58     flags.obj
 0001:00004f68       ??_C@_08FKIDFHCM@CDF_NONE@ 0000000180005f68     flags.obj
 0001:00004f78       ??_C@_0N@ELMEMNDH@FMSG_WARNING@ 0000000180005f78     flags.obj
 0001:00004f88       ??_C@_0P@HHIGLJAP@FMSG_ERRORTYPE@ 0000000180005f88     flags.obj
 0001:00004f98       ??_C@_0BE@FHOOILPH@FMSG_KEEPBACKGROUND@ 0000000180005f98     flags.obj
 0001:00004fb0       ??_C@_0P@KBEMNNEP@FMSG_LEFTALIGN@ 0000000180005fb0     flags.obj
 0001:00004fc0       ??_C@_0O@FOIOKDHJ@FMSG_ALLINONE@ 0000000180005fc0     flags.obj
 0001:00004fd0       ??_C@_0L@BGALGPOK@FMSG_MB_OK@ 0000000180005fd0     flags.obj
 0001:00004fe0       ??_C@_0BB@JGAPGIEP@FMSG_MB_OKCANCEL@ 0000000180005fe0     flags.obj
 0001:00004ff8       ??_C@_0BJ@BKJADAHA@FMSG_MB_ABORTRETRYIGNORE@ 0000000180005ff8     flags.obj
 0001:00005018       ??_C@_0O@GPCAPHCL@FMSG_MB_YESNO@ 0000000180006018     flags.obj
 0001:00005028       ??_C@_0BE@IBNOLCGP@FMSG_MB_YESNOCANCEL@ 0000000180006028     flags.obj
 0001:00005040       ??_C@_0BE@OCLAIENB@FMSG_MB_RETRYCANCEL@ 0000000180006040     flags.obj
 0001:00005058       ??_C@_09NEGPLEAH@FMSG_NONE@ 0000000180006058     flags.obj
 0001:00005068       ??_C@_0N@DHJCDIKM@DIF_BOXCOLOR@ 0000000180006068     flags.obj
 0001:00005078       ??_C@_09IAEPIICA@DIF_GROUP@ 0000000180006078     flags.obj
 0001:00005088       ??_C@_0N@GCKJNBCM@DIF_LEFTTEXT@ 0000000180006088     flags.obj
 0001:00005098       ??_C@_0P@BGPBEDHH@DIF_MOVESELECT@ 0000000180006098     flags.obj
 0001:000050a8       ??_C@_0BC@PDKFKKEI@DIF_SHOWAMPERSAND@ 00000001800060a8     flags.obj
 0001:000050c0       ??_C@_0BA@BLCOKAAO@DIF_CENTERGROUP@ 00000001800060c0     flags.obj
 0001:000050d0       ??_C@_0P@MKFBJPOB@DIF_NOBRACKETS@ 00000001800060d0     flags.obj
 0001:000050e0       ??_C@_0BF@JBCDBJCL@DIF_MANUALADDHISTORY@ 00000001800060e0     flags.obj
 0001:000050f8       ??_C@_0O@JKNMBNLA@DIF_SEPARATOR@ 00000001800060f8     flags.obj
 0001:00005108       ??_C@_0P@CGILDLOA@DIF_SEPARATOR2@ 0000000180006108     flags.obj
 0001:00005118       ??_C@_0L@NBPFNGLB@DIF_EDITOR@ 0000000180006118     flags.obj
 0001:00005128       ??_C@_0BE@PFICAGJF@DIF_LISTNOAMPERSAND@ 0000000180006128     flags.obj
 0001:00005140       ??_C@_0O@FFJNBMAD@DIF_LISTNOBOX@ 0000000180006140     flags.obj
 0001:00005150       ??_C@_0M@IPFBMFDN@DIF_HISTORY@ 0000000180006150     flags.obj
 0001:00005160       ??_C@_0P@EGFAEEDC@DIF_BTNNOCLOSE@ 0000000180006160     flags.obj
 0001:00005170       ??_C@_0P@KOJCCCGB@DIF_CENTERTEXT@ 0000000180006170     flags.obj
 0001:00005180       ??_C@_0BC@ODEMBOPK@DIF_SEPARATORUSER@ 0000000180006180     flags.obj
 0001:00005198       ??_C@_0O@IKJBMPOF@DIF_SETSHIELD@ 0000000180006198     flags.obj
 0001:000051a8       ??_C@_0P@EEJEDBLH@DIF_EDITEXPAND@ 00000001800061a8     flags.obj
 0001:000051b8       ??_C@_0BB@EIMEKEFP@DIF_DROPDOWNLIST@ 00000001800061b8     flags.obj
 0001:000051d0       ??_C@_0BD@MNGIOLFF@DIF_USELASTHISTORY@ 00000001800061d0     flags.obj
 0001:000051e8       ??_C@_0N@MOCGNIKC@DIF_MASKEDIT@ 00000001800061e8     flags.obj
 0001:000051f8       ??_C@_0BD@LPDHCLJI@DIF_LISTTRACKMOUSE@ 00000001800061f8     flags.obj
 0001:00005210       ??_C@_0BK@LEFIBDOA@DIF_LISTTRACKMOUSEINFOCUS@ 0000000180006210     flags.obj
 0001:00005230       ??_C@_0BC@JNLDMGBD@DIF_SELECTONENTRY@ 0000000180006230     flags.obj
 0001:00005248       ??_C@_0L@KKNJDNBK@DIF_3STATE@ 0000000180006248     flags.obj
 0001:00005258       ??_C@_0N@GBGHICKO@DIF_EDITPATH@ 0000000180006258     flags.obj
 0001:00005268       ??_C@_0BB@NPNALIGO@DIF_LISTWRAPMODE@ 0000000180006268     flags.obj
 0001:00005280       ??_C@_0BD@MFOKKGGF@DIF_NOAUTOCOMPLETE@ 0000000180006280     flags.obj
 0001:00005298       ??_C@_0BG@MONEJILE@DIF_LISTAUTOHIGHLIGHT@ 0000000180006298     flags.obj
 0001:000052b0       ??_C@_0BA@JNOKLHOL@DIF_LISTNOCLOSE@ 00000001800062b0     flags.obj
 0001:000052c0       ??_C@_0BB@GMKDKOOP@DIF_EDITPATHEXEC@ 00000001800062c0     flags.obj
 0001:000052d8       ??_C@_0L@EPNFOPAK@DIF_HIDDEN@ 00000001800062d8     flags.obj
 0001:000052e8       ??_C@_0N@KOGKCAKJ@DIF_READONLY@ 00000001800062e8     flags.obj
 0001:000052f8       ??_C@_0M@NLLDINIM@DIF_NOFOCUS@ 00000001800062f8     flags.obj
 0001:00005308       ??_C@_0M@HCFLMDHK@DIF_DISABLE@ 0000000180006308     flags.obj
 0001:00005318       ??_C@_0BC@CHAAKEJO@DIF_DEFAULTBUTTON@ 0000000180006318     flags.obj
 0001:00005330       ??_C@_09LCJIOEMN@DIF_FOCUS@ 0000000180006330     flags.obj
 0001:00005340       ??_C@_0O@KJADCBBN@DIF_RIGHTTEXT@ 0000000180006340     flags.obj
 0001:00005350       ??_C@_0N@LAEOODAD@DIF_WORDWRAP@ 0000000180006350     flags.obj
 0001:00005360       ??_C@_08KFOHCPDE@DIF_NONE@ 0000000180006360     flags.obj
 0001:00005370       ??_C@_0N@EDHAFIIL@LIF_SELECTED@ 0000000180006370     flags.obj
 0001:00005380       ??_C@_0M@BMGIEAIL@LIF_CHECKED@ 0000000180006380     flags.obj
 0001:00005390       ??_C@_0O@KJIFADIG@LIF_SEPARATOR@ 0000000180006390     flags.obj
 0001:000053a0       ??_C@_0M@HEFHLFIE@LIF_DISABLE@ 00000001800063a0     flags.obj
 0001:000053b0       ??_C@_0L@PKDDGEEG@LIF_GRAYED@ 00000001800063b0     flags.obj
 0001:000053c0       ??_C@_0L@PFBGAOEP@LIF_HIDDEN@ 00000001800063c0     flags.obj
 0001:000053d0       ??_C@_0BD@HEPCOIEH@LIF_DELETEUSERDATA@ 00000001800063d0     flags.obj
 0001:000053e8       ??_C@_08BODPINCM@LIF_NONE@ 00000001800063e8     flags.obj
 0001:000053f8       ??_C@_0BC@BGAENNBJ@LIFIND_EXACTMATCH@ 00000001800063f8     flags.obj
 0001:00005410       ??_C@_0M@FPOGKIGO@LIFIND_NONE@ 0000000180006410     flags.obj
 0001:00005420       ??_C@_0BA@OOIEKCFB@LINFO_SHOWNOBOX@ 0000000180006420     flags.obj
 0001:00005430       ??_C@_0BE@DECCEGNO@LINFO_AUTOHIGHLIGHT@ 0000000180006430     flags.obj
 0001:00005448       ??_C@_0BH@BADLEILJ@LINFO_REVERSEHIGHLIGHT@ 0000000180006448     flags.obj
 0001:00005460       ??_C@_0P@KLBMHNCG@LINFO_WRAPMODE@ 0000000180006460     flags.obj
 0001:00005470       ??_C@_0BE@OHJCOKAE@LINFO_SHOWAMPERSAND@ 0000000180006470     flags.obj
 0001:00005488       ??_C@_0L@EPACPANF@LINFO_NONE@ 0000000180006488     flags.obj
 0001:00005498       ??_C@_0N@OLGDMHKL@FDLG_WARNING@ 0000000180006498     flags.obj
 0001:000054a8       ??_C@_0BB@DKMEBDJJ@FDLG_SMALLDIALOG@ 00000001800064a8     flags.obj
 0001:000054c0       ??_C@_0BC@ONGLDAJN@FDLG_NODRAWSHADOW@ 00000001800064c0     flags.obj
 0001:000054d8       ??_C@_0BB@NPLEEAKK@FDLG_NODRAWPANEL@ 00000001800064d8     flags.obj
 0001:000054f0       ??_C@_0BG@GHNOOENB@FDLG_KEEPCONSOLETITLE@ 00000001800064f0     flags.obj
 0001:00005508       ??_C@_0O@MKFABCNE@FDLG_NONMODAL@ 0000000180006508     flags.obj
 0001:00005518       ??_C@_09NNFHCBNL@FDLG_NONE@ 0000000180006518     flags.obj
 0001:00005528       ??_C@_0N@JOOGIBAO@MIF_SELECTED@ 0000000180006528     flags.obj
 0001:00005538       ??_C@_0M@IHMNAMOE@MIF_CHECKED@ 0000000180006538     flags.obj
 0001:00005548       ??_C@_0O@DEIKOCPA@MIF_SEPARATOR@ 0000000180006548     flags.obj
 0001:00005558       ??_C@_0M@OPPCPJOL@MIF_DISABLE@ 0000000180006558     flags.obj
 0001:00005568       ??_C@_0L@DLLNLLIG@MIF_GRAYED@ 0000000180006568     flags.obj
 0001:00005578       ??_C@_0L@DEJINBIP@MIF_HIDDEN@ 0000000180006578     flags.obj
 0001:00005588       ??_C@_08JEEJJGP@MIF_NONE@  0000000180006588     flags.obj
 0001:00005598       ??_C@_0BE@FALMPPJK@FMENU_SHOWAMPERSAND@ 0000000180006598     flags.obj
 0001:000055b0       ??_C@_0P@HICDNKDJ@FMENU_WRAPMODE@ 00000001800065b0     flags.obj
 0001:000055c0       ??_C@_0BE@IDAMFDEA@FMENU_AUTOHIGHLIGHT@ 00000001800065c0     flags.obj
 0001:000055d8       ??_C@_0BL@OKAIKPMN@FMENU_REVERSEAUTOHIGHLIGHT@ 00000001800065d8     flags.obj
 0001:000055f8       ??_C@_0BJ@FCEONOJC@FMENU_CHANGECONSOLETITLE@ 00000001800065f8     flags.obj
 0001:00005618       ??_C@_0BA@GDFPJAAD@FMENU_SHOWNOBOX@ 0000000180006618     flags.obj
 0001:00005628       ??_C@_0BD@PMEPMEOJ@FMENU_SHOWSHORTBOX@ 0000000180006628     flags.obj
 0001:00005640       ??_C@_0BE@PDNJFEDO@FMENU_SHOWSINGLEBOX@ 0000000180006640     flags.obj
 0001:00005658       ??_C@_0BD@JBJJGCBE@FMENU_NODRAWSHADOW@ 0000000180006658     flags.obj
 0001:00005670       ??_C@_0L@DGFIEOMD@FMENU_NONE@ 0000000180006670     flags.obj
 0001:00005680       ??_C@_0O@JEAJLDHC@PPIF_SELECTED@ 0000000180006680     flags.obj
 0001:00005690       ??_C@_0BC@LPBDBIOM@PPIF_PROCESSDESCR@ 0000000180006690     flags.obj
 0001:000056a8       ??_C@_09OIFMMGNJ@PPIF_NONE@ 00000001800066a8     flags.obj
 0001:000056b8       ??_C@_0BC@BONLDOOD@PFLAGS_SHOWHIDDEN@ 00000001800066b8     flags.obj
 0001:000056d0       ??_C@_0BB@BCAJEJEH@PFLAGS_HIGHLIGHT@ 00000001800066d0     flags.obj
 0001:000056e8       ??_C@_0BI@BFAFODJ@PFLAGS_REVERSESORTORDER@ 00000001800066e8     flags.obj
 0001:00005700       ??_C@_0BF@KJNCJPKN@PFLAGS_USESORTGROUPS@ 0000000180006700     flags.obj
 0001:00005718       ??_C@_0BF@LBBAIOCD@PFLAGS_SELECTEDFIRST@ 0000000180006718     flags.obj
 0001:00005730       ??_C@_0BB@KDANIJNM@PFLAGS_REALNAMES@ 0000000180006730     flags.obj
 0001:00005748       ??_C@_0BB@ILEHDKFJ@PFLAGS_PANELLEFT@ 0000000180006748     flags.obj
 0001:00005760       ??_C@_0BI@EHHAJLOH@PFLAGS_DIRECTORIESFIRST@ 0000000180006760     flags.obj
 0001:00005778       ??_C@_0BA@KJEPHDOM@PFLAGS_USECRC32@ 0000000180006778     flags.obj
 0001:00005788       ??_C@_0O@DBPJGING@PFLAGS_PLUGIN@ 0000000180006788     flags.obj
 0001:00005798       ??_C@_0P@MLDEBNPK@PFLAGS_VISIBLE@ 0000000180006798     flags.obj
 0001:000057a8       ??_C@_0N@EOFAELOJ@PFLAGS_FOCUS@ 00000001800067a8     flags.obj
 0001:000057b8       ??_C@_0BI@EOCCAHFA@PFLAGS_ALTERNATIVENAMES@ 00000001800067b8     flags.obj
 0001:000057d0       ??_C@_0BA@GHMDCHHI@PFLAGS_SHORTCUT@ 00000001800067d0     flags.obj
 0001:000057e0       ??_C@_0M@NEMAHHGP@PFLAGS_NONE@ 00000001800067e0     flags.obj
 0001:000057f0       ??_C@_0M@IDNADAFL@VF_NONMODAL@ 00000001800067f0     flags.obj
 0001:00005800       ??_C@_0BB@OCDDPIKL@VF_DELETEONCLOSE@ 0000000180006800     flags.obj
 0001:00005818       ??_C@_0N@LDHALKKM@VF_ENABLE_F6@ 0000000180006818     flags.obj
 0001:00005828       ??_C@_0BC@DLGKMECC@VF_DISABLEHISTORY@ 0000000180006828     flags.obj
 0001:00005840       ??_C@_0BD@DHJCMLFI@VF_IMMEDIATERETURN@ 0000000180006840     flags.obj
 0001:00005858       ??_C@_0BJ@OGNFHEJG@VF_DELETEONLYFILEONCLOSE@ 0000000180006858     flags.obj
 0001:00005878       ??_C@_07CJJFHP@VF_NONE@    0000000180006878     flags.obj
 0001:00005880       ??_C@_0M@PIFGAPFH@EF_NONMODAL@ 0000000180006880     flags.obj
 0001:00005890       ??_C@_0N@DBHFPBEO@EF_CREATENEW@ 0000000180006890     flags.obj
 0001:000058a0       ??_C@_0N@LKLNHALI@EF_ENABLE_F6@ 00000001800068a0     flags.obj
 0001:000058b0       ??_C@_0BC@PPEPEFFI@EF_DISABLEHISTORY@ 00000001800068b0     flags.obj
 0001:000058c8       ??_C@_0BB@KGPIDKFC@EF_DELETEONCLOSE@ 00000001800068c8     flags.obj
 0001:000058e0       ??_C@_0BD@IHIGHGPL@EF_IMMEDIATERETURN@ 00000001800068e0     flags.obj
 0001:000058f8       ??_C@_0BJ@ILCPOFKL@EF_DELETEONLYFILEONCLOSE@ 00000001800068f8     flags.obj
 0001:00005918       ??_C@_09IJMPFPLB@EF_LOCKED@ 0000000180006918     flags.obj
 0001:00005928       ??_C@_0BC@GFHJGKD@EF_DISABLESAVEPOS@ 0000000180006928     flags.obj
 0001:00005940       ??_C@_0BB@NILAHAFO@EF_OPENMODE_MASK@ 0000000180006940     flags.obj
 0001:00005958       ??_C@_0BC@GAIDEJIA@EF_OPENMODE_QUERY@ 0000000180006958     flags.obj
 0001:00005970       ??_C@_0BG@BFKJJBAG@EF_OPENMODE_NEWIFOPEN@ 0000000180006970     flags.obj
 0001:00005988       ??_C@_0BI@KGOKGPEI@EF_OPENMODE_USEEXISTING@ 0000000180006988     flags.obj
 0001:000059a0       ??_C@_0BI@EJBKKDJ@EF_OPENMODE_BREAKIFOPEN@ 00000001800069a0     flags.obj
 0001:000059b8       ??_C@_0BJ@MOLGCBMH@EF_OPENMODE_RELOADIFOPEN@ 00000001800069b8     flags.obj
 0001:000059d8       ??_C@_07MBPCONNA@EN_NONE@  00000001800069d8     flags.obj
 0001:000059e0       ??_C@_0BC@HHNGCBAM@FHELP_NOSHOWERROR@ 00000001800069e0     flags.obj
 0001:000059f8       ??_C@_0P@GANNLHEJ@FHELP_SELFHELP@ 00000001800069f8     flags.obj
 0001:00005a08       ??_C@_0O@FLGGLFLC@FHELP_FARHELP@ 0000000180006a08     flags.obj
 0001:00005a18       ??_C@_0BB@KNKDPNI@FHELP_CUSTOMFILE@ 0000000180006a18     flags.obj
 0001:00005a30       ??_C@_0BB@IHFFPJJA@FHELP_CUSTOMPATH@ 0000000180006a30     flags.obj
 0001:00005a48       ??_C@_0L@OOIMFPBD@FHELP_GUID@ 0000000180006a48     flags.obj
 0001:00005a58       ??_C@_0BC@PNPOIHMG@FHELP_USECONTENTS@ 0000000180006a58     flags.obj
 0001:00005a70       ??_C@_0L@MAGMKNFN@FHELP_NONE@ 0000000180006a70     flags.obj
 0001:00005a80       ??_C@_0BE@GEGKIINM@KMFLAGS_SILENTCHECK@ 0000000180006a80     flags.obj
 0001:00005a98       ??_C@_0BM@BBOPLPKC@KMFLAGS_NOSENDKEYSTOPLUGINS@ 0000000180006a98     flags.obj
 0001:00005ab8       ??_C@_0BF@PHHPAAOK@KMFLAGS_ENABLEOUTPUT@ 0000000180006ab8     flags.obj
 0001:00005ad0       ??_C@_0BB@NCECNBPK@KMFLAGS_LANGMASK@ 0000000180006ad0     flags.obj
 0001:00005ae8       ??_C@_0M@HFBACHCP@KMFLAGS_LUA@ 0000000180006ae8     flags.obj
 0001:00005af8       ??_C@_0BD@JHNPMIGP@KMFLAGS_MOONSCRIPT@ 0000000180006af8     flags.obj
 0001:00005b10       ??_C@_0N@GIJCDFJI@KMFLAGS_NONE@ 0000000180006b10     flags.obj
 0001:00005b20       ??_C@_0O@GKOLBMFK@AKMFLAGS_NONE@ 0000000180006b20     flags.obj
 0001:00005b30       ??_C@_0P@LMBMJIMF@FSETCLR_REDRAW@ 0000000180006b30     flags.obj
 0001:00005b40       ??_C@_0N@LCOHPDHN@FSETCLR_NONE@ 0000000180006b40     flags.obj
 0001:00005b50       ??_C@_0N@MLMCEKPH@WIF_MODIFIED@ 0000000180006b50     flags.obj
 0001:00005b60       ??_C@_0M@ICPAPCOF@WIF_CURRENT@ 0000000180006b60     flags.obj
 0001:00005b70       ??_C@_09FPGEBDGO@WIF_MODAL@ 0000000180006b70     flags.obj
 0001:00005b80       ??_C@_08DAKKFBIA@WIF_NONE@ 0000000180006b80     flags.obj
 0001:00005b90       ??_C@_0BG@JMJAOELH@VOPT_SAVEFILEPOSITION@ 0000000180006b90     flags.obj
 0001:00005ba8       ??_C@_0BI@NCAHLEBN@VOPT_AUTODETECTCODEPAGE@ 0000000180006ba8     flags.obj
 0001:00005bc0       ??_C@_0BC@FGLBHLDI@VOPT_SHOWTITLEBAR@ 0000000180006bc0     flags.obj
 0001:00005bd8       ??_C@_0BA@GAIDGLME@VOPT_SHOWKEYBAR@ 0000000180006bd8     flags.obj
 0001:00005be8       ??_C@_0BD@LEEGOJKA@VOPT_SHOWSCROLLBAR@ 0000000180006be8     flags.obj
 0001:00005c00       ??_C@_0P@NEIKPMJJ@VOPT_QUICKVIEW@ 0000000180006c00     flags.obj
 0001:00005c10       ??_C@_09FIOJMNJ@VOPT_NONE@ 0000000180006c10     flags.obj
 0001:00005c20       ??_C@_0N@ILNDJNNO@VSMFL_REDRAW@ 0000000180006c20     flags.obj
 0001:00005c30       ??_C@_0L@DLLCFLOD@VSMFL_NONE@ 0000000180006c30     flags.obj
 0001:00005c40       ??_C@_0N@GHEHKHJN@VSP_NOREDRAW@ 0000000180006c40     flags.obj
 0001:00005c50       ??_C@_0M@LHNGMHFO@VSP_PERCENT@ 0000000180006c50     flags.obj
 0001:00005c60       ??_C@_0N@JGGGCNIP@VSP_RELATIVE@ 0000000180006c60     flags.obj
 0001:00005c70       ??_C@_0BA@JKDMJLJG@VSP_NORETNEWPOS@ 0000000180006c70     flags.obj
 0001:00005c80       ??_C@_08MOKEMBNE@VSP_NONE@ 0000000180006c80     flags.obj
 0001:00005c90       ??_C@_08FAPBJAKB@VMF_WRAP@ 0000000180006c90     flags.obj
 0001:00005ca0       ??_C@_0N@GHBDMLON@VMF_WORDWRAP@ 0000000180006ca0     flags.obj
 0001:00005cb0       ??_C@_08KDJLELDJ@VMF_NONE@ 0000000180006cb0     flags.obj
 0001:00005cc0       ??_C@_0BB@EDGIEBDF@ECF_TABMARKFIRST@ 0000000180006cc0     flags.obj
 0001:00005cd8       ??_C@_0BD@DKGCCJNG@ECF_TABMARKCURRENT@ 0000000180006cd8     flags.obj
 0001:00005cf0       ??_C@_0P@BAFEMBAJ@ECF_AUTODELETE@ 0000000180006cf0     flags.obj
 0001:00005d00       ??_C@_08CDFMCHLP@ECF_NONE@ 0000000180006d00     flags.obj
 0001:00005d10       ??_C@_0BA@KNNLMGCA@FIB_ENABLEEMPTY@ 0000000180006d10     flags.obj
 0001:00005d20       ??_C@_0N@DLDJCGJI@FIB_PASSWORD@ 0000000180006d20     flags.obj
 0001:00005d30       ??_C@_0O@DOHEGELC@FIB_EXPANDENV@ 0000000180006d30     flags.obj
 0001:00005d40       ??_C@_0BF@CEMIHIOK@FIB_NOUSELASTHISTORY@ 0000000180006d40     flags.obj
 0001:00005d58       ??_C@_0M@KJOJJDIM@FIB_BUTTONS@ 0000000180006d58     flags.obj
 0001:00005d68       ??_C@_0BA@COBBDHNL@FIB_NOAMPERSAND@ 0000000180006d68     flags.obj
 0001:00005d78       ??_C@_0N@LBOCEEGH@FIB_EDITPATH@ 0000000180006d78     flags.obj
 0001:00005d88       ??_C@_0BB@DCODFLEL@FIB_EDITPATHEXEC@ 0000000180006d88     flags.obj
 0001:00005da0       ??_C@_08HPFOCDKB@FIB_NONE@ 0000000180006da0     flags.obj
 0001:00005db0       ??_C@_0L@NMBLFMBN@FPF_LOADED@ 0000000180006db0     flags.obj
 0001:00005dc0       ??_C@_08GKECKCCJ@FPF_ANSI@ 0000000180006dc0     flags.obj
 0001:00005dd0       ??_C@_08OIOFCNLC@FPF_NONE@ 0000000180006dd0     flags.obj
 0001:00005de0       ??_C@_0L@HODJIPGA@PN_CMPNAME@ 0000000180006de0     flags.obj
 0001:00005df0       ??_C@_0P@KDEENAHJ@PN_CMPNAMELIST@ 0000000180006df0     flags.obj
 0001:00005e00       ??_C@_0BA@BJCCEIOI@PN_GENERATENAME@ 0000000180006e00     flags.obj
 0001:00005e10       ??_C@_0N@FEGPCCPJ@PN_CHECKMASK@ 0000000180006e10     flags.obj
 0001:00005e20       ??_C@_0M@NOOLKEBH@PN_SKIPPATH@ 0000000180006e20     flags.obj
 0001:00005e30       ??_C@_0BE@OPDBOAAE@PN_SHOWERRORMESSAGE@ 0000000180006e30     flags.obj
 0001:00005e48       ??_C@_07PFKJNCJP@PN_NONE@  0000000180006e48     flags.obj
 0001:00005e50       ??_C@_0BG@GOMJDMCK@XLAT_SWITCHKEYBLAYOUT@ 0000000180006e50     flags.obj
 0001:00005e68       ??_C@_0BE@KOIJDNLA@XLAT_SWITCHKEYBBEEP@ 0000000180006e68     flags.obj
 0001:00005e80       ??_C@_0BH@KBFAFPNA@XLAT_USEKEYBLAYOUTNAME@ 0000000180006e80     flags.obj
 0001:00005e98       ??_C@_0BH@IANKLOAC@XLAT_CONVERTALLCMDLINE@ 0000000180006e98     flags.obj
 0001:00005eb0       ??_C@_09JCNLKBBK@XLAT_NONE@ 0000000180006eb0     flags.obj
 0001:00005ec0       ??_C@_0N@PJEDCNNJ@FRS_RETUPDIR@ 0000000180006ec0     flags.obj
 0001:00005ed0       ??_C@_09GHEPLOHO@FRS_RECUR@ 0000000180006ed0     flags.obj
 0001:00005ee0       ??_C@_0BA@JCPHOEAE@FRS_SCANSYMLINK@ 0000000180006ee0     flags.obj
 0001:00005ef0       ??_C@_08JPCGJJKG@FRS_NONE@ 0000000180006ef0     flags.obj
 0001:00005f00       ??_C@_0P@LJPBHEIE@MLF_SHOWERRMSG@ 0000000180006f00     flags.obj
 0001:00005f10       ??_C@_0BF@LMAGFLHF@MLF_DONOTUPDATEPANEL@ 0000000180006f10     flags.obj
 0001:00005f28       ??_C@_0P@EPFBLPAE@MLF_HOLDTARGET@ 0000000180006f28     flags.obj
 0001:00005f38       ??_C@_08EBKEJHAL@MLF_NONE@ 0000000180006f38     flags.obj
 0001:00005f48       ??_C@_0M@JDMKDBDH@FFFS_COMMAS@ 0000000180006f48     flags.obj
 0001:00005f58       ??_C@_0P@JPMLNBKL@FFFS_FLOATSIZE@ 0000000180006f58     flags.obj
 0001:00005f68       ??_C@_0BE@NPKCCEJ@FFFS_SHOWBYTESINDEX@ 0000000180006f68     flags.obj
 0001:00005f80       ??_C@_0O@FPIOAIMC@FFFS_ECONOMIC@ 0000000180006f80     flags.obj
 0001:00005f90       ??_C@_0O@HFIGPFIH@FFFS_THOUSAND@ 0000000180006f90     flags.obj
 0001:00005fa0       ??_C@_0BC@LLLANJJO@FFFS_MINSIZEINDEX@ 0000000180006fa0     flags.obj
 0001:00005fb8       ??_C@_0BH@PEGBPJKE@FFFS_MINSIZEINDEX_MASK@ 0000000180006fb8     flags.obj
 0001:00005fd0       ??_C@_09PBPAKNEI@FFFS_NONE@ 0000000180006fd0     flags.obj
 0001:00005fe0       ??_C@_0L@NHEJGKCF@PF_PRELOAD@ 0000000180006fe0     flags.obj
 0001:00005ff0       ??_C@_0BB@GCINAIGN@PF_DISABLEPANELS@ 0000000180006ff0     flags.obj
 0001:00006008       ??_C@_09OENCMPGE@PF_EDITOR@ 0000000180007008     flags.obj
 0001:00006018       ??_C@_09NEKIJNNA@PF_VIEWER@ 0000000180007018     flags.obj
 0001:00006028       ??_C@_0P@MBLBBCNK@PF_FULLCMDLINE@ 0000000180007028     flags.obj
 0001:00006038       ??_C@_09GMFDAFKL@PF_DIALOG@ 0000000180007038     flags.obj
 0001:00006048       ??_C@_07MGEGJMPI@PF_NONE@  0000000180007048     flags.obj
 0001:00006050       ??_C@_0BD@EGELEIIG@IPLFLAGS_SEPARATOR@ 0000000180007050     flags.obj
 0001:00006068       ??_C@_0O@JBNJFHHK@IPLFLAGS_NONE@ 0000000180007068     flags.obj
 0001:00006078       ??_C@_0BD@KGHJOBGM@PMFLAGS_FULLSCREEN@ 0000000180007078     flags.obj
 0001:00006090       ??_C@_0BH@GDAAKEMH@PMFLAGS_DETAILEDSTATUS@ 0000000180007090     flags.obj
 0001:000060a8       ??_C@_0BI@BMHIBDMH@PMFLAGS_ALIGNEXTENSIONS@ 00000001800070a8     flags.obj
 0001:000060c0       ??_C@_0BH@KOFCBJBO@PMFLAGS_CASECONVERSION@ 00000001800070c0     flags.obj
 0001:000060d8       ??_C@_0N@DLFMCMOB@PMFLAGS_NONE@ 00000001800070d8     flags.obj
 0001:000060e8       ??_C@_0BD@PBMGDJEM@OPIF_DISABLEFILTER@ 00000001800070e8     flags.obj
 0001:00006100       ??_C@_0BH@FHBKALPD@OPIF_DISABLESORTGROUPS@ 0000000180007100     flags.obj
 0001:00006118       ??_C@_0BJ@NGLIANCL@OPIF_DISABLEHIGHLIGHTING@ 0000000180007118     flags.obj
 0001:00006138       ??_C@_0N@JANKJMLP@OPIF_ADDDOTS@ 0000000180007138     flags.obj
 0001:00006148       ??_C@_0BC@HOFHNJIG@OPIF_RAWSELECTION@ 0000000180007148     flags.obj
 0001:00006160       ??_C@_0P@OFEDJCO@OPIF_REALNAMES@ 0000000180007160     flags.obj
 0001:00006170       ??_C@_0BD@FPGMNAPD@OPIF_SHOWNAMESONLY@ 0000000180007170     flags.obj
 0001:00006188       ??_C@_0BJ@NMIFAPJD@OPIF_SHOWRIGHTALIGNNAMES@ 0000000180007188     flags.obj
 0001:000061a8       ??_C@_0BG@HGPMKHIE@OPIF_SHOWPRESERVECASE@ 00000001800071a8     flags.obj
 0001:000061c0       ??_C@_0BE@GJEJHNKJ@OPIF_COMPAREFATTIME@ 00000001800071c0     flags.obj
 0001:000061d8       ??_C@_0BB@PELHBPAM@OPIF_EXTERNALGET@ 00000001800071d8     flags.obj
 0001:000061f0       ??_C@_0BB@CFFPNDFK@OPIF_EXTERNALPUT@ 00000001800071f0     flags.obj
 0001:00006208       ??_C@_0BE@LKEMICNM@OPIF_EXTERNALDELETE@ 0000000180007208     flags.obj
 0001:00006220       ??_C@_0BD@JIMJPFEP@OPIF_EXTERNALMKDIR@ 0000000180007220     flags.obj
 0001:00006238       ??_C@_0BJ@CALDMPLF@OPIF_USEATTRHIGHLIGHTING@ 0000000180007238     flags.obj
 0001:00006258       ??_C@_0O@JHHHMHIG@OPIF_USECRC32@ 0000000180007258     flags.obj
 0001:00006268       ??_C@_0BB@PFDFAFHG@OPIF_USEFREESIZE@ 0000000180007268     flags.obj
 0001:00006280       ??_C@_0O@FJPLJDBC@OPIF_SHORTCUT@ 0000000180007280     flags.obj
 0001:00006290       ??_C@_09DOPJBMLM@OPIF_NONE@ 0000000180007290     flags.obj
 0001:000062a0       ??_C@_0L@GEHHKNBL@OPM_SILENT@ 00000001800072a0     flags.obj
 0001:000062b0       ??_C@_08EKEBOKEP@OPM_FIND@ 00000001800072b0     flags.obj
 0001:000062c0       ??_C@_08EHBLNDLO@OPM_VIEW@ 00000001800072c0     flags.obj
 0001:000062d0       ??_C@_08LAAGEMJG@OPM_EDIT@ 00000001800072d0     flags.obj
 0001:000062e0       ??_C@_0N@NDGKAFDM@OPM_TOPLEVEL@ 00000001800072e0     flags.obj
 0001:000062f0       ??_C@_09EBKAPHPA@OPM_DESCR@ 00000001800072f0     flags.obj
 0001:00006300       ??_C@_0O@OPDAGBBE@OPM_QUICKVIEW@ 0000000180007300     flags.obj
 0001:00006310       ??_C@_08LCEGJCAC@OPM_PGDN@ 0000000180007310     flags.obj
 0001:00006320       ??_C@_0N@HKCLLJDG@OPM_COMMANDS@ 0000000180007320     flags.obj
 0001:00006330       ??_C@_08EGEBMPBD@OPM_NONE@ 0000000180007330     flags.obj
 0001:00006340       ??_C@_0M@MIGJPBPE@FOSF_ACTIVE@ 0000000180007340     flags.obj
 0001:00006350       ??_C@_09FMOOJHDF@FOSF_NONE@ 0000000180007350     flags.obj
 0001:00006360       ??_C@_09HNBBLIGN@PCIF_NONE@ 0000000180007360     flags.obj
 0001:00006370       ??_C@_0BA@MAEBFMHC@FOREGROUND_BLUE@ 0000000180007370     flags.obj
 0001:00006380       ??_C@_0BB@PDFNMAI@FOREGROUND_GREEN@ 0000000180007380     flags.obj
 0001:00006398       ??_C@_0P@PBJHCFGA@FOREGROUND_RED@ 0000000180007398     flags.obj
 0001:000063a8       ??_C@_0BF@OOGEJCC@FOREGROUND_INTENSITY@ 00000001800073a8     flags.obj
 0001:000063c0       ??_C@_0BA@PIFINJCK@BACKGROUND_BLUE@ 00000001800073c0     flags.obj
 0001:000063d0       ??_C@_0BB@GKLNBMEL@BACKGROUND_GREEN@ 00000001800073d0     flags.obj
 0001:000063e8       ??_C@_0P@DANALJMC@BACKGROUND_RED@ 00000001800073e8     flags.obj
 0001:000063f8       ??_C@_0BF@NIGKKPCF@BACKGROUND_INTENSITY@ 00000001800073f8     flags.obj
 0001:00006410       ??_C@_0N@FEFOEFHG@CTRL_C_EVENT@ 0000000180007410     flags.obj
 0001:00006420       ??_C@_0BB@ELEIIFAE@CTRL_BREAK_EVENT@ 0000000180007420     flags.obj
 0001:00006438       ??_C@_0BB@KMPDMOKK@CTRL_CLOSE_EVENT@ 0000000180007438     flags.obj
 0001:00006450       ??_C@_0BC@MCKCEPAL@CTRL_LOGOFF_EVENT@ 0000000180007450     flags.obj
 0001:00006468       ??_C@_0BE@BCNEFGKM@CTRL_SHUTDOWN_EVENT@ 0000000180007468     flags.obj
 0001:00006480       ??_C@_0BC@BBOPHMOM@ENABLE_LINE_INPUT@ 0000000180007480     flags.obj
 0001:00006498       ??_C@_0BC@JPFKLHOC@ENABLE_ECHO_INPUT@ 0000000180007498     flags.obj
 0001:000064b0       ??_C@_0BH@EHINFMOF@ENABLE_PROCESSED_INPUT@ 00000001800074b0     flags.obj
 0001:000064c8       ??_C@_0BE@BLAHACNB@ENABLE_WINDOW_INPUT@ 00000001800074c8     flags.obj
 0001:000064e0       ??_C@_0BD@BJECBJPO@ENABLE_MOUSE_INPUT@ 00000001800074e0     flags.obj
 0001:000064f8       ??_C@_0BD@KJBPOMPN@ENABLE_INSERT_MODE@ 00000001800074f8     flags.obj
 0001:00006510       ??_C@_0BH@BJKMFKAO@ENABLE_QUICK_EDIT_MODE@ 0000000180007510     flags.obj
 0001:00006528       ??_C@_0BG@CBCHHIEH@ENABLE_EXTENDED_FLAGS@ 0000000180007528     flags.obj
 0001:00006540       ??_C@_0BF@PEBFEBKN@ENABLE_AUTO_POSITION@ 0000000180007540     flags.obj
 0001:00006558       ??_C@_0BI@MHKNPIFM@ENABLE_PROCESSED_OUTPUT@ 0000000180007558     flags.obj
 0001:00006570       ??_C@_0BK@CDKLKCHJ@ENABLE_WRAP_AT_EOL_OUTPUT@ 0000000180007570     flags.obj
 0001:00006590       ??_C@_09JBABGNAE@KEY_EVENT@ 0000000180007590     flags.obj
 0001:000065a0       ??_C@_0M@CPILDGOO@MOUSE_EVENT@ 00000001800075a0     flags.obj
 0001:000065b0       ??_C@_0BJ@OHDOHJKG@WINDOW_BUFFER_SIZE_EVENT@ 00000001800075b0     flags.obj
 0001:000065d0       ??_C@_0L@MPODFLFH@MENU_EVENT@ 00000001800075d0     flags.obj
 0001:000065e0       ??_C@_0M@LNGHCCGJ@FOCUS_EVENT@ 00000001800075e0     flags.obj
 0001:000065f0       ??_C@_0M@MKBGBFGO@CAPSLOCK_ON@ 00000001800075f0     flags.obj
 0001:00006600       ??_C@_0N@EMEOEKDA@ENHANCED_KEY@ 0000000180007600     flags.obj
 0001:00006610       ??_C@_0BC@GDHABBAP@RIGHT_ALT_PRESSED@ 0000000180007610     flags.obj
 0001:00006628       ??_C@_0BB@MCADLJJO@LEFT_ALT_PRESSED@ 0000000180007628     flags.obj
 0001:00006640       ??_C@_0BD@NEHHNAHO@RIGHT_CTRL_PRESSED@ 0000000180007640     flags.obj
 0001:00006658       ??_C@_0BC@FDNOAAAE@LEFT_CTRL_PRESSED@ 0000000180007658     flags.obj
 0001:00006670       ??_C@_0O@OGDFJMBK@SHIFT_PRESSED@ 0000000180007670     flags.obj
 0001:00006680       ??_C@_0L@IMGKKBIM@NUMLOCK_ON@ 0000000180007680     flags.obj
 0001:00006690       ??_C@_0O@LAHFNPLG@SCROLLLOCK_ON@ 0000000180007690     flags.obj
 0001:000066a0       ??_C@_0BN@HACKHGAB@FROM_LEFT_1ST_BUTTON_PRESSED@ 00000001800076a0     flags.obj
 0001:000066c0       ??_C@_0BJ@JECFAJNJ@RIGHTMOST_BUTTON_PRESSED@ 00000001800076c0     flags.obj
 0001:000066e0       ??_C@_0BN@BJCFPKCG@FROM_LEFT_2ND_BUTTON_PRESSED@ 00000001800076e0     flags.obj
 0001:00006700       ??_C@_0BN@PMJNFPGM@FROM_LEFT_3RD_BUTTON_PRESSED@ 0000000180007700     flags.obj
 0001:00006720       ??_C@_0BN@CNMHAAPD@FROM_LEFT_4TH_BUTTON_PRESSED@ 0000000180007720     flags.obj
 0001:00006740       ??_C@_0M@KKBDEELB@MOUSE_MOVED@ 0000000180007740     flags.obj
 0001:00006750       ??_C@_0N@EDCKBGJE@DOUBLE_CLICK@ 0000000180007750     flags.obj
 0001:00006760       ??_C@_0O@GABDOPO@MOUSE_WHEELED@ 0000000180007760     flags.obj
 0001:00006770       ??_C@_0BA@OOKCCMHH@KEY_WOW64_32KEY@ 0000000180007770     flags.obj
 0001:00006780       ??_C@_0BA@DBCPEIGE@KEY_WOW64_64KEY@ 0000000180007780     flags.obj
 0001:00008b0c       ??_C@_06ICDCBJPI@Colors@   0000000180009b0c     keysandcolors.obj
 0001:00008b14       ??_C@_05GALAPKHH@Guids@    0000000180009b14     keysandcolors.obj
 0001:000093d8       ??_C@_01EEMJAFIK@?6@       000000018000a3d8     lflua.obj
 0001:000093e0       ??_C@_0BB@BJDGDOHH@cannot?5?$CFs?5?$CFs?3?5?$CFs@ 000000018000a3e0     lflua.obj
 0001:000093f4       ??_C@_03PKPBNCAL@?o?$LL?$LP@ 000000018000a3f4     lflua.obj
 0001:000093f8       ??_C@_06CCPPALKB@?$DNstdin@ 000000018000a3f8     lflua.obj
 0001:00009400       ??_C@_01EOFPKCAF@?$EA@     000000018000a400     lflua.obj
 0001:00009404       ??_C@_04PMOCAHAA@open@     000000018000a404     lflua.obj
 0001:0000940c       ??_C@_15JJPIMNBO@?$AAr?$AAb@ 000000018000a40c     lflua.obj
 0001:00009414       ??_C@_06IEGCHAII@reopen@   000000018000a414     lflua.obj
 0001:0000941c       ??_C@_04POLDLDMI@read@     000000018000a41c     lflua.obj
 0001:00009424       ??_C@_02LOCGON@?$AA?$AA@   000000018000a424     lflua.obj
 0001:00009430       regex_methods              000000018000a430     lregex.obj
 0001:000094f0       regex_functions            000000018000a4f0     lregex.obj
 0001:00009e68       ??_C@_04CKFJHKAP@find@     000000018000ae68     lregex.obj
 0001:00009e70       ??_C@_04GOLEAPFD@gsub@     000000018000ae70     lregex.obj
 0001:00009e78       ??_C@_05FNONLPDI@match@    000000018000ae78     lregex.obj
 0001:00009e80       ??_C@_04MGEIEJAD@exec@     000000018000ae80     lregex.obj
 0001:00009e88       ??_C@_05GFGPIPHI@findW@    000000018000ae88     lregex.obj
 0001:00009e90       ??_C@_05HPGHPNC@gsubW@     000000018000ae90     lregex.obj
 0001:00009e98       ??_C@_06NNKFJOLC@matchW@   000000018000ae98     lregex.obj
 0001:00009ea0       ??_C@_05GMDFNCGA@execW@    000000018000aea0     lregex.obj
 0001:00009ea8       ??_C@_0O@OJAOCNID@bracketscount@ 000000018000aea8     lregex.obj
 0001:00009eb8       ??_C@_04BDLIKKMN@__gc@     000000018000aeb8     lregex.obj
 0001:00009ec0       ??_C@_06DPFCLDIO@gmatch@   000000018000aec0     lregex.obj
 0001:00009ec8       ??_C@_07PPMFDHAH@gmatchW@  000000018000aec8     lregex.obj
 0001:00009ed0       ??_C@_09KIEPBIJC@far_regex@ 000000018000aed0     lregex.obj
 0001:00009ee0       ??_C@_0BO@PBOFMCLL@attempt?5to?5access?5freed?5regex@ 000000018000aee0     lregex.obj
 0001:00009f00       ??_C@_07IHINEPFG@?$CFs?5?$CI?$CFp?$CJ@ 000000018000af00     lregex.obj
 0001:00009f08       ??_C@_01KMDKNFGN@?1@       000000018000af08     lregex.obj
 0001:00009f10       ??_C@_0BE@BBBEAHLK@RECTL_CREATE?5failed@ 000000018000af10     lregex.obj
 0001:00009f28       ??_C@_0BL@HEFMPIBG@invalid?5regular?5expression@ 000000018000af28     lregex.obj
 0001:00009f48       ??_C@_0BK@JCLHPPNA@cannot?5add?5?$CFd?5stack?5slots@ 000000018000af48     lregex.obj
 0001:00009f68       ??_C@_0BM@MOHHGMBK@string?5or?5table?5or?5function@ 000000018000af68     lregex.obj
 0001:00009f88       ??_C@_0CG@IDFLGMFM@replace?5string?3?5invalid?5capture@ 000000018000af88     lregex.obj
 0001:00009fb0       ??_C@_0BJ@IMAIDFKH@invalid?5replacement?5type@ 000000018000afb0     lregex.obj
 0001:00009fd0       ??_C@_0BE@KPDOHKBE@invalid?5return?5type@ 000000018000afd0     lregex.obj
 0001:00009fe8       ??_C@_07NHABFFHN@__index@  000000018000afe8     lregex.obj
 0001:00009ff0       ??_C@_05FGAODPCE@regex@    000000018000aff0     lregex.obj
 0001:0000a8c0       ??_C@_0BC@PMGNICBE@MacroPluginReturn@ 000000018000b8c0     luamacro.obj
 0001:0000a8d4       ??_C@_02JIEIHMJD@wl@       000000018000b8d4     luamacro.obj
 0001:0000a8d8       ??_C@_15PMCGDJNJ@?$AAO?$AAK@ 000000018000b8d8     luamacro.obj
 0001:0000a8e0       ??_C@_1BC@GBFPAMBP@?$AAL?$AAu?$AAa?$AAM?$AAa?$AAc?$AAr?$AAo@ 000000018000b8e0     luamacro.obj
 0001:0000a900       ??_C@_1FA@DAFHIDEP@?$AAt?$AAo?$AAo?$AA?5?$AAm?$AAa?$AAn?$AAy?$AA?5?$AAv?$AAa?$AAl?$AAu?$AAe?$AAs@ 000000018000b900     luamacro.obj
 0001:0000a950       ??_C@_0BN@ICDOMFBB@invalid?5argument?5?$CD?$CFd?5to?5?8?$CFs?8@ 000000018000b950     luamacro.obj
 0001:0000a970       ??_C@_0BB@FCMFBGOM@invalid?5argument@ 000000018000b970     luamacro.obj
 0001:0000b230       usercontrol_methods        000000018000c230     lusercontrol.obj
 0001:0000b280       usercontrol_functions      000000018000c280     lusercontrol.obj
 0001:0000b2a0       ??_C@_05MNDELLDN@__len@    000000018000c2a0     lusercontrol.obj
 0001:0000b2a8       ??_C@_0L@GADKNKH@__newindex@ 000000018000c2a8     lusercontrol.obj
 0001:0000b2b8       ??_C@_0BC@KFJDHEIC@CreateUserControl@ 000000018000c2b8     lusercontrol.obj
 0001:0000b2d0       ??_C@_0BA@MDNLMOMP@far_usercontrol@ 000000018000c2d0     lusercontrol.obj
 0001:0000b2e0       ??_C@_0BH@DOPNHMGD@bounds?5checking?5failed@ 000000018000c2e0     lusercontrol.obj
 0001:0000b2f8       ??_C@_09LDLEBFOB@rawhandle@ 000000018000c2f8     lusercontrol.obj
 0001:0000b304       ??_C@_04IMAAEPPE@Char@     000000018000c304     lusercontrol.obj
 0001:0000b310       ??_C@_0L@PLFFHFAH@Attributes@ 000000018000c310     lusercontrol.obj
 0001:0000b320       ??_C@_0BD@BPIMECDH@X?5must?5be?5positive@ 000000018000c320     lusercontrol.obj
 0001:0000b338       ??_C@_0BD@MIGOMCGP@Y?5must?5be?5positive@ 000000018000c338     lusercontrol.obj
 0001:0000b368       FarFileFilterType          000000018000c368     service.obj
 0001:0000b378       FarTimerType               000000018000c378     service.obj
 0001:0000b388       FarTimerQueueKey           000000018000c388     service.obj
 0001:0000b398       FarDialogType              000000018000c398     service.obj
 0001:0000b3a8       SettingsType               000000018000c3a8     service.obj
 0001:0000b3b8       SettingsHandles            000000018000c3b8     service.obj
 0001:0000b3d0       PluginHandleType           000000018000c3d0     service.obj
 0001:0000b3e0       AddMacroDataType           000000018000c3e0     service.obj
 0001:0000b3f0       SavedScreenType            000000018000c3f0     service.obj
 0001:0000b400       FAR_VIRTUALKEYS            000000018000c400     service.obj
 0001:0000b410       FAR_FLAGSTABLE             000000018000c410     service.obj
 0001:0000b420       FAR_DN_STORAGE             000000018000c420     service.obj
 0001:0000bd00       timer_methods              000000018000cd00     service.obj
 0001:0000bd50       filefilter_methods         000000018000cd50     service.obj
 0001:0000bdc0       dialog_methods             000000018000cdc0     service.obj
 0001:0000be10       Settings_methods           000000018000ce10     service.obj
 0001:0000beb0       editor_funcs               000000018000ceb0     service.obj
 0001:0000c140       viewer_funcs               000000018000d140     service.obj
 0001:0000c1e0       panel_funcs                000000018000d1e0     service.obj
 0001:0000c410       far_funcs                  000000018000d410     service.obj
 0001:0000c8b0       far_Dialog                 000000018000d8b0     service.obj
 0001:0000cc00       api_functions              000000018000dc00     service.obj
 0001:0000ccc0       ??_C@_07PHPIFDKI@LBUTTON@  000000018000dcc0     service.obj
 0001:0000ccc8       ??_C@_07JOMJHALB@RBUTTON@  000000018000dcc8     service.obj
 0001:0000ccd0       ??_C@_06JHILMIHF@CANCEL@   000000018000dcd0     service.obj
 0001:0000ccd8       ??_C@_07DLFCFDDG@MBUTTON@  000000018000dcd8     service.obj
 0001:0000cce0       ??_C@_08OPILMHEG@XBUTTON1@ 000000018000dce0     service.obj
 0001:0000ccf0       ??_C@_08MEKGJEIF@XBUTTON2@ 000000018000dcf0     service.obj
 0001:0000ccfc       ??_C@_04FJBHJJME@BACK@     000000018000dcfc     service.obj
 0001:0000cd04       ??_C@_03CJMDHCGG@TAB@      000000018000dd04     service.obj
 0001:0000cd08       ??_C@_05PONODPI@CLEAR@     000000018000dd08     service.obj
 0001:0000cd10       ??_C@_06LJMOENAO@RETURN@   000000018000dd10     service.obj
 0001:0000cd18       ??_C@_05OAHIEJBI@SHIFT@    000000018000dd18     service.obj
 0001:0000cd20       ??_C@_07DBEDOPMC@CONTROL@  000000018000dd20     service.obj
 0001:0000cd28       ??_C@_04IILMDFMO@MENU@     000000018000dd28     service.obj
 0001:0000cd30       ??_C@_05DIAHPDGL@PAUSE@    000000018000dd30     service.obj
 0001:0000cd38       ??_C@_07OPCFNGJB@CAPITAL@  000000018000dd38     service.obj
 0001:0000cd40       ??_C@_04KGDAIAGM@KANA@     000000018000dd40     service.obj
 0001:0000cd48       ??_C@_05PPKJGOLB@JUNJA@    000000018000dd48     service.obj
 0001:0000cd50       ??_C@_05JEIAEFOF@FINAL@    000000018000dd50     service.obj
 0001:0000cd58       ??_C@_05CHABPOPI@HANJA@    000000018000dd58     service.obj
 0001:0000cd60       ??_C@_06CDPDIIDH@ESCAPE@   000000018000dd60     service.obj
 0001:0000cd68       ??_C@_0L@ODNCKDCK@NONCONVERT@ 000000018000dd68     service.obj
 0001:0000cd74       ??_C@_06INBBKPI@ACCEPT@    000000018000dd74     service.obj
 0001:0000cd80       ??_C@_0L@HEHNEBED@MODECHANGE@ 000000018000dd80     service.obj
 0001:0000cd8c       ??_C@_05CAEOFMEP@SPACE@    000000018000dd8c     service.obj
 0001:0000cd94       ??_C@_05BFDHCIJM@PRIOR@    000000018000dd94     service.obj
 0001:0000cd9c       ??_C@_04MOKMKBJN@NEXT@     000000018000dd9c     service.obj
 0001:0000cda4       ??_C@_03JMGAKCCH@END@      000000018000dda4     service.obj
 0001:0000cda8       ??_C@_04GHGFPGNC@HOME@     000000018000dda8     service.obj
 0001:0000cdb0       ??_C@_04KCNEHMIH@LEFT@     000000018000ddb0     service.obj
 0001:0000cdb8       ??_C@_02NAHCJHOC@UP@       000000018000ddb8     service.obj
 0001:0000cdbc       ??_C@_05PMAFOJDE@RIGHT@    000000018000ddbc     service.obj
 0001:0000cdc4       ??_C@_04FANAOELO@DOWN@     000000018000ddc4     service.obj
 0001:0000cdcc       ??_C@_06LCPJPOPK@SELECT@   000000018000ddcc     service.obj
 0001:0000cdd4       ??_C@_05ECKPOFCN@PRINT@    000000018000ddd4     service.obj
 0001:0000cde0       ??_C@_07LBDEDADF@EXECUTE@  000000018000dde0     service.obj
 0001:0000cde8       ??_C@_08EMOKHGD@SNAPSHOT@  000000018000dde8     service.obj
 0001:0000cdf4       ??_C@_06OEMEAEKN@INSERT@   000000018000ddf4     service.obj
 0001:0000cdfc       ??_C@_06FKDAMKFP@DELETE@   000000018000ddfc     service.obj
 0001:0000ce04       ??_C@_04DOKPJKJF@HELP@     000000018000de04     service.obj
 0001:0000ce0c       ??_C@_01GBGANLPD@0@        000000018000de0c     service.obj
 0001:0000ce10       ??_C@_01HIHLOKLC@1@        000000018000de10     service.obj
 0001:0000ce14       ??_C@_01FDFGLJHB@2@        000000018000de14     service.obj
 0001:0000ce18       ??_C@_01EKENIIDA@3@        000000018000de18     service.obj
 0001:0000ce1c       ??_C@_01FAMBOPH@4@         000000018000de1c     service.obj
 0001:0000ce20       ??_C@_01BMBHCPLG@5@        000000018000de20     service.obj
 0001:0000ce24       ??_C@_01DHDKHMHF@6@        000000018000de24     service.obj
 0001:0000ce28       ??_C@_01COCBENDE@7@        000000018000de28     service.obj
 0001:0000ce2c       ??_C@_01KJLJFBPL@8@        000000018000de2c     service.obj
 0001:0000ce30       ??_C@_01LAKCGALK@9@        000000018000de30     service.obj
 0001:0000ce34       ??_C@_01FHEEJDEE@A@        000000018000de34     service.obj
 0001:0000ce38       ??_C@_01HMGJMAIH@B@        000000018000de38     service.obj
 0001:0000ce3c       ??_C@_01GFHCPBMG@C@        000000018000de3c     service.obj
 0001:0000ce40       ??_C@_01CKDDGHAB@D@        000000018000de40     service.obj
 0001:0000ce44       ??_C@_01DDCIFGEA@E@        000000018000de44     service.obj
 0001:0000ce48       ??_C@_01BIAFAFID@F@        000000018000de48     service.obj
 0001:0000ce4c       ??_C@_01BBODEMC@G@         000000018000de4c     service.obj
 0001:0000ce50       ??_C@_01IGIGCIAN@H@        000000018000de50     service.obj
 0001:0000ce54       ??_C@_01JPJNBJEM@I@        000000018000de54     service.obj
 0001:0000ce58       ??_C@_01LELAEKIP@J@        000000018000de58     service.obj
 0001:0000ce5c       ??_C@_01KNKLHLMO@K@        000000018000de5c     service.obj
 0001:0000ce60       ??_C@_01OCOKONAJ@L@        000000018000de60     service.obj
 0001:0000ce64       ??_C@_01PLPBNMEI@M@        000000018000de64     service.obj
 0001:0000ce68       ??_C@_01NANMIPIL@N@        000000018000de68     service.obj
 0001:0000ce6c       ??_C@_01MJMHLOMK@O@        000000018000de6c     service.obj
 0001:0000ce70       ??_C@_01EJNLAFE@P@         000000018000de70     service.obj
 0001:0000ce74       ??_C@_01BNIGIBBF@Q@        000000018000de74     service.obj
 0001:0000ce78       ??_C@_01DGKLNCNG@R@        000000018000de78     service.obj
 0001:0000ce7c       ??_C@_01CPLAODJH@S@        000000018000de7c     service.obj
 0001:0000ce80       ??_C@_01GAPBHFFA@T@        000000018000de80     service.obj
 0001:0000ce84       ??_C@_01HJOKEEBB@U@        000000018000de84     service.obj
 0001:0000ce88       ??_C@_01FCMHBHNC@V@        000000018000de88     service.obj
 0001:0000ce8c       ??_C@_01ELNMCGJD@W@        000000018000de8c     service.obj
 0001:0000ce90       ??_C@_01MMEEDKFM@X@        000000018000de90     service.obj
 0001:0000ce94       ??_C@_01NFFPALBN@Y@        000000018000de94     service.obj
 0001:0000ce98       ??_C@_01POHCFINO@Z@        000000018000de98     service.obj
 0001:0000ce9c       ??_C@_04ODLFFOHF@LWIN@     000000018000de9c     service.obj
 0001:0000cea4       ??_C@_04DMGFHHJG@RWIN@     000000018000dea4     service.obj
 0001:0000ceac       ??_C@_04GKGJFGJO@APPS@     000000018000deac     service.obj
 0001:0000ceb4       ??_C@_05DJAECLDN@SLEEP@    000000018000deb4     service.obj
 0001:0000cec0       ??_C@_07NHIPMMJH@NUMPAD0@  000000018000dec0     service.obj
 0001:0000cec8       ??_C@_07MOJEPNNG@NUMPAD1@  000000018000dec8     service.obj
 0001:0000ced0       ??_C@_07OFLJKOBF@NUMPAD2@  000000018000ded0     service.obj
 0001:0000ced8       ??_C@_07PMKCJPFE@NUMPAD3@  000000018000ded8     service.obj
 0001:0000cee0       ??_C@_07LDODAJJD@NUMPAD4@  000000018000dee0     service.obj
 0001:0000cee8       ??_C@_07KKPIDINC@NUMPAD5@  000000018000dee8     service.obj
 0001:0000cef0       ??_C@_07IBNFGLBB@NUMPAD6@  000000018000def0     service.obj
 0001:0000cef8       ??_C@_07JIMOFKFA@NUMPAD7@  000000018000def8     service.obj
 0001:0000cf00       ??_C@_07BPFGEGJP@NUMPAD8@  000000018000df00     service.obj
 0001:0000cf08       ??_C@_07GENHHNO@NUMPAD9@   000000018000df08     service.obj
 0001:0000cf10       ??_C@_08LDEOAAGM@MULTIPLY@ 000000018000df10     service.obj
 0001:0000cf1c       ??_C@_03BOJFLAKG@ADD@      000000018000df1c     service.obj
 0001:0000cf20       ??_C@_09POPINEFK@SEPARATOR@ 000000018000df20     service.obj
 0001:0000cf30       ??_C@_08MGBEENML@SUBTRACT@ 000000018000df30     service.obj
 0001:0000cf40       ??_C@_07LJPMJDLL@DECIMAL@  000000018000df40     service.obj
 0001:0000cf48       ??_C@_06FBFCJJMP@DIVIDE@   000000018000df48     service.obj
 0001:0000cf50       ??_C@_02LCPENACN@F1@       000000018000df50     service.obj
 0001:0000cf54       ??_C@_02JJNJIDOO@F2@       000000018000df54     service.obj
 0001:0000cf58       ??_C@_02IAMCLCKP@F3@       000000018000df58     service.obj
 0001:0000cf5c       ??_C@_02MPIDCEGI@F4@       000000018000df5c     service.obj
 0001:0000cf60       ??_C@_02NGJIBFCJ@F5@       000000018000df60     service.obj
 0001:0000cf64       ??_C@_02PNLFEGOK@F6@       000000018000df64     service.obj
 0001:0000cf68       ??_C@_02OEKOHHKL@F7@       000000018000df68     service.obj
 0001:0000cf6c       ??_C@_02GDDGGLGE@F8@       000000018000df6c     service.obj
 0001:0000cf70       ??_C@_02HKCNFKCF@F9@       000000018000df70     service.obj
 0001:0000cf74       ??_C@_03JKCLJOFG@F10@      000000018000df74     service.obj
 0001:0000cf78       ??_C@_03IDDAKPBH@F11@      000000018000df78     service.obj
 0001:0000cf7c       ??_C@_03KIBNPMNE@F12@      000000018000df7c     service.obj
 0001:0000cf80       ??_C@_03LBAGMNJF@F13@      000000018000df80     service.obj
 0001:0000cf84       ??_C@_03POEHFLFC@F14@      000000018000df84     service.obj
 0001:0000cf88       ??_C@_03OHFMGKBD@F15@      000000018000df88     service.obj
 0001:0000cf8c       ??_C@_03MMHBDJNA@F16@      000000018000df8c     service.obj
 0001:0000cf90       ??_C@_03NFGKAIJB@F17@      000000018000df90     service.obj
 0001:0000cf94       ??_C@_03FCPCBEFO@F18@      000000018000df94     service.obj
 0001:0000cf98       ??_C@_03ELOJCFBP@F19@      000000018000df98     service.obj
 0001:0000cf9c       ??_C@_03JIGNCAAP@F20@      000000018000df9c     service.obj
 0001:0000cfa0       ??_C@_03IBHGBBEO@F21@      000000018000dfa0     service.obj
 0001:0000cfa4       ??_C@_03KKFLECIN@F22@      000000018000dfa4     service.obj
 0001:0000cfa8       ??_C@_03LDEAHDMM@F23@      000000018000dfa8     service.obj
 0001:0000cfac       ??_C@_03PMABOFAL@F24@      000000018000dfac     service.obj
 0001:0000cfb0       ??_C@_07FLMEHHJP@NUMLOCK@  000000018000dfb0     service.obj
 0001:0000cfb8       ??_C@_06FNIKALAE@SCROLL@   000000018000dfb8     service.obj
 0001:0000cfc0       ??_C@_0O@DBBJDALK@OEM_NEC_EQUAL@ 000000018000dfc0     service.obj
 0001:0000cfd0       ??_C@_0P@JKGCFGCD@OEM_FJ_MASSHOU@ 000000018000dfd0     service.obj
 0001:0000cfe0       ??_C@_0P@NIEOFNLG@OEM_FJ_TOUROKU@ 000000018000dfe0     service.obj
 0001:0000cff0       ??_C@_0M@IBEHGLCM@OEM_FJ_LOYA@ 000000018000dff0     service.obj
 0001:0000d000       ??_C@_0M@FOJHECMP@OEM_FJ_ROYA@ 000000018000e000     service.obj
 0001:0000d00c       ??_C@_06EPHNCIMI@LSHIFT@   000000018000e00c     service.obj
 0001:0000d014       ??_C@_06HIJMMPFL@RSHIFT@   000000018000e014     service.obj
 0001:0000d020       ??_C@_08IKMONEBG@LCONTROL@ 000000018000e020     service.obj
 0001:0000d030       ??_C@_08OOMMENPF@RCONTROL@ 000000018000e030     service.obj
 0001:0000d03c       ??_C@_05IHMGKJGH@LMENU@    000000018000e03c     service.obj
 0001:0000d044       ??_C@_05LOBKMKIM@RMENU@    000000018000e044     service.obj
 0001:0000d050       ??_C@_0N@OAJIELLG@BROWSER_BACK@ 000000018000e050     service.obj
 0001:0000d060       ??_C@_0BA@ENOAJOGH@BROWSER_FORWARD@ 000000018000e060     service.obj
 0001:0000d070       ??_C@_0BA@GDNDIDGJ@BROWSER_REFRESH@ 000000018000e070     service.obj
 0001:0000d080       ??_C@_0N@HKPDGANH@BROWSER_STOP@ 000000018000e080     service.obj
 0001:0000d090       ??_C@_0P@BEAEBJDD@BROWSER_SEARCH@ 000000018000e090     service.obj
 0001:0000d0a0       ??_C@_0BC@BOMJIH@BROWSER_FAVORITES@ 000000018000e0a0     service.obj
 0001:0000d0b8       ??_C@_0N@NOOKCEKA@BROWSER_HOME@ 000000018000e0b8     service.obj
 0001:0000d0c8       ??_C@_0M@ENOHKBMG@VOLUME_MUTE@ 000000018000e0c8     service.obj
 0001:0000d0d8       ??_C@_0M@JOOBBDNO@VOLUME_DOWN@ 000000018000e0d8     service.obj
 0001:0000d0e8       ??_C@_09MGPMNMJC@VOLUME_UP@ 000000018000e0e8     service.obj
 0001:0000d0f8       ??_C@_0BB@KLAENPA@MEDIA_NEXT_TRACK@ 000000018000e0f8     service.obj
 0001:0000d110       ??_C@_0BB@CMOIJKPH@MEDIA_PREV_TRACK@ 000000018000e110     service.obj
 0001:0000d128       ??_C@_0L@KBJOCDHK@MEDIA_STOP@ 000000018000e128     service.obj
 0001:0000d138       ??_C@_0BB@HAEMIJHO@MEDIA_PLAY_PAUSE@ 000000018000e138     service.obj
 0001:0000d150       ??_C@_0M@GCIKMBID@LAUNCH_MAIL@ 000000018000e150     service.obj
 0001:0000d160       ??_C@_0BE@FADJJAPM@LAUNCH_MEDIA_SELECT@ 000000018000e160     service.obj
 0001:0000d178       ??_C@_0M@MGLJIDDM@LAUNCH_APP1@ 000000018000e178     service.obj
 0001:0000d188       ??_C@_0M@ONJENAPP@LAUNCH_APP2@ 000000018000e188     service.obj
 0001:0000d194       ??_C@_05OIODNPAD@OEM_1@    000000018000e194     service.obj
 0001:0000d1a0       ??_C@_08LDJEIPBH@OEM_PLUS@ 000000018000e1a0     service.obj
 0001:0000d1b0       ??_C@_09CLPFJEOD@OEM_COMMA@ 000000018000e1b0     service.obj
 0001:0000d1c0       ??_C@_09OGMLCNMG@OEM_MINUS@ 000000018000e1c0     service.obj
 0001:0000d1d0       ??_C@_0L@DNNMNDGM@OEM_PERIOD@ 000000018000e1d0     service.obj
 0001:0000d1dc       ??_C@_05MDMOIMMA@OEM_2@    000000018000e1dc     service.obj
 0001:0000d1e4       ??_C@_05NKNFLNIB@OEM_3@    000000018000e1e4     service.obj
 0001:0000d1ec       ??_C@_05JFJECLEG@OEM_4@    000000018000e1ec     service.obj
 0001:0000d1f4       ??_C@_05IMIPBKAH@OEM_5@    000000018000e1f4     service.obj
 0001:0000d1fc       ??_C@_05KHKCEJME@OEM_6@    000000018000e1fc     service.obj
 0001:0000d204       ??_C@_05LOLJHIIF@OEM_7@    000000018000e204     service.obj
 0001:0000d20c       ??_C@_05DJCBGEEK@OEM_8@    000000018000e20c     service.obj
 0001:0000d218       ??_C@_07PEFKMFIE@OEM_102@  000000018000e218     service.obj
 0001:0000d220       ??_C@_0L@EFLJCPAM@PROCESSKEY@ 000000018000e220     service.obj
 0001:0000d22c       ??_C@_06HOICDKCB@PACKET@   000000018000e22c     service.obj
 0001:0000d238       ??_C@_09CAKPMKHM@OEM_RESET@ 000000018000e238     service.obj
 0001:0000d248       ??_C@_08INMNLJCK@OEM_JUMP@ 000000018000e248     service.obj
 0001:0000d258       ??_C@_07JNOAEEG@OEM_PA1@   000000018000e258     service.obj
 0001:0000d260       ??_C@_07CCPDFHIF@OEM_PA2@  000000018000e260     service.obj
 0001:0000d268       ??_C@_07DLOIGGME@OEM_PA3@  000000018000e268     service.obj
 0001:0000d270       ??_C@_0L@OCAIHDP@OEM_WSCTRL@ 000000018000e270     service.obj
 0001:0000d27c       ??_C@_04BNGOAFAJ@ATTN@     000000018000e27c     service.obj
 0001:0000d284       ??_C@_05HGAHFFFL@CRSEL@    000000018000e284     service.obj
 0001:0000d28c       ??_C@_05OKOOKOOH@EXSEL@    000000018000e28c     service.obj
 0001:0000d294       ??_C@_05CCFENDFJ@EREOF@    000000018000e294     service.obj
 0001:0000d29c       ??_C@_04MKCNCBEG@PLAY@     000000018000e29c     service.obj
 0001:0000d2a4       ??_C@_04LGBIGMFG@ZOOM@     000000018000e2a4     service.obj
 0001:0000d2ac       ??_C@_06LJIOOKLP@NONAME@   000000018000e2ac     service.obj
 0001:0000d2b4       ??_C@_03KCLDMPAE@PA1@      000000018000e2b4     service.obj
 0001:0000d2b8       ??_C@_09MBBEHOCK@OEM_CLEAR@ 000000018000e2b8     service.obj
 0001:0000d2c4       ??_C@_05LCLENNFI@table@    000000018000e2c4     service.obj
 0001:0000d2cc       ??_C@_06ICGJLFIM@string@   000000018000e2cc     service.obj
 0001:0000d2d8       ??_C@_0P@LKPINHLK@FreeFileFilter@ 000000018000e2d8     service.obj
 0001:0000d2e8       ??_C@_0BA@JGEOEAE@OpenFiltersMenu@ 000000018000e2e8     service.obj
 0001:0000d2f8       ??_C@_0BB@OPPOFOAK@StartingToFilter@ 000000018000e2f8     service.obj
 0001:0000d310       ??_C@_0P@JDMCHDIM@IsFileInFilter@ 000000018000e310     service.obj
 0001:0000d320       ??_C@_04MIIPNNEF@send@     000000018000e320     service.obj
 0001:0000d328       ??_C@_06JBKGCNBB@Delete@   000000018000e328     service.obj
 0001:0000d330       ??_C@_04PAFOOALK@Enum@     000000018000e330     service.obj
 0001:0000d338       ??_C@_04HJMOFLDF@Free@     000000018000e338     service.obj
 0001:0000d340       ??_C@_03NNDHPFFO@Get@      000000018000e340     service.obj
 0001:0000d344       ??_C@_03CEMDFJG@Set@       000000018000e344     service.obj
 0001:0000d348       ??_C@_0N@OELJMCEC@CreateSubkey@ 000000018000e348     service.obj
 0001:0000d358       ??_C@_0L@CPCKAMD@OpenSubkey@ 000000018000e358     service.obj
 0001:0000d368       ??_C@_08EGJLHNCO@AddColor@ 000000018000e368     service.obj
 0001:0000d378       ??_C@_0BD@DOFEEDDC@AddSessionBookmark@ 000000018000e378     service.obj
 0001:0000d390       ??_C@_0BG@IGFHDIIN@ClearSessionBookmarks@ 000000018000e390     service.obj
 0001:0000d3a8       ??_C@_08PDEJHGJI@DelColor@ 000000018000e3a8     service.obj
 0001:0000d3b8       ??_C@_0M@LPIECDD@DeleteBlock@ 000000018000e3b8     service.obj
 0001:0000d3c8       ??_C@_0L@BCLIBKOC@DeleteChar@ 000000018000e3c8     service.obj
 0001:0000d3d8       ??_C@_0BG@KOELEFCN@DeleteSessionBookmark@ 000000018000e3d8     service.obj
 0001:0000d3f0       ??_C@_0N@EKENACAE@DeleteString@ 000000018000e3f0     service.obj
 0001:0000d400       ??_C@_06MJDIICIN@Editor@   000000018000e400     service.obj
 0001:0000d408       ??_C@_0L@HDLPOLMA@ExpandTabs@ 000000018000e408     service.obj
 0001:0000d418       ??_C@_0N@MGAOADJN@GetBookmarks@ 000000018000e418     service.obj
 0001:0000d428       ??_C@_08JOPFJIPE@GetColor@ 000000018000e428     service.obj
 0001:0000d438       ??_C@_0M@FECPLAMN@GetFileName@ 000000018000e438     service.obj
 0001:0000d448       ??_C@_07NAJNLNAF@GetInfo@  000000018000e448     service.obj
 0001:0000d450       ??_C@_0N@KIILHCLH@GetSelection@ 000000018000e450     service.obj
 0001:0000d460       ??_C@_0BE@LBJJGOGD@GetSessionBookmarks@ 000000018000e460     service.obj
 0001:0000d478       ??_C@_09HBLKHMEA@GetString@ 000000018000e478     service.obj
 0001:0000d488       ??_C@_0L@IDFHDAHP@GetStringW@ 000000018000e488     service.obj
 0001:0000d498       ??_C@_0N@ICPGLOEG@InsertString@ 000000018000e498     service.obj
 0001:0000d4a8       ??_C@_0L@JMOIGJIA@InsertText@ 000000018000e4a8     service.obj
 0001:0000d4b8       ??_C@_0M@BINOKANK@InsertTextW@ 000000018000e4b8     service.obj
 0001:0000d4c8       ??_C@_0BE@CNGODNDI@NextSessionBookmark@ 000000018000e4c8     service.obj
 0001:0000d4e0       ??_C@_0BE@IEBIGOAP@PrevSessionBookmark@ 000000018000e4e0     service.obj
 0001:0000d4f8       ??_C@_0N@FNCEPAJJ@ProcessInput@ 000000018000e4f8     service.obj
 0001:0000d508       ??_C@_04GMBKPCGK@Quit@     000000018000e508     service.obj
 0001:0000d510       ??_C@_09KINLOJJJ@ReadInput@ 000000018000e510     service.obj
 0001:0000d520       ??_C@_09DBPLBJBJ@RealToTab@ 000000018000e520     service.obj
 0001:0000d52c       ??_C@_06KAPLBEK@Redraw@    000000018000e52c     service.obj
 0001:0000d538       ??_C@_08FBDDPFPJ@SaveFile@ 000000018000e538     service.obj
 0001:0000d544       ??_C@_06HJGPBJLE@Select@   000000018000e544     service.obj
 0001:0000d550       ??_C@_09PPEOOGEC@SetKeyBar@ 000000018000e550     service.obj
 0001:0000d560       ??_C@_08CCKJEGOF@SetParam@ 000000018000e560     service.obj
 0001:0000d570       ??_C@_0M@GKIFPNAD@SetPosition@ 000000018000e570     service.obj
 0001:0000d580       ??_C@_09FPPPFNNC@SetString@ 000000018000e580     service.obj
 0001:0000d590       ??_C@_0L@JNHIIHDG@SetStringW@ 000000018000e590     service.obj
 0001:0000d5a0       ??_C@_08GMCCAJLF@SetTitle@ 000000018000e5a0     service.obj
 0001:0000d5b0       ??_C@_08JNAOBKMI@GetTitle@ 000000018000e5b0     service.obj
 0001:0000d5c0       ??_C@_0BF@LIMPGNED@SubscribeChangeEvent@ 000000018000e5c0     service.obj
 0001:0000d5d8       ??_C@_09JFBCONJH@TabToReal@ 000000018000e5d8     service.obj
 0001:0000d5e8       ??_C@_08IBJJAHJG@UndoRedo@ 000000018000e5e8     service.obj
 0001:0000d5f8       ??_C@_07JMDLHPJF@SetMode@  000000018000e5f8     service.obj
 0001:0000d600       ??_C@_06PJECNADJ@Viewer@   000000018000e600     service.obj
 0001:0000d608       ??_C@_0P@OAACIGEB@BeginSelection@ 000000018000e608     service.obj
 0001:0000d618       ??_C@_0BB@PJGDGIKA@CheckPanelsExist@ 000000018000e618     service.obj
 0001:0000d630       ??_C@_0P@DFBDDHFA@ClearSelection@ 000000018000e630     service.obj
 0001:0000d640       ??_C@_0N@BHLDKHDJ@EndSelection@ 000000018000e640     service.obj
 0001:0000d650       ??_C@_0L@KOHCMOPM@GetCmdLine@ 000000018000e650     service.obj
 0001:0000d660       ??_C@_0O@NLDIMJEA@GetCmdLinePos@ 000000018000e660     service.obj
 0001:0000d670       ??_C@_0BE@CBPLLCEH@GetCmdLineSelection@ 000000018000e670     service.obj
 0001:0000d688       ??_C@_0P@CMFANDFM@GetColumnTypes@ 000000018000e688     service.obj
 0001:0000d698       ??_C@_0BA@DJGLDCBG@GetColumnWidths@ 000000018000e698     service.obj
 0001:0000d6a8       ??_C@_0BE@JPAIJBCI@GetCurrentPanelItem@ 000000018000e6a8     service.obj
 0001:0000d6c0       ??_C@_0BC@NGKPIKGL@GetPanelDirectory@ 000000018000e6c0     service.obj
 0001:0000d6d8       ??_C@_0P@GODLFFFJ@GetPanelFormat@ 000000018000e6d8     service.obj
 0001:0000d6e8       ??_C@_0BB@LCMBHPNI@GetPanelHostFile@ 000000018000e6e8     service.obj
 0001:0000d700       ??_C@_0N@HPIPGDFA@GetPanelInfo@ 000000018000e700     service.obj
 0001:0000d710       ??_C@_0N@HAFLAIHA@GetPanelItem@ 000000018000e710     service.obj
 0001:0000d720       ??_C@_0P@HCBKDPMP@GetPanelPrefix@ 000000018000e720     service.obj
 0001:0000d730       ??_C@_0BF@MEMFMMGB@GetSelectedPanelItem@ 000000018000e730     service.obj
 0001:0000d748       ??_C@_0O@HEGDGAJG@GetUserScreen@ 000000018000e748     service.obj
 0001:0000d758       ??_C@_0O@EHOCCHAL@InsertCmdLine@ 000000018000e758     service.obj
 0001:0000d768       ??_C@_0O@OMMHIHHH@IsActivePanel@ 000000018000e768     service.obj
 0001:0000d778       ??_C@_0M@LCEPDNPK@RedrawPanel@ 000000018000e778     service.obj
 0001:0000d788       ??_C@_0P@OPKJJMLB@SetActivePanel@ 000000018000e788     service.obj
 0001:0000d798       ??_C@_0L@LAFNHJLF@SetCmdLine@ 000000018000e798     service.obj
 0001:0000d7a8       ??_C@_0O@KECGHKDH@SetCmdLinePos@ 000000018000e7a8     service.obj
 0001:0000d7b8       ??_C@_0BE@IPNAPCDL@SetCmdLineSelection@ 000000018000e7b8     service.obj
 0001:0000d7d0       ??_C@_0BE@PAPEKLCP@SetDirectoriesFirst@ 000000018000e7d0     service.obj
 0001:0000d7e8       ??_C@_0BC@PDKEABHF@SetPanelDirectory@ 000000018000e7e8     service.obj
 0001:0000d800       ??_C@_0N@NMDFLOPL@SetSelection@ 000000018000e800     service.obj
 0001:0000d810       ??_C@_0M@CMMMGIDG@SetSortMode@ 000000018000e810     service.obj
 0001:0000d820       ??_C@_0N@HCHLALN@SetSortOrder@ 000000018000e820     service.obj
 0001:0000d830       ??_C@_0O@LHNNDOB@SetUserScreen@ 000000018000e830     service.obj
 0001:0000d840       ??_C@_0M@IENJPEBA@SetViewMode@ 000000018000e840     service.obj
 0001:0000d850       ??_C@_0M@EICBHAOA@UpdatePanel@ 000000018000e850     service.obj
 0001:0000d860       ??_C@_0BC@BIIKJLKB@PluginStartupInfo@ 000000018000e860     service.obj
 0001:0000d878       ??_C@_0L@PJAHNOGM@DialogInit@ 000000018000e878     service.obj
 0001:0000d888       ??_C@_09DBEDLMHB@DialogRun@ 000000018000e888     service.obj
 0001:0000d898       ??_C@_0L@DLFLHLOO@DialogFree@ 000000018000e898     service.obj
 0001:0000d8a8       ??_C@_0P@HLOFPDFP@SendDlgMessage@ 000000018000e8a8     service.obj
 0001:0000d8b8       ??_C@_0L@CKELNLCE@GetDlgItem@ 000000018000e8b8     service.obj
 0001:0000d8c8       ??_C@_0L@DEGEGMGN@SetDlgItem@ 000000018000e8c8     service.obj
 0001:0000d8d8       ??_C@_0BK@EBIPEKDH@SubscribeDialogDrawEvents@ 000000018000e8d8     service.obj
 0001:0000d8f8       ??_C@_0L@MCFABBED@GetDirList@ 000000018000e8f8     service.obj
 0001:0000d904       ??_C@_06KCCBBIBJ@GetMsg@   000000018000e904     service.obj
 0001:0000d910       ??_C@_0BB@HIDBFOJJ@GetPluginDirList@ 000000018000e910     service.obj
 0001:0000d924       ??_C@_04IFEHPILC@Menu@     000000018000e924     service.obj
 0001:0000d930       ??_C@_07BEIHKDLJ@Message@  000000018000e930     service.obj
 0001:0000d938       ??_C@_0O@CGLFPNOD@RestoreScreen@ 000000018000e938     service.obj
 0001:0000d948       ??_C@_0L@PGGGPLFK@SaveScreen@ 000000018000e948     service.obj
 0001:0000d958       ??_C@_08DAHHHDJC@ShowHelp@ 000000018000e958     service.obj
 0001:0000d968       ??_C@_08IAADAJIH@InputBox@ 000000018000e968     service.obj
 0001:0000d978       ??_C@_0L@HHLOIHOP@AdvControl@ 000000018000e978     service.obj
 0001:0000d988       ??_C@_0N@GHGEMEN@MacroLoadAll@ 000000018000e988     service.obj
 0001:0000d998       ??_C@_0N@NAGBAPAE@MacroSaveAll@ 000000018000e998     service.obj
 0001:0000d9a8       ??_C@_0O@KGHDMPAJ@MacroGetState@ 000000018000e9a8     service.obj
 0001:0000d9b8       ??_C@_0N@PNLHCOIE@MacroGetArea@ 000000018000e9b8     service.obj
 0001:0000d9c8       ??_C@_09KGKKBHMO@MacroPost@ 000000018000e9c8     service.obj
 0001:0000d9d8       ??_C@_0L@KBAKOGFP@MacroCheck@ 000000018000e9d8     service.obj
 0001:0000d9e8       ??_C@_08KAFLEHAN@MacroAdd@ 000000018000e9e8     service.obj
 0001:0000d9f8       ??_C@_0M@KFMHCNNB@MacroDelete@ 000000018000e9f8     service.obj
 0001:0000da08       ??_C@_0BC@MJDKBAPF@MacroGetLastError@ 000000018000ea08     service.obj
 0001:0000da20       ??_C@_0N@COEPENFH@MacroExecute@ 000000018000ea20     service.obj
 0001:0000da30       ??_C@_0BB@BICELPOF@CreateFileFilter@ 000000018000ea30     service.obj
 0001:0000da48       ??_C@_0L@CHJBHF@LoadPlugin@ 000000018000ea48     service.obj
 0001:0000da58       ??_C@_0N@DHIONCLI@UnloadPlugin@ 000000018000ea58     service.obj
 0001:0000da68       ??_C@_0BB@IJHIBGJA@ForcedLoadPlugin@ 000000018000ea68     service.obj
 0001:0000da80       ??_C@_0L@DACPHGGH@FindPlugin@ 000000018000ea80     service.obj
 0001:0000da90       ??_C@_0BF@KLOGLFMF@GetPluginInformation@ 000000018000ea90     service.obj
 0001:0000daa8       ??_C@_0L@JIDCIJHM@GetPlugins@ 000000018000eaa8     service.obj
 0001:0000dab8       ??_C@_0P@IKAEEPOB@IsPluginLoaded@ 000000018000eab8     service.obj
 0001:0000dac8       ??_C@_0P@HMKEDHIE@CreateSettings@ 000000018000eac8     service.obj
 0001:0000dad8       ??_C@_0N@GOMOBHDB@FreeSettings@ 000000018000ead8     service.obj
 0001:0000dae8       ??_C@_0M@IFKFGKML@ColorDialog@ 000000018000eae8     service.obj
 0001:0000daf8       ??_C@_0BA@EOCNNPOG@CopyToClipboard@ 000000018000eaf8     service.obj
 0001:0000db08       ??_C@_0BD@PLIHDKFC@PasteFromClipboard@ 000000018000eb08     service.obj
 0001:0000db20       ??_C@_0BC@FJDIKOMH@InputRecordToName@ 000000018000eb20     service.obj
 0001:0000db38       ??_C@_0BC@FFNOIDFI@NameToInputRecord@ 000000018000eb38     service.obj
 0001:0000db50       ??_C@_08HGLFNLMB@LStricmp@ 000000018000eb50     service.obj
 0001:0000db60       ??_C@_09GALOFBAC@LStrnicmp@ 000000018000eb60     service.obj
 0001:0000db70       ??_C@_0M@KPPMMAOL@ProcessName@ 000000018000eb70     service.obj
 0001:0000db80       ??_C@_0M@KFCNKLDK@GetPathRoot@ 000000018000eb80     service.obj
 0001:0000db90       ??_C@_0BE@EPGHGPJC@GetReparsePointInfo@ 000000018000eb90     service.obj
 0001:0000dba8       ??_C@_08DNJCLFF@LIsAlpha@  000000018000eba8     service.obj
 0001:0000dbb8       ??_C@_0M@LKJIEECA@LIsAlphanum@ 000000018000ebb8     service.obj
 0001:0000dbc8       ??_C@_08MAHKICD@LIsLower@  000000018000ebc8     service.obj
 0001:0000dbd8       ??_C@_08FHLJMDJK@LIsUpper@ 000000018000ebd8     service.obj
 0001:0000dbe8       ??_C@_09LPKAHGM@LLowerBuf@ 000000018000ebe8     service.obj
 0001:0000dbf8       ??_C@_09GLKFOOEP@LUpperBuf@ 000000018000ebf8     service.obj
 0001:0000dc04       ??_C@_06ILCHIEBO@MkTemp@   000000018000ec04     service.obj
 0001:0000dc0c       ??_C@_06DKBBJCCG@MkLink@   000000018000ec0c     service.obj
 0001:0000dc18       ??_C@_0N@CCDDAJK@TruncPathStr@ 000000018000ec18     service.obj
 0001:0000dc28       ??_C@_08BNEIIKEJ@TruncStr@ 000000018000ec28     service.obj
 0001:0000dc38       ??_C@_0BA@CLEHBIPM@RecursiveSearch@ 000000018000ec38     service.obj
 0001:0000dc48       ??_C@_0M@HKHGOOHG@ConvertPath@ 000000018000ec48     service.obj
 0001:0000dc54       ??_C@_04OCDKHGII@XLat@     000000018000ec54     service.obj
 0001:0000dc60       ??_C@_0P@BGLLKGOI@FormatFileSize@ 000000018000ec60     service.obj
 0001:0000dc70       ??_C@_08KJBLDCDF@FarClock@ 000000018000ec70     service.obj
 0001:0000dc80       ??_C@_0BD@ELMHPHAC@CPluginStartupInfo@ 000000018000ec80     service.obj
 0001:0000dc98       ??_C@_0BE@DJLJEKBK@GetCurrentDirectory@ 000000018000ec98     service.obj
 0001:0000dcb0       ??_C@_0N@MOMBJEKA@GetFileOwner@ 000000018000ecb0     service.obj
 0001:0000dcc0       ??_C@_0BB@JBNBALEM@GetNumberOfLinks@ 000000018000ecc0     service.obj
 0001:0000dcd8       ??_C@_0O@BJEAJNBH@MakeMenuItems@ 000000018000ecd8     service.obj
 0001:0000dce8       ??_C@_0BB@HLFLDCHO@RunDefaultScript@ 000000018000ece8     service.obj
 0001:0000dcfc       ??_C@_04JLAJABDJ@Show@     000000018000ecfc     service.obj
 0001:0000dd04       ??_C@_05NHFJDMOA@Timer@    000000018000ed04     service.obj
 0001:0000dd10       ??_C@_0BD@KCMHFGFP@FileTimeResolution@ 000000018000ed10     service.obj
 0001:0000dd24       ??_C@_02KFNNKBCK@io@       000000018000ed24     service.obj
 0001:0000dd28       ??_C@_02EHCHIAMF@os@       000000018000ed28     service.obj
 0001:0000dd2c       ??_C@_04CFDJAKFL@math@     000000018000ed2c     service.obj
 0001:0000dd38       ??_C@_07GAJMMAJO@unicode@  000000018000ed38     service.obj
 0001:0000dd40       ??_C@_04LHHHFLPP@utf8@     000000018000ed40     service.obj
 0001:0000dd48       ??_C@_03JECLAOEA@win@      000000018000ed48     service.obj
 0001:0000dd50       ??_C@_09GJGOMOL@lua51?4dll@ 000000018000ed50     service.obj
 0001:0000dd60       ??_C@_0M@PLOBHAKE@luaopen_bit@ 000000018000ed60     service.obj
 0001:0000dd70       ??_C@_0M@IALDMMNC@luaopen_ffi@ 000000018000ed70     service.obj
 0001:0000dd80       ??_C@_0M@DOFFFIEL@luaopen_jit@ 000000018000ed80     service.obj
 0001:0000dd90       ??_C@_0BE@OEPKKAAB@integer?5or?5userdata@ 000000018000ed90     service.obj
 0001:0000dda8       ??_C@_0BD@PNJHLBDA@invalid?5flag?3?5?$CC?$CFs?$CC@ 000000018000eda8     service.obj
 0001:0000ddc0       ??_C@_0N@JJLBBDOC@invalid?5flag@ 000000018000edc0     service.obj
 0001:0000ddd0       ??_C@_0BJ@MIKGPOKL@invalid?5flag?5combination@ 000000018000edd0     service.obj
 0001:0000ddf0       ??_C@_0P@EANMLDOP@MousePositionX@ 000000018000edf0     service.obj
 0001:0000de00       ??_C@_0P@FJMHICKO@MousePositionY@ 000000018000ee00     service.obj
 0001:0000de10       ??_C@_0M@BJAICPIE@ButtonState@ 000000018000ee10     service.obj
 0001:0000de20       ??_C@_0L@EMFBJIPA@EventFlags@ 000000018000ee20     service.obj
 0001:0000de30       ??_C@_07EEJLMCNH@CurLine@  000000018000ee30     service.obj
 0001:0000de38       ??_C@_06EDBJMJDC@CurPos@   000000018000ee38     service.obj
 0001:0000de40       ??_C@_09EGONKHKB@CurTabPos@ 000000018000ee40     service.obj
 0001:0000de50       ??_C@_0O@OKGGHEJK@TopScreenLine@ 000000018000ee50     service.obj
 0001:0000de60       ??_C@_07GDAKJHLE@LeftPos@  000000018000ee60     service.obj
 0001:0000de68       ??_C@_08LLJICOLD@Overtype@ 000000018000ee68     service.obj
 0001:0000de78       ??_C@_0L@GEIEADPN@ModuleName@ 000000018000ee78     service.obj
 0001:0000de88       ??_C@_09HOIHBHIM@ModuleDir@ 000000018000ee88     service.obj
 0001:0000de98       ??_C@_0L@JLHCLFBG@PluginGuid@ 000000018000ee98     service.obj
 0001:0000dea8       ??_C@_08GGMFPBHM@EditorID@ 000000018000eea8     service.obj
 0001:0000deb8       ??_C@_0M@CPDBGLHN@WindowSizeX@ 000000018000eeb8     service.obj
 0001:0000dec8       ??_C@_0M@DGCKFKDM@WindowSizeY@ 000000018000eec8     service.obj
 0001:0000ded8       ??_C@_0L@PMKENHMA@TotalLines@ 000000018000eed8     service.obj
 0001:0000dee8       ??_C@_09HKBEFIPN@BlockType@ 000000018000eee8     service.obj
 0001:0000def8       ??_C@_0P@GAEEHNHE@BlockStartLine@ 000000018000eef8     service.obj
 0001:0000df08       ??_C@_07KHIHFBFN@Options@  000000018000ef08     service.obj
 0001:0000df10       ??_C@_07FLDNELFM@TabSize@  000000018000ef10     service.obj
 0001:0000df18       ??_C@_0O@EBLDFOPH@BookmarkCount@ 000000018000ef18     service.obj
 0001:0000df28       ??_C@_0BF@ODFKBFAK@SessionBookmarkCount@ 000000018000ef28     service.obj
 0001:0000df40       ??_C@_08CPAOHJDL@CurState@ 000000018000ef40     service.obj
 0001:0000df50       ??_C@_0N@DAJMJAE@StringLength@ 000000018000ef50     service.obj
 0001:0000df60       ??_C@_08JPMALCFA@SelStart@ 000000018000ef60     service.obj
 0001:0000df6c       ??_C@_06JLEHDHII@SelEnd@   000000018000ef6c     service.obj
 0001:0000df78       ??_C@_0L@IFNFGDGN@StringText@ 000000018000ef78     service.obj
 0001:0000df88       ??_C@_09IBGOAAEM@StringEOL@ 000000018000ef88     service.obj
 0001:0000df94       ??_C@_01LOCGONAA@?$AA@     000000018000ef94     service.obj
 0001:0000df98       ??_C@_06MFLCIING@redraw@   000000018000ef98     service.obj
 0001:0000dfa0       ??_C@_07HICINA@restore@    000000018000efa0     service.obj
 0001:0000dfa8       ??_C@_0CG@LAKEGANL@must?5be?5?8redraw?8?0?5?8restore?8?0?5or@ 000000018000efa8     service.obj
 0001:0000dfd0       ??_C@_04LIDDHMOL@Line@     000000018000efd0     service.obj
 0001:0000dfd8       ??_C@_06OIIFPIKD@Cursor@   000000018000efd8     service.obj
 0001:0000dfe0       ??_C@_0L@GDDEHGKI@ScreenLine@ 000000018000efe0     service.obj
 0001:0000dff0       ??_C@_0O@CIAFMMMB@BlockStartPos@ 000000018000eff0     service.obj
 0001:0000e000       ??_C@_0L@EKLJJHPF@BlockWidth@ 000000018000f000     service.obj
 0001:0000e010       ??_C@_0M@NKKGBDGK@BlockHeight@ 000000018000f010     service.obj
 0001:0000e020       ??_C@_09JFPCGCOC@StartLine@ 000000018000f020     service.obj
 0001:0000e030       ??_C@_08JBNOANJG@StartPos@ 000000018000f030     service.obj
 0001:0000e040       ??_C@_07DCKCOCOC@EndLine@  000000018000f040     service.obj
 0001:0000e048       ??_C@_06KGHIGMHC@EndPos@   000000018000f048     service.obj
 0001:0000e050       ??_C@_0BA@HNIJJEO@ForegroundColor@ 000000018000f050     service.obj
 0001:0000e060       ??_C@_0BA@DPMBBMBG@BackgroundColor@ 000000018000f060     service.obj
 0001:0000e070       ??_C@_0O@NHKEGDJF@GUID?5required@ 000000018000f070     service.obj
 0001:0000e080       ??_C@_0BJ@BMOGHFAN@table?5or?5number?5expected@ 000000018000f080     service.obj
 0001:0000e0a0       ??_C@_08KGEIBGG@Priority@  000000018000f0a0     service.obj
 0001:0000e0ac       ??_C@_05PDOBBJNA@Color@    000000018000f0ac     service.obj
 0001:0000e0b8       ??_C@_09KDLBEGCN@EventType@ 000000018000f0b8     service.obj
 0001:0000e0c8       ??_C@_07HPHPOAEG@KeyDown@  000000018000f0c8     service.obj
 0001:0000e0d0       ??_C@_0M@FGGHEADP@RepeatCount@ 000000018000f0d0     service.obj
 0001:0000e0e0       ??_C@_0BA@KCCLHPM@VirtualScanCode@ 000000018000f0e0     service.obj
 0001:0000e0f0       ??_C@_0M@PBJKDIHH@UnicodeChar@ 000000018000f0f0     service.obj
 0001:0000e0fc       ??_C@_05GIPJKPFG@SizeX@    000000018000f0fc     service.obj
 0001:0000e104       ??_C@_05HBOCJOBH@SizeY@    000000018000f104     service.obj
 0001:0000e110       ??_C@_09GEJJJAHL@CommandId@ 000000018000f110     service.obj
 0001:0000e120       ??_C@_08GPNNBNIL@SetFocus@ 000000018000f120     service.obj
 0001:0000e130       ??_C@_0M@BEDENHPD@invalid?5key@ 000000018000f130     service.obj
 0001:0000e140       ??_C@_19IBCFILMC@?$AAM?$AAe?$AAn?$AAu@ 000000018000f140     service.obj
 0001:0000e150       ??_C@_0BN@JBAMKCCJ@must?5be?5table?0?5string?5or?5nil@ 000000018000f150     service.obj
 0001:0000e170       ??_C@_09FDAFFNEA@MaxHeight@ 000000018000f170     service.obj
 0001:0000e17c       ??_C@_06DDHCBBGN@Bottom@   000000018000f17c     service.obj
 0001:0000e188       ??_C@_09CFELDMD@HelpTopic@ 000000018000f188     service.obj
 0001:0000e198       ??_C@_0M@GGMLPAIK@SelectIndex@ 000000018000f198     service.obj
 0001:0000e1a4       ??_C@_02HOGEDOAB@Id@       000000018000f1a4     service.obj
 0001:0000e1a8       ??_C@_07FJOBMBFC@checked@  000000018000f1a8     service.obj
 0001:0000e1b0       ??_C@_09MOAJOJKN@separator@ 000000018000f1b0     service.obj
 0001:0000e1c0       ??_C@_07DBNODEFN@disable@  000000018000f1c0     service.obj
 0001:0000e1c8       ??_C@_06JHIAOIKD@grayed@   000000018000f1c8     service.obj
 0001:0000e1d0       ??_C@_06JIKFICKK@hidden@   000000018000f1d0     service.obj
 0001:0000e1d8       ??_C@_08CJLOJPNI@selected@ 000000018000f1d8     service.obj
 0001:0000e1e8       ??_C@_08MMCKBNNI@AccelKey@ 000000018000f1e8     service.obj
 0001:0000e1f8       ??_C@_08PNHLLJE@BreakKey@  000000018000f1f8     service.obj
 0001:0000e204       ??_C@_15FMBEJGOH@?$AAO?$AAk@ 000000018000f204     service.obj
 0001:0000e210       ??_C@_1BC@IBCAPFAE@?$AAO?$AAk?$AAC?$AAa?$AAn?$AAc?$AAe?$AAl@ 000000018000f210     service.obj
 0001:0000e228       ??_C@_1CC@HODOHOHB@?$AAA?$AAb?$AAo?$AAr?$AAt?$AAR?$AAe?$AAt?$AAr?$AAy?$AAI?$AAg?$AAn?$AAo?$AAr@ 000000018000f228     service.obj
 0001:0000e250       ??_C@_1M@GGPOIMAD@?$AAY?$AAe?$AAs?$AAN?$AAo@ 000000018000f250     service.obj
 0001:0000e260       ??_C@_1BI@BNDFIGCI@?$AAY?$AAe?$AAs?$AAN?$AAo?$AAC?$AAa?$AAn?$AAc?$AAe?$AAl@ 000000018000f260     service.obj
 0001:0000e278       ??_C@_1BI@KMMIHPHF@?$AAR?$AAe?$AAt?$AAr?$AAy?$AAC?$AAa?$AAn?$AAc?$AAe?$AAl@ 000000018000f278     service.obj
 0001:0000e290       ??_C@_1DG@LMKDDADI@?$AA?$DM?$AAn?$AAo?$AAn?$AA?9?$AAs?$AAt?$AAr?$AAi?$AAn?$AAg?$AA?5?$AAe?$AAr?$AAr@ 000000018000f290     service.obj
 0001:0000e2c8       ??_C@_15IEGBJKPD@?$AA?3?$AA?6@ 000000018000f2c8     service.obj
 0001:0000e2d0       ??_C@_19FFLPMPBO@?$AA?6?$AA?5?$AA?5?$AA?5@ 000000018000f2d0     service.obj
 0001:0000e2dc       ??_C@_15JCKODCLA@?$AA?6?$AA?7@ 000000018000f2dc     service.obj
 0001:0000e2e8       ??_C@_1M@ILHOPKA@?$AAE?$AAr?$AAr?$AAo?$AAr@ 000000018000f2e8     service.obj
 0001:0000e2f8       ??_C@_08FNIIFOJC@tostring@ 000000018000f2f8     service.obj
 0001:0000e308       ??_C@_0BJ@JOELOGM@cannot?5convert?5to?5string@ 000000018000f308     service.obj
 0001:0000e328       ??_C@_1BA@HHOMBECE@?$AAM?$AAe?$AAs?$AAs?$AAa?$AAg?$AAe@ 000000018000f328     service.obj
 0001:0000e338       ??_C@_17PAGBAIDI@?$AA?$DL?$AAO?$AAK@ 000000018000f338     service.obj
 0001:0000e340       ??_C@_09ENKGJCEC@OwnerGuid@ 000000018000f340     service.obj
 0001:0000e350       ??_C@_0N@CCPLCIHE@PluginHandle@ 000000018000f350     service.obj
 0001:0000e360       ??_C@_0N@HEHBMBNM@PluginObject@ 000000018000f360     service.obj
 0001:0000e370       ??_C@_09BKHPOLGD@PanelType@ 000000018000f370     service.obj
 0001:0000e37c       ??_C@_04GOOOJOPP@left@     000000018000f37c     service.obj
 0001:0000e384       ??_C@_03FGFCOCMD@top@      000000018000f384     service.obj
 0001:0000e388       ??_C@_05DHJDAOHK@right@    000000018000f388     service.obj
 0001:0000e390       ??_C@_06PMMPCIPB@bottom@   000000018000f390     service.obj
 0001:0000e398       ??_C@_09MCEJMINN@PanelRect@ 000000018000f398     service.obj
 0001:0000e3a8       ??_C@_0M@DDGFKGKJ@ItemsNumber@ 000000018000f3a8     service.obj
 0001:0000e3b8       ??_C@_0BE@EOBAHHNK@SelectedItemsNumber@ 000000018000f3b8     service.obj
 0001:0000e3d0       ??_C@_0M@JMILNLLF@CurrentItem@ 000000018000f3d0     service.obj
 0001:0000e3e0       ??_C@_0N@CDHIFJIH@TopPanelItem@ 000000018000f3e0     service.obj
 0001:0000e3f0       ??_C@_08IMMBLBLF@ViewMode@ 000000018000f3f0     service.obj
 0001:0000e400       ??_C@_08CENECNJD@SortMode@ 000000018000f400     service.obj
 0001:0000e40c       ??_C@_04FABLJDN@Name@      000000018000f40c     service.obj
 0001:0000e414       ??_C@_05LOJBNELM@Param@    000000018000f414     service.obj
 0001:0000e41c       ??_C@_04PBAHLACE@File@     000000018000f41c     service.obj
 0001:0000e428       ??_C@_08HGEAFCFN@PluginId@ 000000018000f428     service.obj
 0001:0000e438       ??_C@_0BA@MLHECKCE@table?5or?5string@ 000000018000f438     service.obj
 0001:0000e448       ??_C@_0BD@CKJHMJBG@non?9positive?5index@ 000000018000f448     service.obj
 0001:0000e460       ??_C@_0BA@GNKNKKDM@number?5or?5table@ 000000018000f460     service.obj
 0001:0000e470       ??_C@_0CI@DDAJHJKO@?$CFs?5?9?5unsupported?5type?5in?5dialog@ 000000018000f470     service.obj
 0001:0000e498       ??_C@_0CD@JIANOKII@unsupported?5flag?5in?5dialog?5item@ 000000018000f498     service.obj
 0001:0000e4c0       ??_C@_0CB@EOGFCCCC@value?5at?5index?5?$CFd?5is?5not?5a?5tabl@ 000000018000f4c0     service.obj
 0001:0000e4e8       ??_C@_0O@FEBHKEHB@closed?5dialog@ 000000018000f4e8     service.obj
 0001:0000e4f8       ??_C@_0BK@NEMPGLFN@operation?5not?5implemented@ 000000018000f4f8     service.obj
 0001:0000e514       ??_C@_04KPCPLBPL@Left@     000000018000f514     service.obj
 0001:0000e51c       ??_C@_03PGGAENPN@Top@      000000018000f51c     service.obj
 0001:0000e520       ??_C@_05DADPALEM@Right@    000000018000f520     service.obj
 0001:0000e528       ??_C@_0CK@JHNDGJBB@element?5?$CD?$CFd?5in?5argument?5?$CD4?5is?5n@ 000000018000f528     service.obj
 0001:0000e558       ??_C@_0L@CECHCPAP@StartIndex@ 000000018000f558     service.obj
 0001:0000e564       ??_C@_05IJGIMMHE@Count@    000000018000f564     service.obj
 0001:0000e570       ??_C@_07NOCIGAPP@Pattern@  000000018000f570     service.obj
 0001:0000e578       ??_C@_09IMOCKOO@SelectPos@ 000000018000f578     service.obj
 0001:0000e584       ??_C@_06DJONBJOP@TopPos@   000000018000f584     service.obj
 0001:0000e590       ??_C@_09OGCBKCAK@MaxLength@ 000000018000f590     service.obj
 0001:0000e59c       ??_C@_05FNNGFGLF@Index@    000000018000f59c     service.obj
 0001:0000e5a8       ??_C@_07GHGHLGFI@GetType@  000000018000f5a8     service.obj
 0001:0000e5b0       ??_C@_07MMLMCDAI@ValType@  000000018000f5b0     service.obj
 0001:0000e5b8       ??_C@_05LPIJGKJ@Value@     000000018000f5b8     service.obj
 0001:0000e5c0       ??_C@_0L@LPFMIAHH@helpstring@ 000000018000f5c0     service.obj
 0001:0000e5d0       ??_C@_0P@NABDHFON@getvaluestring@ 000000018000f5d0     service.obj
 0001:0000e5e0       ??_C@_0BJ@IINAPFDG@Items?$FL?$CFd?$FN?5is?5not?5a?5table@ 000000018000f5e0     service.obj
 0001:0000e600       ??_C@_0CC@GBOJFNBI@error?5occured?5in?5dialog?5procedu@ 000000018000f600     service.obj
 0001:0000e628       ??_C@_0M@EHMONPJO@?$CFs?5?$CIclosed?$CJ@ 000000018000f628     service.obj
 0001:0000e638       ??_C@_08GDAJJKGC@ViewerID@ 000000018000f638     service.obj
 0001:0000e648       ??_C@_07MJHBHMFM@FilePos@  000000018000f648     service.obj
 0001:0000e650       ??_C@_07FBAHDBGN@CurMode@  000000018000f650     service.obj
 0001:0000e658       ??_C@_06IMBBKDFH@iParam@   000000018000f658     service.obj
 0001:0000e660       ??_C@_1BE@CGKCNEEP@?$AAI?$AAn?$AAp?$AAu?$AAt?$AA?5?$AAB?$AAo?$AAx@ 000000018000f660     service.obj
 0001:0000e678       ??_C@_1CA@PCDNIBFH@?$AAE?$AAn?$AAt?$AAe?$AAr?$AA?5?$AAt?$AAh?$AAe?$AA?5?$AAt?$AAe?$AAx?$AAt?$AA?3@ 000000018000f678     service.obj
 0001:0000e698       ??_C@_0BG@GAFLOAPP@command?5not?5supported@ 000000018000f698     service.obj
 0001:0000e6b0       ??_C@_09MIJAKHKB@Completed@ 000000018000f6b0     service.obj
 0001:0000e6bc       ??_C@_05KGEAEGFG@Total@    000000018000f6bc     service.obj
 0001:0000e6c8       ??_C@_0P@DJOANNIK@?$CFd?4?$CFd?4?$CFd?4?$CFd?4?$CFd@ 000000018000f6c8     service.obj
 0001:0000e6d8       ??_C@_03FCCPIJGJ@Pos@      000000018000f6d8     service.obj
 0001:0000e6e0       ??_C@_08NNKIOIN@TypeName@  000000018000f6e0     service.obj
 0001:0000e6f0       ??_C@_07ONPPLIAF@ErrCode@  000000018000f6f0     service.obj
 0001:0000e6f8       ??_C@_07LJDOKIBM@ErrPosX@  000000018000f6f8     service.obj
 0001:0000e700       ??_C@_07KACFJJFN@ErrPosY@  000000018000f700     service.obj
 0001:0000e708       ??_C@_06HBEFEBCM@ErrSrc@   000000018000f708     service.obj
 0001:0000e710       ??_C@_06LDIMCHFC@?$CF?$CKs?$CFs?5@ 000000018000f710     service.obj
 0001:0000e718       ??_C@_09HNJDNMKK@?$CF?$CF?$CFdd?$CF?$CFs?5@ 000000018000f718     service.obj
 0001:0000e728       ??_C@_0CC@JIGPFMKG@global?5?$GAtostring?8?5is?5not?5functi@ 000000018000f728     service.obj
 0001:0000e750       ??_C@_0CH@OINAPBOJ@tostring?$CI?$CJ?5returned?5a?5non?9strin@ 000000018000f750     service.obj
 0001:0000e778       ??_C@_04CIMGMMMG@text@     000000018000f778     service.obj
 0001:0000e780       ??_C@_03CAOIPBNL@arg@      000000018000f780     service.obj
 0001:0000e790       ??_C@_0ME@JDKAEDFJ@local?5items?0n?$DN?4?4?4?6local?5bottom?$DN@ 000000018000f790     service.obj
 0001:0000e858       ??_C@_0CG@FGNNCNLL@attempt?5to?5access?5invalid?5file?5@ 000000018000f858     service.obj
 0001:0000e880       ??_C@_07BJOIOONN@Strings@  000000018000f880     service.obj
 0001:0000e888       ??_C@_08FGAFMHLF@DiskMenu@ 000000018000f888     service.obj
 0001:0000e898       ??_C@_0L@NHENMPLN@PluginMenu@ 000000018000f898     service.obj
 0001:0000e8a8       ??_C@_0N@IEACHFBM@PluginConfig@ 000000018000f8a8     service.obj
 0001:0000e8b8       ??_C@_05GCJGCMFJ@PInfo@    000000018000f8b8     service.obj
 0001:0000e8c0       ??_C@_05HMEFBOHK@GInfo@    000000018000f8c0     service.obj
 0001:0000e8c8       ??_C@_0N@GAMEMCEE@invalid?5GUID@ 000000018000f8c8     service.obj
 0001:0000e8d8       ??_C@_0BP@NJEEOHDB@attempt?5to?5access?5closed?5timer@ 000000018000f8d8     service.obj
 0001:0000e8f8       ??_C@_05LGELBCGM@Close@    000000018000f8f8     service.obj
 0001:0000e900       ??_C@_07DOAOMMKG@Enabled@  000000018000f900     service.obj
 0001:0000e908       ??_C@_08KDKDEPAG@Interval@ 000000018000f908     service.obj
 0001:0000e918       ??_C@_07CIINKFND@OnTimer@  000000018000f918     service.obj
 0001:0000e920       ??_C@_06EFCDMIMC@Closed@   000000018000f920     service.obj
 0001:0000e928       ??_C@_0CE@LHJCBGGH@attempt?5to?5call?5non?9existent?5me@ 000000018000f928     service.obj
 0001:0000e950       ??_C@_0BO@PNFLEJKN@attempt?5to?5access?5a?5closed?5?$CFs@ 000000018000f950     service.obj
 0001:0000e970       ??_C@_04OKOFBOPB@Time@     000000018000f970     service.obj
 0001:0000e978       ??_C@_04LADJNOK@Lock@      000000018000f978     service.obj
 0001:0000e980       ??_C@_0N@ECMJOJJG@MacroCallFar@ 000000018000f980     service.obj
 0001:0000e990       ??_C@_0BC@JJHHFNMP@FarMacroCallToLua@ 000000018000f990     service.obj
 0001:0000e9a4       ??_C@_06GIFLLBB@editor@    000000018000f9a4     service.obj
 0001:0000e9ac       ??_C@_06DGPPOJKF@viewer@   000000018000f9ac     service.obj
 0001:0000e9b4       ??_C@_01DICPFPGM@k@        000000018000f9b4     service.obj
 0001:0000e9b8       ??_C@_06BPGFKLEK@__mode@   000000018000f9b8     service.obj
 0001:0000e9c0       ??_C@_1CC@OPOAGCKN@?$AA?2?$AAl?$AAu?$AAa?$AAf?$AAa?$AAr?$AA_?$AAi?$AAn?$AAi?$AAt?$AA?4?$AAl?$AAu@ 000000018000f9c0     service.obj
 0001:0000e9e8       ??_C@_1BG@BDOBMIBP@?$AAF?$AAA?$AAR?$AAP?$AAR?$AAO?$AAF?$AAI?$AAL?$AAE@ 000000018000f9e8     service.obj
 0001:0000ea00       ??_C@_05NDNJFBEF@cfind@    000000018000fa00     service.obj
 0001:0000ea08       ??_C@_03EDMBFDDG@bit@      000000018000fa08     service.obj
 0001:0000ea0c       ??_C@_03IGHFHLNJ@jit@      000000018000fa0c     service.obj
 0001:0000ea10       ??_C@_08LBNNGFKE@_PRELOAD@ 000000018000fa10     service.obj
 0001:0000ea1c       ??_C@_03DIJDOPEA@ffi@      000000018000fa1c     service.obj
 0001:0000ea20       ??_C@_06ONNDGCDK@dofile@   000000018000fa20     service.obj
 0001:0000ea28       ??_C@_08BNNFLGCJ@loadfile@ 000000018000fa28     service.obj
 0001:0000ea34       ??_C@_03OFAPEBGM@?$CFs?6@  000000018000fa34     service.obj
 0001:0000ea38       __real@3ff0000000000000    000000018000fa38     service.obj
 0001:0000ea40       __real@4059000000000000    000000018000fa40     service.obj
 0001:0000ea48       __real@41e0000000000000    000000018000fa48     service.obj
 0001:0000ea50       __real@43f0000000000000    000000018000fa50     service.obj
 0001:0000ea60       __xmm@ffffffffffffffffffffffffffffffff 000000018000fa60     service.obj
 0001:0000eac0       ??_C@_04GGLOKIEE@dump@     000000018000fac0     slnunico.obj
 0001:0000eac8       ??_C@_06DLEPGFEF@format@   000000018000fac8     slnunico.obj
 0001:0000ead0       ??_C@_03HOKODIMJ@rep@      000000018000fad0     slnunico.obj
 0001:0000ead8       ??_C@_09GCBMKPBD@utf8valid@ 000000018000fad8     slnunico.obj
 0001:0000eae8       ??_C@_0BO@BNLBHKJN@unable?5to?5dump?5given?5function@ 000000018000fae8     slnunico.obj
 0001:0000eb08       ??_C@_02HIBBOKEN@?2r@      000000018000fb08     slnunico.obj
 0001:0000eb0c       ??_C@_04MPDIABOK@?2000@    000000018000fb0c     slnunico.obj
 0001:0000eb14       ??_C@_05GGBDHNF@?9?$CL?5?$CD0@ 000000018000fb14     slnunico.obj
 0001:0000eb20       ??_C@_0CA@COOMGCAO@invalid?5format?5?$CIrepeated?5flags?$CJ@ 000000018000fb20     slnunico.obj
 0001:0000eb40       ??_C@_0CN@KALFEKPN@invalid?5format?5?$CIwidth?5or?5precis@ 000000018000fb40     slnunico.obj
 0001:0000eb70       ??_C@_0CC@KIPBEOBI@invalid?5option?5?8?$CF?$CF?$CFc?8?5to?5?8forma@ 000000018000fb70     slnunico.obj
 0001:0000eb98       ??_C@_0BP@FKCDAMA@number?1string?5expected?0?5got?5?$CFs@ 000000018000fb98     lutf8lib.obj
 0001:0000ebb8       ??_C@_0BG@DFAIEAEC@string?5slice?5too?5long@ 000000018000fbb8     lutf8lib.obj
 0001:0000ebd0       ??_C@_0N@FCPHIMMG@out?5of?5range@ 000000018000fbd0     lutf8lib.obj
 0001:0000ebe0       ??_C@_0BE@MHMGJPCL@invalid?5escape?5?8?$CFc?8@ 000000018000fbe0     lutf8lib.obj
 0001:0000ebf8       ??_C@_0BI@HGMIJEDD@invalid?5escape?5sequence@ 000000018000fbf8     lutf8lib.obj
 0001:0000ec10       ??_C@_0BL@JNACDPC@invalid?5capture?5index?5?$CF?$CF?$CFd@ 000000018000fc10     lutf8lib.obj
 0001:0000ec30       ??_C@_0BI@ECNPHIBF@invalid?5pattern?5capture@ 000000018000fc30     lutf8lib.obj
 0001:0000ec48       ??_C@_0CD@PLJBIEHA@malformed?5pattern?5?$CIends?5with?5?8?$CF@ 000000018000fc48     lutf8lib.obj
 0001:0000ec70       ??_C@_0CA@CFGACOGB@malformed?5pattern?5?$CImissing?5?8?$FN?8?$CJ@ 000000018000fc70     lutf8lib.obj
 0001:0000ec90       ??_C@_0CP@FCNHBCLO@malformed?5pattern?5?$CImissing?5argu@ 000000018000fc90     lutf8lib.obj
 0001:0000ecc0       ??_C@_0BC@IMEAEJPD@too?5many?5captures@ 000000018000fcc0     lutf8lib.obj
 0001:0000ecd8       ??_C@_0BE@LPFFPFJG@pattern?5too?5complex@ 000000018000fcd8     lutf8lib.obj
 0001:0000ecf0       ??_C@_0CD@LOJJMDBH@missing?5?8?$FL?8?5after?5?8?$CF?$CFf?8?5in?5patt@ 000000018000fcf0     lutf8lib.obj
 0001:0000ed18       ??_C@_0BG@LEHNKOGD@invalid?5capture?5index@ 000000018000fd18     lutf8lib.obj
 0001:0000ed30       ??_C@_0BD@BFKNEALP@unfinished?5capture@ 000000018000fd30     lutf8lib.obj
 0001:0000ed48       ??_C@_0L@NLFJOONJ@?$FO$?$CK?$CL?$DP?4?$CI?$FL?$CF?9@ 000000018000fd48     lutf8lib.obj
 0001:0000ed58       ??_C@_0CK@KLCOLAN@invalid?5use?5of?5?8?$CFc?8?5in?5replacem@ 000000018000fd58     lutf8lib.obj
 0001:0000ed88       ??_C@_0CB@LPDIHGGA@invalid?5replacement?5value?5?$CIa?5?$CFs@ 000000018000fd88     lutf8lib.obj
 0001:0000edb0       ??_C@_0BP@PPPOBACA@string?1function?1table?5expected@ 000000018000fdb0     lutf8lib.obj
 0001:0000edd0       ??_C@_06KLHHMIGM@offset@   000000018000fdd0     lutf8lib.obj
 0001:0000edd8       ??_C@_05CFHFIAJO@codes@    000000018000fdd8     lutf8lib.obj
 0001:0000ede0       ??_C@_09HHCEKEIA@codepoint@ 000000018000fde0     lutf8lib.obj
 0001:0000edec       ??_C@_03BKCJCHLK@len@      000000018000fdec     lutf8lib.obj
 0001:0000edf0       ??_C@_07KOIEOCCE@reverse@  000000018000fdf0     lutf8lib.obj
 0001:0000edf8       ??_C@_05IPJEPLHL@lower@    000000018000fdf8     lutf8lib.obj
 0001:0000ee00       ??_C@_05NECKJAMC@upper@    000000018000fe00     lutf8lib.obj
 0001:0000ee08       ??_C@_05PHLGJONK@title@    000000018000fe08     lutf8lib.obj
 0001:0000ee10       ??_C@_04MLGPBLN@fold@      000000018000fe10     lutf8lib.obj
 0001:0000ee18       ??_C@_04IHGKJMLH@byte@     000000018000fe18     lutf8lib.obj
 0001:0000ee20       ??_C@_04ENMBGAPA@char@     000000018000fe20     lutf8lib.obj
 0001:0000ee28       ??_C@_06CHNIFGOF@escape@   000000018000fe28     lutf8lib.obj
 0001:0000ee30       ??_C@_06OAOPNKHP@insert@   000000018000fe30     lutf8lib.obj
 0001:0000ee38       ??_C@_06LEMKAMD@remove@    000000018000fe38     lutf8lib.obj
 0001:0000ee40       ??_C@_07BAPMOMKI@charpos@  000000018000fe40     lutf8lib.obj
 0001:0000ee48       ??_C@_04CJGEDOF@next@      000000018000fe48     lutf8lib.obj
 0001:0000ee50       ??_C@_05IGKADHGO@width@    000000018000fe50     lutf8lib.obj
 0001:0000ee58       ??_C@_0L@OLBIGGEG@widthindex@ 000000018000fe58     lutf8lib.obj
 0001:0000ee68       ??_C@_08GEDFKPFE@ncasecmp@ 000000018000fe68     lutf8lib.obj
 0001:0000ee78       ??_C@_0P@NELPIPKN@?$FL?$AA?9?$HP?B?9?t?$FN?$FL?$IA?9?$LP?$FN?$CK@ 000000018000fe78     lutf8lib.obj
 0001:0000ee88       ??_C@_0M@GMACFGDH@charpattern@ 000000018000fe88     lutf8lib.obj
 0001:0000f080       ??_C@_05DFJCHPDH@input@    0000000180010080     uliolib51.obj
 0001:0000f088       ??_C@_06DKIGHACF@output@   0000000180010088     uliolib51.obj
 0001:0000f090       ??_C@_03KCHOJKKI@set@      0000000180010090     uliolib51.obj
 0001:0000f094       ??_C@_03LIBLMJMB@cur@      0000000180010094     uliolib51.obj
 0001:0000f098       ??_C@_03JBJLGPFL@end@      0000000180010098     uliolib51.obj
 0001:0000f09c       ??_C@_02KAJCLHKP@no@       000000018001009c     uliolib51.obj
 0001:0000f0a0       ??_C@_04PLMLMMEO@full@     00000001800100a0     uliolib51.obj
 0001:0000f0a8       ??_C@_04HJPCFDOP@line@     00000001800100a8     uliolib51.obj
 0001:0000f0b0       ??_C@_05LBOHBHFK@close@    00000001800100b0     uliolib51.obj
 0001:0000f0b8       ??_C@_05GLCAEPFP@flush@    00000001800100b8     uliolib51.obj
 0001:0000f0c0       ??_C@_05DENOCHIP@lines@    00000001800100c0     uliolib51.obj
 0001:0000f0c8       ??_C@_05IACAFMHP@popen@    00000001800100c8     uliolib51.obj
 0001:0000f0d0       ??_C@_07FKJPAINK@tmpfile@  00000001800100d0     uliolib51.obj
 0001:0000f0d8       ??_C@_05NGFEDHGN@write@    00000001800100d8     uliolib51.obj
 0001:0000f0e0       ??_C@_04EDECCOGL@seek@     00000001800100e0     uliolib51.obj
 0001:0000f0e8       ??_C@_07HHBPNGAN@setvbuf@  00000001800100e8     uliolib51.obj
 0001:0000f0f0       ??_C@_06DJHOIPC@?$CFs?3?5?$CFs@ 00000001800100f0     uliolib51.obj
 0001:0000f0f8       ??_C@_02DKCKIIND@?$CFs@    00000001800100f8     uliolib51.obj
 0001:0000f0fc       ??_C@_05KCHOJJD@FILE?$CK@  00000001800100fc     uliolib51.obj
 0001:0000f108       ??_C@_0M@IBKPHHKH@closed?5file@ 0000000180010108     uliolib51.obj
 0001:0000f114       ??_C@_04DAMGJPCA@file@     0000000180010114     uliolib51.obj
 0001:0000f120       ??_C@_0BN@LPOOHAOM@attempt?5to?5use?5a?5closed?5file@ 0000000180010120     uliolib51.obj
 0001:0000f140       ??_C@_0BL@PEFGCPAG@cannot?5close?5standard?5file@ 0000000180010140     uliolib51.obj
 0001:0000f160       ??_C@_07DMJMBBKE@__close@  0000000180010160     uliolib51.obj
 0001:0000f168       ??_C@_0O@PLFAPHPG@file?5?$CIclosed?$CJ@ 0000000180010168     uliolib51.obj
 0001:0000f178       ??_C@_09BPMAMLLD@file?5?$CI?$CFp?$CJ@ 0000000180010178     uliolib51.obj
 0001:0000f188       ??_C@_17OBBFBLGE@?$AAr?$AAw?$AAa@ 0000000180010188     uliolib51.obj
 0001:0000f190       ??_C@_0CP@DHGANCPP@invalid?5mode?5?8?$CFs?8?5?$CIshould?5match@ 0000000180010190     uliolib51.obj
 0001:0000f1c0       ??_C@_0BL@JMNLNGCA@standard?5?$CFs?5file?5is?5closed@ 00000001800101c0     uliolib51.obj
 0001:0000f1dc       ??_C@_13CIFDLIMG@?$AAw@    00000001800101dc     uliolib51.obj
 0001:0000f1e0       ??_C@_03DLDNIBIK@?$CFlf@   00000001800101e0     uliolib51.obj
 0001:0000f1e8       ??_C@_0BD@IOJAAODF@too?5many?5arguments@ 00000001800101e8     uliolib51.obj
 0001:0000f200       ??_C@_0P@PJFAGLMH@invalid?5option@ 0000000180010200     uliolib51.obj
 0001:0000f210       ??_C@_0P@CENJCLHM@invalid?5format@ 0000000180010210     uliolib51.obj
 0001:0000f220       ??_C@_0BH@PBGIDLEF@file?5is?5already?5closed@ 0000000180010220     uliolib51.obj
 0001:0000f238       ??_C@_05CGOEHEFE@?$CF?414g@ 0000000180010238     uliolib51.obj
 0001:0000f240       ??_C@_0DB@KKADAMFH@rawhandle?5is?5only?5available?5in?5@ 0000000180010240     uliolib51.obj
 0001:0000f274       ??_C@_05MHOFLBOO@stdin@    0000000180010274     uliolib51.obj
 0001:0000f27c       ??_C@_06DJDOIFHB@stdout@   000000018001027c     uliolib51.obj
 0001:0000f284       ??_C@_06FJGNEBG@stderr@    0000000180010284     uliolib51.obj
 0001:0000f320       ??_C@_07KOEABFCN@loadlib@  0000000180010320     uloadlib51.obj
 0001:0000f328       ??_C@_06LNOHAKGK@seeall@   0000000180010328     uloadlib51.obj
 0001:0000f330       ??_C@_06BIEEJMKO@module@   0000000180010330     uloadlib51.obj
 0001:0000f338       ??_C@_07FFLLPPLH@require@  0000000180010338     uloadlib51.obj
 0001:0000f340       ??_C@_0BN@GMPFCLAN@unable?5to?5get?5ModuleFileName@ 0000000180010340     uloadlib51.obj
 0001:0000f360       ??_C@_13MGDFOILI@?$AA?$CB@ 0000000180010360     uloadlib51.obj
 0001:0000f368       ??_C@_09GMLHALBF@LOADLIB?3?5@ 0000000180010368     uloadlib51.obj
 0001:0000f374       ??_C@_04HDOCAJNK@?$CFs?$CFs@ 0000000180010374     uloadlib51.obj
 0001:0000f380       ??_C@_08HNNNOMMJ@_LOADLIB@ 0000000180010380     uloadlib51.obj
 0001:0000f38c       ??_C@_04HKFDNBLD@init@     000000018001038c     uloadlib51.obj
 0001:0000f394       ??_C@_13FPGAJAPJ@?$AA?2@   0000000180010394     uloadlib51.obj
 0001:0000f398       ??_C@_13JOFGPIOO@?$AA?4@   0000000180010398     uloadlib51.obj
 0001:0000f3a0       ??_C@_0BO@COFCKCAL@?8package?4?$CFs?8?5must?5be?5a?5string@ 00000001800103a0     uloadlib51.obj
 0001:0000f3c0       ??_C@_0CE@EPEHLLIH@?8package?4?$CFs?8?5contains?5invalid?5U@ 00000001800103c0     uloadlib51.obj
 0001:0000f3e4       ??_C@_13HGPDMIBE@?$AA?$DP@ 00000001800103e4     uloadlib51.obj
 0001:0000f3e8       ??_C@_0P@NEBKIMDC@?6?7no?5file?5?8?$CFs?8@ 00000001800103e8     uloadlib51.obj
 0001:0000f3f8       ??_C@_0CO@KHMIPLKM@error?5loading?5module?5?8?$CFs?8?5from?5@ 00000001800103f8     uloadlib51.obj
 0001:0000f428       ??_C@_04LNEJFJGI@path@     0000000180010428     uloadlib51.obj
 0001:0000f430       ??_C@_01IDAFKMJL@_@        0000000180010430     uloadlib51.obj
 0001:0000f434       ??_C@_01LFCBOECM@?4@       0000000180010434     uloadlib51.obj
 0001:0000f438       ??_C@_0L@KHKMBFOE@luaopen_?$CFs@ 0000000180010438     uloadlib51.obj
 0001:0000f444       ??_C@_05EEMJHCCC@cpath@    0000000180010444     uloadlib51.obj
 0001:0000f450       ??_C@_0BO@KOILFIGK@?6?7no?5module?5?8?$CFs?8?5in?5file?5?8?$CFs?8@ 0000000180010450     uloadlib51.obj
 0001:0000f470       ??_C@_0CC@CCJHFBLH@?8package?4preload?8?5must?5be?5a?5tab@ 0000000180010470     uloadlib51.obj
 0001:0000f498       ??_C@_0CB@NPNABMBF@?6?7no?5field?5package?4preload?$FL?8?$CFs?8@ 0000000180010498     uloadlib51.obj
 0001:0000f4c0       ??_C@_07PINPBNPB@_LOADED@  00000001800104c0     uloadlib51.obj
 0001:0000f4c8       ??_C@_0CL@DIEJCPFH@loop?5or?5previous?5error?5loading?5@ 00000001800104c8     uloadlib51.obj
 0001:0000f4f8       ??_C@_07JAOCDFCG@loaders@  00000001800104f8     uloadlib51.obj
 0001:0000f500       ??_C@_0CC@IGEJMOFI@?8package?4loaders?8?5must?5be?5a?5tab@ 0000000180010500     uloadlib51.obj
 0001:0000f528       ??_C@_0BJ@HFHHABH@module?5?8?$CFs?8?5not?5found?3?$CFs@ 0000000180010528     uloadlib51.obj
 0001:0000f544       ??_C@_01INIBCBCB@f@        0000000180010544     uloadlib51.obj
 0001:0000f548       ??_C@_0CI@GKOMOAFD@?8module?8?5not?5called?5from?5a?5Lua?5@ 0000000180010548     uloadlib51.obj
 0001:0000f570       ??_C@_02CCIJHOCI@_M@       0000000180010570     uloadlib51.obj
 0001:0000f574       ??_C@_05ICMCJINN@_NAME@    0000000180010574     uloadlib51.obj
 0001:0000f580       ??_C@_08HONLOGDK@_PACKAGE@ 0000000180010580     uloadlib51.obj
 0001:0000f590       ??_C@_0BO@CBJIAGLF@name?5conflict?5for?5module?5?8?$CFs?8@ 0000000180010590     uloadlib51.obj
 0001:0000f5b0       ??_C@_17KOAMMDLI@?$AA?$DL?$AA?$AB?$AA?$DL@ 00000001800105b0     uloadlib51.obj
 0001:0000f5b8       ??_C@_15HKKNGJC@?$AA?$DL?$AA?$DL@ 00000001800105b8     uloadlib51.obj
 0001:0000f5c0       ??_C@_13GGAHEHIG@?$AA?$AB@ 00000001800105c0     uloadlib51.obj
 0001:0000f5d0       ??_C@_1HE@JLDBNBHO@?$AA?4?$AA?2?$AA?$DP?$AA?4?$AAl?$AAu?$AAa?$AA?$DL?$AA?$CB?$AA?2?$AAl?$AAu?$AAa?$AA?2?$AA?$DP@ 00000001800105d0     uloadlib51.obj
 0001:0000f648       ??_C@_1BC@ILFFIBFI@?$AAL?$AAU?$AAA?$AA_?$AAP?$AAA?$AAT?$AAH@ 0000000180010648     uloadlib51.obj
 0001:0000f660       ??_C@_1DM@FGPGEDD@?$AA?4?$AA?2?$AA?$DP?$AA?4?$AAd?$AAl?$AAl?$AA?$DL?$AA?$CB?$AA?2?$AA?$DP?$AA?4?$AAd?$AAl?$AAl@ 0000000180010660     uloadlib51.obj
 0001:0000f6a0       ??_C@_1BE@EFNILHBI@?$AAL?$AAU?$AAA?$AA_?$AAC?$AAP?$AAA?$AAT?$AAH@ 00000001800106a0     uloadlib51.obj
 0001:0000f6b8       ??_C@_1BE@CKNDCMBB@?$AA?2?$AA?6?$AA?$DL?$AA?6?$AA?$DP?$AA?6?$AA?$CB?$AA?6?$AA?9@ 00000001800106b8     uloadlib51.obj
 0001:0000f6cc       ??_C@_06HEJKKHEK@config@   00000001800106cc     uloadlib51.obj
 0001:0000f6d4       ??_C@_06IILMCCFO@loaded@   00000001800106d4     uloadlib51.obj
 0001:0000f6e0       ustring_funcs              00000001800106e0     ustring.obj
 0001:0000f8d0       ??_C@_0BE@DEHGONAH@EnumSystemCodePages@ 00000001800108d0     ustring.obj
 0001:0000f8e4       ??_C@_06FMJLOCAF@GetACP@   00000001800108e4     ustring.obj
 0001:0000f8f0       ??_C@_09HLFMNDA@GetCPInfo@ 00000001800108f0     ustring.obj
 0001:0000f900       ??_C@_0O@PIBBCLJF@GetCurrentDir@ 0000000180010900     ustring.obj
 0001:0000f910       ??_C@_0N@IIBOJKJ@GetDriveType@ 0000000180010910     ustring.obj
 0001:0000f920       ??_C@_0M@KHMMJMNI@GetFileAttr@ 0000000180010920     ustring.obj
 0001:0000f930       ??_C@_0M@ONGMCNNE@GetKeyState@ 0000000180010930     ustring.obj
 0001:0000f940       ??_C@_0BH@KKAFOIJJ@GetLogicalDriveStrings@ 0000000180010940     ustring.obj
 0001:0000f958       ??_C@_08OMCNFONF@GetOEMCP@ 0000000180010958     ustring.obj
 0001:0000f968       ??_C@_0N@EBDGNADB@GetConsoleCP@ 0000000180010968     ustring.obj
 0001:0000f978       ??_C@_0N@DFIIBMHN@SetConsoleCP@ 0000000180010978     ustring.obj
 0001:0000f988       ??_C@_0BD@LLGELLLN@GetConsoleOutputCP@ 0000000180010988     ustring.obj
 0001:0000f9a0       ??_C@_0BD@EBEOINFF@SetConsoleOutputCP@ 00000001800109a0     ustring.obj
 0001:0000f9b8       ??_C@_0BD@IHIHPGDL@GlobalMemoryStatus@ 00000001800109b8     ustring.obj
 0001:0000f9d0       ??_C@_0BE@HCIKGJGE@MultiByteToWideChar@ 00000001800109d0     ustring.obj
 0001:0000f9e8       ??_C@_09EPINLGBH@OemToUtf8@ 00000001800109e8     ustring.obj
 0001:0000f9f8       ??_C@_0BC@NFCPMJFM@OutputDebugString@ 00000001800109f8     ustring.obj
 0001:0000fa10       ??_C@_0BA@MNJFBAJH@SHGetFolderPath@ 0000000180010a10     ustring.obj
 0001:0000fa20       ??_C@_0L@PMCLJMMJ@SearchPath@ 0000000180010a20     ustring.obj
 0001:0000fa30       ??_C@_0O@IHAPJIOC@SetCurrentDir@ 0000000180010a30     ustring.obj
 0001:0000fa40       ??_C@_0M@KINCEKFL@SetFileAttr@ 0000000180010a40     ustring.obj
 0001:0000fa4c       ??_C@_05PFDOMJEF@Sleep@    0000000180010a4c     ustring.obj
 0001:0000fa58       ??_C@_0M@KJELMDJD@Utf16ToUtf8@ 0000000180010a58     ustring.obj
 0001:0000fa68       ??_C@_09LCEKPEGC@Utf8ToOem@ 0000000180010a68     ustring.obj
 0001:0000fa78       ??_C@_0M@GJGCILHG@Utf8ToUtf16@ 0000000180010a78     ustring.obj
 0001:0000fa84       ??_C@_04NDFIEGPL@Uuid@     0000000180010a84     ustring.obj
 0001:0000fa90       ??_C@_0BE@LJADKLBD@WideCharToMultiByte@ 0000000180010a90     ustring.obj
 0001:0000faa4       ??_C@_04GFOHBGIO@subW@     0000000180010aa4     ustring.obj
 0001:0000faac       ??_C@_06FHFOAHML@system@   0000000180010aac     ustring.obj
 0001:0000fab4       ??_C@_04NOFELICG@lenW@     0000000180010ab4     ustring.obj
 0001:0000fac0       ??_C@_0BB@BLJKPILH@system?5error?5?$CFd?6@ 0000000180010ac0     ustring.obj
 0001:0000fad8       ??_C@_0BJ@MEAJDMDL@invalid?5multibyte?5string@ 0000000180010ad8     ustring.obj
 0001:0000faf8       ??_C@_0BG@ELIKBHAO@invalid?5UTF?916?5string@ 0000000180010af8     ustring.obj
 0001:0000fb10       ??_C@_0M@KJGJBDLL@MaxCharSize@ 0000000180010b10     ustring.obj
 0001:0000fb20       ??_C@_0M@IMOFNPBB@DefaultChar@ 0000000180010b20     ustring.obj
 0001:0000fb30       ??_C@_08HIIJAENB@LeadByte@ 0000000180010b30     ustring.obj
 0001:0000fb40       ??_C@_0BD@CBNPFFPH@UnicodeDefaultChar@ 0000000180010b40     ustring.obj
 0001:0000fb58       ??_C@_0N@DJCOCBOB@CodePageName@ 0000000180010b58     ustring.obj
 0001:0000fb68       ??_C@_0N@IFJMFGJK@unknown?5type@ 0000000180010b68     ustring.obj
 0001:0000fb78       ??_C@_0BC@GPFCFLGN@no?5root?5directory@ 0000000180010b78     ustring.obj
 0001:0000fb90       ??_C@_09HPGMKNKO@removable@ 0000000180010b90     ustring.obj
 0001:0000fb9c       ??_C@_05OFLEIIDM@fixed@    0000000180010b9c     ustring.obj
 0001:0000fba4       ??_C@_06IMIHEKN@remote@    0000000180010ba4     ustring.obj
 0001:0000fbac       ??_C@_05POABADMF@cdrom@    0000000180010bac     ustring.obj
 0001:0000fbb8       ??_C@_07BHCBOAMP@ramdisk@  0000000180010bb8     ustring.obj
 0001:0000fbc0       ??_C@_0L@PLJFMBIJ@MemoryLoad@ 0000000180010bc0     ustring.obj
 0001:0000fbd0       ??_C@_09MMAOIBBJ@TotalPhys@ 0000000180010bd0     ustring.obj
 0001:0000fbe0       ??_C@_09KFOEOLH@AvailPhys@ 0000000180010be0     ustring.obj
 0001:0000fbf0       ??_C@_0O@PEEMGPEP@TotalPageFile@ 0000000180010bf0     ustring.obj
 0001:0000fc00       ??_C@_0O@LLHOKNF@AvailPageFile@ 0000000180010c00     ustring.obj
 0001:0000fc10       ??_C@_0N@LCJEOHMM@TotalVirtual@ 0000000180010c10     ustring.obj
 0001:0000fc20       ??_C@_0N@EGHLANBF@AvailVirtual@ 0000000180010c20     ustring.obj
 0001:0000fc30       ??_C@_0BF@KKNLCGDE@AvailExtendedVirtual@ 0000000180010c30     ustring.obj
 0001:0000fc48       ??_C@_0P@KJDDGAFH@FileAttributes@ 0000000180010c48     ustring.obj
 0001:0000fc58       ??_C@_07JOJHCKGP@ustring@  0000000180010c58     ustring.obj
 0001:00010518       ??_C@_0DJ@KKHMCMAP@bad?5field?5?$FL?$CFd?$FN?5in?5table?5stackpo@ 0000000180011518     util.obj
 0001:00010558       ??_C@_0DJ@PFHHGAMM@bad?5field?5?8?$CFs?8?5in?5table?5stackpo@ 0000000180011558     util.obj
 0001:00010594       ??_C@_06EBGNBFIA@number@   0000000180011594     util.obj
 0001:000105c0       win_funcs                  00000001800115c0     win.obj
 0001:00011038       ??_C@_0O@CFPMOCDP@CompareString@ 0000000180012038     win.obj
 0001:00011048       ??_C@_08PPLNFCGA@CopyFile@ 0000000180012048     win.obj
 0001:00011058       ??_C@_09INHPLKKM@CreateDir@ 0000000180012058     win.obj
 0001:00011068       ??_C@_0L@GPLPOFDC@DeleteFile@ 0000000180012068     win.obj
 0001:00011078       ??_C@_0N@FOJPHHPH@DeleteRegKey@ 0000000180012078     win.obj
 0001:00011088       ??_C@_0P@PCCDOIAL@DeleteRegValue@ 0000000180012088     win.obj
 0001:00011098       ??_C@_0L@DGAGCFOP@EnumRegKey@ 0000000180012098     win.obj
 0001:000110a8       ??_C@_0N@PFFNCIBD@EnumRegValue@ 00000001800120a8     win.obj
 0001:000110b8       ??_C@_0L@MGMEFCAE@ExtractKey@ 00000001800120b8     win.obj
 0001:000110c8       ??_C@_0N@HALOIPMN@ExtractKeyEx@ 00000001800120c8     win.obj
 0001:000110d8       ??_C@_0N@DNBFBBHK@IsWinVersion@ 00000001800120d8     win.obj
 0001:000110e8       ??_C@_0BI@EKFDIGHI@FileTimeToLocalFileTime@ 00000001800120e8     win.obj
 0001:00011100       ??_C@_0BF@KPJNHALE@FileTimeToSystemTime@ 0000000180012100     win.obj
 0001:00011118       ??_C@_0BL@NAIJNMLL@GetConsoleScreenBufferInfo@ 0000000180012118     win.obj
 0001:00011134       ??_C@_06CALCCDMF@GetEnv@   0000000180012134     win.obj
 0001:00011140       ??_C@_0M@EINGHLOA@GetFileInfo@ 0000000180012140     win.obj
 0001:00011150       ??_C@_09GFGIAJLD@GetRegKey@ 0000000180012150     win.obj
 0001:00011160       ??_C@_0BI@ENMDHCMK@GetSystemTimeAsFileTime@ 0000000180012160     win.obj
 0001:00011178       ??_C@_0P@GGGHOPAD@GetVirtualKeys@ 0000000180012178     win.obj
 0001:00011188       ??_C@_0P@MIPPOCAO@IsProcess64bit@ 0000000180012188     win.obj
 0001:00011198       ??_C@_08CALLHOCI@MoveFile@ 0000000180012198     win.obj
 0001:000111a8       ??_C@_09EDKALOCB@RemoveDir@ 00000001800121a8     win.obj
 0001:000111b8       ??_C@_0L@HBAGBENL@RenameFile@ 00000001800121b8     win.obj
 0001:000111c4       ??_C@_06LDCDJLBI@SetEnv@   00000001800121c4     win.obj
 0001:000111d0       ??_C@_09ELCNCICB@SetRegKey@ 00000001800121d0     win.obj
 0001:000111e0       ??_C@_0N@BFFIJKHB@ShellExecute@ 00000001800121e0     win.obj
 0001:000111f0       ??_C@_0BF@HBHGIPOG@SystemTimeToFileTime@ 00000001800121f0     win.obj
 0001:00011208       ??_C@_06DNONFAKH@wcscmp@   0000000180012208     win.obj
 0001:00011210       ??_C@_0N@OCKOJJEP@WriteConsole@ 0000000180012210     win.obj
 0001:00011220       ??_C@_04CBBMIBLK@HKLM@     0000000180012220     win.obj
 0001:00011228       ??_C@_04LEMDOLAJ@HKCC@     0000000180012228     win.obj
 0001:00011230       ??_C@_04OHBKMIBJ@HKCR@     0000000180012230     win.obj
 0001:00011238       ??_C@_04KIFLFONO@HKCU@     0000000180012238     win.obj
 0001:00011240       ??_C@_03DLBIJLAB@HKU@      0000000180012240     win.obj
 0001:00011248       ??_C@_0DA@DKALLFDI@must?5be?5?8HKLM?8?0?5?8HKCC?8?0?5?8HKCR?8?0@ 0000000180012248     win.obj
 0001:00011278       ??_C@_05KDALNKAH@dword@    0000000180012278     win.obj
 0001:00011280       ??_C@_06FNFBAEBE@binary@   0000000180012280     win.obj
 0001:00011288       ??_C@_0N@CBOMHLPN@expandstring@ 0000000180012288     win.obj
 0001:00011298       ??_C@_0M@PEGIPCHN@multistring@ 0000000180012298     win.obj
 0001:000112a8       ??_C@_0BH@NOJOGNJM@unsupported?5value?5type@ 00000001800122a8     win.obj
 0001:000112c0       ??_C@_0BD@MJODDCFG@OpenRegKey?5failed?4@ 00000001800122c0     win.obj
 0001:000112d8       ??_C@_0BI@COLHBIIE@RegQueryValueEx?5failed?4@ 00000001800122d8     win.obj
 0001:000112f0       ??_C@_1BK@BIGILECK@?$AAA?$AAd?$AAv?$AAa?$AAp?$AAi?$AA3?$AA2?$AA?4?$AAd?$AAl?$AAl@ 00000001800122f0     win.obj
 0001:00011310       ??_C@_0BA@LILAPHGE@RegDeleteKeyExW@ 0000000180012310     win.obj
 0001:00011320       ??_C@_0BG@HHFHBIKG@RegOpenKeyExW?5failed?4@ 0000000180012320     win.obj
 0001:00011338       ??_C@_05DFPNHDMN@wYear@    0000000180012338     win.obj
 0001:00011340       ??_C@_06MGNNJGBJ@wMonth@   0000000180012340     win.obj
 0001:00011348       ??_C@_0L@OAHPHHP@wDayOfWeek@ 0000000180012348     win.obj
 0001:00011354       ??_C@_04NBLBJIPP@wDay@     0000000180012354     win.obj
 0001:0001135c       ??_C@_05BMOPCGDH@wHour@    000000018001235c     win.obj
 0001:00011368       ??_C@_07HPODENI@wMinute@   0000000180012368     win.obj
 0001:00011370       ??_C@_07IIEDHHJN@wSecond@  0000000180012370     win.obj
 0001:00011378       ??_C@_0O@HBAPEOKP@wMilliseconds@ 0000000180012378     win.obj
 0001:00011388       ??_C@_01LKDEMHDF@s@        0000000180012388     win.obj
 0001:00011390       ??_C@_0BA@IAFODGNM@CursorPositionX@ 0000000180012390     win.obj
 0001:000113a0       ??_C@_0BA@JJEFAHJN@CursorPositionY@ 00000001800123a0     win.obj
 0001:000113b0       ??_C@_0L@NFCEOFBF@WindowLeft@ 00000001800123b0     win.obj
 0001:000113c0       ??_C@_09JHGOALHG@WindowTop@ 00000001800123c0     win.obj
 0001:000113d0       ??_C@_0M@HHPHMPGH@WindowRight@ 00000001800123d0     win.obj
 0001:000113e0       ??_C@_0N@JPIJCAOJ@WindowBottom@ 00000001800123e0     win.obj
 0001:000113f0       ??_C@_0BD@DOLDEII@MaximumWindowSizeX@ 00000001800123f0     win.obj
 0001:00011408       ??_C@_0BD@BKPAAFMJ@MaximumWindowSizeY@ 0000000180012408     win.obj
 0001:0001141c       ??_C@_01PFHFFBPC@t@        000000018001241c     win.obj
 0001:00011420       ??_C@_0BJ@LPJMBJJL@directory?5already?5exists@ 0000000180012420     win.obj
 0001:0001143c       ??_C@_02NIKKAELB@XP@       000000018001243c     win.obj
 0001:00011440       ??_C@_05OFKKJCED@XPSP1@    0000000180012440     win.obj
 0001:00011448       ??_C@_05MOIHMBIA@XPSP2@    0000000180012448     win.obj
 0001:00011450       ??_C@_05NHJMPAMB@XPSP3@    0000000180012450     win.obj
 0001:00011458       ??_C@_05FGFMDFJC@Vista@    0000000180012458     win.obj
 0001:00011460       ??_C@_08ENCCDKOP@VistaSP1@ 0000000180012460     win.obj
 0001:00011470       ??_C@_08GGAPGJCM@VistaSP2@ 0000000180012470     win.obj
 0001:0001147c       ??_C@_02PJEKLOOM@W7@       000000018001247c     win.obj
 0001:00011480       ??_C@_05DPOOILML@W7SP1@    0000000180012480     win.obj
 0001:00011488       ??_C@_02HONCKCCD@W8@       0000000180012488     win.obj
 0001:0001148c       ??_C@_04HCPPKHCP@W8?41@    000000018001248c     win.obj
 0001:00011494       ??_C@_03HCIOKOKM@W10@      0000000180012494     win.obj
 0001:00011498       ??_C@_06LGMEBDBC@Server@   0000000180012498     win.obj
 0001:000114a0       ??_C@_0BH@CNFJKJGO@invalid?5argument?5value@ 00000001800124a0     win.obj
 0001:000114b8       ??_C@_0BK@LNHOAEDA@must?5be?5string?5or?5integer@ 00000001800124b8     win.obj
 0001:000114d8       __real@41f0000000000000    00000001800124d8     win.obj
 0001:000114e0       _pRawDllMain               00000001800124e0     LIBCMT:dll_dllmain.obj
 0001:000114e0       _pDefaultRawDllMain        00000001800124e0     LIBCMT:dll_dllmain.obj
 0001:000114e8       _pDestructExceptionObject  00000001800124e8     libvcruntime:ehhelpers.obj
 0001:00011828       ??_C@_08EHJDFFNH@__based?$CI@ 0000000180012828     libvcruntime:undname.obj
 0001:00011838       ??_C@_07KOLFKCDI@__cdecl@  0000000180012838     libvcruntime:undname.obj
 0001:00011840       ??_C@_08GHMPAG@__pascal@   0000000180012840     libvcruntime:undname.obj
 0001:00011850       ??_C@_09IFJBGAPI@__stdcall@ 0000000180012850     libvcruntime:undname.obj
 0001:00011860       ??_C@_0L@NPHFGOKO@__thiscall@ 0000000180012860     libvcruntime:undname.obj
 0001:00011870       ??_C@_0L@JMKHOMEK@__fastcall@ 0000000180012870     libvcruntime:undname.obj
 0001:00011880       ??_C@_0N@BCKKPABJ@__vectorcall@ 0000000180012880     libvcruntime:undname.obj
 0001:00011890       ??_C@_09HIJEGCPM@__clrcall@ 0000000180012890     libvcruntime:undname.obj
 0001:0001189c       ??_C@_06GHPCKEAG@__eabi@   000000018001289c     libvcruntime:undname.obj
 0001:000118a8       ??_C@_09IOPIDJLG@__swift_1@ 00000001800128a8     libvcruntime:undname.obj
 0001:000118b8       ??_C@_09KFNFGKHF@__swift_2@ 00000001800128b8     libvcruntime:undname.obj
 0001:000118c8       ??_C@_07JOMMBBKO@__ptr64@  00000001800128c8     libvcruntime:undname.obj
 0001:000118d0       ??_C@_0L@PILCLIHE@__restrict@ 00000001800128d0     libvcruntime:undname.obj
 0001:000118e0       ??_C@_0M@GFIIJFMG@__unaligned@ 00000001800128e0     libvcruntime:undname.obj
 0001:000118f0       ??_C@_09DHDLOLLB@restrict?$CI@ 00000001800128f0     libvcruntime:undname.obj
 0001:000118fc       ??_C@_04NIHEBCM@?5new@     00000001800128fc     libvcruntime:undname.obj
 0001:00011908       ??_C@_07FPCDHGMM@?5delete@ 0000000180012908     libvcruntime:undname.obj
 0001:00011910       ??_C@_01NEMOKFLO@?$DN@     0000000180012910     libvcruntime:undname.obj
 0001:00011914       ??_C@_02GPIOPFAK@?$DO?$DO@ 0000000180012914     libvcruntime:undname.obj
 0001:00011918       ??_C@_02FODMEDOG@?$DM?$DM@ 0000000180012918     libvcruntime:undname.obj
 0001:0001191c       ??_C@_01DCLJPIOD@?$CB@     000000018001291c     libvcruntime:undname.obj
 0001:00011920       ??_C@_02EGOFBIJA@?$DN?$DN@ 0000000180012920     libvcruntime:undname.obj
 0001:00011924       ??_C@_02FDNJECIE@?$CB?$DN@ 0000000180012924     libvcruntime:undname.obj
 0001:00011928       ??_C@_02GPECMEKF@?$FL?$FN@ 0000000180012928     libvcruntime:undname.obj
 0001:00011930       ??_C@_08LHJFAFGD@operator@ 0000000180012930     libvcruntime:undname.obj
 0001:0001193c       ??_C@_02HBOOOICD@?9?$DO@   000000018001293c     libvcruntime:undname.obj
 0001:00011940       ??_C@_01NBENCBCI@?$CK@     0000000180012940     libvcruntime:undname.obj
 0001:00011944       ??_C@_02ECNGHCIF@?$CL?$CL@ 0000000180012944     libvcruntime:undname.obj
 0001:00011948       ??_C@_02BAABKJLB@?9?9@     0000000180012948     libvcruntime:undname.obj
 0001:0001194c       ??_C@_01JOAMLHOP@?9@       000000018001294c     libvcruntime:undname.obj
 0001:00011950       ??_C@_01MIFGBAGJ@?$CL@     0000000180012950     libvcruntime:undname.obj
 0001:00011954       ??_C@_01HNPIGOCE@?$CG@     0000000180012954     libvcruntime:undname.obj
 0001:00011958       ??_C@_03MNHNFDLC@?9?$DO?$CK@ 0000000180012958     libvcruntime:undname.obj
 0001:0001195c       ??_C@_01FGNFDNOH@?$CF@     000000018001295c     libvcruntime:undname.obj
 0001:00011960       ??_C@_01MNNFJEPP@?$DM@     0000000180012960     libvcruntime:undname.obj
 0001:00011964       ??_C@_02EHCHHCKH@?$DM?$DN@ 0000000180012964     libvcruntime:undname.obj
 0001:00011968       ??_C@_01PPODPGHN@?$DO@     0000000180012968     libvcruntime:undname.obj
 0001:0001196c       ??_C@_02EEKDKGMJ@?$DO?$DN@ 000000018001296c     libvcruntime:undname.obj
 0001:00011970       ??_C@_01IHBHIGKO@?0@       0000000180012970     libvcruntime:undname.obj
 0001:00011974       ??_C@_02HCKGKOFO@?$CI?$CJ@ 0000000180012974     libvcruntime:undname.obj
 0001:00011978       ??_C@_01PJKLJHI@?$HO@      0000000180012978     libvcruntime:undname.obj
 0001:0001197c       ??_C@_01JKBOJNNK@?$FO@     000000018001297c     libvcruntime:undname.obj
 0001:00011980       ??_C@_01DNKMNLPK@?$HM@     0000000180012980     libvcruntime:undname.obj
 0001:00011984       ??_C@_02PPKAJPJL@?$CG?$CG@ 0000000180012984     libvcruntime:undname.obj
 0001:00011988       ??_C@_02NONPIBCD@?$HM?$HM@ 0000000180012988     libvcruntime:undname.obj
 0001:0001198c       ??_C@_02FPIMKNGF@?$CK?$DN@ 000000018001298c     libvcruntime:undname.obj
 0001:00011990       ??_C@_02FOEOMHFC@?$CL?$DN@ 0000000180012990     libvcruntime:undname.obj
 0001:00011994       ??_C@_02FKMDLLOA@?9?$DN@   0000000180012994     libvcruntime:undname.obj
 0001:00011998       ??_C@_02FJEHGPIO@?1?$DN@   0000000180012998     libvcruntime:undname.obj
 0001:0001199c       ??_C@_02FENAOKFI@?$CF?$DN@ 000000018001299c     libvcruntime:undname.obj
 0001:000119a0       ??_C@_03IKFCCPFF@?$DO?$DO?$DN@ 00000001800129a0     libvcruntime:undname.obj
 0001:000119a4       ??_C@_03CDNPDDLA@?$DM?$DM?$DN@ 00000001800129a4     libvcruntime:undname.obj
 0001:000119a8       ??_C@_02FGJGFEAB@?$CG?$DN@ 00000001800129a8     libvcruntime:undname.obj
 0001:000119ac       ??_C@_02DHLNPPGH@?$HM?$DN@ 00000001800129ac     libvcruntime:undname.obj
 0001:000119b0       ??_C@_02MHEGNOJ@?$FO?$DN@  00000001800129b0     libvcruntime:undname.obj
 0001:000119b8       ??_C@_09IFPLHPGF@?$GAvftable?8@ 00000001800129b8     libvcruntime:undname.obj
 0001:000119c8       ??_C@_09BLBHBJP@?$GAvbtable?8@ 00000001800129c8     libvcruntime:undname.obj
 0001:000119d8       ??_C@_07FEEIOKP@?$GAvcall?8@ 00000001800129d8     libvcruntime:undname.obj
 0001:000119e0       ??_C@_08LLFFHHDJ@?$GAtypeof?8@ 00000001800129e0     libvcruntime:undname.obj
 0001:000119f0       ??_C@_0BF@KDPPACIK@?$GAlocal?5static?5guard?8@ 00000001800129f0     libvcruntime:undname.obj
 0001:00011a08       ??_C@_08OBABFOLI@?$GAstring?8@ 0000000180012a08     libvcruntime:undname.obj
 0001:00011a18       ??_C@_0BD@JDLKDPAB@?$GAvbase?5destructor?8@ 0000000180012a18     libvcruntime:undname.obj
 0001:00011a30       ??_C@_0BN@DEGPLNFK@?$GAvector?5deleting?5destructor?8@ 0000000180012a30     libvcruntime:undname.obj
 0001:00011a50       ??_C@_0BO@OBMKPJIG@?$GAdefault?5constructor?5closure?8@ 0000000180012a50     libvcruntime:undname.obj
 0001:00011a70       ??_C@_0BN@IMDCHIKM@?$GAscalar?5deleting?5destructor?8@ 0000000180012a70     libvcruntime:undname.obj
 0001:00011a90       ??_C@_0BO@PFGOCPJJ@?$GAvector?5constructor?5iterator?8@ 0000000180012a90     libvcruntime:undname.obj
 0001:00011ab0       ??_C@_0BN@LFPFMEDL@?$GAvector?5destructor?5iterator?8@ 0000000180012ab0     libvcruntime:undname.obj
 0001:00011ad0       ??_C@_0CE@IKBNEHA@?$GAvector?5vbase?5constructor?5itera@ 0000000180012ad0     libvcruntime:undname.obj
 0001:00011af8       ??_C@_0BL@NILFHHPC@?$GAvirtual?5displacement?5map?8@ 0000000180012af8     libvcruntime:undname.obj
 0001:00011b18       ??_C@_0CB@JONCMFFK@?$GAeh?5vector?5constructor?5iterator@ 0000000180012b18     libvcruntime:undname.obj
 0001:00011b40       ??_C@_0CA@GCEOPDGL@?$GAeh?5vector?5destructor?5iterator?8@ 0000000180012b40     libvcruntime:undname.obj
 0001:00011b60       ??_C@_0CH@OOJPLCPH@?$GAeh?5vector?5vbase?5constructor?5it@ 0000000180012b60     libvcruntime:undname.obj
 0001:00011b88       ??_C@_0BL@LLKPOHJI@?$GAcopy?5constructor?5closure?8@ 0000000180012b88     libvcruntime:undname.obj
 0001:00011ba8       ??_C@_0BA@KBCDOMBN@?$GAudt?5returning?8@ 0000000180012ba8     libvcruntime:undname.obj
 0001:00011bb8       ??_C@_03KLGMFNMG@?$GAEH@   0000000180012bb8     libvcruntime:undname.obj
 0001:00011bbc       ??_C@_05KHLCHHI@?$GARTTI@  0000000180012bbc     libvcruntime:undname.obj
 0001:00011bc8       ??_C@_0BA@KKLDJDLB@?$GAlocal?5vftable?8@ 0000000180012bc8     libvcruntime:undname.obj
 0001:00011bd8       ??_C@_0CE@IIHCMGGL@?$GAlocal?5vftable?5constructor?5clos@ 0000000180012bd8     libvcruntime:undname.obj
 0001:00011bfc       ??_C@_06FHBGPFGH@?5new?$FL?$FN@ 0000000180012bfc     libvcruntime:undname.obj
 0001:00011c08       ??_C@_09LBNFPBCA@?5delete?$FL?$FN@ 0000000180012c08     libvcruntime:undname.obj
 0001:00011c18       ??_C@_0P@HJKNJFNN@?$GAomni?5callsig?8@ 0000000180012c18     libvcruntime:undname.obj
 0001:00011c28       ??_C@_0BL@CNOONJFP@?$GAplacement?5delete?5closure?8@ 0000000180012c28     libvcruntime:undname.obj
 0001:00011c48       ??_C@_0BN@CKNJLHMB@?$GAplacement?5delete?$FL?$FN?5closure?8@ 0000000180012c48     libvcruntime:undname.obj
 0001:00011c68       ??_C@_0CG@CFDHKGGD@?$GAmanaged?5vector?5constructor?5ite@ 0000000180012c68     libvcruntime:undname.obj
 0001:00011c90       ??_C@_0CF@IMGKMJNO@?$GAmanaged?5vector?5destructor?5iter@ 0000000180012c90     libvcruntime:undname.obj
 0001:00011cb8       ??_C@_0CG@HLDDJMAG@?$GAeh?5vector?5copy?5constructor?5ite@ 0000000180012cb8     libvcruntime:undname.obj
 0001:00011ce0       ??_C@_0CM@FCBBDIGB@?$GAeh?5vector?5vbase?5copy?5construct@ 0000000180012ce0     libvcruntime:undname.obj
 0001:00011d10       ??_C@_0BL@CLIPGLGB@?$GAdynamic?5initializer?5for?5?8@ 0000000180012d10     libvcruntime:undname.obj
 0001:00011d30       ??_C@_0CB@PDBIFEP@?$GAdynamic?5atexit?5destructor?5for?5@ 0000000180012d30     libvcruntime:undname.obj
 0001:00011d58       ??_C@_0CD@CGAJBKEJ@?$GAvector?5copy?5constructor?5iterat@ 0000000180012d58     libvcruntime:undname.obj
 0001:00011d80       ??_C@_0CJ@GJELGAMM@?$GAvector?5vbase?5copy?5constructor?5@ 0000000180012d80     libvcruntime:undname.obj
 0001:00011db0       ??_C@_0CL@FGIJHLCE@?$GAmanaged?5vector?5copy?5constructo@ 0000000180012db0     libvcruntime:undname.obj
 0001:00011de0       ??_C@_0BM@PMGGMLDN@?$GAlocal?5static?5thread?5guard?8@ 0000000180012de0     libvcruntime:undname.obj
 0001:00011e00       ??_C@_0N@BDNMDMOL@operator?5?$CC?$CC?5@ 0000000180012e00     libvcruntime:undname.obj
 0001:00011e10       ??_C@_0BC@GGEBGALA@operator?5co_await@ 0000000180012e10     libvcruntime:undname.obj
 0001:00011e28       ??_C@_0BC@DAFEJGAK@?5Type?5Descriptor?8@ 0000000180012e28     libvcruntime:undname.obj
 0001:00011e40       ??_C@_0BM@LDKODKLH@?5Base?5Class?5Descriptor?5at?5?$CI@ 0000000180012e40     libvcruntime:undname.obj
 0001:00011e60       ??_C@_0BD@LGICGFMM@?5Base?5Class?5Array?8@ 0000000180012e60     libvcruntime:undname.obj
 0001:00011e78       ??_C@_0BN@MECKDCOJ@?5Class?5Hierarchy?5Descriptor?8@ 0000000180012e78     libvcruntime:undname.obj
 0001:00011e98       ??_C@_0BK@CFCOFLF@?5Complete?5Object?5Locator?8@ 0000000180012e98     libvcruntime:undname.obj
 0001:00011ed0       ??_C@_1DM@KHCHBNEB@?$AAa?$AAp?$AAi?$AA?9?$AAm?$AAs?$AA?9?$AAw?$AAi?$AAn?$AA?9?$AAc?$AAo?$AAr?$AAe@ 0000000180012ed0     libvcruntime:winapi_downlevel.obj
 0001:00011f10       ??_C@_1DK@LPPGFMPP@?$AAa?$AAp?$AAi?$AA?9?$AAm?$AAs?$AA?9?$AAw?$AAi?$AAn?$AA?9?$AAc?$AAo?$AAr?$AAe@ 0000000180012f10     libvcruntime:winapi_downlevel.obj
 0001:00011f50       ??_C@_1BC@GDMECMAK@?$AAk?$AAe?$AAr?$AAn?$AAe?$AAl?$AA3?$AA2@ 0000000180012f50     libvcruntime:winapi_downlevel.obj
 0001:00011f68       ??_C@_1BA@PFFKHIOG@?$AAa?$AAp?$AAi?$AA?9?$AAm?$AAs?$AA?9@ 0000000180012f68     libvcruntime:winapi_downlevel.obj
 0001:00011f78       ??_C@_1BA@IAIFMGEF@?$AAe?$AAx?$AAt?$AA?9?$AAm?$AAs?$AA?9@ 0000000180012f78     libvcruntime:winapi_downlevel.obj
 0001:00011f90       ??_C@_08KNHFBNJ@FlsAlloc@  0000000180012f90     libvcruntime:winapi_downlevel.obj
 0001:00011fa8       ??_C@_07PEJMOBNF@FlsFree@  0000000180012fa8     libvcruntime:winapi_downlevel.obj
 0001:00011fb8       ??_C@_0M@GDNOONDI@FlsGetValue@ 0000000180012fb8     libvcruntime:winapi_downlevel.obj
 0001:00011fd0       ??_C@_0M@JCPCPOEF@FlsSetValue@ 0000000180012fd0     libvcruntime:winapi_downlevel.obj
 0001:00011fe8       ??_C@_0BM@HCFOFFN@InitializeCriticalSectionEx@ 0000000180012fe8     libvcruntime:winapi_downlevel.obj
 0001:00012010       standard_lookup_table      0000000180013010     libucrt:output.obj
 0001:00012070       ??_C@_1O@CEDCILHN@?$AA?$CI?$AAn?$AAu?$AAl?$AAl?$AA?$CJ?$AA?$AA@ 0000000180013070     libucrt:output.obj
 0001:00012080       ??_C@_06OJHGLDPL@?$CInull?$CJ?$AA@ 0000000180013080     libucrt:output.obj
 0001:00012200       ??_C@_0EA@FCLIIPNN@Visual?5C?$CL?$CL?5CRT?3?5Not?5enough?5memor@ 0000000180013200     libucrt:strerror.obj
 0001:00012290       ?large_power_data@?1??multiply_by_power_of_ten@__crt_strtox@@YA_NAEAUbig_integer@2@I@Z@4QBIB 0000000180013290     libucrt:input.obj
 0001:00012ba0       ?large_power_indices@?1??multiply_by_power_of_ten@__crt_strtox@@YA_NAEAUbig_integer@2@I@Z@4QBUunpack_index@?1??12@YA_N0I@Z@B 0000000180013ba0     libucrt:input.obj
 0001:00012c38       ?small_powers_of_ten@?1??multiply_by_power_of_ten@__crt_strtox@@YA_NAEAUbig_integer@2@I@Z@4QBIB 0000000180013c38     libucrt:input.obj
 0001:00012c60       ??_C@_1GE@DPGDJKLM@?$AAm?$AAi?$AAn?$AAk?$AAe?$AAr?$AAn?$AAe?$AAl?$AA?2?$AAc?$AAr?$AAt?$AAs?$AA?2?$AAu?$AAc?$AAr?$AAt?$AA?2?$AAi?$AAn?$AAc?$AA?2?$AAc?$AAo?$AAr?$AAe?$AAc?$AAr?$AAt?$AA_@ 0000000180013c60     libucrt:input.obj
 0001:00012cd0       ??_C@_1FM@FELNCOBF@?$AA_?$AA_?$AAc?$AAr?$AAt?$AA_?$AAs?$AAt?$AAr?$AAt?$AAo?$AAx?$AA?3?$AA?3?$AAf?$AAl?$AAo?$AAa?$AAt?$AAi?$AAn?$AAg?$AA_?$AAp?$AAo?$AAi?$AAn?$AAt?$AA_?$AAv?$AAa?$AAl@ 0000000180013cd0     libucrt:input.obj
 0001:00012d30       ??_C@_1BG@GEMHBGAF@?$AA_?$AAi?$AAs?$AA_?$AAd?$AAo?$AAu?$AAb?$AAl?$AAe?$AA?$AA@ 0000000180013d30     libucrt:input.obj
 0001:00012d50       ??_C@_1FK@JOJELFFO@?$AA_?$AA_?$AAc?$AAr?$AAt?$AA_?$AAs?$AAt?$AAr?$AAt?$AAo?$AAx?$AA?3?$AA?3?$AAf?$AAl?$AAo?$AAa?$AAt?$AAi?$AAn?$AAg?$AA_?$AAp?$AAo?$AAi?$AAn?$AAt?$AA_?$AAv?$AAa?$AAl@ 0000000180013d50     libucrt:input.obj
 0001:00012db0       ??_C@_1BI@BANMPGJI@?$AA?$CB?$AA_?$AAi?$AAs?$AA_?$AAd?$AAo?$AAu?$AAb?$AAl?$AAe?$AA?$AA@ 0000000180013db0     libucrt:input.obj
 0001:00012dd0       ?constraints@?1??is_length_valid@__crt_stdio_input@@YA_NW4conversion_mode@2@W4length_modifier@2@@Z@4QAY0M@$$CBEA 0000000180013dd0     libucrt:input.obj
 0001:00012e48       ?inf_uppercase@?1???$parse_floating_point_possible_infinity@DV?$input_adapter_character_source@V?$stream_input_adapter@D@__crt_stdio_input@@@__crt_strtox@@_K@__crt_strtox@@YA?AW4floating_point_parse_result@1@AEADAEAV?$input_adapter_character_source@V?$stream_input_adapter@D@__crt_stdio_input@@@1@_K@Z@4QBDB 0000000180013e48     libucrt:input.obj
 0001:00012e4c       ?inf_lowercase@?1???$parse_floating_point_possible_infinity@DV?$input_adapter_character_source@V?$stream_input_adapter@D@__crt_stdio_input@@@__crt_strtox@@_K@__crt_strtox@@YA?AW4floating_point_parse_result@1@AEADAEAV?$input_adapter_character_source@V?$stream_input_adapter@D@__crt_stdio_input@@@1@_K@Z@4QBDB 0000000180013e4c     libucrt:input.obj
 0001:00012e50       ?inity_uppercase@?1???$parse_floating_point_possible_infinity@DV?$input_adapter_character_source@V?$stream_input_adapter@D@__crt_stdio_input@@@__crt_strtox@@_K@__crt_strtox@@YA?AW4floating_point_parse_result@1@AEADAEAV?$input_adapter_character_source@V?$stream_input_adapter@D@__crt_stdio_input@@@1@_K@Z@4QBDB 0000000180013e50     libucrt:input.obj
 0001:00012e58       ?inity_lowercase@?1???$parse_floating_point_possible_infinity@DV?$input_adapter_character_source@V?$stream_input_adapter@D@__crt_stdio_input@@@__crt_strtox@@_K@__crt_strtox@@YA?AW4floating_point_parse_result@1@AEADAEAV?$input_adapter_character_source@V?$stream_input_adapter@D@__crt_stdio_input@@@1@_K@Z@4QBDB 0000000180013e58     libucrt:input.obj
 0001:00012e60       ?uppercase@?1???$parse_floating_point_possible_nan@DV?$input_adapter_character_source@V?$stream_input_adapter@D@__crt_stdio_input@@@__crt_strtox@@_K@__crt_strtox@@YA?AW4floating_point_parse_result@1@AEADAEAV?$input_adapter_character_source@V?$stream_input_adapter@D@__crt_stdio_input@@@1@_K@Z@4QBDB 0000000180013e60     libucrt:input.obj
 0001:00012e64       ?lowercase@?1???$parse_floating_point_possible_nan@DV?$input_adapter_character_source@V?$stream_input_adapter@D@__crt_stdio_input@@@__crt_strtox@@_K@__crt_strtox@@YA?AW4floating_point_parse_result@1@AEADAEAV?$input_adapter_character_source@V?$stream_input_adapter@D@__crt_stdio_input@@@1@_K@Z@4QBDB 0000000180013e64     libucrt:input.obj
 0001:00012e68       ?uppercase@?1???$parse_floating_point_possible_nan_is_snan@DV?$input_adapter_character_source@V?$stream_input_adapter@D@__crt_stdio_input@@@__crt_strtox@@@__crt_strtox@@YA_NAEADAEAV?$input_adapter_character_source@V?$stream_input_adapter@D@__crt_stdio_input@@@1@@Z@4QBDB 0000000180013e68     libucrt:input.obj
 0001:00012e70       ?lowercase@?1???$parse_floating_point_possible_nan_is_snan@DV?$input_adapter_character_source@V?$stream_input_adapter@D@__crt_stdio_input@@@__crt_strtox@@@__crt_strtox@@YA_NAEADAEAV?$input_adapter_character_source@V?$stream_input_adapter@D@__crt_stdio_input@@@1@@Z@4QBDB 0000000180013e70     libucrt:input.obj
 0001:00012e78       ?uppercase@?1???$parse_floating_point_possible_nan_is_ind@DV?$input_adapter_character_source@V?$stream_input_adapter@D@__crt_stdio_input@@@__crt_strtox@@@__crt_strtox@@YA_NAEADAEAV?$input_adapter_character_source@V?$stream_input_adapter@D@__crt_stdio_input@@@1@@Z@4QBDB 0000000180013e78     libucrt:input.obj
 0001:00012e7c       ?lowercase@?1???$parse_floating_point_possible_nan_is_ind@DV?$input_adapter_character_source@V?$stream_input_adapter@D@__crt_stdio_input@@@__crt_strtox@@@__crt_strtox@@YA_NAEADAEAV?$input_adapter_character_source@V?$stream_input_adapter@D@__crt_stdio_input@@@1@@Z@4QBDB 0000000180013e7c     libucrt:input.obj
 0001:00012eb0       __acrt_exception_action_table 0000000180013eb0     libucrt:exception_filter.obj
 0001:00012f70       __acrt_signal_action_table_count 0000000180013f70     libucrt:exception_filter.obj
 0001:00012f78       __acrt_signal_action_first_fpe_index 0000000180013f78     libucrt:exception_filter.obj
 0001:00012f80       __acrt_signal_action_fpe_count 0000000180013f80     libucrt:exception_filter.obj
 0001:00012f88       ??_C@_1BI@BGOHAHKC@?$AAm?$AAs?$AAc?$AAo?$AAr?$AAe?$AAe?$AA?4?$AAd?$AAl?$AAl?$AA?$AA@ 0000000180013f88     libucrt:exit.obj
 0001:00012fa0       ??_C@_0P@MIGLKIOC@CorExitProcess?$AA@ 0000000180013fa0     libucrt:exit.obj
 0001:000130b0       ??_C@_03OEIAHPBN@INF?$AA@  00000001800140b0     libucrt:cvt.obj
 0001:000130b4       ??_C@_03OJHLLCGB@inf?$AA@  00000001800140b4     libucrt:cvt.obj
 0001:000130b8       ??_C@_03LKNCIKJB@NAN?$AA@  00000001800140b8     libucrt:cvt.obj
 0001:000130bc       ??_C@_03LHCJEHON@nan?$AA@  00000001800140bc     libucrt:cvt.obj
 0001:000130c0       ??_C@_09OFJJIMPC@NAN?$CISNAN?$CJ?$AA@ 00000001800140c0     libucrt:cvt.obj
 0001:000130d0       ??_C@_09IPFBKMDL@nan?$CIsnan?$CJ?$AA@ 00000001800140d0     libucrt:cvt.obj
 0001:000130e0       ??_C@_08IKHNHAJ@NAN?$CIIND?$CJ?$AA@ 00000001800140e0     libucrt:cvt.obj
 0001:000130f0       ??_C@_08OFCDMILK@nan?$CIind?$CJ?$AA@ 00000001800140f0     libucrt:cvt.obj
 0001:000130fc       ??_C@_05KLBDPFGC@e?$CL000?$AA@ 00000001800140fc     libucrt:cvt.obj
 0001:00013110       __lc_time_c                0000000180014110     libucrt:nlsdata.obj
 0001:000133d0       ??_C@_03KOEHGMDN@Sun?$AA@  00000001800143d0     libucrt:nlsdata.obj
 0001:000133d4       ??_C@_03PDAGKDH@Mon?$AA@   00000001800143d4     libucrt:nlsdata.obj
 0001:000133d8       ??_C@_03NAGEINEP@Tue?$AA@  00000001800143d8     libucrt:nlsdata.obj
 0001:000133dc       ??_C@_03MHOMLAJA@Wed?$AA@  00000001800143dc     libucrt:nlsdata.obj
 0001:000133e0       ??_C@_03IOFIKPDN@Thu?$AA@  00000001800143e0     libucrt:nlsdata.obj
 0001:000133e4       ??_C@_03IDIOELNC@Fri?$AA@  00000001800143e4     libucrt:nlsdata.obj
 0001:000133e8       ??_C@_03FEFJNEK@Sat?$AA@   00000001800143e8     libucrt:nlsdata.obj
 0001:000133ec       ??_C@_06OOPIFAJ@Sunday?$AA@ 00000001800143ec     libucrt:nlsdata.obj
 0001:000133f4       ??_C@_06JLEDEDGH@Monday?$AA@ 00000001800143f4     libucrt:nlsdata.obj
 0001:00013400       ??_C@_07BAAGCFCM@Tuesday?$AA@ 0000000180014400     libucrt:nlsdata.obj
 0001:00013408       ??_C@_09DLIGFAKA@Wednesday?$AA@ 0000000180014408     libucrt:nlsdata.obj
 0001:00013418       ??_C@_08HACCIKIA@Thursday?$AA@ 0000000180014418     libucrt:nlsdata.obj
 0001:00013424       ??_C@_06JECMNKMI@Friday?$AA@ 0000000180014424     libucrt:nlsdata.obj
 0001:00013430       ??_C@_08INBOOONO@Saturday?$AA@ 0000000180014430     libucrt:nlsdata.obj
 0001:0001343c       ??_C@_03JIHJHPIE@Jan?$AA@  000000018001443c     libucrt:nlsdata.obj
 0001:00013440       ??_C@_03HJBDCHOM@Feb?$AA@  0000000180014440     libucrt:nlsdata.obj
 0001:00013444       ??_C@_03ODNJBKGA@Mar?$AA@  0000000180014444     libucrt:nlsdata.obj
 0001:00013448       ??_C@_03LEOLGMJP@Apr?$AA@  0000000180014448     libucrt:nlsdata.obj
 0001:0001344c       ??_C@_03CNMDKL@May?$AA@    000000018001444c     libucrt:nlsdata.obj
 0001:00013450       ??_C@_03IDFGHECI@Jun?$AA@  0000000180014450     libucrt:nlsdata.obj
 0001:00013454       ??_C@_03LBGABGKK@Jul?$AA@  0000000180014454     libucrt:nlsdata.obj
 0001:00013458       ??_C@_03IFJFEIGA@Aug?$AA@  0000000180014458     libucrt:nlsdata.obj
 0001:0001345c       ??_C@_03GGCAPAJC@Sep?$AA@  000000018001445c     libucrt:nlsdata.obj
 0001:00013460       ??_C@_03BMAOKBAD@Oct?$AA@  0000000180014460     libucrt:nlsdata.obj
 0001:00013464       ??_C@_03JPJOFNIA@Nov?$AA@  0000000180014464     libucrt:nlsdata.obj
 0001:00013468       ??_C@_03MKABNOCG@Dec?$AA@  0000000180014468     libucrt:nlsdata.obj
 0001:00013470       ??_C@_07CGJPFGJA@January?$AA@ 0000000180014470     libucrt:nlsdata.obj
 0001:00013478       ??_C@_08GNJGEPFN@February?$AA@ 0000000180014478     libucrt:nlsdata.obj
 0001:00013484       ??_C@_05HPCKOFNC@March?$AA@ 0000000180014484     libucrt:nlsdata.obj
 0001:0001348c       ??_C@_05DMJDNLEJ@April?$AA@ 000000018001448c     libucrt:nlsdata.obj
 0001:00013494       ??_C@_04CNLMGBGM@June?$AA@ 0000000180014494     libucrt:nlsdata.obj
 0001:0001349c       ??_C@_04MIEPOIFP@July?$AA@ 000000018001449c     libucrt:nlsdata.obj
 0001:000134a4       ??_C@_06LBBHFDDG@August?$AA@ 00000001800144a4     libucrt:nlsdata.obj
 0001:000134b0       ??_C@_09BHHEALKD@September?$AA@ 00000001800144b0     libucrt:nlsdata.obj
 0001:000134c0       ??_C@_07JJNFCEND@October?$AA@ 00000001800144c0     libucrt:nlsdata.obj
 0001:000134c8       ??_C@_08HCHEGEOA@November?$AA@ 00000001800144c8     libucrt:nlsdata.obj
 0001:000134d8       ??_C@_08EDHMEBNP@December?$AA@ 00000001800144d8     libucrt:nlsdata.obj
 0001:000134e4       ??_C@_02DEDBPAFC@AM?$AA@   00000001800144e4     libucrt:nlsdata.obj
 0001:000134e8       ??_C@_02CJNFDJBF@PM?$AA@   00000001800144e8     libucrt:nlsdata.obj
 0001:000134f0       ??_C@_08BPBNCDIB@MM?1dd?1yy?$AA@ 00000001800144f0     libucrt:nlsdata.obj
 0001:00013500       ??_C@_0BE@CKGJFCPC@dddd?0?5MMMM?5dd?0?5yyyy?$AA@ 0000000180014500     libucrt:nlsdata.obj
 0001:00013518       ??_C@_08JCCMCCIL@HH?3mm?3ss?$AA@ 0000000180014518     libucrt:nlsdata.obj
 0001:00013528       ??_C@_17MBGCMIPB@?$AAS?$AAu?$AAn?$AA?$AA@ 0000000180014528     libucrt:nlsdata.obj
 0001:00013530       ??_C@_17KBOMKBF@?$AAM?$AAo?$AAn?$AA?$AA@ 0000000180014530     libucrt:nlsdata.obj
 0001:00013538       ??_C@_17BMKGEGOJ@?$AAT?$AAu?$AAe?$AA?$AA@ 0000000180014538     libucrt:nlsdata.obj
 0001:00013540       ??_C@_17CJEDCEPE@?$AAW?$AAe?$AAd?$AA?$AA@ 0000000180014540     libucrt:nlsdata.obj
 0001:00013548       ??_C@_17PDPHAADD@?$AAT?$AAh?$AAu?$AA?$AA@ 0000000180014548     libucrt:nlsdata.obj
 0001:00013550       ??_C@_17HFOLPPLP@?$AAF?$AAr?$AAi?$AA?$AA@ 0000000180014550     libucrt:nlsdata.obj
 0001:00013558       ??_C@_17GGIBDPIH@?$AAS?$AAa?$AAt?$AA?$AA@ 0000000180014558     libucrt:nlsdata.obj
 0001:00013560       ??_C@_1O@IHNHDHPB@?$AAS?$AAu?$AAn?$AAd?$AAa?$AAy?$AA?$AA@ 0000000180014560     libucrt:nlsdata.obj
 0001:00013570       ??_C@_1O@MMNBFLIA@?$AAM?$AAo?$AAn?$AAd?$AAa?$AAy?$AA?$AA@ 0000000180014570     libucrt:nlsdata.obj
 0001:00013580       ??_C@_1BA@ENFBFFEK@?$AAT?$AAu?$AAe?$AAs?$AAd?$AAa?$AAy?$AA?$AA@ 0000000180014580     libucrt:nlsdata.obj
 0001:00013590       ??_C@_1BE@EBOGMDOH@?$AAW?$AAe?$AAd?$AAn?$AAe?$AAs?$AAd?$AAa?$AAy?$AA?$AA@ 0000000180014590     libucrt:nlsdata.obj
 0001:000135a8       ??_C@_1BC@HHMNLIHE@?$AAT?$AAh?$AAu?$AAr?$AAs?$AAd?$AAa?$AAy?$AA?$AA@ 00000001800145a8     libucrt:nlsdata.obj
 0001:000135c0       ??_C@_1O@PDICJHAG@?$AAF?$AAr?$AAi?$AAd?$AAa?$AAy?$AA?$AA@ 00000001800145c0     libucrt:nlsdata.obj
 0001:000135d0       ??_C@_1BC@ENMNNPAJ@?$AAS?$AAa?$AAt?$AAu?$AAr?$AAd?$AAa?$AAy?$AA?$AA@ 00000001800145d0     libucrt:nlsdata.obj
 0001:000135e8       ??_C@_17DKNBKCHM@?$AAJ?$AAa?$AAn?$AA?$AA@ 00000001800145e8     libucrt:nlsdata.obj
 0001:000135f0       ??_C@_17LMDJEKJN@?$AAF?$AAe?$AAb?$AA?$AA@ 00000001800145f0     libucrt:nlsdata.obj
 0001:000135f8       ??_C@_17CKNLEDEC@?$AAM?$AAa?$AAr?$AA?$AA@ 00000001800145f8     libucrt:nlsdata.obj
 0001:00013600       ??_C@_17LFPOIHDD@?$AAA?$AAp?$AAr?$AA?$AA@ 0000000180014600     libucrt:nlsdata.obj
 0001:00013608       ??_C@_17PNNKMEED@?$AAM?$AAa?$AAy?$AA?$AA@ 0000000180014608     libucrt:nlsdata.obj
 0001:00013610       ??_C@_17KCJGOCPB@?$AAJ?$AAu?$AAn?$AA?$AA@ 0000000180014610     libucrt:nlsdata.obj
 0001:00013618       ??_C@_17IJPCKHK@?$AAJ?$AAu?$AAl?$AA?$AA@ 0000000180014618     libucrt:nlsdata.obj
 0001:00013620       ??_C@_17ICPELBCN@?$AAA?$AAu?$AAg?$AA?$AA@ 0000000180014620     libucrt:nlsdata.obj
 0001:00013628       ??_C@_17HCHCOKMG@?$AAS?$AAe?$AAp?$AA?$AA@ 0000000180014628     libucrt:nlsdata.obj
 0001:00013630       ??_C@_17FNLKOI@?$AAO?$AAc?$AAt?$AA?$AA@ 0000000180014630     libucrt:nlsdata.obj
 0001:00013638       ??_C@_17BBDMLCIG@?$AAN?$AAo?$AAv?$AA?$AA@ 0000000180014638     libucrt:nlsdata.obj
 0001:00013640       ??_C@_17EGKACKIF@?$AAD?$AAe?$AAc?$AA?$AA@ 0000000180014640     libucrt:nlsdata.obj
 0001:00013648       ??_C@_1BA@EFMEIEBA@?$AAJ?$AAa?$AAn?$AAu?$AAa?$AAr?$AAy?$AA?$AA@ 0000000180014648     libucrt:nlsdata.obj
 0001:00013658       ??_C@_1BC@JGDDFFAM@?$AAF?$AAe?$AAb?$AAr?$AAu?$AAa?$AAr?$AAy?$AA?$AA@ 0000000180014658     libucrt:nlsdata.obj
 0001:00013670       ??_C@_1M@IKEENEDF@?$AAM?$AAa?$AAr?$AAc?$AAh?$AA?$AA@ 0000000180014670     libucrt:nlsdata.obj
 0001:00013680       ??_C@_1M@GJNLMHFD@?$AAA?$AAp?$AAr?$AAi?$AAl?$AA?$AA@ 0000000180014680     libucrt:nlsdata.obj
 0001:00013690       ??_C@_19EPFLPGAP@?$AAJ?$AAu?$AAn?$AAe?$AA?$AA@ 0000000180014690     libucrt:nlsdata.obj
 0001:000136a0       ??_C@_19BIFMLPCD@?$AAJ?$AAu?$AAl?$AAy?$AA?$AA@ 00000001800146a0     libucrt:nlsdata.obj
 0001:000136b0       ??_C@_1O@PAHLKOAC@?$AAA?$AAu?$AAg?$AAu?$AAs?$AAt?$AA?$AA@ 00000001800146b0     libucrt:nlsdata.obj
 0001:000136c0       ??_C@_1BE@DKAAMBJL@?$AAS?$AAe?$AAp?$AAt?$AAe?$AAm?$AAb?$AAe?$AAr?$AA?$AA@ 00000001800146c0     libucrt:nlsdata.obj
 0001:000136d8       ??_C@_1BA@EPANDLNG@?$AAO?$AAc?$AAt?$AAo?$AAb?$AAe?$AAr?$AA?$AA@ 00000001800146d8     libucrt:nlsdata.obj
 0001:000136e8       ??_C@_1BC@BGLIFPF@?$AAN?$AAo?$AAv?$AAe?$AAm?$AAb?$AAe?$AAr?$AA?$AA@ 00000001800146e8     libucrt:nlsdata.obj
 0001:00013700       ??_C@_1BC@FEMKIFH@?$AAD?$AAe?$AAc?$AAe?$AAm?$AAb?$AAe?$AAr?$AA?$AA@ 0000000180014700     libucrt:nlsdata.obj
 0001:00013714       ??_C@_15ODEHAHHF@?$AAA?$AAM?$AA?$AA@ 0000000180014714     libucrt:nlsdata.obj
 0001:0001371c       ??_C@_15CLMNNGEL@?$AAP?$AAM?$AA?$AA@ 000000018001471c     libucrt:nlsdata.obj
 0001:00013728       ??_C@_1BC@IEBCMHCM@?$AAM?$AAM?$AA?1?$AAd?$AAd?$AA?1?$AAy?$AAy?$AA?$AA@ 0000000180014728     libucrt:nlsdata.obj
 0001:00013740       ??_C@_1CI@KNAKOEBC@?$AAd?$AAd?$AAd?$AAd?$AA?0?$AA?5?$AAM?$AAM?$AAM?$AAM?$AA?5?$AAd?$AAd?$AA?0?$AA?5?$AAy?$AAy?$AAy?$AAy?$AA?$AA@ 0000000180014740     libucrt:nlsdata.obj
 0001:00013768       ??_C@_1BC@GDGBMEMK@?$AAH?$AAH?$AA?3?$AAm?$AAm?$AA?3?$AAs?$AAs?$AA?$AA@ 0000000180014768     libucrt:nlsdata.obj
 0001:00013780       ??_C@_1M@BMHNFIME@?$AAe?$AAn?$AA?9?$AAU?$AAS?$AA?$AA@ 0000000180014780     libucrt:nlsdata.obj
 0001:0001378c       ?ccs@?1???$__acrt_stdio_parse_mode@_W@@YA?AU__acrt_stdio_stream_mode@@QEB_W@Z@4QB_WB 000000018001478c     libucrt:openfile.obj
 0001:00013798       ?utf8_encoding@?1???$__acrt_stdio_parse_mode@_W@@YA?AU__acrt_stdio_stream_mode@@QEB_W@Z@4QB_WB 0000000180014798     libucrt:openfile.obj
 0001:000137a8       ?utf16_encoding@?1???$__acrt_stdio_parse_mode@_W@@YA?AU__acrt_stdio_stream_mode@@QEB_W@Z@4QB_WB 00000001800147a8     libucrt:openfile.obj
 0001:000137b8       ?unicode_encoding@?1???$__acrt_stdio_parse_mode@_W@@YA?AU__acrt_stdio_stream_mode@@QEB_W@Z@4QB_WB 00000001800147b8     libucrt:openfile.obj
 0001:000137e0       _sys_errlist               00000001800147e0     libucrt:syserr.obj
 0001:00013940       ??_C@_08INEPGKHH@No?5error?$AA@ 0000000180014940     libucrt:syserr.obj
 0001:00013950       ??_C@_0BI@BJFCGOHL@Operation?5not?5permitted?$AA@ 0000000180014950     libucrt:syserr.obj
 0001:00013968       ??_C@_0BK@FMDHKPNF@No?5such?5file?5or?5directory?$AA@ 0000000180014968     libucrt:syserr.obj
 0001:00013988       ??_C@_0BA@FKIAIBGA@No?5such?5process?$AA@ 0000000180014988     libucrt:syserr.obj
 0001:00013998       ??_C@_0BK@FJBOAFDK@Interrupted?5function?5call?$AA@ 0000000180014998     libucrt:syserr.obj
 0001:000139b8       ??_C@_0BD@KKNFOBBD@Input?1output?5error?$AA@ 00000001800149b8     libucrt:syserr.obj
 0001:000139d0       ??_C@_0BK@DPKMCKJ@No?5such?5device?5or?5address?$AA@ 00000001800149d0     libucrt:syserr.obj
 0001:000139f0       ??_C@_0BC@MFFGCDFL@Arg?5list?5too?5long?$AA@ 00000001800149f0     libucrt:syserr.obj
 0001:00013a08       ??_C@_0BC@HKPNECK@Exec?5format?5error?$AA@ 0000000180014a08     libucrt:syserr.obj
 0001:00013a20       ??_C@_0BE@NFGDDCEF@Bad?5file?5descriptor?$AA@ 0000000180014a20     libucrt:syserr.obj
 0001:00013a38       ??_C@_0BD@LOHELEP@No?5child?5processes?$AA@ 0000000180014a38     libucrt:syserr.obj
 0001:00013a50       ??_C@_0CB@EPFKGNAK@Resource?5temporarily?5unavailable@ 0000000180014a50     libucrt:syserr.obj
 0001:00013a78       ??_C@_0BB@IMDKMPFB@Not?5enough?5space?$AA@ 0000000180014a78     libucrt:syserr.obj
 0001:00013a90       ??_C@_0BC@HFNFNKAI@Permission?5denied?$AA@ 0000000180014a90     libucrt:syserr.obj
 0001:00013aa8       ??_C@_0M@LOEHLCJD@Bad?5address?$AA@ 0000000180014aa8     libucrt:syserr.obj
 0001:00013ab8       ??_C@_0O@NIPGCINC@Unknown?5error?$AA@ 0000000180014ab8     libucrt:syserr.obj
 0001:00013ac8       ??_C@_0BA@BIBLIOEK@Resource?5device?$AA@ 0000000180014ac8     libucrt:syserr.obj
 0001:00013ad8       ??_C@_0M@NAAJNNGH@File?5exists?$AA@ 0000000180014ad8     libucrt:syserr.obj
 0001:00013ae8       ??_C@_0O@OAMDNOCP@Improper?5link?$AA@ 0000000180014ae8     libucrt:syserr.obj
 0001:00013af8       ??_C@_0P@NLEIANHE@No?5such?5device?$AA@ 0000000180014af8     libucrt:syserr.obj
 0001:00013b08       ??_C@_0BA@CJBACOOL@Not?5a?5directory?$AA@ 0000000180014b08     libucrt:syserr.obj
 0001:00013b18       ??_C@_0P@NDHGCGKE@Is?5a?5directory?$AA@ 0000000180014b18     libucrt:syserr.obj
 0001:00013b28       ??_C@_0BB@HMGGCEBG@Invalid?5argument?$AA@ 0000000180014b28     libucrt:syserr.obj
 0001:00013b40       ??_C@_0BO@IIFBODJE@Too?5many?5open?5files?5in?5system?$AA@ 0000000180014b40     libucrt:syserr.obj
 0001:00013b60       ??_C@_0BE@INBJMKGG@Too?5many?5open?5files?$AA@ 0000000180014b60     libucrt:syserr.obj
 0001:00013b78       ??_C@_0CE@ONOKNLPF@Inappropriate?5I?1O?5control?5operat@ 0000000180014b78     libucrt:syserr.obj
 0001:00013ba0       ??_C@_0P@LFMMIPAE@File?5too?5large?$AA@ 0000000180014ba0     libucrt:syserr.obj
 0001:00013bb0       ??_C@_0BI@FEALHKLD@No?5space?5left?5on?5device?$AA@ 0000000180014bb0     libucrt:syserr.obj
 0001:00013bc8       ??_C@_0N@FEHLOILP@Invalid?5seek?$AA@ 0000000180014bc8     libucrt:syserr.obj
 0001:00013bd8       ??_C@_0BG@DDBFNKBH@Read?9only?5file?5system?$AA@ 0000000180014bd8     libucrt:syserr.obj
 0001:00013bf0       ??_C@_0P@PKCJJLLM@Too?5many?5links?$AA@ 0000000180014bf0     libucrt:syserr.obj
 0001:00013c00       ??_C@_0M@LHEPIIOM@Broken?5pipe?$AA@ 0000000180014c00     libucrt:syserr.obj
 0001:00013c10       ??_C@_0N@MMJPGLJK@Domain?5error?$AA@ 0000000180014c10     libucrt:syserr.obj
 0001:00013c20       ??_C@_0BB@FCBJFCAJ@Result?5too?5large?$AA@ 0000000180014c20     libucrt:syserr.obj
 0001:00013c38       ??_C@_0BK@JAEBMJJM@Resource?5deadlock?5avoided?$AA@ 0000000180014c38     libucrt:syserr.obj
 0001:00013c58       ??_C@_0BC@BEDIHIDK@Filename?5too?5long?$AA@ 0000000180014c58     libucrt:syserr.obj
 0001:00013c70       ??_C@_0BD@CLHBCGPB@No?5locks?5available?$AA@ 0000000180014c70     libucrt:syserr.obj
 0001:00013c88       ??_C@_0BJ@IHEHINLI@Function?5not?5implemented?$AA@ 0000000180014c88     libucrt:syserr.obj
 0001:00013ca8       ??_C@_0BE@ICMCHPHH@Directory?5not?5empty?$AA@ 0000000180014ca8     libucrt:syserr.obj
 0001:00013cc0       ??_C@_0BG@KLEAJEFJ@Illegal?5byte?5sequence?$AA@ 0000000180014cc0     libucrt:syserr.obj
 0001:00013cd8       _sys_nerr                  0000000180014cd8     libucrt:syserr.obj
 0001:00013d80       ??_C@_1EA@JGEFHKEI@?$AAa?$AAp?$AAi?$AA?9?$AAm?$AAs?$AA?9?$AAw?$AAi?$AAn?$AA?9?$AAc?$AAo?$AAr?$AAe?$AA?9?$AAd?$AAa?$AAt?$AAe?$AAt?$AAi?$AAm?$AAe?$AA?9?$AAl?$AA1?$AA?9?$AA1?$AA?9?$AA1?$AA?$AA@ 0000000180014d80     libucrt:winapi_thunks.obj
 0001:00013dc0       ??_C@_1DM@KHCHBNEB@?$AAa?$AAp?$AAi?$AA?9?$AAm?$AAs?$AA?9?$AAw?$AAi?$AAn?$AA?9?$AAc?$AAo?$AAr?$AAe?$AA?9?$AAf?$AAi?$AAb?$AAe?$AAr?$AAs?$AA?9?$AAl?$AA1?$AA?9?$AA1?$AA?9?$AA1?$AA?$AA@ 0000000180014dc0     libucrt:winapi_thunks.obj
 0001:00013e00       ??_C@_1DI@IJCEHOCB@?$AAa?$AAp?$AAi?$AA?9?$AAm?$AAs?$AA?9?$AAw?$AAi?$AAn?$AA?9?$AAc?$AAo?$AAr?$AAe?$AA?9?$AAf?$AAi?$AAl?$AAe?$AA?9?$AAl?$AA1?$AA?9?$AA2?$AA?9?$AA2?$AA?$AA@ 0000000180014e00     libucrt:winapi_thunks.obj
 0001:00013e40       ??_C@_1EI@MPIAOHOC@?$AAa?$AAp?$AAi?$AA?9?$AAm?$AAs?$AA?9?$AAw?$AAi?$AAn?$AA?9?$AAc?$AAo?$AAr?$AAe?$AA?9?$AAl?$AAo?$AAc?$AAa?$AAl?$AAi?$AAz?$AAa?$AAt?$AAi?$AAo?$AAn?$AA?9?$AAl?$AA1?$AA?9@ 0000000180014e40     libucrt:winapi_thunks.obj
 0001:00013e90       ??_C@_1FK@FPHCKFIE@?$AAa?$AAp?$AAi?$AA?9?$AAm?$AAs?$AA?9?$AAw?$AAi?$AAn?$AA?9?$AAc?$AAo?$AAr?$AAe?$AA?9?$AAl?$AAo?$AAc?$AAa?$AAl?$AAi?$AAz?$AAa?$AAt?$AAi?$AAo?$AAn?$AA?9?$AAo?$AAb?$AAs@ 0000000180014e90     libucrt:winapi_thunks.obj
 0001:00013ef0       ??_C@_1EM@DILCGIIO@?$AAa?$AAp?$AAi?$AA?9?$AAm?$AAs?$AA?9?$AAw?$AAi?$AAn?$AA?9?$AAc?$AAo?$AAr?$AAe?$AA?9?$AAp?$AAr?$AAo?$AAc?$AAe?$AAs?$AAs?$AAt?$AAh?$AAr?$AAe?$AAa?$AAd?$AAs?$AA?9?$AAl@ 0000000180014ef0     libucrt:winapi_thunks.obj
 0001:00013f40       ??_C@_1DM@LNCGDDPN@?$AAa?$AAp?$AAi?$AA?9?$AAm?$AAs?$AA?9?$AAw?$AAi?$AAn?$AA?9?$AAc?$AAo?$AAr?$AAe?$AA?9?$AAs?$AAt?$AAr?$AAi?$AAn?$AAg?$AA?9?$AAl?$AA1?$AA?9?$AA1?$AA?9?$AA0?$AA?$AA@ 0000000180014f40     libucrt:winapi_thunks.obj
 0001:00013f80       ??_C@_1DK@LPPGFMPP@?$AAa?$AAp?$AAi?$AA?9?$AAm?$AAs?$AA?9?$AAw?$AAi?$AAn?$AA?9?$AAc?$AAo?$AAr?$AAe?$AA?9?$AAs?$AAy?$AAn?$AAc?$AAh?$AA?9?$AAl?$AA1?$AA?9?$AA2?$AA?9?$AA0?$AA?$AA@ 0000000180014f80     libucrt:winapi_thunks.obj
 0001:00013fc0       ??_C@_1DO@FPAPJEMD@?$AAa?$AAp?$AAi?$AA?9?$AAm?$AAs?$AA?9?$AAw?$AAi?$AAn?$AA?9?$AAc?$AAo?$AAr?$AAe?$AA?9?$AAs?$AAy?$AAs?$AAi?$AAn?$AAf?$AAo?$AA?9?$AAl?$AA1?$AA?9?$AA2?$AA?9?$AA1?$AA?$AA@ 0000000180014fc0     libucrt:winapi_thunks.obj
 0001:00014000       ??_C@_1DK@NDHNAHIO@?$AAa?$AAp?$AAi?$AA?9?$AAm?$AAs?$AA?9?$AAw?$AAi?$AAn?$AA?9?$AAc?$AAo?$AAr?$AAe?$AA?9?$AAw?$AAi?$AAn?$AAr?$AAt?$AA?9?$AAl?$AA1?$AA?9?$AA1?$AA?9?$AA0?$AA?$AA@ 0000000180015000     libucrt:winapi_thunks.obj
 0001:00014040       ??_C@_1DM@KGHDGBCM@?$AAa?$AAp?$AAi?$AA?9?$AAm?$AAs?$AA?9?$AAw?$AAi?$AAn?$AA?9?$AAc?$AAo?$AAr?$AAe?$AA?9?$AAx?$AAs?$AAt?$AAa?$AAt?$AAe?$AA?9?$AAl?$AA2?$AA?9?$AA1?$AA?9?$AA0?$AA?$AA@ 0000000180015040     libucrt:winapi_thunks.obj
 0001:00014080       ??_C@_1EO@IJIOEFOH@?$AAa?$AAp?$AAi?$AA?9?$AAm?$AAs?$AA?9?$AAw?$AAi?$AAn?$AA?9?$AAr?$AAt?$AAc?$AAo?$AAr?$AAe?$AA?9?$AAn?$AAt?$AAu?$AAs?$AAe?$AAr?$AA?9?$AAw?$AAi?$AAn?$AAd?$AAo?$AAw?$AA?9@ 0000000180015080     libucrt:winapi_thunks.obj
 0001:000140d0       ??_C@_1FG@HHGEKANL@?$AAa?$AAp?$AAi?$AA?9?$AAm?$AAs?$AA?9?$AAw?$AAi?$AAn?$AA?9?$AAs?$AAe?$AAc?$AAu?$AAr?$AAi?$AAt?$AAy?$AA?9?$AAs?$AAy?$AAs?$AAt?$AAe?$AAm?$AAf?$AAu?$AAn?$AAc?$AAt?$AAi@ 00000001800150d0     libucrt:winapi_thunks.obj
 0001:00014130       ??_C@_1EG@DBIOJECG@?$AAe?$AAx?$AAt?$AA?9?$AAm?$AAs?$AA?9?$AAw?$AAi?$AAn?$AA?9?$AAn?$AAt?$AAu?$AAs?$AAe?$AAr?$AA?9?$AAd?$AAi?$AAa?$AAl?$AAo?$AAg?$AAb?$AAo?$AAx?$AA?9?$AAl?$AA1?$AA?9?$AA1@ 0000000180015130     libucrt:winapi_thunks.obj
 0001:00014180       ??_C@_1EO@FIHMJCLF@?$AAe?$AAx?$AAt?$AA?9?$AAm?$AAs?$AA?9?$AAw?$AAi?$AAn?$AA?9?$AAn?$AAt?$AAu?$AAs?$AAe?$AAr?$AA?9?$AAw?$AAi?$AAn?$AAd?$AAo?$AAw?$AAs?$AAt?$AAa?$AAt?$AAi?$AAo?$AAn?$AA?9@ 0000000180015180     libucrt:winapi_thunks.obj
 0001:000141d0       ??_C@_1BC@DNHGCMLG@?$AAa?$AAd?$AAv?$AAa?$AAp?$AAi?$AA3?$AA2?$AA?$AA@ 00000001800151d0     libucrt:winapi_thunks.obj
 0001:000141e8       ??_C@_1BC@GDMECMAK@?$AAk?$AAe?$AAr?$AAn?$AAe?$AAl?$AA3?$AA2?$AA?$AA@ 00000001800151e8     libucrt:winapi_thunks.obj
 0001:00014200       ??_C@_1M@OAIMIKLP@?$AAn?$AAt?$AAd?$AAl?$AAl?$AA?$AA@ 0000000180015200     libucrt:winapi_thunks.obj
 0001:00014210       ??_C@_1EG@DPGNFKGC@?$AAa?$AAp?$AAi?$AA?9?$AAm?$AAs?$AA?9?$AAw?$AAi?$AAn?$AA?9?$AAa?$AAp?$AAp?$AAm?$AAo?$AAd?$AAe?$AAl?$AA?9?$AAr?$AAu?$AAn?$AAt?$AAi?$AAm?$AAe?$AA?9?$AAl?$AA1?$AA?9?$AA1@ 0000000180015210     libucrt:winapi_thunks.obj
 0001:00014258       ??_C@_1O@BCCLBEOE@?$AAu?$AAs?$AAe?$AAr?$AA3?$AA2?$AA?$AA@ 0000000180015258     libucrt:winapi_thunks.obj
 0001:00014268       ??_C@_1BA@PFFKHIOG@?$AAa?$AAp?$AAi?$AA?9?$AAm?$AAs?$AA?9?$AA?$AA@ 0000000180015268     libucrt:winapi_thunks.obj
 0001:00014278       ??_C@_1BA@IAIFMGEF@?$AAe?$AAx?$AAt?$AA?9?$AAm?$AAs?$AA?9?$AA?$AA@ 0000000180015278     libucrt:winapi_thunks.obj
 0001:00014290       ??_C@_0BA@FHFNEAED@AreFileApisANSI?$AA@ 0000000180015290     libucrt:winapi_thunks.obj
 0001:000142a8       ??_C@_0BA@IHGNDAEB@CompareStringEx?$AA@ 00000001800152a8     libucrt:winapi_thunks.obj
 0001:000142c0       ??_C@_08KNHFBNJ@FlsAlloc?$AA@ 00000001800152c0     libucrt:winapi_thunks.obj
 0001:000142d8       ??_C@_07PEJMOBNF@FlsFree?$AA@ 00000001800152d8     libucrt:winapi_thunks.obj
 0001:000142e8       ??_C@_0M@GDNOONDI@FlsGetValue?$AA@ 00000001800152e8     libucrt:winapi_thunks.obj
 0001:00014300       ??_C@_0M@JCPCPOEF@FlsSetValue?$AA@ 0000000180015300     libucrt:winapi_thunks.obj
 0001:00014318       ??_C@_0BM@HCFOFFN@InitializeCriticalSectionEx?$AA@ 0000000180015318     libucrt:winapi_thunks.obj
 0001:00014340       ??_C@_0O@KKBNKAPF@LCMapStringEx?$AA@ 0000000180015340     libucrt:winapi_thunks.obj
 0001:00014358       ??_C@_0BB@HBDEELFH@LocaleNameToLCID?$AA@ 0000000180015358     libucrt:winapi_thunks.obj
 0001:00014370       ??_C@_0CF@OJOFEIGO@AppPolicyGetProcessTerminationMe@ 0000000180015370     libucrt:winapi_thunks.obj
 0001:000143a0       __newctype                 00000001800153a0     libucrt:ctype.obj
 0001:000146a0       __newclmap                 00000001800156a0     libucrt:ctype.obj
 0001:00014820       __newcumap                 0000000180015820     libucrt:ctype.obj
 0001:000149a0       _wctype                    00000001800159a0     libucrt:ctype.obj
 0001:00014bf8       ??_C@_1M@HPNHIDJI@?$AAj?$AAa?$AA?9?$AAJ?$AAP?$AA?$AA@ 0000000180015bf8     libucrt:mbctype.obj
 0001:00014c08       ??_C@_1M@BIBDDEMK@?$AAz?$AAh?$AA?9?$AAC?$AAN?$AA?$AA@ 0000000180015c08     libucrt:mbctype.obj
 0001:00014c18       ??_C@_1M@JLOOOEGK@?$AAk?$AAo?$AA?9?$AAK?$AAR?$AA?$AA@ 0000000180015c18     libucrt:mbctype.obj
 0001:00014c28       ??_C@_1M@CLNBBOPM@?$AAz?$AAh?$AA?9?$AAT?$AAW?$AA?$AA@ 0000000180015c28     libucrt:mbctype.obj
 0001:00014c34       ??_C@_00CNPNBAHC@?$AA@     0000000180015c34     libucrt:mbrtowc.obj
 0001:00014c38       ??_C@_01GBGANLPD@0?$AA@    0000000180015c38     libucrt:cfout.obj
 0001:00014c3c       ??_C@_05DNEBIAHO@1?$CDINF?$AA@ 0000000180015c3c     libucrt:cfout.obj
 0001:00014c44       ??_C@_06IMKFLFPG@1?$CDQNAN?$AA@ 0000000180015c44     libucrt:cfout.obj
 0001:00014c4c       ??_C@_06PGGFOGJG@1?$CDSNAN?$AA@ 0000000180015c4c     libucrt:cfout.obj
 0001:00014c54       ??_C@_05PHHOCPM@1?$CDIND?$AA@ 0000000180015c54     libucrt:cfout.obj
 0001:00014c5c       ??_C@_15PJPFLCCM@?$AAu?$AAk?$AA?$AA@ 0000000180015c5c     libucrt:get_qualified_locale.obj
 0001:00015ab0       ??_C@_15EMKDOKLE@?$AAa?$AAr?$AA?$AA@ 0000000180016ab0     libucrt:lcidtoname_downlevel.obj
 0001:00015ab8       ??_C@_15KNPADPLH@?$AAb?$AAg?$AA?$AA@ 0000000180016ab8     libucrt:lcidtoname_downlevel.obj
 0001:00015ac0       ??_C@_15EDMHLDMO@?$AAc?$AAa?$AA?$AA@ 0000000180016ac0     libucrt:lcidtoname_downlevel.obj
 0001:00015ac8       ??_C@_1O@BPEAJADD@?$AAz?$AAh?$AA?9?$AAC?$AAH?$AAS?$AA?$AA@ 0000000180016ac8     libucrt:lcidtoname_downlevel.obj
 0001:00015ad8       ??_C@_15LJNHCMNK@?$AAc?$AAs?$AA?$AA@ 0000000180016ad8     libucrt:lcidtoname_downlevel.obj
 0001:00015ae0       ??_C@_15FOMCIDHG@?$AAd?$AAa?$AA?$AA@ 0000000180016ae0     libucrt:lcidtoname_downlevel.obj
 0001:00015ae8       ??_C@_15NBKABECB@?$AAd?$AAe?$AA?$AA@ 0000000180016ae8     libucrt:lcidtoname_downlevel.obj
 0001:00015af0       ??_C@_15GHPEIIAO@?$AAe?$AAl?$AA?$AA@ 0000000180016af0     libucrt:lcidtoname_downlevel.obj
 0001:00015af8       ??_C@_15MNPNEAIF@?$AAe?$AAn?$AA?$AA@ 0000000180016af8     libucrt:lcidtoname_downlevel.obj
 0001:00015b00       ??_C@_15GPIOMPMH@?$AAe?$AAs?$AA?$AA@ 0000000180016b00     libucrt:lcidtoname_downlevel.obj
 0001:00015b08       ??_C@_15NGLOAKJC@?$AAf?$AAi?$AA?$AA@ 0000000180016b08     libucrt:lcidtoname_downlevel.obj
 0001:00015b10       ??_C@_15FBKGNKAM@?$AAf?$AAr?$AA?$AA@ 0000000180016b10     libucrt:lcidtoname_downlevel.obj
 0001:00015b18       ??_C@_15KGGCNEFK@?$AAh?$AAe?$AA?$AA@ 0000000180016b18     libucrt:lcidtoname_downlevel.obj
 0001:00015b20       ??_C@_15PGHLIDMF@?$AAh?$AAu?$AA?$AA@ 0000000180016b20     libucrt:lcidtoname_downlevel.obj
 0001:00015b28       ??_C@_15BIEMAPLM@?$AAi?$AAs?$AA?$AA@ 0000000180016b28     libucrt:lcidtoname_downlevel.obj
 0001:00015b30       ??_C@_15IFJLDHAF@?$AAi?$AAt?$AA?$AA@ 0000000180016b30     libucrt:lcidtoname_downlevel.obj
 0001:00015b38       ??_C@_15GEMIOCAG@?$AAj?$AAa?$AA?$AA@ 0000000180016b38     libucrt:lcidtoname_downlevel.obj
 0001:00015b40       ??_C@_15EPELEGJA@?$AAk?$AAo?$AA?$AA@ 0000000180016b40     libucrt:lcidtoname_downlevel.obj
 0001:00015b48       ??_C@_15NDDHIMN@?$AAn?$AAl?$AA?$AA@ 0000000180016b48     libucrt:lcidtoname_downlevel.obj
 0001:00015b50       ??_C@_15BPIGNHCD@?$AAn?$AAo?$AA?$AA@ 0000000180016b50     libucrt:lcidtoname_downlevel.obj
 0001:00015b58       ??_C@_15DEOPBLCG@?$AAp?$AAl?$AA?$AA@ 0000000180016b58     libucrt:lcidtoname_downlevel.obj
 0001:00015b60       ??_C@_15KBECGEFG@?$AAp?$AAt?$AA?$AA@ 0000000180016b60     libucrt:lcidtoname_downlevel.obj
 0001:00015b68       ??_C@_15GLJCBFMD@?$AAr?$AAo?$AA?$AA@ 0000000180016b68     libucrt:lcidtoname_downlevel.obj
 0001:00015b70       ??_C@_15FEDGKCDI@?$AAr?$AAu?$AA?$AA@ 0000000180016b70     libucrt:lcidtoname_downlevel.obj
 0001:00015b78       ??_C@_15GLKMLLHM@?$AAh?$AAr?$AA?$AA@ 0000000180016b78     libucrt:lcidtoname_downlevel.obj
 0001:00015b80       ??_C@_15CPKMFBDB@?$AAs?$AAk?$AA?$AA@ 0000000180016b80     libucrt:lcidtoname_downlevel.obj
 0001:00015b88       ??_C@_15BAAIOGMK@?$AAs?$AAq?$AA?$AA@ 0000000180016b88     libucrt:lcidtoname_downlevel.obj
 0001:00015b90       ??_C@_15INNPNOHD@?$AAs?$AAv?$AA?$AA@ 0000000180016b90     libucrt:lcidtoname_downlevel.obj
 0001:00015b98       ??_C@_15CABMMOGH@?$AAt?$AAh?$AA?$AA@ 0000000180016b98     libucrt:lcidtoname_downlevel.obj
 0001:00015ba0       ??_C@_15BPLIHJJM@?$AAt?$AAr?$AA?$AA@ 0000000180016ba0     libucrt:lcidtoname_downlevel.obj
 0001:00015ba8       ??_C@_15NEOEKKDJ@?$AAu?$AAr?$AA?$AA@ 0000000180016ba8     libucrt:lcidtoname_downlevel.obj
 0001:00015bb0       ??_C@_15NFICGAJK@?$AAi?$AAd?$AA?$AA@ 0000000180016bb0     libucrt:lcidtoname_downlevel.obj
 0001:00015bb8       ??_C@_15HPJPHDM@?$AAb?$AAe?$AA?$AA@ 0000000180016bb8     libucrt:lcidtoname_downlevel.obj
 0001:00015bc0       ??_C@_15LCHLGJII@?$AAs?$AAl?$AA?$AA@ 0000000180016bc0     libucrt:lcidtoname_downlevel.obj
 0001:00015bc8       ??_C@_15PCFJPHHO@?$AAe?$AAt?$AA?$AA@ 0000000180016bc8     libucrt:lcidtoname_downlevel.obj
 0001:00015bd0       ??_C@_15HPFPGODN@?$AAl?$AAv?$AA?$AA@ 0000000180016bd0     libucrt:lcidtoname_downlevel.obj
 0001:00015bd8       ??_C@_15NFFGKGLG@?$AAl?$AAt?$AA?$AA@ 0000000180016bd8     libucrt:lcidtoname_downlevel.obj
 0001:00015be0       ??_C@_15BDAKCCHN@?$AAf?$AAa?$AA?$AA@ 0000000180016be0     libucrt:lcidtoname_downlevel.obj
 0001:00015be8       ??_C@_15NFGIAIAJ@?$AAv?$AAi?$AA?$AA@ 0000000180016be8     libucrt:lcidtoname_downlevel.obj
 0001:00015bf0       ??_C@_15LMKNDMHN@?$AAh?$AAy?$AA?$AA@ 0000000180016bf0     libucrt:lcidtoname_downlevel.obj
 0001:00015bf8       ??_C@_15IJBHMCFL@?$AAa?$AAz?$AA?$AA@ 0000000180016bf8     libucrt:lcidtoname_downlevel.obj
 0001:00015c00       ??_C@_15EKOFJABL@?$AAe?$AAu?$AA?$AA@ 0000000180016c00     libucrt:lcidtoname_downlevel.obj
 0001:00015c08       ??_C@_15BGHADCNK@?$AAm?$AAk?$AA?$AA@ 0000000180016c08     libucrt:lcidtoname_downlevel.obj
 0001:00015c10       ??_C@_15JDNICKHM@?$AAa?$AAf?$AA?$AA@ 0000000180016c10     libucrt:lcidtoname_downlevel.obj
 0001:00015c18       ??_C@_15KPJEDBKD@?$AAk?$AAa?$AA?$AA@ 0000000180016c18     libucrt:lcidtoname_downlevel.obj
 0001:00015c20       ??_C@_15PDNFFFEO@?$AAf?$AAo?$AA?$AA@ 0000000180016c20     libucrt:lcidtoname_downlevel.obj
 0001:00015c28       ??_C@_15OMLEGLOC@?$AAh?$AAi?$AA?$AA@ 0000000180016c28     libucrt:lcidtoname_downlevel.obj
 0001:00015c30       ??_C@_15IDNNENKK@?$AAm?$AAs?$AA?$AA@ 0000000180016c30     libucrt:lcidtoname_downlevel.obj
 0001:00015c38       ??_C@_15MACJNBMH@?$AAk?$AAk?$AA?$AA@ 0000000180016c38     libucrt:lcidtoname_downlevel.obj
 0001:00015c40       ??_C@_15DKDJEOND@?$AAk?$AAy?$AA?$AA@ 0000000180016c40     libucrt:lcidtoname_downlevel.obj
 0001:00015c48       ??_C@_15DFGDLJBG@?$AAs?$AAw?$AA?$AA@ 0000000180016c48     libucrt:lcidtoname_downlevel.obj
 0001:00015c50       ??_C@_15BBFAICNG@?$AAu?$AAz?$AA?$AA@ 0000000180016c50     libucrt:lcidtoname_downlevel.obj
 0001:00015c58       ??_C@_15DKNDCGEA@?$AAt?$AAt?$AA?$AA@ 0000000180016c58     libucrt:lcidtoname_downlevel.obj
 0001:00015c60       ??_C@_15MGIFMDPL@?$AAp?$AAa?$AA?$AA@ 0000000180016c60     libucrt:lcidtoname_downlevel.obj
 0001:00015c68       ??_C@_15HCNDBBA@?$AAg?$AAu?$AA?$AA@ 0000000180016c68     libucrt:lcidtoname_downlevel.obj
 0001:00015c70       ??_C@_15FNBEIBON@?$AAt?$AAa?$AA?$AA@ 0000000180016c70     libucrt:lcidtoname_downlevel.obj
 0001:00015c78       ??_C@_15NCHGBGLK@?$AAt?$AAe?$AA?$AA@ 0000000180016c78     libucrt:lcidtoname_downlevel.obj
 0001:00015c80       ??_C@_15PHPHCBPF@?$AAk?$AAn?$AA?$AA@ 0000000180016c80     libucrt:lcidtoname_downlevel.obj
 0001:00015c88       ??_C@_15DLGBCKMP@?$AAm?$AAr?$AA?$AA@ 0000000180016c88     libucrt:lcidtoname_downlevel.obj
 0001:00015c90       ??_C@_15EABBLBFF@?$AAs?$AAa?$AA?$AA@ 0000000180016c90     libucrt:lcidtoname_downlevel.obj
 0001:00015c98       ??_C@_15CBKOMCOI@?$AAm?$AAn?$AA?$AA@ 0000000180016c98     libucrt:lcidtoname_downlevel.obj
 0001:00015ca0       ??_C@_15CKDMCJAF@?$AAg?$AAl?$AA?$AA@ 0000000180016ca0     libucrt:lcidtoname_downlevel.obj
 0001:00015ca8       ??_C@_17CNJFBPG@?$AAk?$AAo?$AAk?$AA?$AA@ 0000000180016ca8     libucrt:lcidtoname_downlevel.obj
 0001:00015cb0       ??_C@_17FFBJICPL@?$AAs?$AAy?$AAr?$AA?$AA@ 0000000180016cb0     libucrt:lcidtoname_downlevel.obj
 0001:00015cb8       ??_C@_17KPNDCPAF@?$AAd?$AAi?$AAv?$AA?$AA@ 0000000180016cb8     libucrt:lcidtoname_downlevel.obj
 0001:00015cc0       ??_C@_11LOCGONAA@?$AA?$AA@ 0000000180016cc0     libucrt:lcidtoname_downlevel.obj
 0001:00015cc8       ??_C@_1M@OKAHONE@?$AAa?$AAr?$AA?9?$AAS?$AAA?$AA?$AA@ 0000000180016cc8     libucrt:lcidtoname_downlevel.obj
 0001:00015cd8       ??_C@_1M@FFFIGIGK@?$AAb?$AAg?$AA?9?$AAB?$AAG?$AA?$AA@ 0000000180016cd8     libucrt:lcidtoname_downlevel.obj
 0001:00015ce8       ??_C@_1M@BJNKEDC@?$AAc?$AAa?$AA?9?$AAE?$AAS?$AA?$AA@ 0000000180016ce8     libucrt:lcidtoname_downlevel.obj
 0001:00015cf8       ??_C@_1M@IJJHFJHA@?$AAc?$AAs?$AA?9?$AAC?$AAZ?$AA?$AA@ 0000000180016cf8     libucrt:lcidtoname_downlevel.obj
 0001:00015d08       ??_C@_1M@CLPEOBGI@?$AAd?$AAa?$AA?9?$AAD?$AAK?$AA?$AA@ 0000000180016d08     libucrt:lcidtoname_downlevel.obj
 0001:00015d18       ??_C@_1M@MCMADGCB@?$AAd?$AAe?$AA?9?$AAD?$AAE?$AA?$AA@ 0000000180016d18     libucrt:lcidtoname_downlevel.obj
 0001:00015d28       ??_C@_1M@OOCKEMAM@?$AAe?$AAl?$AA?9?$AAG?$AAR?$AA?$AA@ 0000000180016d28     libucrt:lcidtoname_downlevel.obj
 0001:00015d38       ??_C@_1M@DDNJFGID@?$AAf?$AAi?$AA?9?$AAF?$AAI?$AA?$AA@ 0000000180016d38     libucrt:lcidtoname_downlevel.obj
 0001:00015d48       ??_C@_1M@GLIPPMAC@?$AAf?$AAr?$AA?9?$AAF?$AAR?$AA?$AA@ 0000000180016d48     libucrt:lcidtoname_downlevel.obj
 0001:00015d58       ??_C@_1M@GFMCHPE@?$AAh?$AAe?$AA?9?$AAI?$AAL?$AA?$AA@ 0000000180016d58     libucrt:lcidtoname_downlevel.obj
 0001:00015d68       ??_C@_1M@MHLPGNKM@?$AAh?$AAu?$AA?9?$AAH?$AAU?$AA?$AA@ 0000000180016d68     libucrt:lcidtoname_downlevel.obj
 0001:00015d78       ??_C@_1M@LPDDNNPN@?$AAi?$AAs?$AA?9?$AAI?$AAS?$AA?$AA@ 0000000180016d78     libucrt:lcidtoname_downlevel.obj
 0001:00015d88       ??_C@_1M@MADIPODN@?$AAi?$AAt?$AA?9?$AAI?$AAT?$AA?$AA@ 0000000180016d88     libucrt:lcidtoname_downlevel.obj
 0001:00015d98       ??_C@_1M@IHBJJGG@?$AAn?$AAl?$AA?9?$AAN?$AAL?$AA?$AA@ 0000000180016d98     libucrt:lcidtoname_downlevel.obj
 0001:00015da8       ??_C@_1M@EANAGDL@?$AAn?$AAb?$AA?9?$AAN?$AAO?$AA?$AA@ 0000000180016da8     libucrt:lcidtoname_downlevel.obj
 0001:00015db8       ??_C@_1M@NEIEMEGP@?$AAp?$AAl?$AA?9?$AAP?$AAL?$AA?$AA@ 0000000180016db8     libucrt:lcidtoname_downlevel.obj
 0001:00015dc8       ??_C@_1M@BOCFIGEP@?$AAp?$AAt?$AA?9?$AAB?$AAR?$AA?$AA@ 0000000180016dc8     libucrt:lcidtoname_downlevel.obj
 0001:00015dd8       ??_C@_1M@IMPFOPBG@?$AAr?$AAo?$AA?9?$AAR?$AAO?$AA?$AA@ 0000000180016dd8     libucrt:lcidtoname_downlevel.obj
 0001:00015de8       ??_C@_1M@IDNNEJMM@?$AAr?$AAu?$AA?9?$AAR?$AAU?$AA?$AA@ 0000000180016de8     libucrt:lcidtoname_downlevel.obj
 0001:00015df8       ??_C@_1M@LILEEOGM@?$AAh?$AAr?$AA?9?$AAH?$AAR?$AA?$AA@ 0000000180016df8     libucrt:lcidtoname_downlevel.obj
 0001:00015e08       ??_C@_1M@FKIFEHPB@?$AAs?$AAk?$AA?9?$AAS?$AAK?$AA?$AA@ 0000000180016e08     libucrt:lcidtoname_downlevel.obj
 0001:00015e18       ??_C@_1M@LJMAMNPJ@?$AAs?$AAq?$AA?9?$AAA?$AAL?$AA?$AA@ 0000000180016e18     libucrt:lcidtoname_downlevel.obj
 0001:00015e28       ??_C@_1M@GIAKDKJK@?$AAs?$AAv?$AA?9?$AAS?$AAE?$AA?$AA@ 0000000180016e28     libucrt:lcidtoname_downlevel.obj
 0001:00015e38       ??_C@_1M@MKJKIKCL@?$AAt?$AAh?$AA?9?$AAT?$AAH?$AA?$AA@ 0000000180016e38     libucrt:lcidtoname_downlevel.obj
 0001:00015e48       ??_C@_1M@MFLCCMPB@?$AAt?$AAr?$AA?9?$AAT?$AAR?$AA?$AA@ 0000000180016e48     libucrt:lcidtoname_downlevel.obj
 0001:00015e58       ??_C@_1M@OIJHDKJN@?$AAu?$AAr?$AA?9?$AAP?$AAK?$AA?$AA@ 0000000180016e58     libucrt:lcidtoname_downlevel.obj
 0001:00015e68       ??_C@_1M@LHIPCIEK@?$AAi?$AAd?$AA?9?$AAI?$AAD?$AA?$AA@ 0000000180016e68     libucrt:lcidtoname_downlevel.obj
 0001:00015e78       ??_C@_1M@MFMOBGI@?$AAu?$AAk?$AA?9?$AAU?$AAA?$AA?$AA@ 0000000180016e78     libucrt:lcidtoname_downlevel.obj
 0001:00015e88       ??_C@_1M@OBGLJIPL@?$AAb?$AAe?$AA?9?$AAB?$AAY?$AA?$AA@ 0000000180016e88     libucrt:lcidtoname_downlevel.obj
 0001:00015e98       ??_C@_1M@BCFAJEAD@?$AAs?$AAl?$AA?9?$AAS?$AAI?$AA?$AA@ 0000000180016e98     libucrt:lcidtoname_downlevel.obj
 0001:00015ea8       ??_C@_1M@FKFFEDDN@?$AAe?$AAt?$AA?9?$AAE?$AAE?$AA?$AA@ 0000000180016ea8     libucrt:lcidtoname_downlevel.obj
 0001:00015eb8       ??_C@_1M@KGKKAACI@?$AAl?$AAv?$AA?9?$AAL?$AAV?$AA?$AA@ 0000000180016eb8     libucrt:lcidtoname_downlevel.obj
 0001:00015ec8       ??_C@_1M@IFGBIJO@?$AAl?$AAt?$AA?9?$AAL?$AAT?$AA?$AA@ 0000000180016ec8     libucrt:lcidtoname_downlevel.obj
 0001:00015ed8       ??_C@_1M@FGEAHEDM@?$AAf?$AAa?$AA?9?$AAI?$AAR?$AA?$AA@ 0000000180016ed8     libucrt:lcidtoname_downlevel.obj
 0001:00015ee8       ??_C@_1M@KBMAIBFN@?$AAv?$AAi?$AA?9?$AAV?$AAN?$AA?$AA@ 0000000180016ee8     libucrt:lcidtoname_downlevel.obj
 0001:00015ef8       ??_C@_1M@GPCBKDJK@?$AAh?$AAy?$AA?9?$AAA?$AAM?$AA?$AA@ 0000000180016ef8     libucrt:lcidtoname_downlevel.obj
 0001:00015f08       ??_C@_1BG@BECMDDJB@?$AAa?$AAz?$AA?9?$AAA?$AAZ?$AA?9?$AAL?$AAa?$AAt?$AAn?$AA?$AA@ 0000000180016f08     libucrt:lcidtoname_downlevel.obj
 0001:00015f20       ??_C@_1M@MAOFCAEA@?$AAe?$AAu?$AA?9?$AAE?$AAS?$AA?$AA@ 0000000180016f20     libucrt:lcidtoname_downlevel.obj
 0001:00015f30       ??_C@_1M@IGHABKPI@?$AAm?$AAk?$AA?9?$AAM?$AAK?$AA?$AA@ 0000000180016f30     libucrt:lcidtoname_downlevel.obj
 0001:00015f40       ??_C@_1M@IAIGNEJG@?$AAt?$AAn?$AA?9?$AAZ?$AAA?$AA?$AA@ 0000000180016f40     libucrt:lcidtoname_downlevel.obj
 0001:00015f50       ??_C@_1M@IIJCOJFA@?$AAx?$AAh?$AA?9?$AAZ?$AAA?$AA?$AA@ 0000000180016f50     libucrt:lcidtoname_downlevel.obj
 0001:00015f60       ??_C@_1M@LGPJHNJH@?$AAz?$AAu?$AA?9?$AAZ?$AAA?$AA?$AA@ 0000000180016f60     libucrt:lcidtoname_downlevel.obj
 0001:00015f70       ??_C@_1M@HOKAOIO@?$AAa?$AAf?$AA?9?$AAZ?$AAA?$AA?$AA@ 0000000180016f70     libucrt:lcidtoname_downlevel.obj
 0001:00015f80       ??_C@_1M@DPCLHLIE@?$AAk?$AAa?$AA?9?$AAG?$AAE?$AA?$AA@ 0000000180016f80     libucrt:lcidtoname_downlevel.obj
 0001:00015f90       ??_C@_1M@BLKMHJBI@?$AAf?$AAo?$AA?9?$AAF?$AAO?$AA?$AA@ 0000000180016f90     libucrt:lcidtoname_downlevel.obj
 0001:00015fa0       ??_C@_1M@LGGJAPPB@?$AAh?$AAi?$AA?9?$AAI?$AAN?$AA?$AA@ 0000000180016fa0     libucrt:lcidtoname_downlevel.obj
 0001:00015fb0       ??_C@_1M@FIKPIHFE@?$AAm?$AAt?$AA?9?$AAM?$AAT?$AA?$AA@ 0000000180016fb0     libucrt:lcidtoname_downlevel.obj
 0001:00015fc0       ??_C@_1M@HEGGPBFA@?$AAs?$AAe?$AA?9?$AAN?$AAO?$AA?$AA@ 0000000180016fc0     libucrt:lcidtoname_downlevel.obj
 0001:00015fd0       ??_C@_1M@EIBJEEPA@?$AAm?$AAs?$AA?9?$AAM?$AAY?$AA?$AA@ 0000000180016fd0     libucrt:lcidtoname_downlevel.obj
 0001:00015fe0       ??_C@_1M@FHLBGMPP@?$AAk?$AAk?$AA?9?$AAK?$AAZ?$AA?$AA@ 0000000180016fe0     libucrt:lcidtoname_downlevel.obj
 0001:00015ff0       ??_C@_1M@NGJJLCGI@?$AAk?$AAy?$AA?9?$AAK?$AAG?$AA?$AA@ 0000000180016ff0     libucrt:lcidtoname_downlevel.obj
 0001:00016000       ??_C@_1M@GIENNBFC@?$AAs?$AAw?$AA?9?$AAK?$AAE?$AA?$AA@ 0000000180017000     libucrt:lcidtoname_downlevel.obj
 0001:00016010       ??_C@_1BG@NDGMJIMJ@?$AAu?$AAz?$AA?9?$AAU?$AAZ?$AA?9?$AAL?$AAa?$AAt?$AAn?$AA?$AA@ 0000000180017010     libucrt:lcidtoname_downlevel.obj
 0001:00016028       ??_C@_1M@IDCCIHBC@?$AAt?$AAt?$AA?9?$AAR?$AAU?$AA?$AA@ 0000000180017028     libucrt:lcidtoname_downlevel.obj
 0001:00016038       ??_C@_1M@LOICPMOJ@?$AAb?$AAn?$AA?9?$AAI?$AAN?$AA?$AA@ 0000000180017038     libucrt:lcidtoname_downlevel.obj
 0001:00016048       ??_C@_1M@KPKKNEAH@?$AAp?$AAa?$AA?9?$AAI?$AAN?$AA?$AA@ 0000000180017048     libucrt:lcidtoname_downlevel.obj
 0001:00016058       ??_C@_1M@PJGPPBOG@?$AAg?$AAu?$AA?9?$AAI?$AAN?$AA?$AA@ 0000000180017058     libucrt:lcidtoname_downlevel.obj
 0001:00016068       ??_C@_1M@KMKMOPHI@?$AAt?$AAa?$AA?9?$AAI?$AAN?$AA?$AA@ 0000000180017068     libucrt:lcidtoname_downlevel.obj
 0001:00016078       ??_C@_1M@KFEHEPAC@?$AAt?$AAe?$AA?9?$AAI?$AAN?$AA?$AA@ 0000000180017078     libucrt:lcidtoname_downlevel.obj
 0001:00016088       ??_C@_1M@CDCLMGHI@?$AAk?$AAn?$AA?9?$AAI?$AAN?$AA?$AA@ 0000000180017088     libucrt:lcidtoname_downlevel.obj
 0001:00016098       ??_C@_1M@MIODLDKF@?$AAm?$AAl?$AA?9?$AAI?$AAN?$AA?$AA@ 0000000180017098     libucrt:lcidtoname_downlevel.obj
 0001:000160a8       ??_C@_1M@PBIEACPO@?$AAm?$AAr?$AA?9?$AAI?$AAN?$AA?$AA@ 00000001800170a8     libucrt:lcidtoname_downlevel.obj
 0001:000160b8       ??_C@_1M@NIDEAGPH@?$AAs?$AAa?$AA?9?$AAI?$AAN?$AA?$AA@ 00000001800170b8     libucrt:lcidtoname_downlevel.obj
 0001:000160c8       ??_C@_1M@FHIHCBIO@?$AAm?$AAn?$AA?9?$AAM?$AAN?$AA?$AA@ 00000001800170c8     libucrt:lcidtoname_downlevel.obj
 0001:000160d8       ??_C@_1M@JAIJPENP@?$AAc?$AAy?$AA?9?$AAG?$AAB?$AA?$AA@ 00000001800170d8     libucrt:lcidtoname_downlevel.obj
 0001:000160e8       ??_C@_1M@PHGFBEPN@?$AAg?$AAl?$AA?9?$AAE?$AAS?$AA?$AA@ 00000001800170e8     libucrt:lcidtoname_downlevel.obj
 0001:000160f8       ??_C@_1O@KPIPDNCP@?$AAk?$AAo?$AAk?$AA?9?$AAI?$AAN?$AA?$AA@ 00000001800170f8     libucrt:lcidtoname_downlevel.obj
 0001:00016108       ??_C@_1O@KNHJLDJA@?$AAs?$AAy?$AAr?$AA?9?$AAS?$AAY?$AA?$AA@ 0000000180017108     libucrt:lcidtoname_downlevel.obj
 0001:00016118       ??_C@_1O@MKEKBLAH@?$AAd?$AAi?$AAv?$AA?9?$AAM?$AAV?$AA?$AA@ 0000000180017118     libucrt:lcidtoname_downlevel.obj
 0001:00016128       ??_C@_1O@OHDCKDDF@?$AAq?$AAu?$AAz?$AA?9?$AAB?$AAO?$AA?$AA@ 0000000180017128     libucrt:lcidtoname_downlevel.obj
 0001:00016138       ??_C@_1M@LEPJNLFD@?$AAn?$AAs?$AA?9?$AAZ?$AAA?$AA?$AA@ 0000000180017138     libucrt:lcidtoname_downlevel.obj
 0001:00016148       ??_C@_1M@OMLEIIJB@?$AAm?$AAi?$AA?9?$AAN?$AAZ?$AA?$AA@ 0000000180017148     libucrt:lcidtoname_downlevel.obj
 0001:00016158       ??_C@_1M@PMPEAILG@?$AAa?$AAr?$AA?9?$AAI?$AAQ?$AA?$AA@ 0000000180017158     libucrt:lcidtoname_downlevel.obj
 0001:00016168       ??_C@_1M@CNKPNOEE@?$AAd?$AAe?$AA?9?$AAC?$AAH?$AA?$AA@ 0000000180017168     libucrt:lcidtoname_downlevel.obj
 0001:00016178       ??_C@_1M@LKMGMLKO@?$AAe?$AAn?$AA?9?$AAG?$AAB?$AA?$AA@ 0000000180017178     libucrt:lcidtoname_downlevel.obj
 0001:00016188       ??_C@_1M@PGKJFFGL@?$AAe?$AAs?$AA?9?$AAM?$AAX?$AA?$AA@ 0000000180017188     libucrt:lcidtoname_downlevel.obj
 0001:00016198       ??_C@_1M@DNNANBDC@?$AAf?$AAr?$AA?9?$AAB?$AAE?$AA?$AA@ 0000000180017198     libucrt:lcidtoname_downlevel.obj
 0001:000161a8       ??_C@_1M@HLGMDFHM@?$AAi?$AAt?$AA?9?$AAC?$AAH?$AA?$AA@ 00000001800171a8     libucrt:lcidtoname_downlevel.obj
 0001:000161b8       ??_C@_1M@CLLBGJH@?$AAn?$AAl?$AA?9?$AAB?$AAE?$AA?$AA@ 00000001800171b8     libucrt:lcidtoname_downlevel.obj
 0001:000161c8       ??_C@_1M@BODBOGLF@?$AAn?$AAn?$AA?9?$AAN?$AAO?$AA?$AA@ 00000001800171c8     libucrt:lcidtoname_downlevel.obj
 0001:000161d8       ??_C@_1M@HFFAHKAD@?$AAp?$AAt?$AA?9?$AAP?$AAT?$AA?$AA@ 00000001800171d8     libucrt:lcidtoname_downlevel.obj
 0001:000161e8       ??_C@_1BG@LNOAKHIE@?$AAs?$AAr?$AA?9?$AAS?$AAP?$AA?9?$AAL?$AAa?$AAt?$AAn?$AA?$AA@ 00000001800171e8     libucrt:lcidtoname_downlevel.obj
 0001:00016200       ??_C@_1M@HBMHBGAK@?$AAs?$AAv?$AA?9?$AAF?$AAI?$AA?$AA@ 0000000180017200     libucrt:lcidtoname_downlevel.obj
 0001:00016210       ??_C@_1BG@DGCJGJBE@?$AAa?$AAz?$AA?9?$AAA?$AAZ?$AA?9?$AAC?$AAy?$AAr?$AAl?$AA?$AA@ 0000000180017210     libucrt:lcidtoname_downlevel.obj
 0001:00016228       ??_C@_1M@KEJDAAHB@?$AAs?$AAe?$AA?9?$AAS?$AAE?$AA?$AA@ 0000000180017228     libucrt:lcidtoname_downlevel.obj
 0001:00016238       ??_C@_1M@HEIBJJAD@?$AAm?$AAs?$AA?9?$AAB?$AAN?$AA?$AA@ 0000000180017238     libucrt:lcidtoname_downlevel.obj
 0001:00016248       ??_C@_1BG@PBGJMCEM@?$AAu?$AAz?$AA?9?$AAU?$AAZ?$AA?9?$AAC?$AAy?$AAr?$AAl?$AA?$AA@ 0000000180017248     libucrt:lcidtoname_downlevel.obj
 0001:00016260       ??_C@_1O@LAOBCMDF@?$AAq?$AAu?$AAz?$AA?9?$AAE?$AAC?$AA?$AA@ 0000000180017260     libucrt:lcidtoname_downlevel.obj
 0001:00016270       ??_C@_1M@POEEMAIO@?$AAa?$AAr?$AA?9?$AAE?$AAG?$AA?$AA@ 0000000180017270     libucrt:lcidtoname_downlevel.obj
 0001:00016280       ??_C@_1M@EFAKDEDL@?$AAz?$AAh?$AA?9?$AAH?$AAK?$AA?$AA@ 0000000180017280     libucrt:lcidtoname_downlevel.obj
 0001:00016290       ??_C@_1M@HKKIJHGI@?$AAd?$AAe?$AA?9?$AAA?$AAT?$AA?$AA@ 0000000180017290     libucrt:lcidtoname_downlevel.obj
 0001:000162a0       ??_C@_1M@KBFBEHJF@?$AAe?$AAn?$AA?9?$AAA?$AAU?$AA?$AA@ 00000001800172a0     libucrt:lcidtoname_downlevel.obj
 0001:000162b0       ??_C@_1M@MNPLFAAH@?$AAe?$AAs?$AA?9?$AAE?$AAS?$AA?$AA@ 00000001800172b0     libucrt:lcidtoname_downlevel.obj
 0001:000162c0       ??_C@_1M@HJOOJFMA@?$AAf?$AAr?$AA?9?$AAC?$AAA?$AA?$AA@ 00000001800172c0     libucrt:lcidtoname_downlevel.obj
 0001:000162d0       ??_C@_1BG@JPOFPNAB@?$AAs?$AAr?$AA?9?$AAS?$AAP?$AA?9?$AAC?$AAy?$AAr?$AAl?$AA?$AA@ 00000001800172d0     libucrt:lcidtoname_downlevel.obj
 0001:000162e8       ??_C@_1M@LNFOCMOB@?$AAs?$AAe?$AA?9?$AAF?$AAI?$AA?$AA@ 00000001800172e8     libucrt:lcidtoname_downlevel.obj
 0001:000162f8       ??_C@_1O@MGJBOAMB@?$AAq?$AAu?$AAz?$AA?9?$AAP?$AAE?$AA?$AA@ 00000001800172f8     libucrt:lcidtoname_downlevel.obj
 0001:00016308       ??_C@_1M@GJINLBOK@?$AAa?$AAr?$AA?9?$AAL?$AAY?$AA?$AA@ 0000000180017308     libucrt:lcidtoname_downlevel.obj
 0001:00016318       ??_C@_1M@GGMNHJNL@?$AAz?$AAh?$AA?9?$AAS?$AAG?$AA?$AA@ 0000000180017318     libucrt:lcidtoname_downlevel.obj
 0001:00016328       ??_C@_1M@HOIKODND@?$AAd?$AAe?$AA?9?$AAL?$AAU?$AA?$AA@ 0000000180017328     libucrt:lcidtoname_downlevel.obj
 0001:00016338       ??_C@_1M@DDOCCGFG@?$AAe?$AAn?$AA?9?$AAC?$AAA?$AA?$AA@ 0000000180017338     libucrt:lcidtoname_downlevel.obj
 0001:00016348       ??_C@_1M@BNOEMJLF@?$AAe?$AAs?$AA?9?$AAG?$AAT?$AA?$AA@ 0000000180017348     libucrt:lcidtoname_downlevel.obj
 0001:00016358       ??_C@_1M@EOGNKEK@?$AAf?$AAr?$AA?9?$AAC?$AAH?$AA?$AA@ 0000000180017358     libucrt:lcidtoname_downlevel.obj
 0001:00016368       ??_C@_1M@FLIDJFHL@?$AAh?$AAr?$AA?9?$AAB?$AAA?$AA?$AA@ 0000000180017368     libucrt:lcidtoname_downlevel.obj
 0001:00016378       ??_C@_1O@FMCELNAJ@?$AAs?$AAm?$AAj?$AA?9?$AAN?$AAO?$AA?$AA@ 0000000180017378     libucrt:lcidtoname_downlevel.obj
 0001:00016388       ??_C@_1M@JHGLJMGJ@?$AAa?$AAr?$AA?9?$AAD?$AAZ?$AA?$AA@ 0000000180017388     libucrt:lcidtoname_downlevel.obj
 0001:00016398       ??_C@_1M@JKKFDCNP@?$AAz?$AAh?$AA?9?$AAM?$AAO?$AA?$AA@ 0000000180017398     libucrt:lcidtoname_downlevel.obj
 0001:000163a8       ??_C@_1M@GEEFALPE@?$AAd?$AAe?$AA?9?$AAL?$AAI?$AA?$AA@ 00000001800173a8     libucrt:lcidtoname_downlevel.obj
 0001:000163b8       ??_C@_1M@IGEOFBG@?$AAe?$AAn?$AA?9?$AAN?$AAZ?$AA?$AA@ 00000001800173b8     libucrt:lcidtoname_downlevel.obj
 0001:000163c8       ??_C@_1M@KDBONEHP@?$AAe?$AAs?$AA?9?$AAC?$AAR?$AA?$AA@ 00000001800173c8     libucrt:lcidtoname_downlevel.obj
 0001:000163d8       ??_C@_1M@FHMDOHNN@?$AAf?$AAr?$AA?9?$AAL?$AAU?$AA?$AA@ 00000001800173d8     libucrt:lcidtoname_downlevel.obj
 0001:000163e8       ??_C@_1BG@NFKKMAFG@?$AAb?$AAs?$AA?9?$AAB?$AAA?$AA?9?$AAL?$AAa?$AAt?$AAn?$AA?$AA@ 00000001800173e8     libucrt:lcidtoname_downlevel.obj
 0001:00016400       ??_C@_1O@IMNBEMCI@?$AAs?$AAm?$AAj?$AA?9?$AAS?$AAE?$AA?$AA@ 0000000180017400     libucrt:lcidtoname_downlevel.obj
 0001:00016410       ??_C@_1M@DHHMBNDP@?$AAa?$AAr?$AA?9?$AAM?$AAA?$AA?$AA@ 0000000180017410     libucrt:lcidtoname_downlevel.obj
 0001:00016420       ??_C@_1M@BNBLJCGH@?$AAe?$AAn?$AA?9?$AAI?$AAE?$AA?$AA@ 0000000180017420     libucrt:lcidtoname_downlevel.obj
 0001:00016430       ??_C@_1M@GEPAFMDL@?$AAe?$AAs?$AA?9?$AAP?$AAA?$AA?$AA@ 0000000180017430     libucrt:lcidtoname_downlevel.obj
 0001:00016440       ??_C@_1M@OJONDMDL@?$AAf?$AAr?$AA?9?$AAM?$AAC?$AA?$AA@ 0000000180017440     libucrt:lcidtoname_downlevel.obj
 0001:00016450       ??_C@_1BG@OBCNFJB@?$AAs?$AAr?$AA?9?$AAB?$AAA?$AA?9?$AAL?$AAa?$AAt?$AAn?$AA?$AA@ 0000000180017450     libucrt:lcidtoname_downlevel.obj
 0001:00016468       ??_C@_1O@KEMEEGPO@?$AAs?$AAm?$AAa?$AA?9?$AAN?$AAO?$AA?$AA@ 0000000180017468     libucrt:lcidtoname_downlevel.obj
 0001:00016478       ??_C@_1M@ELMGFODK@?$AAa?$AAr?$AA?9?$AAT?$AAN?$AA?$AA@ 0000000180017478     libucrt:lcidtoname_downlevel.obj
 0001:00016488       ??_C@_1M@BHDLHFAF@?$AAe?$AAn?$AA?9?$AAZ?$AAA?$AA?$AA@ 0000000180017488     libucrt:lcidtoname_downlevel.obj
 0001:00016498       ??_C@_1M@BMGIGLIF@?$AAe?$AAs?$AA?9?$AAD?$AAO?$AA?$AA@ 0000000180017498     libucrt:lcidtoname_downlevel.obj
 0001:000164a8       ??_C@_1BG@CMBHIPBE@?$AAs?$AAr?$AA?9?$AAB?$AAA?$AA?9?$AAC?$AAy?$AAr?$AAl?$AA?$AA@ 00000001800174a8     libucrt:lcidtoname_downlevel.obj
 0001:000164c0       ??_C@_1O@HEDBLHNP@?$AAs?$AAm?$AAa?$AA?9?$AAS?$AAE?$AA?$AA@ 00000001800174c0     libucrt:lcidtoname_downlevel.obj
 0001:000164d0       ??_C@_1M@DAGCADIM@?$AAa?$AAr?$AA?9?$AAO?$AAM?$AA?$AA@ 00000001800174d0     libucrt:lcidtoname_downlevel.obj
 0001:000164e0       ??_C@_1M@FODLMICG@?$AAe?$AAn?$AA?9?$AAJ?$AAM?$AA?$AA@ 00000001800174e0     libucrt:lcidtoname_downlevel.obj
 0001:000164f0       ??_C@_1M@DNMLCIHB@?$AAe?$AAs?$AA?9?$AAV?$AAE?$AA?$AA@ 00000001800174f0     libucrt:lcidtoname_downlevel.obj
 0001:00016500       ??_C@_1O@EOKHMKJK@?$AAs?$AAm?$AAs?$AA?9?$AAF?$AAI?$AA?$AA@ 0000000180017500     libucrt:lcidtoname_downlevel.obj
 0001:00016510       ??_C@_1M@CAFJMKOF@?$AAa?$AAr?$AA?9?$AAY?$AAE?$AA?$AA@ 0000000180017510     libucrt:lcidtoname_downlevel.obj
 0001:00016520       ??_C@_1M@CBFHIJLI@?$AAe?$AAn?$AA?9?$AAC?$AAB?$AA?$AA@ 0000000180017520     libucrt:lcidtoname_downlevel.obj
 0001:00016530       ??_C@_1M@BGNFLDN@?$AAe?$AAs?$AA?9?$AAC?$AAO?$AA?$AA@ 0000000180017530     libucrt:lcidtoname_downlevel.obj
 0001:00016540       ??_C@_1O@JMPHMAMC@?$AAs?$AAm?$AAn?$AA?9?$AAF?$AAI?$AA?$AA@ 0000000180017540     libucrt:lcidtoname_downlevel.obj
 0001:00016550       ??_C@_1M@JLANABKE@?$AAa?$AAr?$AA?9?$AAS?$AAY?$AA?$AA@ 0000000180017550     libucrt:lcidtoname_downlevel.obj
 0001:00016560       ??_C@_1M@HPKGCFGN@?$AAe?$AAn?$AA?9?$AAB?$AAZ?$AA?$AA@ 0000000180017560     libucrt:lcidtoname_downlevel.obj
 0001:00016570       ??_C@_1M@OLJCMLGM@?$AAe?$AAs?$AA?9?$AAP?$AAE?$AA?$AA@ 0000000180017570     libucrt:lcidtoname_downlevel.obj
 0001:00016580       ??_C@_1M@MKKGFKLE@?$AAa?$AAr?$AA?9?$AAJ?$AAO?$AA?$AA@ 0000000180017580     libucrt:lcidtoname_downlevel.obj
 0001:00016590       ??_C@_1M@EKPGLDNI@?$AAe?$AAn?$AA?9?$AAT?$AAT?$AA?$AA@ 0000000180017590     libucrt:lcidtoname_downlevel.obj
 0001:000165a0       ??_C@_1M@OONGHFHE@?$AAe?$AAs?$AA?9?$AAA?$AAR?$AA?$AA@ 00000001800175a0     libucrt:lcidtoname_downlevel.obj
 0001:000165b0       ??_C@_1M@OOJFGBHE@?$AAa?$AAr?$AA?9?$AAL?$AAB?$AA?$AA@ 00000001800175b0     libucrt:lcidtoname_downlevel.obj
 0001:000165c0       ??_C@_1M@GCEJHNEG@?$AAe?$AAn?$AA?9?$AAZ?$AAW?$AA?$AA@ 00000001800175c0     libucrt:lcidtoname_downlevel.obj
 0001:000165d0       ??_C@_1M@JNOCAHJI@?$AAe?$AAs?$AA?9?$AAE?$AAC?$AA?$AA@ 00000001800175d0     libucrt:lcidtoname_downlevel.obj
 0001:000165e0       ??_C@_1M@JEFHPGGB@?$AAa?$AAr?$AA?9?$AAK?$AAW?$AA?$AA@ 00000001800175e0     libucrt:lcidtoname_downlevel.obj
 0001:000165f0       ??_C@_1M@MLKIBJOJ@?$AAe?$AAn?$AA?9?$AAP?$AAH?$AA?$AA@ 00000001800175f0     libucrt:lcidtoname_downlevel.obj
 0001:00016600       ??_C@_1M@BDNIPEND@?$AAe?$AAs?$AA?9?$AAC?$AAL?$AA?$AA@ 0000000180017600     libucrt:lcidtoname_downlevel.obj
 0001:00016610       ??_C@_1M@MPNMEKBD@?$AAa?$AAr?$AA?9?$AAA?$AAE?$AA?$AA@ 0000000180017610     libucrt:lcidtoname_downlevel.obj
 0001:00016620       ??_C@_1M@KBJALCPI@?$AAe?$AAs?$AA?9?$AAU?$AAY?$AA?$AA@ 0000000180017620     libucrt:lcidtoname_downlevel.obj
 0001:00016630       ??_C@_1M@LLCCOAGA@?$AAa?$AAr?$AA?9?$AAB?$AAH?$AA?$AA@ 0000000180017630     libucrt:lcidtoname_downlevel.obj
 0001:00016640       ??_C@_1M@PBFNCDEL@?$AAe?$AAs?$AA?9?$AAP?$AAY?$AA?$AA@ 0000000180017640     libucrt:lcidtoname_downlevel.obj
 0001:00016650       ??_C@_1M@EDGINPNP@?$AAa?$AAr?$AA?9?$AAQ?$AAA?$AA?$AA@ 0000000180017650     libucrt:lcidtoname_downlevel.obj
 0001:00016660       ??_C@_1M@MKDBIIJI@?$AAe?$AAs?$AA?9?$AAB?$AAO?$AA?$AA@ 0000000180017660     libucrt:lcidtoname_downlevel.obj
 0001:00016670       ??_C@_1M@CPKKEBLD@?$AAe?$AAs?$AA?9?$AAS?$AAV?$AA?$AA@ 0000000180017670     libucrt:lcidtoname_downlevel.obj
 0001:00016680       ??_C@_1M@NDBGMMJL@?$AAe?$AAs?$AA?9?$AAH?$AAN?$AA?$AA@ 0000000180017680     libucrt:lcidtoname_downlevel.obj
 0001:00016690       ??_C@_1M@JIJIBHDP@?$AAe?$AAs?$AA?9?$AAN?$AAI?$AA?$AA@ 0000000180017690     libucrt:lcidtoname_downlevel.obj
 0001:000166a0       ??_C@_1M@CGFMKEEK@?$AAe?$AAs?$AA?9?$AAP?$AAR?$AA?$AA@ 00000001800176a0     libucrt:lcidtoname_downlevel.obj
 0001:000166b0       ??_C@_1O@ICJHKIIK@?$AAz?$AAh?$AA?9?$AAC?$AAH?$AAT?$AA?$AA@ 00000001800176b0     libucrt:lcidtoname_downlevel.obj
 0001:000166c0       ??_C@_15CLNEJCE@?$AAs?$AAr?$AA?$AA@ 00000001800176c0     libucrt:lcidtoname_downlevel.obj
 0001:00017510       ??_C@_1M@KAHEKEIG@?$AAa?$AAf?$AA?9?$AAz?$AAa?$AA?$AA@ 0000000180018510     libucrt:lcidtoname_downlevel.obj
 0001:00017520       ??_C@_1M@GIECOABL@?$AAa?$AAr?$AA?9?$AAa?$AAe?$AA?$AA@ 0000000180018520     libucrt:lcidtoname_downlevel.obj
 0001:00017530       ??_C@_1M@BMLMEKGI@?$AAa?$AAr?$AA?9?$AAb?$AAh?$AA?$AA@ 0000000180018530     libucrt:lcidtoname_downlevel.obj
 0001:00017540       ??_C@_1M@DAPFDGGB@?$AAa?$AAr?$AA?9?$AAd?$AAz?$AA?$AA@ 0000000180018540     libucrt:lcidtoname_downlevel.obj
 0001:00017550       ??_C@_1M@FJNKGKIG@?$AAa?$AAr?$AA?9?$AAe?$AAg?$AA?$AA@ 0000000180018550     libucrt:lcidtoname_downlevel.obj
 0001:00017560       ??_C@_1M@FLGKKCLO@?$AAa?$AAr?$AA?9?$AAi?$AAq?$AA?$AA@ 0000000180018560     libucrt:lcidtoname_downlevel.obj
 0001:00017570       ??_C@_1M@GNDIPALM@?$AAa?$AAr?$AA?9?$AAj?$AAo?$AA?$AA@ 0000000180018570     libucrt:lcidtoname_downlevel.obj
 0001:00017580       ??_C@_1M@DDMJFMGJ@?$AAa?$AAr?$AA?9?$AAk?$AAw?$AA?$AA@ 0000000180018580     libucrt:lcidtoname_downlevel.obj
 0001:00017590       ??_C@_1M@EJALMLHM@?$AAa?$AAr?$AA?9?$AAl?$AAb?$AA?$AA@ 0000000180018590     libucrt:lcidtoname_downlevel.obj
 0001:000175a0       ??_C@_1M@MOBDBLOC@?$AAa?$AAr?$AA?9?$AAl?$AAy?$AA?$AA@ 00000001800185a0     libucrt:lcidtoname_downlevel.obj
 0001:000175b0       ??_C@_1M@JAOCLHDH@?$AAa?$AAr?$AA?9?$AAm?$AAa?$AA?$AA@ 00000001800185b0     libucrt:lcidtoname_downlevel.obj
 0001:000175c0       ??_C@_1M@JHPMKJIE@?$AAa?$AAr?$AA?9?$AAo?$AAm?$AA?$AA@ 00000001800185c0     libucrt:lcidtoname_downlevel.obj
 0001:000175d0       ??_C@_1M@OEPGHFNH@?$AAa?$AAr?$AA?9?$AAq?$AAa?$AA?$AA@ 00000001800185d0     libucrt:lcidtoname_downlevel.obj
 0001:000175e0       ??_C@_1M@KJDONENM@?$AAa?$AAr?$AA?9?$AAs?$AAa?$AA?$AA@ 00000001800185e0     libucrt:lcidtoname_downlevel.obj
 0001:000175f0       ??_C@_1M@DMJDKLKM@?$AAa?$AAr?$AA?9?$AAs?$AAy?$AA?$AA@ 00000001800185f0     libucrt:lcidtoname_downlevel.obj
 0001:00017600       ??_C@_1M@OMFIPEDC@?$AAa?$AAr?$AA?9?$AAt?$AAn?$AA?$AA@ 0000000180018600     libucrt:lcidtoname_downlevel.obj
 0001:00017610       ??_C@_1M@IHMHGAON@?$AAa?$AAr?$AA?9?$AAy?$AAe?$AA?$AA@ 0000000180018610     libucrt:lcidtoname_downlevel.obj
 0001:00017620       ??_C@_1BG@KDCPGJGB@?$AAa?$AAz?$AA?9?$AAa?$AAz?$AA?9?$AAc?$AAy?$AAr?$AAl?$AA?$AA@ 0000000180018620     libucrt:lcidtoname_downlevel.obj
 0001:00017638       ??_C@_1BG@IBCKDDOE@?$AAa?$AAz?$AA?9?$AAa?$AAz?$AA?9?$AAl?$AAa?$AAt?$AAn?$AA?$AA@ 0000000180018638     libucrt:lcidtoname_downlevel.obj
 0001:00017650       ??_C@_1M@EGPFDCPD@?$AAb?$AAe?$AA?9?$AAb?$AAy?$AA?$AA@ 0000000180018650     libucrt:lcidtoname_downlevel.obj
 0001:00017660       ??_C@_1M@PCMGMCGC@?$AAb?$AAg?$AA?9?$AAb?$AAg?$AA?$AA@ 0000000180018660     libucrt:lcidtoname_downlevel.obj
 0001:00017670       ??_C@_1M@BJBMFGOB@?$AAb?$AAn?$AA?9?$AAi?$AAn?$AA?$AA@ 0000000180018670     libucrt:lcidtoname_downlevel.obj
 0001:00017680       ??_C@_1BG@EAKMMACD@?$AAb?$AAs?$AA?9?$AAb?$AAa?$AA?9?$AAl?$AAa?$AAt?$AAn?$AA?$AA@ 0000000180018680     libucrt:lcidtoname_downlevel.obj
 0001:00017698       ??_C@_1M@KGADAODK@?$AAc?$AAa?$AA?9?$AAe?$AAs?$AA?$AA@ 0000000180018698     libucrt:lcidtoname_downlevel.obj
 0001:000176a8       ??_C@_1M@COAJPDHI@?$AAc?$AAs?$AA?9?$AAc?$AAz?$AA?$AA@ 00000001800186a8     libucrt:lcidtoname_downlevel.obj
 0001:000176b8       ??_C@_1M@DHBHFONH@?$AAc?$AAy?$AA?9?$AAg?$AAb?$AA?$AA@ 00000001800186b8     libucrt:lcidtoname_downlevel.obj
 0001:000176c8       ??_C@_1M@IMGKELGA@?$AAd?$AAa?$AA?9?$AAd?$AAk?$AA?$AA@ 00000001800186c8     libucrt:lcidtoname_downlevel.obj
 0001:000176d8       ??_C@_1M@NNDGDNGA@?$AAd?$AAe?$AA?9?$AAa?$AAt?$AA?$AA@ 00000001800186d8     libucrt:lcidtoname_downlevel.obj
 0001:000176e8       ??_C@_1M@IKDBHEEM@?$AAd?$AAe?$AA?9?$AAc?$AAh?$AA?$AA@ 00000001800186e8     libucrt:lcidtoname_downlevel.obj
 0001:000176f8       ??_C@_1M@GFFOJMCJ@?$AAd?$AAe?$AA?9?$AAd?$AAe?$AA?$AA@ 00000001800186f8     libucrt:lcidtoname_downlevel.obj
 0001:00017708       ??_C@_1M@MDNLKBPM@?$AAd?$AAe?$AA?9?$AAl?$AAi?$AA?$AA@ 0000000180018708     libucrt:lcidtoname_downlevel.obj
 0001:00017718       ??_C@_1M@NJBEEJNL@?$AAd?$AAe?$AA?9?$AAl?$AAu?$AA?$AA@ 0000000180018718     libucrt:lcidtoname_downlevel.obj
 0001:00017728       ??_C@_1O@GNNELBAP@?$AAd?$AAi?$AAv?$AA?9?$AAm?$AAv?$AA?$AA@ 0000000180018728     libucrt:lcidtoname_downlevel.obj
 0001:00017738       ??_C@_1M@EJLEOGAE@?$AAe?$AAl?$AA?9?$AAg?$AAr?$AA?$AA@ 0000000180018738     libucrt:lcidtoname_downlevel.obj
 0001:00017748       ??_C@_1M@GMPONJN@?$AAe?$AAn?$AA?9?$AAa?$AAu?$AA?$AA@ 0000000180018748     libucrt:lcidtoname_downlevel.obj
 0001:00017758       ??_C@_1M@NIDIIPGF@?$AAe?$AAn?$AA?9?$AAb?$AAz?$AA?$AA@ 0000000180018758     libucrt:lcidtoname_downlevel.obj
 0001:00017768       ??_C@_1M@JEHMIMFO@?$AAe?$AAn?$AA?9?$AAc?$AAa?$AA?$AA@ 0000000180018768     libucrt:lcidtoname_downlevel.obj
 0001:00017778       ??_C@_1M@IGMJCDLA@?$AAe?$AAn?$AA?9?$AAc?$AAb?$AA?$AA@ 0000000180018778     libucrt:lcidtoname_downlevel.obj
 0001:00017788       ??_C@_1M@BNFIGBKG@?$AAe?$AAn?$AA?9?$AAg?$AAb?$AA?$AA@ 0000000180018788     libucrt:lcidtoname_downlevel.obj
 0001:00017798       ??_C@_1M@LKIFDIGP@?$AAe?$AAn?$AA?9?$AAi?$AAe?$AA?$AA@ 0000000180018798     libucrt:lcidtoname_downlevel.obj
 0001:000177a8       ??_C@_1M@PJKFGCCO@?$AAe?$AAn?$AA?9?$AAj?$AAm?$AA?$AA@ 00000001800187a8     libucrt:lcidtoname_downlevel.obj
 0001:000177b8       ??_C@_1M@KPPKEPBO@?$AAe?$AAn?$AA?9?$AAn?$AAz?$AA?$AA@ 00000001800187b8     libucrt:lcidtoname_downlevel.obj
 0001:000177c8       ??_C@_1M@GMDGLDOB@?$AAe?$AAn?$AA?9?$AAp?$AAh?$AA?$AA@ 00000001800187c8     libucrt:lcidtoname_downlevel.obj
 0001:000177d8       ??_C@_1M@ONGIBJNA@?$AAe?$AAn?$AA?9?$AAt?$AAt?$AA?$AA@ 00000001800187d8     libucrt:lcidtoname_downlevel.obj
 0001:000177e8       ??_C@_1M@LLODPCMM@?$AAe?$AAn?$AA?9?$AAu?$AAs?$AA?$AA@ 00000001800187e8     libucrt:lcidtoname_downlevel.obj
 0001:000177f8       ??_C@_1M@LAKFNPAN@?$AAe?$AAn?$AA?9?$AAz?$AAa?$AA?$AA@ 00000001800187f8     libucrt:lcidtoname_downlevel.obj
 0001:00017808       ??_C@_1M@MFNHNHEO@?$AAe?$AAn?$AA?9?$AAz?$AAw?$AA?$AA@ 0000000180018808     libucrt:lcidtoname_downlevel.obj
 0001:00017818       ??_C@_1M@EJEINPHM@?$AAe?$AAs?$AA?9?$AAa?$AAr?$AA?$AA@ 0000000180018818     libucrt:lcidtoname_downlevel.obj
 0001:00017828       ??_C@_1M@GNKPCCJA@?$AAe?$AAs?$AA?9?$AAb?$AAo?$AA?$AA@ 0000000180018828     libucrt:lcidtoname_downlevel.obj
 0001:00017838       ??_C@_1M@LEEGFONL@?$AAe?$AAs?$AA?9?$AAc?$AAl?$AA?$AA@ 0000000180018838     libucrt:lcidtoname_downlevel.obj
 0001:00017848       ??_C@_1M@KGPDPBDF@?$AAe?$AAs?$AA?9?$AAc?$AAo?$AA?$AA@ 0000000180018848     libucrt:lcidtoname_downlevel.obj
 0001:00017858       ??_C@_1M@EIAHOHH@?$AAe?$AAs?$AA?9?$AAc?$AAr?$AA?$AA@ 0000000180018858     libucrt:lcidtoname_downlevel.obj
 0001:00017868       ??_C@_1M@LLPGMBIN@?$AAe?$AAs?$AA?9?$AAd?$AAo?$AA?$AA@ 0000000180018868     libucrt:lcidtoname_downlevel.obj
 0001:00017878       ??_C@_1M@DKHMKNJA@?$AAe?$AAs?$AA?9?$AAe?$AAc?$AA?$AA@ 0000000180018878     libucrt:lcidtoname_downlevel.obj
 0001:00017888       ??_C@_1M@GKGFPKAP@?$AAe?$AAs?$AA?9?$AAe?$AAs?$AA?$AA@ 0000000180018888     libucrt:lcidtoname_downlevel.obj
 0001:00017898       ??_C@_1M@LKHKGDLN@?$AAe?$AAs?$AA?9?$AAg?$AAt?$AA?$AA@ 0000000180018898     libucrt:lcidtoname_downlevel.obj
 0001:000178a8       ??_C@_1M@HEIIGGJD@?$AAe?$AAs?$AA?9?$AAh?$AAn?$AA?$AA@ 00000001800188a8     libucrt:lcidtoname_downlevel.obj
 0001:000178b8       ??_C@_1M@FBDHPPGD@?$AAe?$AAs?$AA?9?$AAm?$AAx?$AA?$AA@ 00000001800188b8     libucrt:lcidtoname_downlevel.obj
 0001:000178c8       ??_C@_1M@DPAGLNDH@?$AAe?$AAs?$AA?9?$AAn?$AAi?$AA?$AA@ 00000001800188c8     libucrt:lcidtoname_downlevel.obj
 0001:000178d8       ??_C@_1M@MDGOPGDD@?$AAe?$AAs?$AA?9?$AAp?$AAa?$AA?$AA@ 00000001800188d8     libucrt:lcidtoname_downlevel.obj
 0001:000178e8       ??_C@_1M@EMAMGBGE@?$AAe?$AAs?$AA?9?$AAp?$AAe?$AA?$AA@ 00000001800188e8     libucrt:lcidtoname_downlevel.obj
 0001:000178f8       ??_C@_1M@IBMCAOEC@?$AAe?$AAs?$AA?9?$AAp?$AAr?$AA?$AA@ 00000001800188f8     libucrt:lcidtoname_downlevel.obj
 0001:00017908       ??_C@_1M@FGMDIJED@?$AAe?$AAs?$AA?9?$AAp?$AAy?$AA?$AA@ 0000000180018908     libucrt:lcidtoname_downlevel.obj
 0001:00017918       ??_C@_1M@IIDEOLLL@?$AAe?$AAs?$AA?9?$AAs?$AAv?$AA?$AA@ 0000000180018918     libucrt:lcidtoname_downlevel.obj
 0001:00017928       ??_C@_1M@GAOBIPA@?$AAe?$AAs?$AA?9?$AAu?$AAy?$AA?$AA@ 0000000180018928     libucrt:lcidtoname_downlevel.obj
 0001:00017938       ??_C@_1M@JKFFICHJ@?$AAe?$AAs?$AA?9?$AAv?$AAe?$AA?$AA@ 0000000180018938     libucrt:lcidtoname_downlevel.obj
 0001:00017948       ??_C@_1M@PNMLOJDF@?$AAe?$AAt?$AA?9?$AAe?$AAe?$AA?$AA@ 0000000180018948     libucrt:lcidtoname_downlevel.obj
 0001:00017958       ??_C@_1M@GHHLIKEI@?$AAe?$AAu?$AA?9?$AAe?$AAs?$AA?$AA@ 0000000180018958     libucrt:lcidtoname_downlevel.obj
 0001:00017968       ??_C@_1M@PBNONODE@?$AAf?$AAa?$AA?9?$AAi?$AAr?$AA?$AA@ 0000000180018968     libucrt:lcidtoname_downlevel.obj
 0001:00017978       ??_C@_1M@JEEHPMIL@?$AAf?$AAi?$AA?9?$AAf?$AAi?$AA?$AA@ 0000000180018978     libucrt:lcidtoname_downlevel.obj
 0001:00017988       ??_C@_1M@LMDCNDBA@?$AAf?$AAo?$AA?9?$AAf?$AAo?$AA?$AA@ 0000000180018988     libucrt:lcidtoname_downlevel.obj
 0001:00017998       ??_C@_1M@JKEOHLDK@?$AAf?$AAr?$AA?9?$AAb?$AAe?$AA?$AA@ 0000000180018998     libucrt:lcidtoname_downlevel.obj
 0001:000179a8       ??_C@_1M@NOHADPMI@?$AAf?$AAr?$AA?9?$AAc?$AAa?$AA?$AA@ 00000001800189a8     libucrt:lcidtoname_downlevel.obj
 0001:000179b8       ??_C@_1M@KDHIHAEC@?$AAf?$AAr?$AA?9?$AAc?$AAh?$AA?$AA@ 00000001800189b8     libucrt:lcidtoname_downlevel.obj
 0001:000179c8       ??_C@_1M@MMBBFGAK@?$AAf?$AAr?$AA?9?$AAf?$AAr?$AA?$AA@ 00000001800189c8     libucrt:lcidtoname_downlevel.obj
 0001:000179d8       ??_C@_1M@PAFNENNF@?$AAf?$AAr?$AA?9?$AAl?$AAu?$AA?$AA@ 00000001800189d8     libucrt:lcidtoname_downlevel.obj
 0001:000179e8       ??_C@_1M@EOHDJGDD@?$AAf?$AAr?$AA?9?$AAm?$AAc?$AA?$AA@ 00000001800189e8     libucrt:lcidtoname_downlevel.obj
 0001:000179f8       ??_C@_1M@FAPLLOPF@?$AAg?$AAl?$AA?9?$AAe?$AAs?$AA?$AA@ 00000001800189f8     libucrt:lcidtoname_downlevel.obj
 0001:00017a08       ??_C@_1M@FOPBFLOO@?$AAg?$AAu?$AA?9?$AAi?$AAn?$AA?$AA@ 0000000180018a08     libucrt:lcidtoname_downlevel.obj
 0001:00017a18       ??_C@_1M@KBMCINPM@?$AAh?$AAe?$AA?9?$AAi?$AAl?$AA?$AA@ 0000000180018a18     libucrt:lcidtoname_downlevel.obj
 0001:00017a28       ??_C@_1M@BBPHKFPJ@?$AAh?$AAi?$AA?9?$AAi?$AAn?$AA?$AA@ 0000000180018a28     libucrt:lcidtoname_downlevel.obj
 0001:00017a38       ??_C@_1M@PMBNDPHD@?$AAh?$AAr?$AA?9?$AAb?$AAa?$AA?$AA@ 0000000180018a38     libucrt:lcidtoname_downlevel.obj
 0001:00017a48       ??_C@_1M@BPCKOEGE@?$AAh?$AAr?$AA?9?$AAh?$AAr?$AA?$AA@ 0000000180018a48     libucrt:lcidtoname_downlevel.obj
 0001:00017a58       ??_C@_1M@GACBMHKE@?$AAh?$AAu?$AA?9?$AAh?$AAu?$AA?$AA@ 0000000180018a58     libucrt:lcidtoname_downlevel.obj
 0001:00017a68       ??_C@_1M@MILPAJJC@?$AAh?$AAy?$AA?9?$AAa?$AAm?$AA?$AA@ 0000000180018a68     libucrt:lcidtoname_downlevel.obj
 0001:00017a78       ??_C@_1M@BABBICEC@?$AAi?$AAd?$AA?9?$AAi?$AAd?$AA?$AA@ 0000000180018a78     libucrt:lcidtoname_downlevel.obj
 0001:00017a88       ??_C@_1M@BIKNHHPF@?$AAi?$AAs?$AA?9?$AAi?$AAs?$AA?$AA@ 0000000180018a88     libucrt:lcidtoname_downlevel.obj
 0001:00017a98       ??_C@_1M@NMPCJPHE@?$AAi?$AAt?$AA?9?$AAc?$AAh?$AA?$AA@ 0000000180018a98     libucrt:lcidtoname_downlevel.obj
 0001:00017aa8       ??_C@_1M@GHKGFEDF@?$AAi?$AAt?$AA?9?$AAi?$AAt?$AA?$AA@ 0000000180018aa8     libucrt:lcidtoname_downlevel.obj
 0001:00017ab8       ??_C@_1M@NIEJCJJA@?$AAj?$AAa?$AA?9?$AAj?$AAp?$AA?$AA@ 0000000180018ab8     libucrt:lcidtoname_downlevel.obj
 0001:00017ac8       ??_C@_1M@JILFNBIM@?$AAk?$AAa?$AA?9?$AAg?$AAe?$AA?$AA@ 0000000180018ac8     libucrt:lcidtoname_downlevel.obj
 0001:00017ad8       ??_C@_1M@PACPMGPH@?$AAk?$AAk?$AA?9?$AAk?$AAz?$AA?$AA@ 0000000180018ad8     libucrt:lcidtoname_downlevel.obj
 0001:00017ae8       ??_C@_1M@IELFGMHA@?$AAk?$AAn?$AA?9?$AAi?$AAn?$AA?$AA@ 0000000180018ae8     libucrt:lcidtoname_downlevel.obj
 0001:00017af8       ??_C@_1O@IBBJHCH@?$AAk?$AAo?$AAk?$AA?9?$AAi?$AAn?$AA?$AA@ 0000000180018af8     libucrt:lcidtoname_downlevel.obj
 0001:00017b08       ??_C@_1M@DMHAEOGC@?$AAk?$AAo?$AA?9?$AAk?$AAr?$AA?$AA@ 0000000180018b08     libucrt:lcidtoname_downlevel.obj
 0001:00017b18       ??_C@_1M@HBAHBIGA@?$AAk?$AAy?$AA?9?$AAk?$AAg?$AA?$AA@ 0000000180018b18     libucrt:lcidtoname_downlevel.obj
 0001:00017b28       ??_C@_1M@KPMILCJG@?$AAl?$AAt?$AA?9?$AAl?$AAt?$AA?$AA@ 0000000180018b28     libucrt:lcidtoname_downlevel.obj
 0001:00017b38       ??_C@_1M@BDEKKCA@?$AAl?$AAv?$AA?9?$AAl?$AAv?$AA?$AA@ 0000000180018b38     libucrt:lcidtoname_downlevel.obj
 0001:00017b48       ??_C@_1M@ELCKCCJJ@?$AAm?$AAi?$AA?9?$AAn?$AAz?$AA?$AA@ 0000000180018b48     libucrt:lcidtoname_downlevel.obj
 0001:00017b58       ??_C@_1M@CBOOLAPA@?$AAm?$AAk?$AA?9?$AAm?$AAk?$AA?$AA@ 0000000180018b58     libucrt:lcidtoname_downlevel.obj
 0001:00017b68       ??_C@_1M@GPHNBJKN@?$AAm?$AAl?$AA?9?$AAi?$AAn?$AA?$AA@ 0000000180018b68     libucrt:lcidtoname_downlevel.obj
 0001:00017b78       ??_C@_1M@PABJILIG@?$AAm?$AAn?$AA?9?$AAm?$AAn?$AA?$AA@ 0000000180018b78     libucrt:lcidtoname_downlevel.obj
 0001:00017b88       ??_C@_1M@FGBKKIPG@?$AAm?$AAr?$AA?9?$AAi?$AAn?$AA?$AA@ 0000000180018b88     libucrt:lcidtoname_downlevel.obj
 0001:00017b98       ??_C@_1M@NDBPDDAL@?$AAm?$AAs?$AA?9?$AAb?$AAn?$AA?$AA@ 0000000180018b98     libucrt:lcidtoname_downlevel.obj
 0001:00017ba8       ??_C@_1M@OPIHOOPI@?$AAm?$AAs?$AA?9?$AAm?$AAy?$AA?$AA@ 0000000180018ba8     libucrt:lcidtoname_downlevel.obj
 0001:00017bb8       ??_C@_1M@PPDBCNFM@?$AAm?$AAt?$AA?9?$AAm?$AAt?$AA?$AA@ 0000000180018bb8     libucrt:lcidtoname_downlevel.obj
 0001:00017bc8       ??_C@_1M@KDJDKMDD@?$AAn?$AAb?$AA?9?$AAn?$AAo?$AA?$AA@ 0000000180018bc8     libucrt:lcidtoname_downlevel.obj
 0001:00017bd8       ??_C@_1M@KFCFLMJP@?$AAn?$AAl?$AA?9?$AAb?$AAe?$AA?$AA@ 0000000180018bd8     libucrt:lcidtoname_downlevel.obj
 0001:00017be8       ??_C@_1M@KPOPDDGO@?$AAn?$AAl?$AA?9?$AAn?$AAl?$AA?$AA@ 0000000180018be8     libucrt:lcidtoname_downlevel.obj
 0001:00017bf8       ??_C@_1M@LJKPEMLN@?$AAn?$AAn?$AA?9?$AAn?$AAo?$AA?$AA@ 0000000180018bf8     libucrt:lcidtoname_downlevel.obj
 0001:00017c08       ??_C@_1M@BDGHHBFL@?$AAn?$AAs?$AA?9?$AAz?$AAa?$AA?$AA@ 0000000180018c08     libucrt:lcidtoname_downlevel.obj
 0001:00017c18       ??_C@_1M@IDEHOAP@?$AAp?$AAa?$AA?9?$AAi?$AAn?$AA?$AA@ 0000000180018c18     libucrt:lcidtoname_downlevel.obj
 0001:00017c28       ??_C@_1M@HDBKGOGH@?$AAp?$AAl?$AA?9?$AAp?$AAl?$AA?$AA@ 0000000180018c28     libucrt:lcidtoname_downlevel.obj
 0001:00017c38       ??_C@_1M@LJLLCMEH@?$AAp?$AAt?$AA?9?$AAb?$AAr?$AA?$AA@ 0000000180018c38     libucrt:lcidtoname_downlevel.obj
 0001:00017c48       ??_C@_1M@NCMONAAL@?$AAp?$AAt?$AA?9?$AAp?$AAt?$AA?$AA@ 0000000180018c48     libucrt:lcidtoname_downlevel.obj
 0001:00017c58       ??_C@_1O@EAKMAJDN@?$AAq?$AAu?$AAz?$AA?9?$AAb?$AAo?$AA?$AA@ 0000000180018c58     libucrt:lcidtoname_downlevel.obj
 0001:00017c68       ??_C@_1O@BHHPIGDN@?$AAq?$AAu?$AAz?$AA?9?$AAe?$AAc?$AA?$AA@ 0000000180018c68     libucrt:lcidtoname_downlevel.obj
 0001:00017c78       ??_C@_1O@GBAPEKMJ@?$AAq?$AAu?$AAz?$AA?9?$AAp?$AAe?$AA?$AA@ 0000000180018c78     libucrt:lcidtoname_downlevel.obj
 0001:00017c88       ??_C@_1M@CLGLEFBO@?$AAr?$AAo?$AA?9?$AAr?$AAo?$AA?$AA@ 0000000180018c88     libucrt:lcidtoname_downlevel.obj
 0001:00017c98       ??_C@_1M@CEEDODME@?$AAr?$AAu?$AA?9?$AAr?$AAu?$AA?$AA@ 0000000180018c98     libucrt:lcidtoname_downlevel.obj
 0001:00017ca8       ??_C@_1M@HPKKKMPP@?$AAs?$AAa?$AA?9?$AAi?$AAn?$AA?$AA@ 0000000180018ca8     libucrt:lcidtoname_downlevel.obj
 0001:00017cb8       ??_C@_1M@BKMAIGOJ@?$AAs?$AAe?$AA?9?$AAf?$AAi?$AA?$AA@ 0000000180018cb8     libucrt:lcidtoname_downlevel.obj
 0001:00017cc8       ??_C@_1M@NDPIFLFI@?$AAs?$AAe?$AA?9?$AAn?$AAo?$AA?$AA@ 0000000180018cc8     libucrt:lcidtoname_downlevel.obj
 0001:00017cd8       ??_C@_1M@DANKKHJ@?$AAs?$AAe?$AA?9?$AAs?$AAe?$AA?$AA@ 0000000180018cd8     libucrt:lcidtoname_downlevel.obj
 0001:00017ce8       ??_C@_1M@PNBLONPJ@?$AAs?$AAk?$AA?9?$AAs?$AAk?$AA?$AA@ 0000000180018ce8     libucrt:lcidtoname_downlevel.obj
 0001:00017cf8       ??_C@_1M@LFMODOAL@?$AAs?$AAl?$AA?9?$AAs?$AAi?$AA?$AA@ 0000000180018cf8     libucrt:lcidtoname_downlevel.obj
 0001:00017d08       ??_C@_1O@DFKOMPG@?$AAs?$AAm?$AAa?$AA?9?$AAn?$AAo?$AA?$AA@ 0000000180018d08     libucrt:lcidtoname_downlevel.obj
 0001:00017d18       ??_C@_1O@NDKPBNNH@?$AAs?$AAm?$AAa?$AA?9?$AAs?$AAe?$AA?$AA@ 0000000180018d18     libucrt:lcidtoname_downlevel.obj
 0001:00017d28       ??_C@_1O@PLLKBHAB@?$AAs?$AAm?$AAj?$AA?9?$AAn?$AAo?$AA?$AA@ 0000000180018d28     libucrt:lcidtoname_downlevel.obj
 0001:00017d38       ??_C@_1O@CLEPOGCA@?$AAs?$AAm?$AAj?$AA?9?$AAs?$AAe?$AA?$AA@ 0000000180018d38     libucrt:lcidtoname_downlevel.obj
 0001:00017d48       ??_C@_1O@DLGJGKMK@?$AAs?$AAm?$AAn?$AA?9?$AAf?$AAi?$AA?$AA@ 0000000180018d48     libucrt:lcidtoname_downlevel.obj
 0001:00017d58       ??_C@_1O@OJDJGAJC@?$AAs?$AAm?$AAs?$AA?9?$AAf?$AAi?$AA?$AA@ 0000000180018d58     libucrt:lcidtoname_downlevel.obj
 0001:00017d68       ??_C@_1M@BOFOGHPB@?$AAs?$AAq?$AA?9?$AAa?$AAl?$AA?$AA@ 0000000180018d68     libucrt:lcidtoname_downlevel.obj
 0001:00017d78       ??_C@_1BG@LJBBIPGB@?$AAs?$AAr?$AA?9?$AAb?$AAa?$AA?9?$AAc?$AAy?$AAr?$AAl?$AA?$AA@ 0000000180018d78     libucrt:lcidtoname_downlevel.obj
 0001:00017d90       ??_C@_1BG@JLBENFOE@?$AAs?$AAr?$AA?9?$AAb?$AAa?$AA?9?$AAl?$AAa?$AAt?$AAn?$AA?$AA@ 0000000180018d90     libucrt:lcidtoname_downlevel.obj
 0001:00017da8       ??_C@_1BG@KODPNHE@?$AAs?$AAr?$AA?9?$AAs?$AAp?$AA?9?$AAc?$AAy?$AAr?$AAl?$AA?$AA@ 0000000180018da8     libucrt:lcidtoname_downlevel.obj
 0001:00017dc0       ??_C@_1BG@CIOGKHPB@?$AAs?$AAr?$AA?9?$AAs?$AAp?$AA?9?$AAl?$AAa?$AAt?$AAn?$AA?$AA@ 0000000180018dc0     libucrt:lcidtoname_downlevel.obj
 0001:00017dd8       ??_C@_1M@NGFJLMAC@?$AAs?$AAv?$AA?9?$AAf?$AAi?$AA?$AA@ 0000000180018dd8     libucrt:lcidtoname_downlevel.obj
 0001:00017de8       ??_C@_1M@MPJEJAJC@?$AAs?$AAv?$AA?9?$AAs?$AAe?$AA?$AA@ 0000000180018de8     libucrt:lcidtoname_downlevel.obj
 0001:00017df8       ??_C@_1M@MPNDHLFK@?$AAs?$AAw?$AA?9?$AAk?$AAe?$AA?$AA@ 0000000180018df8     libucrt:lcidtoname_downlevel.obj
 0001:00017e08       ??_C@_1O@KOHBJJI@?$AAs?$AAy?$AAr?$AA?9?$AAs?$AAy?$AA?$AA@ 0000000180018e08     libucrt:lcidtoname_downlevel.obj
 0001:00017e18       ??_C@_1M@LDCEFHA@?$AAt?$AAa?$AA?9?$AAi?$AAn?$AA?$AA@ 0000000180018e18     libucrt:lcidtoname_downlevel.obj
 0001:00017e28       ??_C@_1M@CNJOFAK@?$AAt?$AAe?$AA?9?$AAi?$AAn?$AA?$AA@ 0000000180018e28     libucrt:lcidtoname_downlevel.obj
 0001:00017e38       ??_C@_1M@GNAECACD@?$AAt?$AAh?$AA?9?$AAt?$AAh?$AA?$AA@ 0000000180018e38     libucrt:lcidtoname_downlevel.obj
 0001:00017e48       ??_C@_1M@CHBIHOJO@?$AAt?$AAn?$AA?9?$AAz?$AAa?$AA?$AA@ 0000000180018e48     libucrt:lcidtoname_downlevel.obj
 0001:00017e58       ??_C@_1M@GCCMIGPJ@?$AAt?$AAr?$AA?9?$AAt?$AAr?$AA?$AA@ 0000000180018e58     libucrt:lcidtoname_downlevel.obj
 0001:00017e68       ??_C@_1M@CELMCNBK@?$AAt?$AAt?$AA?9?$AAr?$AAu?$AA?$AA@ 0000000180018e68     libucrt:lcidtoname_downlevel.obj
 0001:00017e78       ??_C@_1M@KLMCELGA@?$AAu?$AAk?$AA?9?$AAu?$AAa?$AA?$AA@ 0000000180018e78     libucrt:lcidtoname_downlevel.obj
 0001:00017e88       ??_C@_1M@EPAJJAJF@?$AAu?$AAr?$AA?9?$AAp?$AAk?$AA?$AA@ 0000000180018e88     libucrt:lcidtoname_downlevel.obj
 0001:00017e98       ??_C@_1BG@GEGPMCDJ@?$AAu?$AAz?$AA?9?$AAu?$AAz?$AA?9?$AAc?$AAy?$AAr?$AAl?$AA?$AA@ 0000000180018e98     libucrt:lcidtoname_downlevel.obj
 0001:00017eb0       ??_C@_1BG@EGGKJILM@?$AAu?$AAz?$AA?9?$AAu?$AAz?$AA?9?$AAl?$AAa?$AAt?$AAn?$AA?$AA@ 0000000180018eb0     libucrt:lcidtoname_downlevel.obj
 0001:00017ec8       ??_C@_1M@GFOCLFF@?$AAv?$AAi?$AA?9?$AAv?$AAn?$AA?$AA@ 0000000180018ec8     libucrt:lcidtoname_downlevel.obj
 0001:00017ed8       ??_C@_1M@CPAMEDFI@?$AAx?$AAh?$AA?9?$AAz?$AAa?$AA?$AA@ 0000000180018ed8     libucrt:lcidtoname_downlevel.obj
 0001:00017ee8       ??_C@_1O@EBKIFIGN@?$AAz?$AAh?$AA?9?$AAc?$AAh?$AAs?$AA?$AA@ 0000000180018ee8     libucrt:lcidtoname_downlevel.obj
 0001:00017ef8       ??_C@_1O@NMHPGANE@?$AAz?$AAh?$AA?9?$AAc?$AAh?$AAt?$AA?$AA@ 0000000180018ef8     libucrt:lcidtoname_downlevel.obj
 0001:00017f08       ??_C@_1M@LPINJOMC@?$AAz?$AAh?$AA?9?$AAc?$AAn?$AA?$AA@ 0000000180018f08     libucrt:lcidtoname_downlevel.obj
 0001:00017f18       ??_C@_1M@OCJEJODD@?$AAz?$AAh?$AA?9?$AAh?$AAk?$AA?$AA@ 0000000180018f18     libucrt:lcidtoname_downlevel.obj
 0001:00017f28       ??_C@_1M@DNDLJINH@?$AAz?$AAh?$AA?9?$AAm?$AAo?$AA?$AA@ 0000000180018f28     libucrt:lcidtoname_downlevel.obj
 0001:00017f38       ??_C@_1M@MBFDNDND@?$AAz?$AAh?$AA?9?$AAs?$AAg?$AA?$AA@ 0000000180018f38     libucrt:lcidtoname_downlevel.obj
 0001:00017f48       ??_C@_1M@IMEPLEPE@?$AAz?$AAh?$AA?9?$AAt?$AAw?$AA?$AA@ 0000000180018f48     libucrt:lcidtoname_downlevel.obj
 0001:00017f58       ??_C@_1M@BBGHNHJP@?$AAz?$AAu?$AA?9?$AAz?$AAa?$AA?$AA@ 0000000180018f58     libucrt:lcidtoname_downlevel.obj
 0001:000181c0       ??_C@_1BA@BALFACEM@?$AAC?$AAO?$AAN?$AAO?$AAU?$AAT?$AA$?$AA?$AA@ 00000001800191c0     libucrt:initcon.obj
 0001:000181d0       __log10_256_lead           00000001800191d0     libucrt:log10_256_lead_tail_table.obj
 0001:000189e0       __log10_256_tail           00000001800199e0     libucrt:log10_256_lead_tail_table.obj
 0001:000191f0       __log_F_inv_qword          000000018001a1f0     libucrt:log_f_inv_qword_table.obj
 0001:00019a00       ??_C@_05HGHHAHAP@log10?$AA@ 000000018001aa00     libucrt:log_special.obj
 0001:00019a40       _load_config_used          000000018001aa40     LIBCMT:loadcfg.obj
 0001:00019dc0       __rtc_iaa                  000000018001adc0     LIBCMT:initsect.obj
 0001:00019dc8       __rtc_izz                  000000018001adc8     LIBCMT:initsect.obj
 0001:00019dd0       __rtc_taa                  000000018001add0     LIBCMT:initsect.obj
 0001:00019dd8       __rtc_tzz                  000000018001add8     LIBCMT:initsect.obj
 0001:00019df0       __chkstk                   000000018001adf0 f   chkstk.obj
 0001:00019df0       _alloca_probe              000000018001adf0 f   chkstk.obj
 0001:0001a940       __local_stdio_printf_options 000000018001b940 f i bit64.obj
 0001:0001a950       bit64_getvalue             000000018001b950 f   bit64.obj
 0001:0001aa00       bit64_push                 000000018001ba00 f   bit64.obj
 0001:0001aa90       bit64_pushuserdata         000000018001ba90 f   bit64.obj
 0001:0001ac20       luaopen_bit64              000000018001bc20 f   bit64.obj
 0001:0001ac70       sprintf                    000000018001bc70 f i bit64.obj
 0001:0001acd0       AddBufToCollector          000000018001bcd0 f   exported.obj
 0001:0001ad50       CreateStringsArray         000000018001bd50 f   exported.obj
 0001:0001ae60       FarPanelItemFreeCallback   000000018001be60 f   exported.obj
 0001:0001b140       FillFindData               000000018001c140 f   exported.obj
 0001:0001b450       FillPluginPanelItem        000000018001c450 f   exported.obj
 0001:0001b740       GetExportFunction          000000018001c740 f   exported.obj
 0001:0001b7e0       LF_Analyse                 000000018001c7e0 f   exported.obj
 0001:0001b8a0       LF_CloseAnalyse            000000018001c8a0 f   exported.obj
 0001:0001b8b0       LF_ClosePanel              000000018001c8b0 f   exported.obj
 0001:0001b9a0       LF_Compare                 000000018001c9a0 f   exported.obj
 0001:0001bab0       LF_Configure               000000018001cab0 f   exported.obj
 0001:0001bb40       LF_DeleteFiles             000000018001cb40 f   exported.obj
 0001:0001bc30       LF_ExitFAR                 000000018001cc30 f   exported.obj
 0001:0001bc90       LF_FreeContentData         000000018001cc90 f   exported.obj
 0001:0001bce0       LF_FreeFindData            000000018001cce0 f   exported.obj
 0001:0001bd60       LF_GetContentData          000000018001cd60 f   exported.obj
 0001:0001bec0       LF_GetContentFields        000000018001cec0 f   exported.obj
 0001:0001bf90       LF_GetFiles                000000018001cf90 f   exported.obj
 0001:0001c130       LF_GetFindData             000000018001d130 f   exported.obj
 0001:0001c250       LF_GetGlobalInfo           000000018001d250 f   exported.obj
 0001:0001c6b0       LF_GetOpenPanelInfo        000000018001d6b0 f   exported.obj
 0001:0001d0a0       LF_GetPluginInfo           000000018001e0a0 f   exported.obj
 0001:0001d1f0       LF_MakeDirectory           000000018001e1f0 f   exported.obj
 0001:0001d340       LF_Open                    000000018001e340 f   exported.obj
 0001:0001d750       LF_ProcessConsoleInput     000000018001e750 f   exported.obj
 0001:0001d840       LF_ProcessDialogEvent      000000018001e840 f   exported.obj
 0001:0001da60       LF_ProcessEditorEvent      000000018001ea60 f   exported.obj
 0001:0001dbd0       LF_ProcessEditorInput      000000018001ebd0 f   exported.obj
 0001:0001dc50       LF_ProcessHostFile         000000018001ec50 f   exported.obj
 0001:0001dd80       LF_ProcessPanelEvent       000000018001ed80 f   exported.obj
 0001:0001de60       LF_ProcessPanelInput       000000018001ee60 f   exported.obj
 0001:0001df40       LF_ProcessSynchroEvent     000000018001ef40 f   exported.obj
 0001:0001e130       LF_ProcessViewerEvent      000000018001f130 f   exported.obj
 0001:0001e1e0       LF_PutFiles                000000018001f1e0 f   exported.obj
 0001:0001e330       LF_RunDefaultScript        000000018001f330 f   exported.obj
 0001:0001e340       LF_SetDirectory            000000018001f340 f   exported.obj
 0001:0001e450       LF_SetFindList             000000018001f450 f   exported.obj
 0001:0001e530       PackMacroValues            000000018001f530 f   exported.obj
 0001:0001e770       PushFarMacroValue          000000018001f770 f   exported.obj
 0001:0001e8d0       PushPluginObject           000000018001f8d0 f   exported.obj
 0001:0001e920       PushPluginPair             000000018001f920 f   exported.obj
 0001:0001ea10       ReplacePluginInfoCollector 000000018001fa10 f   exported.obj
 0001:0001ea50       RunDefaultScript           000000018001fa50 f   exported.obj
 0001:0001ec90       UpdateFileSelection        000000018001fc90 f   exported.obj
 0001:0001ed70       _AddStringToCollector      000000018001fd70 f   exported.obj
 0001:0001edf0       getPluginMenuItems         000000018001fdf0 f   exported.obj
 0001:0001eec0       pcall_msg                  000000018001fec0 f   exported.obj
 0001:0001efc0       traceback                  000000018001ffc0 f   exported.obj
 0001:0001f080       push_flags_table           0000000180020080 f   flags.obj
 0001:0001f100       SetFarColors               0000000180020100 f   keysandcolors.obj
 0001:0001f170       LF_Gsub                    0000000180020170 f   lflua.obj
 0001:0001f2b0       LF_LoadFile                00000001800202b0 f   lflua.obj
 0001:0001f610       luaB_dofileW               0000000180020610 f   lflua.obj
 0001:0001f680       luaB_loadfileW             0000000180020680 f   lflua.obj
 0001:0001f6d0       method_gc                  00000001800206d0 f   lregex.obj
 0001:0001f750       method_tostring            0000000180020750 f   lregex.obj
 0001:0001f7c0       func_Gmatch                00000001800207c0 f   lregex.obj
 0001:0001f7d0       func_GmatchW               00000001800207d0 f   lregex.obj
 0001:0001f7e0       method_bracketscount       00000001800207e0 f   lregex.obj
 0001:0001f860       func_New                   0000000180020860 f   lregex.obj
 0001:0001f8b0       method_find                00000001800208b0 f   lregex.obj
 0001:0001f8c0       func_find                  00000001800208c0 f   lregex.obj
 0001:0001f8d0       method_findW               00000001800208d0 f   lregex.obj
 0001:0001f8e0       func_findW                 00000001800208e0 f   lregex.obj
 0001:0001f8f0       method_match               00000001800208f0 f   lregex.obj
 0001:0001f900       func_match                 0000000180020900 f   lregex.obj
 0001:0001f910       method_matchW              0000000180020910 f   lregex.obj
 0001:0001f930       func_matchW                0000000180020930 f   lregex.obj
 0001:0001f940       method_exec                0000000180020940 f   lregex.obj
 0001:0001f950       func_exec                  0000000180020950 f   lregex.obj
 0001:0001f960       method_execW               0000000180020960 f   lregex.obj
 0001:0001f980       func_execW                 0000000180020980 f   lregex.obj
 0001:0001f9a0       method_gsub                00000001800209a0 f   lregex.obj
 0001:0001f9b0       func_gsub                  00000001800209b0 f   lregex.obj
 0001:0001f9c0       method_gsubW               00000001800209c0 f   lregex.obj
 0001:0001f9d0       func_gsubW                 00000001800209d0 f   lregex.obj
 0001:0001f9e0       _Gmatch                    00000001800209e0 f   lregex.obj
 0001:0001fb00       _regex_gmatch_closure      0000000180020b00 f   lregex.obj
 0001:0001fc40       check_regex_pattern        0000000180020c40 f   lregex.obj
 0001:0001fd20       luaopen_regex              0000000180020d20 f   lregex.obj
 0001:0001fdb0       push_far_regex             0000000180020db0 f   lregex.obj
 0001:0001fe60       regex_gmatch_closure       0000000180020e60 f   lregex.obj
 0001:0001fe70       regex_gmatch_closureW      0000000180020e70 f   lregex.obj
 0001:0001fe80       rx_find_match              0000000180020e80 f   lregex.obj
 0001:000201f0       rx_gsub                    00000001800211f0 f   lregex.obj
 0001:00020b00       Open_Luamacro              0000000180021b00 f   luamacro.obj
 0001:00020f00       far_FarMacroCallToLua      0000000180021f00 f   luamacro.obj
 0001:00020fa0       far_MacroCallFar           0000000180021fa0 f   luamacro.obj
 0001:00021210       uc_len                     0000000180022210 f   lusercontrol.obj
 0001:00021530       CheckFarUserControl        0000000180022530 f   lusercontrol.obj
 0001:00021540       luaopen_usercontrol        0000000180022540 f   lusercontrol.obj
 0001:00021590       CreateRegKey               0000000180022590 f   reg.obj
 0001:000215f0       OpenRegKey                 00000001800225f0 f   reg.obj
 0001:00021630       SetRegKeyArr               0000000180022630 f   reg.obj
 0001:000216f0       SetRegKeyDword             00000001800226f0 f   reg.obj
 0001:000217b0       SetRegKeyStr               00000001800227b0 f   reg.obj
 0001:0002ccf0       ConvertLuaValue            000000018002dcf0 f   service.obj
 0001:0002ce30       CreateList                 000000018002de30 f   service.obj
 0001:0002d030       DeleteLuaStateTimerQueue   000000018002e030 f   service.obj
 0001:0002d060       DialogHandleEqual          000000018002e060 f   service.obj
 0001:0002d0c0       DllMain                    000000018002e0c0 f   service.obj
 0001:0002d310       FillInputRecord            000000018002e310 f   service.obj
 0001:0002d870       GetFarColor                000000018002e870 f   service.obj
 0001:0002d9e0       GetFlagCombination         000000018002e9e0 f   service.obj
 0001:0002dc00       GetFlagsFromTable          000000018002ec00 f   service.obj
 0001:0002dc40       GetLuaStateTimerQueue      000000018002ec40 f   service.obj
 0001:0002dc90       GetPluginData              000000018002ec90 f   service.obj
 0001:0002dcb0       IsLuaJIT                   000000018002ecb0 f   service.obj
 0001:0002dcc0       LF_DlgProc                 000000018002ecc0 f   service.obj
 0001:0002deb0       LF_DoFile                  000000018002eeb0 f   service.obj
 0001:0002df80       LF_Error                   000000018002ef80 f   service.obj
 0001:0002e080       LF_GetLuafarAPI            000000018002f080 f   service.obj
 0001:0002e0c0       LF_InitLuaState1           000000018002f0c0 f   service.obj
 0001:0002e350       LF_InitLuaState2           000000018002f350 f   service.obj
 0001:0002e420       LF_MacroCallback           000000018002f420 f   service.obj
 0001:0002e430       LF_Message                 000000018002f430 f   service.obj
 0001:0002e920       _guard_check_icall_nop     000000018002f920 f   LIBCMT:guard_support.obj
 0001:0002e920       LF_ProcessEnvVars          000000018002f920 f   service.obj
 0001:0002e930       LF_RunLuafarInit           000000018002f930 f   service.obj
 0001:0002ea10       MacroAddCallback           000000018002fa10 f   service.obj
 0001:0002ec70       NewDialogData              000000018002fc70 f   service.obj
 0001:0002ed30       NewVirtualKeyTable         000000018002fd30 f   service.obj
 0001:0002edf0       OptFlags                   000000018002fdf0 f   service.obj
 0001:0002ee60       OptHandle                  000000018002fe60 f   service.obj
 0001:0002efd0       ProcessDNResult            000000018002ffd0 f   service.obj
 0001:0002f430       PushDMParams               0000000180030430 f   service.obj
 0001:0002f530       PushDNParams               0000000180030530 f   service.obj
 0001:0002fb40       PushFarColor               0000000180030b40 f   service.obj
 0001:0002fbc0       PushInputRecord            0000000180030bc0 f   service.obj
 0001:0002fda0       PushPanelItem              0000000180030da0 f   service.obj
 0001:00030010       PushPanelItems             0000000180031010 f   service.obj
 0001:00030340       PutFlagsToTable            0000000180031340 f   service.obj
 0001:00030c50       TimerCallback              0000000180031c50 f   service.obj
 0001:00031300       dir_exist                  0000000180032300 f   service.obj
 0001:00031330       fprintf                    0000000180032330 f i service.obj
 0001:00031b10       luaopen_luafar3            0000000180032b10 f   service.obj
 0001:00031d00       pushFileTime               0000000180032d00 f   service.obj
 0001:000326f0       _snwprintf                 00000001800336f0 f i slnunico.obj
 0001:00032750       luaopen_unicode            0000000180033750 f   slnunico.obj
 0001:000345b0       luaopen_utf8               00000001800355b0 f   lutf8lib.obj
 0001:00036d50       __local_stdio_scanf_options 0000000180037d50 f i uliolib51.obj
 0001:00036e20       fscanf                     0000000180037e20 f i uliolib51.obj
 0001:000374f0       luaopen_uio                00000001800384f0 f   uliolib51.obj
 0001:00038700       luaopen_upackage           0000000180039700 f   uloadlib51.obj
 0001:00038ac0       ustring_WideCharToMultiByte 0000000180039ac0 f   ustring.obj
 0001:00038c50       ustring_MultiByteToWideChar 0000000180039c50 f   ustring.obj
 0001:00038de0       ustring_OemToUtf8          0000000180039de0 f   ustring.obj
 0001:00038ee0       ustring_Utf8ToOem          0000000180039ee0 f   ustring.obj
 0001:00038fd0       ustring_Utf16ToUtf8        0000000180039fd0 f   ustring.obj
 0001:00039020       ustring_Utf8ToUtf16        000000018003a020 f   ustring.obj
 0001:00039100       ustring_GetACP             000000018003a100 f   ustring.obj
 0001:00039130       ustring_GetOEMCP           000000018003a130 f   ustring.obj
 0001:00039160       ustring_GetConsoleCP       000000018003a160 f   ustring.obj
 0001:00039190       ustring_SetConsoleCP       000000018003a190 f   ustring.obj
 0001:00039200       ustring_GetConsoleOutputCP 000000018003a200 f   ustring.obj
 0001:00039230       ustring_SetConsoleOutputCP 000000018003a230 f   ustring.obj
 0001:000392a0       ustring_EnumSystemCodePages 000000018003a2a0 f   ustring.obj
 0001:00039330       ustring_GetCPInfo          000000018003a330 f   ustring.obj
 0001:000395d0       ustring_GetLogicalDriveStrings 000000018003a5d0 f   ustring.obj
 0001:000396f0       ustring_GetDriveType       000000018003a6f0 f   ustring.obj
 0001:00039800       ustring_Uuid               000000018003a800 f   ustring.obj
 0001:000398d0       ustring_SearchPath         000000018003a8d0 f   ustring.obj
 0001:00039ae0       ustring_GlobalMemoryStatus 000000018003aae0 f   ustring.obj
 0001:00039cf0       ustring_Sleep              000000018003acf0 f   ustring.obj
 0001:00039d10       ustring_SetFileAttr        000000018003ad10 f   ustring.obj
 0001:00039f40       ustring_GetFileAttr        000000018003af40 f   ustring.obj
 0001:0003a060       ustring_SHGetFolderPath    000000018003b060 f   ustring.obj
 0001:0003a1a0       ustring_sub                000000018003b1a0 f   ustring.obj
 0001:0003a260       ustring_len                000000018003b260 f   ustring.obj
 0001:0003a510       ustring_GetCurrentDir      000000018003b510 f   ustring.obj
 0001:0003a6a0       ustring_SetCurrentDir      000000018003b6a0 f   ustring.obj
 0001:0003a7c0       ustring_GetKeyState        000000018003b7c0 f   ustring.obj
 0001:0003a810       DecodeAttributes           000000018003b810 f   ustring.obj
 0001:0003a910       EnumCodePagesProc          000000018003b910 f   ustring.obj
 0001:0003a980       GetBoolFromTable           000000018003b980 f   ustring.obj
 0001:0003a9d0       GetOptBoolFromTable        000000018003b9d0 f   ustring.obj
 0001:0003aa30       GetOptIntFromArray         000000018003ba30 f   ustring.obj
 0001:0003aa90       GetOptIntFromTable         000000018003ba90 f   ustring.obj
 0001:0003aaf0       GetOptNumFromTable         000000018003baf0 f   ustring.obj
 0001:0003ab50       PushAttrString             000000018003bb50 f   ustring.obj
 0001:0003ac40       PutAttrToTable             000000018003bc40 f   ustring.obj
 0001:0003ac70       PutBoolToTable             000000018003bc70 f   ustring.obj
 0001:0003acb0       PutIntToArray              000000018003bcb0 f   ustring.obj
 0001:0003acf0       PutIntToTable              000000018003bcf0 f   ustring.obj
 0001:0003ad30       PutLStrToTable             000000018003bd30 f   ustring.obj
 0001:0003ad70       PutNumToTable              000000018003bd70 f   ustring.obj
 0001:0003adb0       PutStrToArray              000000018003bdb0 f   ustring.obj
 0001:0003adf0       PutStrToTable              000000018003bdf0 f   ustring.obj
 0001:0003ae30       PutWStrToArray             000000018003be30 f   ustring.obj
 0001:0003ae90       PutWStrToTable             000000018003be90 f   ustring.obj
 0001:0003aed0       SysErrorReturn             000000018003bed0 f   ustring.obj
 0001:0003af10       check_utf16_string         000000018003bf10 f   ustring.obj
 0001:0003af40       check_utf8_string          000000018003bf40 f   ustring.obj
 0001:0003af70       convert_multibyte_string   000000018003bf70 f   ustring.obj
 0001:0003b0a0       luaopen_ustring            000000018003c0a0 f   ustring.obj
 0001:0003b100       opt_utf16_string           000000018003c100 f   ustring.obj
 0001:0003b110       opt_utf8_string            000000018003c110 f   ustring.obj
 0001:0003b220       push_multibyte_string      000000018003c220 f   ustring.obj
 0001:0003b330       push_utf16_string          000000018003c330 f   ustring.obj
 0001:0003b360       push_utf8_string           000000018003c360 f   ustring.obj
 0001:0003b390       pusherror                  000000018003c390 f   ustring.obj
 0001:0003b3b0       pusherrorcode              000000018003c3b0 f   ustring.obj
 0001:0003b450       utf8_to_utf16              000000018003c450 f   ustring.obj
 0001:0003b480       GetAttrFromTable           000000018003c480 f   util.obj
 0001:0003b4e0       GetFileSizeFromTable       000000018003c4e0 f   util.obj
 0001:0003b570       GetFileTimeFromTable       000000018003c570 f   util.obj
 0001:0003b620       GetIntFromArray            000000018003c620 f   util.obj
 0001:0003b6e0       PutFileTimeToTable         000000018003c6e0 f   util.obj
 0001:0003b790       luaLF_FieldError           000000018003c790 f   util.obj
 0001:0003b810       luaLF_SlotError            000000018003c810 f   util.obj
 0001:0003cf40       win_WriteConsole           000000018003df40 f   win.obj
 0001:0003d080       win_IsWinVersion           000000018003e080 f   win.obj
 0001:0003da80       luaopen_win                000000018003ea80 f   win.obj
 0001:0003dd1c       lua_gettop                 000000018003ed1c f   lua51:lua51.dll
 0001:0003dd22       lua_settop                 000000018003ed22 f   lua51:lua51.dll
 0001:0003dd28       lua_type                   000000018003ed28 f   lua51:lua51.dll
 0001:0003dd2e       lua_rawequal               000000018003ed2e f   lua51:lua51.dll
 0001:0003dd34       lua_tonumber               000000018003ed34 f   lua51:lua51.dll
 0001:0003dd3a       lua_tolstring              000000018003ed3a f   lua51:lua51.dll
 0001:0003dd40       lua_touserdata             000000018003ed40 f   lua51:lua51.dll
 0001:0003dd46       lua_pushnil                000000018003ed46 f   lua51:lua51.dll
 0001:0003dd4c       lua_pushnumber             000000018003ed4c f   lua51:lua51.dll
 0001:0003dd52       lua_pushstring             000000018003ed52 f   lua51:lua51.dll
 0001:0003dd58       lua_pushboolean            000000018003ed58 f   lua51:lua51.dll
 0001:0003dd5e       lua_getfield               000000018003ed5e f   lua51:lua51.dll
 0001:0003dd64       lua_newuserdata            000000018003ed64 f   lua51:lua51.dll
 0001:0003dd6a       lua_getmetatable           000000018003ed6a f   lua51:lua51.dll
 0001:0003dd70       lua_setmetatable           000000018003ed70 f   lua51:lua51.dll
 0001:0003dd76       luaL_register              000000018003ed76 f   lua51:lua51.dll
 0001:0003dd7c       luaL_argerror              000000018003ed7c f   lua51:lua51.dll
 0001:0003dd82       luaL_checkinteger          000000018003ed82 f   lua51:lua51.dll
 0001:0003dd88       luaL_newmetatable          000000018003ed88 f   lua51:lua51.dll
 0001:0003dd8e       lua_pushvalue              000000018003ed8e f   lua51:lua51.dll
 0001:0003dd94       lua_remove                 000000018003ed94 f   lua51:lua51.dll
 0001:0003dd9a       lua_insert                 000000018003ed9a f   lua51:lua51.dll
 0001:0003dda0       lua_isnumber               000000018003eda0 f   lua51:lua51.dll
 0001:0003dda6       lua_isstring               000000018003eda6 f   lua51:lua51.dll
 0001:0003ddac       lua_tointeger              000000018003edac f   lua51:lua51.dll
 0001:0003ddb2       lua_toboolean              000000018003edb2 f   lua51:lua51.dll
 0001:0003ddb8       lua_objlen                 000000018003edb8 f   lua51:lua51.dll
 0001:0003ddbe       lua_topointer              000000018003edbe f   lua51:lua51.dll
 0001:0003ddc4       lua_pushinteger            000000018003edc4 f   lua51:lua51.dll
 0001:0003ddca       lua_pushlstring            000000018003edca f   lua51:lua51.dll
 0001:0003ddd0       lua_pushcclosure           000000018003edd0 f   lua51:lua51.dll
 0001:0003ddd6       lua_pushlightuserdata      000000018003edd6 f   lua51:lua51.dll
 0001:0003dddc       lua_gettable               000000018003eddc f   lua51:lua51.dll
 0001:0003dde2       lua_rawget                 000000018003ede2 f   lua51:lua51.dll
 0001:0003dde8       lua_rawgeti                000000018003ede8 f   lua51:lua51.dll
 0001:0003ddee       lua_createtable            000000018003edee f   lua51:lua51.dll
 0001:0003ddf4       lua_setfield               000000018003edf4 f   lua51:lua51.dll
 0001:0003ddfa       lua_rawset                 000000018003edfa f   lua51:lua51.dll
 0001:0003de00       lua_rawseti                000000018003ee00 f   lua51:lua51.dll
 0001:0003de06       lua_call                   000000018003ee06 f   lua51:lua51.dll
 0001:0003de0c       lua_pcall                  000000018003ee0c f   lua51:lua51.dll
 0001:0003de12       lua_gc                     000000018003ee12 f   lua51:lua51.dll
 0001:0003de18       luaL_ref                   000000018003ee18 f   lua51:lua51.dll
 0001:0003de1e       luaL_unref                 000000018003ee1e f   lua51:lua51.dll
 0001:0003de24       luaL_loadstring            000000018003ee24 f   lua51:lua51.dll
 0001:0003de2a       lua_pushfstring            000000018003ee2a f   lua51:lua51.dll
 0001:0003de30       lua_load                   000000018003ee30 f   lua51:lua51.dll
 0001:0003de36       lua_error                  000000018003ee36 f   lua51:lua51.dll
 0001:0003de3c       lua_concat                 000000018003ee3c f   lua51:lua51.dll
 0001:0003de42       luaL_buffinit              000000018003ee42 f   lua51:lua51.dll
 0001:0003de48       luaL_addlstring            000000018003ee48 f   lua51:lua51.dll
 0001:0003de4e       luaL_pushresult            000000018003ee4e f   lua51:lua51.dll
 0001:0003de54       lua_replace                000000018003ee54 f   lua51:lua51.dll
 0001:0003de5a       lua_checkstack             000000018003ee5a f   lua51:lua51.dll
 0001:0003de60       luaL_checklstring          000000018003ee60 f   lua51:lua51.dll
 0001:0003de66       luaL_optlstring            000000018003ee66 f   lua51:lua51.dll
 0001:0003de6c       luaL_optinteger            000000018003ee6c f   lua51:lua51.dll
 0001:0003de72       luaL_checkudata            000000018003ee72 f   lua51:lua51.dll
 0001:0003de78       luaL_error                 000000018003ee78 f   lua51:lua51.dll
 0001:0003de7e       luaL_addvalue              000000018003ee7e f   lua51:lua51.dll
 0001:0003de84       lua_getstack               000000018003ee84 f   lua51:lua51.dll
 0001:0003de8a       lua_getinfo                000000018003ee8a f   lua51:lua51.dll
 0001:0003de90       luaL_checktype             000000018003ee90 f   lua51:lua51.dll
 0001:0003de96       luaopen_base               000000018003ee96 f   lua51:lua51.dll
 0001:0003de9c       luaopen_table              000000018003ee9c f   lua51:lua51.dll
 0001:0003dea2       luaopen_os                 000000018003eea2 f   lua51:lua51.dll
 0001:0003dea8       luaopen_string             000000018003eea8 f   lua51:lua51.dll
 0001:0003deae       luaopen_math               000000018003eeae f   lua51:lua51.dll
 0001:0003deb4       luaopen_debug              000000018003eeb4 f   lua51:lua51.dll
 0001:0003deba       lua_getfenv                000000018003eeba f   lua51:lua51.dll
 0001:0003dec0       lua_settable               000000018003eec0 f   lua51:lua51.dll
 0001:0003dec6       lua_setfenv                000000018003eec6 f   lua51:lua51.dll
 0001:0003decc       lua_next                   000000018003eecc f   lua51:lua51.dll
 0001:0003ded2       lua_getallocf              000000018003eed2 f   lua51:lua51.dll
 0001:0003ded8       lua_setallocf              000000018003eed8 f   lua51:lua51.dll
 0001:0003dede       luaL_typerror              000000018003eede f   lua51:lua51.dll
 0001:0003dee4       luaL_checknumber           000000018003eee4 f   lua51:lua51.dll
 0001:0003deea       luaL_optnumber             000000018003eeea f   lua51:lua51.dll
 0001:0003def0       luaL_checkany              000000018003eef0 f   lua51:lua51.dll
 0001:0003def6       luaL_findtable             000000018003eef6 f   lua51:lua51.dll
 0001:0003defc       lua_dump                   000000018003eefc f   lua51:lua51.dll
 0001:0003df02       luaL_prepbuffer            000000018003ef02 f   lua51:lua51.dll
 0001:0003df08       lua_typename               000000018003ef08 f   lua51:lua51.dll
 0001:0003df0e       luaL_checkstack            000000018003ef0e f   lua51:lua51.dll
 0001:0003df14       lua_tocfunction            000000018003ef14 f   lua51:lua51.dll
 0001:0003df1a       luaL_checkoption           000000018003ef1a f   lua51:lua51.dll
 0001:0003df20       lua_iscfunction            000000018003ef20 f   lua51:lua51.dll
 0001:0003df26       luaL_gsub                  000000018003ef26 f   lua51:lua51.dll
 0001:0003df2c       lua_isuserdata             000000018003ef2c f   lua51:lua51.dll
 0001:0003e264       _DllMainCRTStartup         000000018003f264 f   LIBCMT:dll_dllmain.obj
 0001:0003e2a4       __security_init_cookie     000000018003f2a4 f   LIBCMT:gs_support.obj
 0001:0003e350       ?__scrt_initialize_type_info@@YAXXZ 000000018003f350 f   LIBCMT:tncleanup.obj
 0001:0003e360       ?__scrt_uninitialize_type_info@@YAXXZ 000000018003f360 f   LIBCMT:tncleanup.obj
 0001:0003e36c       __scrt_initialize_default_local_stdio_options 000000018003f36c f   LIBCMT:default_local_stdio_options.obj
 0001:0003e388       __scrt_acquire_startup_lock 000000018003f388 f   LIBCMT:utility.obj
 0001:0003e3c4       __scrt_dllmain_after_initialize_c 000000018003f3c4 f   LIBCMT:utility.obj
 0001:0003e3f8       __scrt_dllmain_before_initialize_c 000000018003f3f8 f   LIBCMT:utility.obj
 0001:0003e410       __scrt_dllmain_crt_thread_attach 000000018003f410 f   LIBCMT:utility.obj
 0001:0003e438       __scrt_dllmain_crt_thread_detach 000000018003f438 f   LIBCMT:utility.obj
 0001:0003e450       __scrt_dllmain_exception_filter 000000018003f450 f   LIBCMT:utility.obj
 0001:0003e4b0       __scrt_dllmain_uninitialize_c 000000018003f4b0 f   LIBCMT:utility.obj
 0001:0003e4e0       __scrt_dllmain_uninitialize_critical 000000018003f4e0 f   LIBCMT:utility.obj
 0001:0003e4f4       __scrt_initialize_crt      000000018003f4f4 f   LIBCMT:utility.obj
 0001:0003e540       __scrt_initialize_onexit_tables 000000018003f540 f   LIBCMT:utility.obj
 0001:0003e618       __scrt_is_nonwritable_in_current_image 000000018003f618 f   LIBCMT:utility.obj
 0001:0003e6b4       __scrt_release_startup_lock 000000018003f6b4 f   LIBCMT:utility.obj
 0001:0003e6d8       __scrt_uninitialize_crt    000000018003f6d8 f   LIBCMT:utility.obj
 0001:0003e704       __scrt_get_dyn_tls_init_callback 000000018003f704 f   LIBCMT:dyn_tls_init.obj
 0001:0003e70c       __crt_debugger_hook        000000018003f70c f   LIBCMT:utility_desktop.obj
 0001:0003e714       __scrt_fastfail            000000018003f714 f   LIBCMT:utility_desktop.obj
 0001:0003e860       _RTC_Initialize            000000018003f860 f   LIBCMT:initsect.obj
 0001:0003e89c       _RTC_Terminate             000000018003f89c f   LIBCMT:initsect.obj
 0001:0003e8d8       __isa_available_init       000000018003f8d8 f   LIBCMT:cpu_disp.obj
 0001:0003ea54       _get_startup_argv_mode     000000018003fa54 f   LIBCMT:argv_mode.obj
 0001:0003ea5c       __scrt_is_ucrt_dll_in_use  000000018003fa5c f   LIBCMT:ucrt_detection.obj
 0001:0003ea70       wcsrchr                    000000018003fa70 f   libvcruntime:wcsrchr.obj
 0001:0003eb40       memcpy_repmovs             000000018003fb40 f   libvcruntime:memcpy.obj
 0001:0003eb60       memcpy                     000000018003fb60 f   libvcruntime:memcpy.obj
 0001:0003eb60       memmove                    000000018003fb60 f   libvcruntime:memcpy.obj
 0001:0003efa0       memset_repmovs             000000018003ffa0 f   libvcruntime:memset.obj
 0001:0003efc0       memset                     000000018003ffc0 f   libvcruntime:memset.obj
 0001:0003f150       wcsstr                     0000000180040150 f   libvcruntime:wcsstr.obj
 0001:0003f36c       strchr                     000000018004036c f   libvcruntime:strchr.obj
 0001:0003f3f8       wcschr                     00000001800403f8 f   libvcruntime:wcschr.obj
 0001:0003f4a0       memchr                     00000001800404a0 f   libvcruntime:memchr.obj
 0001:0003f520       memcmp                     0000000180040520 f   libvcruntime:memcmp.obj
 0001:0003f5e8       strrchr                    00000001800405e8 f   libvcruntime:strrchr.obj
 0001:0003f734       __C_specific_handler       0000000180040734 f   libvcruntime:riscchandler.obj
 0001:0003f940       __std_type_info_destroy_list 0000000180040940 f   libvcruntime:std_type_info.obj
 0001:0003f96c       __vcrt_initialize          000000018004096c f   libvcruntime:initialization.obj
 0001:0003f9a0       __vcrt_thread_attach       00000001800409a0 f   libvcruntime:initialization.obj
 0001:0003f9b4       __vcrt_thread_detach       00000001800409b4 f   libvcruntime:initialization.obj
 0001:0003f9c8       __vcrt_uninitialize        00000001800409c8 f   libvcruntime:initialization.obj
 0001:0003f9e8       __vcrt_uninitialize_critical 00000001800409e8 f   libvcruntime:initialization.obj
 0001:0003fa10       _NLG_Notify                0000000180040a10 f   libvcruntime:notify.obj
 0001:0003fa30       __NLG_Dispatch2            0000000180040a30 f   libvcruntime:notify.obj
 0001:0003fa40       __NLG_Return2              0000000180040a40 f   libvcruntime:notify.obj
 0001:0003fa44       __except_validate_context_record 0000000180040a44 f   libvcruntime:jbcxrval.obj
 0001:0003fa7c       __DestructExceptionObject  0000000180040a7c f   libvcruntime:ehhelpers.obj
 0001:0003faf0       ?_CallMemberFunction0@@YAXQEAX0@Z 0000000180040af0 f i libvcruntime:ehhelpers.obj
 0001:0003faf4       __vcrt_freefls             0000000180040af4 f   libvcruntime:per_thread_data.obj
 0001:0003fb14       __vcrt_freeptd             0000000180040b14 f   libvcruntime:per_thread_data.obj
 0001:0003fb64       __vcrt_getptd_noexit       0000000180040b64 f   libvcruntime:per_thread_data.obj
 0001:0003fc30       __vcrt_initialize_ptd      0000000180040c30 f   libvcruntime:per_thread_data.obj
 0001:0003fc84       __vcrt_uninitialize_ptd    0000000180040c84 f   libvcruntime:per_thread_data.obj
 0001:0003fca8       __vcrt_initialize_locks    0000000180040ca8 f   libvcruntime:locks.obj
 0001:0003fcf0       __vcrt_uninitialize_locks  0000000180040cf0 f   libvcruntime:locks.obj
 0001:0003ff00       __vcrt_FlsAlloc            0000000180040f00 f   libvcruntime:winapi_downlevel.obj
 0001:0003ff48       __vcrt_FlsFree             0000000180040f48 f   libvcruntime:winapi_downlevel.obj
 0001:0003ff90       __vcrt_FlsGetValue         0000000180040f90 f   libvcruntime:winapi_downlevel.obj
 0001:0003ffd8       __vcrt_FlsSetValue         0000000180040fd8 f   libvcruntime:winapi_downlevel.obj
 0001:0004002c       __vcrt_InitializeCriticalSectionEx 000000018004102c f   libvcruntime:winapi_downlevel.obj
 0001:00040090       __vcrt_initialize_winapi_thunks 0000000180041090 f   libvcruntime:winapi_downlevel.obj
 0001:000400c0       __vcrt_uninitialize_winapi_thunks 00000001800410c0 f   libvcruntime:winapi_downlevel.obj
 0001:00040100       __vcrt_initialize_pure_virtual_call_handler 0000000180041100 f   libvcruntime:purevirt_data.obj
 0001:00040120       _CallSettingFrame          0000000180041120 f   libvcruntime:handlers.obj
 0001:00040170       _CallSettingFrameEncoded   0000000180041170 f   libvcruntime:handlers.obj
 0001:00040598       ??$ensure_buffer_is_big_enough@D@formatting_buffer@__crt_stdio_output@@QEAA_N_K@Z 0000000180041598 f i libucrt:output.obj
 0001:00040640       ??$ensure_buffer_is_big_enough@_W@formatting_buffer@__crt_stdio_output@@QEAA_N_K@Z 0000000180041640 f i libucrt:output.obj
 0001:000406ec       ??$is_wide_character_specifier@_W@__crt_stdio_output@@YA_N_K_WW4length_modifier@0@@Z 00000001800416ec f i libucrt:output.obj
 0001:0004072c       ??$type_case_integer_parse_into_buffer@I@?$output_processor@DV?$string_output_adapter@D@__crt_stdio_output@@V?$standard_base@DV?$string_output_adapter@D@__crt_stdio_output@@@2@@__crt_stdio_output@@AEAAXII_N@Z 000000018004172c f i libucrt:output.obj
 0001:0004072c       ??$type_case_integer_parse_into_buffer@I@?$output_processor@DV?$stream_output_adapter@D@__crt_stdio_output@@V?$standard_base@DV?$stream_output_adapter@D@__crt_stdio_output@@@2@@__crt_stdio_output@@AEAAXII_N@Z 000000018004172c f i libucrt:output.obj
 0001:000407bc       ??$type_case_integer_parse_into_buffer@I@?$output_processor@_WV?$string_output_adapter@_W@__crt_stdio_output@@V?$standard_base@_WV?$string_output_adapter@_W@__crt_stdio_output@@@2@@__crt_stdio_output@@AEAAXII_N@Z 00000001800417bc f i libucrt:output.obj
 0001:00040860       ??$type_case_integer_parse_into_buffer@_K@?$output_processor@DV?$stream_output_adapter@D@__crt_stdio_output@@V?$standard_base@DV?$stream_output_adapter@D@__crt_stdio_output@@@2@@__crt_stdio_output@@AEAAX_KI_N@Z 0000000180041860 f i libucrt:output.obj
 0001:00040860       ??$type_case_integer_parse_into_buffer@_K@?$output_processor@DV?$string_output_adapter@D@__crt_stdio_output@@V?$standard_base@DV?$string_output_adapter@D@__crt_stdio_output@@@2@@__crt_stdio_output@@AEAAX_KI_N@Z 0000000180041860 f i libucrt:output.obj
 0001:000408f4       ??$type_case_integer_parse_into_buffer@_K@?$output_processor@_WV?$string_output_adapter@_W@__crt_stdio_output@@V?$standard_base@_WV?$string_output_adapter@_W@__crt_stdio_output@@@2@@__crt_stdio_output@@AEAAX_KI_N@Z 00000001800418f4 f i libucrt:output.obj
 0001:00040998       ??$write_multiple_characters@V?$stream_output_adapter@D@__crt_stdio_output@@D@__crt_stdio_output@@YAXAEBV?$stream_output_adapter@D@0@DHQEAH@Z 0000000180041998 f i libucrt:output.obj
 0001:00040a24       ??$write_multiple_characters@V?$string_output_adapter@D@__crt_stdio_output@@D@__crt_stdio_output@@YAXAEBV?$string_output_adapter@D@0@DHQEAH@Z 0000000180041a24 f i libucrt:output.obj
 0001:00040a9c       ??$write_multiple_characters@V?$string_output_adapter@_W@__crt_stdio_output@@D@__crt_stdio_output@@YAXAEBV?$string_output_adapter@_W@0@DHQEAH@Z 0000000180041a9c f i libucrt:output.obj
 0001:00040b18       ??0_LocaleUpdate@@QEAA@QEAU__crt_locale_pointers@@@Z 0000000180041b18 f i libucrt:output.obj
 0001:00040ce4       ?crop_zeroes@__crt_stdio_output@@YAXPEADQEAU__crt_locale_pointers@@@Z 0000000180041ce4 f i libucrt:output.obj
 0001:00040d50       ?force_decimal_point@__crt_stdio_output@@YAXPEADQEAU__crt_locale_pointers@@@Z 0000000180041d50 f i libucrt:output.obj
 0001:00040dc0       ?parse_int_from_format_string@?$output_processor@DV?$string_output_adapter@D@__crt_stdio_output@@V?$standard_base@DV?$string_output_adapter@D@__crt_stdio_output@@@2@@__crt_stdio_output@@AEAA_NQEAH@Z 0000000180041dc0 f i libucrt:output.obj
 0001:00040dc0       ?parse_int_from_format_string@?$output_processor@DV?$stream_output_adapter@D@__crt_stdio_output@@V?$standard_base@DV?$stream_output_adapter@D@__crt_stdio_output@@@2@@__crt_stdio_output@@AEAA_NQEAH@Z 0000000180041dc0 f i libucrt:output.obj
 0001:00040e64       ?parse_int_from_format_string@?$output_processor@_WV?$string_output_adapter@_W@__crt_stdio_output@@V?$standard_base@_WV?$string_output_adapter@_W@__crt_stdio_output@@@2@@__crt_stdio_output@@AEAA_NQEAH@Z 0000000180041e64 f i libucrt:output.obj
 0001:00040f08       ?process@?$output_processor@DV?$stream_output_adapter@D@__crt_stdio_output@@V?$standard_base@DV?$stream_output_adapter@D@__crt_stdio_output@@@2@@__crt_stdio_output@@QEAAHXZ 0000000180041f08 f i libucrt:output.obj
 0001:00041120       ?process@?$output_processor@DV?$string_output_adapter@D@__crt_stdio_output@@V?$standard_base@DV?$string_output_adapter@D@__crt_stdio_output@@@2@@__crt_stdio_output@@QEAAHXZ 0000000180042120 f i libucrt:output.obj
 0001:0004132c       ?process@?$output_processor@_WV?$string_output_adapter@_W@__crt_stdio_output@@V?$standard_base@_WV?$string_output_adapter@_W@__crt_stdio_output@@@2@@__crt_stdio_output@@QEAAHXZ 000000018004232c f i libucrt:output.obj
 0001:000415a8       ?state_case_normal@?$output_processor@DV?$stream_output_adapter@D@__crt_stdio_output@@V?$standard_base@DV?$stream_output_adapter@D@__crt_stdio_output@@@2@@__crt_stdio_output@@AEAA_NXZ 00000001800425a8 f i libucrt:output.obj
 0001:00041618       ?state_case_normal@?$output_processor@DV?$string_output_adapter@D@__crt_stdio_output@@V?$standard_base@DV?$string_output_adapter@D@__crt_stdio_output@@@2@@__crt_stdio_output@@AEAA_NXZ 0000000180042618 f i libucrt:output.obj
 0001:0004168c       ?state_case_normal_tchar@?$output_processor@DV?$stream_output_adapter@D@__crt_stdio_output@@V?$standard_base@DV?$stream_output_adapter@D@__crt_stdio_output@@@2@@__crt_stdio_output@@AEAA_ND@Z 000000018004268c f i libucrt:output.obj
 0001:00041730       ?state_case_normal_tchar@?$output_processor@DV?$string_output_adapter@D@__crt_stdio_output@@V?$standard_base@DV?$string_output_adapter@D@__crt_stdio_output@@@2@@__crt_stdio_output@@AEAA_ND@Z 0000000180042730 f i libucrt:output.obj
 0001:000417d8       ?state_case_size@?$output_processor@DV?$stream_output_adapter@D@__crt_stdio_output@@V?$standard_base@DV?$stream_output_adapter@D@__crt_stdio_output@@@2@@__crt_stdio_output@@AEAA_NXZ 00000001800427d8 f i libucrt:output.obj
 0001:0004194c       ?state_case_size@?$output_processor@DV?$string_output_adapter@D@__crt_stdio_output@@V?$standard_base@DV?$string_output_adapter@D@__crt_stdio_output@@@2@@__crt_stdio_output@@AEAA_NXZ 000000018004294c f i libucrt:output.obj
 0001:00041ac0       ?state_case_size@?$output_processor@_WV?$string_output_adapter@_W@__crt_stdio_output@@V?$standard_base@_WV?$string_output_adapter@_W@__crt_stdio_output@@@2@@__crt_stdio_output@@AEAA_NXZ 0000000180042ac0 f i libucrt:output.obj
 0001:00041c58       ?state_case_type@?$output_processor@DV?$stream_output_adapter@D@__crt_stdio_output@@V?$standard_base@DV?$stream_output_adapter@D@__crt_stdio_output@@@2@@__crt_stdio_output@@AEAA_NXZ 0000000180042c58 f i libucrt:output.obj
 0001:00041edc       ?state_case_type@?$output_processor@DV?$string_output_adapter@D@__crt_stdio_output@@V?$standard_base@DV?$string_output_adapter@D@__crt_stdio_output@@@2@@__crt_stdio_output@@AEAA_NXZ 0000000180042edc f i libucrt:output.obj
 0001:00042144       ?state_case_type@?$output_processor@_WV?$string_output_adapter@_W@__crt_stdio_output@@V?$standard_base@_WV?$string_output_adapter@_W@__crt_stdio_output@@@2@@__crt_stdio_output@@AEAA_NXZ 0000000180043144 f i libucrt:output.obj
 0001:00042410       ?type_case_Z@?$output_processor@DV?$stream_output_adapter@D@__crt_stdio_output@@V?$standard_base@DV?$stream_output_adapter@D@__crt_stdio_output@@@2@@__crt_stdio_output@@AEAA_NXZ 0000000180043410 f i libucrt:output.obj
 0001:00042410       ?type_case_Z@?$output_processor@DV?$string_output_adapter@D@__crt_stdio_output@@V?$standard_base@DV?$string_output_adapter@D@__crt_stdio_output@@@2@@__crt_stdio_output@@AEAA_NXZ 0000000180043410 f i libucrt:output.obj
 0001:00042488       ?type_case_Z@?$output_processor@_WV?$string_output_adapter@_W@__crt_stdio_output@@V?$standard_base@_WV?$string_output_adapter@_W@__crt_stdio_output@@@2@@__crt_stdio_output@@AEAA_NXZ 0000000180043488 f i libucrt:output.obj
 0001:00042504       ?type_case_a@?$output_processor@DV?$string_output_adapter@D@__crt_stdio_output@@V?$standard_base@DV?$string_output_adapter@D@__crt_stdio_output@@@2@@__crt_stdio_output@@AEAA_NXZ 0000000180043504 f i libucrt:output.obj
 0001:00042504       ?type_case_a@?$output_processor@DV?$stream_output_adapter@D@__crt_stdio_output@@V?$standard_base@DV?$stream_output_adapter@D@__crt_stdio_output@@@2@@__crt_stdio_output@@AEAA_NXZ 0000000180043504 f i libucrt:output.obj
 0001:000426c0       ?type_case_a@?$output_processor@_WV?$string_output_adapter@_W@__crt_stdio_output@@V?$standard_base@_WV?$string_output_adapter@_W@__crt_stdio_output@@@2@@__crt_stdio_output@@AEAA_NXZ 00000001800436c0 f i libucrt:output.obj
 0001:000428a0       ?type_case_c_tchar@?$output_processor@DV?$stream_output_adapter@D@__crt_stdio_output@@V?$standard_base@DV?$stream_output_adapter@D@__crt_stdio_output@@@2@@__crt_stdio_output@@AEAA_ND@Z 00000001800438a0 f i libucrt:output.obj
 0001:000428a0       ?type_case_c_tchar@?$output_processor@DV?$string_output_adapter@D@__crt_stdio_output@@V?$standard_base@DV?$string_output_adapter@D@__crt_stdio_output@@@2@@__crt_stdio_output@@AEAA_ND@Z 00000001800438a0 f i libucrt:output.obj
 0001:0004295c       ?type_case_c_tchar@?$output_processor@_WV?$string_output_adapter@_W@__crt_stdio_output@@V?$standard_base@_WV?$string_output_adapter@_W@__crt_stdio_output@@@2@@__crt_stdio_output@@AEAA_N_W@Z 000000018004395c f i libucrt:output.obj
 0001:00042a04       ?type_case_integer@?$output_processor@DV?$string_output_adapter@D@__crt_stdio_output@@V?$standard_base@DV?$string_output_adapter@D@__crt_stdio_output@@@2@@__crt_stdio_output@@AEAA_NI_N@Z 0000000180043a04 f i libucrt:output.obj
 0001:00042a04       ?type_case_integer@?$output_processor@DV?$stream_output_adapter@D@__crt_stdio_output@@V?$standard_base@DV?$stream_output_adapter@D@__crt_stdio_output@@@2@@__crt_stdio_output@@AEAA_NI_N@Z 0000000180043a04 f i libucrt:output.obj
 0001:00042bcc       ?type_case_integer@?$output_processor@_WV?$string_output_adapter@_W@__crt_stdio_output@@V?$standard_base@_WV?$string_output_adapter@_W@__crt_stdio_output@@@2@@__crt_stdio_output@@AEAA_NI_N@Z 0000000180043bcc f i libucrt:output.obj
 0001:00042d98       ?type_case_n@?$output_processor@DV?$stream_output_adapter@D@__crt_stdio_output@@V?$standard_base@DV?$stream_output_adapter@D@__crt_stdio_output@@@2@@__crt_stdio_output@@AEAA_NXZ 0000000180043d98 f i libucrt:output.obj
 0001:00042d98       ?type_case_n@?$output_processor@_WV?$string_output_adapter@_W@__crt_stdio_output@@V?$standard_base@_WV?$string_output_adapter@_W@__crt_stdio_output@@@2@@__crt_stdio_output@@AEAA_NXZ 0000000180043d98 f i libucrt:output.obj
 0001:00042d98       ?type_case_n@?$output_processor@DV?$string_output_adapter@D@__crt_stdio_output@@V?$standard_base@DV?$string_output_adapter@D@__crt_stdio_output@@@2@@__crt_stdio_output@@AEAA_NXZ 0000000180043d98 f i libucrt:output.obj
 0001:00042e74       ?type_case_s@?$output_processor@DV?$string_output_adapter@D@__crt_stdio_output@@V?$standard_base@DV?$string_output_adapter@D@__crt_stdio_output@@@2@@__crt_stdio_output@@AEAA_NXZ 0000000180043e74 f i libucrt:output.obj
 0001:00042e74       ?type_case_s@?$output_processor@DV?$stream_output_adapter@D@__crt_stdio_output@@V?$standard_base@DV?$stream_output_adapter@D@__crt_stdio_output@@@2@@__crt_stdio_output@@AEAA_NXZ 0000000180043e74 f i libucrt:output.obj
 0001:00042f0c       ?type_case_s@?$output_processor@_WV?$string_output_adapter@_W@__crt_stdio_output@@V?$standard_base@_WV?$string_output_adapter@_W@__crt_stdio_output@@@2@@__crt_stdio_output@@AEAA_NXZ 0000000180043f0c f i libucrt:output.obj
 0001:00042fd4       ?validate_stream_is_ansi_if_required@?$__acrt_stdio_char_traits@D@@SA_NQEAU_iobuf@@@Z 0000000180043fd4 f i libucrt:output.obj
 0001:00043070       ?write_stored_string_tchar@?$output_processor@DV?$stream_output_adapter@D@__crt_stdio_output@@V?$standard_base@DV?$stream_output_adapter@D@__crt_stdio_output@@@2@@__crt_stdio_output@@AEAA_ND@Z 0000000180044070 f i libucrt:output.obj
 0001:00043194       ?write_stored_string_tchar@?$output_processor@DV?$string_output_adapter@D@__crt_stdio_output@@V?$standard_base@DV?$string_output_adapter@D@__crt_stdio_output@@@2@@__crt_stdio_output@@AEAA_ND@Z 0000000180044194 f i libucrt:output.obj
 0001:0004326c       ?write_stored_string_tchar@?$output_processor@_WV?$string_output_adapter@_W@__crt_stdio_output@@V?$standard_base@_WV?$string_output_adapter@_W@__crt_stdio_output@@@2@@__crt_stdio_output@@AEAA_N_W@Z 000000018004426c f i libucrt:output.obj
 0001:00043358       ?write_string@?$string_output_adapter@D@__crt_stdio_output@@QEBAXQEBDHQEAHAEAV__crt_deferred_errno_cache@@@Z 0000000180044358 f i libucrt:output.obj
 0001:000433fc       ?write_string@?$string_output_adapter@_W@__crt_stdio_output@@QEBAXQEB_WHQEAHAEAV__crt_deferred_errno_cache@@@Z 00000001800443fc f i libucrt:output.obj
 0001:000434a4       ?write_string_impl@?$output_adapter_common@DV?$stream_output_adapter@D@__crt_stdio_output@@@__crt_stdio_output@@IEBAXQEBDHQEAHAEAV__crt_deferred_errno_cache@@@Z 00000001800444a4 f i libucrt:output.obj
 0001:0004359c       __stdio_common_vfprintf    000000018004459c f   libucrt:output.obj
 0001:00043628       __stdio_common_vsprintf    0000000180044628 f   libucrt:output.obj
 0001:00043630       __stdio_common_vswprintf   0000000180044630 f   libucrt:output.obj
 0001:00043638       _wcsdup                    0000000180044638 f   libucrt:wcsdup.obj
 0001:00043638       wcsdup                     0000000180044638 f   libucrt:wcsdup.obj
 0001:000436bc       free                       00000001800446bc f   libucrt:free.obj
 0001:000436d0       malloc                     00000001800446d0 f   libucrt:malloc.obj
 0001:000437a4       _wfopen                    00000001800447a4 f   libucrt:fopen.obj
 0001:000437b0       _fclose_nolock             00000001800447b0 f   libucrt:fclose.obj
 0001:00043834       fclose                     0000000180044834 f   libucrt:fclose.obj
 0001:00043898       _clearfp                   0000000180044898 f   libucrt:ieee.obj
 0001:00043908       _control87                 0000000180044908 f   libucrt:ieee.obj
 0001:00043bd0       __acrt_errno_from_os_error 0000000180044bd0 f   libucrt:errno.obj
 0001:00043c18       __acrt_errno_map_os_error  0000000180044c18 f   libucrt:errno.obj
 0001:00043c68       __doserrno                 0000000180044c68 f   libucrt:errno.obj
 0001:00043c88       _errno                     0000000180044c88 f   libucrt:errno.obj
 0001:00043ca8       strerror                   0000000180044ca8 f   libucrt:strerror.obj
 0001:00043d50       __acrt_initialize_stdio    0000000180044d50 f   libucrt:_file.obj
 0001:00043e70       __acrt_iob_func            0000000180044e70 f   libucrt:_file.obj
 0001:00043e84       __acrt_uninitialize_stdio  0000000180044e84 f   libucrt:_file.obj
 0001:00043ee0       _lock_file                 0000000180044ee0 f   libucrt:_file.obj
 0001:00043eec       _unlock_file               0000000180044eec f   libucrt:_file.obj
 0001:00043ff8       _wfreopen                  0000000180044ff8 f   libucrt:freopen.obj
 0001:00044028       feof                       0000000180045028 f   libucrt:feoferr.obj
 0001:00044054       ferror                     0000000180045054 f   libucrt:feoferr.obj
 0001:00044080       _fread_nolock_s            0000000180045080 f   libucrt:fread.obj
 0001:00044310       fread                      0000000180045310 f   libucrt:fread.obj
 0001:00044330       fread_s                    0000000180045330 f   libucrt:fread.obj
 0001:000443d8       _fgetc_nolock              00000001800453d8 f   libucrt:fgetc.obj
 0001:0004441c       _getc_nolock               000000018004541c f   libucrt:fgetc.obj
 0001:00044424       fgetc                      0000000180045424 f   libucrt:fgetc.obj
 0001:0004452c       getc                       000000018004552c f   libucrt:fgetc.obj
 0001:00044534       rewind                     0000000180045534 f   libucrt:rewind.obj
 0001:000445f8       _ungetc_nolock             00000001800455f8 f   libucrt:ungetc.obj
 0001:00044720       ungetc                     0000000180045720 f   libucrt:ungetc.obj
 0001:00044790       strcmp                     0000000180045790 f   libucrt:strcmp.obj
 0001:000447f8       iswctype                   00000001800457f8 f   libucrt:iswctype.obj
 0001:00044868       isdigit                    0000000180045868 f i libucrt:_ctype.obj
 0001:000448fc       isspace                    00000001800458fc f i libucrt:_ctype.obj
 0001:00044990       wcsncpy                    0000000180045990 f   libucrt:wcsncpy.obj
 0001:000449d8       _wcsicmp                   00000001800459d8 f   libucrt:wcsicmp.obj
 0001:00044a70       _wcsicmp_l                 0000000180045a70 f   libucrt:wcsicmp.obj
 0001:00044b80       strncmp                    0000000180045b80 f   libucrt:strncmp.obj
 0001:00044c10       strncpy                    0000000180045c10 f   libucrt:strncpy.obj
 0001:00044e20       strpbrk                    0000000180045e20 f   libucrt:strpbrk.obj
 0001:0004590c       _pclose                    000000018004690c f   libucrt:popen.obj
 0001:000459e4       _wpopen                    00000001800469e4 f   libucrt:popen.obj
 0001:000459ec       clearerr                   00000001800469ec f   libucrt:clearerr.obj
 0001:000459f4       clearerr_s                 00000001800469f4 f   libucrt:clearerr.obj
 0001:00045cb8       __acrt_stdio_flush_nolock  0000000180046cb8 f   libucrt:fflush.obj
 0001:00045d34       _fflush_nolock             0000000180046d34 f   libucrt:fflush.obj
 0001:00045d80       _flushall                  0000000180046d80 f   libucrt:fflush.obj
 0001:00045d88       fflush                     0000000180046d88 f   libucrt:fflush.obj
 0001:00045ebc       fgets                      0000000180046ebc f   libucrt:fgets.obj
 0001:000460cc       fseek                      00000001800470cc f   libucrt:fseek.obj
 0001:000465c0       _ftelli64_nolock           00000001800475c0 f   libucrt:ftell.obj
 0001:000465c8       ftell                      00000001800475c8 f   libucrt:ftell.obj
 0001:00046674       _fwrite_nolock             0000000180047674 f   libucrt:fwrite.obj
 0001:00046820       fwrite                     0000000180047820 f   libucrt:fwrite.obj
 0001:000469c4       setvbuf                    00000001800479c4 f   libucrt:setvbuf.obj
 0001:00046e00       __acrt_stdio_free_tmpfile_name_buffers_nolock 0000000180047e00 f   libucrt:tmpfile.obj
 0001:00046e88       tmpfile                    0000000180047e88 f   libucrt:tmpfile.obj
 0001:00046eec       ??$is_overflow_condition@_K@__crt_strtox@@YA_NI_K@Z 0000000180047eec f i libucrt:input.obj
 0001:00046f1c       ??$parse_floating_point@V?$input_adapter_character_source@V?$stream_input_adapter@D@__crt_stdio_input@@@__crt_strtox@@M@__crt_strtox@@YA?AW4SLD_STATUS@@QEAU__crt_locale_pointers@@V?$input_adapter_character_source@V?$stream_input_adapter@D@__crt_stdio_input@@@0@QEAM@Z 0000000180047f1c f i libucrt:input.obj
 0001:00046fc4       ??$parse_floating_point@V?$input_adapter_character_source@V?$stream_input_adapter@D@__crt_stdio_input@@@__crt_strtox@@N@__crt_strtox@@YA?AW4SLD_STATUS@@QEAU__crt_locale_pointers@@V?$input_adapter_character_source@V?$stream_input_adapter@D@__crt_stdio_input@@@0@QEAN@Z 0000000180047fc4 f i libucrt:input.obj
 0001:0004706c       ??$parse_floating_point_from_source@V?$input_adapter_character_source@V?$stream_input_adapter@D@__crt_stdio_input@@@__crt_strtox@@@__crt_strtox@@YA?AW4floating_point_parse_result@0@QEAU__crt_locale_pointers@@AEAV?$input_adapter_character_source@V?$stream_input_adapter@D@__crt_stdio_input@@@0@AEAUfloating_point_string@0@@Z 000000018004806c f i libucrt:input.obj
 0001:00047910       ??$parse_floating_point_possible_infinity@DV?$input_adapter_character_source@V?$stream_input_adapter@D@__crt_stdio_input@@@__crt_strtox@@_K@__crt_strtox@@YA?AW4floating_point_parse_result@0@AEADAEAV?$input_adapter_character_source@V?$stream_input_adapter@D@__crt_stdio_input@@@0@_K@Z 0000000180048910 f i libucrt:input.obj
 0001:00047b80       ??$parse_floating_point_possible_nan@DV?$input_adapter_character_source@V?$stream_input_adapter@D@__crt_stdio_input@@@__crt_strtox@@_K@__crt_strtox@@YA?AW4floating_point_parse_result@0@AEADAEAV?$input_adapter_character_source@V?$stream_input_adapter@D@__crt_stdio_input@@@0@_K@Z 0000000180048b80 f i libucrt:input.obj
 0001:00047e1c       ??$parse_floating_point_possible_nan_is_ind@DV?$input_adapter_character_source@V?$stream_input_adapter@D@__crt_stdio_input@@@__crt_strtox@@@__crt_strtox@@YA_NAEADAEAV?$input_adapter_character_source@V?$stream_input_adapter@D@__crt_stdio_input@@@0@@Z 0000000180048e1c f i libucrt:input.obj
 0001:00047eb4       ??$parse_floating_point_possible_nan_is_snan@DV?$input_adapter_character_source@V?$stream_input_adapter@D@__crt_stdio_input@@@__crt_strtox@@@__crt_strtox@@YA_NAEADAEAV?$input_adapter_character_source@V?$stream_input_adapter@D@__crt_stdio_input@@@0@@Z 0000000180048eb4 f i libucrt:input.obj
 0001:00047f4c       ??$parse_floating_point_write_result@M@__crt_strtox@@YA?AW4SLD_STATUS@@W4floating_point_parse_result@0@AEBUfloating_point_string@0@QEAM@Z 0000000180048f4c f i libucrt:input.obj
 0001:000480bc       ??$parse_floating_point_write_result@N@__crt_strtox@@YA?AW4SLD_STATUS@@W4floating_point_parse_result@0@AEBUfloating_point_string@0@QEAN@Z 00000001800490bc f i libucrt:input.obj
 0001:0004829c       ??$parse_integer@_KV?$input_adapter_character_source@V?$stream_input_adapter@D@__crt_stdio_input@@@__crt_strtox@@@__crt_strtox@@YA_KQEAU__crt_locale_pointers@@V?$input_adapter_character_source@V?$stream_input_adapter@D@__crt_stdio_input@@@0@H_N@Z 000000018004929c f i libucrt:input.obj
 0001:00048720       ??$process_floating_point_specifier_t@M@?$input_processor@DV?$stream_input_adapter@D@__crt_stdio_input@@@__crt_stdio_input@@AEAA_NXZ 0000000180049720 f i libucrt:input.obj
 0001:000487c0       ??$process_floating_point_specifier_t@N@?$input_processor@DV?$stream_input_adapter@D@__crt_stdio_input@@@__crt_stdio_input@@AEAA_NXZ 00000001800497c0 f i libucrt:input.obj
 0001:00048860       ??$process_string_specifier_tchar@D@?$input_processor@DV?$stream_input_adapter@D@__crt_stdio_input@@@__crt_stdio_input@@AEAA_NW4conversion_mode@1@D@Z 0000000180049860 f i libucrt:input.obj
 0001:000489fc       ??$process_string_specifier_tchar@_W@?$input_processor@DV?$stream_input_adapter@D@__crt_stdio_input@@@__crt_stdio_input@@AEAA_NW4conversion_mode@1@_W@Z 00000001800499fc f i libucrt:input.obj
 0001:00048bd0       ??$skip_whitespace@Vstream_input_adapter@__crt_stdio_input@@D@__crt_stdio_input@@YAHAEAV?$stream_input_adapter@D@0@QEAU__crt_locale_pointers@@@Z 0000000180049bd0 f i libucrt:input.obj
 0001:00048db0       ?advance@?$format_string_parser@D@__crt_stdio_input@@QEAA_NXZ 0000000180049db0 f i libucrt:input.obj
 0001:00048f78       ?as_double@floating_point_value@__crt_strtox@@QEBAAEANXZ 0000000180049f78 f i libucrt:input.obj
 0001:00048fb4       ?as_float@floating_point_value@__crt_strtox@@QEBAAEAMXZ 0000000180049fb4 f i libucrt:input.obj
 0001:00048ff0       ?assemble_floating_point_value@__crt_strtox@@YA?AW4SLD_STATUS@@_KH_N1AEBVfloating_point_value@1@@Z 0000000180049ff0 f i libucrt:input.obj
 0001:00049398       ?assemble_floating_point_value_from_big_integer@__crt_strtox@@YA?AW4SLD_STATUS@@AEBUbig_integer@1@I_N1AEBVfloating_point_value@1@@Z 000000018004a398 f i libucrt:input.obj
 0001:000494fc       ?convert_decimal_string_to_floating_type_common@__crt_strtox@@YA?AW4SLD_STATUS@@AEBUfloating_point_string@1@AEBVfloating_point_value@1@@Z 000000018004a4fc f i libucrt:input.obj
 0001:0004b27c       ?convert_hexadecimal_string_to_floating_type_common@__crt_strtox@@YA?AW4SLD_STATUS@@AEBUfloating_point_string@1@AEBVfloating_point_value@1@@Z 000000018004c27c f i libucrt:input.obj
 0001:0004b330       ?divide@__crt_strtox@@YA_KAEAUbig_integer@1@AEBU21@@Z 000000018004c330 f i libucrt:input.obj
 0001:0004b75c       ?length@?$format_string_parser@D@__crt_stdio_input@@QEBA_KXZ 000000018004c75c f i libucrt:input.obj
 0001:0004b7f8       ?process@?$input_processor@DV?$stream_input_adapter@D@__crt_stdio_input@@@__crt_stdio_input@@QEAAHXZ 000000018004c7f8 f i libucrt:input.obj
 0001:0004b8b8       ?process_conversion_specifier@?$input_processor@DV?$stream_input_adapter@D@__crt_stdio_input@@@__crt_stdio_input@@AEAA_NXZ 000000018004c8b8 f i libucrt:input.obj
 0001:0004b9d4       ?process_floating_point_specifier@?$input_processor@DV?$stream_input_adapter@D@__crt_stdio_input@@@__crt_stdio_input@@AEAA_NXZ 000000018004c9d4 f i libucrt:input.obj
 0001:0004ba38       ?process_integer_specifier@?$input_processor@DV?$stream_input_adapter@D@__crt_stdio_input@@@__crt_stdio_input@@AEAA_NI_N@Z 000000018004ca38 f i libucrt:input.obj
 0001:0004bae4       ?process_literal_character_tchar@?$input_processor@DV?$stream_input_adapter@D@__crt_stdio_input@@@__crt_stdio_input@@AEAA_ND@Z 000000018004cae4 f i libucrt:input.obj
 0001:0004bb58       ?process_state@?$input_processor@DV?$stream_input_adapter@D@__crt_stdio_input@@@__crt_stdio_input@@AEAA_NXZ 000000018004cb58 f i libucrt:input.obj
 0001:0004bc14       ?process_string_specifier@?$input_processor@DV?$stream_input_adapter@D@__crt_stdio_input@@@__crt_stdio_input@@AEAA_NW4conversion_mode@2@@Z 000000018004cc14 f i libucrt:input.obj
 0001:0004bc94       ?scan_conversion_specifier@?$format_string_parser@D@__crt_stdio_input@@AEAA_NXZ 000000018004cc94 f i libucrt:input.obj
 0001:0004be38       ?scan_optional_field_width@?$format_string_parser@D@__crt_stdio_input@@AEAA_NXZ 000000018004ce38 f i libucrt:input.obj
 0001:0004bee0       ?scan_optional_length_modifier@?$format_string_parser@D@__crt_stdio_input@@AEAAXXZ 000000018004cee0 f i libucrt:input.obj
 0001:0004c01c       ?scan_scanset_range@?$format_string_parser@D@__crt_stdio_input@@AEAA_NXZ 000000018004d01c f i libucrt:input.obj
 0001:0004c1d0       ?write_character@?$input_processor@DV?$stream_input_adapter@D@__crt_stdio_input@@@__crt_stdio_input@@AEAA_NQEFA_W_KAEAPEFA_WAEA_KD@Z 000000018004d1d0 f i libucrt:input.obj
 0001:0004c264       ?write_integer@?$input_processor@DV?$stream_input_adapter@D@__crt_stdio_input@@@__crt_stdio_input@@AEAA_N_K@Z 000000018004d264 f i libucrt:input.obj
 0001:0004c2d8       __stdio_common_vfscanf     000000018004d2d8 f   libucrt:input.obj
 0001:0004c5d8       _wdupenv_s                 000000018004d5d8 f   libucrt:getenv.obj
 0001:0004c5f8       _wgetenv                   000000018004d5f8 f   libucrt:getenv.obj
 0001:0004c600       _wsystem                   000000018004d600 f   libucrt:system.obj
 0001:0004c738       wcscmp                     000000018004d738 f   libucrt:wcscmp.obj
 0001:0004c770       _initterm                  000000018004d770 f   libucrt:initterm.obj
 0001:0004c7d4       _initterm_e                000000018004d7d4 f   libucrt:initterm.obj
 0001:0004c814       _seh_filter_dll            000000018004d814 f   libucrt:exception_filter.obj
 0001:0004c828       _seh_filter_exe            000000018004d828 f   libucrt:exception_filter.obj
 0001:0004cc18       __acrt_initialize_thread_local_exit_callback 000000018004dc18 f   libucrt:exit.obj
 0001:0004cc20       _cexit                     000000018004dc20 f   libucrt:exit.obj
 0001:0004cc30       _exit                      000000018004dc30 f   libucrt:exit.obj
 0001:0004cc3c       _is_c_termination_complete 000000018004dc3c f   libucrt:exit.obj
 0001:0004ce08       __acrt_allocate_buffer_for_argv 000000018004de08 f   libucrt:argv_parsing.obj
 0001:0004ce68       _configure_narrow_argv     000000018004de68 f   libucrt:argv_parsing.obj
 0001:0004d410       __dcrt_get_or_create_wide_environment_nolock 000000018004e410 f   libucrt:environment_initialization.obj
 0001:0004d44c       __dcrt_uninitialize_environments_nolock 000000018004e44c f   libucrt:environment_initialization.obj
 0001:0004d484       _initialize_narrow_environment 000000018004e484 f   libucrt:environment_initialization.obj
 0001:0004d5e0       _execute_onexit_table      000000018004e5e0 f   libucrt:onexit.obj
 0001:0004d61c       _initialize_onexit_table   000000018004e61c f   libucrt:onexit.obj
 0001:0004d67c       __acrt_uninitialize_command_line 000000018004e67c f   libucrt:argv_data.obj
 0001:0004d774       __acrt_initialize          000000018004e774 f   libucrt:initialization.obj
 0001:0004d788       __acrt_thread_attach       000000018004e788 f   libucrt:initialization.obj
 0001:0004d79c       __acrt_thread_detach       000000018004e79c f   libucrt:initialization.obj
 0001:0004d7ac       __acrt_uninitialize        000000018004e7ac f   libucrt:initialization.obj
 0001:0004d7e4       __acrt_uninitialize_critical 000000018004e7e4 f   libucrt:initialization.obj
 0001:0004d7f4       terminate                  000000018004e7f4 f   libucrt:terminate.obj
 0001:0004da18       _strupr                    000000018004ea18 f   libucrt:strupr.obj
 0001:0004da18       strupr                     000000018004ea18 f   libucrt:strupr.obj
 0001:0004da78       _strupr_s_l                000000018004ea78 f   libucrt:strupr.obj
 0001:0004dac4       __ascii_stricmp            000000018004eac4 f   libucrt:stricmp.obj
 0001:0004db04       _stricmp                   000000018004eb04 f   libucrt:stricmp.obj
 0001:0004db04       stricmp                    000000018004eb04 f   libucrt:stricmp.obj
 0001:0004db4c       _stricmp_l                 000000018004eb4c f   libucrt:stricmp.obj
 0001:0004dc00       strcpy_s                   000000018004ec00 f   libucrt:strcpy_s.obj
 0001:0004dc60       ??$parse_integer@KV?$c_string_character_source@D@__crt_strtox@@@__crt_strtox@@YAKQEAU__crt_locale_pointers@@V?$c_string_character_source@D@0@H_N@Z 000000018004ec60 f i libucrt:atox.obj
 0001:0004df9c       ??$parse_integer@KV?$c_string_character_source@_W@__crt_strtox@@@__crt_strtox@@YAKQEAU__crt_locale_pointers@@V?$c_string_character_source@_W@0@H_N@Z 000000018004ef9c f i libucrt:atox.obj
 0001:0004e650       ??$parse_integer@_KV?$c_string_character_source@D@__crt_strtox@@@__crt_strtox@@YA_KQEAU__crt_locale_pointers@@V?$c_string_character_source@D@0@H_N@Z 000000018004f650 f i libucrt:atox.obj
 0001:0004e980       abort                      000000018004f980 f   libucrt:abort.obj
 0001:0004e9d8       calloc                     000000018004f9d8 f   libucrt:calloc.obj
 0001:0004e9e0       wcsncmp                    000000018004f9e0 f   libucrt:wcsncmp.obj
 0001:0004ea0c       __acrt_call_reportfault    000000018004fa0c f   libucrt:invalid_parameter.obj
 0001:0004eb68       __acrt_initialize_invalid_parameter_handler 000000018004fb68 f   libucrt:invalid_parameter.obj
 0001:0004eb70       _invalid_parameter         000000018004fb70 f   libucrt:invalid_parameter.obj
 0001:0004ec20       _invalid_parameter_noinfo  000000018004fc20 f   libucrt:invalid_parameter.obj
 0001:0004ec40       _invoke_watson             000000018004fc40 f   libucrt:invalid_parameter.obj
 0001:0004ece8       _tolower_l                 000000018004fce8 f   libucrt:tolower_toupper.obj
 0001:0004ee28       tolower                    000000018004fe28 f   libucrt:tolower_toupper.obj
 0001:0004ee54       _free_base                 000000018004fe54 f   libucrt:free_base.obj
 0001:0004ee94       _malloc_base               000000018004fe94 f   libucrt:malloc_base.obj
 0001:0004eef4       strtol                     000000018004fef4 f   libucrt:strtox.obj
 0001:0004ef20       strtoull                   000000018004ff20 f   libucrt:strtox.obj
 0001:0004ef4c       wcstol                     000000018004ff4c f   libucrt:strtox.obj
 0001:0004ef78       _mbtowc_l                  000000018004ff78 f   libucrt:mbtowc.obj
 0001:0004f0f4       mbtowc                     00000001800500f4 f   libucrt:mbtowc.obj
 0001:0004f0fc       _wctomb_s_l                00000001800500fc f   libucrt:wctomb.obj
 0001:0004f29c       wctomb_s                   000000018005029c f   libucrt:wctomb.obj
 0001:0004f2b0       strnlen                    00000001800502b0 f   libucrt:strnlen.obj
 0001:0004f400       wcsnlen                    0000000180050400 f   libucrt:strnlen.obj
 0001:0004f950       __acrt_freeptd             0000000180050950 f   libucrt:per_thread_data.obj
 0001:0004f994       __acrt_getptd              0000000180050994 f   libucrt:per_thread_data.obj
 0001:0004fa68       __acrt_getptd_head         0000000180050a68 f   libucrt:per_thread_data.obj
 0001:0004fb10       __acrt_getptd_noexit       0000000180050b10 f   libucrt:per_thread_data.obj
 0001:0004fbdc       __acrt_initialize_ptd      0000000180050bdc f   libucrt:per_thread_data.obj
 0001:0004fc18       __acrt_uninitialize_ptd    0000000180050c18 f   libucrt:per_thread_data.obj
 0001:0004fc3c       __acrt_update_locale_info  0000000180050c3c f   libucrt:locale_update.obj
 0001:0004fc70       __acrt_update_multibyte_info 0000000180050c70 f   libucrt:locale_update.obj
 0001:00050678       __acrt_fp_format           0000000180051678 f   libucrt:cvt.obj
 0001:00050900       _fileno                    0000000180051900 f   libucrt:fileno.obj
 0001:00050928       _fputc_nolock              0000000180051928 f   libucrt:fputc.obj
 0001:00050940       _get_printf_count_output   0000000180051940 f   libucrt:printf_count_output.obj
 0001:00050958       __acrt_stdio_begin_temporary_buffering_nolock 0000000180051958 f   libucrt:_sftbuf.obj
 0001:00050a28       __acrt_stdio_end_temporary_buffering_nolock 0000000180051a28 f   libucrt:_sftbuf.obj
 0001:00050ad4       __acrt_set_locale_changed  0000000180051ad4 f   libucrt:wsetlocale.obj
 0001:00050ae0       __acrt_uninitialize_locale 0000000180051ae0 f   libucrt:wsetlocale.obj
 0001:00050d0c       __acrt_initialize_lowio    0000000180051d0c f   libucrt:ioinit.obj
 0001:00050d48       __acrt_uninitialize_lowio  0000000180051d48 f   libucrt:ioinit.obj
 0001:00050d88       wcscpy_s                   0000000180051d88 f   libucrt:wcscpy_s.obj
 0001:00050df0       ?__acrt_stdio_allocate_stream@@YA?AV__crt_stdio_stream@@XZ 0000000180051df0 f   libucrt:stream.obj
 0001:00050e48       ?__acrt_stdio_free_stream@@YAXV__crt_stdio_stream@@@Z 0000000180051e48 f   libucrt:stream.obj
 0001:00050f50       ??$__acrt_stdio_parse_mode@_W@@YA?AU__acrt_stdio_stream_mode@@QEB_W@Z 0000000180051f50 f i libucrt:openfile.obj
 0001:00051254       _wopenfile                 0000000180052254 f   libucrt:openfile.obj
 0001:00051364       _close                     0000000180052364 f   libucrt:close.obj
 0001:00051408       _close_nolock              0000000180052408 f   libucrt:close.obj
 0001:000514c8       __acrt_stdio_free_buffer_nolock 00000001800524c8 f   libucrt:_freebuf.obj
 0001:00051520       _get_fpsr                  0000000180052520 f   libucrt:fpsr.obj
 0001:00051530       _set_fpsr                  0000000180052530 f   libucrt:fpsr.obj
 0001:0005153a       _fclrf                     000000018005253a f   libucrt:fpsr.obj
 0001:0005154e       _frnd                      000000018005254e f   libucrt:fpsr.obj
 0001:00051570       _calloc_base               0000000180052570 f   libucrt:calloc_base.obj
 0001:000515e8       __sys_errlist              00000001800525e8 f   libucrt:syserr.obj
 0001:000515f0       __sys_nerr                 00000001800525f0 f   libucrt:syserr.obj
 0001:000515f8       strncpy_s                  00000001800525f8 f   libucrt:strncpy_s.obj
 0001:000518a4       __acrt_AppPolicyGetProcessTerminationMethodInternal 00000001800528a4 f   libucrt:winapi_thunks.obj
 0001:000518f4       __acrt_AreFileApisANSI     00000001800528f4 f   libucrt:winapi_thunks.obj
 0001:00051930       __acrt_CompareStringEx     0000000180052930 f   libucrt:winapi_thunks.obj
 0001:00051a0c       __acrt_FlsAlloc            0000000180052a0c f   libucrt:winapi_thunks.obj
 0001:00051a54       __acrt_FlsFree             0000000180052a54 f   libucrt:winapi_thunks.obj
 0001:00051a9c       __acrt_FlsGetValue         0000000180052a9c f   libucrt:winapi_thunks.obj
 0001:00051ae4       __acrt_FlsSetValue         0000000180052ae4 f   libucrt:winapi_thunks.obj
 0001:00051b38       __acrt_InitializeCriticalSectionEx 0000000180052b38 f   libucrt:winapi_thunks.obj
 0001:00051b9c       __acrt_LCMapStringEx       0000000180052b9c f   libucrt:winapi_thunks.obj
 0001:00051c78       __acrt_LocaleNameToLCID    0000000180052c78 f   libucrt:winapi_thunks.obj
 0001:00051cc8       __acrt_initialize_winapi_thunks 0000000180052cc8 f   libucrt:winapi_thunks.obj
 0001:00051cfc       __acrt_uninitialize_winapi_thunks 0000000180052cfc f   libucrt:winapi_thunks.obj
 0001:00051d40       _fcloseall                 0000000180052d40 f   libucrt:closeall.obj
 0001:000523c8       _read                      00000001800533c8 f   libucrt:read.obj
 0001:000524e4       _read_nolock               00000001800534e4 f   libucrt:read.obj
 0001:0005293c       __acrt_stdio_refill_and_read_narrow_nolock 000000018005393c f   libucrt:_filbuf.obj
 0001:00052e14       _lseek                     0000000180053e14 f   libucrt:lseek.obj
 0001:00052e1c       _lseeki64                  0000000180053e1c f   libucrt:lseek.obj
 0001:00052e24       _lseeki64_nolock           0000000180053e24 f   libucrt:lseek.obj
 0001:00052e2c       __acrt_stdio_allocate_buffer_nolock 0000000180053e2c f   libucrt:_getbuf.obj
 0001:00052e94       __acrt_GetStringTypeW      0000000180053e94 f   libucrt:getstringtypew.obj
 0001:00052e9c       __pctype_func              0000000180053e9c f   libucrt:ctype.obj
 0001:00052ecc       _isctype_l                 0000000180053ecc f   libucrt:isctype.obj
 0001:00052fdc       _towlower_l                0000000180053fdc f   libucrt:towlower.obj
 0001:000530a0       _recalloc_base             00000001800540a0 f   libucrt:recalloc.obj
 0001:00053138       wcscat_s                   0000000180054138 f   libucrt:wcscat_s.obj
 0001:000531b8       _cwait                     00000001800541b8 f   libucrt:wait.obj
 0001:00053270       __acrt_wgetpath            0000000180054270 f   libucrt:getpath.obj
 0001:00053364       ??$__acrt_mbs_to_wcs_cp@U__crt_win32_buffer_internal_dynamic_resizing@@@@YAHQEBDAEAV?$__crt_win32_buffer@_WU__crt_win32_buffer_internal_dynamic_resizing@@@@I@Z 0000000180054364 f i libucrt:createprocessa.obj
 0001:000534dc       __acrt_initialize_locks    00000001800544dc f   libucrt:locks.obj
 0001:00053524       __acrt_lock                0000000180054524 f   libucrt:locks.obj
 0001:00053540       __acrt_uninitialize_locks  0000000180054540 f   libucrt:locks.obj
 0001:00053578       __acrt_unlock              0000000180054578 f   libucrt:locks.obj
 0001:00053594       _waccess_s                 0000000180054594 f   libucrt:waccess.obj
 0001:00053640       _pipe                      0000000180054640 f   libucrt:pipe.obj
 0001:000539d0       _wfdopen                   00000001800549d0 f   libucrt:fdopen.obj
 0001:00053a64       _commit                    0000000180054a64 f   libucrt:commit.obj
 0001:00054364       _write                     0000000180055364 f   libucrt:write.obj
 0001:00054450       _write_nolock              0000000180055450 f   libucrt:write.obj
 0001:00054888       __acrt_stdio_flush_and_write_narrow_nolock 0000000180055888 f   libucrt:_flsbuf.obj
 0001:00054aa8       _ui64toa_s                 0000000180055aa8 f   libucrt:xtoa.obj
 0001:00054abc       _strdup                    0000000180055abc f   libucrt:strdup.obj
 0001:00054b34       __acrt_GetTempPathA        0000000180055b34 f   libucrt:gettemppath.obj
 0001:000552c8       _sopen_nolock              00000001800562c8 f   libucrt:open.obj
 0001:000553e0       _sopen_s                   00000001800563e0 f   libucrt:open.obj
 0001:00055414       _wsopen_nolock             0000000180056414 f   libucrt:open.obj
 0001:000557fc       _wsopen_s                  00000001800567fc f   libucrt:open.obj
 0001:00055830       __acrt_uninitialize_tmpfile 0000000180056830 f   libucrt:rmtmp.obj
 0001:00055844       _rmtmp                     0000000180056844 f   libucrt:rmtmp.obj
 0001:000558d8       fegetround                 00000001800568d8 f   libucrt:fegetround.obj
 0001:000558ec       _wcsnicoll                 00000001800568ec f   libucrt:wcsnicol.obj
 0001:0005599c       _wcsnicoll_l               000000018005699c f   libucrt:wcsnicol.obj
 0001:00056224       _wspawnve                  0000000180057224 f   libucrt:spawnv.obj
 0001:00056554       _wspawnvpe                 0000000180057554 f   libucrt:spawnvp.obj
 0001:0005655c       __acrt_get_process_end_policy 000000018005755c f   libucrt:win_policies.obj
 0001:000565ac       ??$__acrt_wcs_to_mbs_cp@U__crt_win32_buffer_internal_dynamic_resizing@@@@YAHQEB_WAEAV?$__crt_win32_buffer@DU__crt_win32_buffer_internal_dynamic_resizing@@@@I@Z 00000001800575ac f i libucrt:argv_wildcards.obj
 0001:00056ddc       __acrt_expand_narrow_argv_wildcards 0000000180057ddc f   libucrt:argv_wildcards.obj
 0001:00056de4       ??$__acrt_wcs_to_mbs_cp@U__crt_win32_buffer_no_resizing@@@@YAHQEB_WAEAV?$__crt_win32_buffer@DU__crt_win32_buffer_no_resizing@@@@I@Z 0000000180057de4 f i libucrt:getmodulefilenamea.obj
 0001:00056ef8       __acrt_GetModuleFileNameA  0000000180057ef8 f   libucrt:getmodulefilenamea.obj
 0001:00057744       __acrt_initialize_multibyte 0000000180058744 f   libucrt:mbctype.obj
 0001:000577a4       __acrt_update_thread_multibyte_data 00000001800587a4 f   libucrt:mbctype.obj
 0001:000577c0       _setmbcp_nolock            00000001800587c0 f   libucrt:mbctype.obj
 0001:00057af4       _ismbblead                 0000000180058af4 f   libucrt:ismbbyte.obj
 0001:00057b08       __acrt_initialize_command_line 0000000180058b08 f   libucrt:argv_data.obj
 0001:00057b30       __acrt_MultiByteToWideChar 0000000180058b30 f   libucrt:multibytetowidechar.obj
 0001:00057b8c       __acrt_WideCharToMultiByte 0000000180058b8c f   libucrt:widechartomultibyte.obj
 0001:00057c24       __dcrt_get_narrow_environment_from_os 0000000180058c24 f   libucrt:get_environment_from_os.obj
 0001:00057d28       __dcrt_get_wide_environment_from_os 0000000180058d28 f   libucrt:get_environment_from_os.obj
 0001:000581dc       __dcrt_set_variable_in_wide_environment_nolock 00000001800591dc f   libucrt:setenv.obj
 0001:000581e4       __acrt_initialize_heap     00000001800591e4 f   libucrt:heap_handle.obj
 0001:00058200       __acrt_uninitialize_heap   0000000180059200 f   libucrt:heap_handle.obj
 0001:0005820c       __acrt_execute_initializers 000000018005920c f   libucrt:shared_initialization.obj
 0001:0005828c       __acrt_execute_uninitializers 000000018005928c f   libucrt:shared_initialization.obj
 0001:000582c8       __acrt_initialize_new_handler 00000001800592c8 f   libucrt:new_handler.obj
 0001:000582d0       _callnewh                  00000001800592d0 f   libucrt:new_handler.obj
 0001:00058300       _query_new_handler         0000000180059300 f   libucrt:new_handler.obj
 0001:0005837c       __acrt_get_sigabrt_handler 000000018005937c f   libucrt:signal.obj
 0001:000583ac       __acrt_initialize_signal_handlers 00000001800593ac f   libucrt:signal.obj
 0001:000583cc       raise                      00000001800593cc f   libucrt:signal.obj
 0001:00058638       __acrt_has_user_matherr    0000000180059638 f   libucrt:matherr.obj
 0001:00058658       __acrt_initialize_user_matherr 0000000180059658 f   libucrt:matherr.obj
 0001:00058660       __acrt_invoke_user_matherr 0000000180059660 f   libucrt:matherr.obj
 0001:000589a8       __acrt_LCMapStringA        00000001800599a8 f   libucrt:lcmapstringa.obj
 0001:00058a40       _isleadbyte_l              0000000180059a40 f i libucrt:_wctype.obj
 0001:00058a8c       _query_new_mode            0000000180059a8c f   libucrt:new_mode.obj
 0001:00058a94       ?__mbrtowc_utf8@__crt_mbstring@@YA_KPEA_WPEBD_KPEAU_Mbstatet@@@Z 0000000180059a94 f   libucrt:mbrtowc.obj
 0001:00058ad0       ?__mbsrtowcs_utf8@__crt_mbstring@@YA_KPEA_WPEAPEBD_KPEAU_Mbstatet@@@Z 0000000180059ad0 f   libucrt:mbrtowc.obj
 0001:00058c48       ?__c32rtomb_utf8@__crt_mbstring@@YA_KPEAD_UPEAU_Mbstatet@@@Z 0000000180059c48 f   libucrt:c32rtomb.obj
 0001:00058d00       __acrt_add_locale_ref      0000000180059d00 f   libucrt:locale_refcounting.obj
 0001:00058d8c       __acrt_free_locale         0000000180059d8c f   libucrt:locale_refcounting.obj
 0001:00058f04       __acrt_locale_add_lc_time_reference 0000000180059f04 f   libucrt:locale_refcounting.obj
 0001:00058f2c       __acrt_locale_free_lc_time_if_unreferenced 0000000180059f2c f   libucrt:locale_refcounting.obj
 0001:00058f64       __acrt_locale_release_lc_time_reference 0000000180059f64 f   libucrt:locale_refcounting.obj
 0001:00058f8c       __acrt_release_locale_ref  0000000180059f8c f   libucrt:locale_refcounting.obj
 0001:00059034       __acrt_update_thread_locale_data 000000018005a034 f   libucrt:locale_refcounting.obj
 0001:000590a4       _updatetlocinfoEx_nolock   000000018005a0a4 f   libucrt:locale_refcounting.obj
 0001:0005910c       __acrt_fp_strflt_to_string 000000018005a10c f   libucrt:_fptostr.obj
 0001:000591f0       __acrt_fltout              000000018005a1f0 f   libucrt:cfout.obj
 0001:0005a424       _isatty                    000000018005b424 f   libucrt:isatty.obj
 0001:0005a484       __acrt_locale_free_monetary 000000018005b484 f   libucrt:initmon.obj
 0001:0005a590       __acrt_locale_free_numeric 000000018005b590 f   libucrt:initnum.obj
 0001:0005a654       __acrt_locale_free_time    000000018005b654 f   libucrt:inittime.obj
 0001:0005a75c       __acrt_GetStringTypeA      000000018005b75c f   libucrt:getstringtypea.obj
 0001:0005a8ec       __acrt_lowio_create_handle_array 000000018005b8ec f   libucrt:osfinfo.obj
 0001:0005a994       __acrt_lowio_destroy_handle_array 000000018005b994 f   libucrt:osfinfo.obj
 0001:0005a9e4       __acrt_lowio_ensure_fh_exists 000000018005b9e4 f   libucrt:osfinfo.obj
 0001:0005aa8c       __acrt_lowio_lock_fh       000000018005ba8c f   libucrt:osfinfo.obj
 0001:0005aab4       __acrt_lowio_set_os_handle 000000018005bab4 f   libucrt:osfinfo.obj
 0001:0005ab74       __acrt_lowio_unlock_fh     000000018005bb74 f   libucrt:osfinfo.obj
 0001:0005ab9c       _alloc_osfhnd              000000018005bb9c f   libucrt:osfinfo.obj
 0001:0005acdc       _free_osfhnd               000000018005bcdc f   libucrt:osfinfo.obj
 0001:0005ad98       _get_osfhandle             000000018005bd98 f   libucrt:osfinfo.obj
 0001:0005ae10       _wcsnicmp                  000000018005be10 f   libucrt:wcsnicmp.obj
 0001:0005aebc       _wcsnicmp_l                000000018005bebc f   libucrt:wcsnicmp.obj
 0001:0005b0cc       __acrt_DownlevelLocaleNameToLCID 000000018005c0cc f   libucrt:lcidtoname_downlevel.obj
 0001:0005b100       __acrt_LCMapStringW        000000018005c100 f   libucrt:lcmapstringw.obj
 0001:0005b188       _msize_base                000000018005c188 f   libucrt:msize.obj
 0001:0005b1c4       _realloc_base              000000018005c1c4 f   libucrt:realloc_base.obj
 0001:0005b240       _get_fmode                 000000018005c240 f   libucrt:setmode.obj
 0001:0005b270       _setmode_nolock            000000018005c270 f   libucrt:setmode.obj
 0001:0005b350       _putwch_nolock             000000018005c350 f   libucrt:putwch.obj
 0001:0005b38c       _chsize_nolock             000000018005c38c f   libucrt:chsize.obj
 0001:0005b4f8       __acrt_fenv_get_common_round_control 000000018005c4f8 f   libucrt:_fenvutils.obj
 0001:0005b504       __acrt_fenv_get_control    000000018005c504 f   libucrt:_fenvutils.obj
 0001:0005b5f8       __acrt_fenv_get_status     000000018005c5f8 f   libucrt:_fenvutils.obj
 0001:0005b64c       __acrt_fenv_set_control    000000018005c64c f   libucrt:_fenvutils.obj
 0001:0005b794       __acrt_fenv_set_status     000000018005c794 f   libucrt:_fenvutils.obj
 0001:0005b818       __acrt_CompareStringW      000000018005c818 f   libucrt:comparestringw.obj
 0001:0005bbf8       __acrt_pack_wide_command_line_and_environment 000000018005cbf8 f   libucrt:cenvarg.obj
 0001:0005bd80       qsort                      000000018005cd80 f   libucrt:qsort.obj
 0001:0005c140       _mbsdec                    000000018005d140 f   libucrt:mbsdec.obj
 0001:0005c148       _mbsdec_l                  000000018005d148 f   libucrt:mbsdec.obj
 0001:0005c1f4       __strncnt                  000000018005d1f4 f   libucrt:strncnt.obj
 0001:0005c20c       ?__mbrtoc32_utf8@__crt_mbstring@@YA_KPEA_UPEBD_KPEAU_Mbstatet@@@Z 000000018005d20c f   libucrt:mbrtoc32.obj
 0001:0005c3e8       fegetenv                   000000018005d3e8 f   libucrt:fegetenv.obj
 0001:0005c408       fesetenv                   000000018005d408 f   libucrt:fesetenv.obj
 0001:0005c458       feholdexcept               000000018005d458 f   libucrt:feholdexcept.obj
 0001:0005c4a8       ceil                       000000018005d4a8 f   libucrt:ceil.obj
 0001:0005c570       log10                      000000018005d570 f   libucrt:log10.obj
 0001:0005cb1c       _query_app_type            000000018005db1c f   libucrt:report_runtime_error.obj
 0001:0005cb24       __dcrt_lowio_ensure_console_output_initialized 000000018005db24 f   libucrt:initcon.obj
 0001:0005cb78       __dcrt_terminate_console_output 000000018005db78 f   libucrt:initcon.obj
 0001:0005cb94       __dcrt_write_console       000000018005db94 f   libucrt:initcon.obj
 0001:0005cd78       _handle_error              000000018005dd78 f   libucrt:libm_error.obj
 0001:0005cea0       _handle_nan                000000018005dea0 f   libucrt:libm_error.obj
 0001:0005cec0       __acrt_initialize_fma3     000000018005dec0 f   libucrt:fma3_available.obj
 0001:0005cf30       _log10_special             000000018005df30 f   libucrt:log_special.obj
 0001:0005cfe8       _raise_exc                 000000018005dfe8 f   libucrt:fpexcept.obj
 0001:0005d010       _raise_exc_ex              000000018005e010 f   libucrt:fpexcept.obj
 0001:0005d320       _set_errno_from_matherr    000000018005e320 f   libucrt:fpexcept.obj
 0001:0005d350       _clrfp                     000000018005e350 f   libucrt:fpctrl.obj
 0001:0005d370       _ctrlfp                    000000018005e370 f   libucrt:fpctrl.obj
 0001:0005d3ec       _set_statfp                000000018005e3ec f   libucrt:fpctrl.obj
 0001:0005d40c       _statfp                    000000018005e40c f   libucrt:fpctrl.obj
 0001:0005d41d       IsProcessorFeaturePresent  000000018005e41d f   kernel32:KERNEL32.dll
 0001:0005d430       _FindPESection             000000018005e430 f   LIBCMT:pesect.obj
 0001:0005d480       _IsNonwritableInCurrentImage 000000018005e480 f   LIBCMT:pesect.obj
 0001:0005d4d0       _ValidateImageBase         000000018005e4d0 f   LIBCMT:pesect.obj
 0001:0005d500       __GSHandlerCheck           000000018005e500 f   LIBCMT:gshandler.obj
 0001:0005d520       __GSHandlerCheckCommon     000000018005e520 f   LIBCMT:gshandler.obj
 0001:0005d590       __security_check_cookie    000000018005e590 f   LIBCMT:amdsecgs.obj
 0001:0005d5b4       __GSHandlerCheck_SEH       000000018005e5b4 f   LIBCMT:gshandlerseh.obj
 0001:0005d63c       __raise_securityfailure    000000018005e63c f   LIBCMT:gs_report.obj
 0001:0005d670       __report_gsfailure         000000018005e670 f   LIBCMT:gs_report.obj
 0001:0005d744       __report_rangecheckfailure 000000018005e744 f   LIBCMT:gs_report.obj
 0001:0005d758       __report_securityfailure   000000018005e758 f   LIBCMT:gs_report.obj
 0001:0005d8d8       _local_unwind              000000018005e8d8 f   libvcruntime:jmpuwind.obj
 0001:0005d920       _guard_dispatch_icall_nop  000000018005e920 f   LIBCMT:guard_dispatch.obj
 0002:00000000       Keys                       0000000180063000     flags.obj
 0002:00001680       VirtualKeyStrings          0000000180064680     service.obj
 0002:0000b554       _fltused                   000000018006e554     LIBCMT:fltused.obj
 0002:0000b558       __scrt_native_dllmain_reason 000000018006e558     LIBCMT:utility.obj
 0002:0000b560       __security_cookie_complement 000000018006e560     LIBCMT:gs_cookie.obj
 0002:0000b568       __security_cookie          000000018006e568     LIBCMT:gs_cookie.obj
 0002:0000b570       __isa_available            000000018006e570     LIBCMT:cpu_disp.obj
 0002:0000b574       __isa_enabled              000000018006e574     LIBCMT:cpu_disp.obj
 0002:0000b578       __memcpy_nt_iters          000000018006e578     LIBCMT:cpu_disp.obj
 0002:0000b5a0       _iob                       000000018006e5a0     libucrt:_file.obj
 0002:0000b6b0       __abort_behavior           000000018006e6b0     libucrt:abort.obj
 0002:0000b6c0       __acrt_initial_locale_data 000000018006e6c0     libucrt:nlsdata.obj
 0002:0000b818       __acrt_initial_locale_pointers 000000018006e818     libucrt:nlsdata.obj
 0002:0000b828       __acrt_wide_c_locale_string 000000018006e828     libucrt:nlsdata.obj
 0002:0000b830       __badioinfo                000000018006e830     libucrt:ioinit.obj
 0002:0000b880       _lookuptrailbytes          000000018006e880     libucrt:read.obj
 0002:0000b980       _pwctype                   000000018006e980     libucrt:ctype.obj
 0002:0000bca0       __acrt_initial_multibyte_data 000000018006eca0     libucrt:mbctype.obj
 0002:0000bec8       __globallocalestatus       000000018006eec8     libucrt:glstatus.obj
 0002:0000bed0       __acrt_lconv_c             000000018006eed0     libucrt:localeconv.obj
 0002:0000bf68       __acrt_lconv_static_decimal 000000018006ef68     libucrt:localeconv.obj
 0002:0000bf6c       __acrt_lconv_static_W_decimal 000000018006ef6c     libucrt:localeconv.obj
 0002:0000bfb0       ?__type_info_root_node@@3U__type_info_node@@A 000000018006efb0     LIBCMT:tncleanup.obj
 0002:0000bfc0       __scrt_current_native_startup_state 000000018006efc0     LIBCMT:utility.obj
 0002:0000bfc8       __scrt_native_startup_lock 000000018006efc8     LIBCMT:utility.obj
 0002:0000c008       __scrt_debugger_hook_flag  000000018006f008     LIBCMT:utility_desktop.obj
 0002:0000c00c       __favor                    000000018006f00c     LIBCMT:cpu_disp.obj
 0002:0000c010       ?__WinRTOutOfMemoryExceptionCallback@@3P6APEAXXZEA 000000018006f010     libvcruntime:ehhelpers.obj
 0002:0000c018       ?pArgList@UnDecorator@@0PEAVReplicator@@EA 000000018006f018     libvcruntime:undname.obj
 0002:0000c020       ?pZNameList@UnDecorator@@0PEAVReplicator@@EA 000000018006f020     libvcruntime:undname.obj
 0002:0000c028       ?pTemplateArgList@UnDecorator@@0PEAVReplicator@@EA 000000018006f028     libvcruntime:undname.obj
 0002:0000c030       ?gName@UnDecorator@@0PEBDEB 000000018006f030     libvcruntime:undname.obj
 0002:0000c038       ?name@UnDecorator@@0PEBDEB 000000018006f038     libvcruntime:undname.obj
 0002:0000c040       ?disableFlags@UnDecorator@@0KA 000000018006f040     libvcruntime:undname.obj
 0002:0000c044       ?fExplicitTemplateParams@UnDecorator@@0_NA 000000018006f044     libvcruntime:undname.obj
 0002:0000c045       ?fGetTemplateArgumentList@UnDecorator@@0_NA 000000018006f045     libvcruntime:undname.obj
 0002:0000c048       ?m_pGetParameter@UnDecorator@@0P6APEADJ@ZEA 000000018006f048     libvcruntime:undname.obj
 0002:0000c050       ?m_CHPENameOffset@UnDecorator@@0KA 000000018006f050     libvcruntime:undname.obj
 0002:0000c054       ?m_recursionLevel@UnDecorator@@0KA 000000018006f054     libvcruntime:undname.obj
 0002:0000c180       __pPurecall                000000018006f180     libvcruntime:purevirt_data.obj
 0002:0000c188       _nstream                   000000018006f188     libucrt:_file.obj
 0002:0000c190       __piob                     000000018006f190     libucrt:_file.obj
 0002:0000c198       _cflush                    000000018006f198     libucrt:_file.obj
 0002:0000c1f0       ?c_exit_complete@?1???R<lambda_6e4b09c48022b2350581041d5f6b0c4c>@@QEBA@XZ@4_NA 000000018006f1f0     libucrt:exit.obj
 0002:0000c308       _environ_table             000000018006f308     libucrt:environment_initialization.obj
 0002:0000c310       _wenviron_table            000000018006f310     libucrt:environment_initialization.obj
 0002:0000c318       __dcrt_initial_wide_environment 000000018006f318     libucrt:environment_initialization.obj
 0002:0000c320       __dcrt_initial_narrow_environment 000000018006f320     libucrt:environment_initialization.obj
 0002:0000c328       __acrt_atexit_table        000000018006f328     libucrt:onexit.obj
 0002:0000c340       __acrt_at_quick_exit_table 000000018006f340     libucrt:onexit.obj
 0002:0000c370       __acrt_stdout_buffer       000000018006f370     libucrt:_sftbuf.obj
 0002:0000c378       __acrt_stderr_buffer       000000018006f378     libucrt:_sftbuf.obj
 0002:0000c380       __acrt_locale_changed_data 000000018006f380     libucrt:wsetlocale.obj
 0002:0000c388       __acrt_current_locale_data 000000018006f388     libucrt:nlsdata.obj
 0002:0000c390       __pioinfo                  000000018006f390     libucrt:ioinit.obj
 0002:0000c790       _nhandle                   000000018006f790     libucrt:ioinit.obj
 0002:0000cb84       _commode                   000000018006fb84     libucrt:ncommode.obj
 0002:0000cb88       _mbctype                   000000018006fb88     libucrt:mbctype.obj
 0002:0000cb90       _mbcasemap                 000000018006fb90     libucrt:mbctype.obj
 0002:0000cb98       __acrt_current_multibyte_data 000000018006fb98     libucrt:mbctype.obj
 0002:0000cba8       _pgmptr                    000000018006fba8     libucrt:argv_data.obj
 0002:0000cbb0       __argc                     000000018006fbb0     libucrt:argv_data.obj
 0002:0000cbb8       __argv                     000000018006fbb8     libucrt:argv_data.obj
 0002:0000cbc0       __wargv                    000000018006fbc0     libucrt:argv_data.obj
 0002:0000cbc8       _acmdln                    000000018006fbc8     libucrt:argv_data.obj
 0002:0000cbd0       _wcmdln                    000000018006fbd0     libucrt:argv_data.obj
 0002:0000cbd8       __acrt_heap                000000018006fbd8     libucrt:heap_handle.obj
 0002:0000cc14       __acrt_lconv_static_null   000000018006fc14     libucrt:localeconv.obj
 0002:0000cc18       __acrt_lconv_static_W_null 000000018006fc18     libucrt:localeconv.obj
 0002:0000cc1c       _umaskval                  000000018006fc1c     libucrt:umask.obj
 0002:0000cc2c       _fmode                     000000018006fc2c     libucrt:txtmode.obj
 0002:0000cc30       __fma3_is_available        000000018006fc30     libucrt:fma3_available.obj
 0002:0000cc34       __use_fma3_lib             000000018006fc34     libucrt:fma3_available.obj
 0002:0000d1b0       EnumCP                     00000001800701b0     <common>
 0002:0000d1c0       ?_OptionsStorage@?1??__local_stdio_scanf_options@@9@9 00000001800701c0     <common>
 0002:0000d1c8       ?_OptionsStorage@?1??__local_stdio_printf_options@@9@9 00000001800701c8     <common>
 0002:0000d1d0       __scrt_ucrt_dll_is_in_use  00000001800701d0     <common>
 0002:0000d1d8       __dyn_tls_init_callback    00000001800701d8     <common>
 0004:00000000       __imp_RegEnumValueW        0000000180075000     advapi32:ADVAPI32.dll
 0004:00000008       __imp_RegEnumKeyExW        0000000180075008     advapi32:ADVAPI32.dll
 0004:00000010       __imp_RegDeleteValueW      0000000180075010     advapi32:ADVAPI32.dll
 0004:00000018       __imp_RegDeleteKeyW        0000000180075018     advapi32:ADVAPI32.dll
 0004:00000020       __imp_RegSetValueExW       0000000180075020     advapi32:ADVAPI32.dll
 0004:00000028       __imp_RegQueryValueExW     0000000180075028     advapi32:ADVAPI32.dll
 0004:00000030       __imp_RegOpenKeyExW        0000000180075030     advapi32:ADVAPI32.dll
 0004:00000038       __imp_RegCreateKeyExW      0000000180075038     advapi32:ADVAPI32.dll
 0004:00000040       __imp_RegCloseKey          0000000180075040     advapi32:ADVAPI32.dll
 0004:00000048       \177ADVAPI32_NULL_THUNK_DATA 0000000180075048     advapi32:ADVAPI32.dll
 0004:00000050       __imp_GetConsoleScreenBufferInfo 0000000180075050     kernel32:KERNEL32.dll
 0004:00000058       __imp_FreeLibrary          0000000180075058     kernel32:KERNEL32.dll
 0004:00000060       __imp_GetModuleFileNameW   0000000180075060     kernel32:KERNEL32.dll
 0004:00000068       __imp_LoadLibraryW         0000000180075068     kernel32:KERNEL32.dll
 0004:00000070       __imp_SetCurrentDirectoryW 0000000180075070     kernel32:KERNEL32.dll
 0004:00000078       __imp_GetCurrentDirectoryW 0000000180075078     kernel32:KERNEL32.dll
 0004:00000080       __imp_SearchPathW          0000000180075080     kernel32:KERNEL32.dll
 0004:00000088       __imp_GetDriveTypeW        0000000180075088     kernel32:KERNEL32.dll
 0004:00000090       __imp_GetLogicalDriveStringsW 0000000180075090     kernel32:KERNEL32.dll
 0004:00000098       __imp_SetFileAttributesW   0000000180075098     kernel32:KERNEL32.dll
 0004:000000a0       __imp_OutputDebugStringW   00000001800750a0     kernel32:KERNEL32.dll
 0004:000000a8       __imp_GetLastError         00000001800750a8     kernel32:KERNEL32.dll
 0004:000000b0       __imp_Sleep                00000001800750b0     kernel32:KERNEL32.dll
 0004:000000b8       __imp_GlobalMemoryStatusEx 00000001800750b8     kernel32:KERNEL32.dll
 0004:000000c0       __imp_FormatMessageW       00000001800750c0     kernel32:KERNEL32.dll
 0004:000000c8       __imp_MultiByteToWideChar  00000001800750c8     kernel32:KERNEL32.dll
 0004:000000d0       __imp_WideCharToMultiByte  00000001800750d0     kernel32:KERNEL32.dll
 0004:000000d8       __imp_GetACP               00000001800750d8     kernel32:KERNEL32.dll
 0004:000000e0       __imp_GetOEMCP             00000001800750e0     kernel32:KERNEL32.dll
 0004:000000e8       __imp_GetCPInfoExW         00000001800750e8     kernel32:KERNEL32.dll
 0004:000000f0       __imp_EnumSystemCodePagesW 00000001800750f0     kernel32:KERNEL32.dll
 0004:000000f8       __imp_GetConsoleCP         00000001800750f8     kernel32:KERNEL32.dll
 0004:00000100       __imp_GetConsoleOutputCP   0000000180075100     kernel32:KERNEL32.dll
 0004:00000108       __imp_GetProcAddress       0000000180075108     kernel32:KERNEL32.dll
 0004:00000110       __imp_SetConsoleOutputCP   0000000180075110     kernel32:KERNEL32.dll
 0004:00000118       __imp_VerSetConditionMask  0000000180075118     kernel32:KERNEL32.dll
 0004:00000120       __imp_SetEnvironmentVariableW 0000000180075120     kernel32:KERNEL32.dll
 0004:00000128       __imp_CreateDirectoryW     0000000180075128     kernel32:KERNEL32.dll
 0004:00000130       __imp_DeleteFileW          0000000180075130     kernel32:KERNEL32.dll
 0004:00000138       __imp_FileTimeToLocalFileTime 0000000180075138     kernel32:KERNEL32.dll
 0004:00000140       __imp_FindClose            0000000180075140     kernel32:KERNEL32.dll
 0004:00000148       __imp_FindFirstFileW       0000000180075148     kernel32:KERNEL32.dll
 0004:00000150       __imp_RemoveDirectoryW     0000000180075150     kernel32:KERNEL32.dll
 0004:00000158       __imp_GetSystemTimeAsFileTime 0000000180075158     kernel32:KERNEL32.dll
 0004:00000160       __imp_GetModuleHandleW     0000000180075160     kernel32:KERNEL32.dll
 0004:00000168       __imp_CopyFileW            0000000180075168     kernel32:KERNEL32.dll
 0004:00000170       __imp_MoveFileExW          0000000180075170     kernel32:KERNEL32.dll
 0004:00000178       __imp_VerifyVersionInfoW   0000000180075178     kernel32:KERNEL32.dll
 0004:00000180       __imp_FileTimeToSystemTime 0000000180075180     kernel32:KERNEL32.dll
 0004:00000188       __imp_SystemTimeToFileTime 0000000180075188     kernel32:KERNEL32.dll
 0004:00000190       __imp_CompareStringW       0000000180075190     kernel32:KERNEL32.dll
 0004:00000198       __imp_ReadConsoleInputW    0000000180075198     kernel32:KERNEL32.dll
 0004:000001a0       __imp_PeekConsoleInputW    00000001800751a0     kernel32:KERNEL32.dll
 0004:000001a8       __imp_WriteConsoleW        00000001800751a8     kernel32:KERNEL32.dll
 0004:000001b0       __imp_SetEndOfFile         00000001800751b0     kernel32:KERNEL32.dll
 0004:000001b8       __imp_HeapReAlloc          00000001800751b8     kernel32:KERNEL32.dll
 0004:000001c0       __imp_HeapSize             00000001800751c0     kernel32:KERNEL32.dll
 0004:000001c8       __imp_GetModuleHandleA     00000001800751c8     kernel32:KERNEL32.dll
 0004:000001d0       __imp_DeleteTimerQueueTimer 00000001800751d0     kernel32:KERNEL32.dll
 0004:000001d8       __imp_ChangeTimerQueueTimer 00000001800751d8     kernel32:KERNEL32.dll
 0004:000001e0       __imp_CreateTimerQueueTimer 00000001800751e0     kernel32:KERNEL32.dll
 0004:000001e8       __imp_CreateTimerQueue     00000001800751e8     kernel32:KERNEL32.dll
 0004:000001f0       __imp_GetFileAttributesW   00000001800751f0     kernel32:KERNEL32.dll
 0004:000001f8       __imp_GetEnvironmentVariableW 00000001800751f8     kernel32:KERNEL32.dll
 0004:00000200       __imp_GetStdHandle         0000000180075200     kernel32:KERNEL32.dll
 0004:00000208       __imp_SetConsoleCP         0000000180075208     kernel32:KERNEL32.dll
 0004:00000210       __imp_DeleteTimerQueueEx   0000000180075210     kernel32:KERNEL32.dll
 0004:00000218       __imp_SetStdHandle         0000000180075218     kernel32:KERNEL32.dll
 0004:00000220       __imp_GetProcessHeap       0000000180075220     kernel32:KERNEL32.dll
 0004:00000228       __imp_FreeEnvironmentStringsW 0000000180075228     kernel32:KERNEL32.dll
 0004:00000230       __imp_GetEnvironmentStringsW 0000000180075230     kernel32:KERNEL32.dll
 0004:00000238       __imp_GetCommandLineW      0000000180075238     kernel32:KERNEL32.dll
 0004:00000240       __imp_GetCommandLineA      0000000180075240     kernel32:KERNEL32.dll
 0004:00000248       __imp_GetCPInfo            0000000180075248     kernel32:KERNEL32.dll
 0004:00000250       __imp_IsValidCodePage      0000000180075250     kernel32:KERNEL32.dll
 0004:00000258       __imp_FindNextFileW        0000000180075258     kernel32:KERNEL32.dll
 0004:00000260       __imp_FindFirstFileExW     0000000180075260     kernel32:KERNEL32.dll
 0004:00000268       __imp_CreateFileW          0000000180075268     kernel32:KERNEL32.dll
 0004:00000270       __imp_GetFileSizeEx        0000000180075270     kernel32:KERNEL32.dll
 0004:00000278       __imp_WriteFile            0000000180075278     kernel32:KERNEL32.dll
 0004:00000280       __imp_FlushFileBuffers     0000000180075280     kernel32:KERNEL32.dll
 0004:00000288       __imp_CreatePipe           0000000180075288     kernel32:KERNEL32.dll
 0004:00000290       __imp_GetFileAttributesExW 0000000180075290     kernel32:KERNEL32.dll
 0004:00000298       __imp_GetExitCodeProcess   0000000180075298     kernel32:KERNEL32.dll
 0004:000002a0       __imp_WaitForSingleObject  00000001800752a0     kernel32:KERNEL32.dll
 0004:000002a8       __imp_GetStringTypeW       00000001800752a8     kernel32:KERNEL32.dll
 0004:000002b0       __imp_SetFilePointerEx     00000001800752b0     kernel32:KERNEL32.dll
 0004:000002b8       __imp_ReadConsoleW         00000001800752b8     kernel32:KERNEL32.dll
 0004:000002c0       __imp_GetConsoleMode       00000001800752c0     kernel32:KERNEL32.dll
 0004:000002c8       __imp_LCMapStringW         00000001800752c8     kernel32:KERNEL32.dll
 0004:000002d0       __imp_GetFileType          00000001800752d0     kernel32:KERNEL32.dll
 0004:000002d8       __imp_HeapAlloc            00000001800752d8     kernel32:KERNEL32.dll
 0004:000002e0       __imp_HeapFree             00000001800752e0     kernel32:KERNEL32.dll
 0004:000002e8       __imp_GetModuleHandleExW   00000001800752e8     kernel32:KERNEL32.dll
 0004:000002f0       __imp_TerminateProcess     00000001800752f0     kernel32:KERNEL32.dll
 0004:000002f8       __imp_ExitProcess          00000001800752f8     kernel32:KERNEL32.dll
 0004:00000300       __imp_GetTempPathW         0000000180075300     kernel32:KERNEL32.dll
 0004:00000308       __imp_ReadFile             0000000180075308     kernel32:KERNEL32.dll
 0004:00000310       __imp_CreateProcessW       0000000180075310     kernel32:KERNEL32.dll
 0004:00000318       __imp_GetCurrentProcess    0000000180075318     kernel32:KERNEL32.dll
 0004:00000320       __imp_DuplicateHandle      0000000180075320     kernel32:KERNEL32.dll
 0004:00000328       __imp_CloseHandle          0000000180075328     kernel32:KERNEL32.dll
 0004:00000330       __imp_RaiseException       0000000180075330     kernel32:KERNEL32.dll
 0004:00000338       __imp_LoadLibraryExW       0000000180075338     kernel32:KERNEL32.dll
 0004:00000340       __imp_TlsFree              0000000180075340     kernel32:KERNEL32.dll
 0004:00000348       __imp_TlsSetValue          0000000180075348     kernel32:KERNEL32.dll
 0004:00000350       __imp_TlsGetValue          0000000180075350     kernel32:KERNEL32.dll
 0004:00000358       __imp_TlsAlloc             0000000180075358     kernel32:KERNEL32.dll
 0004:00000360       __imp_InitializeCriticalSectionAndSpinCount 0000000180075360     kernel32:KERNEL32.dll
 0004:00000368       __imp_DeleteCriticalSection 0000000180075368     kernel32:KERNEL32.dll
 0004:00000370       __imp_RtlUnwind            0000000180075370     kernel32:KERNEL32.dll
 0004:00000378       __imp_LeaveCriticalSection 0000000180075378     kernel32:KERNEL32.dll
 0004:00000380       __imp_EnterCriticalSection 0000000180075380     kernel32:KERNEL32.dll
 0004:00000388       __imp_SetLastError         0000000180075388     kernel32:KERNEL32.dll
 0004:00000390       __imp_InterlockedFlushSList 0000000180075390     kernel32:KERNEL32.dll
 0004:00000398       __imp_RtlUnwindEx          0000000180075398     kernel32:KERNEL32.dll
 0004:000003a0       __imp_IsProcessorFeaturePresent 00000001800753a0     kernel32:KERNEL32.dll
 0004:000003a8       __imp_GetStartupInfoW      00000001800753a8     kernel32:KERNEL32.dll
 0004:000003b0       __imp_SetUnhandledExceptionFilter 00000001800753b0     kernel32:KERNEL32.dll
 0004:000003b8       __imp_UnhandledExceptionFilter 00000001800753b8     kernel32:KERNEL32.dll
 0004:000003c0       __imp_IsDebuggerPresent    00000001800753c0     kernel32:KERNEL32.dll
 0004:000003c8       __imp_RtlVirtualUnwind     00000001800753c8     kernel32:KERNEL32.dll
 0004:000003d0       __imp_RtlLookupFunctionEntry 00000001800753d0     kernel32:KERNEL32.dll
 0004:000003d8       __imp_RtlCaptureContext    00000001800753d8     kernel32:KERNEL32.dll
 0004:000003e0       __imp_InitializeSListHead  00000001800753e0     kernel32:KERNEL32.dll
 0004:000003e8       __imp_GetCurrentThreadId   00000001800753e8     kernel32:KERNEL32.dll
 0004:000003f0       __imp_GetCurrentProcessId  00000001800753f0     kernel32:KERNEL32.dll
 0004:000003f8       __imp_QueryPerformanceCounter 00000001800753f8     kernel32:KERNEL32.dll
 0004:00000400       \177KERNEL32_NULL_THUNK_DATA 0000000180075400     kernel32:KERNEL32.dll
 0004:00000408       __imp_RpcStringFreeA       0000000180075408     rpcrt4:RPCRT4.dll
 0004:00000410       __imp_UuidCreate           0000000180075410     rpcrt4:RPCRT4.dll
 0004:00000418       __imp_UuidToStringA        0000000180075418     rpcrt4:RPCRT4.dll
 0004:00000420       __imp_UuidFromStringA      0000000180075420     rpcrt4:RPCRT4.dll
 0004:00000428       \177RPCRT4_NULL_THUNK_DATA 0000000180075428     rpcrt4:RPCRT4.dll
 0004:00000430       __imp_ShellExecuteW        0000000180075430     shell32:SHELL32.dll
 0004:00000438       __imp_SHGetFolderPathW     0000000180075438     shell32:SHELL32.dll
 0004:00000440       \177SHELL32_NULL_THUNK_DATA 0000000180075440     shell32:SHELL32.dll
 0004:00000448       __imp_GetKeyState          0000000180075448     user32:USER32.dll
 0004:00000450       \177USER32_NULL_THUNK_DATA 0000000180075450     user32:USER32.dll
 0004:00000458       __imp_lua_dump             0000000180075458     lua51:lua51.dll
 0004:00000460       __imp_luaL_prepbuffer      0000000180075460     lua51:lua51.dll
 0004:00000468       __imp_lua_typename         0000000180075468     lua51:lua51.dll
 0004:00000470       __imp_luaL_checkstack      0000000180075470     lua51:lua51.dll
 0004:00000478       __imp_lua_tocfunction      0000000180075478     lua51:lua51.dll
 0004:00000480       __imp_luaL_checkoption     0000000180075480     lua51:lua51.dll
 0004:00000488       __imp_lua_iscfunction      0000000180075488     lua51:lua51.dll
 0004:00000490       __imp_luaL_gsub            0000000180075490     lua51:lua51.dll
 0004:00000498       __imp_lua_isuserdata       0000000180075498     lua51:lua51.dll
 0004:000004a0       __imp_luaL_findtable       00000001800754a0     lua51:lua51.dll
 0004:000004a8       __imp_luaL_checkany        00000001800754a8     lua51:lua51.dll
 0004:000004b0       __imp_luaL_optnumber       00000001800754b0     lua51:lua51.dll
 0004:000004b8       __imp_luaL_checknumber     00000001800754b8     lua51:lua51.dll
 0004:000004c0       __imp_luaL_typerror        00000001800754c0     lua51:lua51.dll
 0004:000004c8       __imp_lua_setallocf        00000001800754c8     lua51:lua51.dll
 0004:000004d0       __imp_luaopen_debug        00000001800754d0     lua51:lua51.dll
 0004:000004d8       __imp_luaopen_math         00000001800754d8     lua51:lua51.dll
 0004:000004e0       __imp_luaopen_string       00000001800754e0     lua51:lua51.dll
 0004:000004e8       __imp_luaopen_os           00000001800754e8     lua51:lua51.dll
 0004:000004f0       __imp_luaopen_table        00000001800754f0     lua51:lua51.dll
 0004:000004f8       __imp_luaopen_base         00000001800754f8     lua51:lua51.dll
 0004:00000500       __imp_luaL_checktype       0000000180075500     lua51:lua51.dll
 0004:00000508       __imp_lua_getinfo          0000000180075508     lua51:lua51.dll
 0004:00000510       __imp_lua_getstack         0000000180075510     lua51:lua51.dll
 0004:00000518       __imp_luaL_addvalue        0000000180075518     lua51:lua51.dll
 0004:00000520       __imp_luaL_error           0000000180075520     lua51:lua51.dll
 0004:00000528       __imp_luaL_checkudata      0000000180075528     lua51:lua51.dll
 0004:00000530       __imp_luaL_optinteger      0000000180075530     lua51:lua51.dll
 0004:00000538       __imp_luaL_optlstring      0000000180075538     lua51:lua51.dll
 0004:00000540       __imp_luaL_checklstring    0000000180075540     lua51:lua51.dll
 0004:00000548       __imp_lua_checkstack       0000000180075548     lua51:lua51.dll
 0004:00000550       __imp_lua_replace          0000000180075550     lua51:lua51.dll
 0004:00000558       __imp_luaL_pushresult      0000000180075558     lua51:lua51.dll
 0004:00000560       __imp_luaL_buffinit        0000000180075560     lua51:lua51.dll
 0004:00000568       __imp_lua_concat           0000000180075568     lua51:lua51.dll
 0004:00000570       __imp_lua_error            0000000180075570     lua51:lua51.dll
 0004:00000578       __imp_lua_load             0000000180075578     lua51:lua51.dll
 0004:00000580       __imp_lua_pushfstring      0000000180075580     lua51:lua51.dll
 0004:00000588       __imp_lua_getallocf        0000000180075588     lua51:lua51.dll
 0004:00000590       __imp_luaL_unref           0000000180075590     lua51:lua51.dll
 0004:00000598       __imp_luaL_ref             0000000180075598     lua51:lua51.dll
 0004:000005a0       __imp_lua_gc               00000001800755a0     lua51:lua51.dll
 0004:000005a8       __imp_lua_pcall            00000001800755a8     lua51:lua51.dll
 0004:000005b0       __imp_lua_call             00000001800755b0     lua51:lua51.dll
 0004:000005b8       __imp_lua_rawseti          00000001800755b8     lua51:lua51.dll
 0004:000005c0       __imp_lua_rawset           00000001800755c0     lua51:lua51.dll
 0004:000005c8       __imp_lua_setfield         00000001800755c8     lua51:lua51.dll
 0004:000005d0       __imp_lua_createtable      00000001800755d0     lua51:lua51.dll
 0004:000005d8       __imp_lua_rawgeti          00000001800755d8     lua51:lua51.dll
 0004:000005e0       __imp_lua_rawget           00000001800755e0     lua51:lua51.dll
 0004:000005e8       __imp_lua_gettable         00000001800755e8     lua51:lua51.dll
 0004:000005f0       __imp_lua_pushlightuserdata 00000001800755f0     lua51:lua51.dll
 0004:000005f8       __imp_lua_pushcclosure     00000001800755f8     lua51:lua51.dll
 0004:00000600       __imp_lua_pushlstring      0000000180075600     lua51:lua51.dll
 0004:00000608       __imp_lua_pushinteger      0000000180075608     lua51:lua51.dll
 0004:00000610       __imp_lua_topointer        0000000180075610     lua51:lua51.dll
 0004:00000618       __imp_lua_objlen           0000000180075618     lua51:lua51.dll
 0004:00000620       __imp_lua_toboolean        0000000180075620     lua51:lua51.dll
 0004:00000628       __imp_lua_tointeger        0000000180075628     lua51:lua51.dll
 0004:00000630       __imp_lua_isstring         0000000180075630     lua51:lua51.dll
 0004:00000638       __imp_lua_isnumber         0000000180075638     lua51:lua51.dll
 0004:00000640       __imp_lua_insert           0000000180075640     lua51:lua51.dll
 0004:00000648       __imp_lua_remove           0000000180075648     lua51:lua51.dll
 0004:00000650       __imp_lua_pushvalue        0000000180075650     lua51:lua51.dll
 0004:00000658       __imp_luaL_newmetatable    0000000180075658     lua51:lua51.dll
 0004:00000660       __imp_luaL_checkinteger    0000000180075660     lua51:lua51.dll
 0004:00000668       __imp_luaL_argerror        0000000180075668     lua51:lua51.dll
 0004:00000670       __imp_luaL_register        0000000180075670     lua51:lua51.dll
 0004:00000678       __imp_lua_setmetatable     0000000180075678     lua51:lua51.dll
 0004:00000680       __imp_lua_getmetatable     0000000180075680     lua51:lua51.dll
 0004:00000688       __imp_lua_newuserdata      0000000180075688     lua51:lua51.dll
 0004:00000690       __imp_lua_getfield         0000000180075690     lua51:lua51.dll
 0004:00000698       __imp_lua_pushboolean      0000000180075698     lua51:lua51.dll
 0004:000006a0       __imp_lua_pushstring       00000001800756a0     lua51:lua51.dll
 0004:000006a8       __imp_lua_pushnumber       00000001800756a8     lua51:lua51.dll
 0004:000006b0       __imp_lua_pushnil          00000001800756b0     lua51:lua51.dll
 0004:000006b8       __imp_lua_touserdata       00000001800756b8     lua51:lua51.dll
 0004:000006c0       __imp_lua_tolstring        00000001800756c0     lua51:lua51.dll
 0004:000006c8       __imp_lua_tonumber         00000001800756c8     lua51:lua51.dll
 0004:000006d0       __imp_lua_rawequal         00000001800756d0     lua51:lua51.dll
 0004:000006d8       __imp_lua_type             00000001800756d8     lua51:lua51.dll
 0004:000006e0       __imp_lua_settop           00000001800756e0     lua51:lua51.dll
 0004:000006e8       __imp_lua_gettop           00000001800756e8     lua51:lua51.dll
 0004:000006f0       __imp_lua_next             00000001800756f0     lua51:lua51.dll
 0004:000006f8       __imp_lua_setfenv          00000001800756f8     lua51:lua51.dll
 0004:00000700       __imp_lua_settable         0000000180075700     lua51:lua51.dll
 0004:00000708       __imp_luaL_loadstring      0000000180075708     lua51:lua51.dll
 0004:00000710       __imp_lua_getfenv          0000000180075710     lua51:lua51.dll
 0004:00000718       __imp_luaL_addlstring      0000000180075718     lua51:lua51.dll
 0004:00000720       \177lua51_NULL_THUNK_DATA  0000000180075720     lua51:lua51.dll
 0004:00000728       __guard_check_icall_fptr   0000000180075728     LIBCMT:guard_support.obj
 0004:00000730       __guard_dispatch_icall_fptr 0000000180075730     LIBCMT:guard_support.obj
 0004:00000738       __IMPORT_DESCRIPTOR_KERNEL32 0000000180075738     kernel32:KERNEL32.dll
 0004:0000074c       __IMPORT_DESCRIPTOR_USER32 000000018007574c     user32:USER32.dll
 0004:00000760       __IMPORT_DESCRIPTOR_ADVAPI32 0000000180075760     advapi32:ADVAPI32.dll
 0004:00000774       __IMPORT_DESCRIPTOR_SHELL32 0000000180075774     shell32:SHELL32.dll
 0004:00000788       __IMPORT_DESCRIPTOR_lua51  0000000180075788     lua51:lua51.dll
 0004:0000079c       __IMPORT_DESCRIPTOR_RPCRT4 000000018007579c     rpcrt4:RPCRT4.dll
 0004:000007b0       __NULL_IMPORT_DESCRIPTOR   00000001800757b0     kernel32:KERNEL32.dll

 entry point at        0001:0003e264

 Static symbols

 0001:00000080       funcs                      0000000180001080     bit64.obj
 0001:000001a0       metamethods                00000001800011a0     bit64.obj
 0001:000003b0       FCF_FG_4BIT                00000001800013b0     exported.obj
 0001:000003b8       FCF_BG_4BIT                00000001800013b8     exported.obj
 0001:000003c0       FCF_4BITMASK               00000001800013c0     exported.obj
 0001:000003c8       FCF_RAWATTR_MASK           00000001800013c8     exported.obj
 0001:000003d0       FCF_EXTENDEDFLAGS          00000001800013d0     exported.obj
 0001:000003d8       FCF_FG_BOLD                00000001800013d8     exported.obj
 0001:000003e0       FCF_FG_ITALIC              00000001800013e0     exported.obj
 0001:000003e8       FCF_FG_UNDERLINE           00000001800013e8     exported.obj
 0001:000003f0       FCF_STYLEMASK              00000001800013f0     exported.obj
 0001:000003f8       FCF_NONE                   00000001800013f8     exported.obj
 0001:00000400       CDF_NONE                   0000000180001400     exported.obj
 0001:00000408       FMSG_WARNING               0000000180001408     exported.obj
 0001:00000410       FMSG_ERRORTYPE             0000000180001410     exported.obj
 0001:00000418       FMSG_KEEPBACKGROUND        0000000180001418     exported.obj
 0001:00000420       FMSG_LEFTALIGN             0000000180001420     exported.obj
 0001:00000428       FMSG_ALLINONE              0000000180001428     exported.obj
 0001:00000430       FMSG_MB_OK                 0000000180001430     exported.obj
 0001:00000438       FMSG_MB_OKCANCEL           0000000180001438     exported.obj
 0001:00000440       FMSG_MB_ABORTRETRYIGNORE   0000000180001440     exported.obj
 0001:00000448       FMSG_MB_YESNO              0000000180001448     exported.obj
 0001:00000450       FMSG_MB_YESNOCANCEL        0000000180001450     exported.obj
 0001:00000458       FMSG_MB_RETRYCANCEL        0000000180001458     exported.obj
 0001:00000460       FMSG_NONE                  0000000180001460     exported.obj
 0001:00000468       DIF_BOXCOLOR               0000000180001468     exported.obj
 0001:00000470       DIF_GROUP                  0000000180001470     exported.obj
 0001:00000478       DIF_LEFTTEXT               0000000180001478     exported.obj
 0001:00000480       DIF_MOVESELECT             0000000180001480     exported.obj
 0001:00000488       DIF_SHOWAMPERSAND          0000000180001488     exported.obj
 0001:00000490       DIF_CENTERGROUP            0000000180001490     exported.obj
 0001:00000498       DIF_NOBRACKETS             0000000180001498     exported.obj
 0001:000004a0       DIF_MANUALADDHISTORY       00000001800014a0     exported.obj
 0001:000004a8       DIF_SEPARATOR              00000001800014a8     exported.obj
 0001:000004b0       DIF_SEPARATOR2             00000001800014b0     exported.obj
 0001:000004b8       DIF_EDITOR                 00000001800014b8     exported.obj
 0001:000004c0       DIF_LISTNOAMPERSAND        00000001800014c0     exported.obj
 0001:000004c8       DIF_LISTNOBOX              00000001800014c8     exported.obj
 0001:000004d0       DIF_HISTORY                00000001800014d0     exported.obj
 0001:000004d8       DIF_BTNNOCLOSE             00000001800014d8     exported.obj
 0001:000004e0       DIF_CENTERTEXT             00000001800014e0     exported.obj
 0001:000004e8       DIF_SEPARATORUSER          00000001800014e8     exported.obj
 0001:000004f0       DIF_SETSHIELD              00000001800014f0     exported.obj
 0001:000004f8       DIF_EDITEXPAND             00000001800014f8     exported.obj
 0001:00000500       DIF_DROPDOWNLIST           0000000180001500     exported.obj
 0001:00000508       DIF_USELASTHISTORY         0000000180001508     exported.obj
 0001:00000510       DIF_MASKEDIT               0000000180001510     exported.obj
 0001:00000518       DIF_LISTTRACKMOUSE         0000000180001518     exported.obj
 0001:00000520       DIF_LISTTRACKMOUSEINFOCUS  0000000180001520     exported.obj
 0001:00000528       DIF_SELECTONENTRY          0000000180001528     exported.obj
 0001:00000530       DIF_3STATE                 0000000180001530     exported.obj
 0001:00000538       DIF_EDITPATH               0000000180001538     exported.obj
 0001:00000540       DIF_LISTWRAPMODE           0000000180001540     exported.obj
 0001:00000548       DIF_NOAUTOCOMPLETE         0000000180001548     exported.obj
 0001:00000550       DIF_LISTAUTOHIGHLIGHT      0000000180001550     exported.obj
 0001:00000558       DIF_LISTNOCLOSE            0000000180001558     exported.obj
 0001:00000560       DIF_EDITPATHEXEC           0000000180001560     exported.obj
 0001:00000568       DIF_HIDDEN                 0000000180001568     exported.obj
 0001:00000570       DIF_READONLY               0000000180001570     exported.obj
 0001:00000578       DIF_NOFOCUS                0000000180001578     exported.obj
 0001:00000580       DIF_DISABLE                0000000180001580     exported.obj
 0001:00000588       DIF_DEFAULTBUTTON          0000000180001588     exported.obj
 0001:00000590       DIF_FOCUS                  0000000180001590     exported.obj
 0001:00000598       DIF_RIGHTTEXT              0000000180001598     exported.obj
 0001:000005a0       DIF_WORDWRAP               00000001800015a0     exported.obj
 0001:000005a8       DIF_NONE                   00000001800015a8     exported.obj
 0001:000005b0       LIF_SELECTED               00000001800015b0     exported.obj
 0001:000005b8       LIF_CHECKED                00000001800015b8     exported.obj
 0001:000005c0       LIF_SEPARATOR              00000001800015c0     exported.obj
 0001:000005c8       LIF_DISABLE                00000001800015c8     exported.obj
 0001:000005d0       LIF_GRAYED                 00000001800015d0     exported.obj
 0001:000005d8       LIF_HIDDEN                 00000001800015d8     exported.obj
 0001:000005e0       LIF_DELETEUSERDATA         00000001800015e0     exported.obj
 0001:000005e8       LIF_NONE                   00000001800015e8     exported.obj
 0001:000005f0       LIFIND_EXACTMATCH          00000001800015f0     exported.obj
 0001:000005f8       LIFIND_NONE                00000001800015f8     exported.obj
 0001:00000600       LINFO_SHOWNOBOX            0000000180001600     exported.obj
 0001:00000608       LINFO_AUTOHIGHLIGHT        0000000180001608     exported.obj
 0001:00000610       LINFO_REVERSEHIGHLIGHT     0000000180001610     exported.obj
 0001:00000618       LINFO_WRAPMODE             0000000180001618     exported.obj
 0001:00000620       LINFO_SHOWAMPERSAND        0000000180001620     exported.obj
 0001:00000628       LINFO_NONE                 0000000180001628     exported.obj
 0001:00000630       FDLG_WARNING               0000000180001630     exported.obj
 0001:00000638       FDLG_SMALLDIALOG           0000000180001638     exported.obj
 0001:00000640       FDLG_NODRAWSHADOW          0000000180001640     exported.obj
 0001:00000648       FDLG_NODRAWPANEL           0000000180001648     exported.obj
 0001:00000650       FDLG_KEEPCONSOLETITLE      0000000180001650     exported.obj
 0001:00000658       FDLG_NONMODAL              0000000180001658     exported.obj
 0001:00000660       FDLG_NONE                  0000000180001660     exported.obj
 0001:00000668       MIF_SELECTED               0000000180001668     exported.obj
 0001:00000670       MIF_CHECKED                0000000180001670     exported.obj
 0001:00000678       MIF_SEPARATOR              0000000180001678     exported.obj
 0001:00000680       MIF_DISABLE                0000000180001680     exported.obj
 0001:00000688       MIF_GRAYED                 0000000180001688     exported.obj
 0001:00000690       MIF_HIDDEN                 0000000180001690     exported.obj
 0001:00000698       MIF_NONE                   0000000180001698     exported.obj
 0001:000006a0       FMENU_SHOWAMPERSAND        00000001800016a0     exported.obj
 0001:000006a8       FMENU_WRAPMODE             00000001800016a8     exported.obj
 0001:000006b0       FMENU_AUTOHIGHLIGHT        00000001800016b0     exported.obj
 0001:000006b8       FMENU_REVERSEAUTOHIGHLIGHT 00000001800016b8     exported.obj
 0001:000006c0       FMENU_CHANGECONSOLETITLE   00000001800016c0     exported.obj
 0001:000006c8       FMENU_SHOWNOBOX            00000001800016c8     exported.obj
 0001:000006d0       FMENU_SHOWSHORTBOX         00000001800016d0     exported.obj
 0001:000006d8       FMENU_SHOWSINGLEBOX        00000001800016d8     exported.obj
 0001:000006e0       FMENU_NODRAWSHADOW         00000001800016e0     exported.obj
 0001:000006e8       FMENU_NONE                 00000001800016e8     exported.obj
 0001:000006f0       PPIF_SELECTED              00000001800016f0     exported.obj
 0001:000006f8       PPIF_PROCESSDESCR          00000001800016f8     exported.obj
 0001:00000700       PPIF_NONE                  0000000180001700     exported.obj
 0001:00000708       PFLAGS_SHOWHIDDEN          0000000180001708     exported.obj
 0001:00000710       PFLAGS_HIGHLIGHT           0000000180001710     exported.obj
 0001:00000718       PFLAGS_REVERSESORTORDER    0000000180001718     exported.obj
 0001:00000720       PFLAGS_USESORTGROUPS       0000000180001720     exported.obj
 0001:00000728       PFLAGS_SELECTEDFIRST       0000000180001728     exported.obj
 0001:00000730       PFLAGS_REALNAMES           0000000180001730     exported.obj
 0001:00000738       PFLAGS_PANELLEFT           0000000180001738     exported.obj
 0001:00000740       PFLAGS_DIRECTORIESFIRST    0000000180001740     exported.obj
 0001:00000748       PFLAGS_USECRC32            0000000180001748     exported.obj
 0001:00000750       PFLAGS_PLUGIN              0000000180001750     exported.obj
 0001:00000758       PFLAGS_VISIBLE             0000000180001758     exported.obj
 0001:00000760       PFLAGS_FOCUS               0000000180001760     exported.obj
 0001:00000768       PFLAGS_ALTERNATIVENAMES    0000000180001768     exported.obj
 0001:00000770       PFLAGS_SHORTCUT            0000000180001770     exported.obj
 0001:00000778       PFLAGS_NONE                0000000180001778     exported.obj
 0001:00000780       VF_NONMODAL                0000000180001780     exported.obj
 0001:00000788       VF_DELETEONCLOSE           0000000180001788     exported.obj
 0001:00000790       VF_ENABLE_F6               0000000180001790     exported.obj
 0001:00000798       VF_DISABLEHISTORY          0000000180001798     exported.obj
 0001:000007a0       VF_IMMEDIATERETURN         00000001800017a0     exported.obj
 0001:000007a8       VF_DELETEONLYFILEONCLOSE   00000001800017a8     exported.obj
 0001:000007b0       VF_NONE                    00000001800017b0     exported.obj
 0001:000007b8       EF_NONMODAL                00000001800017b8     exported.obj
 0001:000007c0       EF_CREATENEW               00000001800017c0     exported.obj
 0001:000007c8       EF_ENABLE_F6               00000001800017c8     exported.obj
 0001:000007d0       EF_DISABLEHISTORY          00000001800017d0     exported.obj
 0001:000007d8       EF_DELETEONCLOSE           00000001800017d8     exported.obj
 0001:000007e0       EF_IMMEDIATERETURN         00000001800017e0     exported.obj
 0001:000007e8       EF_DELETEONLYFILEONCLOSE   00000001800017e8     exported.obj
 0001:000007f0       EF_LOCKED                  00000001800017f0     exported.obj
 0001:000007f8       EF_DISABLESAVEPOS          00000001800017f8     exported.obj
 0001:00000800       EF_OPENMODE_MASK           0000000180001800     exported.obj
 0001:00000808       EF_OPENMODE_QUERY          0000000180001808     exported.obj
 0001:00000810       EF_OPENMODE_NEWIFOPEN      0000000180001810     exported.obj
 0001:00000818       EF_OPENMODE_USEEXISTING    0000000180001818     exported.obj
 0001:00000820       EF_OPENMODE_BREAKIFOPEN    0000000180001820     exported.obj
 0001:00000828       EF_OPENMODE_RELOADIFOPEN   0000000180001828     exported.obj
 0001:00000830       EN_NONE                    0000000180001830     exported.obj
 0001:00000838       FHELP_NOSHOWERROR          0000000180001838     exported.obj
 0001:00000840       FHELP_SELFHELP             0000000180001840     exported.obj
 0001:00000848       FHELP_FARHELP              0000000180001848     exported.obj
 0001:00000850       FHELP_CUSTOMFILE           0000000180001850     exported.obj
 0001:00000858       FHELP_CUSTOMPATH           0000000180001858     exported.obj
 0001:00000860       FHELP_GUID                 0000000180001860     exported.obj
 0001:00000868       FHELP_USECONTENTS          0000000180001868     exported.obj
 0001:00000870       FHELP_NONE                 0000000180001870     exported.obj
 0001:00000878       KMFLAGS_SILENTCHECK        0000000180001878     exported.obj
 0001:00000880       KMFLAGS_NOSENDKEYSTOPLUGINS 0000000180001880     exported.obj
 0001:00000888       KMFLAGS_ENABLEOUTPUT       0000000180001888     exported.obj
 0001:00000890       KMFLAGS_LANGMASK           0000000180001890     exported.obj
 0001:00000898       KMFLAGS_LUA                0000000180001898     exported.obj
 0001:000008a0       KMFLAGS_MOONSCRIPT         00000001800018a0     exported.obj
 0001:000008a8       KMFLAGS_NONE               00000001800018a8     exported.obj
 0001:000008b0       AKMFLAGS_NONE              00000001800018b0     exported.obj
 0001:000008b8       FSETCLR_REDRAW             00000001800018b8     exported.obj
 0001:000008c0       FSETCLR_NONE               00000001800018c0     exported.obj
 0001:000008c8       WIF_MODIFIED               00000001800018c8     exported.obj
 0001:000008d0       WIF_CURRENT                00000001800018d0     exported.obj
 0001:000008d8       WIF_MODAL                  00000001800018d8     exported.obj
 0001:000008e0       WIF_NONE                   00000001800018e0     exported.obj
 0001:000008e8       VOPT_SAVEFILEPOSITION      00000001800018e8     exported.obj
 0001:000008f0       VOPT_AUTODETECTCODEPAGE    00000001800018f0     exported.obj
 0001:000008f8       VOPT_SHOWTITLEBAR          00000001800018f8     exported.obj
 0001:00000900       VOPT_SHOWKEYBAR            0000000180001900     exported.obj
 0001:00000908       VOPT_SHOWSCROLLBAR         0000000180001908     exported.obj
 0001:00000910       VOPT_QUICKVIEW             0000000180001910     exported.obj
 0001:00000918       VOPT_NONE                  0000000180001918     exported.obj
 0001:00000920       VSMFL_REDRAW               0000000180001920     exported.obj
 0001:00000928       VSMFL_NONE                 0000000180001928     exported.obj
 0001:00000930       VSP_NOREDRAW               0000000180001930     exported.obj
 0001:00000938       VSP_PERCENT                0000000180001938     exported.obj
 0001:00000940       VSP_RELATIVE               0000000180001940     exported.obj
 0001:00000948       VSP_NORETNEWPOS            0000000180001948     exported.obj
 0001:00000950       VSP_NONE                   0000000180001950     exported.obj
 0001:00000958       VMF_WRAP                   0000000180001958     exported.obj
 0001:00000960       VMF_WORDWRAP               0000000180001960     exported.obj
 0001:00000968       VMF_NONE                   0000000180001968     exported.obj
 0001:00000970       ECF_TABMARKFIRST           0000000180001970     exported.obj
 0001:00000978       ECF_TABMARKCURRENT         0000000180001978     exported.obj
 0001:00000980       ECF_AUTODELETE             0000000180001980     exported.obj
 0001:00000988       ECF_NONE                   0000000180001988     exported.obj
 0001:00000990       FIB_ENABLEEMPTY            0000000180001990     exported.obj
 0001:00000998       FIB_PASSWORD               0000000180001998     exported.obj
 0001:000009a0       FIB_EXPANDENV              00000001800019a0     exported.obj
 0001:000009a8       FIB_NOUSELASTHISTORY       00000001800019a8     exported.obj
 0001:000009b0       FIB_BUTTONS                00000001800019b0     exported.obj
 0001:000009b8       FIB_NOAMPERSAND            00000001800019b8     exported.obj
 0001:000009c0       FIB_EDITPATH               00000001800019c0     exported.obj
 0001:000009c8       FIB_EDITPATHEXEC           00000001800019c8     exported.obj
 0001:000009d0       FIB_NONE                   00000001800019d0     exported.obj
 0001:000009d8       FPF_LOADED                 00000001800019d8     exported.obj
 0001:000009e0       FPF_ANSI                   00000001800019e0     exported.obj
 0001:000009e8       FPF_NONE                   00000001800019e8     exported.obj
 0001:000009f0       PN_CMPNAME                 00000001800019f0     exported.obj
 0001:000009f8       PN_CMPNAMELIST             00000001800019f8     exported.obj
 0001:00000a00       PN_GENERATENAME            0000000180001a00     exported.obj
 0001:00000a08       PN_CHECKMASK               0000000180001a08     exported.obj
 0001:00000a10       PN_SKIPPATH                0000000180001a10     exported.obj
 0001:00000a18       PN_SHOWERRORMESSAGE        0000000180001a18     exported.obj
 0001:00000a20       PN_NONE                    0000000180001a20     exported.obj
 0001:00000a28       XLAT_SWITCHKEYBLAYOUT      0000000180001a28     exported.obj
 0001:00000a30       XLAT_SWITCHKEYBBEEP        0000000180001a30     exported.obj
 0001:00000a38       XLAT_USEKEYBLAYOUTNAME     0000000180001a38     exported.obj
 0001:00000a40       XLAT_CONVERTALLCMDLINE     0000000180001a40     exported.obj
 0001:00000a48       XLAT_NONE                  0000000180001a48     exported.obj
 0001:00000a50       FRS_RETUPDIR               0000000180001a50     exported.obj
 0001:00000a58       FRS_RECUR                  0000000180001a58     exported.obj
 0001:00000a60       FRS_SCANSYMLINK            0000000180001a60     exported.obj
 0001:00000a68       FRS_NONE                   0000000180001a68     exported.obj
 0001:00000a70       MLF_SHOWERRMSG             0000000180001a70     exported.obj
 0001:00000a78       MLF_DONOTUPDATEPANEL       0000000180001a78     exported.obj
 0001:00000a80       MLF_HOLDTARGET             0000000180001a80     exported.obj
 0001:00000a88       MLF_NONE                   0000000180001a88     exported.obj
 0001:00000a90       FFFS_COMMAS                0000000180001a90     exported.obj
 0001:00000a98       FFFS_FLOATSIZE             0000000180001a98     exported.obj
 0001:00000aa0       FFFS_SHOWBYTESINDEX        0000000180001aa0     exported.obj
 0001:00000aa8       FFFS_ECONOMIC              0000000180001aa8     exported.obj
 0001:00000ab0       FFFS_THOUSAND              0000000180001ab0     exported.obj
 0001:00000ab8       FFFS_MINSIZEINDEX          0000000180001ab8     exported.obj
 0001:00000ac0       FFFS_MINSIZEINDEX_MASK     0000000180001ac0     exported.obj
 0001:00000ac8       FFFS_NONE                  0000000180001ac8     exported.obj
 0001:00000ad0       PF_PRELOAD                 0000000180001ad0     exported.obj
 0001:00000ad8       PF_DISABLEPANELS           0000000180001ad8     exported.obj
 0001:00000ae0       PF_EDITOR                  0000000180001ae0     exported.obj
 0001:00000ae8       PF_VIEWER                  0000000180001ae8     exported.obj
 0001:00000af0       PF_FULLCMDLINE             0000000180001af0     exported.obj
 0001:00000af8       PF_DIALOG                  0000000180001af8     exported.obj
 0001:00000b00       PF_NONE                    0000000180001b00     exported.obj
 0001:00000b08       IPLFLAGS_SEPARATOR         0000000180001b08     exported.obj
 0001:00000b10       IPLFLAGS_NONE              0000000180001b10     exported.obj
 0001:00000b18       PMFLAGS_FULLSCREEN         0000000180001b18     exported.obj
 0001:00000b20       PMFLAGS_DETAILEDSTATUS     0000000180001b20     exported.obj
 0001:00000b28       PMFLAGS_ALIGNEXTENSIONS    0000000180001b28     exported.obj
 0001:00000b30       PMFLAGS_CASECONVERSION     0000000180001b30     exported.obj
 0001:00000b38       PMFLAGS_NONE               0000000180001b38     exported.obj
 0001:00000b40       OPIF_DISABLEFILTER         0000000180001b40     exported.obj
 0001:00000b48       OPIF_DISABLESORTGROUPS     0000000180001b48     exported.obj
 0001:00000b50       OPIF_DISABLEHIGHLIGHTING   0000000180001b50     exported.obj
 0001:00000b58       OPIF_ADDDOTS               0000000180001b58     exported.obj
 0001:00000b60       OPIF_RAWSELECTION          0000000180001b60     exported.obj
 0001:00000b68       OPIF_REALNAMES             0000000180001b68     exported.obj
 0001:00000b70       OPIF_SHOWNAMESONLY         0000000180001b70     exported.obj
 0001:00000b78       OPIF_SHOWRIGHTALIGNNAMES   0000000180001b78     exported.obj
 0001:00000b80       OPIF_SHOWPRESERVECASE      0000000180001b80     exported.obj
 0001:00000b88       OPIF_COMPAREFATTIME        0000000180001b88     exported.obj
 0001:00000b90       OPIF_EXTERNALGET           0000000180001b90     exported.obj
 0001:00000b98       OPIF_EXTERNALPUT           0000000180001b98     exported.obj
 0001:00000ba0       OPIF_EXTERNALDELETE        0000000180001ba0     exported.obj
 0001:00000ba8       OPIF_EXTERNALMKDIR         0000000180001ba8     exported.obj
 0001:00000bb0       OPIF_USEATTRHIGHLIGHTING   0000000180001bb0     exported.obj
 0001:00000bb8       OPIF_USECRC32              0000000180001bb8     exported.obj
 0001:00000bc0       OPIF_USEFREESIZE           0000000180001bc0     exported.obj
 0001:00000bc8       OPIF_SHORTCUT              0000000180001bc8     exported.obj
 0001:00000bd0       OPIF_NONE                  0000000180001bd0     exported.obj
 0001:00000bd8       OPM_SILENT                 0000000180001bd8     exported.obj
 0001:00000be0       OPM_FIND                   0000000180001be0     exported.obj
 0001:00000be8       OPM_VIEW                   0000000180001be8     exported.obj
 0001:00000bf0       OPM_EDIT                   0000000180001bf0     exported.obj
 0001:00000bf8       OPM_TOPLEVEL               0000000180001bf8     exported.obj
 0001:00000c00       OPM_DESCR                  0000000180001c00     exported.obj
 0001:00000c08       OPM_QUICKVIEW              0000000180001c08     exported.obj
 0001:00000c10       OPM_PGDN                   0000000180001c10     exported.obj
 0001:00000c18       OPM_COMMANDS               0000000180001c18     exported.obj
 0001:00000c20       OPM_NONE                   0000000180001c20     exported.obj
 0001:00000c28       FOSF_ACTIVE                0000000180001c28     exported.obj
 0001:00000c30       FOSF_NONE                  0000000180001c30     exported.obj
 0001:00000c38       PCIF_NONE                  0000000180001c38     exported.obj
 0001:00000c40       FarGuid                    0000000180001c40     exported.obj
 0001:00000c50       PDF_DIALOGEVENTDRAWENABLE  0000000180001c50     exported.obj
 0001:00000c58       PDF_PROCESSINGERROR        0000000180001c58     exported.obj
 0001:00000c60       PDF_FULL_TIME_RESOLUTION   0000000180001c60     exported.obj
 0001:00001310       FCF_FG_4BIT                0000000180002310     flags.obj
 0001:00001318       FCF_BG_4BIT                0000000180002318     flags.obj
 0001:00001320       FCF_4BITMASK               0000000180002320     flags.obj
 0001:00001328       FCF_RAWATTR_MASK           0000000180002328     flags.obj
 0001:00001330       FCF_EXTENDEDFLAGS          0000000180002330     flags.obj
 0001:00001338       FCF_FG_BOLD                0000000180002338     flags.obj
 0001:00001340       FCF_FG_ITALIC              0000000180002340     flags.obj
 0001:00001348       FCF_FG_UNDERLINE           0000000180002348     flags.obj
 0001:00001350       FCF_STYLEMASK              0000000180002350     flags.obj
 0001:00001358       FCF_NONE                   0000000180002358     flags.obj
 0001:00001360       CDF_NONE                   0000000180002360     flags.obj
 0001:00001368       FMSG_WARNING               0000000180002368     flags.obj
 0001:00001370       FMSG_ERRORTYPE             0000000180002370     flags.obj
 0001:00001378       FMSG_KEEPBACKGROUND        0000000180002378     flags.obj
 0001:00001380       FMSG_LEFTALIGN             0000000180002380     flags.obj
 0001:00001388       FMSG_ALLINONE              0000000180002388     flags.obj
 0001:00001390       FMSG_MB_OK                 0000000180002390     flags.obj
 0001:00001398       FMSG_MB_OKCANCEL           0000000180002398     flags.obj
 0001:000013a0       FMSG_MB_ABORTRETRYIGNORE   00000001800023a0     flags.obj
 0001:000013a8       FMSG_MB_YESNO              00000001800023a8     flags.obj
 0001:000013b0       FMSG_MB_YESNOCANCEL        00000001800023b0     flags.obj
 0001:000013b8       FMSG_MB_RETRYCANCEL        00000001800023b8     flags.obj
 0001:000013c0       FMSG_NONE                  00000001800023c0     flags.obj
 0001:000013c8       DIF_BOXCOLOR               00000001800023c8     flags.obj
 0001:000013d0       DIF_GROUP                  00000001800023d0     flags.obj
 0001:000013d8       DIF_LEFTTEXT               00000001800023d8     flags.obj
 0001:000013e0       DIF_MOVESELECT             00000001800023e0     flags.obj
 0001:000013e8       DIF_SHOWAMPERSAND          00000001800023e8     flags.obj
 0001:000013f0       DIF_CENTERGROUP            00000001800023f0     flags.obj
 0001:000013f8       DIF_NOBRACKETS             00000001800023f8     flags.obj
 0001:00001400       DIF_MANUALADDHISTORY       0000000180002400     flags.obj
 0001:00001408       DIF_SEPARATOR              0000000180002408     flags.obj
 0001:00001410       DIF_SEPARATOR2             0000000180002410     flags.obj
 0001:00001418       DIF_EDITOR                 0000000180002418     flags.obj
 0001:00001420       DIF_LISTNOAMPERSAND        0000000180002420     flags.obj
 0001:00001428       DIF_LISTNOBOX              0000000180002428     flags.obj
 0001:00001430       DIF_HISTORY                0000000180002430     flags.obj
 0001:00001438       DIF_BTNNOCLOSE             0000000180002438     flags.obj
 0001:00001440       DIF_CENTERTEXT             0000000180002440     flags.obj
 0001:00001448       DIF_SEPARATORUSER          0000000180002448     flags.obj
 0001:00001450       DIF_SETSHIELD              0000000180002450     flags.obj
 0001:00001458       DIF_EDITEXPAND             0000000180002458     flags.obj
 0001:00001460       DIF_DROPDOWNLIST           0000000180002460     flags.obj
 0001:00001468       DIF_USELASTHISTORY         0000000180002468     flags.obj
 0001:00001470       DIF_MASKEDIT               0000000180002470     flags.obj
 0001:00001478       DIF_LISTTRACKMOUSE         0000000180002478     flags.obj
 0001:00001480       DIF_LISTTRACKMOUSEINFOCUS  0000000180002480     flags.obj
 0001:00001488       DIF_SELECTONENTRY          0000000180002488     flags.obj
 0001:00001490       DIF_3STATE                 0000000180002490     flags.obj
 0001:00001498       DIF_EDITPATH               0000000180002498     flags.obj
 0001:000014a0       DIF_LISTWRAPMODE           00000001800024a0     flags.obj
 0001:000014a8       DIF_NOAUTOCOMPLETE         00000001800024a8     flags.obj
 0001:000014b0       DIF_LISTAUTOHIGHLIGHT      00000001800024b0     flags.obj
 0001:000014b8       DIF_LISTNOCLOSE            00000001800024b8     flags.obj
 0001:000014c0       DIF_EDITPATHEXEC           00000001800024c0     flags.obj
 0001:000014c8       DIF_HIDDEN                 00000001800024c8     flags.obj
 0001:000014d0       DIF_READONLY               00000001800024d0     flags.obj
 0001:000014d8       DIF_NOFOCUS                00000001800024d8     flags.obj
 0001:000014e0       DIF_DISABLE                00000001800024e0     flags.obj
 0001:000014e8       DIF_DEFAULTBUTTON          00000001800024e8     flags.obj
 0001:000014f0       DIF_FOCUS                  00000001800024f0     flags.obj
 0001:000014f8       DIF_RIGHTTEXT              00000001800024f8     flags.obj
 0001:00001500       DIF_WORDWRAP               0000000180002500     flags.obj
 0001:00001508       DIF_NONE                   0000000180002508     flags.obj
 0001:00001510       LIF_SELECTED               0000000180002510     flags.obj
 0001:00001518       LIF_CHECKED                0000000180002518     flags.obj
 0001:00001520       LIF_SEPARATOR              0000000180002520     flags.obj
 0001:00001528       LIF_DISABLE                0000000180002528     flags.obj
 0001:00001530       LIF_GRAYED                 0000000180002530     flags.obj
 0001:00001538       LIF_HIDDEN                 0000000180002538     flags.obj
 0001:00001540       LIF_DELETEUSERDATA         0000000180002540     flags.obj
 0001:00001548       LIF_NONE                   0000000180002548     flags.obj
 0001:00001550       LIFIND_EXACTMATCH          0000000180002550     flags.obj
 0001:00001558       LIFIND_NONE                0000000180002558     flags.obj
 0001:00001560       LINFO_SHOWNOBOX            0000000180002560     flags.obj
 0001:00001568       LINFO_AUTOHIGHLIGHT        0000000180002568     flags.obj
 0001:00001570       LINFO_REVERSEHIGHLIGHT     0000000180002570     flags.obj
 0001:00001578       LINFO_WRAPMODE             0000000180002578     flags.obj
 0001:00001580       LINFO_SHOWAMPERSAND        0000000180002580     flags.obj
 0001:00001588       LINFO_NONE                 0000000180002588     flags.obj
 0001:00001590       FDLG_WARNING               0000000180002590     flags.obj
 0001:00001598       FDLG_SMALLDIALOG           0000000180002598     flags.obj
 0001:000015a0       FDLG_NODRAWSHADOW          00000001800025a0     flags.obj
 0001:000015a8       FDLG_NODRAWPANEL           00000001800025a8     flags.obj
 0001:000015b0       FDLG_KEEPCONSOLETITLE      00000001800025b0     flags.obj
 0001:000015b8       FDLG_NONMODAL              00000001800025b8     flags.obj
 0001:000015c0       FDLG_NONE                  00000001800025c0     flags.obj
 0001:000015c8       MIF_SELECTED               00000001800025c8     flags.obj
 0001:000015d0       MIF_CHECKED                00000001800025d0     flags.obj
 0001:000015d8       MIF_SEPARATOR              00000001800025d8     flags.obj
 0001:000015e0       MIF_DISABLE                00000001800025e0     flags.obj
 0001:000015e8       MIF_GRAYED                 00000001800025e8     flags.obj
 0001:000015f0       MIF_HIDDEN                 00000001800025f0     flags.obj
 0001:000015f8       MIF_NONE                   00000001800025f8     flags.obj
 0001:00001600       FMENU_SHOWAMPERSAND        0000000180002600     flags.obj
 0001:00001608       FMENU_WRAPMODE             0000000180002608     flags.obj
 0001:00001610       FMENU_AUTOHIGHLIGHT        0000000180002610     flags.obj
 0001:00001618       FMENU_REVERSEAUTOHIGHLIGHT 0000000180002618     flags.obj
 0001:00001620       FMENU_CHANGECONSOLETITLE   0000000180002620     flags.obj
 0001:00001628       FMENU_SHOWNOBOX            0000000180002628     flags.obj
 0001:00001630       FMENU_SHOWSHORTBOX         0000000180002630     flags.obj
 0001:00001638       FMENU_SHOWSINGLEBOX        0000000180002638     flags.obj
 0001:00001640       FMENU_NODRAWSHADOW         0000000180002640     flags.obj
 0001:00001648       FMENU_NONE                 0000000180002648     flags.obj
 0001:00001650       PPIF_SELECTED              0000000180002650     flags.obj
 0001:00001658       PPIF_PROCESSDESCR          0000000180002658     flags.obj
 0001:00001660       PPIF_NONE                  0000000180002660     flags.obj
 0001:00001668       PFLAGS_SHOWHIDDEN          0000000180002668     flags.obj
 0001:00001670       PFLAGS_HIGHLIGHT           0000000180002670     flags.obj
 0001:00001678       PFLAGS_REVERSESORTORDER    0000000180002678     flags.obj
 0001:00001680       PFLAGS_USESORTGROUPS       0000000180002680     flags.obj
 0001:00001688       PFLAGS_SELECTEDFIRST       0000000180002688     flags.obj
 0001:00001690       PFLAGS_REALNAMES           0000000180002690     flags.obj
 0001:00001698       PFLAGS_PANELLEFT           0000000180002698     flags.obj
 0001:000016a0       PFLAGS_DIRECTORIESFIRST    00000001800026a0     flags.obj
 0001:000016a8       PFLAGS_USECRC32            00000001800026a8     flags.obj
 0001:000016b0       PFLAGS_PLUGIN              00000001800026b0     flags.obj
 0001:000016b8       PFLAGS_VISIBLE             00000001800026b8     flags.obj
 0001:000016c0       PFLAGS_FOCUS               00000001800026c0     flags.obj
 0001:000016c8       PFLAGS_ALTERNATIVENAMES    00000001800026c8     flags.obj
 0001:000016d0       PFLAGS_SHORTCUT            00000001800026d0     flags.obj
 0001:000016d8       PFLAGS_NONE                00000001800026d8     flags.obj
 0001:000016e0       VF_NONMODAL                00000001800026e0     flags.obj
 0001:000016e8       VF_DELETEONCLOSE           00000001800026e8     flags.obj
 0001:000016f0       VF_ENABLE_F6               00000001800026f0     flags.obj
 0001:000016f8       VF_DISABLEHISTORY          00000001800026f8     flags.obj
 0001:00001700       VF_IMMEDIATERETURN         0000000180002700     flags.obj
 0001:00001708       VF_DELETEONLYFILEONCLOSE   0000000180002708     flags.obj
 0001:00001710       VF_NONE                    0000000180002710     flags.obj
 0001:00001718       EF_NONMODAL                0000000180002718     flags.obj
 0001:00001720       EF_CREATENEW               0000000180002720     flags.obj
 0001:00001728       EF_ENABLE_F6               0000000180002728     flags.obj
 0001:00001730       EF_DISABLEHISTORY          0000000180002730     flags.obj
 0001:00001738       EF_DELETEONCLOSE           0000000180002738     flags.obj
 0001:00001740       EF_IMMEDIATERETURN         0000000180002740     flags.obj
 0001:00001748       EF_DELETEONLYFILEONCLOSE   0000000180002748     flags.obj
 0001:00001750       EF_LOCKED                  0000000180002750     flags.obj
 0001:00001758       EF_DISABLESAVEPOS          0000000180002758     flags.obj
 0001:00001760       EF_OPENMODE_MASK           0000000180002760     flags.obj
 0001:00001768       EF_OPENMODE_QUERY          0000000180002768     flags.obj
 0001:00001770       EF_OPENMODE_NEWIFOPEN      0000000180002770     flags.obj
 0001:00001778       EF_OPENMODE_USEEXISTING    0000000180002778     flags.obj
 0001:00001780       EF_OPENMODE_BREAKIFOPEN    0000000180002780     flags.obj
 0001:00001788       EF_OPENMODE_RELOADIFOPEN   0000000180002788     flags.obj
 0001:00001790       EN_NONE                    0000000180002790     flags.obj
 0001:00001798       FHELP_NOSHOWERROR          0000000180002798     flags.obj
 0001:000017a0       FHELP_SELFHELP             00000001800027a0     flags.obj
 0001:000017a8       FHELP_FARHELP              00000001800027a8     flags.obj
 0001:000017b0       FHELP_CUSTOMFILE           00000001800027b0     flags.obj
 0001:000017b8       FHELP_CUSTOMPATH           00000001800027b8     flags.obj
 0001:000017c0       FHELP_GUID                 00000001800027c0     flags.obj
 0001:000017c8       FHELP_USECONTENTS          00000001800027c8     flags.obj
 0001:000017d0       FHELP_NONE                 00000001800027d0     flags.obj
 0001:000017d8       KMFLAGS_SILENTCHECK        00000001800027d8     flags.obj
 0001:000017e0       KMFLAGS_NOSENDKEYSTOPLUGINS 00000001800027e0     flags.obj
 0001:000017e8       KMFLAGS_ENABLEOUTPUT       00000001800027e8     flags.obj
 0001:000017f0       KMFLAGS_LANGMASK           00000001800027f0     flags.obj
 0001:000017f8       KMFLAGS_LUA                00000001800027f8     flags.obj
 0001:00001800       KMFLAGS_MOONSCRIPT         0000000180002800     flags.obj
 0001:00001808       KMFLAGS_NONE               0000000180002808     flags.obj
 0001:00001810       AKMFLAGS_NONE              0000000180002810     flags.obj
 0001:00001818       FSETCLR_REDRAW             0000000180002818     flags.obj
 0001:00001820       FSETCLR_NONE               0000000180002820     flags.obj
 0001:00001828       WIF_MODIFIED               0000000180002828     flags.obj
 0001:00001830       WIF_CURRENT                0000000180002830     flags.obj
 0001:00001838       WIF_MODAL                  0000000180002838     flags.obj
 0001:00001840       WIF_NONE                   0000000180002840     flags.obj
 0001:00001848       VOPT_SAVEFILEPOSITION      0000000180002848     flags.obj
 0001:00001850       VOPT_AUTODETECTCODEPAGE    0000000180002850     flags.obj
 0001:00001858       VOPT_SHOWTITLEBAR          0000000180002858     flags.obj
 0001:00001860       VOPT_SHOWKEYBAR            0000000180002860     flags.obj
 0001:00001868       VOPT_SHOWSCROLLBAR         0000000180002868     flags.obj
 0001:00001870       VOPT_QUICKVIEW             0000000180002870     flags.obj
 0001:00001878       VOPT_NONE                  0000000180002878     flags.obj
 0001:00001880       VSMFL_REDRAW               0000000180002880     flags.obj
 0001:00001888       VSMFL_NONE                 0000000180002888     flags.obj
 0001:00001890       VSP_NOREDRAW               0000000180002890     flags.obj
 0001:00001898       VSP_PERCENT                0000000180002898     flags.obj
 0001:000018a0       VSP_RELATIVE               00000001800028a0     flags.obj
 0001:000018a8       VSP_NORETNEWPOS            00000001800028a8     flags.obj
 0001:000018b0       VSP_NONE                   00000001800028b0     flags.obj
 0001:000018b8       VMF_WRAP                   00000001800028b8     flags.obj
 0001:000018c0       VMF_WORDWRAP               00000001800028c0     flags.obj
 0001:000018c8       VMF_NONE                   00000001800028c8     flags.obj
 0001:000018d0       ECF_TABMARKFIRST           00000001800028d0     flags.obj
 0001:000018d8       ECF_TABMARKCURRENT         00000001800028d8     flags.obj
 0001:000018e0       ECF_AUTODELETE             00000001800028e0     flags.obj
 0001:000018e8       ECF_NONE                   00000001800028e8     flags.obj
 0001:000018f0       FIB_ENABLEEMPTY            00000001800028f0     flags.obj
 0001:000018f8       FIB_PASSWORD               00000001800028f8     flags.obj
 0001:00001900       FIB_EXPANDENV              0000000180002900     flags.obj
 0001:00001908       FIB_NOUSELASTHISTORY       0000000180002908     flags.obj
 0001:00001910       FIB_BUTTONS                0000000180002910     flags.obj
 0001:00001918       FIB_NOAMPERSAND            0000000180002918     flags.obj
 0001:00001920       FIB_EDITPATH               0000000180002920     flags.obj
 0001:00001928       FIB_EDITPATHEXEC           0000000180002928     flags.obj
 0001:00001930       FIB_NONE                   0000000180002930     flags.obj
 0001:00001938       FPF_LOADED                 0000000180002938     flags.obj
 0001:00001940       FPF_ANSI                   0000000180002940     flags.obj
 0001:00001948       FPF_NONE                   0000000180002948     flags.obj
 0001:00001950       PN_CMPNAME                 0000000180002950     flags.obj
 0001:00001958       PN_CMPNAMELIST             0000000180002958     flags.obj
 0001:00001960       PN_GENERATENAME            0000000180002960     flags.obj
 0001:00001968       PN_CHECKMASK               0000000180002968     flags.obj
 0001:00001970       PN_SKIPPATH                0000000180002970     flags.obj
 0001:00001978       PN_SHOWERRORMESSAGE        0000000180002978     flags.obj
 0001:00001980       PN_NONE                    0000000180002980     flags.obj
 0001:00001988       XLAT_SWITCHKEYBLAYOUT      0000000180002988     flags.obj
 0001:00001990       XLAT_SWITCHKEYBBEEP        0000000180002990     flags.obj
 0001:00001998       XLAT_USEKEYBLAYOUTNAME     0000000180002998     flags.obj
 0001:000019a0       XLAT_CONVERTALLCMDLINE     00000001800029a0     flags.obj
 0001:000019a8       XLAT_NONE                  00000001800029a8     flags.obj
 0001:000019b0       FRS_RETUPDIR               00000001800029b0     flags.obj
 0001:000019b8       FRS_RECUR                  00000001800029b8     flags.obj
 0001:000019c0       FRS_SCANSYMLINK            00000001800029c0     flags.obj
 0001:000019c8       FRS_NONE                   00000001800029c8     flags.obj
 0001:000019d0       MLF_SHOWERRMSG             00000001800029d0     flags.obj
 0001:000019d8       MLF_DONOTUPDATEPANEL       00000001800029d8     flags.obj
 0001:000019e0       MLF_HOLDTARGET             00000001800029e0     flags.obj
 0001:000019e8       MLF_NONE                   00000001800029e8     flags.obj
 0001:000019f0       FFFS_COMMAS                00000001800029f0     flags.obj
 0001:000019f8       FFFS_FLOATSIZE             00000001800029f8     flags.obj
 0001:00001a00       FFFS_SHOWBYTESINDEX        0000000180002a00     flags.obj
 0001:00001a08       FFFS_ECONOMIC              0000000180002a08     flags.obj
 0001:00001a10       FFFS_THOUSAND              0000000180002a10     flags.obj
 0001:00001a18       FFFS_MINSIZEINDEX          0000000180002a18     flags.obj
 0001:00001a20       FFFS_MINSIZEINDEX_MASK     0000000180002a20     flags.obj
 0001:00001a28       FFFS_NONE                  0000000180002a28     flags.obj
 0001:00001a30       PF_PRELOAD                 0000000180002a30     flags.obj
 0001:00001a38       PF_DISABLEPANELS           0000000180002a38     flags.obj
 0001:00001a40       PF_EDITOR                  0000000180002a40     flags.obj
 0001:00001a48       PF_VIEWER                  0000000180002a48     flags.obj
 0001:00001a50       PF_FULLCMDLINE             0000000180002a50     flags.obj
 0001:00001a58       PF_DIALOG                  0000000180002a58     flags.obj
 0001:00001a60       PF_NONE                    0000000180002a60     flags.obj
 0001:00001a68       IPLFLAGS_SEPARATOR         0000000180002a68     flags.obj
 0001:00001a70       IPLFLAGS_NONE              0000000180002a70     flags.obj
 0001:00001a78       PMFLAGS_FULLSCREEN         0000000180002a78     flags.obj
 0001:00001a80       PMFLAGS_DETAILEDSTATUS     0000000180002a80     flags.obj
 0001:00001a88       PMFLAGS_ALIGNEXTENSIONS    0000000180002a88     flags.obj
 0001:00001a90       PMFLAGS_CASECONVERSION     0000000180002a90     flags.obj
 0001:00001a98       PMFLAGS_NONE               0000000180002a98     flags.obj
 0001:00001aa0       OPIF_DISABLEFILTER         0000000180002aa0     flags.obj
 0001:00001aa8       OPIF_DISABLESORTGROUPS     0000000180002aa8     flags.obj
 0001:00001ab0       OPIF_DISABLEHIGHLIGHTING   0000000180002ab0     flags.obj
 0001:00001ab8       OPIF_ADDDOTS               0000000180002ab8     flags.obj
 0001:00001ac0       OPIF_RAWSELECTION          0000000180002ac0     flags.obj
 0001:00001ac8       OPIF_REALNAMES             0000000180002ac8     flags.obj
 0001:00001ad0       OPIF_SHOWNAMESONLY         0000000180002ad0     flags.obj
 0001:00001ad8       OPIF_SHOWRIGHTALIGNNAMES   0000000180002ad8     flags.obj
 0001:00001ae0       OPIF_SHOWPRESERVECASE      0000000180002ae0     flags.obj
 0001:00001ae8       OPIF_COMPAREFATTIME        0000000180002ae8     flags.obj
 0001:00001af0       OPIF_EXTERNALGET           0000000180002af0     flags.obj
 0001:00001af8       OPIF_EXTERNALPUT           0000000180002af8     flags.obj
 0001:00001b00       OPIF_EXTERNALDELETE        0000000180002b00     flags.obj
 0001:00001b08       OPIF_EXTERNALMKDIR         0000000180002b08     flags.obj
 0001:00001b10       OPIF_USEATTRHIGHLIGHTING   0000000180002b10     flags.obj
 0001:00001b18       OPIF_USECRC32              0000000180002b18     flags.obj
 0001:00001b20       OPIF_USEFREESIZE           0000000180002b20     flags.obj
 0001:00001b28       OPIF_SHORTCUT              0000000180002b28     flags.obj
 0001:00001b30       OPIF_NONE                  0000000180002b30     flags.obj
 0001:00001b38       OPM_SILENT                 0000000180002b38     flags.obj
 0001:00001b40       OPM_FIND                   0000000180002b40     flags.obj
 0001:00001b48       OPM_VIEW                   0000000180002b48     flags.obj
 0001:00001b50       OPM_EDIT                   0000000180002b50     flags.obj
 0001:00001b58       OPM_TOPLEVEL               0000000180002b58     flags.obj
 0001:00001b60       OPM_DESCR                  0000000180002b60     flags.obj
 0001:00001b68       OPM_QUICKVIEW              0000000180002b68     flags.obj
 0001:00001b70       OPM_PGDN                   0000000180002b70     flags.obj
 0001:00001b78       OPM_COMMANDS               0000000180002b78     flags.obj
 0001:00001b80       OPM_NONE                   0000000180002b80     flags.obj
 0001:00001b88       FOSF_ACTIVE                0000000180002b88     flags.obj
 0001:00001b90       FOSF_NONE                  0000000180002b90     flags.obj
 0001:00001b98       PCIF_NONE                  0000000180002b98     flags.obj
 0001:00001ba0       FarGuid                    0000000180002ba0     flags.obj
 0001:00006790       colors                     0000000180007790     keysandcolors.obj
 0001:000076f0       guids                      00000001800086f0     keysandcolors.obj
 0001:00008b20       FCF_FG_4BIT                0000000180009b20     lflua.obj
 0001:00008b28       FCF_BG_4BIT                0000000180009b28     lflua.obj
 0001:00008b30       FCF_4BITMASK               0000000180009b30     lflua.obj
 0001:00008b38       FCF_RAWATTR_MASK           0000000180009b38     lflua.obj
 0001:00008b40       FCF_EXTENDEDFLAGS          0000000180009b40     lflua.obj
 0001:00008b48       FCF_FG_BOLD                0000000180009b48     lflua.obj
 0001:00008b50       FCF_FG_ITALIC              0000000180009b50     lflua.obj
 0001:00008b58       FCF_FG_UNDERLINE           0000000180009b58     lflua.obj
 0001:00008b60       FCF_STYLEMASK              0000000180009b60     lflua.obj
 0001:00008b68       FCF_NONE                   0000000180009b68     lflua.obj
 0001:00008b70       CDF_NONE                   0000000180009b70     lflua.obj
 0001:00008b78       FMSG_WARNING               0000000180009b78     lflua.obj
 0001:00008b80       FMSG_ERRORTYPE             0000000180009b80     lflua.obj
 0001:00008b88       FMSG_KEEPBACKGROUND        0000000180009b88     lflua.obj
 0001:00008b90       FMSG_LEFTALIGN             0000000180009b90     lflua.obj
 0001:00008b98       FMSG_ALLINONE              0000000180009b98     lflua.obj
 0001:00008ba0       FMSG_MB_OK                 0000000180009ba0     lflua.obj
 0001:00008ba8       FMSG_MB_OKCANCEL           0000000180009ba8     lflua.obj
 0001:00008bb0       FMSG_MB_ABORTRETRYIGNORE   0000000180009bb0     lflua.obj
 0001:00008bb8       FMSG_MB_YESNO              0000000180009bb8     lflua.obj
 0001:00008bc0       FMSG_MB_YESNOCANCEL        0000000180009bc0     lflua.obj
 0001:00008bc8       FMSG_MB_RETRYCANCEL        0000000180009bc8     lflua.obj
 0001:00008bd0       FMSG_NONE                  0000000180009bd0     lflua.obj
 0001:00008bd8       DIF_BOXCOLOR               0000000180009bd8     lflua.obj
 0001:00008be0       DIF_GROUP                  0000000180009be0     lflua.obj
 0001:00008be8       DIF_LEFTTEXT               0000000180009be8     lflua.obj
 0001:00008bf0       DIF_MOVESELECT             0000000180009bf0     lflua.obj
 0001:00008bf8       DIF_SHOWAMPERSAND          0000000180009bf8     lflua.obj
 0001:00008c00       DIF_CENTERGROUP            0000000180009c00     lflua.obj
 0001:00008c08       DIF_NOBRACKETS             0000000180009c08     lflua.obj
 0001:00008c10       DIF_MANUALADDHISTORY       0000000180009c10     lflua.obj
 0001:00008c18       DIF_SEPARATOR              0000000180009c18     lflua.obj
 0001:00008c20       DIF_SEPARATOR2             0000000180009c20     lflua.obj
 0001:00008c28       DIF_EDITOR                 0000000180009c28     lflua.obj
 0001:00008c30       DIF_LISTNOAMPERSAND        0000000180009c30     lflua.obj
 0001:00008c38       DIF_LISTNOBOX              0000000180009c38     lflua.obj
 0001:00008c40       DIF_HISTORY                0000000180009c40     lflua.obj
 0001:00008c48       DIF_BTNNOCLOSE             0000000180009c48     lflua.obj
 0001:00008c50       DIF_CENTERTEXT             0000000180009c50     lflua.obj
 0001:00008c58       DIF_SEPARATORUSER          0000000180009c58     lflua.obj
 0001:00008c60       DIF_SETSHIELD              0000000180009c60     lflua.obj
 0001:00008c68       DIF_EDITEXPAND             0000000180009c68     lflua.obj
 0001:00008c70       DIF_DROPDOWNLIST           0000000180009c70     lflua.obj
 0001:00008c78       DIF_USELASTHISTORY         0000000180009c78     lflua.obj
 0001:00008c80       DIF_MASKEDIT               0000000180009c80     lflua.obj
 0001:00008c88       DIF_LISTTRACKMOUSE         0000000180009c88     lflua.obj
 0001:00008c90       DIF_LISTTRACKMOUSEINFOCUS  0000000180009c90     lflua.obj
 0001:00008c98       DIF_SELECTONENTRY          0000000180009c98     lflua.obj
 0001:00008ca0       DIF_3STATE                 0000000180009ca0     lflua.obj
 0001:00008ca8       DIF_EDITPATH               0000000180009ca8     lflua.obj
 0001:00008cb0       DIF_LISTWRAPMODE           0000000180009cb0     lflua.obj
 0001:00008cb8       DIF_NOAUTOCOMPLETE         0000000180009cb8     lflua.obj
 0001:00008cc0       DIF_LISTAUTOHIGHLIGHT      0000000180009cc0     lflua.obj
 0001:00008cc8       DIF_LISTNOCLOSE            0000000180009cc8     lflua.obj
 0001:00008cd0       DIF_EDITPATHEXEC           0000000180009cd0     lflua.obj
 0001:00008cd8       DIF_HIDDEN                 0000000180009cd8     lflua.obj
 0001:00008ce0       DIF_READONLY               0000000180009ce0     lflua.obj
 0001:00008ce8       DIF_NOFOCUS                0000000180009ce8     lflua.obj
 0001:00008cf0       DIF_DISABLE                0000000180009cf0     lflua.obj
 0001:00008cf8       DIF_DEFAULTBUTTON          0000000180009cf8     lflua.obj
 0001:00008d00       DIF_FOCUS                  0000000180009d00     lflua.obj
 0001:00008d08       DIF_RIGHTTEXT              0000000180009d08     lflua.obj
 0001:00008d10       DIF_WORDWRAP               0000000180009d10     lflua.obj
 0001:00008d18       DIF_NONE                   0000000180009d18     lflua.obj
 0001:00008d20       LIF_SELECTED               0000000180009d20     lflua.obj
 0001:00008d28       LIF_CHECKED                0000000180009d28     lflua.obj
 0001:00008d30       LIF_SEPARATOR              0000000180009d30     lflua.obj
 0001:00008d38       LIF_DISABLE                0000000180009d38     lflua.obj
 0001:00008d40       LIF_GRAYED                 0000000180009d40     lflua.obj
 0001:00008d48       LIF_HIDDEN                 0000000180009d48     lflua.obj
 0001:00008d50       LIF_DELETEUSERDATA         0000000180009d50     lflua.obj
 0001:00008d58       LIF_NONE                   0000000180009d58     lflua.obj
 0001:00008d60       LIFIND_EXACTMATCH          0000000180009d60     lflua.obj
 0001:00008d68       LIFIND_NONE                0000000180009d68     lflua.obj
 0001:00008d70       LINFO_SHOWNOBOX            0000000180009d70     lflua.obj
 0001:00008d78       LINFO_AUTOHIGHLIGHT        0000000180009d78     lflua.obj
 0001:00008d80       LINFO_REVERSEHIGHLIGHT     0000000180009d80     lflua.obj
 0001:00008d88       LINFO_WRAPMODE             0000000180009d88     lflua.obj
 0001:00008d90       LINFO_SHOWAMPERSAND        0000000180009d90     lflua.obj
 0001:00008d98       LINFO_NONE                 0000000180009d98     lflua.obj
 0001:00008da0       FDLG_WARNING               0000000180009da0     lflua.obj
 0001:00008da8       FDLG_SMALLDIALOG           0000000180009da8     lflua.obj
 0001:00008db0       FDLG_NODRAWSHADOW          0000000180009db0     lflua.obj
 0001:00008db8       FDLG_NODRAWPANEL           0000000180009db8     lflua.obj
 0001:00008dc0       FDLG_KEEPCONSOLETITLE      0000000180009dc0     lflua.obj
 0001:00008dc8       FDLG_NONMODAL              0000000180009dc8     lflua.obj
 0001:00008dd0       FDLG_NONE                  0000000180009dd0     lflua.obj
 0001:00008dd8       MIF_SELECTED               0000000180009dd8     lflua.obj
 0001:00008de0       MIF_CHECKED                0000000180009de0     lflua.obj
 0001:00008de8       MIF_SEPARATOR              0000000180009de8     lflua.obj
 0001:00008df0       MIF_DISABLE                0000000180009df0     lflua.obj
 0001:00008df8       MIF_GRAYED                 0000000180009df8     lflua.obj
 0001:00008e00       MIF_HIDDEN                 0000000180009e00     lflua.obj
 0001:00008e08       MIF_NONE                   0000000180009e08     lflua.obj
 0001:00008e10       FMENU_SHOWAMPERSAND        0000000180009e10     lflua.obj
 0001:00008e18       FMENU_WRAPMODE             0000000180009e18     lflua.obj
 0001:00008e20       FMENU_AUTOHIGHLIGHT        0000000180009e20     lflua.obj
 0001:00008e28       FMENU_REVERSEAUTOHIGHLIGHT 0000000180009e28     lflua.obj
 0001:00008e30       FMENU_CHANGECONSOLETITLE   0000000180009e30     lflua.obj
 0001:00008e38       FMENU_SHOWNOBOX            0000000180009e38     lflua.obj
 0001:00008e40       FMENU_SHOWSHORTBOX         0000000180009e40     lflua.obj
 0001:00008e48       FMENU_SHOWSINGLEBOX        0000000180009e48     lflua.obj
 0001:00008e50       FMENU_NODRAWSHADOW         0000000180009e50     lflua.obj
 0001:00008e58       FMENU_NONE                 0000000180009e58     lflua.obj
 0001:00008e60       PPIF_SELECTED              0000000180009e60     lflua.obj
 0001:00008e68       PPIF_PROCESSDESCR          0000000180009e68     lflua.obj
 0001:00008e70       PPIF_NONE                  0000000180009e70     lflua.obj
 0001:00008e78       PFLAGS_SHOWHIDDEN          0000000180009e78     lflua.obj
 0001:00008e80       PFLAGS_HIGHLIGHT           0000000180009e80     lflua.obj
 0001:00008e88       PFLAGS_REVERSESORTORDER    0000000180009e88     lflua.obj
 0001:00008e90       PFLAGS_USESORTGROUPS       0000000180009e90     lflua.obj
 0001:00008e98       PFLAGS_SELECTEDFIRST       0000000180009e98     lflua.obj
 0001:00008ea0       PFLAGS_REALNAMES           0000000180009ea0     lflua.obj
 0001:00008ea8       PFLAGS_PANELLEFT           0000000180009ea8     lflua.obj
 0001:00008eb0       PFLAGS_DIRECTORIESFIRST    0000000180009eb0     lflua.obj
 0001:00008eb8       PFLAGS_USECRC32            0000000180009eb8     lflua.obj
 0001:00008ec0       PFLAGS_PLUGIN              0000000180009ec0     lflua.obj
 0001:00008ec8       PFLAGS_VISIBLE             0000000180009ec8     lflua.obj
 0001:00008ed0       PFLAGS_FOCUS               0000000180009ed0     lflua.obj
 0001:00008ed8       PFLAGS_ALTERNATIVENAMES    0000000180009ed8     lflua.obj
 0001:00008ee0       PFLAGS_SHORTCUT            0000000180009ee0     lflua.obj
 0001:00008ee8       PFLAGS_NONE                0000000180009ee8     lflua.obj
 0001:00008ef0       VF_NONMODAL                0000000180009ef0     lflua.obj
 0001:00008ef8       VF_DELETEONCLOSE           0000000180009ef8     lflua.obj
 0001:00008f00       VF_ENABLE_F6               0000000180009f00     lflua.obj
 0001:00008f08       VF_DISABLEHISTORY          0000000180009f08     lflua.obj
 0001:00008f10       VF_IMMEDIATERETURN         0000000180009f10     lflua.obj
 0001:00008f18       VF_DELETEONLYFILEONCLOSE   0000000180009f18     lflua.obj
 0001:00008f20       VF_NONE                    0000000180009f20     lflua.obj
 0001:00008f28       EF_NONMODAL                0000000180009f28     lflua.obj
 0001:00008f30       EF_CREATENEW               0000000180009f30     lflua.obj
 0001:00008f38       EF_ENABLE_F6               0000000180009f38     lflua.obj
 0001:00008f40       EF_DISABLEHISTORY          0000000180009f40     lflua.obj
 0001:00008f48       EF_DELETEONCLOSE           0000000180009f48     lflua.obj
 0001:00008f50       EF_IMMEDIATERETURN         0000000180009f50     lflua.obj
 0001:00008f58       EF_DELETEONLYFILEONCLOSE   0000000180009f58     lflua.obj
 0001:00008f60       EF_LOCKED                  0000000180009f60     lflua.obj
 0001:00008f68       EF_DISABLESAVEPOS          0000000180009f68     lflua.obj
 0001:00008f70       EF_OPENMODE_MASK           0000000180009f70     lflua.obj
 0001:00008f78       EF_OPENMODE_QUERY          0000000180009f78     lflua.obj
 0001:00008f80       EF_OPENMODE_NEWIFOPEN      0000000180009f80     lflua.obj
 0001:00008f88       EF_OPENMODE_USEEXISTING    0000000180009f88     lflua.obj
 0001:00008f90       EF_OPENMODE_BREAKIFOPEN    0000000180009f90     lflua.obj
 0001:00008f98       EF_OPENMODE_RELOADIFOPEN   0000000180009f98     lflua.obj
 0001:00008fa0       EN_NONE                    0000000180009fa0     lflua.obj
 0001:00008fa8       FHELP_NOSHOWERROR          0000000180009fa8     lflua.obj
 0001:00008fb0       FHELP_SELFHELP             0000000180009fb0     lflua.obj
 0001:00008fb8       FHELP_FARHELP              0000000180009fb8     lflua.obj
 0001:00008fc0       FHELP_CUSTOMFILE           0000000180009fc0     lflua.obj
 0001:00008fc8       FHELP_CUSTOMPATH           0000000180009fc8     lflua.obj
 0001:00008fd0       FHELP_GUID                 0000000180009fd0     lflua.obj
 0001:00008fd8       FHELP_USECONTENTS          0000000180009fd8     lflua.obj
 0001:00008fe0       FHELP_NONE                 0000000180009fe0     lflua.obj
 0001:00008fe8       KMFLAGS_SILENTCHECK        0000000180009fe8     lflua.obj
 0001:00008ff0       KMFLAGS_NOSENDKEYSTOPLUGINS 0000000180009ff0     lflua.obj
 0001:00008ff8       KMFLAGS_ENABLEOUTPUT       0000000180009ff8     lflua.obj
 0001:00009000       KMFLAGS_LANGMASK           000000018000a000     lflua.obj
 0001:00009008       KMFLAGS_LUA                000000018000a008     lflua.obj
 0001:00009010       KMFLAGS_MOONSCRIPT         000000018000a010     lflua.obj
 0001:00009018       KMFLAGS_NONE               000000018000a018     lflua.obj
 0001:00009020       AKMFLAGS_NONE              000000018000a020     lflua.obj
 0001:00009028       FSETCLR_REDRAW             000000018000a028     lflua.obj
 0001:00009030       FSETCLR_NONE               000000018000a030     lflua.obj
 0001:00009038       WIF_MODIFIED               000000018000a038     lflua.obj
 0001:00009040       WIF_CURRENT                000000018000a040     lflua.obj
 0001:00009048       WIF_MODAL                  000000018000a048     lflua.obj
 0001:00009050       WIF_NONE                   000000018000a050     lflua.obj
 0001:00009058       VOPT_SAVEFILEPOSITION      000000018000a058     lflua.obj
 0001:00009060       VOPT_AUTODETECTCODEPAGE    000000018000a060     lflua.obj
 0001:00009068       VOPT_SHOWTITLEBAR          000000018000a068     lflua.obj
 0001:00009070       VOPT_SHOWKEYBAR            000000018000a070     lflua.obj
 0001:00009078       VOPT_SHOWSCROLLBAR         000000018000a078     lflua.obj
 0001:00009080       VOPT_QUICKVIEW             000000018000a080     lflua.obj
 0001:00009088       VOPT_NONE                  000000018000a088     lflua.obj
 0001:00009090       VSMFL_REDRAW               000000018000a090     lflua.obj
 0001:00009098       VSMFL_NONE                 000000018000a098     lflua.obj
 0001:000090a0       VSP_NOREDRAW               000000018000a0a0     lflua.obj
 0001:000090a8       VSP_PERCENT                000000018000a0a8     lflua.obj
 0001:000090b0       VSP_RELATIVE               000000018000a0b0     lflua.obj
 0001:000090b8       VSP_NORETNEWPOS            000000018000a0b8     lflua.obj
 0001:000090c0       VSP_NONE                   000000018000a0c0     lflua.obj
 0001:000090c8       VMF_WRAP                   000000018000a0c8     lflua.obj
 0001:000090d0       VMF_WORDWRAP               000000018000a0d0     lflua.obj
 0001:000090d8       VMF_NONE                   000000018000a0d8     lflua.obj
 0001:000090e0       ECF_TABMARKFIRST           000000018000a0e0     lflua.obj
 0001:000090e8       ECF_TABMARKCURRENT         000000018000a0e8     lflua.obj
 0001:000090f0       ECF_AUTODELETE             000000018000a0f0     lflua.obj
 0001:000090f8       ECF_NONE                   000000018000a0f8     lflua.obj
 0001:00009100       FIB_ENABLEEMPTY            000000018000a100     lflua.obj
 0001:00009108       FIB_PASSWORD               000000018000a108     lflua.obj
 0001:00009110       FIB_EXPANDENV              000000018000a110     lflua.obj
 0001:00009118       FIB_NOUSELASTHISTORY       000000018000a118     lflua.obj
 0001:00009120       FIB_BUTTONS                000000018000a120     lflua.obj
 0001:00009128       FIB_NOAMPERSAND            000000018000a128     lflua.obj
 0001:00009130       FIB_EDITPATH               000000018000a130     lflua.obj
 0001:00009138       FIB_EDITPATHEXEC           000000018000a138     lflua.obj
 0001:00009140       FIB_NONE                   000000018000a140     lflua.obj
 0001:00009148       FPF_LOADED                 000000018000a148     lflua.obj
 0001:00009150       FPF_ANSI                   000000018000a150     lflua.obj
 0001:00009158       FPF_NONE                   000000018000a158     lflua.obj
 0001:00009160       PN_CMPNAME                 000000018000a160     lflua.obj
 0001:00009168       PN_CMPNAMELIST             000000018000a168     lflua.obj
 0001:00009170       PN_GENERATENAME            000000018000a170     lflua.obj
 0001:00009178       PN_CHECKMASK               000000018000a178     lflua.obj
 0001:00009180       PN_SKIPPATH                000000018000a180     lflua.obj
 0001:00009188       PN_SHOWERRORMESSAGE        000000018000a188     lflua.obj
 0001:00009190       PN_NONE                    000000018000a190     lflua.obj
 0001:00009198       XLAT_SWITCHKEYBLAYOUT      000000018000a198     lflua.obj
 0001:000091a0       XLAT_SWITCHKEYBBEEP        000000018000a1a0     lflua.obj
 0001:000091a8       XLAT_USEKEYBLAYOUTNAME     000000018000a1a8     lflua.obj
 0001:000091b0       XLAT_CONVERTALLCMDLINE     000000018000a1b0     lflua.obj
 0001:000091b8       XLAT_NONE                  000000018000a1b8     lflua.obj
 0001:000091c0       FRS_RETUPDIR               000000018000a1c0     lflua.obj
 0001:000091c8       FRS_RECUR                  000000018000a1c8     lflua.obj
 0001:000091d0       FRS_SCANSYMLINK            000000018000a1d0     lflua.obj
 0001:000091d8       FRS_NONE                   000000018000a1d8     lflua.obj
 0001:000091e0       MLF_SHOWERRMSG             000000018000a1e0     lflua.obj
 0001:000091e8       MLF_DONOTUPDATEPANEL       000000018000a1e8     lflua.obj
 0001:000091f0       MLF_HOLDTARGET             000000018000a1f0     lflua.obj
 0001:000091f8       MLF_NONE                   000000018000a1f8     lflua.obj
 0001:00009200       FFFS_COMMAS                000000018000a200     lflua.obj
 0001:00009208       FFFS_FLOATSIZE             000000018000a208     lflua.obj
 0001:00009210       FFFS_SHOWBYTESINDEX        000000018000a210     lflua.obj
 0001:00009218       FFFS_ECONOMIC              000000018000a218     lflua.obj
 0001:00009220       FFFS_THOUSAND              000000018000a220     lflua.obj
 0001:00009228       FFFS_MINSIZEINDEX          000000018000a228     lflua.obj
 0001:00009230       FFFS_MINSIZEINDEX_MASK     000000018000a230     lflua.obj
 0001:00009238       FFFS_NONE                  000000018000a238     lflua.obj
 0001:00009240       PF_PRELOAD                 000000018000a240     lflua.obj
 0001:00009248       PF_DISABLEPANELS           000000018000a248     lflua.obj
 0001:00009250       PF_EDITOR                  000000018000a250     lflua.obj
 0001:00009258       PF_VIEWER                  000000018000a258     lflua.obj
 0001:00009260       PF_FULLCMDLINE             000000018000a260     lflua.obj
 0001:00009268       PF_DIALOG                  000000018000a268     lflua.obj
 0001:00009270       PF_NONE                    000000018000a270     lflua.obj
 0001:00009278       IPLFLAGS_SEPARATOR         000000018000a278     lflua.obj
 0001:00009280       IPLFLAGS_NONE              000000018000a280     lflua.obj
 0001:00009288       PMFLAGS_FULLSCREEN         000000018000a288     lflua.obj
 0001:00009290       PMFLAGS_DETAILEDSTATUS     000000018000a290     lflua.obj
 0001:00009298       PMFLAGS_ALIGNEXTENSIONS    000000018000a298     lflua.obj
 0001:000092a0       PMFLAGS_CASECONVERSION     000000018000a2a0     lflua.obj
 0001:000092a8       PMFLAGS_NONE               000000018000a2a8     lflua.obj
 0001:000092b0       OPIF_DISABLEFILTER         000000018000a2b0     lflua.obj
 0001:000092b8       OPIF_DISABLESORTGROUPS     000000018000a2b8     lflua.obj
 0001:000092c0       OPIF_DISABLEHIGHLIGHTING   000000018000a2c0     lflua.obj
 0001:000092c8       OPIF_ADDDOTS               000000018000a2c8     lflua.obj
 0001:000092d0       OPIF_RAWSELECTION          000000018000a2d0     lflua.obj
 0001:000092d8       OPIF_REALNAMES             000000018000a2d8     lflua.obj
 0001:000092e0       OPIF_SHOWNAMESONLY         000000018000a2e0     lflua.obj
 0001:000092e8       OPIF_SHOWRIGHTALIGNNAMES   000000018000a2e8     lflua.obj
 0001:000092f0       OPIF_SHOWPRESERVECASE      000000018000a2f0     lflua.obj
 0001:000092f8       OPIF_COMPAREFATTIME        000000018000a2f8     lflua.obj
 0001:00009300       OPIF_EXTERNALGET           000000018000a300     lflua.obj
 0001:00009308       OPIF_EXTERNALPUT           000000018000a308     lflua.obj
 0001:00009310       OPIF_EXTERNALDELETE        000000018000a310     lflua.obj
 0001:00009318       OPIF_EXTERNALMKDIR         000000018000a318     lflua.obj
 0001:00009320       OPIF_USEATTRHIGHLIGHTING   000000018000a320     lflua.obj
 0001:00009328       OPIF_USECRC32              000000018000a328     lflua.obj
 0001:00009330       OPIF_USEFREESIZE           000000018000a330     lflua.obj
 0001:00009338       OPIF_SHORTCUT              000000018000a338     lflua.obj
 0001:00009340       OPIF_NONE                  000000018000a340     lflua.obj
 0001:00009348       OPM_SILENT                 000000018000a348     lflua.obj
 0001:00009350       OPM_FIND                   000000018000a350     lflua.obj
 0001:00009358       OPM_VIEW                   000000018000a358     lflua.obj
 0001:00009360       OPM_EDIT                   000000018000a360     lflua.obj
 0001:00009368       OPM_TOPLEVEL               000000018000a368     lflua.obj
 0001:00009370       OPM_DESCR                  000000018000a370     lflua.obj
 0001:00009378       OPM_QUICKVIEW              000000018000a378     lflua.obj
 0001:00009380       OPM_PGDN                   000000018000a380     lflua.obj
 0001:00009388       OPM_COMMANDS               000000018000a388     lflua.obj
 0001:00009390       OPM_NONE                   000000018000a390     lflua.obj
 0001:00009398       FOSF_ACTIVE                000000018000a398     lflua.obj
 0001:000093a0       FOSF_NONE                  000000018000a3a0     lflua.obj
 0001:000093a8       PCIF_NONE                  000000018000a3a8     lflua.obj
 0001:000093b0       FarGuid                    000000018000a3b0     lflua.obj
 0001:000093c0       PDF_DIALOGEVENTDRAWENABLE  000000018000a3c0     lflua.obj
 0001:000093c8       PDF_PROCESSINGERROR        000000018000a3c8     lflua.obj
 0001:000093d0       PDF_FULL_TIME_RESOLUTION   000000018000a3d0     lflua.obj
 0001:000095b0       FCF_FG_4BIT                000000018000a5b0     lregex.obj
 0001:000095b8       FCF_BG_4BIT                000000018000a5b8     lregex.obj
 0001:000095c0       FCF_4BITMASK               000000018000a5c0     lregex.obj
 0001:000095c8       FCF_RAWATTR_MASK           000000018000a5c8     lregex.obj
 0001:000095d0       FCF_EXTENDEDFLAGS          000000018000a5d0     lregex.obj
 0001:000095d8       FCF_FG_BOLD                000000018000a5d8     lregex.obj
 0001:000095e0       FCF_FG_ITALIC              000000018000a5e0     lregex.obj
 0001:000095e8       FCF_FG_UNDERLINE           000000018000a5e8     lregex.obj
 0001:000095f0       FCF_STYLEMASK              000000018000a5f0     lregex.obj
 0001:000095f8       FCF_NONE                   000000018000a5f8     lregex.obj
 0001:00009600       CDF_NONE                   000000018000a600     lregex.obj
 0001:00009608       FMSG_WARNING               000000018000a608     lregex.obj
 0001:00009610       FMSG_ERRORTYPE             000000018000a610     lregex.obj
 0001:00009618       FMSG_KEEPBACKGROUND        000000018000a618     lregex.obj
 0001:00009620       FMSG_LEFTALIGN             000000018000a620     lregex.obj
 0001:00009628       FMSG_ALLINONE              000000018000a628     lregex.obj
 0001:00009630       FMSG_MB_OK                 000000018000a630     lregex.obj
 0001:00009638       FMSG_MB_OKCANCEL           000000018000a638     lregex.obj
 0001:00009640       FMSG_MB_ABORTRETRYIGNORE   000000018000a640     lregex.obj
 0001:00009648       FMSG_MB_YESNO              000000018000a648     lregex.obj
 0001:00009650       FMSG_MB_YESNOCANCEL        000000018000a650     lregex.obj
 0001:00009658       FMSG_MB_RETRYCANCEL        000000018000a658     lregex.obj
 0001:00009660       FMSG_NONE                  000000018000a660     lregex.obj
 0001:00009668       DIF_BOXCOLOR               000000018000a668     lregex.obj
 0001:00009670       DIF_GROUP                  000000018000a670     lregex.obj
 0001:00009678       DIF_LEFTTEXT               000000018000a678     lregex.obj
 0001:00009680       DIF_MOVESELECT             000000018000a680     lregex.obj
 0001:00009688       DIF_SHOWAMPERSAND          000000018000a688     lregex.obj
 0001:00009690       DIF_CENTERGROUP            000000018000a690     lregex.obj
 0001:00009698       DIF_NOBRACKETS             000000018000a698     lregex.obj
 0001:000096a0       DIF_MANUALADDHISTORY       000000018000a6a0     lregex.obj
 0001:000096a8       DIF_SEPARATOR              000000018000a6a8     lregex.obj
 0001:000096b0       DIF_SEPARATOR2             000000018000a6b0     lregex.obj
 0001:000096b8       DIF_EDITOR                 000000018000a6b8     lregex.obj
 0001:000096c0       DIF_LISTNOAMPERSAND        000000018000a6c0     lregex.obj
 0001:000096c8       DIF_LISTNOBOX              000000018000a6c8     lregex.obj
 0001:000096d0       DIF_HISTORY                000000018000a6d0     lregex.obj
 0001:000096d8       DIF_BTNNOCLOSE             000000018000a6d8     lregex.obj
 0001:000096e0       DIF_CENTERTEXT             000000018000a6e0     lregex.obj
 0001:000096e8       DIF_SEPARATORUSER          000000018000a6e8     lregex.obj
 0001:000096f0       DIF_SETSHIELD              000000018000a6f0     lregex.obj
 0001:000096f8       DIF_EDITEXPAND             000000018000a6f8     lregex.obj
 0001:00009700       DIF_DROPDOWNLIST           000000018000a700     lregex.obj
 0001:00009708       DIF_USELASTHISTORY         000000018000a708     lregex.obj
 0001:00009710       DIF_MASKEDIT               000000018000a710     lregex.obj
 0001:00009718       DIF_LISTTRACKMOUSE         000000018000a718     lregex.obj
 0001:00009720       DIF_LISTTRACKMOUSEINFOCUS  000000018000a720     lregex.obj
 0001:00009728       DIF_SELECTONENTRY          000000018000a728     lregex.obj
 0001:00009730       DIF_3STATE                 000000018000a730     lregex.obj
 0001:00009738       DIF_EDITPATH               000000018000a738     lregex.obj
 0001:00009740       DIF_LISTWRAPMODE           000000018000a740     lregex.obj
 0001:00009748       DIF_NOAUTOCOMPLETE         000000018000a748     lregex.obj
 0001:00009750       DIF_LISTAUTOHIGHLIGHT      000000018000a750     lregex.obj
 0001:00009758       DIF_LISTNOCLOSE            000000018000a758     lregex.obj
 0001:00009760       DIF_EDITPATHEXEC           000000018000a760     lregex.obj
 0001:00009768       DIF_HIDDEN                 000000018000a768     lregex.obj
 0001:00009770       DIF_READONLY               000000018000a770     lregex.obj
 0001:00009778       DIF_NOFOCUS                000000018000a778     lregex.obj
 0001:00009780       DIF_DISABLE                000000018000a780     lregex.obj
 0001:00009788       DIF_DEFAULTBUTTON          000000018000a788     lregex.obj
 0001:00009790       DIF_FOCUS                  000000018000a790     lregex.obj
 0001:00009798       DIF_RIGHTTEXT              000000018000a798     lregex.obj
 0001:000097a0       DIF_WORDWRAP               000000018000a7a0     lregex.obj
 0001:000097a8       DIF_NONE                   000000018000a7a8     lregex.obj
 0001:000097b0       LIF_SELECTED               000000018000a7b0     lregex.obj
 0001:000097b8       LIF_CHECKED                000000018000a7b8     lregex.obj
 0001:000097c0       LIF_SEPARATOR              000000018000a7c0     lregex.obj
 0001:000097c8       LIF_DISABLE                000000018000a7c8     lregex.obj
 0001:000097d0       LIF_GRAYED                 000000018000a7d0     lregex.obj
 0001:000097d8       LIF_HIDDEN                 000000018000a7d8     lregex.obj
 0001:000097e0       LIF_DELETEUSERDATA         000000018000a7e0     lregex.obj
 0001:000097e8       LIF_NONE                   000000018000a7e8     lregex.obj
 0001:000097f0       LIFIND_EXACTMATCH          000000018000a7f0     lregex.obj
 0001:000097f8       LIFIND_NONE                000000018000a7f8     lregex.obj
 0001:00009800       LINFO_SHOWNOBOX            000000018000a800     lregex.obj
 0001:00009808       LINFO_AUTOHIGHLIGHT        000000018000a808     lregex.obj
 0001:00009810       LINFO_REVERSEHIGHLIGHT     000000018000a810     lregex.obj
 0001:00009818       LINFO_WRAPMODE             000000018000a818     lregex.obj
 0001:00009820       LINFO_SHOWAMPERSAND        000000018000a820     lregex.obj
 0001:00009828       LINFO_NONE                 000000018000a828     lregex.obj
 0001:00009830       FDLG_WARNING               000000018000a830     lregex.obj
 0001:00009838       FDLG_SMALLDIALOG           000000018000a838     lregex.obj
 0001:00009840       FDLG_NODRAWSHADOW          000000018000a840     lregex.obj
 0001:00009848       FDLG_NODRAWPANEL           000000018000a848     lregex.obj
 0001:00009850       FDLG_KEEPCONSOLETITLE      000000018000a850     lregex.obj
 0001:00009858       FDLG_NONMODAL              000000018000a858     lregex.obj
 0001:00009860       FDLG_NONE                  000000018000a860     lregex.obj
 0001:00009868       MIF_SELECTED               000000018000a868     lregex.obj
 0001:00009870       MIF_CHECKED                000000018000a870     lregex.obj
 0001:00009878       MIF_SEPARATOR              000000018000a878     lregex.obj
 0001:00009880       MIF_DISABLE                000000018000a880     lregex.obj
 0001:00009888       MIF_GRAYED                 000000018000a888     lregex.obj
 0001:00009890       MIF_HIDDEN                 000000018000a890     lregex.obj
 0001:00009898       MIF_NONE                   000000018000a898     lregex.obj
 0001:000098a0       FMENU_SHOWAMPERSAND        000000018000a8a0     lregex.obj
 0001:000098a8       FMENU_WRAPMODE             000000018000a8a8     lregex.obj
 0001:000098b0       FMENU_AUTOHIGHLIGHT        000000018000a8b0     lregex.obj
 0001:000098b8       FMENU_REVERSEAUTOHIGHLIGHT 000000018000a8b8     lregex.obj
 0001:000098c0       FMENU_CHANGECONSOLETITLE   000000018000a8c0     lregex.obj
 0001:000098c8       FMENU_SHOWNOBOX            000000018000a8c8     lregex.obj
 0001:000098d0       FMENU_SHOWSHORTBOX         000000018000a8d0     lregex.obj
 0001:000098d8       FMENU_SHOWSINGLEBOX        000000018000a8d8     lregex.obj
 0001:000098e0       FMENU_NODRAWSHADOW         000000018000a8e0     lregex.obj
 0001:000098e8       FMENU_NONE                 000000018000a8e8     lregex.obj
 0001:000098f0       PPIF_SELECTED              000000018000a8f0     lregex.obj
 0001:000098f8       PPIF_PROCESSDESCR          000000018000a8f8     lregex.obj
 0001:00009900       PPIF_NONE                  000000018000a900     lregex.obj
 0001:00009908       PFLAGS_SHOWHIDDEN          000000018000a908     lregex.obj
 0001:00009910       PFLAGS_HIGHLIGHT           000000018000a910     lregex.obj
 0001:00009918       PFLAGS_REVERSESORTORDER    000000018000a918     lregex.obj
 0001:00009920       PFLAGS_USESORTGROUPS       000000018000a920     lregex.obj
 0001:00009928       PFLAGS_SELECTEDFIRST       000000018000a928     lregex.obj
 0001:00009930       PFLAGS_REALNAMES           000000018000a930     lregex.obj
 0001:00009938       PFLAGS_PANELLEFT           000000018000a938     lregex.obj
 0001:00009940       PFLAGS_DIRECTORIESFIRST    000000018000a940     lregex.obj
 0001:00009948       PFLAGS_USECRC32            000000018000a948     lregex.obj
 0001:00009950       PFLAGS_PLUGIN              000000018000a950     lregex.obj
 0001:00009958       PFLAGS_VISIBLE             000000018000a958     lregex.obj
 0001:00009960       PFLAGS_FOCUS               000000018000a960     lregex.obj
 0001:00009968       PFLAGS_ALTERNATIVENAMES    000000018000a968     lregex.obj
 0001:00009970       PFLAGS_SHORTCUT            000000018000a970     lregex.obj
 0001:00009978       PFLAGS_NONE                000000018000a978     lregex.obj
 0001:00009980       VF_NONMODAL                000000018000a980     lregex.obj
 0001:00009988       VF_DELETEONCLOSE           000000018000a988     lregex.obj
 0001:00009990       VF_ENABLE_F6               000000018000a990     lregex.obj
 0001:00009998       VF_DISABLEHISTORY          000000018000a998     lregex.obj
 0001:000099a0       VF_IMMEDIATERETURN         000000018000a9a0     lregex.obj
 0001:000099a8       VF_DELETEONLYFILEONCLOSE   000000018000a9a8     lregex.obj
 0001:000099b0       VF_NONE                    000000018000a9b0     lregex.obj
 0001:000099b8       EF_NONMODAL                000000018000a9b8     lregex.obj
 0001:000099c0       EF_CREATENEW               000000018000a9c0     lregex.obj
 0001:000099c8       EF_ENABLE_F6               000000018000a9c8     lregex.obj
 0001:000099d0       EF_DISABLEHISTORY          000000018000a9d0     lregex.obj
 0001:000099d8       EF_DELETEONCLOSE           000000018000a9d8     lregex.obj
 0001:000099e0       EF_IMMEDIATERETURN         000000018000a9e0     lregex.obj
 0001:000099e8       EF_DELETEONLYFILEONCLOSE   000000018000a9e8     lregex.obj
 0001:000099f0       EF_LOCKED                  000000018000a9f0     lregex.obj
 0001:000099f8       EF_DISABLESAVEPOS          000000018000a9f8     lregex.obj
 0001:00009a00       EF_OPENMODE_MASK           000000018000aa00     lregex.obj
 0001:00009a08       EF_OPENMODE_QUERY          000000018000aa08     lregex.obj
 0001:00009a10       EF_OPENMODE_NEWIFOPEN      000000018000aa10     lregex.obj
 0001:00009a18       EF_OPENMODE_USEEXISTING    000000018000aa18     lregex.obj
 0001:00009a20       EF_OPENMODE_BREAKIFOPEN    000000018000aa20     lregex.obj
 0001:00009a28       EF_OPENMODE_RELOADIFOPEN   000000018000aa28     lregex.obj
 0001:00009a30       EN_NONE                    000000018000aa30     lregex.obj
 0001:00009a38       FHELP_NOSHOWERROR          000000018000aa38     lregex.obj
 0001:00009a40       FHELP_SELFHELP             000000018000aa40     lregex.obj
 0001:00009a48       FHELP_FARHELP              000000018000aa48     lregex.obj
 0001:00009a50       FHELP_CUSTOMFILE           000000018000aa50     lregex.obj
 0001:00009a58       FHELP_CUSTOMPATH           000000018000aa58     lregex.obj
 0001:00009a60       FHELP_GUID                 000000018000aa60     lregex.obj
 0001:00009a68       FHELP_USECONTENTS          000000018000aa68     lregex.obj
 0001:00009a70       FHELP_NONE                 000000018000aa70     lregex.obj
 0001:00009a78       KMFLAGS_SILENTCHECK        000000018000aa78     lregex.obj
 0001:00009a80       KMFLAGS_NOSENDKEYSTOPLUGINS 000000018000aa80     lregex.obj
 0001:00009a88       KMFLAGS_ENABLEOUTPUT       000000018000aa88     lregex.obj
 0001:00009a90       KMFLAGS_LANGMASK           000000018000aa90     lregex.obj
 0001:00009a98       KMFLAGS_LUA                000000018000aa98     lregex.obj
 0001:00009aa0       KMFLAGS_MOONSCRIPT         000000018000aaa0     lregex.obj
 0001:00009aa8       KMFLAGS_NONE               000000018000aaa8     lregex.obj
 0001:00009ab0       AKMFLAGS_NONE              000000018000aab0     lregex.obj
 0001:00009ab8       FSETCLR_REDRAW             000000018000aab8     lregex.obj
 0001:00009ac0       FSETCLR_NONE               000000018000aac0     lregex.obj
 0001:00009ac8       WIF_MODIFIED               000000018000aac8     lregex.obj
 0001:00009ad0       WIF_CURRENT                000000018000aad0     lregex.obj
 0001:00009ad8       WIF_MODAL                  000000018000aad8     lregex.obj
 0001:00009ae0       WIF_NONE                   000000018000aae0     lregex.obj
 0001:00009ae8       VOPT_SAVEFILEPOSITION      000000018000aae8     lregex.obj
 0001:00009af0       VOPT_AUTODETECTCODEPAGE    000000018000aaf0     lregex.obj
 0001:00009af8       VOPT_SHOWTITLEBAR          000000018000aaf8     lregex.obj
 0001:00009b00       VOPT_SHOWKEYBAR            000000018000ab00     lregex.obj
 0001:00009b08       VOPT_SHOWSCROLLBAR         000000018000ab08     lregex.obj
 0001:00009b10       VOPT_QUICKVIEW             000000018000ab10     lregex.obj
 0001:00009b18       VOPT_NONE                  000000018000ab18     lregex.obj
 0001:00009b20       VSMFL_REDRAW               000000018000ab20     lregex.obj
 0001:00009b28       VSMFL_NONE                 000000018000ab28     lregex.obj
 0001:00009b30       VSP_NOREDRAW               000000018000ab30     lregex.obj
 0001:00009b38       VSP_PERCENT                000000018000ab38     lregex.obj
 0001:00009b40       VSP_RELATIVE               000000018000ab40     lregex.obj
 0001:00009b48       VSP_NORETNEWPOS            000000018000ab48     lregex.obj
 0001:00009b50       VSP_NONE                   000000018000ab50     lregex.obj
 0001:00009b58       VMF_WRAP                   000000018000ab58     lregex.obj
 0001:00009b60       VMF_WORDWRAP               000000018000ab60     lregex.obj
 0001:00009b68       VMF_NONE                   000000018000ab68     lregex.obj
 0001:00009b70       ECF_TABMARKFIRST           000000018000ab70     lregex.obj
 0001:00009b78       ECF_TABMARKCURRENT         000000018000ab78     lregex.obj
 0001:00009b80       ECF_AUTODELETE             000000018000ab80     lregex.obj
 0001:00009b88       ECF_NONE                   000000018000ab88     lregex.obj
 0001:00009b90       FIB_ENABLEEMPTY            000000018000ab90     lregex.obj
 0001:00009b98       FIB_PASSWORD               000000018000ab98     lregex.obj
 0001:00009ba0       FIB_EXPANDENV              000000018000aba0     lregex.obj
 0001:00009ba8       FIB_NOUSELASTHISTORY       000000018000aba8     lregex.obj
 0001:00009bb0       FIB_BUTTONS                000000018000abb0     lregex.obj
 0001:00009bb8       FIB_NOAMPERSAND            000000018000abb8     lregex.obj
 0001:00009bc0       FIB_EDITPATH               000000018000abc0     lregex.obj
 0001:00009bc8       FIB_EDITPATHEXEC           000000018000abc8     lregex.obj
 0001:00009bd0       FIB_NONE                   000000018000abd0     lregex.obj
 0001:00009bd8       FPF_LOADED                 000000018000abd8     lregex.obj
 0001:00009be0       FPF_ANSI                   000000018000abe0     lregex.obj
 0001:00009be8       FPF_NONE                   000000018000abe8     lregex.obj
 0001:00009bf0       PN_CMPNAME                 000000018000abf0     lregex.obj
 0001:00009bf8       PN_CMPNAMELIST             000000018000abf8     lregex.obj
 0001:00009c00       PN_GENERATENAME            000000018000ac00     lregex.obj
 0001:00009c08       PN_CHECKMASK               000000018000ac08     lregex.obj
 0001:00009c10       PN_SKIPPATH                000000018000ac10     lregex.obj
 0001:00009c18       PN_SHOWERRORMESSAGE        000000018000ac18     lregex.obj
 0001:00009c20       PN_NONE                    000000018000ac20     lregex.obj
 0001:00009c28       XLAT_SWITCHKEYBLAYOUT      000000018000ac28     lregex.obj
 0001:00009c30       XLAT_SWITCHKEYBBEEP        000000018000ac30     lregex.obj
 0001:00009c38       XLAT_USEKEYBLAYOUTNAME     000000018000ac38     lregex.obj
 0001:00009c40       XLAT_CONVERTALLCMDLINE     000000018000ac40     lregex.obj
 0001:00009c48       XLAT_NONE                  000000018000ac48     lregex.obj
 0001:00009c50       FRS_RETUPDIR               000000018000ac50     lregex.obj
 0001:00009c58       FRS_RECUR                  000000018000ac58     lregex.obj
 0001:00009c60       FRS_SCANSYMLINK            000000018000ac60     lregex.obj
 0001:00009c68       FRS_NONE                   000000018000ac68     lregex.obj
 0001:00009c70       MLF_SHOWERRMSG             000000018000ac70     lregex.obj
 0001:00009c78       MLF_DONOTUPDATEPANEL       000000018000ac78     lregex.obj
 0001:00009c80       MLF_HOLDTARGET             000000018000ac80     lregex.obj
 0001:00009c88       MLF_NONE                   000000018000ac88     lregex.obj
 0001:00009c90       FFFS_COMMAS                000000018000ac90     lregex.obj
 0001:00009c98       FFFS_FLOATSIZE             000000018000ac98     lregex.obj
 0001:00009ca0       FFFS_SHOWBYTESINDEX        000000018000aca0     lregex.obj
 0001:00009ca8       FFFS_ECONOMIC              000000018000aca8     lregex.obj
 0001:00009cb0       FFFS_THOUSAND              000000018000acb0     lregex.obj
 0001:00009cb8       FFFS_MINSIZEINDEX          000000018000acb8     lregex.obj
 0001:00009cc0       FFFS_MINSIZEINDEX_MASK     000000018000acc0     lregex.obj
 0001:00009cc8       FFFS_NONE                  000000018000acc8     lregex.obj
 0001:00009cd0       PF_PRELOAD                 000000018000acd0     lregex.obj
 0001:00009cd8       PF_DISABLEPANELS           000000018000acd8     lregex.obj
 0001:00009ce0       PF_EDITOR                  000000018000ace0     lregex.obj
 0001:00009ce8       PF_VIEWER                  000000018000ace8     lregex.obj
 0001:00009cf0       PF_FULLCMDLINE             000000018000acf0     lregex.obj
 0001:00009cf8       PF_DIALOG                  000000018000acf8     lregex.obj
 0001:00009d00       PF_NONE                    000000018000ad00     lregex.obj
 0001:00009d08       IPLFLAGS_SEPARATOR         000000018000ad08     lregex.obj
 0001:00009d10       IPLFLAGS_NONE              000000018000ad10     lregex.obj
 0001:00009d18       PMFLAGS_FULLSCREEN         000000018000ad18     lregex.obj
 0001:00009d20       PMFLAGS_DETAILEDSTATUS     000000018000ad20     lregex.obj
 0001:00009d28       PMFLAGS_ALIGNEXTENSIONS    000000018000ad28     lregex.obj
 0001:00009d30       PMFLAGS_CASECONVERSION     000000018000ad30     lregex.obj
 0001:00009d38       PMFLAGS_NONE               000000018000ad38     lregex.obj
 0001:00009d40       OPIF_DISABLEFILTER         000000018000ad40     lregex.obj
 0001:00009d48       OPIF_DISABLESORTGROUPS     000000018000ad48     lregex.obj
 0001:00009d50       OPIF_DISABLEHIGHLIGHTING   000000018000ad50     lregex.obj
 0001:00009d58       OPIF_ADDDOTS               000000018000ad58     lregex.obj
 0001:00009d60       OPIF_RAWSELECTION          000000018000ad60     lregex.obj
 0001:00009d68       OPIF_REALNAMES             000000018000ad68     lregex.obj
 0001:00009d70       OPIF_SHOWNAMESONLY         000000018000ad70     lregex.obj
 0001:00009d78       OPIF_SHOWRIGHTALIGNNAMES   000000018000ad78     lregex.obj
 0001:00009d80       OPIF_SHOWPRESERVECASE      000000018000ad80     lregex.obj
 0001:00009d88       OPIF_COMPAREFATTIME        000000018000ad88     lregex.obj
 0001:00009d90       OPIF_EXTERNALGET           000000018000ad90     lregex.obj
 0001:00009d98       OPIF_EXTERNALPUT           000000018000ad98     lregex.obj
 0001:00009da0       OPIF_EXTERNALDELETE        000000018000ada0     lregex.obj
 0001:00009da8       OPIF_EXTERNALMKDIR         000000018000ada8     lregex.obj
 0001:00009db0       OPIF_USEATTRHIGHLIGHTING   000000018000adb0     lregex.obj
 0001:00009db8       OPIF_USECRC32              000000018000adb8     lregex.obj
 0001:00009dc0       OPIF_USEFREESIZE           000000018000adc0     lregex.obj
 0001:00009dc8       OPIF_SHORTCUT              000000018000adc8     lregex.obj
 0001:00009dd0       OPIF_NONE                  000000018000add0     lregex.obj
 0001:00009dd8       OPM_SILENT                 000000018000add8     lregex.obj
 0001:00009de0       OPM_FIND                   000000018000ade0     lregex.obj
 0001:00009de8       OPM_VIEW                   000000018000ade8     lregex.obj
 0001:00009df0       OPM_EDIT                   000000018000adf0     lregex.obj
 0001:00009df8       OPM_TOPLEVEL               000000018000adf8     lregex.obj
 0001:00009e00       OPM_DESCR                  000000018000ae00     lregex.obj
 0001:00009e08       OPM_QUICKVIEW              000000018000ae08     lregex.obj
 0001:00009e10       OPM_PGDN                   000000018000ae10     lregex.obj
 0001:00009e18       OPM_COMMANDS               000000018000ae18     lregex.obj
 0001:00009e20       OPM_NONE                   000000018000ae20     lregex.obj
 0001:00009e28       FOSF_ACTIVE                000000018000ae28     lregex.obj
 0001:00009e30       FOSF_NONE                  000000018000ae30     lregex.obj
 0001:00009e38       PCIF_NONE                  000000018000ae38     lregex.obj
 0001:00009e40       FarGuid                    000000018000ae40     lregex.obj
 0001:00009e50       PDF_DIALOGEVENTDRAWENABLE  000000018000ae50     lregex.obj
 0001:00009e58       PDF_PROCESSINGERROR        000000018000ae58     lregex.obj
 0001:00009e60       PDF_FULL_TIME_RESOLUTION   000000018000ae60     lregex.obj
 0001:00009ff8       LuamacroGuid               000000018000aff8     luamacro.obj
 0001:0000a008       FCF_FG_4BIT                000000018000b008     luamacro.obj
 0001:0000a010       FCF_BG_4BIT                000000018000b010     luamacro.obj
 0001:0000a018       FCF_4BITMASK               000000018000b018     luamacro.obj
 0001:0000a020       FCF_RAWATTR_MASK           000000018000b020     luamacro.obj
 0001:0000a028       FCF_EXTENDEDFLAGS          000000018000b028     luamacro.obj
 0001:0000a030       FCF_FG_BOLD                000000018000b030     luamacro.obj
 0001:0000a038       FCF_FG_ITALIC              000000018000b038     luamacro.obj
 0001:0000a040       FCF_FG_UNDERLINE           000000018000b040     luamacro.obj
 0001:0000a048       FCF_STYLEMASK              000000018000b048     luamacro.obj
 0001:0000a050       FCF_NONE                   000000018000b050     luamacro.obj
 0001:0000a058       CDF_NONE                   000000018000b058     luamacro.obj
 0001:0000a060       FMSG_WARNING               000000018000b060     luamacro.obj
 0001:0000a068       FMSG_ERRORTYPE             000000018000b068     luamacro.obj
 0001:0000a070       FMSG_KEEPBACKGROUND        000000018000b070     luamacro.obj
 0001:0000a078       FMSG_LEFTALIGN             000000018000b078     luamacro.obj
 0001:0000a080       FMSG_ALLINONE              000000018000b080     luamacro.obj
 0001:0000a088       FMSG_MB_OK                 000000018000b088     luamacro.obj
 0001:0000a090       FMSG_MB_OKCANCEL           000000018000b090     luamacro.obj
 0001:0000a098       FMSG_MB_ABORTRETRYIGNORE   000000018000b098     luamacro.obj
 0001:0000a0a0       FMSG_MB_YESNO              000000018000b0a0     luamacro.obj
 0001:0000a0a8       FMSG_MB_YESNOCANCEL        000000018000b0a8     luamacro.obj
 0001:0000a0b0       FMSG_MB_RETRYCANCEL        000000018000b0b0     luamacro.obj
 0001:0000a0b8       FMSG_NONE                  000000018000b0b8     luamacro.obj
 0001:0000a0c0       DIF_BOXCOLOR               000000018000b0c0     luamacro.obj
 0001:0000a0c8       DIF_GROUP                  000000018000b0c8     luamacro.obj
 0001:0000a0d0       DIF_LEFTTEXT               000000018000b0d0     luamacro.obj
 0001:0000a0d8       DIF_MOVESELECT             000000018000b0d8     luamacro.obj
 0001:0000a0e0       DIF_SHOWAMPERSAND          000000018000b0e0     luamacro.obj
 0001:0000a0e8       DIF_CENTERGROUP            000000018000b0e8     luamacro.obj
 0001:0000a0f0       DIF_NOBRACKETS             000000018000b0f0     luamacro.obj
 0001:0000a0f8       DIF_MANUALADDHISTORY       000000018000b0f8     luamacro.obj
 0001:0000a100       DIF_SEPARATOR              000000018000b100     luamacro.obj
 0001:0000a108       DIF_SEPARATOR2             000000018000b108     luamacro.obj
 0001:0000a110       DIF_EDITOR                 000000018000b110     luamacro.obj
 0001:0000a118       DIF_LISTNOAMPERSAND        000000018000b118     luamacro.obj
 0001:0000a120       DIF_LISTNOBOX              000000018000b120     luamacro.obj
 0001:0000a128       DIF_HISTORY                000000018000b128     luamacro.obj
 0001:0000a130       DIF_BTNNOCLOSE             000000018000b130     luamacro.obj
 0001:0000a138       DIF_CENTERTEXT             000000018000b138     luamacro.obj
 0001:0000a140       DIF_SEPARATORUSER          000000018000b140     luamacro.obj
 0001:0000a148       DIF_SETSHIELD              000000018000b148     luamacro.obj
 0001:0000a150       DIF_EDITEXPAND             000000018000b150     luamacro.obj
 0001:0000a158       DIF_DROPDOWNLIST           000000018000b158     luamacro.obj
 0001:0000a160       DIF_USELASTHISTORY         000000018000b160     luamacro.obj
 0001:0000a168       DIF_MASKEDIT               000000018000b168     luamacro.obj
 0001:0000a170       DIF_LISTTRACKMOUSE         000000018000b170     luamacro.obj
 0001:0000a178       DIF_LISTTRACKMOUSEINFOCUS  000000018000b178     luamacro.obj
 0001:0000a180       DIF_SELECTONENTRY          000000018000b180     luamacro.obj
 0001:0000a188       DIF_3STATE                 000000018000b188     luamacro.obj
 0001:0000a190       DIF_EDITPATH               000000018000b190     luamacro.obj
 0001:0000a198       DIF_LISTWRAPMODE           000000018000b198     luamacro.obj
 0001:0000a1a0       DIF_NOAUTOCOMPLETE         000000018000b1a0     luamacro.obj
 0001:0000a1a8       DIF_LISTAUTOHIGHLIGHT      000000018000b1a8     luamacro.obj
 0001:0000a1b0       DIF_LISTNOCLOSE            000000018000b1b0     luamacro.obj
 0001:0000a1b8       DIF_EDITPATHEXEC           000000018000b1b8     luamacro.obj
 0001:0000a1c0       DIF_HIDDEN                 000000018000b1c0     luamacro.obj
 0001:0000a1c8       DIF_READONLY               000000018000b1c8     luamacro.obj
 0001:0000a1d0       DIF_NOFOCUS                000000018000b1d0     luamacro.obj
 0001:0000a1d8       DIF_DISABLE                000000018000b1d8     luamacro.obj
 0001:0000a1e0       DIF_DEFAULTBUTTON          000000018000b1e0     luamacro.obj
 0001:0000a1e8       DIF_FOCUS                  000000018000b1e8     luamacro.obj
 0001:0000a1f0       DIF_RIGHTTEXT              000000018000b1f0     luamacro.obj
 0001:0000a1f8       DIF_WORDWRAP               000000018000b1f8     luamacro.obj
 0001:0000a200       DIF_NONE                   000000018000b200     luamacro.obj
 0001:0000a208       LIF_SELECTED               000000018000b208     luamacro.obj
 0001:0000a210       LIF_CHECKED                000000018000b210     luamacro.obj
 0001:0000a218       LIF_SEPARATOR              000000018000b218     luamacro.obj
 0001:0000a220       LIF_DISABLE                000000018000b220     luamacro.obj
 0001:0000a228       LIF_GRAYED                 000000018000b228     luamacro.obj
 0001:0000a230       LIF_HIDDEN                 000000018000b230     luamacro.obj
 0001:0000a238       LIF_DELETEUSERDATA         000000018000b238     luamacro.obj
 0001:0000a240       LIF_NONE                   000000018000b240     luamacro.obj
 0001:0000a248       LIFIND_EXACTMATCH          000000018000b248     luamacro.obj
 0001:0000a250       LIFIND_NONE                000000018000b250     luamacro.obj
 0001:0000a258       LINFO_SHOWNOBOX            000000018000b258     luamacro.obj
 0001:0000a260       LINFO_AUTOHIGHLIGHT        000000018000b260     luamacro.obj
 0001:0000a268       LINFO_REVERSEHIGHLIGHT     000000018000b268     luamacro.obj
 0001:0000a270       LINFO_WRAPMODE             000000018000b270     luamacro.obj
 0001:0000a278       LINFO_SHOWAMPERSAND        000000018000b278     luamacro.obj
 0001:0000a280       LINFO_NONE                 000000018000b280     luamacro.obj
 0001:0000a288       FDLG_WARNING               000000018000b288     luamacro.obj
 0001:0000a290       FDLG_SMALLDIALOG           000000018000b290     luamacro.obj
 0001:0000a298       FDLG_NODRAWSHADOW          000000018000b298     luamacro.obj
 0001:0000a2a0       FDLG_NODRAWPANEL           000000018000b2a0     luamacro.obj
 0001:0000a2a8       FDLG_KEEPCONSOLETITLE      000000018000b2a8     luamacro.obj
 0001:0000a2b0       FDLG_NONMODAL              000000018000b2b0     luamacro.obj
 0001:0000a2b8       FDLG_NONE                  000000018000b2b8     luamacro.obj
 0001:0000a2c0       MIF_SELECTED               000000018000b2c0     luamacro.obj
 0001:0000a2c8       MIF_CHECKED                000000018000b2c8     luamacro.obj
 0001:0000a2d0       MIF_SEPARATOR              000000018000b2d0     luamacro.obj
 0001:0000a2d8       MIF_DISABLE                000000018000b2d8     luamacro.obj
 0001:0000a2e0       MIF_GRAYED                 000000018000b2e0     luamacro.obj
 0001:0000a2e8       MIF_HIDDEN                 000000018000b2e8     luamacro.obj
 0001:0000a2f0       MIF_NONE                   000000018000b2f0     luamacro.obj
 0001:0000a2f8       FMENU_SHOWAMPERSAND        000000018000b2f8     luamacro.obj
 0001:0000a300       FMENU_WRAPMODE             000000018000b300     luamacro.obj
 0001:0000a308       FMENU_AUTOHIGHLIGHT        000000018000b308     luamacro.obj
 0001:0000a310       FMENU_REVERSEAUTOHIGHLIGHT 000000018000b310     luamacro.obj
 0001:0000a318       FMENU_CHANGECONSOLETITLE   000000018000b318     luamacro.obj
 0001:0000a320       FMENU_SHOWNOBOX            000000018000b320     luamacro.obj
 0001:0000a328       FMENU_SHOWSHORTBOX         000000018000b328     luamacro.obj
 0001:0000a330       FMENU_SHOWSINGLEBOX        000000018000b330     luamacro.obj
 0001:0000a338       FMENU_NODRAWSHADOW         000000018000b338     luamacro.obj
 0001:0000a340       FMENU_NONE                 000000018000b340     luamacro.obj
 0001:0000a348       PPIF_SELECTED              000000018000b348     luamacro.obj
 0001:0000a350       PPIF_PROCESSDESCR          000000018000b350     luamacro.obj
 0001:0000a358       PPIF_NONE                  000000018000b358     luamacro.obj
 0001:0000a360       PFLAGS_SHOWHIDDEN          000000018000b360     luamacro.obj
 0001:0000a368       PFLAGS_HIGHLIGHT           000000018000b368     luamacro.obj
 0001:0000a370       PFLAGS_REVERSESORTORDER    000000018000b370     luamacro.obj
 0001:0000a378       PFLAGS_USESORTGROUPS       000000018000b378     luamacro.obj
 0001:0000a380       PFLAGS_SELECTEDFIRST       000000018000b380     luamacro.obj
 0001:0000a388       PFLAGS_REALNAMES           000000018000b388     luamacro.obj
 0001:0000a390       PFLAGS_PANELLEFT           000000018000b390     luamacro.obj
 0001:0000a398       PFLAGS_DIRECTORIESFIRST    000000018000b398     luamacro.obj
 0001:0000a3a0       PFLAGS_USECRC32            000000018000b3a0     luamacro.obj
 0001:0000a3a8       PFLAGS_PLUGIN              000000018000b3a8     luamacro.obj
 0001:0000a3b0       PFLAGS_VISIBLE             000000018000b3b0     luamacro.obj
 0001:0000a3b8       PFLAGS_FOCUS               000000018000b3b8     luamacro.obj
 0001:0000a3c0       PFLAGS_ALTERNATIVENAMES    000000018000b3c0     luamacro.obj
 0001:0000a3c8       PFLAGS_SHORTCUT            000000018000b3c8     luamacro.obj
 0001:0000a3d0       PFLAGS_NONE                000000018000b3d0     luamacro.obj
 0001:0000a3d8       VF_NONMODAL                000000018000b3d8     luamacro.obj
 0001:0000a3e0       VF_DELETEONCLOSE           000000018000b3e0     luamacro.obj
 0001:0000a3e8       VF_ENABLE_F6               000000018000b3e8     luamacro.obj
 0001:0000a3f0       VF_DISABLEHISTORY          000000018000b3f0     luamacro.obj
 0001:0000a3f8       VF_IMMEDIATERETURN         000000018000b3f8     luamacro.obj
 0001:0000a400       VF_DELETEONLYFILEONCLOSE   000000018000b400     luamacro.obj
 0001:0000a408       VF_NONE                    000000018000b408     luamacro.obj
 0001:0000a410       EF_NONMODAL                000000018000b410     luamacro.obj
 0001:0000a418       EF_CREATENEW               000000018000b418     luamacro.obj
 0001:0000a420       EF_ENABLE_F6               000000018000b420     luamacro.obj
 0001:0000a428       EF_DISABLEHISTORY          000000018000b428     luamacro.obj
 0001:0000a430       EF_DELETEONCLOSE           000000018000b430     luamacro.obj
 0001:0000a438       EF_IMMEDIATERETURN         000000018000b438     luamacro.obj
 0001:0000a440       EF_DELETEONLYFILEONCLOSE   000000018000b440     luamacro.obj
 0001:0000a448       EF_LOCKED                  000000018000b448     luamacro.obj
 0001:0000a450       EF_DISABLESAVEPOS          000000018000b450     luamacro.obj
 0001:0000a458       EF_OPENMODE_MASK           000000018000b458     luamacro.obj
 0001:0000a460       EF_OPENMODE_QUERY          000000018000b460     luamacro.obj
 0001:0000a468       EF_OPENMODE_NEWIFOPEN      000000018000b468     luamacro.obj
 0001:0000a470       EF_OPENMODE_USEEXISTING    000000018000b470     luamacro.obj
 0001:0000a478       EF_OPENMODE_BREAKIFOPEN    000000018000b478     luamacro.obj
 0001:0000a480       EF_OPENMODE_RELOADIFOPEN   000000018000b480     luamacro.obj
 0001:0000a488       EN_NONE                    000000018000b488     luamacro.obj
 0001:0000a490       FHELP_NOSHOWERROR          000000018000b490     luamacro.obj
 0001:0000a498       FHELP_SELFHELP             000000018000b498     luamacro.obj
 0001:0000a4a0       FHELP_FARHELP              000000018000b4a0     luamacro.obj
 0001:0000a4a8       FHELP_CUSTOMFILE           000000018000b4a8     luamacro.obj
 0001:0000a4b0       FHELP_CUSTOMPATH           000000018000b4b0     luamacro.obj
 0001:0000a4b8       FHELP_GUID                 000000018000b4b8     luamacro.obj
 0001:0000a4c0       FHELP_USECONTENTS          000000018000b4c0     luamacro.obj
 0001:0000a4c8       FHELP_NONE                 000000018000b4c8     luamacro.obj
 0001:0000a4d0       KMFLAGS_SILENTCHECK        000000018000b4d0     luamacro.obj
 0001:0000a4d8       KMFLAGS_NOSENDKEYSTOPLUGINS 000000018000b4d8     luamacro.obj
 0001:0000a4e0       KMFLAGS_ENABLEOUTPUT       000000018000b4e0     luamacro.obj
 0001:0000a4e8       KMFLAGS_LANGMASK           000000018000b4e8     luamacro.obj
 0001:0000a4f0       KMFLAGS_LUA                000000018000b4f0     luamacro.obj
 0001:0000a4f8       KMFLAGS_MOONSCRIPT         000000018000b4f8     luamacro.obj
 0001:0000a500       KMFLAGS_NONE               000000018000b500     luamacro.obj
 0001:0000a508       AKMFLAGS_NONE              000000018000b508     luamacro.obj
 0001:0000a510       FSETCLR_REDRAW             000000018000b510     luamacro.obj
 0001:0000a518       FSETCLR_NONE               000000018000b518     luamacro.obj
 0001:0000a520       WIF_MODIFIED               000000018000b520     luamacro.obj
 0001:0000a528       WIF_CURRENT                000000018000b528     luamacro.obj
 0001:0000a530       WIF_MODAL                  000000018000b530     luamacro.obj
 0001:0000a538       WIF_NONE                   000000018000b538     luamacro.obj
 0001:0000a540       VOPT_SAVEFILEPOSITION      000000018000b540     luamacro.obj
 0001:0000a548       VOPT_AUTODETECTCODEPAGE    000000018000b548     luamacro.obj
 0001:0000a550       VOPT_SHOWTITLEBAR          000000018000b550     luamacro.obj
 0001:0000a558       VOPT_SHOWKEYBAR            000000018000b558     luamacro.obj
 0001:0000a560       VOPT_SHOWSCROLLBAR         000000018000b560     luamacro.obj
 0001:0000a568       VOPT_QUICKVIEW             000000018000b568     luamacro.obj
 0001:0000a570       VOPT_NONE                  000000018000b570     luamacro.obj
 0001:0000a578       VSMFL_REDRAW               000000018000b578     luamacro.obj
 0001:0000a580       VSMFL_NONE                 000000018000b580     luamacro.obj
 0001:0000a588       VSP_NOREDRAW               000000018000b588     luamacro.obj
 0001:0000a590       VSP_PERCENT                000000018000b590     luamacro.obj
 0001:0000a598       VSP_RELATIVE               000000018000b598     luamacro.obj
 0001:0000a5a0       VSP_NORETNEWPOS            000000018000b5a0     luamacro.obj
 0001:0000a5a8       VSP_NONE                   000000018000b5a8     luamacro.obj
 0001:0000a5b0       VMF_WRAP                   000000018000b5b0     luamacro.obj
 0001:0000a5b8       VMF_WORDWRAP               000000018000b5b8     luamacro.obj
 0001:0000a5c0       VMF_NONE                   000000018000b5c0     luamacro.obj
 0001:0000a5c8       ECF_TABMARKFIRST           000000018000b5c8     luamacro.obj
 0001:0000a5d0       ECF_TABMARKCURRENT         000000018000b5d0     luamacro.obj
 0001:0000a5d8       ECF_AUTODELETE             000000018000b5d8     luamacro.obj
 0001:0000a5e0       ECF_NONE                   000000018000b5e0     luamacro.obj
 0001:0000a5e8       FIB_ENABLEEMPTY            000000018000b5e8     luamacro.obj
 0001:0000a5f0       FIB_PASSWORD               000000018000b5f0     luamacro.obj
 0001:0000a5f8       FIB_EXPANDENV              000000018000b5f8     luamacro.obj
 0001:0000a600       FIB_NOUSELASTHISTORY       000000018000b600     luamacro.obj
 0001:0000a608       FIB_BUTTONS                000000018000b608     luamacro.obj
 0001:0000a610       FIB_NOAMPERSAND            000000018000b610     luamacro.obj
 0001:0000a618       FIB_EDITPATH               000000018000b618     luamacro.obj
 0001:0000a620       FIB_EDITPATHEXEC           000000018000b620     luamacro.obj
 0001:0000a628       FIB_NONE                   000000018000b628     luamacro.obj
 0001:0000a630       FPF_LOADED                 000000018000b630     luamacro.obj
 0001:0000a638       FPF_ANSI                   000000018000b638     luamacro.obj
 0001:0000a640       FPF_NONE                   000000018000b640     luamacro.obj
 0001:0000a648       PN_CMPNAME                 000000018000b648     luamacro.obj
 0001:0000a650       PN_CMPNAMELIST             000000018000b650     luamacro.obj
 0001:0000a658       PN_GENERATENAME            000000018000b658     luamacro.obj
 0001:0000a660       PN_CHECKMASK               000000018000b660     luamacro.obj
 0001:0000a668       PN_SKIPPATH                000000018000b668     luamacro.obj
 0001:0000a670       PN_SHOWERRORMESSAGE        000000018000b670     luamacro.obj
 0001:0000a678       PN_NONE                    000000018000b678     luamacro.obj
 0001:0000a680       XLAT_SWITCHKEYBLAYOUT      000000018000b680     luamacro.obj
 0001:0000a688       XLAT_SWITCHKEYBBEEP        000000018000b688     luamacro.obj
 0001:0000a690       XLAT_USEKEYBLAYOUTNAME     000000018000b690     luamacro.obj
 0001:0000a698       XLAT_CONVERTALLCMDLINE     000000018000b698     luamacro.obj
 0001:0000a6a0       XLAT_NONE                  000000018000b6a0     luamacro.obj
 0001:0000a6a8       FRS_RETUPDIR               000000018000b6a8     luamacro.obj
 0001:0000a6b0       FRS_RECUR                  000000018000b6b0     luamacro.obj
 0001:0000a6b8       FRS_SCANSYMLINK            000000018000b6b8     luamacro.obj
 0001:0000a6c0       FRS_NONE                   000000018000b6c0     luamacro.obj
 0001:0000a6c8       MLF_SHOWERRMSG             000000018000b6c8     luamacro.obj
 0001:0000a6d0       MLF_DONOTUPDATEPANEL       000000018000b6d0     luamacro.obj
 0001:0000a6d8       MLF_HOLDTARGET             000000018000b6d8     luamacro.obj
 0001:0000a6e0       MLF_NONE                   000000018000b6e0     luamacro.obj
 0001:0000a6e8       FFFS_COMMAS                000000018000b6e8     luamacro.obj
 0001:0000a6f0       FFFS_FLOATSIZE             000000018000b6f0     luamacro.obj
 0001:0000a6f8       FFFS_SHOWBYTESINDEX        000000018000b6f8     luamacro.obj
 0001:0000a700       FFFS_ECONOMIC              000000018000b700     luamacro.obj
 0001:0000a708       FFFS_THOUSAND              000000018000b708     luamacro.obj
 0001:0000a710       FFFS_MINSIZEINDEX          000000018000b710     luamacro.obj
 0001:0000a718       FFFS_MINSIZEINDEX_MASK     000000018000b718     luamacro.obj
 0001:0000a720       FFFS_NONE                  000000018000b720     luamacro.obj
 0001:0000a728       PF_PRELOAD                 000000018000b728     luamacro.obj
 0001:0000a730       PF_DISABLEPANELS           000000018000b730     luamacro.obj
 0001:0000a738       PF_EDITOR                  000000018000b738     luamacro.obj
 0001:0000a740       PF_VIEWER                  000000018000b740     luamacro.obj
 0001:0000a748       PF_FULLCMDLINE             000000018000b748     luamacro.obj
 0001:0000a750       PF_DIALOG                  000000018000b750     luamacro.obj
 0001:0000a758       PF_NONE                    000000018000b758     luamacro.obj
 0001:0000a760       IPLFLAGS_SEPARATOR         000000018000b760     luamacro.obj
 0001:0000a768       IPLFLAGS_NONE              000000018000b768     luamacro.obj
 0001:0000a770       PMFLAGS_FULLSCREEN         000000018000b770     luamacro.obj
 0001:0000a778       PMFLAGS_DETAILEDSTATUS     000000018000b778     luamacro.obj
 0001:0000a780       PMFLAGS_ALIGNEXTENSIONS    000000018000b780     luamacro.obj
 0001:0000a788       PMFLAGS_CASECONVERSION     000000018000b788     luamacro.obj
 0001:0000a790       PMFLAGS_NONE               000000018000b790     luamacro.obj
 0001:0000a798       OPIF_DISABLEFILTER         000000018000b798     luamacro.obj
 0001:0000a7a0       OPIF_DISABLESORTGROUPS     000000018000b7a0     luamacro.obj
 0001:0000a7a8       OPIF_DISABLEHIGHLIGHTING   000000018000b7a8     luamacro.obj
 0001:0000a7b0       OPIF_ADDDOTS               000000018000b7b0     luamacro.obj
 0001:0000a7b8       OPIF_RAWSELECTION          000000018000b7b8     luamacro.obj
 0001:0000a7c0       OPIF_REALNAMES             000000018000b7c0     luamacro.obj
 0001:0000a7c8       OPIF_SHOWNAMESONLY         000000018000b7c8     luamacro.obj
 0001:0000a7d0       OPIF_SHOWRIGHTALIGNNAMES   000000018000b7d0     luamacro.obj
 0001:0000a7d8       OPIF_SHOWPRESERVECASE      000000018000b7d8     luamacro.obj
 0001:0000a7e0       OPIF_COMPAREFATTIME        000000018000b7e0     luamacro.obj
 0001:0000a7e8       OPIF_EXTERNALGET           000000018000b7e8     luamacro.obj
 0001:0000a7f0       OPIF_EXTERNALPUT           000000018000b7f0     luamacro.obj
 0001:0000a7f8       OPIF_EXTERNALDELETE        000000018000b7f8     luamacro.obj
 0001:0000a800       OPIF_EXTERNALMKDIR         000000018000b800     luamacro.obj
 0001:0000a808       OPIF_USEATTRHIGHLIGHTING   000000018000b808     luamacro.obj
 0001:0000a810       OPIF_USECRC32              000000018000b810     luamacro.obj
 0001:0000a818       OPIF_USEFREESIZE           000000018000b818     luamacro.obj
 0001:0000a820       OPIF_SHORTCUT              000000018000b820     luamacro.obj
 0001:0000a828       OPIF_NONE                  000000018000b828     luamacro.obj
 0001:0000a830       OPM_SILENT                 000000018000b830     luamacro.obj
 0001:0000a838       OPM_FIND                   000000018000b838     luamacro.obj
 0001:0000a840       OPM_VIEW                   000000018000b840     luamacro.obj
 0001:0000a848       OPM_EDIT                   000000018000b848     luamacro.obj
 0001:0000a850       OPM_TOPLEVEL               000000018000b850     luamacro.obj
 0001:0000a858       OPM_DESCR                  000000018000b858     luamacro.obj
 0001:0000a860       OPM_QUICKVIEW              000000018000b860     luamacro.obj
 0001:0000a868       OPM_PGDN                   000000018000b868     luamacro.obj
 0001:0000a870       OPM_COMMANDS               000000018000b870     luamacro.obj
 0001:0000a878       OPM_NONE                   000000018000b878     luamacro.obj
 0001:0000a880       FOSF_ACTIVE                000000018000b880     luamacro.obj
 0001:0000a888       FOSF_NONE                  000000018000b888     luamacro.obj
 0001:0000a890       PCIF_NONE                  000000018000b890     luamacro.obj
 0001:0000a898       FarGuid                    000000018000b898     luamacro.obj
 0001:0000a8a8       PDF_DIALOGEVENTDRAWENABLE  000000018000b8a8     luamacro.obj
 0001:0000a8b0       PDF_PROCESSINGERROR        000000018000b8b0     luamacro.obj
 0001:0000a8b8       PDF_FULL_TIME_RESOLUTION   000000018000b8b8     luamacro.obj
 0001:0000a990       FCF_FG_4BIT                000000018000b990     lusercontrol.obj
 0001:0000a998       FCF_BG_4BIT                000000018000b998     lusercontrol.obj
 0001:0000a9a0       FCF_4BITMASK               000000018000b9a0     lusercontrol.obj
 0001:0000a9a8       FCF_RAWATTR_MASK           000000018000b9a8     lusercontrol.obj
 0001:0000a9b0       FCF_EXTENDEDFLAGS          000000018000b9b0     lusercontrol.obj
 0001:0000a9b8       FCF_FG_BOLD                000000018000b9b8     lusercontrol.obj
 0001:0000a9c0       FCF_FG_ITALIC              000000018000b9c0     lusercontrol.obj
 0001:0000a9c8       FCF_FG_UNDERLINE           000000018000b9c8     lusercontrol.obj
 0001:0000a9d0       FCF_STYLEMASK              000000018000b9d0     lusercontrol.obj
 0001:0000a9d8       FCF_NONE                   000000018000b9d8     lusercontrol.obj
 0001:0000a9e0       CDF_NONE                   000000018000b9e0     lusercontrol.obj
 0001:0000a9e8       FMSG_WARNING               000000018000b9e8     lusercontrol.obj
 0001:0000a9f0       FMSG_ERRORTYPE             000000018000b9f0     lusercontrol.obj
 0001:0000a9f8       FMSG_KEEPBACKGROUND        000000018000b9f8     lusercontrol.obj
 0001:0000aa00       FMSG_LEFTALIGN             000000018000ba00     lusercontrol.obj
 0001:0000aa08       FMSG_ALLINONE              000000018000ba08     lusercontrol.obj
 0001:0000aa10       FMSG_MB_OK                 000000018000ba10     lusercontrol.obj
 0001:0000aa18       FMSG_MB_OKCANCEL           000000018000ba18     lusercontrol.obj
 0001:0000aa20       FMSG_MB_ABORTRETRYIGNORE   000000018000ba20     lusercontrol.obj
 0001:0000aa28       FMSG_MB_YESNO              000000018000ba28     lusercontrol.obj
 0001:0000aa30       FMSG_MB_YESNOCANCEL        000000018000ba30     lusercontrol.obj
 0001:0000aa38       FMSG_MB_RETRYCANCEL        000000018000ba38     lusercontrol.obj
 0001:0000aa40       FMSG_NONE                  000000018000ba40     lusercontrol.obj
 0001:0000aa48       DIF_BOXCOLOR               000000018000ba48     lusercontrol.obj
 0001:0000aa50       DIF_GROUP                  000000018000ba50     lusercontrol.obj
 0001:0000aa58       DIF_LEFTTEXT               000000018000ba58     lusercontrol.obj
 0001:0000aa60       DIF_MOVESELECT             000000018000ba60     lusercontrol.obj
 0001:0000aa68       DIF_SHOWAMPERSAND          000000018000ba68     lusercontrol.obj
 0001:0000aa70       DIF_CENTERGROUP            000000018000ba70     lusercontrol.obj
 0001:0000aa78       DIF_NOBRACKETS             000000018000ba78     lusercontrol.obj
 0001:0000aa80       DIF_MANUALADDHISTORY       000000018000ba80     lusercontrol.obj
 0001:0000aa88       DIF_SEPARATOR              000000018000ba88     lusercontrol.obj
 0001:0000aa90       DIF_SEPARATOR2             000000018000ba90     lusercontrol.obj
 0001:0000aa98       DIF_EDITOR                 000000018000ba98     lusercontrol.obj
 0001:0000aaa0       DIF_LISTNOAMPERSAND        000000018000baa0     lusercontrol.obj
 0001:0000aaa8       DIF_LISTNOBOX              000000018000baa8     lusercontrol.obj
 0001:0000aab0       DIF_HISTORY                000000018000bab0     lusercontrol.obj
 0001:0000aab8       DIF_BTNNOCLOSE             000000018000bab8     lusercontrol.obj
 0001:0000aac0       DIF_CENTERTEXT             000000018000bac0     lusercontrol.obj
 0001:0000aac8       DIF_SEPARATORUSER          000000018000bac8     lusercontrol.obj
 0001:0000aad0       DIF_SETSHIELD              000000018000bad0     lusercontrol.obj
 0001:0000aad8       DIF_EDITEXPAND             000000018000bad8     lusercontrol.obj
 0001:0000aae0       DIF_DROPDOWNLIST           000000018000bae0     lusercontrol.obj
 0001:0000aae8       DIF_USELASTHISTORY         000000018000bae8     lusercontrol.obj
 0001:0000aaf0       DIF_MASKEDIT               000000018000baf0     lusercontrol.obj
 0001:0000aaf8       DIF_LISTTRACKMOUSE         000000018000baf8     lusercontrol.obj
 0001:0000ab00       DIF_LISTTRACKMOUSEINFOCUS  000000018000bb00     lusercontrol.obj
 0001:0000ab08       DIF_SELECTONENTRY          000000018000bb08     lusercontrol.obj
 0001:0000ab10       DIF_3STATE                 000000018000bb10     lusercontrol.obj
 0001:0000ab18       DIF_EDITPATH               000000018000bb18     lusercontrol.obj
 0001:0000ab20       DIF_LISTWRAPMODE           000000018000bb20     lusercontrol.obj
 0001:0000ab28       DIF_NOAUTOCOMPLETE         000000018000bb28     lusercontrol.obj
 0001:0000ab30       DIF_LISTAUTOHIGHLIGHT      000000018000bb30     lusercontrol.obj
 0001:0000ab38       DIF_LISTNOCLOSE            000000018000bb38     lusercontrol.obj
 0001:0000ab40       DIF_EDITPATHEXEC           000000018000bb40     lusercontrol.obj
 0001:0000ab48       DIF_HIDDEN                 000000018000bb48     lusercontrol.obj
 0001:0000ab50       DIF_READONLY               000000018000bb50     lusercontrol.obj
 0001:0000ab58       DIF_NOFOCUS                000000018000bb58     lusercontrol.obj
 0001:0000ab60       DIF_DISABLE                000000018000bb60     lusercontrol.obj
 0001:0000ab68       DIF_DEFAULTBUTTON          000000018000bb68     lusercontrol.obj
 0001:0000ab70       DIF_FOCUS                  000000018000bb70     lusercontrol.obj
 0001:0000ab78       DIF_RIGHTTEXT              000000018000bb78     lusercontrol.obj
 0001:0000ab80       DIF_WORDWRAP               000000018000bb80     lusercontrol.obj
 0001:0000ab88       DIF_NONE                   000000018000bb88     lusercontrol.obj
 0001:0000ab90       LIF_SELECTED               000000018000bb90     lusercontrol.obj
 0001:0000ab98       LIF_CHECKED                000000018000bb98     lusercontrol.obj
 0001:0000aba0       LIF_SEPARATOR              000000018000bba0     lusercontrol.obj
 0001:0000aba8       LIF_DISABLE                000000018000bba8     lusercontrol.obj
 0001:0000abb0       LIF_GRAYED                 000000018000bbb0     lusercontrol.obj
 0001:0000abb8       LIF_HIDDEN                 000000018000bbb8     lusercontrol.obj
 0001:0000abc0       LIF_DELETEUSERDATA         000000018000bbc0     lusercontrol.obj
 0001:0000abc8       LIF_NONE                   000000018000bbc8     lusercontrol.obj
 0001:0000abd0       LIFIND_EXACTMATCH          000000018000bbd0     lusercontrol.obj
 0001:0000abd8       LIFIND_NONE                000000018000bbd8     lusercontrol.obj
 0001:0000abe0       LINFO_SHOWNOBOX            000000018000bbe0     lusercontrol.obj
 0001:0000abe8       LINFO_AUTOHIGHLIGHT        000000018000bbe8     lusercontrol.obj
 0001:0000abf0       LINFO_REVERSEHIGHLIGHT     000000018000bbf0     lusercontrol.obj
 0001:0000abf8       LINFO_WRAPMODE             000000018000bbf8     lusercontrol.obj
 0001:0000ac00       LINFO_SHOWAMPERSAND        000000018000bc00     lusercontrol.obj
 0001:0000ac08       LINFO_NONE                 000000018000bc08     lusercontrol.obj
 0001:0000ac10       FDLG_WARNING               000000018000bc10     lusercontrol.obj
 0001:0000ac18       FDLG_SMALLDIALOG           000000018000bc18     lusercontrol.obj
 0001:0000ac20       FDLG_NODRAWSHADOW          000000018000bc20     lusercontrol.obj
 0001:0000ac28       FDLG_NODRAWPANEL           000000018000bc28     lusercontrol.obj
 0001:0000ac30       FDLG_KEEPCONSOLETITLE      000000018000bc30     lusercontrol.obj
 0001:0000ac38       FDLG_NONMODAL              000000018000bc38     lusercontrol.obj
 0001:0000ac40       FDLG_NONE                  000000018000bc40     lusercontrol.obj
 0001:0000ac48       MIF_SELECTED               000000018000bc48     lusercontrol.obj
 0001:0000ac50       MIF_CHECKED                000000018000bc50     lusercontrol.obj
 0001:0000ac58       MIF_SEPARATOR              000000018000bc58     lusercontrol.obj
 0001:0000ac60       MIF_DISABLE                000000018000bc60     lusercontrol.obj
 0001:0000ac68       MIF_GRAYED                 000000018000bc68     lusercontrol.obj
 0001:0000ac70       MIF_HIDDEN                 000000018000bc70     lusercontrol.obj
 0001:0000ac78       MIF_NONE                   000000018000bc78     lusercontrol.obj
 0001:0000ac80       FMENU_SHOWAMPERSAND        000000018000bc80     lusercontrol.obj
 0001:0000ac88       FMENU_WRAPMODE             000000018000bc88     lusercontrol.obj
 0001:0000ac90       FMENU_AUTOHIGHLIGHT        000000018000bc90     lusercontrol.obj
 0001:0000ac98       FMENU_REVERSEAUTOHIGHLIGHT 000000018000bc98     lusercontrol.obj
 0001:0000aca0       FMENU_CHANGECONSOLETITLE   000000018000bca0     lusercontrol.obj
 0001:0000aca8       FMENU_SHOWNOBOX            000000018000bca8     lusercontrol.obj
 0001:0000acb0       FMENU_SHOWSHORTBOX         000000018000bcb0     lusercontrol.obj
 0001:0000acb8       FMENU_SHOWSINGLEBOX        000000018000bcb8     lusercontrol.obj
 0001:0000acc0       FMENU_NODRAWSHADOW         000000018000bcc0     lusercontrol.obj
 0001:0000acc8       FMENU_NONE                 000000018000bcc8     lusercontrol.obj
 0001:0000acd0       PPIF_SELECTED              000000018000bcd0     lusercontrol.obj
 0001:0000acd8       PPIF_PROCESSDESCR          000000018000bcd8     lusercontrol.obj
 0001:0000ace0       PPIF_NONE                  000000018000bce0     lusercontrol.obj
 0001:0000ace8       PFLAGS_SHOWHIDDEN          000000018000bce8     lusercontrol.obj
 0001:0000acf0       PFLAGS_HIGHLIGHT           000000018000bcf0     lusercontrol.obj
 0001:0000acf8       PFLAGS_REVERSESORTORDER    000000018000bcf8     lusercontrol.obj
 0001:0000ad00       PFLAGS_USESORTGROUPS       000000018000bd00     lusercontrol.obj
 0001:0000ad08       PFLAGS_SELECTEDFIRST       000000018000bd08     lusercontrol.obj
 0001:0000ad10       PFLAGS_REALNAMES           000000018000bd10     lusercontrol.obj
 0001:0000ad18       PFLAGS_PANELLEFT           000000018000bd18     lusercontrol.obj
 0001:0000ad20       PFLAGS_DIRECTORIESFIRST    000000018000bd20     lusercontrol.obj
 0001:0000ad28       PFLAGS_USECRC32            000000018000bd28     lusercontrol.obj
 0001:0000ad30       PFLAGS_PLUGIN              000000018000bd30     lusercontrol.obj
 0001:0000ad38       PFLAGS_VISIBLE             000000018000bd38     lusercontrol.obj
 0001:0000ad40       PFLAGS_FOCUS               000000018000bd40     lusercontrol.obj
 0001:0000ad48       PFLAGS_ALTERNATIVENAMES    000000018000bd48     lusercontrol.obj
 0001:0000ad50       PFLAGS_SHORTCUT            000000018000bd50     lusercontrol.obj
 0001:0000ad58       PFLAGS_NONE                000000018000bd58     lusercontrol.obj
 0001:0000ad60       VF_NONMODAL                000000018000bd60     lusercontrol.obj
 0001:0000ad68       VF_DELETEONCLOSE           000000018000bd68     lusercontrol.obj
 0001:0000ad70       VF_ENABLE_F6               000000018000bd70     lusercontrol.obj
 0001:0000ad78       VF_DISABLEHISTORY          000000018000bd78     lusercontrol.obj
 0001:0000ad80       VF_IMMEDIATERETURN         000000018000bd80     lusercontrol.obj
 0001:0000ad88       VF_DELETEONLYFILEONCLOSE   000000018000bd88     lusercontrol.obj
 0001:0000ad90       VF_NONE                    000000018000bd90     lusercontrol.obj
 0001:0000ad98       EF_NONMODAL                000000018000bd98     lusercontrol.obj
 0001:0000ada0       EF_CREATENEW               000000018000bda0     lusercontrol.obj
 0001:0000ada8       EF_ENABLE_F6               000000018000bda8     lusercontrol.obj
 0001:0000adb0       EF_DISABLEHISTORY          000000018000bdb0     lusercontrol.obj
 0001:0000adb8       EF_DELETEONCLOSE           000000018000bdb8     lusercontrol.obj
 0001:0000adc0       EF_IMMEDIATERETURN         000000018000bdc0     lusercontrol.obj
 0001:0000adc8       EF_DELETEONLYFILEONCLOSE   000000018000bdc8     lusercontrol.obj
 0001:0000add0       EF_LOCKED                  000000018000bdd0     lusercontrol.obj
 0001:0000add8       EF_DISABLESAVEPOS          000000018000bdd8     lusercontrol.obj
 0001:0000ade0       EF_OPENMODE_MASK           000000018000bde0     lusercontrol.obj
 0001:0000ade8       EF_OPENMODE_QUERY          000000018000bde8     lusercontrol.obj
 0001:0000adf0       EF_OPENMODE_NEWIFOPEN      000000018000bdf0     lusercontrol.obj
 0001:0000adf8       EF_OPENMODE_USEEXISTING    000000018000bdf8     lusercontrol.obj
 0001:0000ae00       EF_OPENMODE_BREAKIFOPEN    000000018000be00     lusercontrol.obj
 0001:0000ae08       EF_OPENMODE_RELOADIFOPEN   000000018000be08     lusercontrol.obj
 0001:0000ae10       EN_NONE                    000000018000be10     lusercontrol.obj
 0001:0000ae18       FHELP_NOSHOWERROR          000000018000be18     lusercontrol.obj
 0001:0000ae20       FHELP_SELFHELP             000000018000be20     lusercontrol.obj
 0001:0000ae28       FHELP_FARHELP              000000018000be28     lusercontrol.obj
 0001:0000ae30       FHELP_CUSTOMFILE           000000018000be30     lusercontrol.obj
 0001:0000ae38       FHELP_CUSTOMPATH           000000018000be38     lusercontrol.obj
 0001:0000ae40       FHELP_GUID                 000000018000be40     lusercontrol.obj
 0001:0000ae48       FHELP_USECONTENTS          000000018000be48     lusercontrol.obj
 0001:0000ae50       FHELP_NONE                 000000018000be50     lusercontrol.obj
 0001:0000ae58       KMFLAGS_SILENTCHECK        000000018000be58     lusercontrol.obj
 0001:0000ae60       KMFLAGS_NOSENDKEYSTOPLUGINS 000000018000be60     lusercontrol.obj
 0001:0000ae68       KMFLAGS_ENABLEOUTPUT       000000018000be68     lusercontrol.obj
 0001:0000ae70       KMFLAGS_LANGMASK           000000018000be70     lusercontrol.obj
 0001:0000ae78       KMFLAGS_LUA                000000018000be78     lusercontrol.obj
 0001:0000ae80       KMFLAGS_MOONSCRIPT         000000018000be80     lusercontrol.obj
 0001:0000ae88       KMFLAGS_NONE               000000018000be88     lusercontrol.obj
 0001:0000ae90       AKMFLAGS_NONE              000000018000be90     lusercontrol.obj
 0001:0000ae98       FSETCLR_REDRAW             000000018000be98     lusercontrol.obj
 0001:0000aea0       FSETCLR_NONE               000000018000bea0     lusercontrol.obj
 0001:0000aea8       WIF_MODIFIED               000000018000bea8     lusercontrol.obj
 0001:0000aeb0       WIF_CURRENT                000000018000beb0     lusercontrol.obj
 0001:0000aeb8       WIF_MODAL                  000000018000beb8     lusercontrol.obj
 0001:0000aec0       WIF_NONE                   000000018000bec0     lusercontrol.obj
 0001:0000aec8       VOPT_SAVEFILEPOSITION      000000018000bec8     lusercontrol.obj
 0001:0000aed0       VOPT_AUTODETECTCODEPAGE    000000018000bed0     lusercontrol.obj
 0001:0000aed8       VOPT_SHOWTITLEBAR          000000018000bed8     lusercontrol.obj
 0001:0000aee0       VOPT_SHOWKEYBAR            000000018000bee0     lusercontrol.obj
 0001:0000aee8       VOPT_SHOWSCROLLBAR         000000018000bee8     lusercontrol.obj
 0001:0000aef0       VOPT_QUICKVIEW             000000018000bef0     lusercontrol.obj
 0001:0000aef8       VOPT_NONE                  000000018000bef8     lusercontrol.obj
 0001:0000af00       VSMFL_REDRAW               000000018000bf00     lusercontrol.obj
 0001:0000af08       VSMFL_NONE                 000000018000bf08     lusercontrol.obj
 0001:0000af10       VSP_NOREDRAW               000000018000bf10     lusercontrol.obj
 0001:0000af18       VSP_PERCENT                000000018000bf18     lusercontrol.obj
 0001:0000af20       VSP_RELATIVE               000000018000bf20     lusercontrol.obj
 0001:0000af28       VSP_NORETNEWPOS            000000018000bf28     lusercontrol.obj
 0001:0000af30       VSP_NONE                   000000018000bf30     lusercontrol.obj
 0001:0000af38       VMF_WRAP                   000000018000bf38     lusercontrol.obj
 0001:0000af40       VMF_WORDWRAP               000000018000bf40     lusercontrol.obj
 0001:0000af48       VMF_NONE                   000000018000bf48     lusercontrol.obj
 0001:0000af50       ECF_TABMARKFIRST           000000018000bf50     lusercontrol.obj
 0001:0000af58       ECF_TABMARKCURRENT         000000018000bf58     lusercontrol.obj
 0001:0000af60       ECF_AUTODELETE             000000018000bf60     lusercontrol.obj
 0001:0000af68       ECF_NONE                   000000018000bf68     lusercontrol.obj
 0001:0000af70       FIB_ENABLEEMPTY            000000018000bf70     lusercontrol.obj
 0001:0000af78       FIB_PASSWORD               000000018000bf78     lusercontrol.obj
 0001:0000af80       FIB_EXPANDENV              000000018000bf80     lusercontrol.obj
 0001:0000af88       FIB_NOUSELASTHISTORY       000000018000bf88     lusercontrol.obj
 0001:0000af90       FIB_BUTTONS                000000018000bf90     lusercontrol.obj
 0001:0000af98       FIB_NOAMPERSAND            000000018000bf98     lusercontrol.obj
 0001:0000afa0       FIB_EDITPATH               000000018000bfa0     lusercontrol.obj
 0001:0000afa8       FIB_EDITPATHEXEC           000000018000bfa8     lusercontrol.obj
 0001:0000afb0       FIB_NONE                   000000018000bfb0     lusercontrol.obj
 0001:0000afb8       FPF_LOADED                 000000018000bfb8     lusercontrol.obj
 0001:0000afc0       FPF_ANSI                   000000018000bfc0     lusercontrol.obj
 0001:0000afc8       FPF_NONE                   000000018000bfc8     lusercontrol.obj
 0001:0000afd0       PN_CMPNAME                 000000018000bfd0     lusercontrol.obj
 0001:0000afd8       PN_CMPNAMELIST             000000018000bfd8     lusercontrol.obj
 0001:0000afe0       PN_GENERATENAME            000000018000bfe0     lusercontrol.obj
 0001:0000afe8       PN_CHECKMASK               000000018000bfe8     lusercontrol.obj
 0001:0000aff0       PN_SKIPPATH                000000018000bff0     lusercontrol.obj
 0001:0000aff8       PN_SHOWERRORMESSAGE        000000018000bff8     lusercontrol.obj
 0001:0000b000       PN_NONE                    000000018000c000     lusercontrol.obj
 0001:0000b008       XLAT_SWITCHKEYBLAYOUT      000000018000c008     lusercontrol.obj
 0001:0000b010       XLAT_SWITCHKEYBBEEP        000000018000c010     lusercontrol.obj
 0001:0000b018       XLAT_USEKEYBLAYOUTNAME     000000018000c018     lusercontrol.obj
 0001:0000b020       XLAT_CONVERTALLCMDLINE     000000018000c020     lusercontrol.obj
 0001:0000b028       XLAT_NONE                  000000018000c028     lusercontrol.obj
 0001:0000b030       FRS_RETUPDIR               000000018000c030     lusercontrol.obj
 0001:0000b038       FRS_RECUR                  000000018000c038     lusercontrol.obj
 0001:0000b040       FRS_SCANSYMLINK            000000018000c040     lusercontrol.obj
 0001:0000b048       FRS_NONE                   000000018000c048     lusercontrol.obj
 0001:0000b050       MLF_SHOWERRMSG             000000018000c050     lusercontrol.obj
 0001:0000b058       MLF_DONOTUPDATEPANEL       000000018000c058     lusercontrol.obj
 0001:0000b060       MLF_HOLDTARGET             000000018000c060     lusercontrol.obj
 0001:0000b068       MLF_NONE                   000000018000c068     lusercontrol.obj
 0001:0000b070       FFFS_COMMAS                000000018000c070     lusercontrol.obj
 0001:0000b078       FFFS_FLOATSIZE             000000018000c078     lusercontrol.obj
 0001:0000b080       FFFS_SHOWBYTESINDEX        000000018000c080     lusercontrol.obj
 0001:0000b088       FFFS_ECONOMIC              000000018000c088     lusercontrol.obj
 0001:0000b090       FFFS_THOUSAND              000000018000c090     lusercontrol.obj
 0001:0000b098       FFFS_MINSIZEINDEX          000000018000c098     lusercontrol.obj
 0001:0000b0a0       FFFS_MINSIZEINDEX_MASK     000000018000c0a0     lusercontrol.obj
 0001:0000b0a8       FFFS_NONE                  000000018000c0a8     lusercontrol.obj
 0001:0000b0b0       PF_PRELOAD                 000000018000c0b0     lusercontrol.obj
 0001:0000b0b8       PF_DISABLEPANELS           000000018000c0b8     lusercontrol.obj
 0001:0000b0c0       PF_EDITOR                  000000018000c0c0     lusercontrol.obj
 0001:0000b0c8       PF_VIEWER                  000000018000c0c8     lusercontrol.obj
 0001:0000b0d0       PF_FULLCMDLINE             000000018000c0d0     lusercontrol.obj
 0001:0000b0d8       PF_DIALOG                  000000018000c0d8     lusercontrol.obj
 0001:0000b0e0       PF_NONE                    000000018000c0e0     lusercontrol.obj
 0001:0000b0e8       IPLFLAGS_SEPARATOR         000000018000c0e8     lusercontrol.obj
 0001:0000b0f0       IPLFLAGS_NONE              000000018000c0f0     lusercontrol.obj
 0001:0000b0f8       PMFLAGS_FULLSCREEN         000000018000c0f8     lusercontrol.obj
 0001:0000b100       PMFLAGS_DETAILEDSTATUS     000000018000c100     lusercontrol.obj
 0001:0000b108       PMFLAGS_ALIGNEXTENSIONS    000000018000c108     lusercontrol.obj
 0001:0000b110       PMFLAGS_CASECONVERSION     000000018000c110     lusercontrol.obj
 0001:0000b118       PMFLAGS_NONE               000000018000c118     lusercontrol.obj
 0001:0000b120       OPIF_DISABLEFILTER         000000018000c120     lusercontrol.obj
 0001:0000b128       OPIF_DISABLESORTGROUPS     000000018000c128     lusercontrol.obj
 0001:0000b130       OPIF_DISABLEHIGHLIGHTING   000000018000c130     lusercontrol.obj
 0001:0000b138       OPIF_ADDDOTS               000000018000c138     lusercontrol.obj
 0001:0000b140       OPIF_RAWSELECTION          000000018000c140     lusercontrol.obj
 0001:0000b148       OPIF_REALNAMES             000000018000c148     lusercontrol.obj
 0001:0000b150       OPIF_SHOWNAMESONLY         000000018000c150     lusercontrol.obj
 0001:0000b158       OPIF_SHOWRIGHTALIGNNAMES   000000018000c158     lusercontrol.obj
 0001:0000b160       OPIF_SHOWPRESERVECASE      000000018000c160     lusercontrol.obj
 0001:0000b168       OPIF_COMPAREFATTIME        000000018000c168     lusercontrol.obj
 0001:0000b170       OPIF_EXTERNALGET           000000018000c170     lusercontrol.obj
 0001:0000b178       OPIF_EXTERNALPUT           000000018000c178     lusercontrol.obj
 0001:0000b180       OPIF_EXTERNALDELETE        000000018000c180     lusercontrol.obj
 0001:0000b188       OPIF_EXTERNALMKDIR         000000018000c188     lusercontrol.obj
 0001:0000b190       OPIF_USEATTRHIGHLIGHTING   000000018000c190     lusercontrol.obj
 0001:0000b198       OPIF_USECRC32              000000018000c198     lusercontrol.obj
 0001:0000b1a0       OPIF_USEFREESIZE           000000018000c1a0     lusercontrol.obj
 0001:0000b1a8       OPIF_SHORTCUT              000000018000c1a8     lusercontrol.obj
 0001:0000b1b0       OPIF_NONE                  000000018000c1b0     lusercontrol.obj
 0001:0000b1b8       OPM_SILENT                 000000018000c1b8     lusercontrol.obj
 0001:0000b1c0       OPM_FIND                   000000018000c1c0     lusercontrol.obj
 0001:0000b1c8       OPM_VIEW                   000000018000c1c8     lusercontrol.obj
 0001:0000b1d0       OPM_EDIT                   000000018000c1d0     lusercontrol.obj
 0001:0000b1d8       OPM_TOPLEVEL               000000018000c1d8     lusercontrol.obj
 0001:0000b1e0       OPM_DESCR                  000000018000c1e0     lusercontrol.obj
 0001:0000b1e8       OPM_QUICKVIEW              000000018000c1e8     lusercontrol.obj
 0001:0000b1f0       OPM_PGDN                   000000018000c1f0     lusercontrol.obj
 0001:0000b1f8       OPM_COMMANDS               000000018000c1f8     lusercontrol.obj
 0001:0000b200       OPM_NONE                   000000018000c200     lusercontrol.obj
 0001:0000b208       FOSF_ACTIVE                000000018000c208     lusercontrol.obj
 0001:0000b210       FOSF_NONE                  000000018000c210     lusercontrol.obj
 0001:0000b218       PCIF_NONE                  000000018000c218     lusercontrol.obj
 0001:0000b220       FarGuid                    000000018000c220     lusercontrol.obj
 0001:0000b350       PDF_DIALOGEVENTDRAWENABLE  000000018000c350     service.obj
 0001:0000b358       PDF_PROCESSINGERROR        000000018000c358     service.obj
 0001:0000b360       PDF_FULL_TIME_RESOLUTION   000000018000c360     service.obj
 0001:0000b430       FCF_FG_4BIT                000000018000c430     service.obj
 0001:0000b438       FCF_BG_4BIT                000000018000c438     service.obj
 0001:0000b440       FCF_4BITMASK               000000018000c440     service.obj
 0001:0000b448       FCF_RAWATTR_MASK           000000018000c448     service.obj
 0001:0000b450       FCF_EXTENDEDFLAGS          000000018000c450     service.obj
 0001:0000b458       FCF_FG_BOLD                000000018000c458     service.obj
 0001:0000b460       FCF_FG_ITALIC              000000018000c460     service.obj
 0001:0000b468       FCF_FG_UNDERLINE           000000018000c468     service.obj
 0001:0000b470       FCF_STYLEMASK              000000018000c470     service.obj
 0001:0000b478       FCF_NONE                   000000018000c478     service.obj
 0001:0000b480       CDF_NONE                   000000018000c480     service.obj
 0001:0000b488       FMSG_WARNING               000000018000c488     service.obj
 0001:0000b490       FMSG_ERRORTYPE             000000018000c490     service.obj
 0001:0000b498       FMSG_KEEPBACKGROUND        000000018000c498     service.obj
 0001:0000b4a0       FMSG_LEFTALIGN             000000018000c4a0     service.obj
 0001:0000b4a8       FMSG_ALLINONE              000000018000c4a8     service.obj
 0001:0000b4b0       FMSG_MB_OK                 000000018000c4b0     service.obj
 0001:0000b4b8       FMSG_MB_OKCANCEL           000000018000c4b8     service.obj
 0001:0000b4c0       FMSG_MB_ABORTRETRYIGNORE   000000018000c4c0     service.obj
 0001:0000b4c8       FMSG_MB_YESNO              000000018000c4c8     service.obj
 0001:0000b4d0       FMSG_MB_YESNOCANCEL        000000018000c4d0     service.obj
 0001:0000b4d8       FMSG_MB_RETRYCANCEL        000000018000c4d8     service.obj
 0001:0000b4e0       FMSG_NONE                  000000018000c4e0     service.obj
 0001:0000b4e8       DIF_BOXCOLOR               000000018000c4e8     service.obj
 0001:0000b4f0       DIF_GROUP                  000000018000c4f0     service.obj
 0001:0000b4f8       DIF_LEFTTEXT               000000018000c4f8     service.obj
 0001:0000b500       DIF_MOVESELECT             000000018000c500     service.obj
 0001:0000b508       DIF_SHOWAMPERSAND          000000018000c508     service.obj
 0001:0000b510       DIF_CENTERGROUP            000000018000c510     service.obj
 0001:0000b518       DIF_NOBRACKETS             000000018000c518     service.obj
 0001:0000b520       DIF_MANUALADDHISTORY       000000018000c520     service.obj
 0001:0000b528       DIF_SEPARATOR              000000018000c528     service.obj
 0001:0000b530       DIF_SEPARATOR2             000000018000c530     service.obj
 0001:0000b538       DIF_EDITOR                 000000018000c538     service.obj
 0001:0000b540       DIF_LISTNOAMPERSAND        000000018000c540     service.obj
 0001:0000b548       DIF_LISTNOBOX              000000018000c548     service.obj
 0001:0000b550       DIF_HISTORY                000000018000c550     service.obj
 0001:0000b558       DIF_BTNNOCLOSE             000000018000c558     service.obj
 0001:0000b560       DIF_CENTERTEXT             000000018000c560     service.obj
 0001:0000b568       DIF_SEPARATORUSER          000000018000c568     service.obj
 0001:0000b570       DIF_SETSHIELD              000000018000c570     service.obj
 0001:0000b578       DIF_EDITEXPAND             000000018000c578     service.obj
 0001:0000b580       ?key@?3??far_Menu@@9@9     000000018000c580     service.obj
 0001:0000b588       DIF_DROPDOWNLIST           000000018000c588     service.obj
 0001:0000b590       DIF_USELASTHISTORY         000000018000c590     service.obj
 0001:0000b598       DIF_MASKEDIT               000000018000c598     service.obj
 0001:0000b5a0       DIF_LISTTRACKMOUSE         000000018000c5a0     service.obj
 0001:0000b5a8       DIF_LISTTRACKMOUSEINFOCUS  000000018000c5a8     service.obj
 0001:0000b5b0       DIF_SELECTONENTRY          000000018000c5b0     service.obj
 0001:0000b5b8       DIF_3STATE                 000000018000c5b8     service.obj
 0001:0000b5c0       DIF_EDITPATH               000000018000c5c0     service.obj
 0001:0000b5c8       DIF_LISTWRAPMODE           000000018000c5c8     service.obj
 0001:0000b5d0       DIF_NOAUTOCOMPLETE         000000018000c5d0     service.obj
 0001:0000b5d8       DIF_LISTAUTOHIGHLIGHT      000000018000c5d8     service.obj
 0001:0000b5e0       DIF_LISTNOCLOSE            000000018000c5e0     service.obj
 0001:0000b5e8       DIF_EDITPATHEXEC           000000018000c5e8     service.obj
 0001:0000b5f0       DIF_HIDDEN                 000000018000c5f0     service.obj
 0001:0000b5f8       DIF_READONLY               000000018000c5f8     service.obj
 0001:0000b600       DIF_NOFOCUS                000000018000c600     service.obj
 0001:0000b608       DIF_DISABLE                000000018000c608     service.obj
 0001:0000b610       DIF_DEFAULTBUTTON          000000018000c610     service.obj
 0001:0000b618       DIF_FOCUS                  000000018000c618     service.obj
 0001:0000b620       DIF_RIGHTTEXT              000000018000c620     service.obj
 0001:0000b628       DIF_WORDWRAP               000000018000c628     service.obj
 0001:0000b630       DIF_NONE                   000000018000c630     service.obj
 0001:0000b638       LIF_SELECTED               000000018000c638     service.obj
 0001:0000b640       LIF_CHECKED                000000018000c640     service.obj
 0001:0000b648       LIF_SEPARATOR              000000018000c648     service.obj
 0001:0000b650       LIF_DISABLE                000000018000c650     service.obj
 0001:0000b658       LIF_GRAYED                 000000018000c658     service.obj
 0001:0000b660       LIF_HIDDEN                 000000018000c660     service.obj
 0001:0000b668       LIF_DELETEUSERDATA         000000018000c668     service.obj
 0001:0000b670       LIF_NONE                   000000018000c670     service.obj
 0001:0000b678       LIFIND_EXACTMATCH          000000018000c678     service.obj
 0001:0000b680       LIFIND_NONE                000000018000c680     service.obj
 0001:0000b688       LINFO_SHOWNOBOX            000000018000c688     service.obj
 0001:0000b690       LINFO_AUTOHIGHLIGHT        000000018000c690     service.obj
 0001:0000b698       LINFO_REVERSEHIGHLIGHT     000000018000c698     service.obj
 0001:0000b6a0       LINFO_WRAPMODE             000000018000c6a0     service.obj
 0001:0000b6a8       LINFO_SHOWAMPERSAND        000000018000c6a8     service.obj
 0001:0000b6b0       LINFO_NONE                 000000018000c6b0     service.obj
 0001:0000b6b8       FDLG_WARNING               000000018000c6b8     service.obj
 0001:0000b6c0       FDLG_SMALLDIALOG           000000018000c6c0     service.obj
 0001:0000b6c8       FDLG_NODRAWSHADOW          000000018000c6c8     service.obj
 0001:0000b6d0       FDLG_NODRAWPANEL           000000018000c6d0     service.obj
 0001:0000b6d8       FDLG_KEEPCONSOLETITLE      000000018000c6d8     service.obj
 0001:0000b6e0       FDLG_NONMODAL              000000018000c6e0     service.obj
 0001:0000b6e8       FDLG_NONE                  000000018000c6e8     service.obj
 0001:0000b6f0       MIF_SELECTED               000000018000c6f0     service.obj
 0001:0000b6f8       MIF_CHECKED                000000018000c6f8     service.obj
 0001:0000b700       MIF_SEPARATOR              000000018000c700     service.obj
 0001:0000b708       MIF_DISABLE                000000018000c708     service.obj
 0001:0000b710       MIF_GRAYED                 000000018000c710     service.obj
 0001:0000b718       MIF_HIDDEN                 000000018000c718     service.obj
 0001:0000b720       MIF_NONE                   000000018000c720     service.obj
 0001:0000b728       FMENU_SHOWAMPERSAND        000000018000c728     service.obj
 0001:0000b730       FMENU_WRAPMODE             000000018000c730     service.obj
 0001:0000b738       FMENU_AUTOHIGHLIGHT        000000018000c738     service.obj
 0001:0000b740       FMENU_REVERSEAUTOHIGHLIGHT 000000018000c740     service.obj
 0001:0000b748       FMENU_CHANGECONSOLETITLE   000000018000c748     service.obj
 0001:0000b750       FMENU_SHOWNOBOX            000000018000c750     service.obj
 0001:0000b758       FMENU_SHOWSHORTBOX         000000018000c758     service.obj
 0001:0000b760       FMENU_SHOWSINGLEBOX        000000018000c760     service.obj
 0001:0000b768       FMENU_NODRAWSHADOW         000000018000c768     service.obj
 0001:0000b770       FMENU_NONE                 000000018000c770     service.obj
 0001:0000b778       PPIF_SELECTED              000000018000c778     service.obj
 0001:0000b780       PPIF_PROCESSDESCR          000000018000c780     service.obj
 0001:0000b788       PPIF_NONE                  000000018000c788     service.obj
 0001:0000b790       PFLAGS_SHOWHIDDEN          000000018000c790     service.obj
 0001:0000b798       PFLAGS_HIGHLIGHT           000000018000c798     service.obj
 0001:0000b7a0       PFLAGS_REVERSESORTORDER    000000018000c7a0     service.obj
 0001:0000b7a8       PFLAGS_USESORTGROUPS       000000018000c7a8     service.obj
 0001:0000b7b0       PFLAGS_SELECTEDFIRST       000000018000c7b0     service.obj
 0001:0000b7b8       PFLAGS_REALNAMES           000000018000c7b8     service.obj
 0001:0000b7c0       PFLAGS_PANELLEFT           000000018000c7c0     service.obj
 0001:0000b7c8       PFLAGS_DIRECTORIESFIRST    000000018000c7c8     service.obj
 0001:0000b7d0       PFLAGS_USECRC32            000000018000c7d0     service.obj
 0001:0000b7d8       PFLAGS_PLUGIN              000000018000c7d8     service.obj
 0001:0000b7e0       PFLAGS_VISIBLE             000000018000c7e0     service.obj
 0001:0000b7e8       PFLAGS_FOCUS               000000018000c7e8     service.obj
 0001:0000b7f0       PFLAGS_ALTERNATIVENAMES    000000018000c7f0     service.obj
 0001:0000b7f8       PFLAGS_SHORTCUT            000000018000c7f8     service.obj
 0001:0000b800       PFLAGS_NONE                000000018000c800     service.obj
 0001:0000b808       VF_NONMODAL                000000018000c808     service.obj
 0001:0000b810       VF_DELETEONCLOSE           000000018000c810     service.obj
 0001:0000b818       VF_ENABLE_F6               000000018000c818     service.obj
 0001:0000b820       VF_DISABLEHISTORY          000000018000c820     service.obj
 0001:0000b828       VF_IMMEDIATERETURN         000000018000c828     service.obj
 0001:0000b830       VF_DELETEONLYFILEONCLOSE   000000018000c830     service.obj
 0001:0000b838       VF_NONE                    000000018000c838     service.obj
 0001:0000b840       EF_NONMODAL                000000018000c840     service.obj
 0001:0000b848       EF_CREATENEW               000000018000c848     service.obj
 0001:0000b850       EF_ENABLE_F6               000000018000c850     service.obj
 0001:0000b858       EF_DISABLEHISTORY          000000018000c858     service.obj
 0001:0000b860       EF_DELETEONCLOSE           000000018000c860     service.obj
 0001:0000b868       EF_IMMEDIATERETURN         000000018000c868     service.obj
 0001:0000b870       EF_DELETEONLYFILEONCLOSE   000000018000c870     service.obj
 0001:0000b878       EF_LOCKED                  000000018000c878     service.obj
 0001:0000b880       EF_DISABLESAVEPOS          000000018000c880     service.obj
 0001:0000b888       EF_OPENMODE_MASK           000000018000c888     service.obj
 0001:0000b890       EF_OPENMODE_QUERY          000000018000c890     service.obj
 0001:0000b898       EF_OPENMODE_NEWIFOPEN      000000018000c898     service.obj
 0001:0000b8a0       EF_OPENMODE_USEEXISTING    000000018000c8a0     service.obj
 0001:0000b8a8       EF_OPENMODE_BREAKIFOPEN    000000018000c8a8     service.obj
 0001:0000b8b0       EF_OPENMODE_RELOADIFOPEN   000000018000c8b0     service.obj
 0001:0000b8b8       EN_NONE                    000000018000c8b8     service.obj
 0001:0000b8c0       FHELP_NOSHOWERROR          000000018000c8c0     service.obj
 0001:0000b8c8       FHELP_SELFHELP             000000018000c8c8     service.obj
 0001:0000b8d0       FHELP_FARHELP              000000018000c8d0     service.obj
 0001:0000b8d8       FHELP_CUSTOMFILE           000000018000c8d8     service.obj
 0001:0000b8e0       FHELP_CUSTOMPATH           000000018000c8e0     service.obj
 0001:0000b8e8       FHELP_GUID                 000000018000c8e8     service.obj
 0001:0000b8f0       FHELP_USECONTENTS          000000018000c8f0     service.obj
 0001:0000b8f8       FHELP_NONE                 000000018000c8f8     service.obj
 0001:0000b900       KMFLAGS_SILENTCHECK        000000018000c900     service.obj
 0001:0000b908       KMFLAGS_NOSENDKEYSTOPLUGINS 000000018000c908     service.obj
 0001:0000b910       KMFLAGS_ENABLEOUTPUT       000000018000c910     service.obj
 0001:0000b918       KMFLAGS_LANGMASK           000000018000c918     service.obj
 0001:0000b920       KMFLAGS_LUA                000000018000c920     service.obj
 0001:0000b928       KMFLAGS_MOONSCRIPT         000000018000c928     service.obj
 0001:0000b930       KMFLAGS_NONE               000000018000c930     service.obj
 0001:0000b938       AKMFLAGS_NONE              000000018000c938     service.obj
 0001:0000b940       FSETCLR_REDRAW             000000018000c940     service.obj
 0001:0000b948       FSETCLR_NONE               000000018000c948     service.obj
 0001:0000b950       WIF_MODIFIED               000000018000c950     service.obj
 0001:0000b958       WIF_CURRENT                000000018000c958     service.obj
 0001:0000b960       WIF_MODAL                  000000018000c960     service.obj
 0001:0000b968       WIF_NONE                   000000018000c968     service.obj
 0001:0000b970       VOPT_SAVEFILEPOSITION      000000018000c970     service.obj
 0001:0000b978       VOPT_AUTODETECTCODEPAGE    000000018000c978     service.obj
 0001:0000b980       VOPT_SHOWTITLEBAR          000000018000c980     service.obj
 0001:0000b988       VOPT_SHOWKEYBAR            000000018000c988     service.obj
 0001:0000b990       VOPT_SHOWSCROLLBAR         000000018000c990     service.obj
 0001:0000b998       VOPT_QUICKVIEW             000000018000c998     service.obj
 0001:0000b9a0       VOPT_NONE                  000000018000c9a0     service.obj
 0001:0000b9a8       VSMFL_REDRAW               000000018000c9a8     service.obj
 0001:0000b9b0       VSMFL_NONE                 000000018000c9b0     service.obj
 0001:0000b9b8       VSP_NOREDRAW               000000018000c9b8     service.obj
 0001:0000b9c0       VSP_PERCENT                000000018000c9c0     service.obj
 0001:0000b9c8       VSP_RELATIVE               000000018000c9c8     service.obj
 0001:0000b9d0       VSP_NORETNEWPOS            000000018000c9d0     service.obj
 0001:0000b9d8       VSP_NONE                   000000018000c9d8     service.obj
 0001:0000b9e0       VMF_WRAP                   000000018000c9e0     service.obj
 0001:0000b9e8       VMF_WORDWRAP               000000018000c9e8     service.obj
 0001:0000b9f0       VMF_NONE                   000000018000c9f0     service.obj
 0001:0000b9f8       ECF_TABMARKFIRST           000000018000c9f8     service.obj
 0001:0000ba00       ECF_TABMARKCURRENT         000000018000ca00     service.obj
 0001:0000ba08       ECF_AUTODELETE             000000018000ca08     service.obj
 0001:0000ba10       ECF_NONE                   000000018000ca10     service.obj
 0001:0000ba18       FIB_ENABLEEMPTY            000000018000ca18     service.obj
 0001:0000ba20       FIB_PASSWORD               000000018000ca20     service.obj
 0001:0000ba28       FIB_EXPANDENV              000000018000ca28     service.obj
 0001:0000ba30       FIB_NOUSELASTHISTORY       000000018000ca30     service.obj
 0001:0000ba38       FIB_BUTTONS                000000018000ca38     service.obj
 0001:0000ba40       FIB_NOAMPERSAND            000000018000ca40     service.obj
 0001:0000ba48       FIB_EDITPATH               000000018000ca48     service.obj
 0001:0000ba50       FIB_EDITPATHEXEC           000000018000ca50     service.obj
 0001:0000ba58       FIB_NONE                   000000018000ca58     service.obj
 0001:0000ba60       FPF_LOADED                 000000018000ca60     service.obj
 0001:0000ba68       FPF_ANSI                   000000018000ca68     service.obj
 0001:0000ba70       FPF_NONE                   000000018000ca70     service.obj
 0001:0000ba78       ?C@?3??far_InputRecordToName@@9@9 000000018000ca78     service.obj
 0001:0000ba80       ?A@?3??far_InputRecordToName@@9@9 000000018000ca80     service.obj
 0001:0000ba88       ?S@?3??far_InputRecordToName@@9@9 000000018000ca88     service.obj
 0001:0000ba90       PN_CMPNAME                 000000018000ca90     service.obj
 0001:0000ba98       PN_CMPNAMELIST             000000018000ca98     service.obj
 0001:0000baa0       PN_GENERATENAME            000000018000caa0     service.obj
 0001:0000baa8       PN_CHECKMASK               000000018000caa8     service.obj
 0001:0000bab0       PN_SKIPPATH                000000018000cab0     service.obj
 0001:0000bab8       PN_SHOWERRORMESSAGE        000000018000cab8     service.obj
 0001:0000bac0       PN_NONE                    000000018000cac0     service.obj
 0001:0000bac8       XLAT_SWITCHKEYBLAYOUT      000000018000cac8     service.obj
 0001:0000bad0       XLAT_SWITCHKEYBBEEP        000000018000cad0     service.obj
 0001:0000bad8       XLAT_USEKEYBLAYOUTNAME     000000018000cad8     service.obj
 0001:0000bae0       XLAT_CONVERTALLCMDLINE     000000018000cae0     service.obj
 0001:0000bae8       XLAT_NONE                  000000018000cae8     service.obj
 0001:0000baf0       FRS_RETUPDIR               000000018000caf0     service.obj
 0001:0000baf8       FRS_RECUR                  000000018000caf8     service.obj
 0001:0000bb00       FRS_SCANSYMLINK            000000018000cb00     service.obj
 0001:0000bb08       FRS_NONE                   000000018000cb08     service.obj
 0001:0000bb10       MLF_SHOWERRMSG             000000018000cb10     service.obj
 0001:0000bb18       MLF_DONOTUPDATEPANEL       000000018000cb18     service.obj
 0001:0000bb20       MLF_HOLDTARGET             000000018000cb20     service.obj
 0001:0000bb28       MLF_NONE                   000000018000cb28     service.obj
 0001:0000bb30       FFFS_COMMAS                000000018000cb30     service.obj
 0001:0000bb38       FFFS_FLOATSIZE             000000018000cb38     service.obj
 0001:0000bb40       FFFS_SHOWBYTESINDEX        000000018000cb40     service.obj
 0001:0000bb48       FFFS_ECONOMIC              000000018000cb48     service.obj
 0001:0000bb50       FFFS_THOUSAND              000000018000cb50     service.obj
 0001:0000bb58       FFFS_MINSIZEINDEX          000000018000cb58     service.obj
 0001:0000bb60       FFFS_MINSIZEINDEX_MASK     000000018000cb60     service.obj
 0001:0000bb68       FFFS_NONE                  000000018000cb68     service.obj
 0001:0000bb70       PF_PRELOAD                 000000018000cb70     service.obj
 0001:0000bb78       PF_DISABLEPANELS           000000018000cb78     service.obj
 0001:0000bb80       PF_EDITOR                  000000018000cb80     service.obj
 0001:0000bb88       PF_VIEWER                  000000018000cb88     service.obj
 0001:0000bb90       PF_FULLCMDLINE             000000018000cb90     service.obj
 0001:0000bb98       PF_DIALOG                  000000018000cb98     service.obj
 0001:0000bba0       PF_NONE                    000000018000cba0     service.obj
 0001:0000bba8       IPLFLAGS_SEPARATOR         000000018000cba8     service.obj
 0001:0000bbb0       IPLFLAGS_NONE              000000018000cbb0     service.obj
 0001:0000bbb8       PMFLAGS_FULLSCREEN         000000018000cbb8     service.obj
 0001:0000bbc0       PMFLAGS_DETAILEDSTATUS     000000018000cbc0     service.obj
 0001:0000bbc8       PMFLAGS_ALIGNEXTENSIONS    000000018000cbc8     service.obj
 0001:0000bbd0       PMFLAGS_CASECONVERSION     000000018000cbd0     service.obj
 0001:0000bbd8       PMFLAGS_NONE               000000018000cbd8     service.obj
 0001:0000bbe0       OPIF_DISABLEFILTER         000000018000cbe0     service.obj
 0001:0000bbe8       OPIF_DISABLESORTGROUPS     000000018000cbe8     service.obj
 0001:0000bbf0       OPIF_DISABLEHIGHLIGHTING   000000018000cbf0     service.obj
 0001:0000bbf8       OPIF_ADDDOTS               000000018000cbf8     service.obj
 0001:0000bc00       OPIF_RAWSELECTION          000000018000cc00     service.obj
 0001:0000bc08       OPIF_REALNAMES             000000018000cc08     service.obj
 0001:0000bc10       OPIF_SHOWNAMESONLY         000000018000cc10     service.obj
 0001:0000bc18       OPIF_SHOWRIGHTALIGNNAMES   000000018000cc18     service.obj
 0001:0000bc20       OPIF_SHOWPRESERVECASE      000000018000cc20     service.obj
 0001:0000bc28       OPIF_COMPAREFATTIME        000000018000cc28     service.obj
 0001:0000bc30       OPIF_EXTERNALGET           000000018000cc30     service.obj
 0001:0000bc38       OPIF_EXTERNALPUT           000000018000cc38     service.obj
 0001:0000bc40       OPIF_EXTERNALDELETE        000000018000cc40     service.obj
 0001:0000bc48       OPIF_EXTERNALMKDIR         000000018000cc48     service.obj
 0001:0000bc50       OPIF_USEATTRHIGHLIGHTING   000000018000cc50     service.obj
 0001:0000bc58       OPIF_USECRC32              000000018000cc58     service.obj
 0001:0000bc60       OPIF_USEFREESIZE           000000018000cc60     service.obj
 0001:0000bc68       OPIF_SHORTCUT              000000018000cc68     service.obj
 0001:0000bc70       OPIF_NONE                  000000018000cc70     service.obj
 0001:0000bc78       OPM_SILENT                 000000018000cc78     service.obj
 0001:0000bc80       OPM_FIND                   000000018000cc80     service.obj
 0001:0000bc88       OPM_VIEW                   000000018000cc88     service.obj
 0001:0000bc90       OPM_EDIT                   000000018000cc90     service.obj
 0001:0000bc98       OPM_TOPLEVEL               000000018000cc98     service.obj
 0001:0000bca0       OPM_DESCR                  000000018000cca0     service.obj
 0001:0000bca8       OPM_QUICKVIEW              000000018000cca8     service.obj
 0001:0000bcb0       OPM_PGDN                   000000018000ccb0     service.obj
 0001:0000bcb8       OPM_COMMANDS               000000018000ccb8     service.obj
 0001:0000bcc0       OPM_NONE                   000000018000ccc0     service.obj
 0001:0000bcc8       FOSF_ACTIVE                000000018000ccc8     service.obj
 0001:0000bcd0       FOSF_NONE                  000000018000ccd0     service.obj
 0001:0000bcd8       PCIF_NONE                  000000018000ccd8     service.obj
 0001:0000bce0       FarGuid                    000000018000cce0     service.obj
 0001:0000bcf0       ?FarGuid@?1??far_CreateSettings@@9@9 000000018000ccf0     service.obj
 0001:0000cae0       lualibs                    000000018000dae0     service.obj
 0001:0000cbb0       lualibs_extra              000000018000dbb0     service.obj
 0001:0000ea70       uniclib                    000000018000fa70     slnunico.obj
 0001:0000eea0       fnames                     000000018000fea0     uliolib51.obj
 0001:0000eeb0       ?mode@?1??f_seek@@9@9      000000018000feb0     uliolib51.obj
 0001:0000eec0       ?modenames@?1??f_seek@@9@9 000000018000fec0     uliolib51.obj
 0001:0000eee0       ?mode@?1??f_setvbuf@@9@9   000000018000fee0     uliolib51.obj
 0001:0000eef0       ?modenames@?1??f_setvbuf@@9@9 000000018000fef0     uliolib51.obj
 0001:0000ef10       iolib                      000000018000ff10     uliolib51.obj
 0001:0000efd0       flib                       000000018000ffd0     uliolib51.obj
 0001:0000f290       sentinel_                  0000000180010290     uloadlib51.obj
 0001:0000f298       pk_funcs                   0000000180010298     uloadlib51.obj
 0001:0000f2c8       ll_funcs                   00000001800102c8     uloadlib51.obj
 0001:0000f2f8       loaders                    00000001800102f8     uloadlib51.obj
 0001:0000fc60       FCF_FG_4BIT                0000000180010c60     util.obj
 0001:0000fc68       FCF_BG_4BIT                0000000180010c68     util.obj
 0001:0000fc70       FCF_4BITMASK               0000000180010c70     util.obj
 0001:0000fc78       FCF_RAWATTR_MASK           0000000180010c78     util.obj
 0001:0000fc80       FCF_EXTENDEDFLAGS          0000000180010c80     util.obj
 0001:0000fc88       FCF_FG_BOLD                0000000180010c88     util.obj
 0001:0000fc90       FCF_FG_ITALIC              0000000180010c90     util.obj
 0001:0000fc98       FCF_FG_UNDERLINE           0000000180010c98     util.obj
 0001:0000fca0       FCF_STYLEMASK              0000000180010ca0     util.obj
 0001:0000fca8       FCF_NONE                   0000000180010ca8     util.obj
 0001:0000fcb0       CDF_NONE                   0000000180010cb0     util.obj
 0001:0000fcb8       FMSG_WARNING               0000000180010cb8     util.obj
 0001:0000fcc0       FMSG_ERRORTYPE             0000000180010cc0     util.obj
 0001:0000fcc8       FMSG_KEEPBACKGROUND        0000000180010cc8     util.obj
 0001:0000fcd0       FMSG_LEFTALIGN             0000000180010cd0     util.obj
 0001:0000fcd8       FMSG_ALLINONE              0000000180010cd8     util.obj
 0001:0000fce0       FMSG_MB_OK                 0000000180010ce0     util.obj
 0001:0000fce8       FMSG_MB_OKCANCEL           0000000180010ce8     util.obj
 0001:0000fcf0       FMSG_MB_ABORTRETRYIGNORE   0000000180010cf0     util.obj
 0001:0000fcf8       FMSG_MB_YESNO              0000000180010cf8     util.obj
 0001:0000fd00       FMSG_MB_YESNOCANCEL        0000000180010d00     util.obj
 0001:0000fd08       FMSG_MB_RETRYCANCEL        0000000180010d08     util.obj
 0001:0000fd10       FMSG_NONE                  0000000180010d10     util.obj
 0001:0000fd18       DIF_BOXCOLOR               0000000180010d18     util.obj
 0001:0000fd20       DIF_GROUP                  0000000180010d20     util.obj
 0001:0000fd28       DIF_LEFTTEXT               0000000180010d28     util.obj
 0001:0000fd30       DIF_MOVESELECT             0000000180010d30     util.obj
 0001:0000fd38       DIF_SHOWAMPERSAND          0000000180010d38     util.obj
 0001:0000fd40       DIF_CENTERGROUP            0000000180010d40     util.obj
 0001:0000fd48       DIF_NOBRACKETS             0000000180010d48     util.obj
 0001:0000fd50       DIF_MANUALADDHISTORY       0000000180010d50     util.obj
 0001:0000fd58       DIF_SEPARATOR              0000000180010d58     util.obj
 0001:0000fd60       DIF_SEPARATOR2             0000000180010d60     util.obj
 0001:0000fd68       DIF_EDITOR                 0000000180010d68     util.obj
 0001:0000fd70       DIF_LISTNOAMPERSAND        0000000180010d70     util.obj
 0001:0000fd78       DIF_LISTNOBOX              0000000180010d78     util.obj
 0001:0000fd80       DIF_HISTORY                0000000180010d80     util.obj
 0001:0000fd88       DIF_BTNNOCLOSE             0000000180010d88     util.obj
 0001:0000fd90       DIF_CENTERTEXT             0000000180010d90     util.obj
 0001:0000fd98       DIF_SEPARATORUSER          0000000180010d98     util.obj
 0001:0000fda0       DIF_SETSHIELD              0000000180010da0     util.obj
 0001:0000fda8       DIF_EDITEXPAND             0000000180010da8     util.obj
 0001:0000fdb0       DIF_DROPDOWNLIST           0000000180010db0     util.obj
 0001:0000fdb8       DIF_USELASTHISTORY         0000000180010db8     util.obj
 0001:0000fdc0       DIF_MASKEDIT               0000000180010dc0     util.obj
 0001:0000fdc8       DIF_LISTTRACKMOUSE         0000000180010dc8     util.obj
 0001:0000fdd0       DIF_LISTTRACKMOUSEINFOCUS  0000000180010dd0     util.obj
 0001:0000fdd8       DIF_SELECTONENTRY          0000000180010dd8     util.obj
 0001:0000fde0       DIF_3STATE                 0000000180010de0     util.obj
 0001:0000fde8       DIF_EDITPATH               0000000180010de8     util.obj
 0001:0000fdf0       DIF_LISTWRAPMODE           0000000180010df0     util.obj
 0001:0000fdf8       DIF_NOAUTOCOMPLETE         0000000180010df8     util.obj
 0001:0000fe00       DIF_LISTAUTOHIGHLIGHT      0000000180010e00     util.obj
 0001:0000fe08       DIF_LISTNOCLOSE            0000000180010e08     util.obj
 0001:0000fe10       DIF_EDITPATHEXEC           0000000180010e10     util.obj
 0001:0000fe18       DIF_HIDDEN                 0000000180010e18     util.obj
 0001:0000fe20       DIF_READONLY               0000000180010e20     util.obj
 0001:0000fe28       DIF_NOFOCUS                0000000180010e28     util.obj
 0001:0000fe30       DIF_DISABLE                0000000180010e30     util.obj
 0001:0000fe38       DIF_DEFAULTBUTTON          0000000180010e38     util.obj
 0001:0000fe40       DIF_FOCUS                  0000000180010e40     util.obj
 0001:0000fe48       DIF_RIGHTTEXT              0000000180010e48     util.obj
 0001:0000fe50       DIF_WORDWRAP               0000000180010e50     util.obj
 0001:0000fe58       DIF_NONE                   0000000180010e58     util.obj
 0001:0000fe60       LIF_SELECTED               0000000180010e60     util.obj
 0001:0000fe68       LIF_CHECKED                0000000180010e68     util.obj
 0001:0000fe70       LIF_SEPARATOR              0000000180010e70     util.obj
 0001:0000fe78       LIF_DISABLE                0000000180010e78     util.obj
 0001:0000fe80       LIF_GRAYED                 0000000180010e80     util.obj
 0001:0000fe88       LIF_HIDDEN                 0000000180010e88     util.obj
 0001:0000fe90       LIF_DELETEUSERDATA         0000000180010e90     util.obj
 0001:0000fe98       LIF_NONE                   0000000180010e98     util.obj
 0001:0000fea0       LIFIND_EXACTMATCH          0000000180010ea0     util.obj
 0001:0000fea8       LIFIND_NONE                0000000180010ea8     util.obj
 0001:0000feb0       LINFO_SHOWNOBOX            0000000180010eb0     util.obj
 0001:0000feb8       LINFO_AUTOHIGHLIGHT        0000000180010eb8     util.obj
 0001:0000fec0       LINFO_REVERSEHIGHLIGHT     0000000180010ec0     util.obj
 0001:0000fec8       LINFO_WRAPMODE             0000000180010ec8     util.obj
 0001:0000fed0       LINFO_SHOWAMPERSAND        0000000180010ed0     util.obj
 0001:0000fed8       LINFO_NONE                 0000000180010ed8     util.obj
 0001:0000fee0       FDLG_WARNING               0000000180010ee0     util.obj
 0001:0000fee8       FDLG_SMALLDIALOG           0000000180010ee8     util.obj
 0001:0000fef0       FDLG_NODRAWSHADOW          0000000180010ef0     util.obj
 0001:0000fef8       FDLG_NODRAWPANEL           0000000180010ef8     util.obj
 0001:0000ff00       FDLG_KEEPCONSOLETITLE      0000000180010f00     util.obj
 0001:0000ff08       FDLG_NONMODAL              0000000180010f08     util.obj
 0001:0000ff10       FDLG_NONE                  0000000180010f10     util.obj
 0001:0000ff18       MIF_SELECTED               0000000180010f18     util.obj
 0001:0000ff20       MIF_CHECKED                0000000180010f20     util.obj
 0001:0000ff28       MIF_SEPARATOR              0000000180010f28     util.obj
 0001:0000ff30       MIF_DISABLE                0000000180010f30     util.obj
 0001:0000ff38       MIF_GRAYED                 0000000180010f38     util.obj
 0001:0000ff40       MIF_HIDDEN                 0000000180010f40     util.obj
 0001:0000ff48       MIF_NONE                   0000000180010f48     util.obj
 0001:0000ff50       FMENU_SHOWAMPERSAND        0000000180010f50     util.obj
 0001:0000ff58       FMENU_WRAPMODE             0000000180010f58     util.obj
 0001:0000ff60       FMENU_AUTOHIGHLIGHT        0000000180010f60     util.obj
 0001:0000ff68       FMENU_REVERSEAUTOHIGHLIGHT 0000000180010f68     util.obj
 0001:0000ff70       FMENU_CHANGECONSOLETITLE   0000000180010f70     util.obj
 0001:0000ff78       FMENU_SHOWNOBOX            0000000180010f78     util.obj
 0001:0000ff80       FMENU_SHOWSHORTBOX         0000000180010f80     util.obj
 0001:0000ff88       FMENU_SHOWSINGLEBOX        0000000180010f88     util.obj
 0001:0000ff90       FMENU_NODRAWSHADOW         0000000180010f90     util.obj
 0001:0000ff98       FMENU_NONE                 0000000180010f98     util.obj
 0001:0000ffa0       PPIF_SELECTED              0000000180010fa0     util.obj
 0001:0000ffa8       PPIF_PROCESSDESCR          0000000180010fa8     util.obj
 0001:0000ffb0       PPIF_NONE                  0000000180010fb0     util.obj
 0001:0000ffb8       PFLAGS_SHOWHIDDEN          0000000180010fb8     util.obj
 0001:0000ffc0       PFLAGS_HIGHLIGHT           0000000180010fc0     util.obj
 0001:0000ffc8       PFLAGS_REVERSESORTORDER    0000000180010fc8     util.obj
 0001:0000ffd0       PFLAGS_USESORTGROUPS       0000000180010fd0     util.obj
 0001:0000ffd8       PFLAGS_SELECTEDFIRST       0000000180010fd8     util.obj
 0001:0000ffe0       PFLAGS_REALNAMES           0000000180010fe0     util.obj
 0001:0000ffe8       PFLAGS_PANELLEFT           0000000180010fe8     util.obj
 0001:0000fff0       PFLAGS_DIRECTORIESFIRST    0000000180010ff0     util.obj
 0001:0000fff8       PFLAGS_USECRC32            0000000180010ff8     util.obj
 0001:00010000       PFLAGS_PLUGIN              0000000180011000     util.obj
 0001:00010008       PFLAGS_VISIBLE             0000000180011008     util.obj
 0001:00010010       PFLAGS_FOCUS               0000000180011010     util.obj
 0001:00010018       PFLAGS_ALTERNATIVENAMES    0000000180011018     util.obj
 0001:00010020       PFLAGS_SHORTCUT            0000000180011020     util.obj
 0001:00010028       PFLAGS_NONE                0000000180011028     util.obj
 0001:00010030       VF_NONMODAL                0000000180011030     util.obj
 0001:00010038       VF_DELETEONCLOSE           0000000180011038     util.obj
 0001:00010040       VF_ENABLE_F6               0000000180011040     util.obj
 0001:00010048       VF_DISABLEHISTORY          0000000180011048     util.obj
 0001:00010050       VF_IMMEDIATERETURN         0000000180011050     util.obj
 0001:00010058       VF_DELETEONLYFILEONCLOSE   0000000180011058     util.obj
 0001:00010060       VF_NONE                    0000000180011060     util.obj
 0001:00010068       EF_NONMODAL                0000000180011068     util.obj
 0001:00010070       EF_CREATENEW               0000000180011070     util.obj
 0001:00010078       EF_ENABLE_F6               0000000180011078     util.obj
 0001:00010080       EF_DISABLEHISTORY          0000000180011080     util.obj
 0001:00010088       EF_DELETEONCLOSE           0000000180011088     util.obj
 0001:00010090       EF_IMMEDIATERETURN         0000000180011090     util.obj
 0001:00010098       EF_DELETEONLYFILEONCLOSE   0000000180011098     util.obj
 0001:000100a0       EF_LOCKED                  00000001800110a0     util.obj
 0001:000100a8       EF_DISABLESAVEPOS          00000001800110a8     util.obj
 0001:000100b0       EF_OPENMODE_MASK           00000001800110b0     util.obj
 0001:000100b8       EF_OPENMODE_QUERY          00000001800110b8     util.obj
 0001:000100c0       EF_OPENMODE_NEWIFOPEN      00000001800110c0     util.obj
 0001:000100c8       EF_OPENMODE_USEEXISTING    00000001800110c8     util.obj
 0001:000100d0       EF_OPENMODE_BREAKIFOPEN    00000001800110d0     util.obj
 0001:000100d8       EF_OPENMODE_RELOADIFOPEN   00000001800110d8     util.obj
 0001:000100e0       EN_NONE                    00000001800110e0     util.obj
 0001:000100e8       FHELP_NOSHOWERROR          00000001800110e8     util.obj
 0001:000100f0       FHELP_SELFHELP             00000001800110f0     util.obj
 0001:000100f8       FHELP_FARHELP              00000001800110f8     util.obj
 0001:00010100       FHELP_CUSTOMFILE           0000000180011100     util.obj
 0001:00010108       FHELP_CUSTOMPATH           0000000180011108     util.obj
 0001:00010110       FHELP_GUID                 0000000180011110     util.obj
 0001:00010118       FHELP_USECONTENTS          0000000180011118     util.obj
 0001:00010120       FHELP_NONE                 0000000180011120     util.obj
 0001:00010128       KMFLAGS_SILENTCHECK        0000000180011128     util.obj
 0001:00010130       KMFLAGS_NOSENDKEYSTOPLUGINS 0000000180011130     util.obj
 0001:00010138       KMFLAGS_ENABLEOUTPUT       0000000180011138     util.obj
 0001:00010140       KMFLAGS_LANGMASK           0000000180011140     util.obj
 0001:00010148       KMFLAGS_LUA                0000000180011148     util.obj
 0001:00010150       KMFLAGS_MOONSCRIPT         0000000180011150     util.obj
 0001:00010158       KMFLAGS_NONE               0000000180011158     util.obj
 0001:00010160       AKMFLAGS_NONE              0000000180011160     util.obj
 0001:00010168       FSETCLR_REDRAW             0000000180011168     util.obj
 0001:00010170       FSETCLR_NONE               0000000180011170     util.obj
 0001:00010178       WIF_MODIFIED               0000000180011178     util.obj
 0001:00010180       WIF_CURRENT                0000000180011180     util.obj
 0001:00010188       WIF_MODAL                  0000000180011188     util.obj
 0001:00010190       WIF_NONE                   0000000180011190     util.obj
 0001:00010198       VOPT_SAVEFILEPOSITION      0000000180011198     util.obj
 0001:000101a0       VOPT_AUTODETECTCODEPAGE    00000001800111a0     util.obj
 0001:000101a8       VOPT_SHOWTITLEBAR          00000001800111a8     util.obj
 0001:000101b0       VOPT_SHOWKEYBAR            00000001800111b0     util.obj
 0001:000101b8       VOPT_SHOWSCROLLBAR         00000001800111b8     util.obj
 0001:000101c0       VOPT_QUICKVIEW             00000001800111c0     util.obj
 0001:000101c8       VOPT_NONE                  00000001800111c8     util.obj
 0001:000101d0       VSMFL_REDRAW               00000001800111d0     util.obj
 0001:000101d8       VSMFL_NONE                 00000001800111d8     util.obj
 0001:000101e0       VSP_NOREDRAW               00000001800111e0     util.obj
 0001:000101e8       VSP_PERCENT                00000001800111e8     util.obj
 0001:000101f0       VSP_RELATIVE               00000001800111f0     util.obj
 0001:000101f8       VSP_NORETNEWPOS            00000001800111f8     util.obj
 0001:00010200       VSP_NONE                   0000000180011200     util.obj
 0001:00010208       VMF_WRAP                   0000000180011208     util.obj
 0001:00010210       VMF_WORDWRAP               0000000180011210     util.obj
 0001:00010218       VMF_NONE                   0000000180011218     util.obj
 0001:00010220       ECF_TABMARKFIRST           0000000180011220     util.obj
 0001:00010228       ECF_TABMARKCURRENT         0000000180011228     util.obj
 0001:00010230       ECF_AUTODELETE             0000000180011230     util.obj
 0001:00010238       ECF_NONE                   0000000180011238     util.obj
 0001:00010240       FIB_ENABLEEMPTY            0000000180011240     util.obj
 0001:00010248       FIB_PASSWORD               0000000180011248     util.obj
 0001:00010250       FIB_EXPANDENV              0000000180011250     util.obj
 0001:00010258       FIB_NOUSELASTHISTORY       0000000180011258     util.obj
 0001:00010260       FIB_BUTTONS                0000000180011260     util.obj
 0001:00010268       FIB_NOAMPERSAND            0000000180011268     util.obj
 0001:00010270       FIB_EDITPATH               0000000180011270     util.obj
 0001:00010278       FIB_EDITPATHEXEC           0000000180011278     util.obj
 0001:00010280       FIB_NONE                   0000000180011280     util.obj
 0001:00010288       FPF_LOADED                 0000000180011288     util.obj
 0001:00010290       FPF_ANSI                   0000000180011290     util.obj
 0001:00010298       FPF_NONE                   0000000180011298     util.obj
 0001:000102a0       PN_CMPNAME                 00000001800112a0     util.obj
 0001:000102a8       PN_CMPNAMELIST             00000001800112a8     util.obj
 0001:000102b0       PN_GENERATENAME            00000001800112b0     util.obj
 0001:000102b8       PN_CHECKMASK               00000001800112b8     util.obj
 0001:000102c0       PN_SKIPPATH                00000001800112c0     util.obj
 0001:000102c8       PN_SHOWERRORMESSAGE        00000001800112c8     util.obj
 0001:000102d0       PN_NONE                    00000001800112d0     util.obj
 0001:000102d8       XLAT_SWITCHKEYBLAYOUT      00000001800112d8     util.obj
 0001:000102e0       XLAT_SWITCHKEYBBEEP        00000001800112e0     util.obj
 0001:000102e8       XLAT_USEKEYBLAYOUTNAME     00000001800112e8     util.obj
 0001:000102f0       XLAT_CONVERTALLCMDLINE     00000001800112f0     util.obj
 0001:000102f8       XLAT_NONE                  00000001800112f8     util.obj
 0001:00010300       FRS_RETUPDIR               0000000180011300     util.obj
 0001:00010308       FRS_RECUR                  0000000180011308     util.obj
 0001:00010310       FRS_SCANSYMLINK            0000000180011310     util.obj
 0001:00010318       FRS_NONE                   0000000180011318     util.obj
 0001:00010320       MLF_SHOWERRMSG             0000000180011320     util.obj
 0001:00010328       MLF_DONOTUPDATEPANEL       0000000180011328     util.obj
 0001:00010330       MLF_HOLDTARGET             0000000180011330     util.obj
 0001:00010338       MLF_NONE                   0000000180011338     util.obj
 0001:00010340       FFFS_COMMAS                0000000180011340     util.obj
 0001:00010348       FFFS_FLOATSIZE             0000000180011348     util.obj
 0001:00010350       FFFS_SHOWBYTESINDEX        0000000180011350     util.obj
 0001:00010358       FFFS_ECONOMIC              0000000180011358     util.obj
 0001:00010360       FFFS_THOUSAND              0000000180011360     util.obj
 0001:00010368       FFFS_MINSIZEINDEX          0000000180011368     util.obj
 0001:00010370       FFFS_MINSIZEINDEX_MASK     0000000180011370     util.obj
 0001:00010378       FFFS_NONE                  0000000180011378     util.obj
 0001:00010380       PF_PRELOAD                 0000000180011380     util.obj
 0001:00010388       PF_DISABLEPANELS           0000000180011388     util.obj
 0001:00010390       PF_EDITOR                  0000000180011390     util.obj
 0001:00010398       PF_VIEWER                  0000000180011398     util.obj
 0001:000103a0       PF_FULLCMDLINE             00000001800113a0     util.obj
 0001:000103a8       PF_DIALOG                  00000001800113a8     util.obj
 0001:000103b0       PF_NONE                    00000001800113b0     util.obj
 0001:000103b8       IPLFLAGS_SEPARATOR         00000001800113b8     util.obj
 0001:000103c0       IPLFLAGS_NONE              00000001800113c0     util.obj
 0001:000103c8       PMFLAGS_FULLSCREEN         00000001800113c8     util.obj
 0001:000103d0       PMFLAGS_DETAILEDSTATUS     00000001800113d0     util.obj
 0001:000103d8       PMFLAGS_ALIGNEXTENSIONS    00000001800113d8     util.obj
 0001:000103e0       PMFLAGS_CASECONVERSION     00000001800113e0     util.obj
 0001:000103e8       PMFLAGS_NONE               00000001800113e8     util.obj
 0001:000103f0       OPIF_DISABLEFILTER         00000001800113f0     util.obj
 0001:000103f8       OPIF_DISABLESORTGROUPS     00000001800113f8     util.obj
 0001:00010400       OPIF_DISABLEHIGHLIGHTING   0000000180011400     util.obj
 0001:00010408       OPIF_ADDDOTS               0000000180011408     util.obj
 0001:00010410       OPIF_RAWSELECTION          0000000180011410     util.obj
 0001:00010418       OPIF_REALNAMES             0000000180011418     util.obj
 0001:00010420       OPIF_SHOWNAMESONLY         0000000180011420     util.obj
 0001:00010428       OPIF_SHOWRIGHTALIGNNAMES   0000000180011428     util.obj
 0001:00010430       OPIF_SHOWPRESERVECASE      0000000180011430     util.obj
 0001:00010438       OPIF_COMPAREFATTIME        0000000180011438     util.obj
 0001:00010440       OPIF_EXTERNALGET           0000000180011440     util.obj
 0001:00010448       OPIF_EXTERNALPUT           0000000180011448     util.obj
 0001:00010450       OPIF_EXTERNALDELETE        0000000180011450     util.obj
 0001:00010458       OPIF_EXTERNALMKDIR         0000000180011458     util.obj
 0001:00010460       OPIF_USEATTRHIGHLIGHTING   0000000180011460     util.obj
 0001:00010468       OPIF_USECRC32              0000000180011468     util.obj
 0001:00010470       OPIF_USEFREESIZE           0000000180011470     util.obj
 0001:00010478       OPIF_SHORTCUT              0000000180011478     util.obj
 0001:00010480       OPIF_NONE                  0000000180011480     util.obj
 0001:00010488       OPM_SILENT                 0000000180011488     util.obj
 0001:00010490       OPM_FIND                   0000000180011490     util.obj
 0001:00010498       OPM_VIEW                   0000000180011498     util.obj
 0001:000104a0       OPM_EDIT                   00000001800114a0     util.obj
 0001:000104a8       OPM_TOPLEVEL               00000001800114a8     util.obj
 0001:000104b0       OPM_DESCR                  00000001800114b0     util.obj
 0001:000104b8       OPM_QUICKVIEW              00000001800114b8     util.obj
 0001:000104c0       OPM_PGDN                   00000001800114c0     util.obj
 0001:000104c8       OPM_COMMANDS               00000001800114c8     util.obj
 0001:000104d0       OPM_NONE                   00000001800114d0     util.obj
 0001:000104d8       FOSF_ACTIVE                00000001800114d8     util.obj
 0001:000104e0       FOSF_NONE                  00000001800114e0     util.obj
 0001:000104e8       PCIF_NONE                  00000001800114e8     util.obj
 0001:000104f0       FarGuid                    00000001800114f0     util.obj
 0001:00010500       PDF_DIALOGEVENTDRAWENABLE  0000000180011500     util.obj
 0001:00010508       PDF_PROCESSINGERROR        0000000180011508     util.obj
 0001:00010510       PDF_FULL_TIME_RESOLUTION   0000000180011510     util.obj
 0001:000105a0       PDF_DIALOGEVENTDRAWENABLE  00000001800115a0     win.obj
 0001:000105a8       PDF_PROCESSINGERROR        00000001800115a8     win.obj
 0001:000105b0       PDF_FULL_TIME_RESOLUTION   00000001800115b0     win.obj
 0001:000105b8       FCF_FG_4BIT                00000001800115b8     win.obj
 0001:000107a0       FCF_BG_4BIT                00000001800117a0     win.obj
 0001:000107a8       FCF_4BITMASK               00000001800117a8     win.obj
 0001:000107b0       FCF_RAWATTR_MASK           00000001800117b0     win.obj
 0001:000107b8       FCF_EXTENDEDFLAGS          00000001800117b8     win.obj
 0001:000107c0       FCF_FG_BOLD                00000001800117c0     win.obj
 0001:000107c8       FCF_FG_ITALIC              00000001800117c8     win.obj
 0001:000107d0       FCF_FG_UNDERLINE           00000001800117d0     win.obj
 0001:000107d8       FCF_STYLEMASK              00000001800117d8     win.obj
 0001:000107e0       FCF_NONE                   00000001800117e0     win.obj
 0001:000107e8       CDF_NONE                   00000001800117e8     win.obj
 0001:000107f0       FMSG_WARNING               00000001800117f0     win.obj
 0001:000107f8       FMSG_ERRORTYPE             00000001800117f8     win.obj
 0001:00010800       FMSG_KEEPBACKGROUND        0000000180011800     win.obj
 0001:00010808       FMSG_LEFTALIGN             0000000180011808     win.obj
 0001:00010810       FMSG_ALLINONE              0000000180011810     win.obj
 0001:00010818       FMSG_MB_OK                 0000000180011818     win.obj
 0001:00010820       FMSG_MB_OKCANCEL           0000000180011820     win.obj
 0001:00010828       FMSG_MB_ABORTRETRYIGNORE   0000000180011828     win.obj
 0001:00010830       FMSG_MB_YESNO              0000000180011830     win.obj
 0001:00010838       FMSG_MB_YESNOCANCEL        0000000180011838     win.obj
 0001:00010840       FMSG_MB_RETRYCANCEL        0000000180011840     win.obj
 0001:00010848       FMSG_NONE                  0000000180011848     win.obj
 0001:00010850       DIF_BOXCOLOR               0000000180011850     win.obj
 0001:00010858       DIF_GROUP                  0000000180011858     win.obj
 0001:00010860       DIF_LEFTTEXT               0000000180011860     win.obj
 0001:00010868       DIF_MOVESELECT             0000000180011868     win.obj
 0001:00010870       DIF_SHOWAMPERSAND          0000000180011870     win.obj
 0001:00010878       DIF_CENTERGROUP            0000000180011878     win.obj
 0001:00010880       DIF_NOBRACKETS             0000000180011880     win.obj
 0001:00010888       DIF_MANUALADDHISTORY       0000000180011888     win.obj
 0001:00010890       DIF_SEPARATOR              0000000180011890     win.obj
 0001:00010898       DIF_SEPARATOR2             0000000180011898     win.obj
 0001:000108a0       DIF_EDITOR                 00000001800118a0     win.obj
 0001:000108a8       DIF_LISTNOAMPERSAND        00000001800118a8     win.obj
 0001:000108b0       DIF_LISTNOBOX              00000001800118b0     win.obj
 0001:000108b8       DIF_HISTORY                00000001800118b8     win.obj
 0001:000108c0       DIF_BTNNOCLOSE             00000001800118c0     win.obj
 0001:000108c8       DIF_CENTERTEXT             00000001800118c8     win.obj
 0001:000108d0       DIF_SEPARATORUSER          00000001800118d0     win.obj
 0001:000108d8       DIF_SETSHIELD              00000001800118d8     win.obj
 0001:000108e0       DIF_EDITEXPAND             00000001800118e0     win.obj
 0001:000108e8       DIF_DROPDOWNLIST           00000001800118e8     win.obj
 0001:000108f0       DIF_USELASTHISTORY         00000001800118f0     win.obj
 0001:000108f8       DIF_MASKEDIT               00000001800118f8     win.obj
 0001:00010900       DIF_LISTTRACKMOUSE         0000000180011900     win.obj
 0001:00010908       DIF_LISTTRACKMOUSEINFOCUS  0000000180011908     win.obj
 0001:00010910       DIF_SELECTONENTRY          0000000180011910     win.obj
 0001:00010918       DIF_3STATE                 0000000180011918     win.obj
 0001:00010920       DIF_EDITPATH               0000000180011920     win.obj
 0001:00010928       DIF_LISTWRAPMODE           0000000180011928     win.obj
 0001:00010930       DIF_NOAUTOCOMPLETE         0000000180011930     win.obj
 0001:00010938       DIF_LISTAUTOHIGHLIGHT      0000000180011938     win.obj
 0001:00010940       DIF_LISTNOCLOSE            0000000180011940     win.obj
 0001:00010948       DIF_EDITPATHEXEC           0000000180011948     win.obj
 0001:00010950       DIF_HIDDEN                 0000000180011950     win.obj
 0001:00010958       DIF_READONLY               0000000180011958     win.obj
 0001:00010960       DIF_NOFOCUS                0000000180011960     win.obj
 0001:00010968       DIF_DISABLE                0000000180011968     win.obj
 0001:00010970       DIF_DEFAULTBUTTON          0000000180011970     win.obj
 0001:00010978       DIF_FOCUS                  0000000180011978     win.obj
 0001:00010980       DIF_RIGHTTEXT              0000000180011980     win.obj
 0001:00010988       DIF_WORDWRAP               0000000180011988     win.obj
 0001:00010990       DIF_NONE                   0000000180011990     win.obj
 0001:00010998       LIF_SELECTED               0000000180011998     win.obj
 0001:000109a0       LIF_CHECKED                00000001800119a0     win.obj
 0001:000109a8       LIF_SEPARATOR              00000001800119a8     win.obj
 0001:000109b0       LIF_DISABLE                00000001800119b0     win.obj
 0001:000109b8       LIF_GRAYED                 00000001800119b8     win.obj
 0001:000109c0       LIF_HIDDEN                 00000001800119c0     win.obj
 0001:000109c8       LIF_DELETEUSERDATA         00000001800119c8     win.obj
 0001:000109d0       LIF_NONE                   00000001800119d0     win.obj
 0001:000109d8       LIFIND_EXACTMATCH          00000001800119d8     win.obj
 0001:000109e0       LIFIND_NONE                00000001800119e0     win.obj
 0001:000109e8       LINFO_SHOWNOBOX            00000001800119e8     win.obj
 0001:000109f0       LINFO_AUTOHIGHLIGHT        00000001800119f0     win.obj
 0001:000109f8       LINFO_REVERSEHIGHLIGHT     00000001800119f8     win.obj
 0001:00010a00       LINFO_WRAPMODE             0000000180011a00     win.obj
 0001:00010a08       LINFO_SHOWAMPERSAND        0000000180011a08     win.obj
 0001:00010a10       LINFO_NONE                 0000000180011a10     win.obj
 0001:00010a18       FDLG_WARNING               0000000180011a18     win.obj
 0001:00010a20       FDLG_SMALLDIALOG           0000000180011a20     win.obj
 0001:00010a28       FDLG_NODRAWSHADOW          0000000180011a28     win.obj
 0001:00010a30       FDLG_NODRAWPANEL           0000000180011a30     win.obj
 0001:00010a38       FDLG_KEEPCONSOLETITLE      0000000180011a38     win.obj
 0001:00010a40       FDLG_NONMODAL              0000000180011a40     win.obj
 0001:00010a48       FDLG_NONE                  0000000180011a48     win.obj
 0001:00010a50       MIF_SELECTED               0000000180011a50     win.obj
 0001:00010a58       MIF_CHECKED                0000000180011a58     win.obj
 0001:00010a60       MIF_SEPARATOR              0000000180011a60     win.obj
 0001:00010a68       MIF_DISABLE                0000000180011a68     win.obj
 0001:00010a70       MIF_GRAYED                 0000000180011a70     win.obj
 0001:00010a78       MIF_HIDDEN                 0000000180011a78     win.obj
 0001:00010a80       MIF_NONE                   0000000180011a80     win.obj
 0001:00010a88       FMENU_SHOWAMPERSAND        0000000180011a88     win.obj
 0001:00010a90       FMENU_WRAPMODE             0000000180011a90     win.obj
 0001:00010a98       FMENU_AUTOHIGHLIGHT        0000000180011a98     win.obj
 0001:00010aa0       FMENU_REVERSEAUTOHIGHLIGHT 0000000180011aa0     win.obj
 0001:00010aa8       FMENU_CHANGECONSOLETITLE   0000000180011aa8     win.obj
 0001:00010ab0       FMENU_SHOWNOBOX            0000000180011ab0     win.obj
 0001:00010ab8       FMENU_SHOWSHORTBOX         0000000180011ab8     win.obj
 0001:00010ac0       FMENU_SHOWSINGLEBOX        0000000180011ac0     win.obj
 0001:00010ac8       FMENU_NODRAWSHADOW         0000000180011ac8     win.obj
 0001:00010ad0       FMENU_NONE                 0000000180011ad0     win.obj
 0001:00010ad8       PPIF_SELECTED              0000000180011ad8     win.obj
 0001:00010ae0       PPIF_PROCESSDESCR          0000000180011ae0     win.obj
 0001:00010ae8       PPIF_NONE                  0000000180011ae8     win.obj
 0001:00010af0       PFLAGS_SHOWHIDDEN          0000000180011af0     win.obj
 0001:00010af8       PFLAGS_HIGHLIGHT           0000000180011af8     win.obj
 0001:00010b00       PFLAGS_REVERSESORTORDER    0000000180011b00     win.obj
 0001:00010b08       PFLAGS_USESORTGROUPS       0000000180011b08     win.obj
 0001:00010b10       PFLAGS_SELECTEDFIRST       0000000180011b10     win.obj
 0001:00010b18       PFLAGS_REALNAMES           0000000180011b18     win.obj
 0001:00010b20       PFLAGS_PANELLEFT           0000000180011b20     win.obj
 0001:00010b28       PFLAGS_DIRECTORIESFIRST    0000000180011b28     win.obj
 0001:00010b30       PFLAGS_USECRC32            0000000180011b30     win.obj
 0001:00010b38       PFLAGS_PLUGIN              0000000180011b38     win.obj
 0001:00010b40       PFLAGS_VISIBLE             0000000180011b40     win.obj
 0001:00010b48       PFLAGS_FOCUS               0000000180011b48     win.obj
 0001:00010b50       PFLAGS_ALTERNATIVENAMES    0000000180011b50     win.obj
 0001:00010b58       PFLAGS_SHORTCUT            0000000180011b58     win.obj
 0001:00010b60       PFLAGS_NONE                0000000180011b60     win.obj
 0001:00010b68       VF_NONMODAL                0000000180011b68     win.obj
 0001:00010b70       VF_DELETEONCLOSE           0000000180011b70     win.obj
 0001:00010b78       VF_ENABLE_F6               0000000180011b78     win.obj
 0001:00010b80       VF_DISABLEHISTORY          0000000180011b80     win.obj
 0001:00010b88       VF_IMMEDIATERETURN         0000000180011b88     win.obj
 0001:00010b90       VF_DELETEONLYFILEONCLOSE   0000000180011b90     win.obj
 0001:00010b98       VF_NONE                    0000000180011b98     win.obj
 0001:00010ba0       EF_NONMODAL                0000000180011ba0     win.obj
 0001:00010ba8       EF_CREATENEW               0000000180011ba8     win.obj
 0001:00010bb0       EF_ENABLE_F6               0000000180011bb0     win.obj
 0001:00010bb8       EF_DISABLEHISTORY          0000000180011bb8     win.obj
 0001:00010bc0       EF_DELETEONCLOSE           0000000180011bc0     win.obj
 0001:00010bc8       EF_IMMEDIATERETURN         0000000180011bc8     win.obj
 0001:00010bd0       EF_DELETEONLYFILEONCLOSE   0000000180011bd0     win.obj
 0001:00010bd8       EF_LOCKED                  0000000180011bd8     win.obj
 0001:00010be0       EF_DISABLESAVEPOS          0000000180011be0     win.obj
 0001:00010be8       EF_OPENMODE_MASK           0000000180011be8     win.obj
 0001:00010bf0       EF_OPENMODE_QUERY          0000000180011bf0     win.obj
 0001:00010bf8       EF_OPENMODE_NEWIFOPEN      0000000180011bf8     win.obj
 0001:00010c00       EF_OPENMODE_USEEXISTING    0000000180011c00     win.obj
 0001:00010c08       EF_OPENMODE_BREAKIFOPEN    0000000180011c08     win.obj
 0001:00010c10       EF_OPENMODE_RELOADIFOPEN   0000000180011c10     win.obj
 0001:00010c18       EN_NONE                    0000000180011c18     win.obj
 0001:00010c20       FHELP_NOSHOWERROR          0000000180011c20     win.obj
 0001:00010c28       FHELP_SELFHELP             0000000180011c28     win.obj
 0001:00010c30       FHELP_FARHELP              0000000180011c30     win.obj
 0001:00010c38       FHELP_CUSTOMFILE           0000000180011c38     win.obj
 0001:00010c40       FHELP_CUSTOMPATH           0000000180011c40     win.obj
 0001:00010c48       FHELP_GUID                 0000000180011c48     win.obj
 0001:00010c50       FHELP_USECONTENTS          0000000180011c50     win.obj
 0001:00010c58       FHELP_NONE                 0000000180011c58     win.obj
 0001:00010c60       KMFLAGS_SILENTCHECK        0000000180011c60     win.obj
 0001:00010c68       KMFLAGS_NOSENDKEYSTOPLUGINS 0000000180011c68     win.obj
 0001:00010c70       KMFLAGS_ENABLEOUTPUT       0000000180011c70     win.obj
 0001:00010c78       KMFLAGS_LANGMASK           0000000180011c78     win.obj
 0001:00010c80       KMFLAGS_LUA                0000000180011c80     win.obj
 0001:00010c88       KMFLAGS_MOONSCRIPT         0000000180011c88     win.obj
 0001:00010c90       KMFLAGS_NONE               0000000180011c90     win.obj
 0001:00010c98       AKMFLAGS_NONE              0000000180011c98     win.obj
 0001:00010ca0       FSETCLR_REDRAW             0000000180011ca0     win.obj
 0001:00010ca8       FSETCLR_NONE               0000000180011ca8     win.obj
 0001:00010cb0       WIF_MODIFIED               0000000180011cb0     win.obj
 0001:00010cb8       WIF_CURRENT                0000000180011cb8     win.obj
 0001:00010cc0       WIF_MODAL                  0000000180011cc0     win.obj
 0001:00010cc8       WIF_NONE                   0000000180011cc8     win.obj
 0001:00010cd0       VOPT_SAVEFILEPOSITION      0000000180011cd0     win.obj
 0001:00010cd8       VOPT_AUTODETECTCODEPAGE    0000000180011cd8     win.obj
 0001:00010ce0       VOPT_SHOWTITLEBAR          0000000180011ce0     win.obj
 0001:00010ce8       VOPT_SHOWKEYBAR            0000000180011ce8     win.obj
 0001:00010cf0       VOPT_SHOWSCROLLBAR         0000000180011cf0     win.obj
 0001:00010cf8       VOPT_QUICKVIEW             0000000180011cf8     win.obj
 0001:00010d00       VOPT_NONE                  0000000180011d00     win.obj
 0001:00010d08       VSMFL_REDRAW               0000000180011d08     win.obj
 0001:00010d10       VSMFL_NONE                 0000000180011d10     win.obj
 0001:00010d18       VSP_NOREDRAW               0000000180011d18     win.obj
 0001:00010d20       VSP_PERCENT                0000000180011d20     win.obj
 0001:00010d28       VSP_RELATIVE               0000000180011d28     win.obj
 0001:00010d30       VSP_NORETNEWPOS            0000000180011d30     win.obj
 0001:00010d38       VSP_NONE                   0000000180011d38     win.obj
 0001:00010d40       VMF_WRAP                   0000000180011d40     win.obj
 0001:00010d48       VMF_WORDWRAP               0000000180011d48     win.obj
 0001:00010d50       VMF_NONE                   0000000180011d50     win.obj
 0001:00010d58       ECF_TABMARKFIRST           0000000180011d58     win.obj
 0001:00010d60       ECF_TABMARKCURRENT         0000000180011d60     win.obj
 0001:00010d68       ECF_AUTODELETE             0000000180011d68     win.obj
 0001:00010d70       ECF_NONE                   0000000180011d70     win.obj
 0001:00010d78       FIB_ENABLEEMPTY            0000000180011d78     win.obj
 0001:00010d80       FIB_PASSWORD               0000000180011d80     win.obj
 0001:00010d88       FIB_EXPANDENV              0000000180011d88     win.obj
 0001:00010d90       FIB_NOUSELASTHISTORY       0000000180011d90     win.obj
 0001:00010d98       FIB_BUTTONS                0000000180011d98     win.obj
 0001:00010da0       FIB_NOAMPERSAND            0000000180011da0     win.obj
 0001:00010da8       FIB_EDITPATH               0000000180011da8     win.obj
 0001:00010db0       FIB_EDITPATHEXEC           0000000180011db0     win.obj
 0001:00010db8       FIB_NONE                   0000000180011db8     win.obj
 0001:00010dc0       FPF_LOADED                 0000000180011dc0     win.obj
 0001:00010dc8       FPF_ANSI                   0000000180011dc8     win.obj
 0001:00010dd0       FPF_NONE                   0000000180011dd0     win.obj
 0001:00010dd8       PN_CMPNAME                 0000000180011dd8     win.obj
 0001:00010de0       PN_CMPNAMELIST             0000000180011de0     win.obj
 0001:00010de8       PN_GENERATENAME            0000000180011de8     win.obj
 0001:00010df0       PN_CHECKMASK               0000000180011df0     win.obj
 0001:00010df8       PN_SKIPPATH                0000000180011df8     win.obj
 0001:00010e00       PN_SHOWERRORMESSAGE        0000000180011e00     win.obj
 0001:00010e08       PN_NONE                    0000000180011e08     win.obj
 0001:00010e10       XLAT_SWITCHKEYBLAYOUT      0000000180011e10     win.obj
 0001:00010e18       XLAT_SWITCHKEYBBEEP        0000000180011e18     win.obj
 0001:00010e20       XLAT_USEKEYBLAYOUTNAME     0000000180011e20     win.obj
 0001:00010e28       XLAT_CONVERTALLCMDLINE     0000000180011e28     win.obj
 0001:00010e30       XLAT_NONE                  0000000180011e30     win.obj
 0001:00010e38       FRS_RETUPDIR               0000000180011e38     win.obj
 0001:00010e40       FRS_RECUR                  0000000180011e40     win.obj
 0001:00010e48       FRS_SCANSYMLINK            0000000180011e48     win.obj
 0001:00010e50       FRS_NONE                   0000000180011e50     win.obj
 0001:00010e58       MLF_SHOWERRMSG             0000000180011e58     win.obj
 0001:00010e60       MLF_DONOTUPDATEPANEL       0000000180011e60     win.obj
 0001:00010e68       MLF_HOLDTARGET             0000000180011e68     win.obj
 0001:00010e70       MLF_NONE                   0000000180011e70     win.obj
 0001:00010e78       FFFS_COMMAS                0000000180011e78     win.obj
 0001:00010e80       FFFS_FLOATSIZE             0000000180011e80     win.obj
 0001:00010e88       FFFS_SHOWBYTESINDEX        0000000180011e88     win.obj
 0001:00010e90       FFFS_ECONOMIC              0000000180011e90     win.obj
 0001:00010e98       FFFS_THOUSAND              0000000180011e98     win.obj
 0001:00010ea0       FFFS_MINSIZEINDEX          0000000180011ea0     win.obj
 0001:00010ea8       FFFS_MINSIZEINDEX_MASK     0000000180011ea8     win.obj
 0001:00010eb0       FFFS_NONE                  0000000180011eb0     win.obj
 0001:00010eb8       PF_PRELOAD                 0000000180011eb8     win.obj
 0001:00010ec0       PF_DISABLEPANELS           0000000180011ec0     win.obj
 0001:00010ec8       PF_EDITOR                  0000000180011ec8     win.obj
 0001:00010ed0       PF_VIEWER                  0000000180011ed0     win.obj
 0001:00010ed8       PF_FULLCMDLINE             0000000180011ed8     win.obj
 0001:00010ee0       PF_DIALOG                  0000000180011ee0     win.obj
 0001:00010ee8       PF_NONE                    0000000180011ee8     win.obj
 0001:00010ef0       IPLFLAGS_SEPARATOR         0000000180011ef0     win.obj
 0001:00010ef8       IPLFLAGS_NONE              0000000180011ef8     win.obj
 0001:00010f00       PMFLAGS_FULLSCREEN         0000000180011f00     win.obj
 0001:00010f08       PMFLAGS_DETAILEDSTATUS     0000000180011f08     win.obj
 0001:00010f10       PMFLAGS_ALIGNEXTENSIONS    0000000180011f10     win.obj
 0001:00010f18       PMFLAGS_CASECONVERSION     0000000180011f18     win.obj
 0001:00010f20       PMFLAGS_NONE               0000000180011f20     win.obj
 0001:00010f28       OPIF_DISABLEFILTER         0000000180011f28     win.obj
 0001:00010f30       OPIF_DISABLESORTGROUPS     0000000180011f30     win.obj
 0001:00010f38       OPIF_DISABLEHIGHLIGHTING   0000000180011f38     win.obj
 0001:00010f40       OPIF_ADDDOTS               0000000180011f40     win.obj
 0001:00010f48       OPIF_RAWSELECTION          0000000180011f48     win.obj
 0001:00010f50       OPIF_REALNAMES             0000000180011f50     win.obj
 0001:00010f58       OPIF_SHOWNAMESONLY         0000000180011f58     win.obj
 0001:00010f60       OPIF_SHOWRIGHTALIGNNAMES   0000000180011f60     win.obj
 0001:00010f68       OPIF_SHOWPRESERVECASE      0000000180011f68     win.obj
 0001:00010f70       OPIF_COMPAREFATTIME        0000000180011f70     win.obj
 0001:00010f78       OPIF_EXTERNALGET           0000000180011f78     win.obj
 0001:00010f80       OPIF_EXTERNALPUT           0000000180011f80     win.obj
 0001:00010f88       OPIF_EXTERNALDELETE        0000000180011f88     win.obj
 0001:00010f90       OPIF_EXTERNALMKDIR         0000000180011f90     win.obj
 0001:00010f98       OPIF_USEATTRHIGHLIGHTING   0000000180011f98     win.obj
 0001:00010fa0       OPIF_USECRC32              0000000180011fa0     win.obj
 0001:00010fa8       OPIF_USEFREESIZE           0000000180011fa8     win.obj
 0001:00010fb0       OPIF_SHORTCUT              0000000180011fb0     win.obj
 0001:00010fb8       OPIF_NONE                  0000000180011fb8     win.obj
 0001:00010fc0       OPM_SILENT                 0000000180011fc0     win.obj
 0001:00010fc8       OPM_FIND                   0000000180011fc8     win.obj
 0001:00010fd0       OPM_VIEW                   0000000180011fd0     win.obj
 0001:00010fd8       OPM_EDIT                   0000000180011fd8     win.obj
 0001:00010fe0       OPM_TOPLEVEL               0000000180011fe0     win.obj
 0001:00010fe8       OPM_DESCR                  0000000180011fe8     win.obj
 0001:00010ff0       OPM_QUICKVIEW              0000000180011ff0     win.obj
 0001:00010ff8       OPM_PGDN                   0000000180011ff8     win.obj
 0001:00011000       OPM_COMMANDS               0000000180012000     win.obj
 0001:00011008       OPM_NONE                   0000000180012008     win.obj
 0001:00011010       FOSF_ACTIVE                0000000180012010     win.obj
 0001:00011018       FOSF_NONE                  0000000180012018     win.obj
 0001:00011020       PCIF_NONE                  0000000180012020     win.obj
 0001:00011028       FarGuid                    0000000180012028     win.obj
 0001:000114f0       ?tokenTable@@3QBQEBDB      00000001800124f0     libvcruntime:undname.obj
 0001:00011570       ?nameTable@@3QBQEBDB       0000000180012570     libvcruntime:undname.obj
 0001:00011800       ?rttiTable@@3QBQEBDB       0000000180012800     libvcruntime:undname.obj
 0001:00011eb8       ?module_names@?A0x14c33c87@@3QBQEB_WB 0000000180012eb8     libvcruntime:winapi_downlevel.obj
 0001:00011f88       ?candidate_modules@?1??try_get_FlsAlloc@@YAP6AKP6AXPEAX@Z@ZXZ@4QBW4module_id@?A0x14c33c87@@B 0000000180012f88     libvcruntime:winapi_downlevel.obj
 0001:00011fa0       ?candidate_modules@?1??try_get_FlsFree@@YAP6AHK@ZXZ@4QBW4module_id@?A0x14c33c87@@B 0000000180012fa0     libvcruntime:winapi_downlevel.obj
 0001:00011fb0       ?candidate_modules@?1??try_get_FlsGetValue@@YAP6APEAXK@ZXZ@4QBW4module_id@?A0x14c33c87@@B 0000000180012fb0     libvcruntime:winapi_downlevel.obj
 0001:00011fc8       ?candidate_modules@?1??try_get_FlsSetValue@@YAP6AHKPEAX@ZXZ@4QBW4module_id@?A0x14c33c87@@B 0000000180012fc8     libvcruntime:winapi_downlevel.obj
 0001:00011fe0       ?candidate_modules@?1??try_get_InitializeCriticalSectionEx@@YAP6AHPEAU_RTL_CRITICAL_SECTION@@KK@ZXZ@4QBW4module_id@?A0x14c33c87@@B 0000000180012fe0     libvcruntime:winapi_downlevel.obj
 0001:00012090       ?errtable@@3QBUerrentry@?A0x31fdb9ec@@B 0000000180013090     libucrt:errno.obj
 0001:00012240       ?default_cmd_exe@?1???$common_popen_nolock@_W@@YAPEAU_iobuf@@QEB_W0HAEAY01H@Z@4QB_WB 0000000180013240     libucrt:popen.obj
 0001:00012250       ?slash_c@?1???$common_popen_nolock@_W@@YAPEAU_iobuf@@QEB_W0HAEAY01H@Z@4QB_WB 0000000180013250     libucrt:popen.obj
 0001:00012260       ?comspec_name@?1???$get_comspec@_W@@YAPEB_WXZ@4QB_WB 0000000180013260     libucrt:popen.obj
 0001:00012270       ?backslash@?L@???$get_executable_path@_W@@YAPEB_WQEB_W@Z@4QB_WB 0000000180013270     libucrt:popen.obj
 0001:00012278       ?path_name@?1???$get_path@_W@@YAPEB_WXZ@4QB_WB 0000000180013278     libucrt:popen.obj
 0001:00012e80       ?comspec_name@?1???$common_system@_W@@YAHQEB_W@Z@4QB_WB 0000000180013e80     libucrt:system.obj
 0001:00012e90       ?cmd_exe@?1???$common_system@_W@@YAHQEB_W@Z@4QB_WB 0000000180013e90     libucrt:system.obj
 0001:00012ea0       ?slash_c@?1???$common_system@_W@@YAHQEB_W@Z@4QB_WB 0000000180013ea0     libucrt:system.obj
 0001:00012fb0       __acrt_initializers        0000000180013fb0     libucrt:initialization.obj
 0001:000137d0       __real@433fffffffffffff    00000001800147d0     libucrt:fpsr.obj
 0001:000137d8       __real@c33fffffffffffff    00000001800147d8     libucrt:fpsr.obj
 0001:00013ce0       ?module_names@?A0x391cf84c@@3QBQEB_WB 0000000180014ce0     libucrt:winapi_thunks.obj
 0001:00014288       ?candidate_modules@?1??try_get_AreFileApisANSI@@YAP6AHXZXZ@4QBW4module_id@?A0x391cf84c@@B 0000000180015288     libucrt:winapi_thunks.obj
 0001:000142a0       ?candidate_modules@?1??try_get_CompareStringEx@@YAP6AHPEB_WK0H0HPEAU_nlsversioninfo@@PEAX_J@ZXZ@4QBW4module_id@?A0x391cf84c@@B 00000001800152a0     libucrt:winapi_thunks.obj
 0001:000142b8       ?candidate_modules@?1??try_get_FlsAlloc@@YAP6AKP6AXPEAX@Z@ZXZ@4QBW4module_id@?A0x391cf84c@@B 00000001800152b8     libucrt:winapi_thunks.obj
 0001:000142d0       ?candidate_modules@?1??try_get_FlsFree@@YAP6AHK@ZXZ@4QBW4module_id@?A0x391cf84c@@B 00000001800152d0     libucrt:winapi_thunks.obj
 0001:000142e0       ?candidate_modules@?1??try_get_FlsGetValue@@YAP6APEAXK@ZXZ@4QBW4module_id@?A0x391cf84c@@B 00000001800152e0     libucrt:winapi_thunks.obj
 0001:000142f8       ?candidate_modules@?1??try_get_FlsSetValue@@YAP6AHKPEAX@ZXZ@4QBW4module_id@?A0x391cf84c@@B 00000001800152f8     libucrt:winapi_thunks.obj
 0001:00014310       ?candidate_modules@?1??try_get_InitializeCriticalSectionEx@@YAP6AHPEAU_RTL_CRITICAL_SECTION@@KK@ZXZ@4QBW4module_id@?A0x391cf84c@@B 0000000180015310     libucrt:winapi_thunks.obj
 0001:00014338       ?candidate_modules@?1??try_get_LCMapStringEx@@YAP6AHPEB_WK0HPEA_WHPEAU_nlsversioninfo@@PEAX_J@ZXZ@4QBW4module_id@?A0x391cf84c@@B 0000000180015338     libucrt:winapi_thunks.obj
 0001:00014350       ?candidate_modules@?1??try_get_LocaleNameToLCID@@YAP6AKPEB_WK@ZXZ@4QBW4module_id@?A0x391cf84c@@B 0000000180015350     libucrt:winapi_thunks.obj
 0001:0001436c       ?candidate_modules@?1??try_get_AppPolicyGetProcessTerminationMethod@@YAP6AJPEAXPEAW4AppPolicyProcessTerminationMethod@@@ZXZ@4QBW4module_id@?A0x391cf84c@@B 000000018001536c     libucrt:winapi_thunks.obj
 0001:00014ba4       ?dot_slash@?CB@???$common_spawnv@_W@@YA_JHQEB_WQEBQEB_W1@Z@4QB_WB 0000000180015ba4     libucrt:spawnv.obj
 0001:00014bb0       ?extensions@?CP@???$common_spawnv@_W@@YA_JHQEB_WQEBQEB_W1@Z@4QAY04$$CB_WA 0000000180015bb0     libucrt:spawnv.obj
 0001:00014bd8       ?_mb_locale_names@@3QBQEB_WB 0000000180015bd8     libucrt:mbctype.obj
 0001:00014c70       ?LcidToLocaleNameTable@?A0x881e4c05@@3QBULcidToLocaleName@1@B 0000000180015c70     libucrt:lcidtoname_downlevel.obj
 0001:000166d0       ?LocaleNameToIndexTable@?A0x881e4c05@@3QBULocaleNameIndex@1@B 00000001800176d0     libucrt:lcidtoname_downlevel.obj
 0001:00017f64       ?equal_sign@?BD@???$construct_environment_block@_W@@YAHQEBQEB_WQEAPEA_W@Z@4QB_WB 0000000180018f64     libucrt:cenvarg.obj
 0001:00017f70       __real_ninf                0000000180018f70     libucrt:log10.obj
 0001:00017f80       __real_inf                 0000000180018f80     libucrt:log10.obj
 0001:00017f90       __real_neg_qnan            0000000180018f90     libucrt:log10.obj
 0001:00017fa0       __real_qnanbit             0000000180018fa0     libucrt:log10.obj
 0001:00017fb0       __int_1023                 0000000180018fb0     libucrt:log10.obj
 0001:00017fc0       __mask_001                 0000000180018fc0     libucrt:log10.obj
 0001:00017fd0       __mask_mant                0000000180018fd0     libucrt:log10.obj
 0001:00017fe0       __mask_mant_top8           0000000180018fe0     libucrt:log10.obj
 0001:00017ff0       __mask_mant9               0000000180018ff0     libucrt:log10.obj
 0001:00018000       __real_log10_e             0000000180019000     libucrt:log10.obj
 0001:00018010       __real_log10_e_lead        0000000180019010     libucrt:log10.obj
 0001:00018020       __real_log10_e_tail        0000000180019020     libucrt:log10.obj
 0001:00018030       __real_log10_2_lead        0000000180019030     libucrt:log10.obj
 0001:00018040       __real_log10_2_tail        0000000180019040     libucrt:log10.obj
 0001:00018050       __real_two                 0000000180019050     libucrt:log10.obj
 0001:00018060       __real_one                 0000000180019060     libucrt:log10.obj
 0001:00018070       __real_half                0000000180019070     libucrt:log10.obj
 0001:00018080       __mask_100                 0000000180019080     libucrt:log10.obj
 0001:00018090       __real_1_over_512          0000000180019090     libucrt:log10.obj
 0001:000180a0       __real_1_over_2            00000001800190a0     libucrt:log10.obj
 0001:000180b0       __real_1_over_3            00000001800190b0     libucrt:log10.obj
 0001:000180c0       __real_1_over_4            00000001800190c0     libucrt:log10.obj
 0001:000180d0       __real_1_over_5            00000001800190d0     libucrt:log10.obj
 0001:000180e0       __real_1_over_6            00000001800190e0     libucrt:log10.obj
 0001:000180f0       __real_neg_1023            00000001800190f0     libucrt:log10.obj
 0001:00018100       __mask_2045                0000000180019100     libucrt:log10.obj
 0001:00018110       __real_threshold           0000000180019110     libucrt:log10.obj
 0001:00018120       __real_near_one_lt         0000000180019120     libucrt:log10.obj
 0001:00018130       __real_near_one_gt         0000000180019130     libucrt:log10.obj
 0001:00018140       __real_min_norm            0000000180019140     libucrt:log10.obj
 0001:00018150       __real_notsign             0000000180019150     libucrt:log10.obj
 0001:00018160       __real_ca1                 0000000180019160     libucrt:log10.obj
 0001:00018170       __real_ca2                 0000000180019170     libucrt:log10.obj
 0001:00018180       __real_ca3                 0000000180019180     libucrt:log10.obj
 0001:00018190       __real_ca4                 0000000180019190     libucrt:log10.obj
 0001:000181a0       __mask_lower               00000001800191a0     libucrt:log10.obj
 0001:000181b0       __flag_x_zero              00000001800191b0     libucrt:log10.obj
 0001:000181b4       __flag_x_neg               00000001800191b4     libucrt:log10.obj
 0001:000181b8       __flag_x_nan               00000001800191b8     libucrt:log10.obj
 0001:00019a08       GS_ExceptionPointers       000000018001aa08     LIBCMT:gs_report.obj
 0001:00019de0       $$000000                   000000018001ade0     chkstk.obj
 0001:00019e50       f_sub                      000000018001ae50 f   bit64.obj
 0001:00019ea0       f_mul                      000000018001aea0 f   bit64.obj
 0001:00019f70       f_div                      000000018001af70 f   bit64.obj
 0001:00019ff0       f_mod                      000000018001aff0 f   bit64.obj
 0001:0001a050       f_unm                      000000018001b050 f   bit64.obj
 0001:0001a080       f_eq                       000000018001b080 f   bit64.obj
 0001:0001a0d0       f_lt                       000000018001b0d0 f   bit64.obj
 0001:0001a120       f_le                       000000018001b120 f   bit64.obj
 0001:0001a170       band                       000000018001b170 f   bit64.obj
 0001:0001a240       bor                        000000018001b240 f   bit64.obj
 0001:0001a310       bxor                       000000018001b310 f   bit64.obj
 0001:0001a3e0       bnot                       000000018001b3e0 f   bit64.obj
 0001:0001a410       lshift                     000000018001b410 f   bit64.obj
 0001:0001a460       rshift                     000000018001b460 f   bit64.obj
 0001:0001a4b0       arshift                    000000018001b4b0 f   bit64.obj
 0001:0001a510       f_new                      000000018001b510 f   bit64.obj
 0001:0001a780       f_tostring                 000000018001b780 f   bit64.obj
 0001:0001a7d0       f_type                     000000018001b7d0 f   bit64.obj
 0001:0001a870       f_add                      000000018001b870 f   bit64.obj
 0001:0001aae0       check64                    000000018001bae0 f   bit64.obj
 0001:0001ae90       FillFarMacroCall           000000018001be90 f   exported.obj
 0001:0001b0d0       FillFarMacroCall_Callback  000000018001c0d0 f   exported.obj
 0001:0001e6c0       $LN22                      000000018001f6c0     exported.obj
 0001:0001e6f0       PushAnalyseInfo            000000018001f6f0 f   exported.obj
 0001:0001e8a8       $LN18                      000000018001f8a8     exported.obj
 0001:0001e980       RegisterObject             000000018001f980 f   exported.obj
 0001:0001f500       errfile                    0000000180020500 f   lflua.obj
 0001:0001f580       getF                       0000000180020580 f   lflua.obj
 0001:000209c0       FL_PushParams              00000001800219c0 f   luamacro.obj
 0001:00020a60       InitMPR                    0000000180021a60 f   luamacro.obj
 0001:00020ad0       MacroCallFarCallback       0000000180021ad0 f   luamacro.obj
 0001:000211d0       uc_tostring                00000001800221d0 f   lusercontrol.obj
 0001:00021250       uc_index                   0000000180022250 f   lusercontrol.obj
 0001:00021350       uc_newindex                0000000180022350 f   lusercontrol.obj
 0001:00021460       uc_New                     0000000180022460 f   lusercontrol.obj
 0001:00021890       far_GetFileOwner           0000000180022890 f   service.obj
 0001:00021940       far_GetNumberOfLinks       0000000180022940 f   service.obj
 0001:000219a0       far_PluginStartupInfo      00000001800229a0 f   service.obj
 0001:00021a70       far_GetCurrentDirectory    0000000180022a70 f   service.obj
 0001:00021af0       editor_GetFileName         0000000180022af0 f   service.obj
 0001:00021bc0       editor_GetInfo             0000000180022bc0 f   service.obj
 0001:00021f40       editor_GetString           0000000180022f40 f   service.obj
 0001:00021f50       editor_GetStringW          0000000180022f50 f   service.obj
 0001:00021f60       editor_SetString           0000000180022f60 f   service.obj
 0001:00021f70       editor_SetStringW          0000000180022f70 f   service.obj
 0001:00021f80       editor_InsertString        0000000180022f80 f   service.obj
 0001:00022010       editor_DeleteString        0000000180023010 f   service.obj
 0001:00022080       editor_InsertText          0000000180023080 f   service.obj
 0001:00022100       editor_InsertTextW         0000000180023100 f   service.obj
 0001:00022110       editor_DeleteChar          0000000180023110 f   service.obj
 0001:00022180       editor_DeleteBlock         0000000180023180 f   service.obj
 0001:000221f0       editor_UndoRedo            00000001800231f0 f   service.obj
 0001:00022290       editor_SetKeyBar           0000000180023290 f   service.obj
 0001:000222a0       viewer_SetKeyBar           00000001800232a0 f   service.obj
 0001:000222b0       editor_SetParam            00000001800232b0 f   service.obj
 0001:00022410       editor_SetPosition         0000000180023410 f   service.obj
 0001:00022540       editor_Redraw              0000000180023540 f   service.obj
 0001:000225b0       editor_ExpandTabs          00000001800235b0 f   service.obj
 0001:00022640       editor_GetBookmarks        0000000180023640 f   service.obj
 0001:00022650       editor_GetSessionBookmarks 0000000180023650 f   service.obj
 0001:00022660       editor_AddSessionBookmark  0000000180023660 f   service.obj
 0001:000226d0       editor_ClearSessionBookmarks 00000001800236d0 f   service.obj
 0001:00022740       editor_DeleteSessionBookmark 0000000180023740 f   service.obj
 0001:000227d0       editor_NextSessionBookmark 00000001800237d0 f   service.obj
 0001:00022840       editor_PrevSessionBookmark 0000000180023840 f   service.obj
 0001:000228b0       editor_SetTitle            00000001800238b0 f   service.obj
 0001:00022930       editor_GetTitle            0000000180023930 f   service.obj
 0001:000229f0       editor_Quit                00000001800239f0 f   service.obj
 0001:00022a60       editor_Select              0000000180023a60 f   service.obj
 0001:00022b90       editor_GetSelection        0000000180023b90 f   service.obj
 0001:00022f30       editor_TabToReal           0000000180023f30 f   service.obj
 0001:00022f40       editor_RealToTab           0000000180023f40 f   service.obj
 0001:00022f50       editor_AddColor            0000000180023f50 f   service.obj
 0001:00023150       editor_DelColor            0000000180024150 f   service.obj
 0001:00023280       editor_GetColor            0000000180024280 f   service.obj
 0001:00023470       editor_SaveFile            0000000180024470 f   service.obj
 0001:00023530       editor_ReadInput           0000000180024530 f   service.obj
 0001:000235b0       editor_ProcessInput        00000001800245b0 f   service.obj
 0001:00023640       editor_SubscribeChangeEvent 0000000180024640 f   service.obj
 0001:000236d0       far_Menu                   00000001800246d0 f   service.obj
 0001:00024150       far_Message                0000000180025150 f   service.obj
 0001:00024310       panel_CheckPanelsExist     0000000180025310 f   service.obj
 0001:00024370       panel_ClosePanel           0000000180025370 f   service.obj
 0001:000243e0       panel_GetPanelInfo         00000001800253e0 f   service.obj
 0001:00024680       panel_GetPanelItem         0000000180025680 f   service.obj
 0001:00024690       panel_GetSelectedPanelItem 0000000180025690 f   service.obj
 0001:000246a0       panel_GetCurrentPanelItem  00000001800256a0 f   service.obj
 0001:000246b0       panel_GetPanelFormat       00000001800256b0 f   service.obj
 0001:000246c0       panel_GetPanelHostFile     00000001800256c0 f   service.obj
 0001:000246d0       panel_GetColumnTypes       00000001800256d0 f   service.obj
 0001:000246e0       panel_GetColumnWidths      00000001800256e0 f   service.obj
 0001:000246f0       panel_GetPanelPrefix       00000001800256f0 f   service.obj
 0001:00024700       panel_RedrawPanel          0000000180025700 f   service.obj
 0001:00024810       panel_SetSortOrder         0000000180025810 f   service.obj
 0001:00024820       panel_SetDirectoriesFirst  0000000180025820 f   service.obj
 0001:00024830       panel_UpdatePanel          0000000180025830 f   service.obj
 0001:00024840       panel_SetSortMode          0000000180025840 f   service.obj
 0001:00024850       panel_SetViewMode          0000000180025850 f   service.obj
 0001:00024860       panel_GetPanelDirectory    0000000180025860 f   service.obj
 0001:000249c0       panel_SetPanelDirectory    00000001800259c0 f   service.obj
 0001:00024bb0       panel_GetCmdLine           0000000180025bb0 f   service.obj
 0001:00024c50       panel_SetCmdLine           0000000180025c50 f   service.obj
 0001:00024cd0       panel_GetCmdLinePos        0000000180025cd0 f   service.obj
 0001:00024d50       panel_SetCmdLinePos        0000000180025d50 f   service.obj
 0001:00024dd0       panel_InsertCmdLine        0000000180025dd0 f   service.obj
 0001:00024e50       panel_GetCmdLineSelection  0000000180025e50 f   service.obj
 0001:00024f00       panel_SetCmdLineSelection  0000000180025f00 f   service.obj
 0001:00024fc0       panel_SetSelection         0000000180025fc0 f   service.obj
 0001:00024fd0       panel_ClearSelection       0000000180025fd0 f   service.obj
 0001:00024fe0       panel_BeginSelection       0000000180025fe0 f   service.obj
 0001:00025070       panel_EndSelection         0000000180026070 f   service.obj
 0001:00025100       panel_SetUserScreen        0000000180026100 f   service.obj
 0001:00025180       panel_GetUserScreen        0000000180026180 f   service.obj
 0001:00025200       panel_IsActivePanel        0000000180026200 f   service.obj
 0001:00025260       panel_SetActivePanel       0000000180026260 f   service.obj
 0001:00025300       far_GetDirList             0000000180026300 f   service.obj
 0001:00025660       far_GetPluginDirList       0000000180026660 f   service.obj
 0001:00025700       far_RestoreScreen          0000000180026700 f   service.obj
 0001:00025790       far_SaveScreen             0000000180026790 f   service.obj
 0001:00025870       far_SendDlgMessage         0000000180026870 f   service.obj
 0001:00026b6c       $LN156                     0000000180027b6c     service.obj
 0001:00026b78       $LN155                     0000000180027b78     service.obj
 0001:00026bbc       $LN154                     0000000180027bbc     service.obj
 0001:00026c44       $LN153                     0000000180027c44     service.obj
 0001:00026c90       far_DialogInit             0000000180027c90 f   service.obj
 0001:00027090       far_DialogRun              0000000180028090 f   service.obj
 0001:00027130       far_DialogFree             0000000180028130 f   service.obj
 0001:00027160       dialog_tostring            0000000180028160 f   service.obj
 0001:000271c0       dialog_rawhandle           00000001800281c0 f   service.obj
 0001:00027210       far_GetDlgItem             0000000180028210 f   service.obj
 0001:000272c0       far_SetDlgItem             00000001800282c0 f   service.obj
 0001:00027360       far_SubscribeDialogDrawEvents 0000000180028360 f   service.obj
 0001:00027380       editor_Editor              0000000180028380 f   service.obj
 0001:00027530       viewer_Viewer              0000000180028530 f   service.obj
 0001:000276c0       viewer_GetFileName         00000001800286c0 f   service.obj
 0001:00027790       viewer_GetInfo             0000000180028790 f   service.obj
 0001:00027a60       viewer_Quit                0000000180028a60 f   service.obj
 0001:00027ac0       viewer_Redraw              0000000180028ac0 f   service.obj
 0001:00027b20       viewer_Select              0000000180028b20 f   service.obj
 0001:00027bd0       viewer_SetPosition         0000000180028bd0 f   service.obj
 0001:00027dd0       viewer_SetMode             0000000180028dd0 f   service.obj
 0001:00027f00       far_ShowHelp               0000000180028f00 f   service.obj
 0001:00027ff0       far_InputBox               0000000180028ff0 f   service.obj
 0001:000281f0       far_GetMsg                 00000001800291f0 f   service.obj
 0001:00028270       far_Text                   0000000180029270 f   service.obj
 0001:00028320       far_CopyToClipboard        0000000180029320 f   service.obj
 0001:00028410       far_PasteFromClipboard     0000000180029410 f   service.obj
 0001:00028500       far_InputRecordToName      0000000180029500 f   service.obj
 0001:00028700       far_NameToInputRecord      0000000180029700 f   service.obj
 0001:00028780       far_LStricmp               0000000180029780 f   service.obj
 0001:00028800       far_LStrnicmp              0000000180029800 f   service.obj
 0001:000288a0       far_ProcessName            00000001800298a0 f   service.obj
 0001:00028af0       far_GetReparsePointInfo    0000000180029af0 f   service.obj
 0001:00028b90       far_LIsAlpha               0000000180029b90 f   service.obj
 0001:00028bf0       far_LIsAlphanum            0000000180029bf0 f   service.obj
 0001:00028c50       far_LIsLower               0000000180029c50 f   service.obj
 0001:00028cb0       far_LIsUpper               0000000180029cb0 f   service.obj
 0001:00028d10       far_LLowerBuf              0000000180029d10 f   service.obj
 0001:00028d80       far_LUpperBuf              0000000180029d80 f   service.obj
 0001:00028df0       far_MkTemp                 0000000180029df0 f   service.obj
 0001:00028e80       far_MkLink                 0000000180029e80 f   service.obj
 0001:00028fa0       far_GetPathRoot            0000000180029fa0 f   service.obj
 0001:00029040       far_TruncPathStr           000000018002a040 f   service.obj
 0001:00029050       far_TruncStr               000000018002a050 f   service.obj
 0001:00029060       far_RecursiveSearch        000000018002a060 f   service.obj
 0001:000291d0       far_ConvertPath            000000018002a1d0 f   service.obj
 0001:000292a0       far_AdvControl             000000018002a2a0 f   service.obj
 0001:00029a9c       $LN62                      000000018002aa9c     service.obj
 0001:00029b10       far_MacroLoadAll           000000018002ab10 f   service.obj
 0001:00029bf0       far_MacroSaveAll           000000018002abf0 f   service.obj
 0001:00029c40       far_MacroGetState          000000018002ac40 f   service.obj
 0001:00029c90       far_MacroGetArea           000000018002ac90 f   service.obj
 0001:00029ce0       far_MacroPost              000000018002ace0 f   service.obj
 0001:00029cf0       far_MacroCheck             000000018002acf0 f   service.obj
 0001:00029d00       far_MacroGetLastError      000000018002ad00 f   service.obj
 0001:00029e00       far_MacroAdd               000000018002ae00 f   service.obj
 0001:0002a0d0       far_MacroDelete            000000018002b0d0 f   service.obj
 0001:0002a190       far_MacroExecute           000000018002b190 f   service.obj
 0001:0002a320       far_CPluginStartupInfo     000000018002b320 f   service.obj
 0001:0002a350       far_MakeMenuItems          000000018002b350 f   service.obj
 0001:0002a6f0       far_Show                   000000018002b6f0 f   service.obj
 0001:0002a7a0       far_CreateFileFilter       000000018002b7a0 f   service.obj
 0001:0002a860       filefilter_Free            000000018002b860 f   service.obj
 0001:0002a8f0       filefilter_gc              000000018002b8f0 f   service.obj
 0001:0002a980       filefilter_tostring        000000018002b980 f   service.obj
 0001:0002a9e0       filefilter_OpenMenu        000000018002b9e0 f   service.obj
 0001:0002aa70       filefilter_Starting        000000018002ba70 f   service.obj
 0001:0002ab00       filefilter_IsFileInFilter  000000018002bb00 f   service.obj
 0001:0002abd0       far_LoadPlugin             000000018002bbd0 f   service.obj
 0001:0002abe0       far_ForcedLoadPlugin       000000018002bbe0 f   service.obj
 0001:0002abf0       far_UnloadPlugin           000000018002bbf0 f   service.obj
 0001:0002ac60       far_FindPlugin             000000018002bc60 f   service.obj
 0001:0002ad10       far_GetPluginInformation   000000018002bd10 f   service.obj
 0001:0002afb0       far_GetPlugins             000000018002bfb0 f   service.obj
 0001:0002b0d0       far_IsPluginLoaded         000000018002c0d0 f   service.obj
 0001:0002b1e0       far_XLat                   000000018002c1e0 f   service.obj
 0001:0002b310       far_FormatFileSize         000000018002c310 f   service.obj
 0001:0002b460       far_FarClock               000000018002c460 f   service.obj
 0001:0002b4b0       far_Timer                  000000018002c4b0 f   service.obj
 0001:0002b6a0       timer_gc                   000000018002c6a0 f   service.obj
 0001:0002b740       timer_tostring             000000018002c740 f   service.obj
 0001:0002b7a0       timer_index                000000018002c7a0 f   service.obj
 0001:0002b910       timer_newindex             000000018002c910 f   service.obj
 0001:0002bac0       far_CreateSettings         000000018002cac0 f   service.obj
 0001:0002bca0       Settings_set               000000018002cca0 f   service.obj
 0001:0002bdd0       Settings_get               000000018002cdd0 f   service.obj
 0001:0002bf20       Settings_delete            000000018002cf20 f   service.obj
 0001:0002bff0       Settings_createsubkey      000000018002cff0 f   service.obj
 0001:0002c130       Settings_opensubkey        000000018002d130 f   service.obj
 0001:0002c210       Settings_enum              000000018002d210 f   service.obj
 0001:0002c580       Settings_free              000000018002d580 f   service.obj
 0001:0002c620       far_FreeSettings           000000018002d620 f   service.obj
 0001:0002c6c0       Settings_tostring          000000018002d6c0 f   service.obj
 0001:0002c720       far_ColorDialog            000000018002d720 f   service.obj
 0001:0002c8a0       far_RunDefaultScript       000000018002d8a0 f   service.obj
 0001:0002c8d0       far_FileTimeResolution     000000018002d8d0 f   service.obj
 0001:0002c950       AddMacroData_gc            000000018002d950 f   service.obj
 0001:0002ca00       ChangePanelSelection       000000018002da00 f   service.obj
 0001:0002cc70       CheckFlagsFromTable        000000018002dc70 f   service.obj
 0001:0002d020       CustomAllocator            000000018002e020 f   service.obj
 0001:0002d150       FillEditorSelect           000000018002e150 f   service.obj
 0001:0002d250       FillEditorSetPosition      000000018002e250 f   service.obj
 0001:0002d560       FillKeyBarTitles           000000018002e560 f   service.obj
 0001:0002d770       FrsUserFunc                000000018002e770 f   service.obj
 0001:0002eae0       MacroSendString            000000018002fae0 f   service.obj
 0001:0002eef0       OptInputRecord             000000018002fef0 f   service.obj
 0001:0002efa0       PluginHandle_rawhandle     000000018002ffa0 f   service.obj
 0001:0002f250       $LN30                      0000000180030250     service.obj
 0001:0002f268       $LN29                      0000000180030268     service.obj
 0001:0002f280       PushBookmarks              0000000180030280 f   service.obj
 0001:0002f4d4       $LN15                      00000001800304d4     service.obj
 0001:0002f4e0       $LN14                      00000001800304e0     service.obj
 0001:0002f780       $LN32                      0000000180030780     service.obj
 0001:0002f78c       $LN31                      000000018003078c     service.obj
 0001:0002f7a4       $LN30                      00000001800307a4     service.obj
 0001:0002f800       PushDlgItem                0000000180030800 f   service.obj
 0001:0002fa60       PushDlgItemNum             0000000180030a60 f   service.obj
 0001:000302e0       PushPluginHandle           00000001800312e0 f   service.obj
 0001:00030380       PutPluginMenuItemToTable   0000000180031380 f   service.obj
 0001:000304a0       PutVersionInfoToTable      00000001800314a0 f   service.obj
 0001:00030540       SetDlgItem                 0000000180031540 f   service.obj
 0001:00030600       SetFarDialogItem           0000000180031600 f   service.obj
 0001:00030990       SetKeyBar                  0000000180031990 f   service.obj
 0001:00030af0       SetPanelBooleanProperty    0000000180031af0 f   service.obj
 0001:00030ba0       SetPanelIntegerProperty    0000000180031ba0 f   service.obj
 0001:00030ca0       _EditorGetString           0000000180031ca0 f   service.obj
 0001:00030f40       _EditorInsertText          0000000180031f40 f   service.obj
 0001:00031050       _EditorSetString           0000000180032050 f   service.obj
 0001:00031190       _EditorTabConvert          0000000180032190 f   service.obj
 0001:00031250       check_env_flag             0000000180032250 f   service.obj
 0001:00031380       free_dialog                0000000180032380 f   service.obj
 0001:000313f0       get_env_flag               00000001800323f0 f   service.obj
 0001:00031520       get_panel_item             0000000180032520 f   service.obj
 0001:00031630       get_string_info            0000000180032630 f   service.obj
 0001:00031720       luaopen_far                0000000180032720 f   service.obj
 0001:00031c40       plugin_load                0000000180032c40 f   service.obj
 0001:00031d80       timer_Close                0000000180032d80 f   service.obj
 0001:00031e40       truncstring                0000000180032e40 f   service.obj
 0001:00031f30       str_rep                    0000000180032f30 f   slnunico.obj
 0001:00031fc0       str_dump                   0000000180032fc0 f   slnunico.obj
 0001:00032040       str_format                 0000000180033040 f   slnunico.obj
 0001:00032584       $LN74                      0000000180033584     slnunico.obj
 0001:000325a0       $LN73                      00000001800335a0     slnunico.obj
 0001:000325e0       utf8_valid                 00000001800335e0 f   slnunico.obj
 0001:00032770       writer                     0000000180033770 f   slnunico.obj
 0001:00032790       Lutf8_byte                 0000000180033790 f   lutf8lib.obj
 0001:000328c0       Lutf8_char                 00000001800338c0 f   lutf8lib.obj
 0001:00032a40       Lutf8_charpos              0000000180033a40 f   lutf8lib.obj
 0001:00032b40       Lutf8_codepoint            0000000180033b40 f   lutf8lib.obj
 0001:00032c90       Lutf8_codes                0000000180033c90 f   lutf8lib.obj
 0001:00032ce0       Lutf8_escape               0000000180033ce0 f   lutf8lib.obj
 0001:00032ed8       $LN40                      0000000180033ed8     lutf8lib.obj
 0001:00032ee8       $LN39                      0000000180033ee8     lutf8lib.obj
 0001:00032f40       Lutf8_find                 0000000180033f40 f   lutf8lib.obj
 0001:00032f50       Lutf8_fold                 0000000180033f50 f   lutf8lib.obj
 0001:00032f60       Lutf8_gmatch               0000000180033f60 f   lutf8lib.obj
 0001:00032fc0       Lutf8_gsub                 0000000180033fc0 f   lutf8lib.obj
 0001:00033190       Lutf8_insert               0000000180034190 f   lutf8lib.obj
 0001:00033290       Lutf8_len                  0000000180034290 f   lutf8lib.obj
 0001:00033370       Lutf8_lower                0000000180034370 f   lutf8lib.obj
 0001:00033380       Lutf8_match                0000000180034380 f   lutf8lib.obj
 0001:00033390       Lutf8_ncasecmp             0000000180034390 f   lutf8lib.obj
 0001:00033550       Lutf8_next                 0000000180034550 f   lutf8lib.obj
 0001:00033600       Lutf8_offset               0000000180034600 f   lutf8lib.obj
 0001:00033630       Lutf8_remove               0000000180034630 f   lutf8lib.obj
 0001:00033780       Lutf8_reverse              0000000180034780 f   lutf8lib.obj
 0001:00033840       Lutf8_sub                  0000000180034840 f   lutf8lib.obj
 0001:00033950       Lutf8_title                0000000180034950 f   lutf8lib.obj
 0001:00033960       Lutf8_upper                0000000180034960 f   lutf8lib.obj
 0001:00033970       Lutf8_width                0000000180034970 f   lutf8lib.obj
 0001:00033a80       Lutf8_widthindex           0000000180034a80 f   lutf8lib.obj
 0001:00033b90       add_utf8char               0000000180034b90 f   lutf8lib.obj
 0001:00033c90       add_value                  0000000180034c90 f   lutf8lib.obj
 0001:00033ee0       classend                   0000000180034ee0 f   lutf8lib.obj
 0001:00033fb0       convert                    0000000180034fb0 f   lutf8lib.obj
 0001:000340d0       find_aux                   00000001800350d0 f   lutf8lib.obj
 0001:00034490       gmatch_aux                 0000000180035490 f   lutf8lib.obj
 0001:00034860       match                      0000000180035860 f   lutf8lib.obj
 0001:00034d60       match_class                0000000180035d60 f   lutf8lib.obj
 0001:000351c4       $LN151                     00000001800361c4     lutf8lib.obj
 0001:00035230       matchbalance               0000000180036230 f   lutf8lib.obj
 0001:00035420       matchbracketclass          0000000180036420 f   lutf8lib.obj
 0001:00035520       push_captures              0000000180036520 f   lutf8lib.obj
 0001:00035680       push_offset                0000000180036680 f   lutf8lib.obj
 0001:00035770       push_onecapture            0000000180036770 f   lutf8lib.obj
 0001:00035880       singlematch                0000000180036880 f   lutf8lib.obj
 0001:00035970       start_capture              0000000180036970 f   lutf8lib.obj
 0001:00035a00       utf8_decode                0000000180036a00 f   lutf8lib.obj
 0001:00035b30       utf8_index                 0000000180036b30 f   lutf8lib.obj
 0001:00035be0       utf8_isdigit               0000000180036be0 f   lutf8lib.obj
 0001:00035c60       utf8_isgraph               0000000180036c60 f   lutf8lib.obj
 0001:00035d80       utf8_islower               0000000180036d80 f   lutf8lib.obj
 0001:00035e00       utf8_length                0000000180036e00 f   lutf8lib.obj
 0001:00035e60       utf8_tofold                0000000180036e60 f   lutf8lib.obj
 0001:00035ec0       utf8_tolower               0000000180036ec0 f   lutf8lib.obj
 0001:00035f20       utf8_totitle               0000000180036f20 f   lutf8lib.obj
 0001:00035f80       utf8_toupper               0000000180036f80 f   lutf8lib.obj
 0001:00035fe0       utf8_width                 0000000180036fe0 f   lutf8lib.obj
 0001:00036190       io_type                    0000000180037190 f   uliolib51.obj
 0001:00036260       io_close                   0000000180037260 f   uliolib51.obj
 0001:000362f0       io_gc                      00000001800372f0 f   uliolib51.obj
 0001:00036350       io_tostring                0000000180037350 f   uliolib51.obj
 0001:000363b0       io_open                    00000001800373b0 f   uliolib51.obj
 0001:000364d0       io_popen                   00000001800374d0 f   uliolib51.obj
 0001:00036590       io_tmpfile                 0000000180037590 f   uliolib51.obj
 0001:00036640       io_input                   0000000180037640 f   uliolib51.obj
 0001:00036660       io_output                  0000000180037660 f   uliolib51.obj
 0001:00036680       f_lines                    0000000180037680 f   uliolib51.obj
 0001:000366f0       io_lines                   00000001800376f0 f   uliolib51.obj
 0001:00036840       io_read                    0000000180037840 f   uliolib51.obj
 0001:000368b0       f_read                     00000001800378b0 f   uliolib51.obj
 0001:00036910       io_write                   0000000180037910 f   uliolib51.obj
 0001:00036980       f_write                    0000000180037980 f   uliolib51.obj
 0001:000369e0       f_seek                     00000001800379e0 f   uliolib51.obj
 0001:00036ae0       f_setvbuf                  0000000180037ae0 f   uliolib51.obj
 0001:00036bd0       io_flush                   0000000180037bd0 f   uliolib51.obj
 0001:00036c90       f_flush                    0000000180037c90 f   uliolib51.obj
 0001:00036d40       f_rawhandle                0000000180037d40 f   uliolib51.obj
 0001:00036d60       aux_close                  0000000180037d60 f   uliolib51.obj
 0001:00036da0       fileerror                  0000000180037da0 f   uliolib51.obj
 0001:00036e70       g_iofile                   0000000180037e70 f   uliolib51.obj
 0001:00036f80       g_read                     0000000180037f80 f   uliolib51.obj
 0001:00037180       g_write                    0000000180038180 f   uliolib51.obj
 0001:00037290       io_fclose                  0000000180038290 f   uliolib51.obj
 0001:00037330       io_noclose                 0000000180038330 f   uliolib51.obj
 0001:00037360       io_pclose                  0000000180038360 f   uliolib51.obj
 0001:00037410       io_readline                0000000180038410 f   uliolib51.obj
 0001:000377f0       newfile                    00000001800387f0 f   uliolib51.obj
 0001:00037840       pushresult                 0000000180038840 f   uliolib51.obj
 0001:00037910       read_chars                 0000000180038910 f   uliolib51.obj
 0001:000379c0       read_line                  00000001800389c0 f   uliolib51.obj
 0001:00037ab0       ll_loadlib                 0000000180038ab0 f   uloadlib51.obj
 0001:00037b40       loader_Lua                 0000000180038b40 f   uloadlib51.obj
 0001:00037ba0       loader_C                   0000000180038ba0 f   uloadlib51.obj
 0001:00037c20       loader_Croot               0000000180038c20 f   uloadlib51.obj
 0001:00037cf0       loader_preload             0000000180038cf0 f   uloadlib51.obj
 0001:00037d90       ll_require                 0000000180038d90 f   uloadlib51.obj
 0001:00037fe0       ll_module                  0000000180038fe0 f   uloadlib51.obj
 0001:00038230       ll_seeall                  0000000180039230 f   uloadlib51.obj
 0001:000382b0       findfile                   00000001800392b0 f   uloadlib51.obj
 0001:000384d0       gctm                       00000001800394d0 f   uloadlib51.obj
 0001:00038520       ll_loadfunc                0000000180039520 f   uloadlib51.obj
 0001:00038690       loaderror                  0000000180039690 f   uloadlib51.obj
 0001:000388f0       mkfuncname                 00000001800398f0 f   uloadlib51.obj
 0001:00038960       setpath                    0000000180039960 f   uloadlib51.obj
 0001:000397e4       $LN12                      000000018003a7e4     ustring.obj
 0001:0003a2a0       ustring_OutputDebugString  000000018003b2a0 f   ustring.obj
 0001:0003a4d0       ustring_system             000000018003b4d0 f   ustring.obj
 0001:0003b880       win_GetEnv                 000000018003c880 f   win.obj
 0001:0003b950       win_SetEnv                 000000018003c950 f   win.obj
 0001:0003b9b0       win_SetRegKey              000000018003c9b0 f   win.obj
 0001:0003bc20       win_GetRegKey              000000018003cc20 f   win.obj
 0001:0003bdf0       win_DeleteRegKey           000000018003cdf0 f   win.obj
 0001:0003beb0       win_DeleteRegValue         000000018003ceb0 f   win.obj
 0001:0003bf70       win_EnumRegKey             000000018003cf70 f   win.obj
 0001:0003c0a0       win_EnumRegValue           000000018003d0a0 f   win.obj
 0001:0003c1d0       win_ExtractKey             000000018003d1d0 f   win.obj
 0001:0003c290       win_ExtractKeyEx           000000018003d290 f   win.obj
 0001:0003c330       win_GetFileInfo            000000018003d330 f   win.obj
 0001:0003c460       win_GetSystemTimeAsFileTime 000000018003d460 f   win.obj
 0001:0003c490       win_FileTimeToSystemTime   000000018003d490 f   win.obj
 0001:0003c5c0       win_SystemTimeToFileTime   000000018003d5c0 f   win.obj
 0001:0003c6e0       win_FileTimeToLocalFileTime 000000018003d6e0 f   win.obj
 0001:0003c760       win_CompareString          000000018003d760 f   win.obj
 0001:0003c8f0       win_wcscmp                 000000018003d8f0 f   win.obj
 0001:0003c970       win_GetVirtualKeys         000000018003d970 f   win.obj
 0001:0003c990       win_GetConsoleScreenBufferInfo 000000018003d990 f   win.obj
 0001:0003cad0       win_CopyFile               000000018003dad0 f   win.obj
 0001:0003cb70       win_MoveFile               000000018003db70 f   win.obj
 0001:0003cc80       win_DeleteFile             000000018003dc80 f   win.obj
 0001:0003ccd0       win_CreateDir              000000018003dcd0 f   win.obj
 0001:0003cdf0       win_RemoveDir              000000018003ddf0 f   win.obj
 0001:0003ce40       win_ShellExecute           000000018003de40 f   win.obj
 0001:0003cf20       win_IsProcess64bit         000000018003df20 f   win.obj
 0001:0003d940       CheckHKey                  000000018003e940 f   win.obj
 0001:0003db10       mkdir                      000000018003eb10 f   win.obj
 0001:0003df34       ?dllmain_crt_dispatch@@YAHQEAUHINSTANCE__@@KQEAX@Z 000000018003ef34 f   LIBCMT:dll_dllmain.obj
 0001:0003df84       ?dllmain_crt_process_attach@@YAHQEAUHINSTANCE__@@QEAX@Z 000000018003ef84 f   LIBCMT:dll_dllmain.obj
 0001:0003e0a0       ?dllmain_crt_process_detach@@YAH_N@Z 000000018003f0a0 f   LIBCMT:dll_dllmain.obj
 0001:0003e130       ?dllmain_dispatch@@YAHQEAUHINSTANCE__@@KQEAX@Z 000000018003f130 f   LIBCMT:dll_dllmain.obj
 0001:0003eb30       $$000000                   000000018003fb30     libvcruntime:memcpy.obj
 0001:0003ebe7       MoveSmall                  000000018003fbe7     libvcruntime:memcpy.obj
 0001:0003ef90       $$000000                   000000018003ff90     libvcruntime:memset.obj
 0001:0003f08c       MsetTab                    000000018004008c     libvcruntime:memset.obj
 0001:0003f490       $$000000                   0000000180040490     libvcruntime:memchr.obj
 0001:0003f510       $$000000                   0000000180040510     libvcruntime:memcmp.obj
 0001:0003fa00       $$000000                   0000000180040a00     libvcruntime:notify.obj
 0001:0003fd28       ?try_get_function@@YAPEAXW4function_id@?A0x14c33c87@@QEBDQEBW4module_id@2@2@Z 0000000180040d28 f   libvcruntime:winapi_downlevel.obj
 0001:00040110       $$000000                   0000000180041110     libvcruntime:handlers.obj
 0001:000401b8       ??$?RV<lambda_a62c933ada0517137acf5807a1eeac1f>@@AEAV<lambda_a31071773b9a94e445cbd5d04ef99106>@@V<lambda_56065050dbf3ada7e59a83db45153de3>@@@?$__crt_seh_guarded_call@H@@QEAAH$$QEAV<lambda_a62c933ada0517137acf5807a1eeac1f>@@AEAV<lambda_a31071773b9a94e445cbd5d04ef99106>@@$$QEAV<lambda_56065050dbf3ada7e59a83db45153de3>@@@Z 00000001800411b8 f   libucrt:output.obj
 0001:000401f8       ??$common_vsprintf@Vstandard_base@__crt_stdio_output@@D@@YAH_KQEAD0QEBDQEAU__crt_locale_pointers@@1@Z 00000001800411f8 f   libucrt:output.obj
 0001:000403c4       ??$common_vsprintf@Vstandard_base@__crt_stdio_output@@_W@@YAH_KQEA_W0QEB_WQEAU__crt_locale_pointers@@QEAD@Z 00000001800413c4 f   libucrt:output.obj
 0001:00040bb4       ??R<lambda_a31071773b9a94e445cbd5d04ef99106>@@QEBAHXZ 0000000180041bb4 f   libucrt:output.obj
 0001:000436d8       ??$common_fsopen@_W@@YAPEAU_iobuf@@QEB_W0H@Z 00000001800446d8 f   libucrt:fopen.obj
 0001:00043910       common_control87           0000000180044910 f   libucrt:ieee.obj
 0001:00043ef8       ??$common_freopen@_W@@YAHQEAPEAU_iobuf@@QEB_W1V__crt_stdio_stream@@H@Z 0000000180044ef8 f   libucrt:freopen.obj
 0001:00044780       $$000000                   0000000180045780     libucrt:strcmp.obj
 0001:00044b70       $$000000                   0000000180045b70     libucrt:strncmp.obj
 0001:00044c00       $$000000                   0000000180045c00     libucrt:strncpy.obj
 0001:00044d74       fallbackMethod             0000000180045d74 f   libucrt:strpbrk.obj
 0001:00045144       $LN78                      0000000180046144     libucrt:strpbrk.obj
 0001:00045180       $LN77                      0000000180046180     libucrt:strpbrk.obj
 0001:000451c0       $LN76                      00000001800461c0     libucrt:strpbrk.obj
 0001:00045200       ??$common_popen@_W@@YAPEAU_iobuf@@QEB_W0@Z 0000000180046200 f   libucrt:popen.obj
 0001:000453cc       ??$common_popen_nolock@_W@@YAPEAU_iobuf@@QEB_W0HAEAY01H@Z 00000001800463cc f   libucrt:popen.obj
 0001:000456ec       ??$get_executable_path@_W@@YAPEB_WQEB_W@Z 00000001800466ec f   libucrt:popen.obj
 0001:00045884       ?idtab@@YAPEAUprocess_handle_pair@?A0xe43b7539@@QEAU_iobuf@@@Z 0000000180046884 f   libucrt:popen.obj
 0001:00045a9c       ??$?RV<lambda_842d9ff0dc9ef11c61343bbaebe7f885>@@AEAV<lambda_c5860995281e5c4ce005b3de8f5874ee>@@V<lambda_d90129c13df834fdcbf8d2b88dafcf2d>@@@?$__crt_seh_guarded_call@X@@QEAAX$$QEAV<lambda_842d9ff0dc9ef11c61343bbaebe7f885>@@AEAV<lambda_c5860995281e5c4ce005b3de8f5874ee>@@$$QEAV<lambda_d90129c13df834fdcbf8d2b88dafcf2d>@@@Z 0000000180046a9c f   libucrt:fflush.obj
 0001:00045b38       ??$?RV<lambda_886d6c58226a84441f68b9f2b8217b83>@@AEAV<lambda_ab61a845afdef5b7c387490eaf3616ee>@@V<lambda_f7f22ab5edc0698d5f6905b0d3f44752>@@@?$__crt_seh_guarded_call@X@@QEAAX$$QEAV<lambda_886d6c58226a84441f68b9f2b8217b83>@@AEAV<lambda_ab61a845afdef5b7c387490eaf3616ee>@@$$QEAV<lambda_f7f22ab5edc0698d5f6905b0d3f44752>@@@Z 0000000180046b38 f   libucrt:fflush.obj
 0001:00045c18       ??$?RV<lambda_c376a267cfb53b6959b3b692ec76b120>@@AEAV<lambda_9a32fed5bf61b6b509b2d3f6003082a1>@@V<lambda_572fbb9fa0ab338edf41edfd4b5fcc8d>@@@?$__crt_seh_guarded_call@H@@QEAAH$$QEAV<lambda_c376a267cfb53b6959b3b692ec76b120>@@AEAV<lambda_9a32fed5bf61b6b509b2d3f6003082a1>@@$$QEAV<lambda_572fbb9fa0ab338edf41edfd4b5fcc8d>@@@Z 0000000180046c18 f   libucrt:fflush.obj
 0001:00045c58       ?common_flush_all@@YAH_N@Z 0000000180046c58 f   libucrt:fflush.obj
 0001:00045df0       ??$common_fgets@D@@YAPEADQEADHV__crt_stdio_stream@@@Z 0000000180046df0 f   libucrt:fgets.obj
 0001:00045ec4       ?common_fseek@@YAHV__crt_stdio_stream@@_JH@Z 0000000180046ec4 f   libucrt:fseek.obj
 0001:00045f30       ?common_fseek_binary_mode_read_only_fast_track_nolock@@YA_NV__crt_stdio_stream@@_JH@Z 0000000180046f30 f   libucrt:fseek.obj
 0001:00046014       ?common_fseek_nolock@@YAHV__crt_stdio_stream@@_JH@Z 0000000180047014 f   libucrt:fseek.obj
 0001:000460d4       ??$common_ftell@J@@YAJV__crt_stdio_stream@@@Z 00000001800470d4 f   libucrt:ftell.obj
 0001:00046144       ??$common_ftell_nolock@_J@@YA_JV__crt_stdio_stream@@@Z 0000000180047144 f   libucrt:ftell.obj
 0001:00046274       ?common_ftell_read_mode_nolock@@YA_JV__crt_stdio_stream@@_J1@Z 0000000180047274 f   libucrt:ftell.obj
 0001:000463c0       ?common_ftell_translated_utf8_nolock@@YA_JV__crt_stdio_stream@@_J@Z 00000001800473c0 f   libucrt:ftell.obj
 0001:0004653c       ?count_newline_bytes@@YA_JQEBD0W4__crt_lowio_text_mode@@@Z 000000018004753c f   libucrt:ftell.obj
 0001:000465d0       ??$?RV<lambda_bdbcead8b570fa3d5ec6d9679862a6e5>@@AEAV<lambda_96f4279ff90247a4c5c5d9824f56f8c1>@@V<lambda_4606be27f17b5e5579e09050fab91818>@@@?$__crt_seh_guarded_call@_K@@QEAA_K$$QEAV<lambda_bdbcead8b570fa3d5ec6d9679862a6e5>@@AEAV<lambda_96f4279ff90247a4c5c5d9824f56f8c1>@@$$QEAV<lambda_4606be27f17b5e5579e09050fab91818>@@@Z 00000001800475d0 f   libucrt:fwrite.obj
 0001:00046610       ??R<lambda_96f4279ff90247a4c5c5d9824f56f8c1>@@QEBA_KXZ 0000000180047610 f   libucrt:fwrite.obj
 0001:000468a4       ??$?RV<lambda_84ec643ea9557e2f7dc01bb0e9624395>@@AEAV<lambda_ca71763b3c0644891230e4f79ea54fa6>@@V<lambda_439a761618c59b0600e24586724d733b>@@@?$__crt_seh_guarded_call@H@@QEAAH$$QEAV<lambda_84ec643ea9557e2f7dc01bb0e9624395>@@AEAV<lambda_ca71763b3c0644891230e4f79ea54fa6>@@$$QEAV<lambda_439a761618c59b0600e24586724d733b>@@@Z 00000001800478a4 f   libucrt:setvbuf.obj
 0001:000468e4       ??R<lambda_ca71763b3c0644891230e4f79ea54fa6>@@QEBAHXZ 00000001800478e4 f   libucrt:setvbuf.obj
 0001:00046a60       ??$generate_tmpfile_file_name@D@@YA_NQEAD_K@Z 0000000180047a60 f   libucrt:tmpfile.obj
 0001:00046afc       ??$get_tmpfile_buffer_nolock@D@@YAPEADW4buffer_id@?A0x5b9a7937@@@Z 0000000180047afc f   libucrt:tmpfile.obj
 0001:00046b40       ??$initialize_tmpfile_buffer_nolock@D@@YA_NW4buffer_id@?A0x5b9a7937@@@Z 0000000180047b40 f   libucrt:tmpfile.obj
 0001:00046c1c       ?common_tmpfile@@YAHQEAPEAU_iobuf@@H@Z 0000000180047c1c f   libucrt:tmpfile.obj
 0001:00046c80       ?common_tmpfile_nolock@@YAHQEAPEAU_iobuf@@H@Z 0000000180047c80 f   libucrt:tmpfile.obj
 0001:00046eac       ??$?RV<lambda_082dd7c0feb7dbdaf245f261e54a6583>@@AEAV<lambda_f3caf1ecae5fe01a9a1a6239afa44510>@@V<lambda_c640b76c0755ae85b317b35c67c61e6b>@@@?$__crt_seh_guarded_call@H@@QEAAH$$QEAV<lambda_082dd7c0feb7dbdaf245f261e54a6583>@@AEAV<lambda_f3caf1ecae5fe01a9a1a6239afa44510>@@$$QEAV<lambda_c640b76c0755ae85b317b35c67c61e6b>@@@Z 0000000180047eac f   libucrt:input.obj
 0001:00048c44       ??R<lambda_156378f40168adef48d7ddfcff3a1264>@@QEBA_NXZ 0000000180049c44 f   libucrt:input.obj
 0001:00048cc0       ??R<lambda_f3caf1ecae5fe01a9a1a6239afa44510>@@QEBAHXZ 0000000180049cc0 f   libucrt:input.obj
 0001:0004c364       memcpy_s                   000000018004d364 f   libucrt:cfout.obj
 0001:0004c364       memcpy_s                   000000018004d364 f   libucrt:input.obj
 0001:0004c3ec       ??$common_dupenv_s@_W@@YAHQEAPEA_WQEA_KQEB_WHQEBDH@Z 000000018004d3ec f   libucrt:getenv.obj
 0001:0004c4e0       ??$common_getenv@_W@@YAPEA_WQEB_W@Z 000000018004d4e0 f   libucrt:getenv.obj
 0001:0004c540       ??$common_getenv_nolock@_W@@YAPEA_WQEB_W@Z 000000018004d540 f   libucrt:getenv.obj
 0001:0004c9ac       ??$?RV<lambda_d80eeec6fff315bfe5c115232f3240e3>@@AEAV<lambda_6e4b09c48022b2350581041d5f6b0c4c>@@V<lambda_2358e3775559c9db80273638284d5e45>@@@?$__crt_seh_guarded_call@X@@QEAAX$$QEAV<lambda_d80eeec6fff315bfe5c115232f3240e3>@@AEAV<lambda_6e4b09c48022b2350581041d5f6b0c4c>@@$$QEAV<lambda_2358e3775559c9db80273638284d5e45>@@@Z 000000018004d9ac f   libucrt:exit.obj
 0001:0004c9e4       ??R<lambda_6e4b09c48022b2350581041d5f6b0c4c>@@QEBA@XZ 000000018004d9e4 f   libucrt:exit.obj
 0001:0004caa8       ?atexit_exception_filter@@YAHK@Z 000000018004daa8 f   libucrt:exit.obj
 0001:0004cab4       ?common_exit@@YAXHW4_crt_exit_cleanup_mode@@W4_crt_exit_return_mode@@@Z 000000018004dab4 f   libucrt:exit.obj
 0001:0004cb70       ?exit_or_terminate_process@@YAXI@Z 000000018004db70 f   libucrt:exit.obj
 0001:0004cbbc       ?try_cor_exit_process@@YAXI@Z 000000018004dbbc f   libucrt:exit.obj
 0001:0004cc44       ??$parse_command_line@D@@YAXPEADPEAPEAD0PEA_K2@Z 000000018004dc44 f   libucrt:argv_parsing.obj
 0001:0004cff0       ??$common_initialize_environment_nolock@D@@YAHXZ 000000018004dff0 f   libucrt:environment_initialization.obj
 0001:0004d05c       ??$common_initialize_environment_nolock@_W@@YAHXZ 000000018004e05c f   libucrt:environment_initialization.obj
 0001:0004d0c4       ??$create_environment@D@@YAQEAPEADQEAD@Z 000000018004e0c4 f   libucrt:environment_initialization.obj
 0001:0004d1cc       ??$create_environment@_W@@YAQEAPEA_WQEA_W@Z 000000018004e1cc f   libucrt:environment_initialization.obj
 0001:0004d2e0       ??$free_environment@D@@YAXQEAPEAD@Z 000000018004e2e0 f   libucrt:environment_initialization.obj
 0001:0004d2e0       ??$free_environment@_W@@YAXQEAPEA_W@Z 000000018004e2e0 f   libucrt:environment_initialization.obj
 0001:0004d324       ??$initialize_environment_by_cloning_nolock@_W@@YAHXZ 000000018004e324 f   libucrt:environment_initialization.obj
 0001:0004d3d8       ??$uninitialize_environment_internal@D@@YAXAEAPEAPEAD@Z 000000018004e3d8 f   libucrt:environment_initialization.obj
 0001:0004d3f4       ??$uninitialize_environment_internal@_W@@YAXAEAPEAPEA_W@Z 000000018004e3f4 f   libucrt:environment_initialization.obj
 0001:0004d48c       ??$?RV<lambda_7777bce6b2f8c936911f934f8298dc43>@@AEAV<lambda_f03950bc5685219e0bcd2087efbe011e>@@V<lambda_3883c3dff614d5e0c5f61bb1ac94921c>@@@?$__crt_seh_guarded_call@H@@QEAAH$$QEAV<lambda_7777bce6b2f8c936911f934f8298dc43>@@AEAV<lambda_f03950bc5685219e0bcd2087efbe011e>@@$$QEAV<lambda_3883c3dff614d5e0c5f61bb1ac94921c>@@@Z 000000018004e48c f   libucrt:onexit.obj
 0001:0004d4c8       ??R<lambda_f03950bc5685219e0bcd2087efbe011e>@@QEBAHXZ 000000018004e4c8 f   libucrt:onexit.obj
 0001:0004d644       initialize_global_variables 000000018004e644 f   libucrt:initialization.obj
 0001:0004d658       initialize_c               000000018004e658 f   libucrt:initialization.obj
 0001:0004d67c       uninitialize_global_state_isolation 000000018004e67c f   libucrt:initialization.obj
 0001:0004d67c       initialize_environment     000000018004e67c f   libucrt:initialization.obj
 0001:0004d67c       initialize_global_state_isolation 000000018004e67c f   libucrt:initialization.obj
 0001:0004d67c       uninitialize_c             000000018004e67c f   libucrt:initialization.obj
 0001:0004d67c       report_memory_leaks        000000018004e67c f   libucrt:initialization.obj
 0001:0004d680       uninitialize_environment   000000018004e680 f   libucrt:initialization.obj
 0001:0004d690       initialize_pointers        000000018004e690 f   libucrt:initialization.obj
 0001:0004d6d0       uninitialize_vcruntime     000000018004e6d0 f   libucrt:initialization.obj
 0001:0004d6d8       uninitialize_allocated_memory 000000018004e6d8 f   libucrt:initialization.obj
 0001:0004d718       uninitialize_allocated_io_buffers 000000018004e718 f   libucrt:initialization.obj
 0001:0004d814       ?_strupr_s_l_stat@@YAHQEAD_KQEAU__crt_locale_pointers@@@Z 000000018004e814 f   libucrt:strupr.obj
 0001:0004ec88       ?internal_isupper_l@@YA_NHQEAU__crt_locale_pointers@@@Z 000000018004fc88 f   libucrt:tolower_toupper.obj
 0001:0004f5d8       ??$?RV<lambda_0ae27a3a962d80f24befdcbee591983d>@@AEAV<lambda_8d0ee55de4b1038c4002e0adecdf1839>@@V<lambda_dc504788e8f1664fe9b84e20bfb512f2>@@@?$__crt_seh_guarded_call@X@@QEAAX$$QEAV<lambda_0ae27a3a962d80f24befdcbee591983d>@@AEAV<lambda_8d0ee55de4b1038c4002e0adecdf1839>@@$$QEAV<lambda_dc504788e8f1664fe9b84e20bfb512f2>@@@Z 00000001800505d8 f   libucrt:per_thread_data.obj
 0001:0004f618       ??$?RV<lambda_2d41944a1d46af3157314b8a01080d33>@@AEAV<lambda_8f455de75cd7d7f24b4096f044d8b9e6>@@V<lambda_aa500f224e6afead328df44964fe2772>@@@?$__crt_seh_guarded_call@X@@QEAAX$$QEAV<lambda_2d41944a1d46af3157314b8a01080d33>@@AEAV<lambda_8f455de75cd7d7f24b4096f044d8b9e6>@@$$QEAV<lambda_aa500f224e6afead328df44964fe2772>@@@Z 0000000180050618 f   libucrt:per_thread_data.obj
 0001:0004f658       ??$?RV<lambda_aa87e3671a710a21b5dc78c0bdf72e11>@@AEAV<lambda_92619d2358a28f41a33ba319515a20b9>@@V<lambda_6992ecaafeb10aed2b74cb1fae11a551>@@@?$__crt_seh_guarded_call@X@@QEAAX$$QEAV<lambda_aa87e3671a710a21b5dc78c0bdf72e11>@@AEAV<lambda_92619d2358a28f41a33ba319515a20b9>@@$$QEAV<lambda_6992ecaafeb10aed2b74cb1fae11a551>@@@Z 0000000180050658 f   libucrt:per_thread_data.obj
 0001:0004f6a0       ??$?RV<lambda_f2e299630e499de9f9a165e60fcd3db5>@@AEAV<lambda_2ae9d31cdba2644fcbeaf08da7c24588>@@V<lambda_40d01ff24d0e7b3814fdbdcee8eab3c7>@@@?$__crt_seh_guarded_call@X@@QEAAX$$QEAV<lambda_f2e299630e499de9f9a165e60fcd3db5>@@AEAV<lambda_2ae9d31cdba2644fcbeaf08da7c24588>@@$$QEAV<lambda_40d01ff24d0e7b3814fdbdcee8eab3c7>@@@Z 00000001800506a0 f   libucrt:per_thread_data.obj
 0001:0004f700       ?construct_ptd_array@@YAXQEAU__acrt_ptd@@@Z 0000000180050700 f   libucrt:per_thread_data.obj
 0001:0004f7d0       ?destroy_fls@@YAXPEAX@Z    00000001800507d0 f   libucrt:per_thread_data.obj
 0001:0004f7f0       ?destroy_ptd_array@@YAXQEAU__acrt_ptd@@@Z 00000001800507f0 f   libucrt:per_thread_data.obj
 0001:0004f8e8       ?replace_current_thread_locale_nolock@@YAXQEAU__acrt_ptd@@QEAU__crt_locale_data@@@Z 00000001800508e8 f   libucrt:per_thread_data.obj
 0001:0004fca4       ?fp_format_a@@YAHQEBNPEAD_KQEAD2H_NIQEAU__crt_locale_pointers@@@Z 0000000180050ca4 f   libucrt:cvt.obj
 0001:00050014       ?fp_format_e@@YAHQEBNQEAD_K12H_NIQEAU__crt_locale_pointers@@@Z 0000000180051014 f   libucrt:cvt.obj
 0001:000500f0       ?fp_format_e_internal@@YAHQEAD_KH_NIQEAU_strflt@@2QEAU__crt_locale_pointers@@@Z 00000001800510f0 f   libucrt:cvt.obj
 0001:000502c4       ?fp_format_f_internal@@YAHQEAD_KHQEAU_strflt@@_NQEAU__crt_locale_pointers@@@Z 00000001800512c4 f   libucrt:cvt.obj
 0001:00050408       ?fp_format_g@@YAHQEBNQEAD_K12H_NIQEAU__crt_locale_pointers@@@Z 0000000180051408 f   libucrt:cvt.obj
 0001:0005053c       ?fp_format_nan_or_infinity@@YAHW4__acrt_fp_class@@_NPEAD_K1@Z 000000018005153c f   libucrt:cvt.obj
 0001:00050a64       ??$?RV<lambda_410d79af7f07d98d83a3f525b3859a53>@@AEAV<lambda_3e16ef9562a7dcce91392c22ab16ea36>@@V<lambda_38119f0e861e05405d8a144b9b982f0a>@@@?$__crt_seh_guarded_call@X@@QEAAX$$QEAV<lambda_410d79af7f07d98d83a3f525b3859a53>@@AEAV<lambda_3e16ef9562a7dcce91392c22ab16ea36>@@$$QEAV<lambda_38119f0e861e05405d8a144b9b982f0a>@@@Z 0000000180051a64 f   libucrt:wsetlocale.obj
 0001:00050b10       ?initialize_inherited_file_handles_nolock@@YAXXZ 0000000180051b10 f   libucrt:ioinit.obj
 0001:00050c00       ?initialize_stdio_handles_nolock@@YAXXZ 0000000180051c00 f   libucrt:ioinit.obj
 0001:00050e64       ?find_or_allocate_unused_stream_nolock@@YA?AV__crt_stdio_stream@@XZ 0000000180051e64 f   libucrt:stream.obj
 0001:000512f0       ??$?RV<lambda_751a882b2c74d4b022dec766aa51a29a>@@AEAV<lambda_628dfdc04ba53c8bfc02c9951375f3f5>@@V<lambda_f6c7be5f7998530c34de24c7437d6b54>@@@?$__crt_seh_guarded_call@H@@QEAAH$$QEAV<lambda_751a882b2c74d4b022dec766aa51a29a>@@AEAV<lambda_628dfdc04ba53c8bfc02c9951375f3f5>@@$$QEAV<lambda_f6c7be5f7998530c34de24c7437d6b54>@@@Z 00000001800522f0 f   libucrt:close.obj
 0001:00051510       $$000000                   0000000180052510     libucrt:fpsr.obj
 0001:000516cc       ?try_get_function@@YAPEAXW4function_id@?A0x391cf84c@@QEBDQEBW4module_id@2@2@Z 00000001800526cc f   libucrt:winapi_thunks.obj
 0001:00051df4       ??$translate_text_mode_nolock@D@@YAHHQEAD_K@Z 0000000180052df4 f   libucrt:read.obj
 0001:00051fc0       ??$translate_text_mode_nolock@_W@@YAHHQEA_W_K@Z 0000000180052fc0 f   libucrt:read.obj
 0001:0005222c       ?translate_ansi_or_utf8_nolock@@YAHHQEAD_KQEA_W1@Z 000000018005322c f   libucrt:read.obj
 0001:00052aa8       ??$common_lseek@J@@YAJHJH@Z 0000000180053aa8 f   libucrt:lseek.obj
 0001:00052b94       ??$common_lseek@_J@@YA_JH_JH@Z 0000000180053b94 f   libucrt:lseek.obj
 0001:00052c84       ??$common_lseek_nolock@J@@YAJHJH@Z 0000000180053c84 f   libucrt:lseek.obj
 0001:00052d78       ??$common_lseek_nolock@_J@@YA_JH_JH@Z 0000000180053d78 f   libucrt:lseek.obj
 0001:000538e4       ??$common_fdopen@_W@@YAPEAU_iobuf@@HQEB_W@Z 00000001800548e4 f   libucrt:fdopen.obj
 0001:000539d8       ??$?RV<lambda_a37b2b86f63e897a80ea819b0eb08c01>@@AEAV<lambda_38ce7e780aa69e748d6df282ebc68efe>@@V<lambda_99fb1378e971ab6e7edea83e3a7a83a2>@@@?$__crt_seh_guarded_call@H@@QEAAH$$QEAV<lambda_a37b2b86f63e897a80ea819b0eb08c01>@@AEAV<lambda_38ce7e780aa69e748d6df282ebc68efe>@@$$QEAV<lambda_99fb1378e971ab6e7edea83e3a7a83a2>@@@Z 00000001800549d8 f   libucrt:commit.obj
 0001:00053af8       ?write_double_translated_ansi_nolock@@YA?AUwrite_result@?A0x17268360@@HQEBDI@Z 0000000180054af8 f   libucrt:write.obj
 0001:00053fd4       ?write_text_ansi_nolock@@YA?AUwrite_result@?A0x17268360@@HQEBDI@Z 0000000180054fd4 f   libucrt:write.obj
 0001:000540d8       ?write_text_utf16le_nolock@@YA?AUwrite_result@?A0x17268360@@HQEBDI@Z 00000001800550d8 f   libucrt:write.obj
 0001:000541f4       ?write_text_utf8_nolock@@YA?AUwrite_result@?A0x17268360@@HQEBDI@Z 00000001800551f4 f   libucrt:write.obj
 0001:0005472c       ??$write_buffer_nolock@D@@YA_NDV__crt_stdio_stream@@@Z 000000018005572c f   libucrt:_flsbuf.obj
 0001:00054810       ?stream_is_at_end_of_file_nolock@@YA_NV__crt_stdio_stream@@@Z 0000000180055810 f   libucrt:_flsbuf.obj
 0001:00054974       ??$common_xtox@_KD@@YAH_KQEAD0I_N@Z 0000000180055974 f   libucrt:xtoa.obj
 0001:00054a40       ??$common_xtox_s@_KD@@YAH_KQEAD0I_N@Z 0000000180055a40 f   libucrt:xtoa.obj
 0001:00054bdc       ??$common_sopen_dispatch@D@@YAHQEBDHHHQEAHH@Z 0000000180055bdc f   libucrt:open.obj
 0001:00054ca0       ??$common_sopen_dispatch@_W@@YAHQEB_WHHHQEAHH@Z 0000000180055ca0 f   libucrt:open.obj
 0001:00054d64       ?configure_text_mode@@YAHHUfile_options@?A0xa9d50aae@@HAEAW4__crt_lowio_text_mode@@@Z 0000000180055d64 f   libucrt:open.obj
 0001:00054ff8       ?decode_options@@YA?AUfile_options@?A0xa9d50aae@@HHH@Z 0000000180055ff8 f   libucrt:open.obj
 0001:00055204       ?truncate_ctrl_z_if_present@@YAHH@Z 0000000180056204 f   libucrt:open.obj
 0001:00055ae0       ??$?RV<lambda_a22f0c497e5168315e06dae667770027>@@AEAV<lambda_a094494068278ba5130ab06e1292f60a>@@V<lambda_24dc10c13f43218c635520766e23e324>@@@?$__crt_seh_guarded_call@_N@@QEAA_N$$QEAV<lambda_a22f0c497e5168315e06dae667770027>@@AEAV<lambda_a094494068278ba5130ab06e1292f60a>@@$$QEAV<lambda_24dc10c13f43218c635520766e23e324>@@@Z 0000000180056ae0 f   libucrt:spawnv.obj
 0001:00055b20       ??$common_spawnv@_W@@YA_JHQEB_WQEBQEB_W1@Z 0000000180056b20 f   libucrt:spawnv.obj
 0001:00055d70       ??$execute_command@_W@@YA_JHQEB_WQEBQEB_W1@Z 0000000180056d70 f   libucrt:spawnv.obj
 0001:00055fd0       ??R<lambda_a094494068278ba5130ab06e1292f60a>@@QEBA_NXZ 0000000180056fd0 f   libucrt:spawnv.obj
 0001:000561cc       ?accumulate_inheritable_handles@@YA_NQEAPEAEQEA_K_N@Z 00000001800571cc f   libucrt:spawnv.obj
 0001:0005622c       ??$common_spawnvp@_W@@YA_JHQEB_WQEBQEB_W1@Z 000000018005722c f   libucrt:spawnvp.obj
 0001:00056598       ?<lambda_invoker_cdecl>@<lambda_c2303d2482d7c3675ea2e24c4cfb6115>@@CAHPEBX0@Z 0000000180057598 f   libucrt:argv_wildcards.obj
 0001:00056738       ??$common_expand_argv_wildcards@D@@YAHQEAPEADQEAPEAPEAD@Z 0000000180057738 f   libucrt:argv_wildcards.obj
 0001:00056944       ??$copy_and_add_argument_to_buffer@D@@YAHQEBD0_KAEAV?$argument_list@D@?A0x5f5c8891@@@Z 0000000180057944 f   libucrt:argv_wildcards.obj
 0001:00056acc       ??$expand_argument_wildcards@D@@YAHQEAD0AEAV?$argument_list@D@?A0x5f5c8891@@@Z 0000000180057acc f   libucrt:argv_wildcards.obj
 0001:00057018       ??$?RV<lambda_efdfa57d1f175319df784efa44bb7b81>@@AEAV<lambda_5f0a4c1567f8adc6734073e5d1e1b35c>@@V<lambda_2e8a7d3640ea6ccb4c2413664c2db6fd>@@@?$__crt_seh_guarded_call@X@@QEAAX$$QEAV<lambda_efdfa57d1f175319df784efa44bb7b81>@@AEAV<lambda_5f0a4c1567f8adc6734073e5d1e1b35c>@@$$QEAV<lambda_2e8a7d3640ea6ccb4c2413664c2db6fd>@@@Z 0000000180058018 f   libucrt:mbctype.obj
 0001:000571d4       ?getSystemCP@@YAHH@Z       00000001800581d4 f   libucrt:mbctype.obj
 0001:00057254       ?setSBCS@@YAXPEAU__crt_multibyte_data@@@Z 0000000180058254 f   libucrt:mbctype.obj
 0001:000572e4       ?setSBUpLow@@YAXPEAU__crt_multibyte_data@@@Z 00000001800582e4 f   libucrt:mbctype.obj
 0001:000574c8       ?setmbcp_internal@@YAHH_NQEAU__acrt_ptd@@QEAPEAU__crt_multibyte_data@@@Z 00000001800584c8 f   libucrt:mbctype.obj
 0001:0005768c       ?update_thread_multibyte_data_internal@@YAPEAU__crt_multibyte_data@@QEAU__acrt_ptd@@QEAPEAU1@@Z 000000018005868c f   libucrt:mbctype.obj
 0001:00057a7c       ?x_ismbbtype_l@@YAHPEAU__crt_locale_pointers@@IHH@Z 0000000180058a7c f   libucrt:ismbbyte.obj
 0001:00057dc8       ??$common_set_variable_in_environment_nolock@_W@@YAHQEA_WH@Z 0000000180058dc8 f   libucrt:setenv.obj
 0001:000580ec       ??$copy_environment@_W@@YAPEAPEA_WQEAPEA_W@Z 00000001800590ec f   libucrt:setenv.obj
 0001:00058334       ??$?RV<lambda_450d765d439847d4c735a33c368b5fc0>@@AEAV<lambda_44731a7d0e6d81c3e6aa82d741081786>@@V<lambda_601a2a7da3b7a96e9554ac7215c4b07c>@@@?$__crt_seh_guarded_call@P6AXH@Z@@QEAAP6AXH@Z$$QEAV<lambda_450d765d439847d4c735a33c368b5fc0>@@AEAV<lambda_44731a7d0e6d81c3e6aa82d741081786>@@$$QEAV<lambda_601a2a7da3b7a96e9554ac7215c4b07c>@@@Z 0000000180059334 f   libucrt:signal.obj
 0001:00058690       ?__acrt_LCMapStringA_stat@@YAHPEAU__crt_locale_pointers@@PEB_WKPEBDHPEADHHH@Z 0000000180059690 f   libucrt:lcmapstringa.obj
 0001:0005a5fc       ?free_crt_array_internal@@YAXQEAPEBX_K@Z 000000018005b5fc f   libucrt:inittime.obj
 0001:0005afe4       ?GetTableIndexFromLocaleName@@YAHPEB_W@Z 000000018005bfe4 f   libucrt:lcidtoname_downlevel.obj
 0001:0005b8d8       ??$construct_environment_block@_W@@YAHQEBQEB_WQEAPEA_W@Z 000000018005c8d8 f   libucrt:cenvarg.obj
 0001:0005c1dc       ?initialize_multibyte@@YAHXZ 000000018005d1dc f   libucrt:multibyte_initializer.obj
 0001:0005c570       $$000000                   000000018005d570     libucrt:log10.obj
 0001:0005cc54       _call_matherr              000000018005dc54 f   libucrt:libm_error.obj
 0001:0005ccbc       _exception_enabled         000000018005dcbc f   libucrt:libm_error.obj
 0001:0005cf50       _log_special_common        000000018005df50 f   libucrt:log_special.obj
 0001:0005d580       $$000000                   000000018005e580     LIBCMT:amdsecgs.obj
 0001:0005d7f4       capture_current_context    000000018005e7f4 f   LIBCMT:gs_report.obj
 0001:0005d864       capture_previous_context   000000018005e864 f   LIBCMT:gs_report.obj
 0001:0005d910       $$000000                   000000018005e910     LIBCMT:guard_dispatch.obj
 0001:0005d930       ?fin$0@?0??dllmain_crt_process_attach@@YAHQEAUHINSTANCE__@@QEAX@Z@4HA 000000018005e930 f   LIBCMT:dll_dllmain.obj
 0001:0005d947       ?fin$0@?0??dllmain_crt_process_detach@@YAH_N@Z@4HA 000000018005e947 f   LIBCMT:dll_dllmain.obj
 0001:0005d963       ?filt$0@?0??dllmain_dispatch@@YAHQEAUHINSTANCE__@@KQEAX@Z@4HA 000000018005e963 f   LIBCMT:dll_dllmain.obj
 0001:0005d999       __scrt_is_nonwritable_in_current_image$filt$0 000000018005e999 f   LIBCMT:utility.obj
 0001:0005d9b1       __DestructExceptionObject$filt$0 000000018005e9b1 f   libvcruntime:ehhelpers.obj
 0001:0005d9c9       ?fin$0@?0???$?RV<lambda_842d9ff0dc9ef11c61343bbaebe7f885>@@AEAV<lambda_c5860995281e5c4ce005b3de8f5874ee>@@V<lambda_d90129c13df834fdcbf8d2b88dafcf2d>@@@?$__crt_seh_guarded_call@X@@QEAAX$$QEAV<lambda_842d9ff0dc9ef11c61343bbaebe7f885>@@AEAV<lambda_c5860995281e5c4ce005b3de8f5874ee>@@$$QEAV<lambda_d90129c13df834fdcbf8d2b88dafcf2d>@@@Z@4HA 000000018005e9c9 f   libucrt:fflush.obj
 0001:0005d9c9       ?fin$0@?0???$?RV<lambda_082dd7c0feb7dbdaf245f261e54a6583>@@AEAV<lambda_f3caf1ecae5fe01a9a1a6239afa44510>@@V<lambda_c640b76c0755ae85b317b35c67c61e6b>@@@?$__crt_seh_guarded_call@H@@QEAAH$$QEAV<lambda_082dd7c0feb7dbdaf245f261e54a6583>@@AEAV<lambda_f3caf1ecae5fe01a9a1a6239afa44510>@@$$QEAV<lambda_c640b76c0755ae85b317b35c67c61e6b>@@@Z@4HA 000000018005e9c9 f   libucrt:input.obj
 0001:0005d9c9       ?fin$0@?0???$?RV<lambda_84ec643ea9557e2f7dc01bb0e9624395>@@AEAV<lambda_ca71763b3c0644891230e4f79ea54fa6>@@V<lambda_439a761618c59b0600e24586724d733b>@@@?$__crt_seh_guarded_call@H@@QEAAH$$QEAV<lambda_84ec643ea9557e2f7dc01bb0e9624395>@@AEAV<lambda_ca71763b3c0644891230e4f79ea54fa6>@@$$QEAV<lambda_439a761618c59b0600e24586724d733b>@@@Z@4HA 000000018005e9c9 f   libucrt:setvbuf.obj
 0001:0005d9c9       ?fin$0@?0???$?RV<lambda_a62c933ada0517137acf5807a1eeac1f>@@AEAV<lambda_a31071773b9a94e445cbd5d04ef99106>@@V<lambda_56065050dbf3ada7e59a83db45153de3>@@@?$__crt_seh_guarded_call@H@@QEAAH$$QEAV<lambda_a62c933ada0517137acf5807a1eeac1f>@@AEAV<lambda_a31071773b9a94e445cbd5d04ef99106>@@$$QEAV<lambda_56065050dbf3ada7e59a83db45153de3>@@@Z@4HA 000000018005e9c9 f   libucrt:output.obj
 0001:0005d9c9       ?fin$0@?0???$?RV<lambda_bdbcead8b570fa3d5ec6d9679862a6e5>@@AEAV<lambda_96f4279ff90247a4c5c5d9824f56f8c1>@@V<lambda_4606be27f17b5e5579e09050fab91818>@@@?$__crt_seh_guarded_call@_K@@QEAA_K$$QEAV<lambda_bdbcead8b570fa3d5ec6d9679862a6e5>@@AEAV<lambda_96f4279ff90247a4c5c5d9824f56f8c1>@@$$QEAV<lambda_4606be27f17b5e5579e09050fab91818>@@@Z@4HA 000000018005e9c9 f   libucrt:fwrite.obj
 0001:0005d9c9       ?fin$0@?0???$?RV<lambda_c376a267cfb53b6959b3b692ec76b120>@@AEAV<lambda_9a32fed5bf61b6b509b2d3f6003082a1>@@V<lambda_572fbb9fa0ab338edf41edfd4b5fcc8d>@@@?$__crt_seh_guarded_call@H@@QEAAH$$QEAV<lambda_c376a267cfb53b6959b3b692ec76b120>@@AEAV<lambda_9a32fed5bf61b6b509b2d3f6003082a1>@@$$QEAV<lambda_572fbb9fa0ab338edf41edfd4b5fcc8d>@@@Z@4HA 000000018005e9c9 f   libucrt:fflush.obj
 0001:0005d9e4       ?fin$0@?0???$common_fsopen@_W@@YAPEAU_iobuf@@QEB_W0H@Z@4HA 000000018005e9e4 f   libucrt:fopen.obj
 0001:0005da0f       ?fin$0@?0??common_fseek@@YAHV__crt_stdio_stream@@_JH@Z@4HA 000000018005ea0f f   libucrt:fseek.obj
 0001:0005da0f       fclose$fin$0               000000018005ea0f f   libucrt:fclose.obj
 0001:0005da0f       clearerr_s$fin$0           000000018005ea0f f   libucrt:clearerr.obj
 0001:0005da0f       rewind$fin$0               000000018005ea0f f   libucrt:rewind.obj
 0001:0005da0f       ?fin$0@?0???$common_ftell@J@@YAJV__crt_stdio_stream@@@Z@4HA 000000018005ea0f f   libucrt:ftell.obj
 0001:0005da27       common_control87$filt$0    000000018005ea27 f   libucrt:ieee.obj
 0001:0005da27       _ctrlfp$filt$0             000000018005ea27 f   libucrt:fpctrl.obj
 0001:0005da53       ?fin$0@?0???$common_freopen@_W@@YAHQEAPEAU_iobuf@@QEB_W1V__crt_stdio_stream@@H@Z@4HA 000000018005ea53 f   libucrt:freopen.obj
 0001:0005da6b       fread_s$fin$0              000000018005ea6b f   libucrt:fread.obj
 0001:0005da83       fgetc$fin$0                000000018005ea83 f   libucrt:fgetc.obj
 0001:0005da9d       ungetc$fin$0               000000018005ea9d f   libucrt:ungetc.obj
 0001:0005dab5       ?fin$0@?0???$common_popen@_W@@YAPEAU_iobuf@@QEB_W0@Z@4HA 000000018005eab5 f   libucrt:popen.obj
 0001:0005dad0       _pclose$fin$0              000000018005ead0 f   libucrt:popen.obj
 0001:0005dae9       ?fin$0@?0???$?RV<lambda_886d6c58226a84441f68b9f2b8217b83>@@AEAV<lambda_ab61a845afdef5b7c387490eaf3616ee>@@V<lambda_f7f22ab5edc0698d5f6905b0d3f44752>@@@?$__crt_seh_guarded_call@X@@QEAAX$$QEAV<lambda_886d6c58226a84441f68b9f2b8217b83>@@AEAV<lambda_ab61a845afdef5b7c387490eaf3616ee>@@$$QEAV<lambda_f7f22ab5edc0698d5f6905b0d3f44752>@@@Z@4HA 000000018005eae9 f   libucrt:fflush.obj
 0001:0005db06       ?fin$0@?0???$common_fgets@D@@YAPEADQEADHV__crt_stdio_stream@@@Z@4HA 000000018005eb06 f   libucrt:fgets.obj
 0001:0005db1e       ?fin$0@?0??common_tmpfile@@YAHQEAPEAU_iobuf@@H@Z@4HA 000000018005eb1e f   libucrt:tmpfile.obj
 0001:0005db37       ?fin$0@?0??common_tmpfile_nolock@@YAHQEAPEAU_iobuf@@H@Z@4HA 000000018005eb37 f   libucrt:tmpfile.obj
 0001:0005db60       ?fin$0@?0???$common_dupenv_s@_W@@YAHQEAPEA_WQEA_KQEB_WHQEBDH@Z@4HA 000000018005eb60 f   libucrt:getenv.obj
 0001:0005db79       ?fin$0@?0???$common_getenv@_W@@YAPEA_WQEB_W@Z@4HA 000000018005eb79 f   libucrt:getenv.obj
 0001:0005db92       ?fin$0@?0???$?RV<lambda_a22f0c497e5168315e06dae667770027>@@AEAV<lambda_a094494068278ba5130ab06e1292f60a>@@V<lambda_24dc10c13f43218c635520766e23e324>@@@?$__crt_seh_guarded_call@_N@@QEAA_N$$QEAV<lambda_a22f0c497e5168315e06dae667770027>@@AEAV<lambda_a094494068278ba5130ab06e1292f60a>@@$$QEAV<lambda_24dc10c13f43218c635520766e23e324>@@@Z@4HA 000000018005eb92 f   libucrt:spawnv.obj
 0001:0005db92       ?fin$0@?0???$?RV<lambda_7777bce6b2f8c936911f934f8298dc43>@@AEAV<lambda_f03950bc5685219e0bcd2087efbe011e>@@V<lambda_3883c3dff614d5e0c5f61bb1ac94921c>@@@?$__crt_seh_guarded_call@H@@QEAAH$$QEAV<lambda_7777bce6b2f8c936911f934f8298dc43>@@AEAV<lambda_f03950bc5685219e0bcd2087efbe011e>@@$$QEAV<lambda_3883c3dff614d5e0c5f61bb1ac94921c>@@@Z@4HA 000000018005eb92 f   libucrt:onexit.obj
 0001:0005db92       ?fin$0@?0???$?RV<lambda_efdfa57d1f175319df784efa44bb7b81>@@AEAV<lambda_5f0a4c1567f8adc6734073e5d1e1b35c>@@V<lambda_2e8a7d3640ea6ccb4c2413664c2db6fd>@@@?$__crt_seh_guarded_call@X@@QEAAX$$QEAV<lambda_efdfa57d1f175319df784efa44bb7b81>@@AEAV<lambda_5f0a4c1567f8adc6734073e5d1e1b35c>@@$$QEAV<lambda_2e8a7d3640ea6ccb4c2413664c2db6fd>@@@Z@4HA 000000018005eb92 f   libucrt:mbctype.obj
 0001:0005db92       ?fin$0@?0???$?RV<lambda_aa87e3671a710a21b5dc78c0bdf72e11>@@AEAV<lambda_92619d2358a28f41a33ba319515a20b9>@@V<lambda_6992ecaafeb10aed2b74cb1fae11a551>@@@?$__crt_seh_guarded_call@X@@QEAAX$$QEAV<lambda_aa87e3671a710a21b5dc78c0bdf72e11>@@AEAV<lambda_92619d2358a28f41a33ba319515a20b9>@@$$QEAV<lambda_6992ecaafeb10aed2b74cb1fae11a551>@@@Z@4HA 000000018005eb92 f   libucrt:per_thread_data.obj
 0001:0005db92       ?fin$0@?0???$?RV<lambda_f2e299630e499de9f9a165e60fcd3db5>@@AEAV<lambda_2ae9d31cdba2644fcbeaf08da7c24588>@@V<lambda_40d01ff24d0e7b3814fdbdcee8eab3c7>@@@?$__crt_seh_guarded_call@X@@QEAAX$$QEAV<lambda_f2e299630e499de9f9a165e60fcd3db5>@@AEAV<lambda_2ae9d31cdba2644fcbeaf08da7c24588>@@$$QEAV<lambda_40d01ff24d0e7b3814fdbdcee8eab3c7>@@@Z@4HA 000000018005eb92 f   libucrt:per_thread_data.obj
 0001:0005db92       ?fin$0@?0???$?RV<lambda_0ae27a3a962d80f24befdcbee591983d>@@AEAV<lambda_8d0ee55de4b1038c4002e0adecdf1839>@@V<lambda_dc504788e8f1664fe9b84e20bfb512f2>@@@?$__crt_seh_guarded_call@X@@QEAAX$$QEAV<lambda_0ae27a3a962d80f24befdcbee591983d>@@AEAV<lambda_8d0ee55de4b1038c4002e0adecdf1839>@@$$QEAV<lambda_dc504788e8f1664fe9b84e20bfb512f2>@@@Z@4HA 000000018005eb92 f   libucrt:per_thread_data.obj
 0001:0005db92       ?fin$0@?0???$?RV<lambda_450d765d439847d4c735a33c368b5fc0>@@AEAV<lambda_44731a7d0e6d81c3e6aa82d741081786>@@V<lambda_601a2a7da3b7a96e9554ac7215c4b07c>@@@?$__crt_seh_guarded_call@P6AXH@Z@@QEAAP6AXH@Z$$QEAV<lambda_450d765d439847d4c735a33c368b5fc0>@@AEAV<lambda_44731a7d0e6d81c3e6aa82d741081786>@@$$QEAV<lambda_601a2a7da3b7a96e9554ac7215c4b07c>@@@Z@4HA 000000018005eb92 f   libucrt:signal.obj
 0001:0005db92       ?fin$0@?0???$?RV<lambda_2d41944a1d46af3157314b8a01080d33>@@AEAV<lambda_8f455de75cd7d7f24b4096f044d8b9e6>@@V<lambda_aa500f224e6afead328df44964fe2772>@@@?$__crt_seh_guarded_call@X@@QEAAX$$QEAV<lambda_2d41944a1d46af3157314b8a01080d33>@@AEAV<lambda_8f455de75cd7d7f24b4096f044d8b9e6>@@$$QEAV<lambda_aa500f224e6afead328df44964fe2772>@@@Z@4HA 000000018005eb92 f   libucrt:per_thread_data.obj
 0001:0005db92       ?fin$0@?0???$?RV<lambda_d80eeec6fff315bfe5c115232f3240e3>@@AEAV<lambda_6e4b09c48022b2350581041d5f6b0c4c>@@V<lambda_2358e3775559c9db80273638284d5e45>@@@?$__crt_seh_guarded_call@X@@QEAAX$$QEAV<lambda_d80eeec6fff315bfe5c115232f3240e3>@@AEAV<lambda_6e4b09c48022b2350581041d5f6b0c4c>@@$$QEAV<lambda_2358e3775559c9db80273638284d5e45>@@@Z@4HA 000000018005eb92 f   libucrt:exit.obj
 0001:0005dbac       ?filt$0@?0???R<lambda_6e4b09c48022b2350581041d5f6b0c4c>@@QEBA@XZ@4HA 000000018005ebac f   libucrt:exit.obj
 0001:0005dbc7       ?fin$0@?0???$?RV<lambda_410d79af7f07d98d83a3f525b3859a53>@@AEAV<lambda_3e16ef9562a7dcce91392c22ab16ea36>@@V<lambda_38119f0e861e05405d8a144b9b982f0a>@@@?$__crt_seh_guarded_call@X@@QEAAX$$QEAV<lambda_410d79af7f07d98d83a3f525b3859a53>@@AEAV<lambda_3e16ef9562a7dcce91392c22ab16ea36>@@$$QEAV<lambda_38119f0e861e05405d8a144b9b982f0a>@@@Z@4HA 000000018005ebc7 f   libucrt:wsetlocale.obj
 0001:0005dbe1       __acrt_initialize_lowio$fin$0 000000018005ebe1 f   libucrt:ioinit.obj
 0001:0005dbe1       _alloc_osfhnd$fin$0        000000018005ebe1 f   libucrt:osfinfo.obj
 0001:0005dbe1       __acrt_lowio_ensure_fh_exists$fin$0 000000018005ebe1 f   libucrt:osfinfo.obj
 0001:0005dbfa       ?fin$0@?0??__acrt_stdio_allocate_stream@@YA?AV__crt_stdio_stream@@XZ@4HA 000000018005ebfa f   libucrt:stream.obj
 0001:0005dbfa       _fcloseall$fin$0           000000018005ebfa f   libucrt:closeall.obj
 0001:0005dc13       ?fin$0@?0???$?RV<lambda_a37b2b86f63e897a80ea819b0eb08c01>@@AEAV<lambda_38ce7e780aa69e748d6df282ebc68efe>@@V<lambda_99fb1378e971ab6e7edea83e3a7a83a2>@@@?$__crt_seh_guarded_call@H@@QEAAH$$QEAV<lambda_a37b2b86f63e897a80ea819b0eb08c01>@@AEAV<lambda_38ce7e780aa69e748d6df282ebc68efe>@@$$QEAV<lambda_99fb1378e971ab6e7edea83e3a7a83a2>@@@Z@4HA 000000018005ec13 f   libucrt:commit.obj
 0001:0005dc13       ?fin$0@?0???$?RV<lambda_751a882b2c74d4b022dec766aa51a29a>@@AEAV<lambda_628dfdc04ba53c8bfc02c9951375f3f5>@@V<lambda_f6c7be5f7998530c34de24c7437d6b54>@@@?$__crt_seh_guarded_call@H@@QEAAH$$QEAV<lambda_751a882b2c74d4b022dec766aa51a29a>@@AEAV<lambda_628dfdc04ba53c8bfc02c9951375f3f5>@@$$QEAV<lambda_f6c7be5f7998530c34de24c7437d6b54>@@@Z@4HA 000000018005ec13 f   libucrt:close.obj
 0001:0005dc2d       _read$fin$0                000000018005ec2d f   libucrt:read.obj
 0001:0005dc44       ?fin$0@?0???$common_lseek@_J@@YA_JH_JH@Z@4HA 000000018005ec44 f   libucrt:lseek.obj
 0001:0005dc44       _write$fin$0               000000018005ec44 f   libucrt:write.obj
 0001:0005dc44       ?fin$0@?0???$common_lseek@J@@YAJHJH@Z@4HA 000000018005ec44 f   libucrt:lseek.obj
 0001:0005dc5b       _pipe$fin$1                000000018005ec5b f   libucrt:pipe.obj
 0001:0005dc77       _pipe$fin$0                000000018005ec77 f   libucrt:pipe.obj
 0001:0005dc93       ?fin$0@?0???$common_fdopen@_W@@YAPEAU_iobuf@@HQEB_W@Z@4HA 000000018005ec93 f   libucrt:fdopen.obj
 0001:0005dcad       ?fin$0@?0???$common_sopen_dispatch@_W@@YAHQEB_WHHHQEAHH@Z@4HA 000000018005ecad f   libucrt:open.obj
 0001:0005dcad       ?fin$0@?0???$common_sopen_dispatch@D@@YAHQEBDHHHQEAHH@Z@4HA 000000018005ecad f   libucrt:open.obj
 0001:0005dd00       _rmtmp$fin$0               000000018005ed00 f   libucrt:rmtmp.obj
 0001:0005dd1a       _rmtmp$fin$1               000000018005ed1a f   libucrt:rmtmp.obj
 0001:0005dd33       ?fin$0@?0??update_thread_multibyte_data_internal@@YAPEAU__crt_multibyte_data@@QEAU__acrt_ptd@@QEAPEAU1@@Z@4HA 000000018005ed33 f   libucrt:mbctype.obj
 0001:0005dd4c       _query_new_handler$fin$0   000000018005ed4c f   libucrt:new_handler.obj
 0001:0005dd62       raise$fin$0                000000018005ed62 f   libucrt:signal.obj
 0001:0005dd83       __acrt_update_thread_locale_data$fin$0 000000018005ed83 f   libucrt:locale_refcounting.obj
 0001:0005dda0       _IsNonwritableInCurrentImage$filt$0 000000018005eda0 f   LIBCMT:pesect.obj
 0001:0005ddc0       $xdatasym                  000000018005edc0     chkstk.obj
 0001:0005ddc8       $unwind$fprintf            000000018005edc8     service.obj
 0001:0005ddc8       $unwind$sprintf            000000018005edc8     bit64.obj
 0001:0005ddc8       $unwind$fscanf             000000018005edc8     uliolib51.obj
 0001:0005ddd4       $unwind$far_LIsLower       000000018005edd4     service.obj
 0001:0005ddd4       $unwind$far_LIsUpper       000000018005edd4     service.obj
 0001:0005ddd4       $unwind$LF_FreeFindData    000000018005edd4     exported.obj
 0001:0005ddd4       $unwind$LF_ExitFAR         000000018005edd4     exported.obj
 0001:0005ddd4       $unwind$editor_PrevSessionBookmark 000000018005edd4     service.obj
 0001:0005ddd4       $unwind$_ungetc_nolock     000000018005edd4     libucrt:ungetc.obj
 0001:0005ddd4       $unwind$editor_NextSessionBookmark 000000018005edd4     service.obj
 0001:0005ddd4       $unwind$?common_fseek_binary_mode_read_only_fast_track_nolock@@YA_NV__crt_stdio_stream@@_JH@Z 000000018005edd4     libucrt:fseek.obj
 0001:0005ddd4       $unwind$pushFileTime       000000018005edd4     service.obj
 0001:0005ddd4       $unwind$__acrt_errno_map_os_error 000000018005edd4     libucrt:errno.obj
 0001:0005ddd4       $unwind$editor_ClearSessionBookmarks 000000018005edd4     service.obj
 0001:0005ddd4       $unwind$far_Show           000000018005edd4     service.obj
 0001:0005ddd4       $unwind$editor_AddSessionBookmark 000000018005edd4     service.obj
 0001:0005ddd4       $unwind$filefilter_Free    000000018005edd4     service.obj
 0001:0005ddd4       $unwind$_fclose_nolock     000000018005edd4     libucrt:fclose.obj
 0001:0005ddd4       $unwind$??$get_tmpfile_buffer_nolock@D@@YAPEADW4buffer_id@?A0x5b9a7937@@@Z 000000018005edd4     libucrt:tmpfile.obj
 0001:0005ddd4       $unwind$LF_Analyse         000000018005edd4     exported.obj
 0001:0005ddd4       $unwind$filefilter_gc      000000018005edd4     service.obj
 0001:0005ddd4       $unwind$?process@?$input_processor@DV?$stream_input_adapter@D@__crt_stdio_input@@@__crt_stdio_input@@QEAAHXZ 000000018005edd4     libucrt:input.obj
 0001:0005ddd4       $unwind$?process_state@?$input_processor@DV?$stream_input_adapter@D@__crt_stdio_input@@@__crt_stdio_input@@AEAA_NXZ 000000018005edd4     libucrt:input.obj
 0001:0005ddd4       $unwind$?process_literal_character_tchar@?$input_processor@DV?$stream_input_adapter@D@__crt_stdio_input@@@__crt_stdio_input@@AEAA_ND@Z 000000018005edd4     libucrt:input.obj
 0001:0005ddd4       $unwind$filefilter_OpenMenu 000000018005edd4     service.obj
 0001:0005ddd4       $unwind$editor_Redraw      000000018005edd4     service.obj
 0001:0005ddd4       $unwind$filefilter_Starting 000000018005edd4     service.obj
 0001:0005ddd4       $unwind$far_LIsAlphanum    000000018005edd4     service.obj
 0001:0005ddd4       $unwind$?process_floating_point_specifier@?$input_processor@DV?$stream_input_adapter@D@__crt_stdio_input@@@__crt_stdio_input@@AEAA_NXZ 000000018005edd4     libucrt:input.obj
 0001:0005ddd4       $unwind$?write_integer@?$input_processor@DV?$stream_input_adapter@D@__crt_stdio_input@@@__crt_stdio_input@@AEAA_N_K@Z 000000018005edd4     libucrt:input.obj
 0001:0005ddd4       $unwind$far_UnloadPlugin   000000018005edd4     service.obj
 0001:0005ddd4       $unwind$Settings_free      000000018005edd4     service.obj
 0001:0005ddd4       $unwind$far_GetMsg         000000018005edd4     service.obj
 0001:0005ddd4       $unwind$??R<lambda_156378f40168adef48d7ddfcff3a1264>@@QEBA_NXZ 000000018005edd4     libucrt:input.obj
 0001:0005ddd4       $unwind$LF_ProcessEditorInput 000000018005edd4     exported.obj
 0001:0005ddd4       $unwind$far_FileTimeResolution 000000018005edd4     service.obj
 0001:0005ddd4       $unwind$luaopen_luafar3    000000018005edd4     service.obj
 0001:0005ddd4       $unwind$add_utf8char       000000018005edd4     lutf8lib.obj
 0001:0005ddd4       $unwind$editor_Quit        000000018005edd4     service.obj
 0001:0005ddd4       $unwind$__acrt_execute_uninitializers 000000018005edd4     libucrt:shared_initialization.obj
 0001:0005ddd4       $unwind$viewer_Redraw      000000018005edd4     service.obj
 0001:0005ddd4       $unwind$editor_DeleteBlock 000000018005edd4     service.obj
 0001:0005ddd4       $unwind$bit64_pushuserdata 000000018005edd4     bit64.obj
 0001:0005ddd4       $unwind$editor_DeleteChar  000000018005edd4     service.obj
 0001:0005ddd4       $unwind$_initterm_e        000000018005edd4     libucrt:initterm.obj
 0001:0005ddd4       $unwind$f_le               000000018005edd4     bit64.obj
 0001:0005ddd4       $unwind$bit64_push         000000018005edd4     bit64.obj
 0001:0005ddd4       $unwind$viewer_Quit        000000018005edd4     service.obj
 0001:0005ddd4       $unwind$__acrt_wgetpath    000000018005edd4     libucrt:getpath.obj
 0001:0005ddd4       $unwind$editor_DeleteString 000000018005edd4     service.obj
 0001:0005ddd4       $unwind$f_lt               000000018005edd4     bit64.obj
 0001:0005ddd4       $unwind$f_eq               000000018005edd4     bit64.obj
 0001:0005ddd4       $unwind$__acrt_stdio_allocate_buffer_nolock 000000018005edd4     libucrt:_getbuf.obj
 0001:0005ddd4       $unwind$?process_conversion_specifier@?$input_processor@DV?$stream_input_adapter@D@__crt_stdio_input@@@__crt_stdio_input@@AEAA_NXZ 000000018005edd4     libucrt:input.obj
 0001:0005ddd4       $unwind$io_type            000000018005edd4     uliolib51.obj
 0001:0005ddd4       $unwind$newfile            000000018005edd4     uliolib51.obj
 0001:0005ddd4       $unwind$f_div              000000018005edd4     bit64.obj
 0001:0005ddd4       $unwind$??$common_initialize_environment_nolock@D@@YAHXZ 000000018005edd4     libucrt:environment_initialization.obj
 0001:0005ddd4       $unwind$io_tmpfile         000000018005edd4     uliolib51.obj
 0001:0005ddd4       $unwind$??$common_initialize_environment_nolock@_W@@YAHXZ 000000018005edd4     libucrt:environment_initialization.obj
 0001:0005ddd4       $unwind$_updatetlocinfoEx_nolock 000000018005edd4     libucrt:locale_refcounting.obj
 0001:0005ddd4       $unwind$io_read            000000018005edd4     uliolib51.obj
 0001:0005ddd4       $unwind$f_sub              000000018005edd4     bit64.obj
 0001:0005ddd4       $unwind$f_read             000000018005edd4     uliolib51.obj
 0001:0005ddd4       $unwind$free_dialog        000000018005edd4     service.obj
 0001:0005ddd4       $unwind$__acrt_fp_strflt_to_string 000000018005edd4     libucrt:_fptostr.obj
 0001:0005ddd4       $unwind$io_write           000000018005edd4     uliolib51.obj
 0001:0005ddd4       $unwind$f_write            000000018005edd4     uliolib51.obj
 0001:0005ddd4       $unwind$ll_loadlib         000000018005edd4     uloadlib51.obj
 0001:0005ddd4       $unwind$loader_Lua         000000018005edd4     uloadlib51.obj
 0001:0005ddd4       $unwind$mkfuncname         000000018005edd4     uloadlib51.obj
 0001:0005ddd4       $unwind$loader_preload     000000018005edd4     uloadlib51.obj
 0001:0005ddd4       $unwind$DialogHandleEqual  000000018005edd4     service.obj
 0001:0005ddd4       $unwind$FillEditorSetPosition 000000018005edd4     service.obj
 0001:0005ddd4       $unwind$SysErrorReturn     000000018005edd4     ustring.obj
 0001:0005ddd4       $unwind$far_GetNumberOfLinks 000000018005edd4     service.obj
 0001:0005ddd4       $unwind$GetBoolFromTable   000000018005edd4     ustring.obj
 0001:0005ddd4       $unwind$GetOptBoolFromTable 000000018005edd4     ustring.obj
 0001:0005ddd4       $unwind$GetOptIntFromArray 000000018005edd4     ustring.obj
 0001:0005ddd4       $unwind$LF_FreeContentData 000000018005edd4     exported.obj
 0001:0005ddd4       $unwind$GetOptIntFromTable 000000018005edd4     ustring.obj
 0001:0005ddd4       $unwind$PutIntToArray      000000018005edd4     ustring.obj
 0001:0005ddd4       $unwind$PutIntToTable      000000018005edd4     ustring.obj
 0001:0005ddd4       $unwind$PushPluginHandle   000000018005edd4     service.obj
 0001:0005ddd4       $unwind$PushInputRecord    000000018005edd4     service.obj
 0001:0005ddd4       $unwind$PutFlagsToTable    000000018005edd4     service.obj
 0001:0005ddd4       $unwind$?force_decimal_point@__crt_stdio_output@@YAXPEADQEAU__crt_locale_pointers@@@Z 000000018005edd4     libucrt:output.obj
 0001:0005ddd4       $unwind$GetFlagsFromTable  000000018005edd4     service.obj
 0001:0005ddd4       $unwind$PutLStrToTable     000000018005edd4     ustring.obj
 0001:0005ddd4       $unwind$CheckFlagsFromTable 000000018005edd4     service.obj
 0001:0005ddd4       $unwind$PutNumToTable      000000018005edd4     ustring.obj
 0001:0005ddd4       $unwind$func_New           000000018005edd4     lregex.obj
 0001:0005ddd4       $unwind$PutStrToArray      000000018005edd4     ustring.obj
 0001:0005ddd4       $unwind$method_bracketscount 000000018005edd4     lregex.obj
 0001:0005ddd4       $unwind$PutStrToTable      000000018005edd4     ustring.obj
 0001:0005ddd4       $unwind$__vcrt_FlsSetValue 000000018005edd4     libvcruntime:winapi_downlevel.obj
 0001:0005ddd4       $unwind$GetExportFunction  000000018005edd4     exported.obj
 0001:0005ddd4       $unwind$ustring_EnumSystemCodePages 000000018005edd4     ustring.obj
 0001:0005ddd4       $unwind$panel_IsActivePanel 000000018005edd4     service.obj
 0001:0005ddd4       $unwind$ustring_GetKeyState 000000018005edd4     ustring.obj
 0001:0005ddd4       $unwind$_realloc_base      000000018005edd4     libucrt:realloc_base.obj
 0001:0005ddd4       $unwind$GetAttrFromTable   000000018005edd4     util.obj
 0001:0005ddd4       $unwind$panel_EndSelection 000000018005edd4     service.obj
 0001:0005ddd4       $unwind$GetLuaStateTimerQueue 000000018005edd4     service.obj
 0001:0005ddd4       $unwind$GetFileSizeFromTable 000000018005edd4     util.obj
 0001:0005ddd4       $unwind$panel_BeginSelection 000000018005edd4     service.obj
 0001:0005ddd4       $unwind$win_SetEnv         000000018005edd4     win.obj
 0001:0005ddd4       $unwind$CheckHKey          000000018005edd4     win.obj
 0001:0005ddd4       $unwind$win_FileTimeToLocalFileTime 000000018005edd4     win.obj
 0001:0005ddd4       $unwind$__acrt_LocaleNameToLCID 000000018005edd4     libucrt:winapi_thunks.obj
 0001:0005ddd4       $unwind$PushPluginPair     000000018005edd4     exported.obj
 0001:0005ddd4       $unwind$PushFarColor       000000018005edd4     service.obj
 0001:0005ddd4       $unwind$lshift             000000018005edd4     bit64.obj
 0001:0005ddd4       $unwind$__acrt_FlsSetValue 000000018005edd4     libucrt:winapi_thunks.obj
 0001:0005ddd4       $unwind$method_tostring    000000018005edd4     lregex.obj
 0001:0005ddd4       $unwind$panel_GetCmdLinePos 000000018005edd4     service.obj
 0001:0005ddd4       $unwind$method_gc          000000018005edd4     lregex.obj
 0001:0005ddd4       $unwind$PutBoolToTable     000000018005edd4     ustring.obj
 0001:0005ddd4       $unwind$strncpy_s          000000018005edd4     libucrt:strncpy_s.obj
 0001:0005ddd4       $unwind$LF_GetLuafarAPI    000000018005edd4     service.obj
 0001:0005ddd4       $unwind$panel_CheckPanelsExist 000000018005edd4     service.obj
 0001:0005ddd4       $unwind$far_LIsAlpha       000000018005edd4     service.obj
 0001:0005ddd4       $unwind$rshift             000000018005edd4     bit64.obj
 0001:0005ddd4       $unwind$_close_nolock      000000018005edd4     libucrt:close.obj
 0001:0005ddd4       $unwind$_RTC_Terminate     000000018005edd4     LIBCMT:initsect.obj
 0001:0005ddd4       $unwind$_RTC_Initialize    000000018005edd4     LIBCMT:initsect.obj
 0001:0005ddd4       $unwind$LF_InitLuaState2   000000018005edd4     service.obj
 0001:0005ddd4       $unwind$PushFarMacroValue  000000018005edd4     exported.obj
 0001:0005ddd4       $unwind$__acrt_uninitialize_lowio 000000018005edd4     libucrt:ioinit.obj
 0001:0005ddd4       $unwind$PushAnalyseInfo    000000018005edd4     exported.obj
 0001:0005ddd4       $unwind$arshift            000000018005edd4     bit64.obj
 0001:0005ddd4       $unwind$?replace_current_thread_locale_nolock@@YAXQEAU__acrt_ptd@@QEAU__crt_locale_data@@@Z 000000018005edd4     libucrt:per_thread_data.obj
 0001:0005ddd4       $unwind$RegisterObject     000000018005edd4     exported.obj
 0001:0005ddd4       $unwind$__acrt_stdio_begin_temporary_buffering_nolock 000000018005edd4     libucrt:_sftbuf.obj
 0001:0005dde0       $unwind$_cwait             000000018005ede0     libucrt:wait.obj
 0001:0005dde0       $unwind$LF_ProcessEditorEvent 000000018005ede0     exported.obj
 0001:0005dde0       $unwind$utf8_length        000000018005ede0     lutf8lib.obj
 0001:0005dde0       $unwind$bit64_getvalue     000000018005ede0     bit64.obj
 0001:0005dde0       $unwind$?type_case_c_tchar@?$output_processor@_WV?$string_output_adapter@_W@__crt_stdio_output@@V?$standard_base@_WV?$string_output_adapter@_W@__crt_stdio_output@@@2@@__crt_stdio_output@@AEAA_N_W@Z 000000018005ede0     libucrt:output.obj
 0001:0005dde0       $unwind$GetFarColor        000000018005ede0     service.obj
 0001:0005dde0       $unwind$LF_ProcessConsoleInput 000000018005ede0     exported.obj
 0001:0005ddf0       $chain$0$bit64_getvalue    000000018005edf0     bit64.obj
 0001:0005de04       $chain$1$bit64_getvalue    000000018005ee04     bit64.obj
 0001:0005de14       $unwind$check64            000000018005ee14     bit64.obj
 0001:0005de24       $chain$0$check64           000000018005ee24     bit64.obj
 0001:0005de38       $chain$1$check64           000000018005ee38     bit64.obj
 0001:0005de48       $unwind$??$common_getenv_nolock@_W@@YAPEA_WQEB_W@Z 000000018005ee48     libucrt:getenv.obj
 0001:0005de48       $unwind$_initterm          000000018005ee48     libucrt:initterm.obj
 0001:0005de48       $unwind$_seh_filter_exe    000000018005ee48     libucrt:exception_filter.obj
 0001:0005de48       $unwind$?find_or_allocate_unused_stream_nolock@@YA?AV__crt_stdio_stream@@XZ 000000018005ee48     libucrt:stream.obj
 0001:0005de48       $unwind$??$ensure_buffer_is_big_enough@D@formatting_buffer@__crt_stdio_output@@QEAA_N_K@Z 000000018005ee48     libucrt:output.obj
 0001:0005de48       $unwind$??$ensure_buffer_is_big_enough@_W@formatting_buffer@__crt_stdio_output@@QEAA_N_K@Z 000000018005ee48     libucrt:output.obj
 0001:0005de48       $unwind$_recalloc_base     000000018005ee48     libucrt:recalloc.obj
 0001:0005de48       $unwind$__dcrt_get_wide_environment_from_os 000000018005ee48     libucrt:get_environment_from_os.obj
 0001:0005de48       $unwind$pushresult         000000018005ee48     uliolib51.obj
 0001:0005de48       $unwind$__acrt_free_locale 000000018005ee48     libucrt:locale_refcounting.obj
 0001:0005de48       $unwind$io_popen           000000018005ee48     uliolib51.obj
 0001:0005de48       $unwind$__scrt_dllmain_exception_filter 000000018005ee48     LIBCMT:utility.obj
 0001:0005de48       $unwind$uc_New             000000018005ee48     lusercontrol.obj
 0001:0005de48       $unwind$?scan_scanset_range@?$format_string_parser@D@__crt_stdio_input@@AEAA_NXZ 000000018005ee48     libucrt:input.obj
 0001:0005de48       $unwind$f_mul              000000018005ee48     bit64.obj
 0001:0005de48       $unwind$timer_index        000000018005ee48     service.obj
 0001:0005de48       $unwind$?setSBCS@@YAXPEAU__crt_multibyte_data@@@Z 000000018005ee48     libucrt:mbctype.obj
 0001:0005de48       $unwind$win_CopyFile       000000018005ee48     win.obj
 0001:0005de48       $unwind$InitMPR            000000018005ee48     luamacro.obj
 0001:0005de48       $unwind$findfile           000000018005ee48     uloadlib51.obj
 0001:0005de48       $unwind$band               000000018005ee48     bit64.obj
 0001:0005de48       $unwind$f_add              000000018005ee48     bit64.obj
 0001:0005de48       $unwind$bor                000000018005ee48     bit64.obj
 0001:0005de48       $unwind$bxor               000000018005ee48     bit64.obj
 0001:0005de48       $unwind$FillInputRecord    000000018005ee48     service.obj
 0001:0005de48       $unwind$win_DeleteRegKey   000000018005ee48     win.obj
 0001:0005de48       $unwind$OptInputRecord     000000018005ee48     service.obj
 0001:0005de48       $unwind$__acrt_lowio_create_handle_array 000000018005ee48     libucrt:osfinfo.obj
 0001:0005de48       $unwind$push_far_regex     000000018005ee48     lregex.obj
 0001:0005de48       $unwind$pcall_msg          000000018005ee48     exported.obj
 0001:0005de5c       $unwind$__vcrt_FlsAlloc    000000018005ee5c     libvcruntime:winapi_downlevel.obj
 0001:0005de5c       $unwind$bnot               000000018005ee5c     bit64.obj
 0001:0005de5c       $unwind$GetFileTimeFromTable 000000018005ee5c     util.obj
 0001:0005de5c       $unwind$__vcrt_uninitialize_locks 000000018005ee5c     libvcruntime:locks.obj
 0001:0005de5c       $unwind$DeleteLuaStateTimerQueue 000000018005ee5c     service.obj
 0001:0005de5c       $unwind$__raise_securityfailure 000000018005ee5c     LIBCMT:gs_report.obj
 0001:0005de5c       $unwind$OptHandle          000000018005ee5c     service.obj
 0001:0005de5c       $unwind$ustring_system     000000018005ee5c     ustring.obj
 0001:0005de5c       $unwind$__vcrt_FlsFree     000000018005ee5c     libvcruntime:winapi_downlevel.obj
 0001:0005de5c       $unwind$?idtab@@YAPEAUprocess_handle_pair@?A0xe43b7539@@QEAU_iobuf@@@Z 000000018005ee5c     libucrt:popen.obj
 0001:0005de5c       $unwind$ustring_len        000000018005ee5c     ustring.obj
 0001:0005de5c       $unwind$ustring_GetDriveType 000000018005ee5c     ustring.obj
 0001:0005de5c       $unwind$__vcrt_FlsGetValue 000000018005ee5c     libvcruntime:winapi_downlevel.obj
 0001:0005de5c       $unwind$_fflush_nolock     000000018005ee5c     libucrt:fflush.obj
 0001:0005de5c       $unwind$ustring_GetConsoleOutputCP 000000018005ee5c     ustring.obj
 0001:0005de5c       $unwind$ustring_GetConsoleCP 000000018005ee5c     ustring.obj
 0001:0005de5c       $unwind$ustring_GetOEMCP   000000018005ee5c     ustring.obj
 0001:0005de5c       $unwind$far_MacroSaveAll   000000018005ee5c     service.obj
 0001:0005de5c       $unwind$ustring_GetACP     000000018005ee5c     ustring.obj
 0001:0005de5c       $unwind$PutAttrToTable     000000018005ee5c     ustring.obj
 0001:0005de5c       $unwind$check_utf16_string 000000018005ee5c     ustring.obj
 0001:0005de5c       $unwind$traceback          000000018005ee5c     exported.obj
 0001:0005de5c       $unwind$far_MacroGetState  000000018005ee5c     service.obj
 0001:0005de5c       $unwind$win_GetSystemTimeAsFileTime 000000018005ee5c     win.obj
 0001:0005de5c       $unwind$PushPluginObject   000000018005ee5c     exported.obj
 0001:0005de5c       $unwind$luaB_loadfileW     000000018005ee5c     lflua.obj
 0001:0005de5c       $unwind$PluginHandle_rawhandle 000000018005ee5c     service.obj
 0001:0005de5c       $unwind$far_MacroGetArea   000000018005ee5c     service.obj
 0001:0005de5c       $unwind$far_CPluginStartupInfo 000000018005ee5c     service.obj
 0001:0005de5c       $unwind$luaopen_regex      000000018005ee5c     lregex.obj
 0001:0005de5c       $unwind$strcpy_s           000000018005ee5c     libucrt:strcpy_s.obj
 0001:0005de5c       $unwind$?state_case_normal@?$output_processor@DV?$stream_output_adapter@D@__crt_stdio_output@@V?$standard_base@DV?$stream_output_adapter@D@__crt_stdio_output@@@2@@__crt_stdio_output@@AEAA_NXZ 000000018005ee5c     libucrt:output.obj
 0001:0005de5c       $unwind$__acrt_AppPolicyGetProcessTerminationMethodInternal 000000018005ee5c     libucrt:winapi_thunks.obj
 0001:0005de5c       $unwind$__vcrt_initialize_locks 000000018005ee5c     libvcruntime:locks.obj
 0001:0005de5c       $unwind$pusherror          000000018005ee5c     ustring.obj
 0001:0005de5c       $unwind$luaopen_ustring    000000018005ee5c     ustring.obj
 0001:0005de5c       $unwind$ll_seeall          000000018005ee5c     uloadlib51.obj
 0001:0005de5c       $unwind$?state_case_normal_tchar@?$output_processor@DV?$stream_output_adapter@D@__crt_stdio_output@@V?$standard_base@DV?$stream_output_adapter@D@__crt_stdio_output@@@2@@__crt_stdio_output@@AEAA_ND@Z 000000018005ee5c     libucrt:output.obj
 0001:0005de5c       $unwind$_strupr            000000018005ee5c     libucrt:strupr.obj
 0001:0005de5c       $unwind$__vcrt_freeptd     000000018005ee5c     libvcruntime:per_thread_data.obj
 0001:0005de5c       $unwind$?type_case_c_tchar@?$output_processor@DV?$stream_output_adapter@D@__crt_stdio_output@@V?$standard_base@DV?$stream_output_adapter@D@__crt_stdio_output@@@2@@__crt_stdio_output@@AEAA_ND@Z 000000018005ee5c     libucrt:output.obj
 0001:0005de5c       $unwind$ReplacePluginInfoCollector 000000018005ee5c     exported.obj
 0001:0005de5c       $unwind$__acrt_FlsGetValue 000000018005ee5c     libucrt:winapi_thunks.obj
 0001:0005de5c       $unwind$gctm               000000018005ee5c     uloadlib51.obj
 0001:0005de5c       $unwind$uninitialize_allocated_memory 000000018005ee5c     libucrt:initialization.obj
 0001:0005de5c       $unwind$?type_case_s@?$output_processor@DV?$stream_output_adapter@D@__crt_stdio_output@@V?$standard_base@DV?$stream_output_adapter@D@__crt_stdio_output@@@2@@__crt_stdio_output@@AEAA_NXZ 000000018005ee5c     libucrt:output.obj
 0001:0005de5c       $unwind$initialize_pointers 000000018005ee5c     libucrt:initialization.obj
 0001:0005de5c       $unwind$?state_case_normal@?$output_processor@DV?$string_output_adapter@D@__crt_stdio_output@@V?$standard_base@DV?$string_output_adapter@D@__crt_stdio_output@@@2@@__crt_stdio_output@@AEAA_NXZ 000000018005ee5c     libucrt:output.obj
 0001:0005de5c       $unwind$?type_case_c_tchar@?$output_processor@DV?$string_output_adapter@D@__crt_stdio_output@@V?$standard_base@DV?$string_output_adapter@D@__crt_stdio_output@@@2@@__crt_stdio_output@@AEAA_ND@Z 000000018005ee5c     libucrt:output.obj
 0001:0005de5c       $unwind$__acrt_FlsFree     000000018005ee5c     libucrt:winapi_thunks.obj
 0001:0005de5c       $unwind$?type_case_s@?$output_processor@DV?$string_output_adapter@D@__crt_stdio_output@@V?$standard_base@DV?$string_output_adapter@D@__crt_stdio_output@@@2@@__crt_stdio_output@@AEAA_NXZ 000000018005ee5c     libucrt:output.obj
 0001:0005de5c       $unwind$fegetenv           000000018005ee5c     libucrt:fegetenv.obj
 0001:0005de5c       $unwind$dialog_tostring    000000018005ee5c     service.obj
 0001:0005de5c       $unwind$f_lines            000000018005ee5c     uliolib51.obj
 0001:0005de5c       $unwind$dialog_rawhandle   000000018005ee5c     service.obj
 0001:0005de5c       $unwind$luaopen_usercontrol 000000018005ee5c     lusercontrol.obj
 0001:0005de5c       $unwind$__acrt_FlsAlloc    000000018005ee5c     libucrt:winapi_thunks.obj
 0001:0005de5c       $unwind$fesetenv           000000018005ee5c     libucrt:fesetenv.obj
 0001:0005de5c       $unwind$__acrt_uninitialize_winapi_thunks 000000018005ee5c     libucrt:winapi_thunks.obj
 0001:0005de5c       $unwind$uc_len             000000018005ee5c     lusercontrol.obj
 0001:0005de5c       $unwind$io_tostring        000000018005ee5c     uliolib51.obj
 0001:0005de5c       $unwind$io_gc              000000018005ee5c     uliolib51.obj
 0001:0005de5c       $unwind$io_close           000000018005ee5c     uliolib51.obj
 0001:0005de5c       $unwind$aux_close          000000018005ee5c     uliolib51.obj
 0001:0005de5c       $unwind$io_noclose         000000018005ee5c     uliolib51.obj
 0001:0005de5c       $unwind$__acrt_allocate_buffer_for_argv 000000018005ee5c     libucrt:argv_parsing.obj
 0001:0005de5c       $unwind$feholdexcept       000000018005ee5c     libucrt:feholdexcept.obj
 0001:0005de5c       $unwind$f_unm              000000018005ee5c     bit64.obj
 0001:0005de5c       $unwind$__std_type_info_destroy_list 000000018005ee5c     libvcruntime:std_type_info.obj
 0001:0005de5c       $unwind$?internal_isupper_l@@YA_NHQEAU__crt_locale_pointers@@@Z 000000018005ee5c     libucrt:tolower_toupper.obj
 0001:0005de5c       $unwind$?exit_or_terminate_process@@YAXI@Z 000000018005ee5c     libucrt:exit.obj
 0001:0005de5c       $unwind$__acrt_uninitialize_stdio 000000018005ee5c     libucrt:_file.obj
 0001:0005de5c       $unwind$uc_tostring        000000018005ee5c     lusercontrol.obj
 0001:0005de5c       $unwind$?try_cor_exit_process@@YAXI@Z 000000018005ee5c     libucrt:exit.obj
 0001:0005de5c       $unwind$wcscat_s           000000018005ee5c     libucrt:wcscat_s.obj
 0001:0005de5c       $unwind$_calloc_base       000000018005ee5c     libucrt:calloc_base.obj
 0001:0005de5c       $unwind$_malloc_base       000000018005ee5c     libucrt:malloc_base.obj
 0001:0005de5c       $unwind$_set_statfp        000000018005ee5c     libucrt:fpctrl.obj
 0001:0005de5c       $unwind$__acrt_stdio_free_buffer_nolock 000000018005ee5c     libucrt:_freebuf.obj
 0001:0005de5c       $unwind$win_DeleteFile     000000018005ee5c     win.obj
 0001:0005de5c       $unwind$FarPanelItemFreeCallback 000000018005ee5c     exported.obj
 0001:0005de5c       $unwind$__acrt_initialize_locks 000000018005ee5c     libucrt:locks.obj
 0001:0005de5c       $unwind$__acrt_uninitialize_locks 000000018005ee5c     libucrt:locks.obj
 0001:0005de5c       $unwind$luaopen_bit64      000000018005ee5c     bit64.obj
 0001:0005de5c       $unwind$?stream_is_at_end_of_file_nolock@@YA_NV__crt_stdio_stream@@@Z 000000018005ee5c     libucrt:_flsbuf.obj
 0001:0005de5c       $unwind$Lutf8_gmatch       000000018005ee5c     lutf8lib.obj
 0001:0005de5c       $unwind$Lutf8_codes        000000018005ee5c     lutf8lib.obj
 0001:0005de5c       $unwind$_callnewh          000000018005ee5c     libucrt:new_handler.obj
 0001:0005de5c       $unwind$Lutf8_offset       000000018005ee5c     lutf8lib.obj
 0001:0005de5c       $unwind$_clearfp           000000018005ee5c     libucrt:ieee.obj
 0001:0005de5c       $unwind$win_RemoveDir      000000018005ee5c     win.obj
 0001:0005de5c       $unwind$wcscpy_s           000000018005ee5c     libucrt:wcscpy_s.obj
 0001:0005de5c       $unwind$__acrt_getptd_head 000000018005ee5c     libucrt:per_thread_data.obj
 0001:0005de5c       $unwind$__acrt_freeptd     000000018005ee5c     libucrt:per_thread_data.obj
 0001:0005de5c       $unwind$far_RunDefaultScript 000000018005ee5c     service.obj
 0001:0005de5c       $unwind$luaopen_win        000000018005ee5c     win.obj
 0001:0005de5c       $unwind$__acrt_update_locale_info 000000018005ee5c     libucrt:locale_update.obj
 0001:0005de5c       $unwind$Settings_tostring  000000018005ee5c     service.obj
 0001:0005de5c       $unwind$far_FreeSettings   000000018005ee5c     service.obj
 0001:0005de5c       $unwind$filefilter_tostring 000000018005ee5c     service.obj
 0001:0005de5c       $unwind$far_CopyToClipboard 000000018005ee5c     service.obj
 0001:0005de5c       $unwind$__scrt_uninitialize_crt 000000018005ee5c     LIBCMT:utility.obj
 0001:0005de5c       $unwind$timer_tostring     000000018005ee5c     service.obj
 0001:0005de5c       $unwind$__scrt_initialize_crt 000000018005ee5c     LIBCMT:utility.obj
 0001:0005de5c       $unwind$TimerCallback      000000018005ee5c     service.obj
 0001:0005de5c       $unwind$__acrt_get_process_end_policy 000000018005ee5c     libucrt:win_policies.obj
 0001:0005de5c       $unwind$far_FarClock       000000018005ee5c     service.obj
 0001:0005de5c       $unwind$SetFarColors       000000018005ee5c     keysandcolors.obj
 0001:0005de5c       $unwind$?scan_optional_field_width@?$format_string_parser@D@__crt_stdio_input@@AEAA_NXZ 000000018005ee5c     libucrt:input.obj
 0001:0005de5c       $unwind$__acrt_update_multibyte_info 000000018005ee5c     libucrt:locale_update.obj
 0001:0005de5c       $unwind$_clrfp             000000018005ee5c     libucrt:fpctrl.obj
 0001:0005de5c       $unwind$__scrt_release_startup_lock 000000018005ee5c     LIBCMT:utility.obj
 0001:0005de64       $unwind$editor_UndoRedo    000000018005ee64     service.obj
 0001:0005de64       $unwind$f_new              000000018005ee64     bit64.obj
 0001:0005de74       $chain$0$f_new             000000018005ee74     bit64.obj
 0001:0005de88       $chain$1$f_new             000000018005ee88     bit64.obj
 0001:0005de98       $unwind$far_FarMacroCallToLua 000000018005ee98     luamacro.obj
 0001:0005de98       $unwind$win_GetConsoleScreenBufferInfo 000000018005ee98     win.obj
 0001:0005de98       $unwind$__scrt_initialize_onexit_tables 000000018005ee98     LIBCMT:utility.obj
 0001:0005de98       $unwind$_isleadbyte_l      000000018005ee98     libucrt:_wctype.obj
 0001:0005de98       $unwind$__dcrt_lowio_ensure_console_output_initialized 000000018005ee98     libucrt:initcon.obj
 0001:0005de98       $unwind$f_tostring         000000018005ee98     bit64.obj
 0001:0005de98       $unwind$?getSystemCP@@YAHH@Z 000000018005ee98     libucrt:mbctype.obj
 0001:0005dea0       $unwind$io_lines           000000018005eea0     uliolib51.obj
 0001:0005dea0       $unwind$f_type             000000018005eea0     bit64.obj
 0001:0005dea8       $chain$0$f_type            000000018005eea8     bit64.obj
 0001:0005debc       $chain$1$f_type            000000018005eebc     bit64.obj
 0001:0005decc       $unwind$__acrt_getptd_noexit 000000018005eecc     libucrt:per_thread_data.obj
 0001:0005decc       $unwind$_DllMainCRTStartup 000000018005eecc     LIBCMT:dll_dllmain.obj
 0001:0005decc       $unwind$LF_InitLuaState1   000000018005eecc     service.obj
 0001:0005decc       $unwind$uc_newindex        000000018005eecc     lusercontrol.obj
 0001:0005decc       $unwind$__acrt_InitializeCriticalSectionEx 000000018005eecc     libucrt:winapi_thunks.obj
 0001:0005decc       $unwind$LF_Configure       000000018005eecc     exported.obj
 0001:0005decc       $unwind$win_wcscmp         000000018005eecc     win.obj
 0001:0005decc       $unwind$__vcrt_getptd_noexit 000000018005eecc     libvcruntime:per_thread_data.obj
 0001:0005decc       $unwind$luaB_dofileW       000000018005eecc     lflua.obj
 0001:0005decc       $unwind$get_env_flag       000000018005eecc     service.obj
 0001:0005decc       $unwind$__acrt_getptd      000000018005eecc     libucrt:per_thread_data.obj
 0001:0005decc       $unwind$__vcrt_InitializeCriticalSectionEx 000000018005eecc     libvcruntime:winapi_downlevel.obj
 0001:0005decc       $unwind$??0_LocaleUpdate@@QEAA@QEAU__crt_locale_pointers@@@Z 000000018005eecc     libucrt:output.obj
 0001:0005decc       $unwind$OptFlags           000000018005eecc     service.obj
 0001:0005decc       $unwind$?type_case_n@?$output_processor@DV?$stream_output_adapter@D@__crt_stdio_output@@V?$standard_base@DV?$stream_output_adapter@D@__crt_stdio_output@@@2@@__crt_stdio_output@@AEAA_NXZ 000000018005eecc     libucrt:output.obj
 0001:0005decc       $unwind$LF_SetFindList     000000018005eecc     exported.obj
 0001:0005decc       $unwind$LF_SetDirectory    000000018005eecc     exported.obj
 0001:0005decc       $unwind$LF_PutFiles        000000018005eecc     exported.obj
 0001:0005decc       $unwind$__acrt_stdio_flush_nolock 000000018005eecc     libucrt:fflush.obj
 0001:0005decc       $unwind$?free_crt_array_internal@@YAXQEAPEBX_K@Z 000000018005eecc     libucrt:inittime.obj
 0001:0005decc       $unwind$LF_ProcessViewerEvent 000000018005eecc     exported.obj
 0001:0005decc       $unwind$??R<lambda_ca71763b3c0644891230e4f79ea54fa6>@@QEBAHXZ 000000018005eecc     libucrt:setvbuf.obj
 0001:0005decc       $unwind$check_env_flag     000000018005eecc     service.obj
 0001:0005decc       $unwind$?type_case_n@?$output_processor@DV?$string_output_adapter@D@__crt_stdio_output@@V?$standard_base@DV?$string_output_adapter@D@__crt_stdio_output@@@2@@__crt_stdio_output@@AEAA_NXZ 000000018005eecc     libucrt:output.obj
 0001:0005decc       $unwind$PutVersionInfoToTable 000000018005eecc     service.obj
 0001:0005decc       $unwind$ll_require         000000018005eecc     uloadlib51.obj
 0001:0005decc       $unwind$PushDMParams       000000018005eecc     service.obj
 0001:0005decc       $unwind$loader_C           000000018005eecc     uloadlib51.obj
 0001:0005decc       $unwind$memcpy_s           000000018005eecc     libucrt:cfout.obj
 0001:0005decc       $unwind$luaopen_uio        000000018005eecc     uliolib51.obj
 0001:0005decc       $unwind$f_flush            000000018005eecc     uliolib51.obj
 0001:0005decc       $unwind$io_flush           000000018005eecc     uliolib51.obj
 0001:0005decc       $unwind$f_setvbuf          000000018005eecc     uliolib51.obj
 0001:0005decc       $unwind$f_seek             000000018005eecc     uliolib51.obj
 0001:0005decc       $unwind$far_DialogRun      000000018005eecc     service.obj
 0001:0005decc       $unwind$io_readline        000000018005eecc     uliolib51.obj
 0001:0005decc       $unwind$?type_case_Z@?$output_processor@_WV?$string_output_adapter@_W@__crt_stdio_output@@V?$standard_base@_WV?$string_output_adapter@_W@__crt_stdio_output@@@2@@__crt_stdio_output@@AEAA_NXZ 000000018005eecc     libucrt:output.obj
 0001:0005decc       $unwind$?type_case_s@?$output_processor@_WV?$string_output_adapter@_W@__crt_stdio_output@@V?$standard_base@_WV?$string_output_adapter@_W@__crt_stdio_output@@@2@@__crt_stdio_output@@AEAA_NXZ 000000018005eecc     libucrt:output.obj
 0001:0005decc       $unwind$f_mod              000000018005eecc     bit64.obj
 0001:0005decc       $unwind$io_fclose          000000018005eecc     uliolib51.obj
 0001:0005decc       $unwind$io_pclose          000000018005eecc     uliolib51.obj
 0001:0005decc       $unwind$?common_fseek_nolock@@YAHV__crt_stdio_stream@@_JH@Z 000000018005eecc     libucrt:fseek.obj
 0001:0005decc       $unwind$fileerror          000000018005eecc     uliolib51.obj
 0001:0005decc       $unwind$??$common_lseek_nolock@_J@@YA_JH_JH@Z 000000018005eecc     libucrt:lseek.obj
 0001:0005decc       $unwind$?type_case_n@?$output_processor@_WV?$string_output_adapter@_W@__crt_stdio_output@@V?$standard_base@_WV?$string_output_adapter@_W@__crt_stdio_output@@@2@@__crt_stdio_output@@AEAA_NXZ 000000018005eecc     libucrt:output.obj
 0001:0005decc       $unwind$LF_ProcessPanelInput 000000018005eecc     exported.obj
 0001:0005decc       $unwind$__acrt_stdio_flush_and_write_narrow_nolock 000000018005eecc     libucrt:_flsbuf.obj
 0001:0005decc       $unwind$_exception_enabled 000000018005eecc     libucrt:libm_error.obj
 0001:0005decc       $unwind$LF_ProcessPanelEvent 000000018005eecc     exported.obj
 0001:0005decc       $unwind$LF_ProcessHostFile 000000018005eecc     exported.obj
 0001:0005decc       $unwind$??$skip_whitespace@Vstream_input_adapter@__crt_stdio_input@@D@__crt_stdio_input@@YAHAEAV?$stream_input_adapter@D@0@QEAU__crt_locale_pointers@@@Z 000000018005eecc     libucrt:input.obj
 0001:0005decc       $unwind$match_class        000000018005eecc     lutf8lib.obj
 0001:0005decc       $unwind$?advance@?$format_string_parser@D@__crt_stdio_input@@QEAA_NXZ 000000018005eecc     libucrt:input.obj
 0001:0005decc       $unwind$?process_string_specifier@?$input_processor@DV?$stream_input_adapter@D@__crt_stdio_input@@@__crt_stdio_input@@AEAA_NW4conversion_mode@2@@Z 000000018005eecc     libucrt:input.obj
 0001:0005decc       $unwind$memcpy_s           000000018005eecc     libucrt:input.obj
 0001:0005decc       $unwind$utf8_index         000000018005eecc     lutf8lib.obj
 0001:0005decc       $unwind$__acrt_execute_initializers 000000018005eecc     libucrt:shared_initialization.obj
 0001:0005decc       $unwind$push_flags_table   000000018005eecc     flags.obj
 0001:0005decc       $unwind$FillEditorSelect   000000018005eecc     service.obj
 0001:0005decc       $unwind$??$common_ftell_nolock@_J@@YA_JV__crt_stdio_stream@@@Z 000000018005eecc     libucrt:ftell.obj
 0001:0005decc       $unwind$__acrt_stdio_free_tmpfile_name_buffers_nolock 000000018005eecc     libucrt:tmpfile.obj
 0001:0005decc       $unwind$??R<lambda_96f4279ff90247a4c5c5d9824f56f8c1>@@QEBA_KXZ 000000018005eecc     libucrt:fwrite.obj
 0001:0005dedc       $unwind$LF_GetFindData     000000018005eedc     exported.obj
 0001:0005dedc       $unwind$LF_Compare         000000018005eedc     exported.obj
 0001:0005dedc       $unwind$LF_GetFiles        000000018005eedc     exported.obj
 0001:0005dedc       $unwind$_AddStringToCollector 000000018005eedc     exported.obj
 0001:0005dedc       $unwind$LF_ClosePanel      000000018005eedc     exported.obj
 0001:0005dedc       $unwind$LF_MakeDirectory   000000018005eedc     exported.obj
 0001:0005dee8       $chain$0$LF_ClosePanel     000000018005eee8     exported.obj
 0001:0005defc       $chain$1$LF_ClosePanel     000000018005eefc     exported.obj
 0001:0005df0c       $chain$0$LF_Compare        000000018005ef0c     exported.obj
 0001:0005df20       $chain$2$LF_Compare        000000018005ef20     exported.obj
 0001:0005df34       $chain$3$LF_Compare        000000018005ef34     exported.obj
 0001:0005df44       $unwind$LF_DeleteFiles     000000018005ef44     exported.obj
 0001:0005df54       $chain$0$LF_DeleteFiles    000000018005ef54     exported.obj
 0001:0005df68       $chain$2$LF_DeleteFiles    000000018005ef68     exported.obj
 0001:0005df7c       $chain$3$LF_DeleteFiles    000000018005ef7c     exported.obj
 0001:0005df8c       $chain$0$LF_GetFiles       000000018005ef8c     exported.obj
 0001:0005dfa0       $chain$2$LF_GetFiles       000000018005efa0     exported.obj
 0001:0005dfb4       $chain$3$LF_GetFiles       000000018005efb4     exported.obj
 0001:0005dfc4       $chain$0$LF_GetFindData    000000018005efc4     exported.obj
 0001:0005dfd8       $chain$1$LF_GetFindData    000000018005efd8     exported.obj
 0001:0005dfe8       $unwind$LF_GetGlobalInfo   000000018005efe8     exported.obj
 0001:0005dffc       $chain$2$LF_GetGlobalInfo  000000018005effc     exported.obj
 0001:0005e014       $chain$3$LF_GetGlobalInfo  000000018005f014     exported.obj
 0001:0005e028       $chain$4$LF_GetGlobalInfo  000000018005f028     exported.obj
 0001:0005e038       $unwind$LF_GetOpenPanelInfo 000000018005f038     exported.obj
 0001:0005e044       $chain$1$LF_GetOpenPanelInfo 000000018005f044     exported.obj
 0001:0005e05c       $chain$3$LF_GetOpenPanelInfo 000000018005f05c     exported.obj
 0001:0005e074       $chain$5$LF_GetOpenPanelInfo 000000018005f074     exported.obj
 0001:0005e08c       $chain$7$LF_GetOpenPanelInfo 000000018005f08c     exported.obj
 0001:0005e0a4       $chain$8$LF_GetOpenPanelInfo 000000018005f0a4     exported.obj
 0001:0005e0b4       $chain$9$LF_GetOpenPanelInfo 000000018005f0b4     exported.obj
 0001:0005e0c4       $chain$10$LF_GetOpenPanelInfo 000000018005f0c4     exported.obj
 0001:0005e0d4       $unwind$LF_GetPluginInfo   000000018005f0d4     exported.obj
 0001:0005e0e0       $chain$1$LF_GetPluginInfo  000000018005f0e0     exported.obj
 0001:0005e0f8       $chain$2$LF_GetPluginInfo  000000018005f0f8     exported.obj
 0001:0005e108       $chain$0$LF_MakeDirectory  000000018005f108     exported.obj
 0001:0005e11c       $chain$2$LF_MakeDirectory  000000018005f11c     exported.obj
 0001:0005e130       $chain$3$LF_MakeDirectory  000000018005f130     exported.obj
 0001:0005e140       $unwind$AddBufToCollector  000000018005f140     exported.obj
 0001:0005e140       $unwind$LF_DoFile          000000018005f140     service.obj
 0001:0005e140       $unwind$ll_loadfunc        000000018005f140     uloadlib51.obj
 0001:0005e140       $unwind$PushDNParams       000000018005f140     service.obj
 0001:0005e140       $unwind$luaopen_far        000000018005f140     service.obj
 0001:0005e140       $unwind$win_MoveFile       000000018005f140     win.obj
 0001:0005e140       $unwind$push_offset        000000018005f140     lutf8lib.obj
 0001:0005e140       $unwind$win_CreateDir      000000018005f140     win.obj
 0001:0005e140       $unwind$timer_newindex     000000018005f140     service.obj
 0001:0005e140       $unwind$FrsUserFunc        000000018005f140     service.obj
 0001:0005e140       $unwind$start_capture      000000018005f140     lutf8lib.obj
 0001:0005e140       $unwind$LF_ProcessDialogEvent 000000018005f140     exported.obj
 0001:0005e140       $unwind$LF_Open            000000018005f140     exported.obj
 0001:0005e158       $chain$0$LF_ProcessEditorEvent 000000018005f158     exported.obj
 0001:0005e16c       $chain$1$LF_ProcessEditorEvent 000000018005f16c     exported.obj
 0001:0005e17c       $chain$0$LF_ProcessConsoleInput 000000018005f17c     exported.obj
 0001:0005e190       $chain$1$LF_ProcessConsoleInput 000000018005f190     exported.obj
 0001:0005e1a0       $unwind$capture_previous_context 000000018005f1a0     LIBCMT:gs_report.obj
 0001:0005e1a0       $unwind$LF_ProcessSynchroEvent 000000018005f1a0     exported.obj
 0001:0005e1ac       $chain$1$LF_ProcessSynchroEvent 000000018005f1ac     exported.obj
 0001:0005e1c4       $chain$2$LF_ProcessSynchroEvent 000000018005f1c4     exported.obj
 0001:0005e1d8       $chain$3$LF_ProcessSynchroEvent 000000018005f1d8     exported.obj
 0001:0005e1e8       $chain$5$LF_ProcessSynchroEvent 000000018005f1e8     exported.obj
 0001:0005e1fc       $chain$6$LF_ProcessSynchroEvent 000000018005f1fc     exported.obj
 0001:0005e20c       $unwind$PutPluginMenuItemToTable 000000018005f20c     service.obj
 0001:0005e20c       $unwind$LF_GetContentFields 000000018005f20c     exported.obj
 0001:0005e20c       $unwind$?parse_int_from_format_string@?$output_processor@_WV?$string_output_adapter@_W@__crt_stdio_output@@V?$standard_base@_WV?$string_output_adapter@_W@__crt_stdio_output@@@2@@__crt_stdio_output@@AEAA_NQEAH@Z 000000018005f20c     libucrt:output.obj
 0001:0005e20c       $unwind$LF_GetContentData  000000018005f20c     exported.obj
 0001:0005e220       $chain$0$LF_GetContentFields 000000018005f220     exported.obj
 0001:0005e234       $chain$1$LF_GetContentFields 000000018005f234     exported.obj
 0001:0005e244       $chain$0$LF_GetContentData 000000018005f244     exported.obj
 0001:0005e258       $chain$1$LF_GetContentData 000000018005f258     exported.obj
 0001:0005e268       $unwind$classend           000000018005f268     lutf8lib.obj
 0001:0005e268       $unwind$PackMacroValues    000000018005f268     exported.obj
 0001:0005e27c       $chain$0$PackMacroValues   000000018005f27c     exported.obj
 0001:0005e290       $chain$1$PackMacroValues   000000018005f290     exported.obj
 0001:0005e2a0       $chain$0$_AddStringToCollector 000000018005f2a0     exported.obj
 0001:0005e2b4       $chain$1$_AddStringToCollector 000000018005f2b4     exported.obj
 0001:0005e2c4       $unwind$CreateStringsArray 000000018005f2c4     exported.obj
 0001:0005e2d8       $chain$1$CreateStringsArray 000000018005f2d8     exported.obj
 0001:0005e2f0       $chain$2$CreateStringsArray 000000018005f2f0     exported.obj
 0001:0005e300       $unwind$FillPluginPanelItem 000000018005f300     exported.obj
 0001:0005e300       $unwind$far_GetPlugins     000000018005f300     service.obj
 0001:0005e30c       $chain$1$FillPluginPanelItem 000000018005f30c     exported.obj
 0001:0005e324       $chain$2$FillPluginPanelItem 000000018005f324     exported.obj
 0001:0005e338       $chain$3$FillPluginPanelItem 000000018005f338     exported.obj
 0001:0005e348       $chain$4$FillPluginPanelItem 000000018005f348     exported.obj
 0001:0005e358       $unwind$FillFindData       000000018005f358     exported.obj
 0001:0005e368       $chain$2$FillFindData      000000018005f368     exported.obj
 0001:0005e384       $chain$3$FillFindData      000000018005f384     exported.obj
 0001:0005e394       $unwind$UpdateFileSelection 000000018005f394     exported.obj
 0001:0005e3a4       $chain$0$UpdateFileSelection 000000018005f3a4     exported.obj
 0001:0005e3b8       $chain$1$UpdateFileSelection 000000018005f3b8     exported.obj
 0001:0005e3c8       $unwind$RunDefaultScript   000000018005f3c8     exported.obj
 0001:0005e3e0       $chain$0$RunDefaultScript  000000018005f3e0     exported.obj
 0001:0005e3f4       $chain$1$RunDefaultScript  000000018005f3f4     exported.obj
 0001:0005e404       $unwind$FillFarMacroCall_Callback 000000018005f404     exported.obj
 0001:0005e410       $chain$0$FillFarMacroCall_Callback 000000018005f410     exported.obj
 0001:0005e424       $chain$1$FillFarMacroCall_Callback 000000018005f424     exported.obj
 0001:0005e434       $unwind$FillFarMacroCall   000000018005f434     exported.obj
 0001:0005e444       $chain$3$FillFarMacroCall  000000018005f444     exported.obj
 0001:0005e464       $chain$4$FillFarMacroCall  000000018005f464     exported.obj
 0001:0005e474       $unwind$getPluginMenuItems 000000018005f474     exported.obj
 0001:0005e48c       $unwind$LF_Gsub            000000018005f48c     lflua.obj
 0001:0005e4ac       $unwind$LF_LoadFile        000000018005f4ac     lflua.obj
 0001:0005e4c0       $chain$1$LF_LoadFile       000000018005f4c0     lflua.obj
 0001:0005e4d8       $chain$2$LF_LoadFile       000000018005f4d8     lflua.obj
 0001:0005e4d8       $chain$4$LF_LoadFile       000000018005f4d8     lflua.obj
 0001:0005e4e8       $chain$3$LF_LoadFile       000000018005f4e8     lflua.obj
 0001:0005e500       $unwind$getF               000000018005f500     lflua.obj
 0001:0005e510       $unwind$errfile            000000018005f510     lflua.obj
 0001:0005e510       $unwind$_invalid_parameter 000000018005f510     libucrt:invalid_parameter.obj
 0001:0005e510       $unwind$??$common_lseek_nolock@J@@YAJHJH@Z 000000018005f510     libucrt:lseek.obj
 0001:0005e510       $unwind$luaLF_FieldError   000000018005f510     util.obj
 0001:0005e510       $unwind$luaLF_SlotError    000000018005f510     util.obj
 0001:0005e510       $unwind$_wcsdup            000000018005f510     libucrt:wcsdup.obj
 0001:0005e524       $unwind$check_regex_pattern 000000018005f524     lregex.obj
 0001:0005e534       $chain$1$check_regex_pattern 000000018005f534     lregex.obj
 0001:0005e54c       $chain$2$check_regex_pattern 000000018005f54c     lregex.obj
 0001:0005e55c       $unwind$_regex_gmatch_closure 000000018005f55c     lregex.obj
 0001:0005e56c       $chain$1$_regex_gmatch_closure 000000018005f56c     lregex.obj
 0001:0005e584       $chain$2$_regex_gmatch_closure 000000018005f584     lregex.obj
 0001:0005e598       $chain$3$_regex_gmatch_closure 000000018005f598     lregex.obj
 0001:0005e5a8       $unwind$_Gmatch            000000018005f5a8     lregex.obj
 0001:0005e5c0       $unwind$rx_find_match      000000018005f5c0     lregex.obj
 0001:0005e5dc       $unwind$rx_gsub            000000018005f5dc     lregex.obj
 0001:0005e5f8       $unwind$FL_PushParams      000000018005f5f8     luamacro.obj
 0001:0005e604       $chain$0$FL_PushParams     000000018005f604     luamacro.obj
 0001:0005e618       $chain$1$FL_PushParams     000000018005f618     luamacro.obj
 0001:0005e62c       $chain$2$FL_PushParams     000000018005f62c     luamacro.obj
 0001:0005e640       $chain$3$FL_PushParams     000000018005f640     luamacro.obj
 0001:0005e650       $chain$4$FL_PushParams     000000018005f650     luamacro.obj
 0001:0005e660       $chain$5$FL_PushParams     000000018005f660     luamacro.obj
 0001:0005e670       $unwind$Open_Luamacro      000000018005f670     luamacro.obj
 0001:0005e684       $chain$0$Open_Luamacro     000000018005f684     luamacro.obj
 0001:0005e698       $chain$1$Open_Luamacro     000000018005f698     luamacro.obj
 0001:0005e6a8       $unwind$far_MacroCallFar   000000018005f6a8     luamacro.obj
 0001:0005e6b8       $chain$2$far_MacroCallFar  000000018005f6b8     luamacro.obj
 0001:0005e6d4       $chain$3$far_MacroCallFar  000000018005f6d4     luamacro.obj
 0001:0005e6e8       $chain$4$far_MacroCallFar  000000018005f6e8     luamacro.obj
 0001:0005e6f8       $chain$5$far_MacroCallFar  000000018005f6f8     luamacro.obj
 0001:0005e708       $chain$0$far_FarMacroCallToLua 000000018005f708     luamacro.obj
 0001:0005e71c       $chain$1$far_FarMacroCallToLua 000000018005f71c     luamacro.obj
 0001:0005e72c       $unwind$uc_index           000000018005f72c     lusercontrol.obj
 0001:0005e73c       $unwind$CreateRegKey       000000018005f73c     reg.obj
 0001:0005e73c       $unwind$viewer_SetPosition 000000018005f73c     service.obj
 0001:0005e744       $unwind$check_utf8_string  000000018005f744     ustring.obj
 0001:0005e744       $unwind$_ui64toa_s         000000018005f744     libucrt:xtoa.obj
 0001:0005e744       $unwind$utf8_to_utf16      000000018005f744     ustring.obj
 0001:0005e744       $unwind$strtol             000000018005f744     libucrt:strtox.obj
 0001:0005e744       $unwind$_sopen_s           000000018005f744     libucrt:open.obj
 0001:0005e744       $unwind$??$parse_floating_point_write_result@N@__crt_strtox@@YA?AW4SLD_STATUS@@W4floating_point_parse_result@0@AEBUfloating_point_string@0@QEAN@Z 000000018005f744     libucrt:input.obj
 0001:0005e744       $unwind$_wfreopen          000000018005f744     libucrt:freopen.obj
 0001:0005e744       $unwind$?as_float@floating_point_value@__crt_strtox@@QEBAAEAMXZ 000000018005f744     libucrt:input.obj
 0001:0005e744       $unwind$_log10_special     000000018005f744     libucrt:log_special.obj
 0001:0005e744       $unwind$fread              000000018005f744     libucrt:fread.obj
 0001:0005e744       $unwind$OpenRegKey         000000018005f744     reg.obj
 0001:0005e744       $unwind$push_utf8_string   000000018005f744     ustring.obj
 0001:0005e744       $unwind$?as_double@floating_point_value@__crt_strtox@@QEBAAEANXZ 000000018005f744     libucrt:input.obj
 0001:0005e744       $unwind$_wdupenv_s         000000018005f744     libucrt:getenv.obj
 0001:0005e744       $unwind$fflush             000000018005f744     libucrt:fflush.obj
 0001:0005e744       $unwind$strtoull           000000018005f744     libucrt:strtox.obj
 0001:0005e744       $unwind$wctomb_s           000000018005f744     libucrt:wctomb.obj
 0001:0005e744       $unwind$wcstol             000000018005f744     libucrt:strtox.obj
 0001:0005e744       $unwind$_wsopen_s          000000018005f744     libucrt:open.obj
 0001:0005e744       $unwind$??$parse_floating_point_write_result@M@__crt_strtox@@YA?AW4SLD_STATUS@@W4floating_point_parse_result@0@AEBUfloating_point_string@0@QEAM@Z 000000018005f744     libucrt:input.obj
 0001:0005e744       $unwind$_invalid_parameter_noinfo 000000018005f744     libucrt:invalid_parameter.obj
 0001:0005e74c       $unwind$SetRegKeyStr       000000018005f74c     reg.obj
 0001:0005e75c       $chain$0$SetRegKeyStr      000000018005f75c     reg.obj
 0001:0005e770       $chain$1$SetRegKeyStr      000000018005f770     reg.obj
 0001:0005e780       $unwind$SetRegKeyDword     000000018005f780     reg.obj
 0001:0005e78c       $chain$0$SetRegKeyDword    000000018005f78c     reg.obj
 0001:0005e7a0       $chain$1$SetRegKeyDword    000000018005f7a0     reg.obj
 0001:0005e7b0       $unwind$SetRegKeyArr       000000018005f7b0     reg.obj
 0001:0005e7c0       $chain$0$SetRegKeyArr      000000018005f7c0     reg.obj
 0001:0005e7d4       $chain$1$SetRegKeyArr      000000018005f7d4     reg.obj
 0001:0005e7e4       $unwind$__dcrt_uninitialize_environments_nolock 000000018005f7e4     libucrt:environment_initialization.obj
 0001:0005e7e4       $unwind$__dcrt_get_or_create_wide_environment_nolock 000000018005f7e4     libucrt:environment_initialization.obj
 0001:0005e7e4       $unwind$_wcsicmp           000000018005f7e4     libucrt:wcsicmp.obj
 0001:0005e7e4       $unwind$_fileno            000000018005f7e4     libucrt:fileno.obj
 0001:0005e7e4       $unwind$__scrt_initialize_default_local_stdio_options 000000018005f7e4     LIBCMT:default_local_stdio_options.obj
 0001:0005e7e4       $unwind$?state_case_size@?$output_processor@_WV?$string_output_adapter@_W@__crt_stdio_output@@V?$standard_base@_WV?$string_output_adapter@_W@__crt_stdio_output@@@2@@__crt_stdio_output@@AEAA_NXZ 000000018005f7e4     libucrt:output.obj
 0001:0005e7e4       $unwind$??$uninitialize_environment_internal@D@@YAXAEAPEAPEAD@Z 000000018005f7e4     libucrt:environment_initialization.obj
 0001:0005e7e4       $unwind$far_DialogFree     000000018005f7e4     service.obj
 0001:0005e7e4       $unwind$??$uninitialize_environment_internal@_W@@YAXAEAPEAPEA_W@Z 000000018005f7e4     libucrt:environment_initialization.obj
 0001:0005e7e4       $unwind$_invoke_watson     000000018005f7e4     libucrt:invalid_parameter.obj
 0001:0005e7e4       $unwind$__scrt_dllmain_crt_thread_detach 000000018005f7e4     LIBCMT:utility.obj
 0001:0005e7e4       $unwind$__report_rangecheckfailure 000000018005f7e4     LIBCMT:gs_report.obj
 0001:0005e7e4       $unwind$fegetround         000000018005f7e4     libucrt:fegetround.obj
 0001:0005e7e4       $unwind$_set_errno_from_matherr 000000018005f7e4     libucrt:fpexcept.obj
 0001:0005e7e4       $unwind$__vcrt_uninitialize 000000018005f7e4     libvcruntime:initialization.obj
 0001:0005e7e4       $unwind$?dllmain_crt_dispatch@@YAHQEAUHINSTANCE__@@KQEAX@Z 000000018005f7e4     LIBCMT:dll_dllmain.obj
 0001:0005e7e4       $unwind$__acrt_update_thread_multibyte_data 000000018005f7e4     libucrt:mbctype.obj
 0001:0005e7e4       $unwind$abort              000000018005f7e4     libucrt:abort.obj
 0001:0005e7e4       $unwind$__acrt_AreFileApisANSI 000000018005f7e4     libucrt:winapi_thunks.obj
 0001:0005e7e4       $unwind$__vcrt_initialize_ptd 000000018005f7e4     libvcruntime:per_thread_data.obj
 0001:0005e7e4       $unwind$__scrt_dllmain_uninitialize_critical 000000018005f7e4     LIBCMT:utility.obj
 0001:0005e7e4       $unwind$_isatty            000000018005f7e4     libucrt:isatty.obj
 0001:0005e7e4       $unwind$__vcrt_thread_detach 000000018005f7e4     libvcruntime:initialization.obj
 0001:0005e7e4       $unwind$__acrt_uninitialize_tmpfile 000000018005f7e4     libucrt:rmtmp.obj
 0001:0005e7e4       $unwind$__vcrt_uninitialize_ptd 000000018005f7e4     libvcruntime:per_thread_data.obj
 0001:0005e7e4       $unwind$__acrt_DownlevelLocaleNameToLCID 000000018005f7e4     libucrt:lcidtoname_downlevel.obj
 0001:0005e7e4       $unwind$win_GetVirtualKeys 000000018005f7e4     win.obj
 0001:0005e7e4       $unwind$far_SubscribeDialogDrawEvents 000000018005f7e4     service.obj
 0001:0005e7e4       $unwind$tolower            000000018005f7e4     libucrt:tolower_toupper.obj
 0001:0005e7e4       $unwind$__GSHandlerCheck   000000018005f7e4     LIBCMT:gshandler.obj
 0001:0005e7e4       $unwind$?state_case_size@?$output_processor@DV?$string_output_adapter@D@__crt_stdio_output@@V?$standard_base@DV?$string_output_adapter@D@__crt_stdio_output@@@2@@__crt_stdio_output@@AEAA_NXZ 000000018005f7e4     libucrt:output.obj
 0001:0005e7e4       $unwind$__scrt_dllmain_crt_thread_attach 000000018005f7e4     LIBCMT:utility.obj
 0001:0005e7e4       $unwind$__vcrt_thread_attach 000000018005f7e4     libvcruntime:initialization.obj
 0001:0005e7e4       $unwind$?__c32rtomb_utf8@__crt_mbstring@@YA_KPEAD_UPEAU_Mbstatet@@@Z 000000018005f7e4     libucrt:c32rtomb.obj
 0001:0005e7e4       $unwind$feof               000000018005f7e4     libucrt:feoferr.obj
 0001:0005e7e4       $unwind$?state_case_normal_tchar@?$output_processor@DV?$string_output_adapter@D@__crt_stdio_output@@V?$standard_base@DV?$string_output_adapter@D@__crt_stdio_output@@@2@@__crt_stdio_output@@AEAA_ND@Z 000000018005f7e4     libucrt:output.obj
 0001:0005e7e4       $unwind$_fgetc_nolock      000000018005f7e4     libucrt:fgetc.obj
 0001:0005e7e4       $unwind$?initialize_multibyte@@YAHXZ 000000018005f7e4     libucrt:multibyte_initializer.obj
 0001:0005e7e4       $unwind$win_IsProcess64bit 000000018005f7e4     win.obj
 0001:0005e7e4       $unwind$__acrt_uninitialize 000000018005f7e4     libucrt:initialization.obj
 0001:0005e7e4       $unwind$__acrt_uninitialize_critical 000000018005f7e4     libucrt:initialization.obj
 0001:0005e7e4       $unwind$__acrt_thread_attach 000000018005f7e4     libucrt:initialization.obj
 0001:0005e7e4       $unwind$__dcrt_terminate_console_output 000000018005f7e4     libucrt:initcon.obj
 0001:0005e7e4       $unwind$__acrt_thread_detach 000000018005f7e4     libucrt:initialization.obj
 0001:0005e7e4       $unwind$initialize_c       000000018005f7e4     libucrt:initialization.obj
 0001:0005e7e4       $unwind$ferror             000000018005f7e4     libucrt:feoferr.obj
 0001:0005e7e4       $unwind$_wcsnicmp          000000018005f7e4     libucrt:wcsnicmp.obj
 0001:0005e7e4       $unwind$uninitialize_environment 000000018005f7e4     libucrt:initialization.obj
 0001:0005e7e4       $unwind$__vcrt_freefls     000000018005f7e4     libvcruntime:per_thread_data.obj
 0001:0005e7e4       $unwind$__vcrt_initialize  000000018005f7e4     libvcruntime:initialization.obj
 0001:0005e7e4       $unwind$__pctype_func      000000018005f7e4     libucrt:ctype.obj
 0001:0005e7e4       $unwind$__scrt_acquire_startup_lock 000000018005f7e4     LIBCMT:utility.obj
 0001:0005e7e4       $unwind$_statfp            000000018005f7e4     libucrt:fpctrl.obj
 0001:0005e7e4       $unwind$_get_osfhandle     000000018005f7e4     libucrt:osfinfo.obj
 0001:0005e7e4       $unwind$DllMain            000000018005f7e4     service.obj
 0001:0005e7e4       $unwind$_msize_base        000000018005f7e4     libucrt:msize.obj
 0001:0005e7e4       $unwind$__acrt_initialize_multibyte 000000018005f7e4     libucrt:mbctype.obj
 0001:0005e7e4       $unwind$luaopen_unicode    000000018005f7e4     slnunico.obj
 0001:0005e7e4       $unwind$_wcsnicoll         000000018005f7e4     libucrt:wcsnicol.obj
 0001:0005e7e4       $unwind$uninitialize_allocated_io_buffers 000000018005f7e4     libucrt:initialization.obj
 0001:0005e7e4       $unwind$__acrt_initialize_ptd 000000018005f7e4     libucrt:per_thread_data.obj
 0001:0005e7e4       $unwind$?state_case_size@?$output_processor@DV?$stream_output_adapter@D@__crt_stdio_output@@V?$standard_base@DV?$stream_output_adapter@D@__crt_stdio_output@@@2@@__crt_stdio_output@@AEAA_NXZ 000000018005f7e4     libucrt:output.obj
 0001:0005e7e4       $unwind$writer             000000018005f7e4     slnunico.obj
 0001:0005e7e4       $unwind$__vcrt_uninitialize_critical 000000018005f7e4     libvcruntime:initialization.obj
 0001:0005e7e4       $unwind$GetPluginData      000000018005f7e4     service.obj
 0001:0005e7e4       $unwind$__scrt_dllmain_before_initialize_c 000000018005f7e4     LIBCMT:utility.obj
 0001:0005e7e4       $unwind$_get_fmode         000000018005f7e4     libucrt:setmode.obj
 0001:0005e7e4       $unwind$_stricmp           000000018005f7e4     libucrt:stricmp.obj
 0001:0005e7e4       $unwind$__acrt_initialize_heap 000000018005f7e4     libucrt:heap_handle.obj
 0001:0005e7e4       $unwind$ustring_Sleep      000000018005f7e4     ustring.obj
 0001:0005e7e4       $unwind$__scrt_dllmain_after_initialize_c 000000018005f7e4     LIBCMT:utility.obj
 0001:0005e7e4       $unwind$__acrt_initialize_command_line 000000018005f7e4     libucrt:argv_data.obj
 0001:0005e7e4       $unwind$dir_exist          000000018005f7e4     service.obj
 0001:0005e7e4       $unwind$__doserrno         000000018005f7e4     libucrt:errno.obj
 0001:0005e7e4       $unwind$?validate_stream_is_ansi_if_required@?$__acrt_stdio_char_traits@D@@SA_NQEAU_iobuf@@@Z 000000018005f7e4     libucrt:output.obj
 0001:0005e7e4       $unwind$__scrt_dllmain_uninitialize_c 000000018005f7e4     LIBCMT:utility.obj
 0001:0005e7e4       $unwind$tmpfile            000000018005f7e4     libucrt:tmpfile.obj
 0001:0005e7e4       $unwind$__acrt_release_locale_ref 000000018005f7e4     libucrt:locale_refcounting.obj
 0001:0005e7e4       $unwind$_errno             000000018005f7e4     libucrt:errno.obj
 0001:0005e7e4       $unwind$__acrt_uninitialize_ptd 000000018005f7e4     libucrt:per_thread_data.obj
 0001:0005e7ec       $unwind$LF_DlgProc         000000018005f7ec     service.obj
 0001:0005e7fc       $chain$1$LF_DlgProc        000000018005f7fc     service.obj
 0001:0005e814       $chain$2$LF_DlgProc        000000018005f814     service.obj
 0001:0005e824       $unwind$LF_Message         000000018005f824     service.obj
 0001:0005e840       $unwind$LF_RunLuafarInit   000000018005f840     service.obj
 0001:0005e84c       $unwind$PushPanelItem      000000018005f84c     service.obj
 0001:0005e858       $chain$0$PushPanelItem     000000018005f858     service.obj
 0001:0005e86c       $chain$1$PushPanelItem     000000018005f86c     service.obj
 0001:0005e87c       $chain$3$PushPanelItem     000000018005f87c     service.obj
 0001:0005e894       $chain$4$PushPanelItem     000000018005f894     service.obj
 0001:0005e8a4       $unwind$PushPanelItems     000000018005f8a4     service.obj
 0001:0005e8b4       $chain$3$PushPanelItems    000000018005f8b4     service.obj
 0001:0005e8d4       $chain$4$PushPanelItems    000000018005f8d4     service.obj
 0001:0005e8e4       $unwind$editor_GetFileName 000000018005f8e4     service.obj
 0001:0005e8e4       $unwind$far_GetPluginInformation 000000018005f8e4     service.obj
 0001:0005e8e4       $unwind$viewer_GetFileName 000000018005f8e4     service.obj
 0001:0005e8e4       $unwind$far_MkLink         000000018005f8e4     service.obj
 0001:0005e8e4       $unwind$far_GetPathRoot    000000018005f8e4     service.obj
 0001:0005e8e4       $unwind$editor_GetTitle    000000018005f8e4     service.obj
 0001:0005e8e4       $unwind$far_ShowHelp       000000018005f8e4     service.obj
 0001:0005e8e4       $unwind$NewDialogData      000000018005f8e4     service.obj
 0001:0005e8e4       $unwind$panel_GetCmdLine   000000018005f8e4     service.obj
 0001:0005e8f8       $chain$0$GetFarColor       000000018005f8f8     service.obj
 0001:0005e90c       $chain$1$GetFarColor       000000018005f90c     service.obj
 0001:0005e91c       $chain$0$DllMain           000000018005f91c     service.obj
 0001:0005e930       $chain$1$DllMain           000000018005f930     service.obj
 0001:0005e940       $unwind$GetFlagCombination 000000018005f940     service.obj
 0001:0005e958       $unwind$ConvertLuaValue    000000018005f958     service.obj
 0001:0005e958       $unwind$plugin_load        000000018005f958     service.obj
 0001:0005e96c       $unwind$far_GetFileOwner   000000018005f96c     service.obj
 0001:0005e980       $unwind$editor_InsertText  000000018005f980     service.obj
 0001:0005e980       $unwind$panel_GetUserScreen 000000018005f980     service.obj
 0001:0005e980       $unwind$panel_SetCmdLinePos 000000018005f980     service.obj
 0001:0005e980       $unwind$far_LStricmp       000000018005f980     service.obj
 0001:0005e980       $unwind$editor_DeleteSessionBookmark 000000018005f980     service.obj
 0001:0005e980       $unwind$far_PluginStartupInfo 000000018005f980     service.obj
 0001:0005e980       $unwind$editor_SetTitle    000000018005f980     service.obj
 0001:0005e980       $unwind$AddMacroData_gc    000000018005f980     service.obj
 0001:0005e980       $unwind$far_MacroDelete    000000018005f980     service.obj
 0001:0005e980       $unwind$far_MkTemp         000000018005f980     service.obj
 0001:0005e980       $unwind$panel_SetUserScreen 000000018005f980     service.obj
 0001:0005e980       $unwind$utf8_valid         000000018005f980     slnunico.obj
 0001:0005e980       $unwind$panel_ClosePanel   000000018005f980     service.obj
 0001:0005e980       $unwind$ustring_sub        000000018005f980     ustring.obj
 0001:0005e980       $unwind$panel_SetCmdLine   000000018005f980     service.obj
 0001:0005e980       $unwind$panel_SetActivePanel 000000018005f980     service.obj
 0001:0005e980       $unwind$panel_InsertCmdLine 000000018005f980     service.obj
 0001:0005e990       $unwind$Lutf8_len          000000018005f990     lutf8lib.obj
 0001:0005e990       $unwind$far_GetCurrentDirectory 000000018005f990     service.obj
 0001:0005e990       $unwind$far_CreateFileFilter 000000018005f990     service.obj
 0001:0005e990       $unwind$far_LStrnicmp      000000018005f990     service.obj
 0001:0005e9a4       $unwind$editor_GetInfo     000000018005f9a4     service.obj
 0001:0005e9b4       $chain$2$editor_GetInfo    000000018005f9b4     service.obj
 0001:0005e9d0       $chain$3$editor_GetInfo    000000018005f9d0     service.obj
 0001:0005e9e4       $chain$4$editor_GetInfo    000000018005f9e4     service.obj
 0001:0005e9f4       $chain$5$editor_GetInfo    000000018005f9f4     service.obj
 0001:0005ea08       $unwind$_EditorGetString   000000018005fa08     service.obj
 0001:0005ea24       $unwind$_EditorSetString   000000018005fa24     service.obj
 0001:0005ea34       $unwind$far_FindPlugin     000000018005fa34     service.obj
 0001:0005ea34       $unwind$editor_InsertString 000000018005fa34     service.obj
 0001:0005ea34       $unwind$far_LUpperBuf      000000018005fa34     service.obj
 0001:0005ea34       $unwind$far_LLowerBuf      000000018005fa34     service.obj
 0001:0005ea34       $unwind$editor_ExpandTabs  000000018005fa34     service.obj
 0001:0005ea44       $unwind$_EditorInsertText  000000018005fa44     service.obj
 0001:0005ea54       $unwind$FillKeyBarTitles   000000018005fa54     service.obj
 0001:0005ea68       $chain$1$FillKeyBarTitles  000000018005fa68     service.obj
 0001:0005ea80       $chain$2$FillKeyBarTitles  000000018005fa80     service.obj
 0001:0005ea90       $unwind$SetKeyBar          000000018005fa90     service.obj
 0001:0005eaa8       $unwind$editor_SetParam    000000018005faa8     service.obj
 0001:0005eac0       $unwind$editor_SetPosition 000000018005fac0     service.obj
 0001:0005ead0       $unwind$PushBookmarks      000000018005fad0     service.obj
 0001:0005eae4       $chain$0$PushBookmarks     000000018005fae4     service.obj
 0001:0005eaf8       $chain$1$PushBookmarks     000000018005faf8     service.obj
 0001:0005eb08       $unwind$editor_Select      000000018005fb08     service.obj
 0001:0005eb18       $unwind$editor_GetSelection 000000018005fb18     service.obj
 0001:0005eb34       $unwind$_EditorTabConvert  000000018005fb34     service.obj
 0001:0005eb48       $unwind$editor_AddColor    000000018005fb48     service.obj
 0001:0005eb5c       $unwind$editor_DelColor    000000018005fb5c     service.obj
 0001:0005eb70       $unwind$editor_GetColor    000000018005fb70     service.obj
 0001:0005eb80       $unwind$viewer_Select      000000018005fb80     service.obj
 0001:0005eb80       $unwind$panel_SetCmdLineSelection 000000018005fb80     service.obj
 0001:0005eb80       $unwind$editor_SaveFile    000000018005fb80     service.obj
 0001:0005eb80       $unwind$viewer_SetMode     000000018005fb80     service.obj
 0001:0005eb90       $unwind$_mbsdec_l          000000018005fb90     libucrt:mbsdec.obj
 0001:0005eb90       $unwind$win_ExtractKeyEx   000000018005fb90     win.obj
 0001:0005eb90       $unwind$LF_Error           000000018005fb90     service.obj
 0001:0005eb90       $unwind$isdigit            000000018005fb90     libucrt:_ctype.obj
 0001:0005eb90       $unwind$Settings_opensubkey 000000018005fb90     service.obj
 0001:0005eb90       $unwind$editor_ReadInput   000000018005fb90     service.obj
 0001:0005eb90       $unwind$Settings_delete    000000018005fb90     service.obj
 0001:0005eb90       $unwind$far_NameToInputRecord 000000018005fb90     service.obj
 0001:0005eb90       $unwind$isspace            000000018005fb90     libucrt:_ctype.obj
 0001:0005eb90       $unwind$editor_ProcessInput 000000018005fb90     service.obj
 0001:0005eb90       $unwind$_strupr_s_l        000000018005fb90     libucrt:strupr.obj
 0001:0005eb90       $unwind$panel_GetCmdLineSelection 000000018005fb90     service.obj
 0001:0005eb90       $unwind$editor_SubscribeChangeEvent 000000018005fb90     service.obj
 0001:0005eb90       $unwind$win_ExtractKey     000000018005fb90     win.obj
 0001:0005eb9c       $unwind$far_Menu           000000018005fb9c     service.obj
 0001:0005ebb4       $chain$0$far_Menu          000000018005fbb4     service.obj
 0001:0005ebc8       $chain$1$far_Menu          000000018005fbc8     service.obj
 0001:0005ebd8       $unwind$far_Message        000000018005fbd8     service.obj
 0001:0005ebf4       $unwind$panel_GetPanelInfo 000000018005fbf4     service.obj
 0001:0005ec04       $chain$0$panel_GetPanelInfo 000000018005fc04     service.obj
 0001:0005ec18       $chain$1$panel_GetPanelInfo 000000018005fc18     service.obj
 0001:0005ec28       $unwind$get_panel_item     000000018005fc28     service.obj
 0001:0005ec3c       $unwind$get_string_info    000000018005fc3c     service.obj
 0001:0005ec54       $unwind$panel_RedrawPanel  000000018005fc54     service.obj
 0001:0005ec68       $unwind$g_write            000000018005fc68     uliolib51.obj
 0001:0005ec68       $unwind$SetPanelBooleanProperty 000000018005fc68     service.obj
 0001:0005ec68       $unwind$SetPanelIntegerProperty 000000018005fc68     service.obj
 0001:0005ec68       $unwind$truncstring        000000018005fc68     service.obj
 0001:0005ec7c       $unwind$panel_GetPanelDirectory 000000018005fc7c     service.obj
 0001:0005ec90       $unwind$panel_SetPanelDirectory 000000018005fc90     service.obj
 0001:0005eca0       $unwind$ChangePanelSelection 000000018005fca0     service.obj
 0001:0005ecb8       $chain$1$ChangePanelSelection 000000018005fcb8     service.obj
 0001:0005eccc       $chain$2$ChangePanelSelection 000000018005fccc     service.obj
 0001:0005ecdc       $unwind$far_GetDirList     000000018005fcdc     service.obj
 0001:0005ece8       $chain$0$far_GetDirList    000000018005fce8     service.obj
 0001:0005ecfc       $chain$6$far_GetDirList    000000018005fcfc     service.obj
 0001:0005ed24       $chain$7$far_GetDirList    000000018005fd24     service.obj
 0001:0005ed34       $chain$8$far_GetDirList    000000018005fd34     service.obj
 0001:0005ed44       $unwind$matchbalance       000000018005fd44     lutf8lib.obj
 0001:0005ed44       $unwind$far_GetPluginDirList 000000018005fd44     service.obj
 0001:0005ed50       $unwind$far_RestoreScreen  000000018005fd50     service.obj
 0001:0005ed5c       $unwind$far_SaveScreen     000000018005fd5c     service.obj
 0001:0005ed74       $unwind$CreateList         000000018005fd74     service.obj
 0001:0005ed84       $chain$2$CreateList        000000018005fd84     service.obj
 0001:0005eda0       $chain$3$CreateList        000000018005fda0     service.obj
 0001:0005edb0       $unwind$far_ConvertPath    000000018005fdb0     service.obj
 0001:0005edb0       $unwind$SetFarDialogItem   000000018005fdb0     service.obj
 0001:0005edc8       $unwind$PushDlgItem        000000018005fdc8     service.obj
 0001:0005eddc       $chain$1$PushDlgItem       000000018005fddc     service.obj
 0001:0005edf0       $chain$2$PushDlgItem       000000018005fdf0     service.obj
 0001:0005ee00       $unwind$PushDlgItemNum     000000018005fe00     service.obj
 0001:0005ee18       $unwind$SetDlgItem         000000018005fe18     service.obj
 0001:0005ee30       $unwind$far_SendDlgMessage 000000018005fe30     service.obj
 0001:0005ee4c       $unwind$ProcessDNResult    000000018005fe4c     service.obj
 0001:0005ee60       $chain$0$ProcessDNResult   000000018005fe60     service.obj
 0001:0005ee74       $chain$1$ProcessDNResult   000000018005fe74     service.obj
 0001:0005ee84       $unwind$far_DialogInit     000000018005fe84     service.obj
 0001:0005eea0       $unwind$far_SetDlgItem     000000018005fea0     service.obj
 0001:0005eea0       $unwind$far_GetDlgItem     000000018005fea0     service.obj
 0001:0005eea0       $unwind$Lutf8_next         000000018005fea0     lutf8lib.obj
 0001:0005eeb4       $unwind$editor_Editor      000000018005feb4     service.obj
 0001:0005eeb4       $unwind$far_InputBox       000000018005feb4     service.obj
 0001:0005eecc       $unwind$viewer_Viewer      000000018005fecc     service.obj
 0001:0005eee4       $unwind$viewer_GetInfo     000000018005fee4     service.obj
 0001:0005eef0       $chain$1$viewer_GetInfo    000000018005fef0     service.obj
 0001:0005ef08       $chain$2$viewer_GetInfo    000000018005ff08     service.obj
 0001:0005ef1c       $chain$3$viewer_GetInfo    000000018005ff1c     service.obj
 0001:0005ef2c       $chain$4$viewer_GetInfo    000000018005ff2c     service.obj
 0001:0005ef3c       $chain$2$viewer_SetPosition 000000018005ff3c     service.obj
 0001:0005ef58       $chain$3$viewer_SetPosition 000000018005ff58     service.obj
 0001:0005ef68       $unwind$far_Text           000000018005ff68     service.obj
 0001:0005ef7c       $chain$1$far_CopyToClipboard 000000018005ff7c     service.obj
 0001:0005ef94       $chain$2$far_CopyToClipboard 000000018005ff94     service.obj
 0001:0005efa4       $unwind$far_PasteFromClipboard 000000018005ffa4     service.obj
 0001:0005efb8       $unwind$far_InputRecordToName 000000018005ffb8     service.obj
 0001:0005efb8       $unwind$pusherrorcode      000000018005ffb8     ustring.obj
 0001:0005efc8       $unwind$far_ProcessName    000000018005ffc8     service.obj
 0001:0005efe0       $chain$2$far_ProcessName   000000018005ffe0     service.obj
 0001:0005eff4       $chain$3$far_ProcessName   000000018005fff4     service.obj
 0001:0005f008       $chain$4$far_ProcessName   0000000180060008     service.obj
 0001:0005f018       $chain$7$far_ProcessName   0000000180060018     service.obj
 0001:0005f018       $chain$5$far_ProcessName   0000000180060018     service.obj
 0001:0005f028       $chain$6$far_ProcessName   0000000180060028     service.obj
 0001:0005f03c       $unwind$far_GetReparsePointInfo 000000018006003c     service.obj
 0001:0005f04c       $chain$0$far_GetReparsePointInfo 000000018006004c     service.obj
 0001:0005f060       $chain$1$far_GetReparsePointInfo 0000000180060060     service.obj
 0001:0005f070       $unwind$?process_integer_specifier@?$input_processor@DV?$stream_input_adapter@D@__crt_stdio_input@@@__crt_stdio_input@@AEAA_NI_N@Z 0000000180060070     libucrt:input.obj
 0001:0005f070       $unwind$far_RecursiveSearch 0000000180060070     service.obj
 0001:0005f084       $unwind$far_AdvControl     0000000180060084     service.obj
 0001:0005f0a4       $chain$0$far_AdvControl    00000001800600a4     service.obj
 0001:0005f0b8       $chain$1$far_AdvControl    00000001800600b8     service.obj
 0001:0005f0c8       $unwind$capture_current_context 00000001800600c8     LIBCMT:gs_report.obj
 0001:0005f0c8       $unwind$far_MacroLoadAll   00000001800600c8     service.obj
 0001:0005f0d4       $chain$0$far_MacroLoadAll  00000001800600d4     service.obj
 0001:0005f0e8       $chain$1$far_MacroLoadAll  00000001800600e8     service.obj
 0001:0005f0f8       $unwind$MacroSendString    00000001800600f8     service.obj
 0001:0005f10c       $unwind$far_MacroGetLastError 000000018006010c     service.obj
 0001:0005f11c       $chain$0$far_MacroGetLastError 000000018006011c     service.obj
 0001:0005f130       $chain$1$far_MacroGetLastError 0000000180060130     service.obj
 0001:0005f140       $unwind$MacroAddCallback   0000000180060140     service.obj
 0001:0005f154       $unwind$far_MacroAdd       0000000180060154     service.obj
 0001:0005f168       $unwind$far_MacroExecute   0000000180060168     service.obj
 0001:0005f170       $chain$2$far_MacroExecute  0000000180060170     service.obj
 0001:0005f18c       $chain$3$far_MacroExecute  000000018006018c     service.obj
 0001:0005f19c       $unwind$far_MakeMenuItems  000000018006019c     service.obj
 0001:0005f1a8       $chain$1$far_MakeMenuItems 00000001800601a8     service.obj
 0001:0005f1c0       $chain$5$far_MakeMenuItems 00000001800601c0     service.obj
 0001:0005f1e0       $chain$6$far_MakeMenuItems 00000001800601e0     service.obj
 0001:0005f1f0       $chain$8$far_MakeMenuItems 00000001800601f0     service.obj
 0001:0005f208       $chain$9$far_MakeMenuItems 0000000180060208     service.obj
 0001:0005f218       $unwind$?type_case_integer@?$output_processor@_WV?$string_output_adapter@_W@__crt_stdio_output@@V?$standard_base@_WV?$string_output_adapter@_W@__crt_stdio_output@@@2@@__crt_stdio_output@@AEAA_NI_N@Z 0000000180060218     libucrt:output.obj
 0001:0005f218       $unwind$io_open            0000000180060218     uliolib51.obj
 0001:0005f218       $unwind$??$parse_floating_point_possible_nan_is_ind@DV?$input_adapter_character_source@V?$stream_input_adapter@D@__crt_stdio_input@@@__crt_strtox@@@__crt_strtox@@YA_NAEADAEAV?$input_adapter_character_source@V?$stream_input_adapter@D@__crt_stdio_input@@@0@@Z 0000000180060218     libucrt:input.obj
 0001:0005f218       $unwind$??$parse_floating_point_possible_nan_is_snan@DV?$input_adapter_character_source@V?$stream_input_adapter@D@__crt_stdio_input@@@__crt_strtox@@@__crt_strtox@@YA_NAEADAEAV?$input_adapter_character_source@V?$stream_input_adapter@D@__crt_stdio_input@@@0@@Z 0000000180060218     libucrt:input.obj
 0001:0005f218       $unwind$??R<lambda_f03950bc5685219e0bcd2087efbe011e>@@QEBAHXZ 0000000180060218     libucrt:onexit.obj
 0001:0005f218       $unwind$??$parse_floating_point_possible_infinity@DV?$input_adapter_character_source@V?$stream_input_adapter@D@__crt_stdio_input@@@__crt_strtox@@_K@__crt_strtox@@YA?AW4floating_point_parse_result@0@AEADAEAV?$input_adapter_character_source@V?$stream_input_adapter@D@__crt_stdio_input@@@0@_K@Z 0000000180060218     libucrt:input.obj
 0001:0005f218       $unwind$NewVirtualKeyTable 0000000180060218     service.obj
 0001:0005f218       $unwind$?type_case_integer@?$output_processor@DV?$stream_output_adapter@D@__crt_stdio_output@@V?$standard_base@DV?$stream_output_adapter@D@__crt_stdio_output@@@2@@__crt_stdio_output@@AEAA_NI_N@Z 0000000180060218     libucrt:output.obj
 0001:0005f218       $unwind$?type_case_integer@?$output_processor@DV?$string_output_adapter@D@__crt_stdio_output@@V?$standard_base@DV?$string_output_adapter@D@__crt_stdio_output@@@2@@__crt_stdio_output@@AEAA_NI_N@Z 0000000180060218     libucrt:output.obj
 0001:0005f230       $unwind$filefilter_IsFileInFilter 0000000180060230     service.obj
 0001:0005f244       $chain$0$PutPluginMenuItemToTable 0000000180060244     service.obj
 0001:0005f258       $chain$1$PutPluginMenuItemToTable 0000000180060258     service.obj
 0001:0005f268       $chain$1$far_GetPlugins    0000000180060268     service.obj
 0001:0005f280       $chain$2$far_GetPlugins    0000000180060280     service.obj
 0001:0005f294       $chain$3$far_GetPlugins    0000000180060294     service.obj
 0001:0005f2a4       $chain$4$far_GetPlugins    00000001800602a4     service.obj
 0001:0005f2b4       $unwind$far_IsPluginLoaded 00000001800602b4     service.obj
 0001:0005f2c4       $chain$0$far_IsPluginLoaded 00000001800602c4     service.obj
 0001:0005f2d8       $chain$1$far_IsPluginLoaded 00000001800602d8     service.obj
 0001:0005f2e8       $unwind$far_XLat           00000001800602e8     service.obj
 0001:0005f2e8       $unwind$Lutf8_byte         00000001800602e8     lutf8lib.obj
 0001:0005f2fc       $unwind$far_FormatFileSize 00000001800602fc     service.obj
 0001:0005f314       $unwind$far_Timer          0000000180060314     service.obj
 0001:0005f32c       $unwind$timer_gc           000000018006032c     service.obj
 0001:0005f32c       $unwind$iswctype           000000018006032c     libucrt:iswctype.obj
 0001:0005f32c       $unwind$timer_Close        000000018006032c     service.obj
 0001:0005f338       $chain$0$timer_Close       0000000180060338     service.obj
 0001:0005f34c       $chain$1$timer_Close       000000018006034c     service.obj
 0001:0005f35c       $chain$0$timer_gc          000000018006035c     service.obj
 0001:0005f370       $chain$1$timer_gc          0000000180060370     service.obj
 0001:0005f380       $unwind$far_CreateSettings 0000000180060380     service.obj
 0001:0005f390       $unwind$Settings_set       0000000180060390     service.obj
 0001:0005f390       $unwind$Settings_get       0000000180060390     service.obj
 0001:0005f39c       $unwind$Settings_createsubkey 000000018006039c     service.obj
 0001:0005f3b0       $unwind$Settings_enum      00000001800603b0     service.obj
 0001:0005f3c0       $chain$2$Settings_enum     00000001800603c0     service.obj
 0001:0005f3dc       $chain$4$Settings_enum     00000001800603dc     service.obj
 0001:0005f3f0       $chain$5$Settings_enum     00000001800603f0     service.obj
 0001:0005f400       $unwind$far_ColorDialog    0000000180060400     service.obj
 0001:0005f410       $unwind$_snwprintf         0000000180060410     slnunico.obj
 0001:0005f420       $unwind$Lutf8_reverse      0000000180060420     lutf8lib.obj
 0001:0005f420       $unwind$str_rep            0000000180060420     slnunico.obj
 0001:0005f434       $unwind$str_dump           0000000180060434     slnunico.obj
 0001:0005f440       $unwind$str_format         0000000180060440     slnunico.obj
 0001:0005f45c       $unwind$??$type_case_integer_parse_into_buffer@I@?$output_processor@DV?$stream_output_adapter@D@__crt_stdio_output@@V?$standard_base@DV?$stream_output_adapter@D@__crt_stdio_output@@@2@@__crt_stdio_output@@AEAAXII_N@Z 000000018006045c     libucrt:output.obj
 0001:0005f45c       $unwind$??$type_case_integer_parse_into_buffer@_K@?$output_processor@DV?$string_output_adapter@D@__crt_stdio_output@@V?$standard_base@DV?$string_output_adapter@D@__crt_stdio_output@@@2@@__crt_stdio_output@@AEAAX_KI_N@Z 000000018006045c     libucrt:output.obj
 0001:0005f45c       $unwind$??$type_case_integer_parse_into_buffer@I@?$output_processor@DV?$string_output_adapter@D@__crt_stdio_output@@V?$standard_base@DV?$string_output_adapter@D@__crt_stdio_output@@@2@@__crt_stdio_output@@AEAAXII_N@Z 000000018006045c     libucrt:output.obj
 0001:0005f45c       $unwind$??$type_case_integer_parse_into_buffer@I@?$output_processor@_WV?$string_output_adapter@_W@__crt_stdio_output@@V?$standard_base@_WV?$string_output_adapter@_W@__crt_stdio_output@@@2@@__crt_stdio_output@@AEAAXII_N@Z 000000018006045c     libucrt:output.obj
 0001:0005f45c       $unwind$utf8_isgraph       000000018006045c     lutf8lib.obj
 0001:0005f45c       $unwind$utf8_isdigit       000000018006045c     lutf8lib.obj
 0001:0005f45c       $unwind$utf8_islower       000000018006045c     lutf8lib.obj
 0001:0005f45c       $unwind$??$type_case_integer_parse_into_buffer@_K@?$output_processor@DV?$stream_output_adapter@D@__crt_stdio_output@@V?$standard_base@DV?$stream_output_adapter@D@__crt_stdio_output@@@2@@__crt_stdio_output@@AEAAX_KI_N@Z 000000018006045c     libucrt:output.obj
 0001:0005f45c       $unwind$??$type_case_integer_parse_into_buffer@_K@?$output_processor@_WV?$string_output_adapter@_W@__crt_stdio_output@@V?$standard_base@_WV?$string_output_adapter@_W@__crt_stdio_output@@@2@@__crt_stdio_output@@AEAAX_KI_N@Z 000000018006045c     libucrt:output.obj
 0001:0005f464       $unwind$utf8_width         0000000180060464     lutf8lib.obj
 0001:0005f470       $unwind$Lutf8_sub          0000000180060470     lutf8lib.obj
 0001:0005f484       $unwind$convert            0000000180060484     lutf8lib.obj
 0001:0005f498       $unwind$Lutf8_codepoint    0000000180060498     lutf8lib.obj
 0001:0005f4b0       $unwind$Lutf8_char         00000001800604b0     lutf8lib.obj
 0001:0005f4c0       $chain$0$Lutf8_char        00000001800604c0     lutf8lib.obj
 0001:0005f4d4       $chain$1$Lutf8_char        00000001800604d4     lutf8lib.obj
 0001:0005f4e4       $unwind$Lutf8_escape       00000001800604e4     lutf8lib.obj
 0001:0005f4f4       $chain$3$Lutf8_escape      00000001800604f4     lutf8lib.obj
 0001:0005f514       $chain$4$Lutf8_escape      0000000180060514     lutf8lib.obj
 0001:0005f524       $unwind$Lutf8_insert       0000000180060524     lutf8lib.obj
 0001:0005f53c       $unwind$Lutf8_remove       000000018006053c     lutf8lib.obj
 0001:0005f554       $unwind$Lutf8_charpos      0000000180060554     lutf8lib.obj
 0001:0005f568       $unwind$Lutf8_width        0000000180060568     lutf8lib.obj
 0001:0005f578       $chain$0$Lutf8_width       0000000180060578     lutf8lib.obj
 0001:0005f58c       $chain$1$Lutf8_width       000000018006058c     lutf8lib.obj
 0001:0005f59c       $unwind$Lutf8_widthindex   000000018006059c     lutf8lib.obj
 0001:0005f59c       $unwind$matchbracketclass  000000018006059c     lutf8lib.obj
 0001:0005f5b4       $unwind$win_SetRegKey      00000001800605b4     win.obj
 0001:0005f5b4       $unwind$win_CompareString  00000001800605b4     win.obj
 0001:0005f5b4       $unwind$Lutf8_ncasecmp     00000001800605b4     lutf8lib.obj
 0001:0005f5cc       $unwind$match              00000001800605cc     lutf8lib.obj
 0001:0005f5dc       $chain$3$match             00000001800605dc     lutf8lib.obj
 0001:0005f5fc       $chain$4$match             00000001800605fc     lutf8lib.obj
 0001:0005f60c       $unwind$singlematch        000000018006060c     lutf8lib.obj
 0001:0005f61c       $chain$1$matchbalance      000000018006061c     lutf8lib.obj
 0001:0005f634       $chain$2$matchbalance      0000000180060634     lutf8lib.obj
 0001:0005f648       $unwind$push_onecapture    0000000180060648     lutf8lib.obj
 0001:0005f650       $chain$3$push_onecapture   0000000180060650     lutf8lib.obj
 0001:0005f670       $chain$5$push_onecapture   0000000180060670     lutf8lib.obj
 0001:0005f688       $unwind$push_captures      0000000180060688     lutf8lib.obj
 0001:0005f698       $chain$2$push_captures     0000000180060698     lutf8lib.obj
 0001:0005f6b4       $chain$3$push_captures     00000001800606b4     lutf8lib.obj
 0001:0005f6c4       $unwind$find_aux           00000001800606c4     lutf8lib.obj
 0001:0005f6e0       $unwind$gmatch_aux         00000001800606e0     lutf8lib.obj
 0001:0005f6f8       $unwind$add_value          00000001800606f8     lutf8lib.obj
 0001:0005f708       $chain$1$add_value         0000000180060708     lutf8lib.obj
 0001:0005f720       $chain$2$add_value         0000000180060720     lutf8lib.obj
 0001:0005f734       $chain$3$add_value         0000000180060734     lutf8lib.obj
 0001:0005f744       $chain$4$add_value         0000000180060744     lutf8lib.obj
 0001:0005f754       $unwind$Lutf8_gsub         0000000180060754     lutf8lib.obj
 0001:0005f76c       $unwind$luaopen_utf8       000000018006076c     lutf8lib.obj
 0001:0005f77c       $unwind$g_iofile           000000018006077c     uliolib51.obj
 0001:0005f78c       $chain$0$g_iofile          000000018006078c     uliolib51.obj
 0001:0005f7a0       $chain$1$g_iofile          00000001800607a0     uliolib51.obj
 0001:0005f7b4       $chain$2$g_iofile          00000001800607b4     uliolib51.obj
 0001:0005f7c4       $chain$3$g_iofile          00000001800607c4     uliolib51.obj
 0001:0005f7d4       $chain$1$io_lines          00000001800607d4     uliolib51.obj
 0001:0005f7ec       $chain$2$io_lines          00000001800607ec     uliolib51.obj
 0001:0005f800       $unwind$read_line          0000000180060800     uliolib51.obj
 0001:0005f814       $unwind$read_chars         0000000180060814     uliolib51.obj
 0001:0005f82c       $unwind$g_read             000000018006082c     uliolib51.obj
 0001:0005f844       $unwind$??$initialize_environment_by_cloning_nolock@_W@@YAHXZ 0000000180060844     libucrt:environment_initialization.obj
 0001:0005f844       $unwind$GetIntFromArray    0000000180060844     util.obj
 0001:0005f844       $unwind$strpbrk            0000000180060844     libucrt:strpbrk.obj
 0001:0005f844       $unwind$PutWStrToArray     0000000180060844     ustring.obj
 0001:0005f844       $unwind$_strdup            0000000180060844     libucrt:strdup.obj
 0001:0005f844       $unwind$loaderror          0000000180060844     uloadlib51.obj
 0001:0005f844       $unwind$??$generate_tmpfile_file_name@D@@YA_NQEAD_K@Z 0000000180060844     libucrt:tmpfile.obj
 0001:0005f854       $unwind$loader_Croot       0000000180060854     uloadlib51.obj
 0001:0005f864       $unwind$ll_module          0000000180060864     uloadlib51.obj
 0001:0005f878       $chain$0$ll_module         0000000180060878     uloadlib51.obj
 0001:0005f88c       $chain$1$ll_module         000000018006088c     uloadlib51.obj
 0001:0005f89c       $unwind$setpath            000000018006089c     uloadlib51.obj
 0001:0005f8b0       $unwind$luaopen_upackage   00000001800608b0     uloadlib51.obj
 0001:0005f8b0       $unwind$__acrt_stdio_refill_and_read_narrow_nolock 00000001800608b0     libucrt:_filbuf.obj
 0001:0005f8b0       $unwind$_free_osfhnd       00000001800608b0     libucrt:osfinfo.obj
 0001:0005f8c4       $unwind$GetOptNumFromTable 00000001800608c4     ustring.obj
 0001:0005f8d0       $unwind$win_FileTimeToSystemTime 00000001800608d0     win.obj
 0001:0005f8d0       $unwind$?convert_hexadecimal_string_to_floating_type_common@__crt_strtox@@YA?AW4SLD_STATUS@@AEBUfloating_point_string@1@AEBVfloating_point_value@1@@Z 00000001800608d0     libucrt:input.obj
 0001:0005f8d0       $unwind$strerror           00000001800608d0     libucrt:strerror.obj
 0001:0005f8d0       $unwind$PutWStrToTable     00000001800608d0     ustring.obj
 0001:0005f8d0       $unwind$EnumCodePagesProc  00000001800608d0     ustring.obj
 0001:0005f8dc       $unwind$opt_utf8_string    00000001800608dc     ustring.obj
 0001:0005f8f4       $unwind$PushAttrString     00000001800608f4     ustring.obj
 0001:0005f8f4       $unwind$_raise_exc         00000001800608f4     libucrt:fpexcept.obj
 0001:0005f8fc       $unwind$convert_multibyte_string 00000001800608fc     ustring.obj
 0001:0005f918       $unwind$push_multibyte_string 0000000180060918     ustring.obj
 0001:0005f92c       $chain$2$push_multibyte_string 000000018006092c     ustring.obj
 0001:0005f944       $chain$3$push_multibyte_string 0000000180060944     ustring.obj
 0001:0005f958       $unwind$ustring_WideCharToMultiByte 0000000180060958     ustring.obj
 0001:0005f96c       $chain$1$ustring_WideCharToMultiByte 000000018006096c     ustring.obj
 0001:0005f984       $chain$2$ustring_WideCharToMultiByte 0000000180060984     ustring.obj
 0001:0005f994       $unwind$ustring_MultiByteToWideChar 0000000180060994     ustring.obj
 0001:0005f9b0       $unwind$ustring_OemToUtf8  00000001800609b0     ustring.obj
 0001:0005f9bc       $chain$1$ustring_OemToUtf8 00000001800609bc     ustring.obj
 0001:0005f9d4       $chain$2$ustring_OemToUtf8 00000001800609d4     ustring.obj
 0001:0005f9e4       $unwind$win_DeleteRegValue 00000001800609e4     win.obj
 0001:0005f9e4       $unwind$ustring_Utf8ToOem  00000001800609e4     ustring.obj
 0001:0005f9e4       $unwind$?decode_options@@YA?AUfile_options@?A0xa9d50aae@@HHH@Z 00000001800609e4     libucrt:open.obj
 0001:0005f9f8       $unwind$??$common_xtox_s@_KD@@YAH_KQEAD0I_N@Z 00000001800609f8     libucrt:xtoa.obj
 0001:0005f9f8       $unwind$win_SystemTimeToFileTime 00000001800609f8     win.obj
 0001:0005f9f8       $unwind$ustring_Utf16ToUtf8 00000001800609f8     ustring.obj
 0001:0005f9f8       $unwind$?__mbrtowc_utf8@__crt_mbstring@@YA_KPEA_WPEBD_KPEAU_Mbstatet@@@Z 00000001800609f8     libucrt:mbrtowc.obj
 0001:0005f9f8       $unwind$ustring_Uuid       00000001800609f8     ustring.obj
 0001:0005fa00       $unwind$ustring_Utf8ToUtf16 0000000180060a00     ustring.obj
 0001:0005fa10       $chain$0$ustring_Utf8ToUtf16 0000000180060a10     ustring.obj
 0001:0005fa24       $chain$1$ustring_Utf8ToUtf16 0000000180060a24     ustring.obj
 0001:0005fa34       $unwind$ustring_SetConsoleOutputCP 0000000180060a34     ustring.obj
 0001:0005fa34       $unwind$ustring_SetConsoleCP 0000000180060a34     ustring.obj
 0001:0005fa40       $unwind$ustring_GetCPInfo  0000000180060a40     ustring.obj
 0001:0005fa58       $unwind$ustring_GetLogicalDriveStrings 0000000180060a58     ustring.obj
 0001:0005fa68       $chain$0$ustring_GetLogicalDriveStrings 0000000180060a68     ustring.obj
 0001:0005fa7c       $chain$1$ustring_GetLogicalDriveStrings 0000000180060a7c     ustring.obj
 0001:0005fa8c       $unwind$ustring_SearchPath 0000000180060a8c     ustring.obj
 0001:0005faa4       $unwind$ustring_GlobalMemoryStatus 0000000180060aa4     ustring.obj
 0001:0005faac       $chain$0$ustring_GlobalMemoryStatus 0000000180060aac     ustring.obj
 0001:0005fac0       $chain$2$ustring_GlobalMemoryStatus 0000000180060ac0     ustring.obj
 0001:0005fad4       $unwind$ustring_SetFileAttr 0000000180060ad4     ustring.obj
 0001:0005fae0       $chain$2$ustring_SetFileAttr 0000000180060ae0     ustring.obj
 0001:0005fafc       $chain$3$ustring_SetFileAttr 0000000180060afc     ustring.obj
 0001:0005fb10       $chain$4$ustring_SetFileAttr 0000000180060b10     ustring.obj
 0001:0005fb20       $chain$5$ustring_SetFileAttr 0000000180060b20     ustring.obj
 0001:0005fb30       $unwind$ustring_GetFileAttr 0000000180060b30     ustring.obj
 0001:0005fb30       $unwind$ustring_SetCurrentDir 0000000180060b30     ustring.obj
 0001:0005fb3c       $chain$2$ustring_GetFileAttr 0000000180060b3c     ustring.obj
 0001:0005fb58       $chain$3$ustring_GetFileAttr 0000000180060b58     ustring.obj
 0001:0005fb68       $unwind$ustring_SHGetFolderPath 0000000180060b68     ustring.obj
 0001:0005fb78       $chain$1$ustring_SHGetFolderPath 0000000180060b78     ustring.obj
 0001:0005fb90       $chain$2$ustring_SHGetFolderPath 0000000180060b90     ustring.obj
 0001:0005fba0       $unwind$ustring_OutputDebugString 0000000180060ba0     ustring.obj
 0001:0005fbb4       $chain$0$ustring_OutputDebugString 0000000180060bb4     ustring.obj
 0001:0005fbc8       $chain$1$ustring_OutputDebugString 0000000180060bc8     ustring.obj
 0001:0005fbd8       $unwind$ustring_GetCurrentDir 0000000180060bd8     ustring.obj
 0001:0005fbec       $chain$0$ustring_GetCurrentDir 0000000180060bec     ustring.obj
 0001:0005fc00       $chain$1$ustring_GetCurrentDir 0000000180060c00     ustring.obj
 0001:0005fc14       $chain$2$ustring_GetCurrentDir 0000000180060c14     ustring.obj
 0001:0005fc24       $chain$3$ustring_GetCurrentDir 0000000180060c24     ustring.obj
 0001:0005fc34       $chain$2$ustring_SetCurrentDir 0000000180060c34     ustring.obj
 0001:0005fc50       $chain$3$ustring_SetCurrentDir 0000000180060c50     ustring.obj
 0001:0005fc60       $unwind$__acrt_lowio_destroy_handle_array 0000000180060c60     libucrt:osfinfo.obj
 0001:0005fc60       $unwind$PutFileTimeToTable 0000000180060c60     util.obj
 0001:0005fc70       $unwind$win_GetEnv         0000000180060c70     win.obj
 0001:0005fc84       $chain$0$win_GetEnv        0000000180060c84     win.obj
 0001:0005fc98       $chain$1$win_GetEnv        0000000180060c98     win.obj
 0001:0005fca8       $unwind$win_GetRegKey      0000000180060ca8     win.obj
 0001:0005fcbc       $unwind$win_EnumRegValue   0000000180060cbc     win.obj
 0001:0005fcbc       $unwind$win_EnumRegKey     0000000180060cbc     win.obj
 0001:0005fcd0       $unwind$win_GetFileInfo    0000000180060cd0     win.obj
 0001:0005fce0       $unwind$mkdir              0000000180060ce0     win.obj
 0001:0005fcf8       $chain$0$mkdir             0000000180060cf8     win.obj
 0001:0005fd0c       $unwind$??$create_environment@_W@@YAQEAPEA_WQEA_W@Z 0000000180060d0c     libucrt:environment_initialization.obj
 0001:0005fd0c       $unwind$??$create_environment@D@@YAQEAPEADQEAD@Z 0000000180060d0c     libucrt:environment_initialization.obj
 0001:0005fd0c       $unwind$win_ShellExecute   0000000180060d0c     win.obj
 0001:0005fd24       $unwind$win_WriteConsole   0000000180060d24     win.obj
 0001:0005fd38       $unwind$win_IsWinVersion   0000000180060d38     win.obj
 0001:0005fd50       $chain$1$win_IsWinVersion  0000000180060d50     win.obj
 0001:0005fd68       $chain$2$win_IsWinVersion  0000000180060d68     win.obj
 0001:0005fd78       $unwind$?dllmain_crt_process_attach@@YAHQEAUHINSTANCE__@@QEAX@Z 0000000180060d78     LIBCMT:dll_dllmain.obj
 0001:0005fdb4       $unwind$?fin$0@?0???$common_fdopen@_W@@YAPEAU_iobuf@@HQEB_W@Z@4HA 0000000180060db4     libucrt:fdopen.obj
 0001:0005fdb4       $unwind$fgetc$fin$0        0000000180060db4     libucrt:fgetc.obj
 0001:0005fdb4       $unwind$?fin$0@?0???$?RV<lambda_c376a267cfb53b6959b3b692ec76b120>@@AEAV<lambda_9a32fed5bf61b6b509b2d3f6003082a1>@@V<lambda_572fbb9fa0ab338edf41edfd4b5fcc8d>@@@?$__crt_seh_guarded_call@H@@QEAAH$$QEAV<lambda_c376a267cfb53b6959b3b692ec76b120>@@AEAV<lambda_9a32fed5bf61b6b509b2d3f6003082a1>@@$$QEAV<lambda_572fbb9fa0ab338edf41edfd4b5fcc8d>@@@Z@4HA 0000000180060db4     libucrt:fflush.obj
 0001:0005fdb4       $unwind$?fin$0@?0???$?RV<lambda_a37b2b86f63e897a80ea819b0eb08c01>@@AEAV<lambda_38ce7e780aa69e748d6df282ebc68efe>@@V<lambda_99fb1378e971ab6e7edea83e3a7a83a2>@@@?$__crt_seh_guarded_call@H@@QEAAH$$QEAV<lambda_a37b2b86f63e897a80ea819b0eb08c01>@@AEAV<lambda_38ce7e780aa69e748d6df282ebc68efe>@@$$QEAV<lambda_99fb1378e971ab6e7edea83e3a7a83a2>@@@Z@4HA 0000000180060db4     libucrt:commit.obj
 0001:0005fdb4       $unwind$?fin$0@?0???$?RV<lambda_a62c933ada0517137acf5807a1eeac1f>@@AEAV<lambda_a31071773b9a94e445cbd5d04ef99106>@@V<lambda_56065050dbf3ada7e59a83db45153de3>@@@?$__crt_seh_guarded_call@H@@QEAAH$$QEAV<lambda_a62c933ada0517137acf5807a1eeac1f>@@AEAV<lambda_a31071773b9a94e445cbd5d04ef99106>@@$$QEAV<lambda_56065050dbf3ada7e59a83db45153de3>@@@Z@4HA 0000000180060db4     libucrt:output.obj
 0001:0005fdb4       $unwind$?fin$0@?0???$?RV<lambda_7777bce6b2f8c936911f934f8298dc43>@@AEAV<lambda_f03950bc5685219e0bcd2087efbe011e>@@V<lambda_3883c3dff614d5e0c5f61bb1ac94921c>@@@?$__crt_seh_guarded_call@H@@QEAAH$$QEAV<lambda_7777bce6b2f8c936911f934f8298dc43>@@AEAV<lambda_f03950bc5685219e0bcd2087efbe011e>@@$$QEAV<lambda_3883c3dff614d5e0c5f61bb1ac94921c>@@@Z@4HA 0000000180060db4     libucrt:onexit.obj
 0001:0005fdb4       $unwind$_write$fin$0       0000000180060db4     libucrt:write.obj
 0001:0005fdb4       $unwind$?fin$0@?0???$common_getenv@_W@@YAPEA_WQEB_W@Z@4HA 0000000180060db4     libucrt:getenv.obj
 0001:0005fdb4       $unwind$?fin$0@?0??common_tmpfile@@YAHQEAPEAU_iobuf@@H@Z@4HA 0000000180060db4     libucrt:tmpfile.obj
 0001:0005fdb4       $unwind$_query_new_handler$fin$0 0000000180060db4     libucrt:new_handler.obj
 0001:0005fdb4       $unwind$?fin$0@?0???$common_fsopen@_W@@YAPEAU_iobuf@@QEB_W0H@Z@4HA 0000000180060db4     libucrt:fopen.obj
 0001:0005fdb4       $unwind$?fin$0@?0???$?RV<lambda_d80eeec6fff315bfe5c115232f3240e3>@@AEAV<lambda_6e4b09c48022b2350581041d5f6b0c4c>@@V<lambda_2358e3775559c9db80273638284d5e45>@@@?$__crt_seh_guarded_call@X@@QEAAX$$QEAV<lambda_d80eeec6fff315bfe5c115232f3240e3>@@AEAV<lambda_6e4b09c48022b2350581041d5f6b0c4c>@@$$QEAV<lambda_2358e3775559c9db80273638284d5e45>@@@Z@4HA 0000000180060db4     libucrt:exit.obj
 0001:0005fdb4       $unwind$__acrt_update_thread_locale_data$fin$0 0000000180060db4     libucrt:locale_refcounting.obj
 0001:0005fdb4       $unwind$?fin$0@?0???$common_lseek@_J@@YA_JH_JH@Z@4HA 0000000180060db4     libucrt:lseek.obj
 0001:0005fdb4       $unwind$_alloc_osfhnd$fin$0 0000000180060db4     libucrt:osfinfo.obj
 0001:0005fdb4       $unwind$?fin$0@?0???$?RV<lambda_0ae27a3a962d80f24befdcbee591983d>@@AEAV<lambda_8d0ee55de4b1038c4002e0adecdf1839>@@V<lambda_dc504788e8f1664fe9b84e20bfb512f2>@@@?$__crt_seh_guarded_call@X@@QEAAX$$QEAV<lambda_0ae27a3a962d80f24befdcbee591983d>@@AEAV<lambda_8d0ee55de4b1038c4002e0adecdf1839>@@$$QEAV<lambda_dc504788e8f1664fe9b84e20bfb512f2>@@@Z@4HA 0000000180060db4     libucrt:per_thread_data.obj
 0001:0005fdb4       $unwind$rewind$fin$0       0000000180060db4     libucrt:rewind.obj
 0001:0005fdb4       $unwind$_read$fin$0        0000000180060db4     libucrt:read.obj
 0001:0005fdb4       $unwind$?fin$0@?0???$?RV<lambda_a22f0c497e5168315e06dae667770027>@@AEAV<lambda_a094494068278ba5130ab06e1292f60a>@@V<lambda_24dc10c13f43218c635520766e23e324>@@@?$__crt_seh_guarded_call@_N@@QEAA_N$$QEAV<lambda_a22f0c497e5168315e06dae667770027>@@AEAV<lambda_a094494068278ba5130ab06e1292f60a>@@$$QEAV<lambda_24dc10c13f43218c635520766e23e324>@@@Z@4HA 0000000180060db4     libucrt:spawnv.obj
 0001:0005fdb4       $unwind$?fin$0@?0???$?RV<lambda_efdfa57d1f175319df784efa44bb7b81>@@AEAV<lambda_5f0a4c1567f8adc6734073e5d1e1b35c>@@V<lambda_2e8a7d3640ea6ccb4c2413664c2db6fd>@@@?$__crt_seh_guarded_call@X@@QEAAX$$QEAV<lambda_efdfa57d1f175319df784efa44bb7b81>@@AEAV<lambda_5f0a4c1567f8adc6734073e5d1e1b35c>@@$$QEAV<lambda_2e8a7d3640ea6ccb4c2413664c2db6fd>@@@Z@4HA 0000000180060db4     libucrt:mbctype.obj
 0001:0005fdb4       $unwind$_fcloseall$fin$0   0000000180060db4     libucrt:closeall.obj
 0001:0005fdb4       $unwind$__DestructExceptionObject$filt$0 0000000180060db4     libvcruntime:ehhelpers.obj
 0001:0005fdb4       $unwind$ungetc$fin$0       0000000180060db4     libucrt:ungetc.obj
 0001:0005fdb4       $unwind$common_control87$filt$0 0000000180060db4     libucrt:ieee.obj
 0001:0005fdb4       $unwind$?fin$0@?0???$?RV<lambda_751a882b2c74d4b022dec766aa51a29a>@@AEAV<lambda_628dfdc04ba53c8bfc02c9951375f3f5>@@V<lambda_f6c7be5f7998530c34de24c7437d6b54>@@@?$__crt_seh_guarded_call@H@@QEAAH$$QEAV<lambda_751a882b2c74d4b022dec766aa51a29a>@@AEAV<lambda_628dfdc04ba53c8bfc02c9951375f3f5>@@$$QEAV<lambda_f6c7be5f7998530c34de24c7437d6b54>@@@Z@4HA 0000000180060db4     libucrt:close.obj
 0001:0005fdb4       $unwind$?fin$0@?0???$?RV<lambda_082dd7c0feb7dbdaf245f261e54a6583>@@AEAV<lambda_f3caf1ecae5fe01a9a1a6239afa44510>@@V<lambda_c640b76c0755ae85b317b35c67c61e6b>@@@?$__crt_seh_guarded_call@H@@QEAAH$$QEAV<lambda_082dd7c0feb7dbdaf245f261e54a6583>@@AEAV<lambda_f3caf1ecae5fe01a9a1a6239afa44510>@@$$QEAV<lambda_c640b76c0755ae85b317b35c67c61e6b>@@@Z@4HA 0000000180060db4     libucrt:input.obj
 0001:0005fdb4       $unwind$raise$fin$0        0000000180060db4     libucrt:signal.obj
 0001:0005fdb4       $unwind$?fin$0@?0??__acrt_stdio_allocate_stream@@YA?AV__crt_stdio_stream@@XZ@4HA 0000000180060db4     libucrt:stream.obj
 0001:0005fdb4       $unwind$?fin$0@?0???$?RV<lambda_84ec643ea9557e2f7dc01bb0e9624395>@@AEAV<lambda_ca71763b3c0644891230e4f79ea54fa6>@@V<lambda_439a761618c59b0600e24586724d733b>@@@?$__crt_seh_guarded_call@H@@QEAAH$$QEAV<lambda_84ec643ea9557e2f7dc01bb0e9624395>@@AEAV<lambda_ca71763b3c0644891230e4f79ea54fa6>@@$$QEAV<lambda_439a761618c59b0600e24586724d733b>@@@Z@4HA 0000000180060db4     libucrt:setvbuf.obj
 0001:0005fdb4       $unwind$_ctrlfp$filt$0     0000000180060db4     libucrt:fpctrl.obj
 0001:0005fdb4       $unwind$?fin$0@?0??update_thread_multibyte_data_internal@@YAPEAU__crt_multibyte_data@@QEAU__acrt_ptd@@QEAPEAU1@@Z@4HA 0000000180060db4     libucrt:mbctype.obj
 0001:0005fdb4       $unwind$_IsNonwritableInCurrentImage$filt$0 0000000180060db4     LIBCMT:pesect.obj
 0001:0005fdb4       $unwind$?fin$0@?0???$?RV<lambda_450d765d439847d4c735a33c368b5fc0>@@AEAV<lambda_44731a7d0e6d81c3e6aa82d741081786>@@V<lambda_601a2a7da3b7a96e9554ac7215c4b07c>@@@?$__crt_seh_guarded_call@P6AXH@Z@@QEAAP6AXH@Z$$QEAV<lambda_450d765d439847d4c735a33c368b5fc0>@@AEAV<lambda_44731a7d0e6d81c3e6aa82d741081786>@@$$QEAV<lambda_601a2a7da3b7a96e9554ac7215c4b07c>@@@Z@4HA 0000000180060db4     libucrt:signal.obj
 0001:0005fdb4       $unwind$?fin$0@?0??common_fseek@@YAHV__crt_stdio_stream@@_JH@Z@4HA 0000000180060db4     libucrt:fseek.obj
 0001:0005fdb4       $unwind$?fin$0@?0???$common_lseek@J@@YAJHJH@Z@4HA 0000000180060db4     libucrt:lseek.obj
 0001:0005fdb4       $unwind$__acrt_initialize_lowio$fin$0 0000000180060db4     libucrt:ioinit.obj
 0001:0005fdb4       $unwind$?fin$0@?0???$?RV<lambda_410d79af7f07d98d83a3f525b3859a53>@@AEAV<lambda_3e16ef9562a7dcce91392c22ab16ea36>@@V<lambda_38119f0e861e05405d8a144b9b982f0a>@@@?$__crt_seh_guarded_call@X@@QEAAX$$QEAV<lambda_410d79af7f07d98d83a3f525b3859a53>@@AEAV<lambda_3e16ef9562a7dcce91392c22ab16ea36>@@$$QEAV<lambda_38119f0e861e05405d8a144b9b982f0a>@@@Z@4HA 0000000180060db4     libucrt:wsetlocale.obj
 0001:0005fdb4       $unwind$?filt$0@?0???R<lambda_6e4b09c48022b2350581041d5f6b0c4c>@@QEBA@XZ@4HA 0000000180060db4     libucrt:exit.obj
 0001:0005fdb4       $unwind$?fin$0@?0???$?RV<lambda_886d6c58226a84441f68b9f2b8217b83>@@AEAV<lambda_ab61a845afdef5b7c387490eaf3616ee>@@V<lambda_f7f22ab5edc0698d5f6905b0d3f44752>@@@?$__crt_seh_guarded_call@X@@QEAAX$$QEAV<lambda_886d6c58226a84441f68b9f2b8217b83>@@AEAV<lambda_ab61a845afdef5b7c387490eaf3616ee>@@$$QEAV<lambda_f7f22ab5edc0698d5f6905b0d3f44752>@@@Z@4HA 0000000180060db4     libucrt:fflush.obj
 0001:0005fdb4       $unwind$?fin$0@?0??dllmain_crt_process_attach@@YAHQEAUHINSTANCE__@@QEAX@Z@4HA 0000000180060db4     LIBCMT:dll_dllmain.obj
 0001:0005fdb4       $unwind$?fin$0@?0???$?RV<lambda_bdbcead8b570fa3d5ec6d9679862a6e5>@@AEAV<lambda_96f4279ff90247a4c5c5d9824f56f8c1>@@V<lambda_4606be27f17b5e5579e09050fab91818>@@@?$__crt_seh_guarded_call@_K@@QEAA_K$$QEAV<lambda_bdbcead8b570fa3d5ec6d9679862a6e5>@@AEAV<lambda_96f4279ff90247a4c5c5d9824f56f8c1>@@$$QEAV<lambda_4606be27f17b5e5579e09050fab91818>@@@Z@4HA 0000000180060db4     libucrt:fwrite.obj
 0001:0005fdb4       $unwind$?fin$0@?0???$?RV<lambda_842d9ff0dc9ef11c61343bbaebe7f885>@@AEAV<lambda_c5860995281e5c4ce005b3de8f5874ee>@@V<lambda_d90129c13df834fdcbf8d2b88dafcf2d>@@@?$__crt_seh_guarded_call@X@@QEAAX$$QEAV<lambda_842d9ff0dc9ef11c61343bbaebe7f885>@@AEAV<lambda_c5860995281e5c4ce005b3de8f5874ee>@@$$QEAV<lambda_d90129c13df834fdcbf8d2b88dafcf2d>@@@Z@4HA 0000000180060db4     libucrt:fflush.obj
 0001:0005fdb4       $unwind$?fin$0@?0??dllmain_crt_process_detach@@YAH_N@Z@4HA 0000000180060db4     LIBCMT:dll_dllmain.obj
 0001:0005fdb4       $unwind$?fin$0@?0???$common_freopen@_W@@YAHQEAPEAU_iobuf@@QEB_W1V__crt_stdio_stream@@H@Z@4HA 0000000180060db4     libucrt:freopen.obj
 0001:0005fdb4       $unwind$_pclose$fin$0      0000000180060db4     libucrt:popen.obj
 0001:0005fdb4       $unwind$_rmtmp$fin$1       0000000180060db4     libucrt:rmtmp.obj
 0001:0005fdb4       $unwind$_rmtmp$fin$0       0000000180060db4     libucrt:rmtmp.obj
 0001:0005fdb4       $unwind$?fin$0@?0???$?RV<lambda_2d41944a1d46af3157314b8a01080d33>@@AEAV<lambda_8f455de75cd7d7f24b4096f044d8b9e6>@@V<lambda_aa500f224e6afead328df44964fe2772>@@@?$__crt_seh_guarded_call@X@@QEAAX$$QEAV<lambda_2d41944a1d46af3157314b8a01080d33>@@AEAV<lambda_8f455de75cd7d7f24b4096f044d8b9e6>@@$$QEAV<lambda_aa500f224e6afead328df44964fe2772>@@@Z@4HA 0000000180060db4     libucrt:per_thread_data.obj
 0001:0005fdb4       $unwind$?fin$0@?0???$?RV<lambda_f2e299630e499de9f9a165e60fcd3db5>@@AEAV<lambda_2ae9d31cdba2644fcbeaf08da7c24588>@@V<lambda_40d01ff24d0e7b3814fdbdcee8eab3c7>@@@?$__crt_seh_guarded_call@X@@QEAAX$$QEAV<lambda_f2e299630e499de9f9a165e60fcd3db5>@@AEAV<lambda_2ae9d31cdba2644fcbeaf08da7c24588>@@$$QEAV<lambda_40d01ff24d0e7b3814fdbdcee8eab3c7>@@@Z@4HA 0000000180060db4     libucrt:per_thread_data.obj
 0001:0005fdb4       $unwind$?fin$0@?0???$common_ftell@J@@YAJV__crt_stdio_stream@@@Z@4HA 0000000180060db4     libucrt:ftell.obj
 0001:0005fdb4       $unwind$clearerr_s$fin$0   0000000180060db4     libucrt:clearerr.obj
 0001:0005fdb4       $unwind$?fin$0@?0???$common_popen@_W@@YAPEAU_iobuf@@QEB_W0@Z@4HA 0000000180060db4     libucrt:popen.obj
 0001:0005fdb4       $unwind$?fin$0@?0???$?RV<lambda_aa87e3671a710a21b5dc78c0bdf72e11>@@AEAV<lambda_92619d2358a28f41a33ba319515a20b9>@@V<lambda_6992ecaafeb10aed2b74cb1fae11a551>@@@?$__crt_seh_guarded_call@X@@QEAAX$$QEAV<lambda_aa87e3671a710a21b5dc78c0bdf72e11>@@AEAV<lambda_92619d2358a28f41a33ba319515a20b9>@@$$QEAV<lambda_6992ecaafeb10aed2b74cb1fae11a551>@@@Z@4HA 0000000180060db4     libucrt:per_thread_data.obj
 0001:0005fdb4       $unwind$__acrt_lowio_ensure_fh_exists$fin$0 0000000180060db4     libucrt:osfinfo.obj
 0001:0005fdb4       $unwind$fclose$fin$0       0000000180060db4     libucrt:fclose.obj
 0001:0005fdb4       $unwind$?fin$0@?0???$common_fgets@D@@YAPEADQEADHV__crt_stdio_stream@@@Z@4HA 0000000180060db4     libucrt:fgets.obj
 0001:0005fdbc       $unwind$?dllmain_crt_process_detach@@YAH_N@Z 0000000180060dbc     LIBCMT:dll_dllmain.obj
 0001:0005fdf4       $unwind$?dllmain_dispatch@@YAHQEAUHINSTANCE__@@KQEAX@Z 0000000180060df4     LIBCMT:dll_dllmain.obj
 0001:0005fe1c       $unwind$?fin$0@?0??common_tmpfile_nolock@@YAHQEAPEAU_iobuf@@H@Z@4HA 0000000180060e1c     libucrt:tmpfile.obj
 0001:0005fe1c       $unwind$fread_s$fin$0      0000000180060e1c     libucrt:fread.obj
 0001:0005fe1c       $unwind$?filt$0@?0??dllmain_dispatch@@YAHQEAUHINSTANCE__@@KQEAX@Z@4HA 0000000180060e1c     LIBCMT:dll_dllmain.obj
 0001:0005fe1c       $unwind$?fin$0@?0???$common_dupenv_s@_W@@YAHQEAPEA_WQEA_KQEB_WHQEBDH@Z@4HA 0000000180060e1c     libucrt:getenv.obj
 0001:0005fe1c       $unwind$_pipe$fin$0        0000000180060e1c     libucrt:pipe.obj
 0001:0005fe1c       $unwind$_pipe$fin$1        0000000180060e1c     libucrt:pipe.obj
 0001:0005fe24       $unwind$__security_init_cookie 0000000180060e24     LIBCMT:gs_support.obj
 0001:0005fe30       $unwind$__scrt_is_nonwritable_in_current_image 0000000180060e30     LIBCMT:utility.obj
 0001:0005fe50       $unwind$__scrt_is_nonwritable_in_current_image$filt$0 0000000180060e50     LIBCMT:utility.obj
 0001:0005fe58       $unwind$__scrt_fastfail    0000000180060e58     LIBCMT:utility_desktop.obj
 0001:0005fe68       $unwind$__isa_available_init 0000000180060e68     LIBCMT:cpu_disp.obj
 0001:0005fe78       $xdatasym                  0000000180060e78     LIBCMT:guard_dispatch.obj
 0001:0005fe80       $xdatasym                  0000000180060e80     libvcruntime:memcpy.obj
 0001:0005fe90       $xdatasym                  0000000180060e90     libvcruntime:memset.obj
 0001:0005fea0       $unwind$wcsstr             0000000180060ea0     libvcruntime:wcsstr.obj
 0001:0005feb4       $unwind$wcschr             0000000180060eb4     libvcruntime:wcschr.obj
 0001:0005feb4       $unwind$strrchr            0000000180060eb4     libvcruntime:strrchr.obj
 0001:0005feb4       $unwind$strchr             0000000180060eb4     libvcruntime:strchr.obj
 0001:0005fec0       $xdatasym                  0000000180060ec0     libvcruntime:memchr.obj
 0001:0005fec8       $xdatasym                  0000000180060ec8     libvcruntime:memcmp.obj
 0001:0005fecc       $unwind$__C_specific_handler 0000000180060ecc     libvcruntime:riscchandler.obj
 0001:0005fee8       $xdatasym                  0000000180060ee8     libvcruntime:notify.obj
 0001:0005fef4       $unwind$__DestructExceptionObject 0000000180060ef4     libvcruntime:ehhelpers.obj
 0001:0005ff14       $unwind$__acrt_initialize_winapi_thunks 0000000180060f14     libucrt:winapi_thunks.obj
 0001:0005ff14       $unwind$__vcrt_initialize_winapi_thunks 0000000180060f14     libvcruntime:winapi_downlevel.obj
 0001:0005ff14       $unwind$wcsncpy            0000000180060f14     libucrt:wcsncpy.obj
 0001:0005ff1c       $unwind$__vcrt_uninitialize_winapi_thunks 0000000180060f1c     libvcruntime:winapi_downlevel.obj
 0001:0005ff1c       $unwind$__acrt_stdio_end_temporary_buffering_nolock 0000000180060f1c     libucrt:_sftbuf.obj
 0001:0005ff24       $unwind$?try_get_function@@YAPEAXW4function_id@?A0x391cf84c@@QEBDQEBW4module_id@2@2@Z 0000000180060f24     libucrt:winapi_thunks.obj
 0001:0005ff24       $unwind$?try_get_function@@YAPEAXW4function_id@?A0x14c33c87@@QEBDQEBW4module_id@2@2@Z 0000000180060f24     libvcruntime:winapi_downlevel.obj
 0001:0005ff24       $unwind$??$process_string_specifier_tchar@D@?$input_processor@DV?$stream_input_adapter@D@__crt_stdio_input@@@__crt_stdio_input@@AEAA_NW4conversion_mode@1@D@Z 0000000180060f24     libucrt:input.obj
 0001:0005ff40       $xdatasym                  0000000180060f40     libvcruntime:handlers.obj
 0001:0005ff50       $unwind$__stdio_common_vfscanf 0000000180060f50     libucrt:input.obj
 0001:0005ff50       $unwind$__stdio_common_vfprintf 0000000180060f50     libucrt:output.obj
 0001:0005ff58       $unwind$??$common_vsprintf@Vstandard_base@__crt_stdio_output@@_W@@YAH_KQEA_W0QEB_WQEAU__crt_locale_pointers@@QEAD@Z 0000000180060f58     libucrt:output.obj
 0001:0005ff58       $unwind$??$common_vsprintf@Vstandard_base@__crt_stdio_output@@D@@YAH_KQEAD0QEBDQEAU__crt_locale_pointers@@1@Z 0000000180060f58     libucrt:output.obj
 0001:0005ff78       $unwind$?write_string_impl@?$output_adapter_common@DV?$stream_output_adapter@D@__crt_stdio_output@@@__crt_stdio_output@@IEBAXQEBDHQEAHAEAV__crt_deferred_errno_cache@@@Z 0000000180060f78     libucrt:output.obj
 0001:0005ff78       $unwind$_chsize_nolock     0000000180060f78     libucrt:chsize.obj
 0001:0005ff78       $unwind$??$parse_command_line@D@@YAXPEADPEAPEAD0PEA_K2@Z 0000000180060f78     libucrt:argv_parsing.obj
 0001:0005ff94       $unwind$?process@?$output_processor@DV?$stream_output_adapter@D@__crt_stdio_output@@V?$standard_base@DV?$stream_output_adapter@D@__crt_stdio_output@@@2@@__crt_stdio_output@@QEAAHXZ 0000000180060f94     libucrt:output.obj
 0001:0005ff94       $unwind$?process@?$output_processor@DV?$string_output_adapter@D@__crt_stdio_output@@V?$standard_base@DV?$string_output_adapter@D@__crt_stdio_output@@@2@@__crt_stdio_output@@QEAAHXZ 0000000180060f94     libucrt:output.obj
 0001:0005ff94       $unwind$?truncate_ctrl_z_if_present@@YAHH@Z 0000000180060f94     libucrt:open.obj
 0001:0005ffa4       $unwind$?parse_int_from_format_string@?$output_processor@DV?$stream_output_adapter@D@__crt_stdio_output@@V?$standard_base@DV?$stream_output_adapter@D@__crt_stdio_output@@@2@@__crt_stdio_output@@AEAA_NQEAH@Z 0000000180060fa4     libucrt:output.obj
 0001:0005ffa4       $unwind$?process@?$output_processor@_WV?$string_output_adapter@_W@__crt_stdio_output@@V?$standard_base@_WV?$string_output_adapter@_W@__crt_stdio_output@@@2@@__crt_stdio_output@@QEAAHXZ 0000000180060fa4     libucrt:output.obj
 0001:0005ffa4       $unwind$?parse_int_from_format_string@?$output_processor@DV?$string_output_adapter@D@__crt_stdio_output@@V?$standard_base@DV?$string_output_adapter@D@__crt_stdio_output@@@2@@__crt_stdio_output@@AEAA_NQEAH@Z 0000000180060fa4     libucrt:output.obj
 0001:0005ffb8       $unwind$?state_case_type@?$output_processor@DV?$stream_output_adapter@D@__crt_stdio_output@@V?$standard_base@DV?$stream_output_adapter@D@__crt_stdio_output@@@2@@__crt_stdio_output@@AEAA_NXZ 0000000180060fb8     libucrt:output.obj
 0001:0005ffb8       $unwind$?configure_text_mode@@YAHHUfile_options@?A0xa9d50aae@@HAEAW4__crt_lowio_text_mode@@@Z 0000000180060fb8     libucrt:open.obj
 0001:0005ffb8       $unwind$?state_case_type@?$output_processor@DV?$string_output_adapter@D@__crt_stdio_output@@V?$standard_base@DV?$string_output_adapter@D@__crt_stdio_output@@@2@@__crt_stdio_output@@AEAA_NXZ 0000000180060fb8     libucrt:output.obj
 0001:0005ffd0       $unwind$?type_case_a@?$output_processor@DV?$stream_output_adapter@D@__crt_stdio_output@@V?$standard_base@DV?$stream_output_adapter@D@__crt_stdio_output@@@2@@__crt_stdio_output@@AEAA_NXZ 0000000180060fd0     libucrt:output.obj
 0001:0005ffd0       $unwind$?type_case_a@?$output_processor@DV?$string_output_adapter@D@__crt_stdio_output@@V?$standard_base@DV?$string_output_adapter@D@__crt_stdio_output@@@2@@__crt_stdio_output@@AEAA_NXZ 0000000180060fd0     libucrt:output.obj
 0001:0005ffdc       $unwind$?write_stored_string_tchar@?$output_processor@DV?$stream_output_adapter@D@__crt_stdio_output@@V?$standard_base@DV?$stream_output_adapter@D@__crt_stdio_output@@@2@@__crt_stdio_output@@AEAA_ND@Z 0000000180060fdc     libucrt:output.obj
 0001:0005ffdc       $unwind$?write_stored_string_tchar@?$output_processor@DV?$string_output_adapter@D@__crt_stdio_output@@V?$standard_base@DV?$string_output_adapter@D@__crt_stdio_output@@@2@@__crt_stdio_output@@AEAA_ND@Z 0000000180060fdc     libucrt:output.obj
 0001:0005fff4       $unwind$??R<lambda_a31071773b9a94e445cbd5d04ef99106>@@QEBAHXZ 0000000180060ff4     libucrt:output.obj
 0001:00060014       $unwind$??$write_multiple_characters@V?$stream_output_adapter@D@__crt_stdio_output@@D@__crt_stdio_output@@YAXAEBV?$stream_output_adapter@D@0@DHQEAH@Z 0000000180061014     libucrt:output.obj
 0001:00060014       $unwind$?write_string@?$string_output_adapter@D@__crt_stdio_output@@QEBAXQEBDHQEAHAEAV__crt_deferred_errno_cache@@@Z 0000000180061014     libucrt:output.obj
 0001:0006002c       $unwind$?write_string@?$string_output_adapter@_W@__crt_stdio_output@@QEBAXQEB_WHQEAHAEAV__crt_deferred_errno_cache@@@Z 000000018006102c     libucrt:output.obj
 0001:00060044       $unwind$?state_case_type@?$output_processor@_WV?$string_output_adapter@_W@__crt_stdio_output@@V?$standard_base@_WV?$string_output_adapter@_W@__crt_stdio_output@@@2@@__crt_stdio_output@@AEAA_NXZ 0000000180061044     libucrt:output.obj
 0001:00060068       $unwind$?type_case_a@?$output_processor@_WV?$string_output_adapter@_W@__crt_stdio_output@@V?$standard_base@_WV?$string_output_adapter@_W@__crt_stdio_output@@@2@@__crt_stdio_output@@AEAA_NXZ 0000000180061068     libucrt:output.obj
 0001:00060078       $unwind$?write_stored_string_tchar@?$output_processor@_WV?$string_output_adapter@_W@__crt_stdio_output@@V?$standard_base@_WV?$string_output_adapter@_W@__crt_stdio_output@@@2@@__crt_stdio_output@@AEAA_N_W@Z 0000000180061078     libucrt:output.obj
 0001:0006008c       $unwind$??$write_multiple_characters@V?$string_output_adapter@D@__crt_stdio_output@@D@__crt_stdio_output@@YAXAEBV?$string_output_adapter@D@0@DHQEAH@Z 000000018006108c     libucrt:output.obj
 0001:0006008c       $unwind$??$write_multiple_characters@V?$string_output_adapter@_W@__crt_stdio_output@@D@__crt_stdio_output@@YAXAEBV?$string_output_adapter@_W@0@DHQEAH@Z 000000018006108c     libucrt:output.obj
 0001:00060098       $unwind$??$?RV<lambda_a62c933ada0517137acf5807a1eeac1f>@@AEAV<lambda_a31071773b9a94e445cbd5d04ef99106>@@V<lambda_56065050dbf3ada7e59a83db45153de3>@@@?$__crt_seh_guarded_call@H@@QEAAH$$QEAV<lambda_a62c933ada0517137acf5807a1eeac1f>@@AEAV<lambda_a31071773b9a94e445cbd5d04ef99106>@@$$QEAV<lambda_56065050dbf3ada7e59a83db45153de3>@@@Z 0000000180061098     libucrt:output.obj
 0001:000600bc       $unwind$??$common_fsopen@_W@@YAPEAU_iobuf@@QEB_W0H@Z 00000001800610bc     libucrt:fopen.obj
 0001:000600e8       $unwind$fclose             00000001800610e8     libucrt:fclose.obj
 0001:0006010c       $unwind$common_control87   000000018006110c     libucrt:ieee.obj
 0001:00060138       $unwind$??$__acrt_stdio_parse_mode@_W@@YA?AU__acrt_stdio_stream_mode@@QEB_W@Z 0000000180061138     libucrt:openfile.obj
 0001:00060138       $unwind$__acrt_initialize_stdio 0000000180061138     libucrt:_file.obj
 0001:00060138       $unwind$?initialize_stdio_handles_nolock@@YAXXZ 0000000180061138     libucrt:ioinit.obj
 0001:00060138       $unwind$__GSHandlerCheck_SEH 0000000180061138     LIBCMT:gshandlerseh.obj
 0001:00060138       $unwind$__acrt_lowio_set_os_handle 0000000180061138     libucrt:osfinfo.obj
 0001:00060138       $unwind$??$common_xtox@_KD@@YAH_KQEAD0I_N@Z 0000000180061138     libucrt:xtoa.obj
 0001:00060150       $unwind$??$common_freopen@_W@@YAHQEAPEAU_iobuf@@QEB_W1V__crt_stdio_stream@@H@Z 0000000180061150     libucrt:freopen.obj
 0001:0006017c       $unwind$fread_s            000000018006117c     libucrt:fread.obj
 0001:000601ac       $unwind$_fread_nolock_s    00000001800611ac     libucrt:fread.obj
 0001:000601c4       $unwind$fgetc              00000001800611c4     libucrt:fgetc.obj
 0001:000601f8       $unwind$rewind             00000001800611f8     libucrt:rewind.obj
 0001:0006021c       $unwind$ungetc             000000018006121c     libucrt:ungetc.obj
 0001:00060240       $xdatasym                  0000000180061240     libucrt:strcmp.obj
 0001:00060244       $unwind$__dcrt_write_console 0000000180061244     libucrt:initcon.obj
 0001:00060244       $unwind$_wcsicmp_l         0000000180061244     libucrt:wcsicmp.obj
 0001:00060244       $unwind$??$__acrt_wcs_to_mbs_cp@U__crt_win32_buffer_no_resizing@@@@YAHQEB_WAEAV?$__crt_win32_buffer@DU__crt_win32_buffer_no_resizing@@@@I@Z 0000000180061244     libucrt:getmodulefilenamea.obj
 0001:00060258       $xdatasym                  0000000180061258     libucrt:strncmp.obj
 0001:00060260       $xdatasym                  0000000180061260     libucrt:strncpy.obj
 0001:00060264       $unwind$fallbackMethod     0000000180061264     libucrt:strpbrk.obj
 0001:00060274       $unwind$_pclose            0000000180061274     libucrt:popen.obj
 0001:0006029c       $unwind$??$common_popen@_W@@YAPEAU_iobuf@@QEB_W0@Z 000000018006129c     libucrt:popen.obj
 0001:000602cc       $unwind$??$common_popen_nolock@_W@@YAPEAU_iobuf@@QEB_W0HAEAY01H@Z 00000001800612cc     libucrt:popen.obj
 0001:000602ec       $unwind$??$get_executable_path@_W@@YAPEB_WQEB_W@Z 00000001800612ec     libucrt:popen.obj
 0001:00060304       $unwind$clearerr_s         0000000180061304     libucrt:clearerr.obj
 0001:0006032c       $unwind$?common_flush_all@@YAH_N@Z 000000018006132c     libucrt:fflush.obj
 0001:00060334       $unwind$??$?RV<lambda_842d9ff0dc9ef11c61343bbaebe7f885>@@AEAV<lambda_c5860995281e5c4ce005b3de8f5874ee>@@V<lambda_d90129c13df834fdcbf8d2b88dafcf2d>@@@?$__crt_seh_guarded_call@X@@QEAAX$$QEAV<lambda_842d9ff0dc9ef11c61343bbaebe7f885>@@AEAV<lambda_c5860995281e5c4ce005b3de8f5874ee>@@$$QEAV<lambda_d90129c13df834fdcbf8d2b88dafcf2d>@@@Z 0000000180061334     libucrt:fflush.obj
 0001:00060358       $unwind$??$?RV<lambda_886d6c58226a84441f68b9f2b8217b83>@@AEAV<lambda_ab61a845afdef5b7c387490eaf3616ee>@@V<lambda_f7f22ab5edc0698d5f6905b0d3f44752>@@@?$__crt_seh_guarded_call@X@@QEAAX$$QEAV<lambda_886d6c58226a84441f68b9f2b8217b83>@@AEAV<lambda_ab61a845afdef5b7c387490eaf3616ee>@@$$QEAV<lambda_f7f22ab5edc0698d5f6905b0d3f44752>@@@Z 0000000180061358     libucrt:fflush.obj
 0001:00060380       $unwind$??$?RV<lambda_c376a267cfb53b6959b3b692ec76b120>@@AEAV<lambda_9a32fed5bf61b6b509b2d3f6003082a1>@@V<lambda_572fbb9fa0ab338edf41edfd4b5fcc8d>@@@?$__crt_seh_guarded_call@H@@QEAAH$$QEAV<lambda_c376a267cfb53b6959b3b692ec76b120>@@AEAV<lambda_9a32fed5bf61b6b509b2d3f6003082a1>@@$$QEAV<lambda_572fbb9fa0ab338edf41edfd4b5fcc8d>@@@Z 0000000180061380     libucrt:fflush.obj
 0001:000603a4       $unwind$??$common_fgets@D@@YAPEADQEADHV__crt_stdio_stream@@@Z 00000001800613a4     libucrt:fgets.obj
 0001:000603d0       $unwind$?common_fseek@@YAHV__crt_stdio_stream@@_JH@Z 00000001800613d0     libucrt:fseek.obj
 0001:000603f8       $unwind$?common_ftell_translated_utf8_nolock@@YA_JV__crt_stdio_stream@@_J@Z 00000001800613f8     libucrt:ftell.obj
 0001:00060420       $unwind$?common_ftell_read_mode_nolock@@YA_JV__crt_stdio_stream@@_J1@Z 0000000180061420     libucrt:ftell.obj
 0001:00060438       $unwind$??$common_ftell@J@@YAJV__crt_stdio_stream@@@Z 0000000180061438     libucrt:ftell.obj
 0001:0006045c       $unwind$fwrite             000000018006145c     libucrt:fwrite.obj
 0001:00060464       $unwind$_fwrite_nolock     0000000180061464     libucrt:fwrite.obj
 0001:00060480       $unwind$??$?RV<lambda_bdbcead8b570fa3d5ec6d9679862a6e5>@@AEAV<lambda_96f4279ff90247a4c5c5d9824f56f8c1>@@V<lambda_4606be27f17b5e5579e09050fab91818>@@@?$__crt_seh_guarded_call@_K@@QEAA_K$$QEAV<lambda_bdbcead8b570fa3d5ec6d9679862a6e5>@@AEAV<lambda_96f4279ff90247a4c5c5d9824f56f8c1>@@$$QEAV<lambda_4606be27f17b5e5579e09050fab91818>@@@Z 0000000180061480     libucrt:fwrite.obj
 0001:000604a4       $unwind$setvbuf            00000001800614a4     libucrt:setvbuf.obj
 0001:000604ac       $unwind$??$?RV<lambda_84ec643ea9557e2f7dc01bb0e9624395>@@AEAV<lambda_ca71763b3c0644891230e4f79ea54fa6>@@V<lambda_439a761618c59b0600e24586724d733b>@@@?$__crt_seh_guarded_call@H@@QEAAH$$QEAV<lambda_84ec643ea9557e2f7dc01bb0e9624395>@@AEAV<lambda_ca71763b3c0644891230e4f79ea54fa6>@@$$QEAV<lambda_439a761618c59b0600e24586724d733b>@@@Z 00000001800614ac     libucrt:setvbuf.obj
 0001:000604d0       $unwind$?common_tmpfile_nolock@@YAHQEAPEAU_iobuf@@H@Z 00000001800614d0     libucrt:tmpfile.obj
 0001:000604fc       $unwind$??$initialize_tmpfile_buffer_nolock@D@@YA_NW4buffer_id@?A0x5b9a7937@@@Z 00000001800614fc     libucrt:tmpfile.obj
 0001:00060510       $unwind$?common_tmpfile@@YAHQEAPEAU_iobuf@@H@Z 0000000180061510     libucrt:tmpfile.obj
 0001:00060534       $unwind$?divide@__crt_strtox@@YA_KAEAUbig_integer@1@AEBU21@@Z 0000000180061534     libucrt:input.obj
 0001:0006054c       $chain$0$?divide@__crt_strtox@@YA_KAEAUbig_integer@1@AEBU21@@Z 000000018006154c     libucrt:input.obj
 0001:00060560       $chain$1$?divide@__crt_strtox@@YA_KAEAUbig_integer@1@AEBU21@@Z 0000000180061560     libucrt:input.obj
 0001:00060570       $unwind$?assemble_floating_point_value@__crt_strtox@@YA?AW4SLD_STATUS@@_KH_N1AEBVfloating_point_value@1@@Z 0000000180061570     libucrt:input.obj
 0001:00060588       $unwind$?assemble_floating_point_value_from_big_integer@__crt_strtox@@YA?AW4SLD_STATUS@@AEBUbig_integer@1@I_N1AEBVfloating_point_value@1@@Z 0000000180061588     libucrt:input.obj
 0001:000605a4       $unwind$?convert_decimal_string_to_floating_type_common@__crt_strtox@@YA?AW4SLD_STATUS@@AEBUfloating_point_string@1@AEBVfloating_point_value@1@@Z 00000001800615a4     libucrt:input.obj
 0001:000605c8       $unwind$?write_character@?$input_processor@DV?$stream_input_adapter@D@__crt_stdio_input@@@__crt_stdio_input@@AEAA_NQEFA_W_KAEAPEFA_WAEA_KD@Z 00000001800615c8     libucrt:input.obj
 0001:000605d8       $unwind$??R<lambda_f3caf1ecae5fe01a9a1a6239afa44510>@@QEBAHXZ 00000001800615d8     libucrt:input.obj
 0001:000605f8       $unwind$??$process_floating_point_specifier_t@N@?$input_processor@DV?$stream_input_adapter@D@__crt_stdio_input@@@__crt_stdio_input@@AEAA_NXZ 00000001800615f8     libucrt:input.obj
 0001:000605f8       $unwind$??$process_floating_point_specifier_t@M@?$input_processor@DV?$stream_input_adapter@D@__crt_stdio_input@@@__crt_stdio_input@@AEAA_NXZ 00000001800615f8     libucrt:input.obj
 0001:00060604       $unwind$??$parse_integer@_KV?$input_adapter_character_source@V?$stream_input_adapter@D@__crt_stdio_input@@@__crt_strtox@@@__crt_strtox@@YA_KQEAU__crt_locale_pointers@@V?$input_adapter_character_source@V?$stream_input_adapter@D@__crt_stdio_input@@@0@H_N@Z 0000000180061604     libucrt:input.obj
 0001:00060620       $unwind$??$process_string_specifier_tchar@_W@?$input_processor@DV?$stream_input_adapter@D@__crt_stdio_input@@@__crt_stdio_input@@AEAA_NW4conversion_mode@1@_W@Z 0000000180061620     libucrt:input.obj
 0001:00060638       $unwind$??$?RV<lambda_082dd7c0feb7dbdaf245f261e54a6583>@@AEAV<lambda_f3caf1ecae5fe01a9a1a6239afa44510>@@V<lambda_c640b76c0755ae85b317b35c67c61e6b>@@@?$__crt_seh_guarded_call@H@@QEAAH$$QEAV<lambda_082dd7c0feb7dbdaf245f261e54a6583>@@AEAV<lambda_f3caf1ecae5fe01a9a1a6239afa44510>@@$$QEAV<lambda_c640b76c0755ae85b317b35c67c61e6b>@@@Z 0000000180061638     libucrt:input.obj
 0001:0006065c       $unwind$??$parse_floating_point@V?$input_adapter_character_source@V?$stream_input_adapter@D@__crt_stdio_input@@@__crt_strtox@@M@__crt_strtox@@YA?AW4SLD_STATUS@@QEAU__crt_locale_pointers@@V?$input_adapter_character_source@V?$stream_input_adapter@D@__crt_stdio_input@@@0@QEAM@Z 000000018006165c     libucrt:input.obj
 0001:0006065c       $unwind$??$parse_floating_point@V?$input_adapter_character_source@V?$stream_input_adapter@D@__crt_stdio_input@@@__crt_strtox@@N@__crt_strtox@@YA?AW4SLD_STATUS@@QEAU__crt_locale_pointers@@V?$input_adapter_character_source@V?$stream_input_adapter@D@__crt_stdio_input@@@0@QEAN@Z 000000018006165c     libucrt:input.obj
 0001:00060674       $unwind$??$parse_floating_point_from_source@V?$input_adapter_character_source@V?$stream_input_adapter@D@__crt_stdio_input@@@__crt_strtox@@@__crt_strtox@@YA?AW4floating_point_parse_result@0@QEAU__crt_locale_pointers@@AEAV?$input_adapter_character_source@V?$stream_input_adapter@D@__crt_stdio_input@@@0@AEAUfloating_point_string@0@@Z 0000000180061674     libucrt:input.obj
 0001:0006068c       $unwind$??$parse_floating_point_possible_nan@DV?$input_adapter_character_source@V?$stream_input_adapter@D@__crt_stdio_input@@@__crt_strtox@@_K@__crt_strtox@@YA?AW4floating_point_parse_result@0@AEADAEAV?$input_adapter_character_source@V?$stream_input_adapter@D@__crt_stdio_input@@@0@_K@Z 000000018006168c     libucrt:input.obj
 0001:000606a0       $unwind$??$common_getenv@_W@@YAPEA_WQEB_W@Z 00000001800616a0     libucrt:getenv.obj
 0001:000606c0       $unwind$??$common_dupenv_s@_W@@YAHQEAPEA_WQEA_KQEB_WHQEBDH@Z 00000001800616c0     libucrt:getenv.obj
 0001:00060700       $unwind$_wsystem           0000000180061700     libucrt:system.obj
 0001:00060718       $unwind$?common_exit@@YAXHW4_crt_exit_cleanup_mode@@W4_crt_exit_return_mode@@@Z 0000000180061718     libucrt:exit.obj
 0001:00060724       $unwind$??R<lambda_6e4b09c48022b2350581041d5f6b0c4c>@@QEBA@XZ 0000000180061724     libucrt:exit.obj
 0001:00060744       $unwind$??$?RV<lambda_d80eeec6fff315bfe5c115232f3240e3>@@AEAV<lambda_6e4b09c48022b2350581041d5f6b0c4c>@@V<lambda_2358e3775559c9db80273638284d5e45>@@@?$__crt_seh_guarded_call@X@@QEAAX$$QEAV<lambda_d80eeec6fff315bfe5c115232f3240e3>@@AEAV<lambda_6e4b09c48022b2350581041d5f6b0c4c>@@$$QEAV<lambda_2358e3775559c9db80273638284d5e45>@@@Z 0000000180061744     libucrt:exit.obj
 0001:00060768       $unwind$_configure_narrow_argv 0000000180061768     libucrt:argv_parsing.obj
 0001:0006077c       $unwind$??$free_environment@D@@YAXQEAPEAD@Z 000000018006177c     libucrt:environment_initialization.obj
 0001:0006077c       $unwind$??$free_environment@_W@@YAXQEAPEA_W@Z 000000018006177c     libucrt:environment_initialization.obj
 0001:00060788       $unwind$_execute_onexit_table 0000000180061788     libucrt:onexit.obj
 0001:00060790       $unwind$??$?RV<lambda_7777bce6b2f8c936911f934f8298dc43>@@AEAV<lambda_f03950bc5685219e0bcd2087efbe011e>@@V<lambda_3883c3dff614d5e0c5f61bb1ac94921c>@@@?$__crt_seh_guarded_call@H@@QEAAH$$QEAV<lambda_7777bce6b2f8c936911f934f8298dc43>@@AEAV<lambda_f03950bc5685219e0bcd2087efbe011e>@@$$QEAV<lambda_3883c3dff614d5e0c5f61bb1ac94921c>@@@Z 0000000180061790     libucrt:onexit.obj
 0001:000607b4       $unwind$terminate          00000001800617b4     libucrt:terminate.obj
 0001:000607d4       $unwind$?_strupr_s_l_stat@@YAHQEAD_KQEAU__crt_locale_pointers@@@Z 00000001800617d4     libucrt:strupr.obj
 0001:000607f8       $unwind$?x_ismbbtype_l@@YAHPEAU__crt_locale_pointers@@IHH@Z 00000001800617f8     libucrt:ismbbyte.obj
 0001:000607f8       $unwind$_stricmp_l         00000001800617f8     libucrt:stricmp.obj
 0001:00060808       $unwind$??$parse_integer@_KV?$c_string_character_source@D@__crt_strtox@@@__crt_strtox@@YA_KQEAU__crt_locale_pointers@@V?$c_string_character_source@D@0@H_N@Z 0000000180061808     libucrt:atox.obj
 0001:00060808       $unwind$??$parse_integer@KV?$c_string_character_source@D@__crt_strtox@@@__crt_strtox@@YAKQEAU__crt_locale_pointers@@V?$c_string_character_source@D@0@H_N@Z 0000000180061808     libucrt:atox.obj
 0001:00060824       $unwind$??$parse_integer@KV?$c_string_character_source@_W@__crt_strtox@@@__crt_strtox@@YAKQEAU__crt_locale_pointers@@V?$c_string_character_source@_W@0@H_N@Z 0000000180061824     libucrt:atox.obj
 0001:0006083c       $unwind$__acrt_call_reportfault 000000018006183c     libucrt:invalid_parameter.obj
 0001:0006085c       $unwind$_tolower_l         000000018006185c     libucrt:tolower_toupper.obj
 0001:0006086c       $unwind$__acrt_locale_free_numeric 000000018006186c     libucrt:initnum.obj
 0001:0006086c       $unwind$__acrt_locale_free_lc_time_if_unreferenced 000000018006186c     libucrt:locale_refcounting.obj
 0001:0006086c       $unwind$_free_base         000000018006186c     libucrt:free_base.obj
 0001:0006086c       $unwind$?destroy_fls@@YAXPEAX@Z 000000018006186c     libucrt:per_thread_data.obj
 0001:00060874       $unwind$__acrt_LCMapStringEx 0000000180061874     libucrt:winapi_thunks.obj
 0001:00060874       $unwind$_mbtowc_l          0000000180061874     libucrt:mbtowc.obj
 0001:00060874       $unwind$?fp_format_e@@YAHQEBNQEAD_K12H_NIQEAU__crt_locale_pointers@@@Z 0000000180061874     libucrt:cvt.obj
 0001:00060874       $unwind$__acrt_CompareStringEx 0000000180061874     libucrt:winapi_thunks.obj
 0001:00060874       $unwind$__acrt_LCMapStringW 0000000180061874     libucrt:lcmapstringw.obj
 0001:00060888       $unwind$_wctomb_s_l        0000000180061888     libucrt:wctomb.obj
 0001:00060898       $unwind$?construct_ptd_array@@YAXQEAU__acrt_ptd@@@Z 0000000180061898     libucrt:per_thread_data.obj
 0001:000608a0       $unwind$?destroy_ptd_array@@YAXQEAU__acrt_ptd@@@Z 00000001800618a0     libucrt:per_thread_data.obj
 0001:000608a8       $unwind$??$?RV<lambda_0ae27a3a962d80f24befdcbee591983d>@@AEAV<lambda_8d0ee55de4b1038c4002e0adecdf1839>@@V<lambda_dc504788e8f1664fe9b84e20bfb512f2>@@@?$__crt_seh_guarded_call@X@@QEAAX$$QEAV<lambda_0ae27a3a962d80f24befdcbee591983d>@@AEAV<lambda_8d0ee55de4b1038c4002e0adecdf1839>@@$$QEAV<lambda_dc504788e8f1664fe9b84e20bfb512f2>@@@Z 00000001800618a8     libucrt:per_thread_data.obj
 0001:000608cc       $unwind$??$?RV<lambda_aa87e3671a710a21b5dc78c0bdf72e11>@@AEAV<lambda_92619d2358a28f41a33ba319515a20b9>@@V<lambda_6992ecaafeb10aed2b74cb1fae11a551>@@@?$__crt_seh_guarded_call@X@@QEAAX$$QEAV<lambda_aa87e3671a710a21b5dc78c0bdf72e11>@@AEAV<lambda_92619d2358a28f41a33ba319515a20b9>@@$$QEAV<lambda_6992ecaafeb10aed2b74cb1fae11a551>@@@Z 00000001800618cc     libucrt:per_thread_data.obj
 0001:000608f0       $unwind$??$?RV<lambda_f2e299630e499de9f9a165e60fcd3db5>@@AEAV<lambda_2ae9d31cdba2644fcbeaf08da7c24588>@@V<lambda_40d01ff24d0e7b3814fdbdcee8eab3c7>@@@?$__crt_seh_guarded_call@X@@QEAAX$$QEAV<lambda_f2e299630e499de9f9a165e60fcd3db5>@@AEAV<lambda_2ae9d31cdba2644fcbeaf08da7c24588>@@$$QEAV<lambda_40d01ff24d0e7b3814fdbdcee8eab3c7>@@@Z 00000001800618f0     libucrt:per_thread_data.obj
 0001:00060914       $unwind$??$?RV<lambda_2d41944a1d46af3157314b8a01080d33>@@AEAV<lambda_8f455de75cd7d7f24b4096f044d8b9e6>@@V<lambda_aa500f224e6afead328df44964fe2772>@@@?$__crt_seh_guarded_call@X@@QEAAX$$QEAV<lambda_2d41944a1d46af3157314b8a01080d33>@@AEAV<lambda_8f455de75cd7d7f24b4096f044d8b9e6>@@$$QEAV<lambda_aa500f224e6afead328df44964fe2772>@@@Z 0000000180061914     libucrt:per_thread_data.obj
 0001:00060938       $unwind$__acrt_fp_format   0000000180061938     libucrt:cvt.obj
 0001:0006094c       $unwind$?fp_format_nan_or_infinity@@YAHW4__acrt_fp_class@@_NPEAD_K1@Z 000000018006194c     libucrt:cvt.obj
 0001:00060960       $unwind$?fp_format_e_internal@@YAHQEAD_KH_NIQEAU_strflt@@2QEAU__crt_locale_pointers@@@Z 0000000180061960     libucrt:cvt.obj
 0001:00060978       $unwind$?fp_format_a@@YAHQEBNPEAD_KQEAD2H_NIQEAU__crt_locale_pointers@@@Z 0000000180061978     libucrt:cvt.obj
 0001:00060994       $unwind$??$__acrt_wcs_to_mbs_cp@U__crt_win32_buffer_internal_dynamic_resizing@@@@YAHQEB_WAEAV?$__crt_win32_buffer@DU__crt_win32_buffer_internal_dynamic_resizing@@@@I@Z 0000000180061994     libucrt:argv_wildcards.obj
 0001:00060994       $unwind$__dcrt_get_narrow_environment_from_os 0000000180061994     libucrt:get_environment_from_os.obj
 0001:00060994       $unwind$?fp_format_f_internal@@YAHQEAD_KHQEAU_strflt@@_NQEAU__crt_locale_pointers@@@Z 0000000180061994     libucrt:cvt.obj
 0001:00060994       $unwind$_wcsnicmp_l        0000000180061994     libucrt:wcsnicmp.obj
 0001:000609ac       $unwind$?fp_format_g@@YAHQEBNQEAD_K12H_NIQEAU__crt_locale_pointers@@@Z 00000001800619ac     libucrt:cvt.obj
 0001:000609c0       $unwind$__acrt_get_sigabrt_handler 00000001800619c0     libucrt:signal.obj
 0001:000609c0       $unwind$__acrt_uninitialize_locale 00000001800619c0     libucrt:wsetlocale.obj
 0001:000609c8       $unwind$??$?RV<lambda_410d79af7f07d98d83a3f525b3859a53>@@AEAV<lambda_3e16ef9562a7dcce91392c22ab16ea36>@@V<lambda_38119f0e861e05405d8a144b9b982f0a>@@@?$__crt_seh_guarded_call@X@@QEAAX$$QEAV<lambda_410d79af7f07d98d83a3f525b3859a53>@@AEAV<lambda_3e16ef9562a7dcce91392c22ab16ea36>@@$$QEAV<lambda_38119f0e861e05405d8a144b9b982f0a>@@@Z 00000001800619c8     libucrt:wsetlocale.obj
 0001:000609f0       $unwind$__acrt_initialize_lowio 00000001800619f0     libucrt:ioinit.obj
 0001:00060a10       $unwind$?initialize_inherited_file_handles_nolock@@YAXXZ 0000000180061a10     libucrt:ioinit.obj
 0001:00060a2c       $unwind$?__acrt_stdio_allocate_stream@@YA?AV__crt_stdio_stream@@XZ 0000000180061a2c     libucrt:stream.obj
 0001:00060a4c       $unwind$_wopenfile         0000000180061a4c     libucrt:openfile.obj
 0001:00060a60       $unwind$_commit            0000000180061a60     libucrt:commit.obj
 0001:00060a60       $unwind$_close             0000000180061a60     libucrt:close.obj
 0001:00060a68       $unwind$??$?RV<lambda_751a882b2c74d4b022dec766aa51a29a>@@AEAV<lambda_628dfdc04ba53c8bfc02c9951375f3f5>@@V<lambda_f6c7be5f7998530c34de24c7437d6b54>@@@?$__crt_seh_guarded_call@H@@QEAAH$$QEAV<lambda_751a882b2c74d4b022dec766aa51a29a>@@AEAV<lambda_628dfdc04ba53c8bfc02c9951375f3f5>@@$$QEAV<lambda_f6c7be5f7998530c34de24c7437d6b54>@@@Z 0000000180061a68     libucrt:close.obj
 0001:00060a90       $xdatasym                  0000000180061a90     libucrt:fpsr.obj
 0001:00060a98       $unwind$_fcloseall         0000000180061a98     libucrt:closeall.obj
 0001:00060abc       $unwind$_read              0000000180061abc     libucrt:read.obj
 0001:00060aec       $unwind$_read_nolock       0000000180061aec     libucrt:read.obj
 0001:00060b04       $unwind$?translate_ansi_or_utf8_nolock@@YAHHQEAD_KQEA_W1@Z 0000000180061b04     libucrt:read.obj
 0001:00060b20       $unwind$??$translate_text_mode_nolock@D@@YAHHQEAD_K@Z 0000000180061b20     libucrt:read.obj
 0001:00060b38       $unwind$??$translate_text_mode_nolock@_W@@YAHHQEA_W_K@Z 0000000180061b38     libucrt:read.obj
 0001:00060b50       $unwind$??$common_lseek@J@@YAJHJH@Z 0000000180061b50     libucrt:lseek.obj
 0001:00060b80       $unwind$??$common_lseek@_J@@YA_JH_JH@Z 0000000180061b80     libucrt:lseek.obj
 0001:00060bb0       $unwind$_isctype_l         0000000180061bb0     libucrt:isctype.obj
 0001:00060bcc       $unwind$_towlower_l        0000000180061bcc     libucrt:towlower.obj
 0001:00060bd4       $unwind$??$__acrt_mbs_to_wcs_cp@U__crt_win32_buffer_internal_dynamic_resizing@@@@YAHQEBDAEAV?$__crt_win32_buffer@_WU__crt_win32_buffer_internal_dynamic_resizing@@@@I@Z 0000000180061bd4     libucrt:createprocessa.obj
 0001:00060bd4       $unwind$??$copy_environment@_W@@YAPEAPEA_WQEAPEA_W@Z 0000000180061bd4     libucrt:setenv.obj
 0001:00060bec       $unwind$_waccess_s         0000000180061bec     libucrt:waccess.obj
 0001:00060bfc       $unwind$_pipe              0000000180061bfc     libucrt:pipe.obj
 0001:00060c3c       $unwind$??$common_fdopen@_W@@YAPEAU_iobuf@@HQEB_W@Z 0000000180061c3c     libucrt:fdopen.obj
 0001:00060c5c       $unwind$??$?RV<lambda_a37b2b86f63e897a80ea819b0eb08c01>@@AEAV<lambda_38ce7e780aa69e748d6df282ebc68efe>@@V<lambda_99fb1378e971ab6e7edea83e3a7a83a2>@@@?$__crt_seh_guarded_call@H@@QEAAH$$QEAV<lambda_a37b2b86f63e897a80ea819b0eb08c01>@@AEAV<lambda_38ce7e780aa69e748d6df282ebc68efe>@@$$QEAV<lambda_99fb1378e971ab6e7edea83e3a7a83a2>@@@Z 0000000180061c5c     libucrt:commit.obj
 0001:00060c80       $unwind$_write             0000000180061c80     libucrt:write.obj
 0001:00060cb0       $unwind$_write_nolock      0000000180061cb0     libucrt:write.obj
 0001:00060cc8       $unwind$?write_double_translated_ansi_nolock@@YA?AUwrite_result@?A0x17268360@@HQEBDI@Z 0000000180061cc8     libucrt:write.obj
 0001:00060cec       $unwind$?write_text_ansi_nolock@@YA?AUwrite_result@?A0x17268360@@HQEBDI@Z 0000000180061cec     libucrt:write.obj
 0001:00060cec       $unwind$?write_text_utf16le_nolock@@YA?AUwrite_result@?A0x17268360@@HQEBDI@Z 0000000180061cec     libucrt:write.obj
 0001:00060d0c       $unwind$?write_text_utf8_nolock@@YA?AUwrite_result@?A0x17268360@@HQEBDI@Z 0000000180061d0c     libucrt:write.obj
 0001:00060d30       $unwind$??$write_buffer_nolock@D@@YA_NDV__crt_stdio_stream@@@Z 0000000180061d30     libucrt:_flsbuf.obj
 0001:00060d40       $unwind$__acrt_GetTempPathA 0000000180061d40     libucrt:gettemppath.obj
 0001:00060d58       $unwind$_sopen_nolock      0000000180061d58     libucrt:open.obj
 0001:00060d74       $unwind$_wsopen_nolock     0000000180061d74     libucrt:open.obj
 0001:00060d94       $unwind$??$common_sopen_dispatch@D@@YAHQEBDHHHQEAHH@Z 0000000180061d94     libucrt:open.obj
 0001:00060db8       $unwind$?fin$0@?0???$common_sopen_dispatch@_W@@YAHQEB_WHHHQEAHH@Z@4HA 0000000180061db8     libucrt:open.obj
 0001:00060db8       $unwind$?fin$0@?0???$common_sopen_dispatch@D@@YAHQEBDHHHQEAHH@Z@4HA 0000000180061db8     libucrt:open.obj
 0001:00060dc0       $unwind$??$common_sopen_dispatch@_W@@YAHQEB_WHHHQEAHH@Z 0000000180061dc0     libucrt:open.obj
 0001:00060de4       $unwind$_rmtmp             0000000180061de4     libucrt:rmtmp.obj
 0001:00060e18       $unwind$_wcsnicoll_l       0000000180061e18     libucrt:wcsnicol.obj
 0001:00060e18       $unwind$__acrt_CompareStringW 0000000180061e18     libucrt:comparestringw.obj
 0001:00060e30       $unwind$?accumulate_inheritable_handles@@YA_NQEAPEAEQEA_K_N@Z 0000000180061e30     libucrt:spawnv.obj
 0001:00060e38       $unwind$??R<lambda_a094494068278ba5130ab06e1292f60a>@@QEBA_NXZ 0000000180061e38     libucrt:spawnv.obj
 0001:00060e54       $unwind$??$common_spawnv@_W@@YA_JHQEB_WQEBQEB_W1@Z 0000000180061e54     libucrt:spawnv.obj
 0001:00060e70       $unwind$??$?RV<lambda_a22f0c497e5168315e06dae667770027>@@AEAV<lambda_a094494068278ba5130ab06e1292f60a>@@V<lambda_24dc10c13f43218c635520766e23e324>@@@?$__crt_seh_guarded_call@_N@@QEAA_N$$QEAV<lambda_a22f0c497e5168315e06dae667770027>@@AEAV<lambda_a094494068278ba5130ab06e1292f60a>@@$$QEAV<lambda_24dc10c13f43218c635520766e23e324>@@@Z 0000000180061e70     libucrt:spawnv.obj
 0001:00060e94       $unwind$??$execute_command@_W@@YA_JHQEB_WQEBQEB_W1@Z 0000000180061e94     libucrt:spawnv.obj
 0001:00060eb0       $unwind$??$common_spawnvp@_W@@YA_JHQEB_WQEBQEB_W1@Z 0000000180061eb0     libucrt:spawnvp.obj
 0001:00060ed0       $unwind$??$common_expand_argv_wildcards@D@@YAHQEAPEADQEAPEAPEAD@Z 0000000180061ed0     libucrt:argv_wildcards.obj
 0001:00060ee8       $unwind$??$copy_and_add_argument_to_buffer@D@@YAHQEBD0_KAEAV?$argument_list@D@?A0x5f5c8891@@@Z 0000000180061ee8     libucrt:argv_wildcards.obj
 0001:00060ee8       $unwind$??$common_set_variable_in_environment_nolock@_W@@YAHQEA_WH@Z 0000000180061ee8     libucrt:setenv.obj
 0001:00060f04       $unwind$??$expand_argument_wildcards@D@@YAHQEAD0AEAV?$argument_list@D@?A0x5f5c8891@@@Z 0000000180061f04     libucrt:argv_wildcards.obj
 0001:00060f28       $unwind$__acrt_GetModuleFileNameA 0000000180061f28     libucrt:getmodulefilenamea.obj
 0001:00060f44       $unwind$_setmbcp_nolock    0000000180061f44     libucrt:mbctype.obj
 0001:00060f64       $unwind$?update_thread_multibyte_data_internal@@YAPEAU__crt_multibyte_data@@QEAU__acrt_ptd@@QEAPEAU1@@Z 0000000180061f64     libucrt:mbctype.obj
 0001:00060f8c       $unwind$?setmbcp_internal@@YAHH_NQEAU__acrt_ptd@@QEAPEAU__crt_multibyte_data@@@Z 0000000180061f8c     libucrt:mbctype.obj
 0001:00060f9c       $unwind$?setSBUpLow@@YAXPEAU__crt_multibyte_data@@@Z 0000000180061f9c     libucrt:mbctype.obj
 0001:00060fb8       $unwind$??$?RV<lambda_efdfa57d1f175319df784efa44bb7b81>@@AEAV<lambda_5f0a4c1567f8adc6734073e5d1e1b35c>@@V<lambda_2e8a7d3640ea6ccb4c2413664c2db6fd>@@@?$__crt_seh_guarded_call@X@@QEAAX$$QEAV<lambda_efdfa57d1f175319df784efa44bb7b81>@@AEAV<lambda_5f0a4c1567f8adc6734073e5d1e1b35c>@@$$QEAV<lambda_2e8a7d3640ea6ccb4c2413664c2db6fd>@@@Z 0000000180061fb8     libucrt:mbctype.obj
 0001:00060fdc       $unwind$__acrt_WideCharToMultiByte 0000000180061fdc     libucrt:widechartomultibyte.obj
 0001:00060fdc       $unwind$__GSHandlerCheckCommon 0000000180061fdc     LIBCMT:gshandler.obj
 0001:00060fe4       $unwind$_query_new_handler 0000000180061fe4     libucrt:new_handler.obj
 0001:00061004       $unwind$raise              0000000180062004     libucrt:signal.obj
 0001:00061040       $unwind$??$?RV<lambda_450d765d439847d4c735a33c368b5fc0>@@AEAV<lambda_44731a7d0e6d81c3e6aa82d741081786>@@V<lambda_601a2a7da3b7a96e9554ac7215c4b07c>@@@?$__crt_seh_guarded_call@P6AXH@Z@@QEAAP6AXH@Z$$QEAV<lambda_450d765d439847d4c735a33c368b5fc0>@@AEAV<lambda_44731a7d0e6d81c3e6aa82d741081786>@@$$QEAV<lambda_601a2a7da3b7a96e9554ac7215c4b07c>@@@Z 0000000180062040     libucrt:signal.obj
 0001:00061064       $unwind$__acrt_LCMapStringA 0000000180062064     libucrt:lcmapstringa.obj
 0001:00061074       $unwind$?__acrt_LCMapStringA_stat@@YAHPEAU__crt_locale_pointers@@PEB_WKPEBDHPEADHHH@Z 0000000180062074     libucrt:lcmapstringa.obj
 0001:0006109c       $unwind$?__mbsrtowcs_utf8@__crt_mbstring@@YA_KPEA_WPEAPEBD_KPEAU_Mbstatet@@@Z 000000018006209c     libucrt:mbrtowc.obj
 0001:000610b4       $unwind$__acrt_update_thread_locale_data 00000001800620b4     libucrt:locale_refcounting.obj
 0001:000610d8       $unwind$__acrt_fltout      00000001800620d8     libucrt:cfout.obj
 0001:000610f8       $unwind$__acrt_locale_free_monetary 00000001800620f8     libucrt:initmon.obj
 0001:00061100       $unwind$__acrt_locale_free_time 0000000180062100     libucrt:inittime.obj
 0001:00061110       $unwind$__acrt_GetStringTypeA 0000000180062110     libucrt:getstringtypea.obj
 0001:00061138       $unwind$_alloc_osfhnd      0000000180062138     libucrt:osfinfo.obj
 0001:00061168       $unwind$__acrt_lowio_ensure_fh_exists 0000000180062168     libucrt:osfinfo.obj
 0001:00061194       $unwind$?GetTableIndexFromLocaleName@@YAHPEB_W@Z 0000000180062194     libucrt:lcidtoname_downlevel.obj
 0001:000611ac       $unwind$_setmode_nolock    00000001800621ac     libucrt:setmode.obj
 0001:000611bc       $unwind$_putwch_nolock     00000001800621bc     libucrt:putwch.obj
 0001:000611c4       $unwind$__acrt_fenv_set_control 00000001800621c4     libucrt:_fenvutils.obj
 0001:000611d4       $unwind$__acrt_pack_wide_command_line_and_environment 00000001800621d4     libucrt:cenvarg.obj
 0001:000611f0       $unwind$??$construct_environment_block@_W@@YAHQEBQEB_WQEAPEA_W@Z 00000001800621f0     libucrt:cenvarg.obj
 0001:00061210       $unwind$qsort              0000000180062210     libucrt:qsort.obj
 0001:00061228       $chain$4$qsort             0000000180062228     libucrt:qsort.obj
 0001:0006124c       $chain$5$qsort             000000018006224c     libucrt:qsort.obj
 0001:0006125c       $unwind$?__mbrtoc32_utf8@__crt_mbstring@@YA_KPEA_UPEBD_KPEAU_Mbstatet@@@Z 000000018006225c     libucrt:mbrtoc32.obj
 0001:00061278       $xdatasym                  0000000180062278     libucrt:log10.obj
 0001:00061284       $unwind$_call_matherr      0000000180062284     libucrt:libm_error.obj
 0001:0006128c       $unwind$_handle_error      000000018006228c     libucrt:libm_error.obj
 0001:000612ac       $unwind$__acrt_initialize_fma3 00000001800622ac     libucrt:fma3_available.obj
 0001:000612b4       $unwind$_log_special_common 00000001800622b4     libucrt:log_special.obj
 0001:000612c0       $unwind$_raise_exc_ex      00000001800622c0     libucrt:fpexcept.obj
 0001:000612d4       $unwind$_ctrlfp            00000001800622d4     libucrt:fpctrl.obj
 0001:000612fc       $unwind$_IsNonwritableInCurrentImage 00000001800622fc     LIBCMT:pesect.obj
 0001:00061320       $xdatasym                  0000000180062320     LIBCMT:amdsecgs.obj
 0001:00061324       $unwind$__report_securityfailure 0000000180062324     LIBCMT:gs_report.obj
 0001:0006132c       $unwind$__report_gsfailure 000000018006232c     LIBCMT:gs_report.obj
 0001:00061334       $unwind$_local_unwind      0000000180062334     libvcruntime:jmpuwind.obj
 0001:00061340       .edata                     0000000180062340     luafar3.exp
 0001:00061368       rgpv                       0000000180062368     luafar3.exp
 0001:00061414       rgszName                   0000000180062414     luafar3.exp
 0001:000614c0       rgwOrd                     00000001800624c0     luafar3.exp
 0001:00061516       szName                     0000000180062516     luafar3.exp
 0001:00061522       $N00001                    0000000180062522     luafar3.exp
 0001:0006152d       $N00002                    000000018006252d     luafar3.exp
 0001:0006153d       $N00003                    000000018006253d     luafar3.exp
 0001:0006154b       $N00004                    000000018006254b     luafar3.exp
 0001:00061556       $N00005                    0000000180062556     luafar3.exp
 0001:00061563       $N00006                    0000000180062563     luafar3.exp
 0001:00061572       $N00007                    0000000180062572     luafar3.exp
 0001:0006157d       $N00008                    000000018006257d     luafar3.exp
 0001:00061587       $N00009                    0000000180062587     luafar3.exp
 0001:00061592       $N00010                    0000000180062592     luafar3.exp
 0001:000615a5       $N00011                    00000001800625a5     luafar3.exp
 0001:000615b5       $N00012                    00000001800625b5     luafar3.exp
 0001:000615c7       $N00013                    00000001800625c7     luafar3.exp
 0001:000615db       $N00014                    00000001800625db     luafar3.exp
 0001:000615e7       $N00015                    00000001800625e7     luafar3.exp
 0001:000615f6       $N00016                    00000001800625f6     luafar3.exp
 0001:00061607       $N00017                    0000000180062607     luafar3.exp
 0001:00061617       $N00018                    0000000180062617     luafar3.exp
 0001:0006162b       $N00019                    000000018006262b     luafar3.exp
 0001:0006163c       $N00020                    000000018006263c     luafar3.exp
 0001:00061644       $N00021                    0000000180062644     luafar3.exp
 0001:00061655       $N00022                    0000000180062655     luafar3.exp
 0001:00061666       $N00023                    0000000180062666     luafar3.exp
 0001:00061672       $N00024                    0000000180062672     luafar3.exp
 0001:00061683       $N00025                    0000000180062683     luafar3.exp
 0001:00061694       $N00026                    0000000180062694     luafar3.exp
 0001:0006169f       $N00027                    000000018006269f     luafar3.exp
 0001:000616a7       $N00028                    00000001800626a7     luafar3.exp
 0001:000616be       $N00029                    00000001800626be     luafar3.exp
 0001:000616d4       $N00030                    00000001800626d4     luafar3.exp
 0001:000616ea       $N00031                    00000001800626ea     luafar3.exp
 0001:00061700       $N00032                    0000000180062700     luafar3.exp
 0001:00061712       $N00033                    0000000180062712     luafar3.exp
 0001:00061725       $N00034                    0000000180062725     luafar3.exp
 0001:0006173a       $N00035                    000000018006273a     luafar3.exp
 0001:0006174f       $N00036                    000000018006274f     luafar3.exp
 0001:00061766       $N00037                    0000000180062766     luafar3.exp
 0001:0006177c       $N00038                    000000018006277c     luafar3.exp
 0001:00061788       $N00039                    0000000180062788     luafar3.exp
 0001:0006179c       $N00040                    000000018006279c     luafar3.exp
 0001:000617ad       $N00041                    00000001800627ad     luafar3.exp
 0001:000617bd       $N00042                    00000001800627bd     luafar3.exp
 0001:000617cc       $N00043                    00000001800627cc     luafar3.exp
 0002:00001e80       alpha_table                0000000180064e80     lutf8lib.obj
 0002:00003930       lower_table                0000000180066930     lutf8lib.obj
 0002:00004050       upper_table                0000000180067050     lutf8lib.obj
 0002:000046e0       xdigit_table               00000001800676e0     lutf8lib.obj
 0002:00004730       space_table                0000000180067730     lutf8lib.obj
 0002:00004790       unprintable_table          0000000180067790     lutf8lib.obj
 0002:00004850       graph_table                0000000180067850     lutf8lib.obj
 0002:000068c0       compose_table              00000001800698c0     lutf8lib.obj
 0002:000073c0       cntrl_table                000000018006a3c0     lutf8lib.obj
 0002:000074e0       digit_table                000000018006a4e0     lutf8lib.obj
 0002:00007740       alnum_extend_table         000000018006a740     lutf8lib.obj
 0002:00007c50       punct_table                000000018006ac50     lutf8lib.obj
 0002:000084b0       tolower_table              000000018006b4b0     lutf8lib.obj
 0002:00008e70       toupper_table              000000018006be70     lutf8lib.obj
 0002:00009890       totitle_table              000000018006c890     lutf8lib.obj
 0002:0000a2d0       tofold_table               000000018006d2d0     lutf8lib.obj
 0002:0000ad50       doublewidth_table          000000018006dd50     lutf8lib.obj
 0002:0000af00       ambiwidth_table            000000018006df00     lutf8lib.obj
 0002:0000b580       ?__vcrt_flsindex@@3KA      000000018006e580     libvcruntime:per_thread_data.obj
 0002:0000b590       ?dazSupported@?1??common_control87@@9@9 000000018006e590     libucrt:ieee.obj
 0002:0000b594       ?errno_no_memory@@3HA      000000018006e594     libucrt:errno.obj
 0002:0000b598       ?doserrno_no_memory@@3KA   000000018006e598     libucrt:errno.obj
 0002:0000b6b4       ?__acrt_flsindex@@3KA      000000018006e6b4     libucrt:per_thread_data.obj
 0002:0000b990       _mbctypes                  000000018006e990     libucrt:mbctype.obj
 0002:0000baa0       _mbcasemaps                000000018006eaa0     libucrt:mbctype.obj
 0002:0000bba0       ?__rgctypeflag@@3PADA      000000018006eba0     libucrt:mbctype.obj
 0002:0000bbb0       ?__rgcode_page_info@@3PAUcode_page_info@@A 000000018006ebb0     libucrt:mbctype.obj
 0002:0000bf70       ?__dcrt_lowio_console_output_handle@@3PEAXEA 000000018006ef70     libucrt:initcon.obj
 0002:0000bf80       ?dazSupported@?1??_ctrlfp@@9@9 000000018006ef80     libucrt:fpctrl.obj
 0002:0000bf90       luaopen_bit                000000018006ef90     service.obj
 0002:0000bf98       luaopen_ffi                000000018006ef98     service.obj
 0002:0000bfa0       luaopen_jit                000000018006efa0     service.obj
 0002:0000bfa8       ?__proc_attached@@3HA      000000018006efa8     LIBCMT:dll_dllmain.obj
 0002:0000bfd0       ?is_initialized_as_dll@@3_NA 000000018006efd0     LIBCMT:utility.obj
 0002:0000bfd1       ?module_local_atexit_table_initialized@@3_NA 000000018006efd1     LIBCMT:utility.obj
 0002:0000bfd8       ?module_local_atexit_table@@3U_onexit_table_t@@A 000000018006efd8     LIBCMT:utility.obj
 0002:0000bff0       ?module_local_at_quick_exit_table@@3U_onexit_table_t@@A 000000018006eff0     LIBCMT:utility.obj
 0002:0000c058       ?heap@@3V_HeapManager@@A   000000018006f058     libvcruntime:undname.obj
 0002:0000c080       ?__vcrt_startup_thread_ptd@@3U__vcrt_ptd@@A 000000018006f080     libvcruntime:per_thread_data.obj
 0002:0000c110       __vcrt_lock_table          000000018006f110     libvcruntime:locks.obj
 0002:0000c138       __vcrt_locks_initialized   000000018006f138     libvcruntime:locks.obj
 0002:0000c140       ?module_handles@@3PAPEAUHINSTANCE__@@A 000000018006f140     libvcruntime:winapi_downlevel.obj
 0002:0000c158       ?encoded_function_pointers@@3PAPEAXA 000000018006f158     libvcruntime:winapi_downlevel.obj
 0002:0000c1a0       ?__idtabsiz@@3IA           000000018006f1a0     libucrt:popen.obj
 0002:0000c1a8       ?__idpairs@@3PEAUprocess_handle_pair@?A0xe43b7539@@EA 000000018006f1a8     libucrt:popen.obj
 0002:0000c1b0       ?narrow_tmpfile_buffer_pointers@@3PAPEADA 000000018006f1b0     libucrt:tmpfile.obj
 0002:0000c1c8       ?wide_tmpfile_buffer_pointers@@3PAPEA_WA 000000018006f1c8     libucrt:tmpfile.obj
 0002:0000c1e0       ?c_termination_complete@@3JA 000000018006f1e0     libucrt:exit.obj
 0002:0000c1e8       ?thread_local_exit_callback_func@@3P6AXPEAXK0@ZEA 000000018006f1e8     libucrt:exit.obj
 0002:0000c200       ?program_name@?1???$common_configure_argv@D@@YAHW4_crt_argv_mode@@@Z@4PADA 000000018006f200     libucrt:argv_parsing.obj
 0002:0000c358       ?__acrt_invalid_parameter_handler@@3V?$dual_state_global@P6AXPEB_W00I_K@Z@__crt_state_management@@A 000000018006f358     libucrt:invalid_parameter.obj
 0002:0000c360       ?internal_state@?1??_mbtowc_l@@9@4U_Mbstatet@@A 000000018006f360     libucrt:mbtowc.obj
 0002:0000c368       ?enable_percent_n@@3_KA    000000018006f368     libucrt:printf_count_output.obj
 0002:0000c7a0       ?module_handles@@3PAPEAUHINSTANCE__@@A 000000018006f7a0     libucrt:winapi_thunks.obj
 0002:0000c840       ?encoded_function_pointers@@3PAPEAXA 000000018006f840     libucrt:winapi_thunks.obj
 0002:0000c950       ?__acrt_lock_table@@3PAU_RTL_CRITICAL_SECTION@@A 000000018006f950     libucrt:locks.obj
 0002:0000cb80       ?__acrt_locks_initialized@@3IA 000000018006fb80     libucrt:locks.obj
 0002:0000cba0       ?fSystemSet@@3HA           000000018006fba0     libucrt:mbctype.obj
 0002:0000cba4       ?initialized@?1??__acrt_initialize_multibyte@@9@4_NA 000000018006fba4     libucrt:mbctype.obj
 0002:0000cbe0       ?__acrt_new_handler@@3V?$dual_state_global@P6AH_K@Z@__crt_state_management@@A 000000018006fbe0     libucrt:new_handler.obj
 0002:0000cbe8       ?ctrlc_action@@3V?$dual_state_global@P6AXH@Z@__crt_state_management@@A 000000018006fbe8     libucrt:signal.obj
 0002:0000cbf0       ?ctrlbreak_action@@3V?$dual_state_global@P6AXH@Z@__crt_state_management@@A 000000018006fbf0     libucrt:signal.obj
 0002:0000cbf8       ?abort_action@@3V?$dual_state_global@P6AXH@Z@__crt_state_management@@A 000000018006fbf8     libucrt:signal.obj
 0002:0000cc00       ?term_action@@3V?$dual_state_global@P6AXH@Z@__crt_state_management@@A 000000018006fc00     libucrt:signal.obj
 0002:0000cc08       ?user_matherr@@3V?$dual_state_global@P6AHPEAU_exception@@@Z@__crt_state_management@@A 000000018006fc08     libucrt:matherr.obj
 0002:0000cc10       ?__acrt_global_new_mode@@3V?$dual_state_global@J@__crt_state_management@@A 000000018006fc10     libucrt:new_mode.obj
 0002:0000cc20       ?internal_pst@?1??__mbrtoc32_utf8@__crt_mbstring@@YA_KPEA_UPEBD_KPEAU_Mbstatet@@@Z@4U3@A 000000018006fc20     libucrt:mbrtoc32.obj
 0002:0000cc28       ?__acrt_app_type@@3W4_crt_app_type@@A 000000018006fc28     libucrt:report_runtime_error.obj
 0002:0000cc40       GS_ExceptionRecord         000000018006fc40     LIBCMT:gs_report.obj
 0002:0000cce0       GS_ContextRecord           000000018006fce0     LIBCMT:gs_report.obj
 0003:0000000c       $pdata$f_sub               000000018007100c     bit64.obj
 0003:00000018       $pdata$f_mul               0000000180071018     bit64.obj
 0003:00000024       $pdata$f_div               0000000180071024     bit64.obj
 0003:00000030       $pdata$f_mod               0000000180071030     bit64.obj
 0003:0000003c       $pdata$f_unm               000000018007103c     bit64.obj
 0003:00000048       $pdata$f_eq                0000000180071048     bit64.obj
 0003:00000054       $pdata$f_lt                0000000180071054     bit64.obj
 0003:00000060       $pdata$f_le                0000000180071060     bit64.obj
 0003:0000006c       $pdata$band                000000018007106c     bit64.obj
 0003:00000078       $pdata$bor                 0000000180071078     bit64.obj
 0003:00000084       $pdata$bxor                0000000180071084     bit64.obj
 0003:00000090       $pdata$bnot                0000000180071090     bit64.obj
 0003:0000009c       $pdata$lshift              000000018007109c     bit64.obj
 0003:000000a8       $pdata$rshift              00000001800710a8     bit64.obj
 0003:000000b4       $pdata$arshift             00000001800710b4     bit64.obj
 0003:000000c0       $pdata$f_new               00000001800710c0     bit64.obj
 0003:000000cc       $pdata$0$f_new             00000001800710cc     bit64.obj
 0003:000000d8       $pdata$1$f_new             00000001800710d8     bit64.obj
 0003:000000e4       $pdata$f_tostring          00000001800710e4     bit64.obj
 0003:000000f0       $pdata$f_type              00000001800710f0     bit64.obj
 0003:000000fc       $pdata$0$f_type            00000001800710fc     bit64.obj
 0003:00000108       $pdata$1$f_type            0000000180071108     bit64.obj
 0003:00000114       $pdata$f_add               0000000180071114     bit64.obj
 0003:00000120       $pdata$bit64_getvalue      0000000180071120     bit64.obj
 0003:0000012c       $pdata$0$bit64_getvalue    000000018007112c     bit64.obj
 0003:00000138       $pdata$1$bit64_getvalue    0000000180071138     bit64.obj
 0003:00000144       $pdata$bit64_push          0000000180071144     bit64.obj
 0003:00000150       $pdata$bit64_pushuserdata  0000000180071150     bit64.obj
 0003:0000015c       $pdata$check64             000000018007115c     bit64.obj
 0003:00000168       $pdata$0$check64           0000000180071168     bit64.obj
 0003:00000174       $pdata$1$check64           0000000180071174     bit64.obj
 0003:00000180       $pdata$luaopen_bit64       0000000180071180     bit64.obj
 0003:0000018c       $pdata$sprintf             000000018007118c     bit64.obj
 0003:00000198       $pdata$AddBufToCollector   0000000180071198     exported.obj
 0003:000001a4       $pdata$CreateStringsArray  00000001800711a4     exported.obj
 0003:000001b0       $pdata$1$CreateStringsArray 00000001800711b0     exported.obj
 0003:000001bc       $pdata$2$CreateStringsArray 00000001800711bc     exported.obj
 0003:000001c8       $pdata$FarPanelItemFreeCallback 00000001800711c8     exported.obj
 0003:000001d4       $pdata$FillFarMacroCall    00000001800711d4     exported.obj
 0003:000001e0       $pdata$3$FillFarMacroCall  00000001800711e0     exported.obj
 0003:000001ec       $pdata$4$FillFarMacroCall  00000001800711ec     exported.obj
 0003:000001f8       $pdata$FillFarMacroCall_Callback 00000001800711f8     exported.obj
 0003:00000204       $pdata$0$FillFarMacroCall_Callback 0000000180071204     exported.obj
 0003:00000210       $pdata$1$FillFarMacroCall_Callback 0000000180071210     exported.obj
 0003:0000021c       $pdata$FillFindData        000000018007121c     exported.obj
 0003:00000228       $pdata$2$FillFindData      0000000180071228     exported.obj
 0003:00000234       $pdata$3$FillFindData      0000000180071234     exported.obj
 0003:00000240       $pdata$FillPluginPanelItem 0000000180071240     exported.obj
 0003:0000024c       $pdata$1$FillPluginPanelItem 000000018007124c     exported.obj
 0003:00000258       $pdata$2$FillPluginPanelItem 0000000180071258     exported.obj
 0003:00000264       $pdata$3$FillPluginPanelItem 0000000180071264     exported.obj
 0003:00000270       $pdata$4$FillPluginPanelItem 0000000180071270     exported.obj
 0003:0000027c       $pdata$GetExportFunction   000000018007127c     exported.obj
 0003:00000288       $pdata$LF_Analyse          0000000180071288     exported.obj
 0003:00000294       $pdata$LF_ClosePanel       0000000180071294     exported.obj
 0003:000002a0       $pdata$0$LF_ClosePanel     00000001800712a0     exported.obj
 0003:000002ac       $pdata$1$LF_ClosePanel     00000001800712ac     exported.obj
 0003:000002b8       $pdata$LF_Compare          00000001800712b8     exported.obj
 0003:000002c4       $pdata$0$LF_Compare        00000001800712c4     exported.obj
 0003:000002d0       $pdata$2$LF_Compare        00000001800712d0     exported.obj
 0003:000002dc       $pdata$3$LF_Compare        00000001800712dc     exported.obj
 0003:000002e8       $pdata$LF_Configure        00000001800712e8     exported.obj
 0003:000002f4       $pdata$LF_DeleteFiles      00000001800712f4     exported.obj
 0003:00000300       $pdata$0$LF_DeleteFiles    0000000180071300     exported.obj
 0003:0000030c       $pdata$2$LF_DeleteFiles    000000018007130c     exported.obj
 0003:00000318       $pdata$3$LF_DeleteFiles    0000000180071318     exported.obj
 0003:00000324       $pdata$LF_ExitFAR          0000000180071324     exported.obj
 0003:00000330       $pdata$LF_FreeContentData  0000000180071330     exported.obj
 0003:0000033c       $pdata$LF_FreeFindData     000000018007133c     exported.obj
 0003:00000348       $pdata$LF_GetContentData   0000000180071348     exported.obj
 0003:00000354       $pdata$0$LF_GetContentData 0000000180071354     exported.obj
 0003:00000360       $pdata$1$LF_GetContentData 0000000180071360     exported.obj
 0003:0000036c       $pdata$LF_GetContentFields 000000018007136c     exported.obj
 0003:00000378       $pdata$0$LF_GetContentFields 0000000180071378     exported.obj
 0003:00000384       $pdata$1$LF_GetContentFields 0000000180071384     exported.obj
 0003:00000390       $pdata$LF_GetFiles         0000000180071390     exported.obj
 0003:0000039c       $pdata$0$LF_GetFiles       000000018007139c     exported.obj
 0003:000003a8       $pdata$2$LF_GetFiles       00000001800713a8     exported.obj
 0003:000003b4       $pdata$3$LF_GetFiles       00000001800713b4     exported.obj
 0003:000003c0       $pdata$LF_GetFindData      00000001800713c0     exported.obj
 0003:000003cc       $pdata$0$LF_GetFindData    00000001800713cc     exported.obj
 0003:000003d8       $pdata$1$LF_GetFindData    00000001800713d8     exported.obj
 0003:000003e4       $pdata$LF_GetGlobalInfo    00000001800713e4     exported.obj
 0003:000003f0       $pdata$2$LF_GetGlobalInfo  00000001800713f0     exported.obj
 0003:000003fc       $pdata$3$LF_GetGlobalInfo  00000001800713fc     exported.obj
 0003:00000408       $pdata$4$LF_GetGlobalInfo  0000000180071408     exported.obj
 0003:00000414       $pdata$LF_GetOpenPanelInfo 0000000180071414     exported.obj
 0003:00000420       $pdata$1$LF_GetOpenPanelInfo 0000000180071420     exported.obj
 0003:0000042c       $pdata$3$LF_GetOpenPanelInfo 000000018007142c     exported.obj
 0003:00000438       $pdata$5$LF_GetOpenPanelInfo 0000000180071438     exported.obj
 0003:00000444       $pdata$7$LF_GetOpenPanelInfo 0000000180071444     exported.obj
 0003:00000450       $pdata$8$LF_GetOpenPanelInfo 0000000180071450     exported.obj
 0003:0000045c       $pdata$9$LF_GetOpenPanelInfo 000000018007145c     exported.obj
 0003:00000468       $pdata$10$LF_GetOpenPanelInfo 0000000180071468     exported.obj
 0003:00000474       $pdata$LF_GetPluginInfo    0000000180071474     exported.obj
 0003:00000480       $pdata$1$LF_GetPluginInfo  0000000180071480     exported.obj
 0003:0000048c       $pdata$2$LF_GetPluginInfo  000000018007148c     exported.obj
 0003:00000498       $pdata$LF_MakeDirectory    0000000180071498     exported.obj
 0003:000004a4       $pdata$0$LF_MakeDirectory  00000001800714a4     exported.obj
 0003:000004b0       $pdata$2$LF_MakeDirectory  00000001800714b0     exported.obj
 0003:000004bc       $pdata$3$LF_MakeDirectory  00000001800714bc     exported.obj
 0003:000004c8       $pdata$LF_Open             00000001800714c8     exported.obj
 0003:000004d4       $pdata$LF_ProcessConsoleInput 00000001800714d4     exported.obj
 0003:000004e0       $pdata$0$LF_ProcessConsoleInput 00000001800714e0     exported.obj
 0003:000004ec       $pdata$1$LF_ProcessConsoleInput 00000001800714ec     exported.obj
 0003:000004f8       $pdata$LF_ProcessDialogEvent 00000001800714f8     exported.obj
 0003:00000504       $pdata$LF_ProcessEditorEvent 0000000180071504     exported.obj
 0003:00000510       $pdata$0$LF_ProcessEditorEvent 0000000180071510     exported.obj
 0003:0000051c       $pdata$1$LF_ProcessEditorEvent 000000018007151c     exported.obj
 0003:00000528       $pdata$LF_ProcessEditorInput 0000000180071528     exported.obj
 0003:00000534       $pdata$LF_ProcessHostFile  0000000180071534     exported.obj
 0003:00000540       $pdata$LF_ProcessPanelEvent 0000000180071540     exported.obj
 0003:0000054c       $pdata$LF_ProcessPanelInput 000000018007154c     exported.obj
 0003:00000558       $pdata$LF_ProcessSynchroEvent 0000000180071558     exported.obj
 0003:00000564       $pdata$1$LF_ProcessSynchroEvent 0000000180071564     exported.obj
 0003:00000570       $pdata$2$LF_ProcessSynchroEvent 0000000180071570     exported.obj
 0003:0000057c       $pdata$3$LF_ProcessSynchroEvent 000000018007157c     exported.obj
 0003:00000588       $pdata$5$LF_ProcessSynchroEvent 0000000180071588     exported.obj
 0003:00000594       $pdata$6$LF_ProcessSynchroEvent 0000000180071594     exported.obj
 0003:000005a0       $pdata$LF_ProcessViewerEvent 00000001800715a0     exported.obj
 0003:000005ac       $pdata$LF_PutFiles         00000001800715ac     exported.obj
 0003:000005b8       $pdata$LF_SetDirectory     00000001800715b8     exported.obj
 0003:000005c4       $pdata$LF_SetFindList      00000001800715c4     exported.obj
 0003:000005d0       $pdata$PackMacroValues     00000001800715d0     exported.obj
 0003:000005dc       $pdata$0$PackMacroValues   00000001800715dc     exported.obj
 0003:000005e8       $pdata$1$PackMacroValues   00000001800715e8     exported.obj
 0003:000005f4       $pdata$PushAnalyseInfo     00000001800715f4     exported.obj
 0003:00000600       $pdata$PushFarMacroValue   0000000180071600     exported.obj
 0003:0000060c       $pdata$PushPluginObject    000000018007160c     exported.obj
 0003:00000618       $pdata$PushPluginPair      0000000180071618     exported.obj
 0003:00000624       $pdata$RegisterObject      0000000180071624     exported.obj
 0003:00000630       $pdata$ReplacePluginInfoCollector 0000000180071630     exported.obj
 0003:0000063c       $pdata$RunDefaultScript    000000018007163c     exported.obj
 0003:00000648       $pdata$0$RunDefaultScript  0000000180071648     exported.obj
 0003:00000654       $pdata$1$RunDefaultScript  0000000180071654     exported.obj
 0003:00000660       $pdata$UpdateFileSelection 0000000180071660     exported.obj
 0003:0000066c       $pdata$0$UpdateFileSelection 000000018007166c     exported.obj
 0003:00000678       $pdata$1$UpdateFileSelection 0000000180071678     exported.obj
 0003:00000684       $pdata$_AddStringToCollector 0000000180071684     exported.obj
 0003:00000690       $pdata$0$_AddStringToCollector 0000000180071690     exported.obj
 0003:0000069c       $pdata$1$_AddStringToCollector 000000018007169c     exported.obj
 0003:000006a8       $pdata$getPluginMenuItems  00000001800716a8     exported.obj
 0003:000006b4       $pdata$pcall_msg           00000001800716b4     exported.obj
 0003:000006c0       $pdata$traceback           00000001800716c0     exported.obj
 0003:000006cc       $pdata$push_flags_table    00000001800716cc     flags.obj
 0003:000006d8       $pdata$SetFarColors        00000001800716d8     keysandcolors.obj
 0003:000006e4       $pdata$LF_Gsub             00000001800716e4     lflua.obj
 0003:000006f0       $pdata$LF_LoadFile         00000001800716f0     lflua.obj
 0003:000006fc       $pdata$1$LF_LoadFile       00000001800716fc     lflua.obj
 0003:00000708       $pdata$2$LF_LoadFile       0000000180071708     lflua.obj
 0003:00000714       $pdata$3$LF_LoadFile       0000000180071714     lflua.obj
 0003:00000720       $pdata$4$LF_LoadFile       0000000180071720     lflua.obj
 0003:0000072c       $pdata$errfile             000000018007172c     lflua.obj
 0003:00000738       $pdata$getF                0000000180071738     lflua.obj
 0003:00000744       $pdata$luaB_dofileW        0000000180071744     lflua.obj
 0003:00000750       $pdata$luaB_loadfileW      0000000180071750     lflua.obj
 0003:0000075c       $pdata$method_gc           000000018007175c     lregex.obj
 0003:00000768       $pdata$method_tostring     0000000180071768     lregex.obj
 0003:00000774       $pdata$method_bracketscount 0000000180071774     lregex.obj
 0003:00000780       $pdata$func_New            0000000180071780     lregex.obj
 0003:0000078c       $pdata$_Gmatch             000000018007178c     lregex.obj
 0003:00000798       $pdata$_regex_gmatch_closure 0000000180071798     lregex.obj
 0003:000007a4       $pdata$1$_regex_gmatch_closure 00000001800717a4     lregex.obj
 0003:000007b0       $pdata$2$_regex_gmatch_closure 00000001800717b0     lregex.obj
 0003:000007bc       $pdata$3$_regex_gmatch_closure 00000001800717bc     lregex.obj
 0003:000007c8       $pdata$check_regex_pattern 00000001800717c8     lregex.obj
 0003:000007d4       $pdata$1$check_regex_pattern 00000001800717d4     lregex.obj
 0003:000007e0       $pdata$2$check_regex_pattern 00000001800717e0     lregex.obj
 0003:000007ec       $pdata$luaopen_regex       00000001800717ec     lregex.obj
 0003:000007f8       $pdata$push_far_regex      00000001800717f8     lregex.obj
 0003:00000804       $pdata$rx_find_match       0000000180071804     lregex.obj
 0003:00000810       $pdata$rx_gsub             0000000180071810     lregex.obj
 0003:0000081c       $pdata$FL_PushParams       000000018007181c     luamacro.obj
 0003:00000828       $pdata$0$FL_PushParams     0000000180071828     luamacro.obj
 0003:00000834       $pdata$1$FL_PushParams     0000000180071834     luamacro.obj
 0003:00000840       $pdata$2$FL_PushParams     0000000180071840     luamacro.obj
 0003:0000084c       $pdata$3$FL_PushParams     000000018007184c     luamacro.obj
 0003:00000858       $pdata$4$FL_PushParams     0000000180071858     luamacro.obj
 0003:00000864       $pdata$5$FL_PushParams     0000000180071864     luamacro.obj
 0003:00000870       $pdata$InitMPR             0000000180071870     luamacro.obj
 0003:0000087c       $pdata$Open_Luamacro       000000018007187c     luamacro.obj
 0003:00000888       $pdata$0$Open_Luamacro     0000000180071888     luamacro.obj
 0003:00000894       $pdata$1$Open_Luamacro     0000000180071894     luamacro.obj
 0003:000008a0       $pdata$far_FarMacroCallToLua 00000001800718a0     luamacro.obj
 0003:000008ac       $pdata$0$far_FarMacroCallToLua 00000001800718ac     luamacro.obj
 0003:000008b8       $pdata$1$far_FarMacroCallToLua 00000001800718b8     luamacro.obj
 0003:000008c4       $pdata$far_MacroCallFar    00000001800718c4     luamacro.obj
 0003:000008d0       $pdata$2$far_MacroCallFar  00000001800718d0     luamacro.obj
 0003:000008dc       $pdata$3$far_MacroCallFar  00000001800718dc     luamacro.obj
 0003:000008e8       $pdata$4$far_MacroCallFar  00000001800718e8     luamacro.obj
 0003:000008f4       $pdata$5$far_MacroCallFar  00000001800718f4     luamacro.obj
 0003:00000900       $pdata$uc_tostring         0000000180071900     lusercontrol.obj
 0003:0000090c       $pdata$uc_len              000000018007190c     lusercontrol.obj
 0003:00000918       $pdata$uc_index            0000000180071918     lusercontrol.obj
 0003:00000924       $pdata$uc_newindex         0000000180071924     lusercontrol.obj
 0003:00000930       $pdata$uc_New              0000000180071930     lusercontrol.obj
 0003:0000093c       $pdata$luaopen_usercontrol 000000018007193c     lusercontrol.obj
 0003:00000948       $pdata$CreateRegKey        0000000180071948     reg.obj
 0003:00000954       $pdata$OpenRegKey          0000000180071954     reg.obj
 0003:00000960       $pdata$SetRegKeyArr        0000000180071960     reg.obj
 0003:0000096c       $pdata$0$SetRegKeyArr      000000018007196c     reg.obj
 0003:00000978       $pdata$1$SetRegKeyArr      0000000180071978     reg.obj
 0003:00000984       $pdata$SetRegKeyDword      0000000180071984     reg.obj
 0003:00000990       $pdata$0$SetRegKeyDword    0000000180071990     reg.obj
 0003:0000099c       $pdata$1$SetRegKeyDword    000000018007199c     reg.obj
 0003:000009a8       $pdata$SetRegKeyStr        00000001800719a8     reg.obj
 0003:000009b4       $pdata$0$SetRegKeyStr      00000001800719b4     reg.obj
 0003:000009c0       $pdata$1$SetRegKeyStr      00000001800719c0     reg.obj
 0003:000009cc       $pdata$far_GetFileOwner    00000001800719cc     service.obj
 0003:000009d8       $pdata$far_GetNumberOfLinks 00000001800719d8     service.obj
 0003:000009e4       $pdata$far_PluginStartupInfo 00000001800719e4     service.obj
 0003:000009f0       $pdata$far_GetCurrentDirectory 00000001800719f0     service.obj
 0003:000009fc       $pdata$editor_GetFileName  00000001800719fc     service.obj
 0003:00000a08       $pdata$editor_GetInfo      0000000180071a08     service.obj
 0003:00000a14       $pdata$2$editor_GetInfo    0000000180071a14     service.obj
 0003:00000a20       $pdata$3$editor_GetInfo    0000000180071a20     service.obj
 0003:00000a2c       $pdata$4$editor_GetInfo    0000000180071a2c     service.obj
 0003:00000a38       $pdata$5$editor_GetInfo    0000000180071a38     service.obj
 0003:00000a44       $pdata$editor_InsertString 0000000180071a44     service.obj
 0003:00000a50       $pdata$editor_DeleteString 0000000180071a50     service.obj
 0003:00000a5c       $pdata$editor_InsertText   0000000180071a5c     service.obj
 0003:00000a68       $pdata$editor_DeleteChar   0000000180071a68     service.obj
 0003:00000a74       $pdata$editor_DeleteBlock  0000000180071a74     service.obj
 0003:00000a80       $pdata$editor_UndoRedo     0000000180071a80     service.obj
 0003:00000a8c       $pdata$editor_SetParam     0000000180071a8c     service.obj
 0003:00000a98       $pdata$editor_SetPosition  0000000180071a98     service.obj
 0003:00000aa4       $pdata$editor_Redraw       0000000180071aa4     service.obj
 0003:00000ab0       $pdata$editor_ExpandTabs   0000000180071ab0     service.obj
 0003:00000abc       $pdata$editor_AddSessionBookmark 0000000180071abc     service.obj
 0003:00000ac8       $pdata$editor_ClearSessionBookmarks 0000000180071ac8     service.obj
 0003:00000ad4       $pdata$editor_DeleteSessionBookmark 0000000180071ad4     service.obj
 0003:00000ae0       $pdata$editor_NextSessionBookmark 0000000180071ae0     service.obj
 0003:00000aec       $pdata$editor_PrevSessionBookmark 0000000180071aec     service.obj
 0003:00000af8       $pdata$editor_SetTitle     0000000180071af8     service.obj
 0003:00000b04       $pdata$editor_GetTitle     0000000180071b04     service.obj
 0003:00000b10       $pdata$editor_Quit         0000000180071b10     service.obj
 0003:00000b1c       $pdata$editor_Select       0000000180071b1c     service.obj
 0003:00000b28       $pdata$editor_GetSelection 0000000180071b28     service.obj
 0003:00000b34       $pdata$editor_AddColor     0000000180071b34     service.obj
 0003:00000b40       $pdata$editor_DelColor     0000000180071b40     service.obj
 0003:00000b4c       $pdata$editor_GetColor     0000000180071b4c     service.obj
 0003:00000b58       $pdata$editor_SaveFile     0000000180071b58     service.obj
 0003:00000b64       $pdata$editor_ReadInput    0000000180071b64     service.obj
 0003:00000b70       $pdata$editor_ProcessInput 0000000180071b70     service.obj
 0003:00000b7c       $pdata$editor_SubscribeChangeEvent 0000000180071b7c     service.obj
 0003:00000b88       $pdata$far_Menu            0000000180071b88     service.obj
 0003:00000b94       $pdata$0$far_Menu          0000000180071b94     service.obj
 0003:00000ba0       $pdata$1$far_Menu          0000000180071ba0     service.obj
 0003:00000bac       $pdata$far_Message         0000000180071bac     service.obj
 0003:00000bb8       $pdata$panel_CheckPanelsExist 0000000180071bb8     service.obj
 0003:00000bc4       $pdata$panel_ClosePanel    0000000180071bc4     service.obj
 0003:00000bd0       $pdata$panel_GetPanelInfo  0000000180071bd0     service.obj
 0003:00000bdc       $pdata$0$panel_GetPanelInfo 0000000180071bdc     service.obj
 0003:00000be8       $pdata$1$panel_GetPanelInfo 0000000180071be8     service.obj
 0003:00000bf4       $pdata$panel_RedrawPanel   0000000180071bf4     service.obj
 0003:00000c00       $pdata$panel_GetPanelDirectory 0000000180071c00     service.obj
 0003:00000c0c       $pdata$panel_SetPanelDirectory 0000000180071c0c     service.obj
 0003:00000c18       $pdata$panel_GetCmdLine    0000000180071c18     service.obj
 0003:00000c24       $pdata$panel_SetCmdLine    0000000180071c24     service.obj
 0003:00000c30       $pdata$panel_GetCmdLinePos 0000000180071c30     service.obj
 0003:00000c3c       $pdata$panel_SetCmdLinePos 0000000180071c3c     service.obj
 0003:00000c48       $pdata$panel_InsertCmdLine 0000000180071c48     service.obj
 0003:00000c54       $pdata$panel_GetCmdLineSelection 0000000180071c54     service.obj
 0003:00000c60       $pdata$panel_SetCmdLineSelection 0000000180071c60     service.obj
 0003:00000c6c       $pdata$panel_BeginSelection 0000000180071c6c     service.obj
 0003:00000c78       $pdata$panel_EndSelection  0000000180071c78     service.obj
 0003:00000c84       $pdata$panel_SetUserScreen 0000000180071c84     service.obj
 0003:00000c90       $pdata$panel_GetUserScreen 0000000180071c90     service.obj
 0003:00000c9c       $pdata$panel_IsActivePanel 0000000180071c9c     service.obj
 0003:00000ca8       $pdata$panel_SetActivePanel 0000000180071ca8     service.obj
 0003:00000cb4       $pdata$far_GetDirList      0000000180071cb4     service.obj
 0003:00000cc0       $pdata$0$far_GetDirList    0000000180071cc0     service.obj
 0003:00000ccc       $pdata$6$far_GetDirList    0000000180071ccc     service.obj
 0003:00000cd8       $pdata$7$far_GetDirList    0000000180071cd8     service.obj
 0003:00000ce4       $pdata$8$far_GetDirList    0000000180071ce4     service.obj
 0003:00000cf0       $pdata$far_GetPluginDirList 0000000180071cf0     service.obj
 0003:00000cfc       $pdata$far_RestoreScreen   0000000180071cfc     service.obj
 0003:00000d08       $pdata$far_SaveScreen      0000000180071d08     service.obj
 0003:00000d14       $pdata$far_SendDlgMessage  0000000180071d14     service.obj
 0003:00000d20       $pdata$far_DialogInit      0000000180071d20     service.obj
 0003:00000d2c       $pdata$far_DialogRun       0000000180071d2c     service.obj
 0003:00000d38       $pdata$far_DialogFree      0000000180071d38     service.obj
 0003:00000d44       $pdata$dialog_tostring     0000000180071d44     service.obj
 0003:00000d50       $pdata$dialog_rawhandle    0000000180071d50     service.obj
 0003:00000d5c       $pdata$far_GetDlgItem      0000000180071d5c     service.obj
 0003:00000d68       $pdata$far_SetDlgItem      0000000180071d68     service.obj
 0003:00000d74       $pdata$far_SubscribeDialogDrawEvents 0000000180071d74     service.obj
 0003:00000d80       $pdata$editor_Editor       0000000180071d80     service.obj
 0003:00000d8c       $pdata$viewer_Viewer       0000000180071d8c     service.obj
 0003:00000d98       $pdata$viewer_GetFileName  0000000180071d98     service.obj
 0003:00000da4       $pdata$viewer_GetInfo      0000000180071da4     service.obj
 0003:00000db0       $pdata$1$viewer_GetInfo    0000000180071db0     service.obj
 0003:00000dbc       $pdata$2$viewer_GetInfo    0000000180071dbc     service.obj
 0003:00000dc8       $pdata$3$viewer_GetInfo    0000000180071dc8     service.obj
 0003:00000dd4       $pdata$4$viewer_GetInfo    0000000180071dd4     service.obj
 0003:00000de0       $pdata$viewer_Quit         0000000180071de0     service.obj
 0003:00000dec       $pdata$viewer_Redraw       0000000180071dec     service.obj
 0003:00000df8       $pdata$viewer_Select       0000000180071df8     service.obj
 0003:00000e04       $pdata$viewer_SetPosition  0000000180071e04     service.obj
 0003:00000e10       $pdata$2$viewer_SetPosition 0000000180071e10     service.obj
 0003:00000e1c       $pdata$3$viewer_SetPosition 0000000180071e1c     service.obj
 0003:00000e28       $pdata$viewer_SetMode      0000000180071e28     service.obj
 0003:00000e34       $pdata$far_ShowHelp        0000000180071e34     service.obj
 0003:00000e40       $pdata$far_InputBox        0000000180071e40     service.obj
 0003:00000e4c       $pdata$far_GetMsg          0000000180071e4c     service.obj
 0003:00000e58       $pdata$far_Text            0000000180071e58     service.obj
 0003:00000e64       $pdata$far_CopyToClipboard 0000000180071e64     service.obj
 0003:00000e70       $pdata$1$far_CopyToClipboard 0000000180071e70     service.obj
 0003:00000e7c       $pdata$2$far_CopyToClipboard 0000000180071e7c     service.obj
 0003:00000e88       $pdata$far_PasteFromClipboard 0000000180071e88     service.obj
 0003:00000e94       $pdata$far_InputRecordToName 0000000180071e94     service.obj
 0003:00000ea0       $pdata$far_NameToInputRecord 0000000180071ea0     service.obj
 0003:00000eac       $pdata$far_LStricmp        0000000180071eac     service.obj
 0003:00000eb8       $pdata$far_LStrnicmp       0000000180071eb8     service.obj
 0003:00000ec4       $pdata$far_ProcessName     0000000180071ec4     service.obj
 0003:00000ed0       $pdata$2$far_ProcessName   0000000180071ed0     service.obj
 0003:00000edc       $pdata$3$far_ProcessName   0000000180071edc     service.obj
 0003:00000ee8       $pdata$4$far_ProcessName   0000000180071ee8     service.obj
 0003:00000ef4       $pdata$5$far_ProcessName   0000000180071ef4     service.obj
 0003:00000f00       $pdata$6$far_ProcessName   0000000180071f00     service.obj
 0003:00000f0c       $pdata$7$far_ProcessName   0000000180071f0c     service.obj
 0003:00000f18       $pdata$far_GetReparsePointInfo 0000000180071f18     service.obj
 0003:00000f24       $pdata$0$far_GetReparsePointInfo 0000000180071f24     service.obj
 0003:00000f30       $pdata$1$far_GetReparsePointInfo 0000000180071f30     service.obj
 0003:00000f3c       $pdata$far_LIsAlpha        0000000180071f3c     service.obj
 0003:00000f48       $pdata$far_LIsAlphanum     0000000180071f48     service.obj
 0003:00000f54       $pdata$far_LIsLower        0000000180071f54     service.obj
 0003:00000f60       $pdata$far_LIsUpper        0000000180071f60     service.obj
 0003:00000f6c       $pdata$far_LLowerBuf       0000000180071f6c     service.obj
 0003:00000f78       $pdata$far_LUpperBuf       0000000180071f78     service.obj
 0003:00000f84       $pdata$far_MkTemp          0000000180071f84     service.obj
 0003:00000f90       $pdata$far_MkLink          0000000180071f90     service.obj
 0003:00000f9c       $pdata$far_GetPathRoot     0000000180071f9c     service.obj
 0003:00000fa8       $pdata$far_RecursiveSearch 0000000180071fa8     service.obj
 0003:00000fb4       $pdata$far_ConvertPath     0000000180071fb4     service.obj
 0003:00000fc0       $pdata$far_AdvControl      0000000180071fc0     service.obj
 0003:00000fcc       $pdata$0$far_AdvControl    0000000180071fcc     service.obj
 0003:00000fd8       $pdata$1$far_AdvControl    0000000180071fd8     service.obj
 0003:00000fe4       $pdata$far_MacroLoadAll    0000000180071fe4     service.obj
 0003:00000ff0       $pdata$0$far_MacroLoadAll  0000000180071ff0     service.obj
 0003:00000ffc       $pdata$1$far_MacroLoadAll  0000000180071ffc     service.obj
 0003:00001008       $pdata$far_MacroSaveAll    0000000180072008     service.obj
 0003:00001014       $pdata$far_MacroGetState   0000000180072014     service.obj
 0003:00001020       $pdata$far_MacroGetArea    0000000180072020     service.obj
 0003:0000102c       $pdata$far_MacroGetLastError 000000018007202c     service.obj
 0003:00001038       $pdata$0$far_MacroGetLastError 0000000180072038     service.obj
 0003:00001044       $pdata$1$far_MacroGetLastError 0000000180072044     service.obj
 0003:00001050       $pdata$far_MacroAdd        0000000180072050     service.obj
 0003:0000105c       $pdata$far_MacroDelete     000000018007205c     service.obj
 0003:00001068       $pdata$far_MacroExecute    0000000180072068     service.obj
 0003:00001074       $pdata$2$far_MacroExecute  0000000180072074     service.obj
 0003:00001080       $pdata$3$far_MacroExecute  0000000180072080     service.obj
 0003:0000108c       $pdata$far_CPluginStartupInfo 000000018007208c     service.obj
 0003:00001098       $pdata$far_MakeMenuItems   0000000180072098     service.obj
 0003:000010a4       $pdata$1$far_MakeMenuItems 00000001800720a4     service.obj
 0003:000010b0       $pdata$5$far_MakeMenuItems 00000001800720b0     service.obj
 0003:000010bc       $pdata$6$far_MakeMenuItems 00000001800720bc     service.obj
 0003:000010c8       $pdata$8$far_MakeMenuItems 00000001800720c8     service.obj
 0003:000010d4       $pdata$9$far_MakeMenuItems 00000001800720d4     service.obj
 0003:000010e0       $pdata$far_Show            00000001800720e0     service.obj
 0003:000010ec       $pdata$far_CreateFileFilter 00000001800720ec     service.obj
 0003:000010f8       $pdata$filefilter_Free     00000001800720f8     service.obj
 0003:00001104       $pdata$filefilter_gc       0000000180072104     service.obj
 0003:00001110       $pdata$filefilter_tostring 0000000180072110     service.obj
 0003:0000111c       $pdata$filefilter_OpenMenu 000000018007211c     service.obj
 0003:00001128       $pdata$filefilter_Starting 0000000180072128     service.obj
 0003:00001134       $pdata$filefilter_IsFileInFilter 0000000180072134     service.obj
 0003:00001140       $pdata$far_UnloadPlugin    0000000180072140     service.obj
 0003:0000114c       $pdata$far_FindPlugin      000000018007214c     service.obj
 0003:00001158       $pdata$far_GetPluginInformation 0000000180072158     service.obj
 0003:00001164       $pdata$far_GetPlugins      0000000180072164     service.obj
 0003:00001170       $pdata$1$far_GetPlugins    0000000180072170     service.obj
 0003:0000117c       $pdata$2$far_GetPlugins    000000018007217c     service.obj
 0003:00001188       $pdata$3$far_GetPlugins    0000000180072188     service.obj
 0003:00001194       $pdata$4$far_GetPlugins    0000000180072194     service.obj
 0003:000011a0       $pdata$far_IsPluginLoaded  00000001800721a0     service.obj
 0003:000011ac       $pdata$0$far_IsPluginLoaded 00000001800721ac     service.obj
 0003:000011b8       $pdata$1$far_IsPluginLoaded 00000001800721b8     service.obj
 0003:000011c4       $pdata$far_XLat            00000001800721c4     service.obj
 0003:000011d0       $pdata$far_FormatFileSize  00000001800721d0     service.obj
 0003:000011dc       $pdata$far_FarClock        00000001800721dc     service.obj
 0003:000011e8       $pdata$far_Timer           00000001800721e8     service.obj
 0003:000011f4       $pdata$timer_gc            00000001800721f4     service.obj
 0003:00001200       $pdata$0$timer_gc          0000000180072200     service.obj
 0003:0000120c       $pdata$1$timer_gc          000000018007220c     service.obj
 0003:00001218       $pdata$timer_tostring      0000000180072218     service.obj
 0003:00001224       $pdata$timer_index         0000000180072224     service.obj
 0003:00001230       $pdata$timer_newindex      0000000180072230     service.obj
 0003:0000123c       $pdata$far_CreateSettings  000000018007223c     service.obj
 0003:00001248       $pdata$Settings_set        0000000180072248     service.obj
 0003:00001254       $pdata$Settings_get        0000000180072254     service.obj
 0003:00001260       $pdata$Settings_delete     0000000180072260     service.obj
 0003:0000126c       $pdata$Settings_createsubkey 000000018007226c     service.obj
 0003:00001278       $pdata$Settings_opensubkey 0000000180072278     service.obj
 0003:00001284       $pdata$Settings_enum       0000000180072284     service.obj
 0003:00001290       $pdata$2$Settings_enum     0000000180072290     service.obj
 0003:0000129c       $pdata$4$Settings_enum     000000018007229c     service.obj
 0003:000012a8       $pdata$5$Settings_enum     00000001800722a8     service.obj
 0003:000012b4       $pdata$Settings_free       00000001800722b4     service.obj
 0003:000012c0       $pdata$far_FreeSettings    00000001800722c0     service.obj
 0003:000012cc       $pdata$Settings_tostring   00000001800722cc     service.obj
 0003:000012d8       $pdata$far_ColorDialog     00000001800722d8     service.obj
 0003:000012e4       $pdata$far_RunDefaultScript 00000001800722e4     service.obj
 0003:000012f0       $pdata$far_FileTimeResolution 00000001800722f0     service.obj
 0003:000012fc       $pdata$AddMacroData_gc     00000001800722fc     service.obj
 0003:00001308       $pdata$ChangePanelSelection 0000000180072308     service.obj
 0003:00001314       $pdata$1$ChangePanelSelection 0000000180072314     service.obj
 0003:00001320       $pdata$2$ChangePanelSelection 0000000180072320     service.obj
 0003:0000132c       $pdata$CheckFlagsFromTable 000000018007232c     service.obj
 0003:00001338       $pdata$ConvertLuaValue     0000000180072338     service.obj
 0003:00001344       $pdata$CreateList          0000000180072344     service.obj
 0003:00001350       $pdata$2$CreateList        0000000180072350     service.obj
 0003:0000135c       $pdata$3$CreateList        000000018007235c     service.obj
 0003:00001368       $pdata$DeleteLuaStateTimerQueue 0000000180072368     service.obj
 0003:00001374       $pdata$DialogHandleEqual   0000000180072374     service.obj
 0003:00001380       $pdata$DllMain             0000000180072380     service.obj
 0003:0000138c       $pdata$0$DllMain           000000018007238c     service.obj
 0003:00001398       $pdata$1$DllMain           0000000180072398     service.obj
 0003:000013a4       $pdata$FillEditorSelect    00000001800723a4     service.obj
 0003:000013b0       $pdata$FillEditorSetPosition 00000001800723b0     service.obj
 0003:000013bc       $pdata$FillInputRecord     00000001800723bc     service.obj
 0003:000013c8       $pdata$FillKeyBarTitles    00000001800723c8     service.obj
 0003:000013d4       $pdata$1$FillKeyBarTitles  00000001800723d4     service.obj
 0003:000013e0       $pdata$2$FillKeyBarTitles  00000001800723e0     service.obj
 0003:000013ec       $pdata$FrsUserFunc         00000001800723ec     service.obj
 0003:000013f8       $pdata$GetFarColor         00000001800723f8     service.obj
 0003:00001404       $pdata$0$GetFarColor       0000000180072404     service.obj
 0003:00001410       $pdata$1$GetFarColor       0000000180072410     service.obj
 0003:0000141c       $pdata$GetFlagCombination  000000018007241c     service.obj
 0003:00001428       $pdata$GetFlagsFromTable   0000000180072428     service.obj
 0003:00001434       $pdata$GetLuaStateTimerQueue 0000000180072434     service.obj
 0003:00001440       $pdata$GetPluginData       0000000180072440     service.obj
 0003:0000144c       $pdata$LF_DlgProc          000000018007244c     service.obj
 0003:00001458       $pdata$1$LF_DlgProc        0000000180072458     service.obj
 0003:00001464       $pdata$2$LF_DlgProc        0000000180072464     service.obj
 0003:00001470       $pdata$LF_DoFile           0000000180072470     service.obj
 0003:0000147c       $pdata$LF_Error            000000018007247c     service.obj
 0003:00001488       $pdata$LF_GetLuafarAPI     0000000180072488     service.obj
 0003:00001494       $pdata$LF_InitLuaState1    0000000180072494     service.obj
 0003:000014a0       $pdata$LF_InitLuaState2    00000001800724a0     service.obj
 0003:000014ac       $pdata$LF_Message          00000001800724ac     service.obj
 0003:000014b8       $pdata$LF_RunLuafarInit    00000001800724b8     service.obj
 0003:000014c4       $pdata$MacroAddCallback    00000001800724c4     service.obj
 0003:000014d0       $pdata$MacroSendString     00000001800724d0     service.obj
 0003:000014dc       $pdata$NewDialogData       00000001800724dc     service.obj
 0003:000014e8       $pdata$NewVirtualKeyTable  00000001800724e8     service.obj
 0003:000014f4       $pdata$OptFlags            00000001800724f4     service.obj
 0003:00001500       $pdata$OptHandle           0000000180072500     service.obj
 0003:0000150c       $pdata$OptInputRecord      000000018007250c     service.obj
 0003:00001518       $pdata$PluginHandle_rawhandle 0000000180072518     service.obj
 0003:00001524       $pdata$ProcessDNResult     0000000180072524     service.obj
 0003:00001530       $pdata$0$ProcessDNResult   0000000180072530     service.obj
 0003:0000153c       $pdata$1$ProcessDNResult   000000018007253c     service.obj
 0003:00001548       $pdata$PushBookmarks       0000000180072548     service.obj
 0003:00001554       $pdata$0$PushBookmarks     0000000180072554     service.obj
 0003:00001560       $pdata$1$PushBookmarks     0000000180072560     service.obj
 0003:0000156c       $pdata$PushDMParams        000000018007256c     service.obj
 0003:00001578       $pdata$PushDNParams        0000000180072578     service.obj
 0003:00001584       $pdata$PushDlgItem         0000000180072584     service.obj
 0003:00001590       $pdata$1$PushDlgItem       0000000180072590     service.obj
 0003:0000159c       $pdata$2$PushDlgItem       000000018007259c     service.obj
 0003:000015a8       $pdata$PushDlgItemNum      00000001800725a8     service.obj
 0003:000015b4       $pdata$PushFarColor        00000001800725b4     service.obj
 0003:000015c0       $pdata$PushInputRecord     00000001800725c0     service.obj
 0003:000015cc       $pdata$PushPanelItem       00000001800725cc     service.obj
 0003:000015d8       $pdata$0$PushPanelItem     00000001800725d8     service.obj
 0003:000015e4       $pdata$1$PushPanelItem     00000001800725e4     service.obj
 0003:000015f0       $pdata$3$PushPanelItem     00000001800725f0     service.obj
 0003:000015fc       $pdata$4$PushPanelItem     00000001800725fc     service.obj
 0003:00001608       $pdata$PushPanelItems      0000000180072608     service.obj
 0003:00001614       $pdata$3$PushPanelItems    0000000180072614     service.obj
 0003:00001620       $pdata$4$PushPanelItems    0000000180072620     service.obj
 0003:0000162c       $pdata$PushPluginHandle    000000018007262c     service.obj
 0003:00001638       $pdata$PutFlagsToTable     0000000180072638     service.obj
 0003:00001644       $pdata$PutPluginMenuItemToTable 0000000180072644     service.obj
 0003:00001650       $pdata$0$PutPluginMenuItemToTable 0000000180072650     service.obj
 0003:0000165c       $pdata$1$PutPluginMenuItemToTable 000000018007265c     service.obj
 0003:00001668       $pdata$PutVersionInfoToTable 0000000180072668     service.obj
 0003:00001674       $pdata$SetDlgItem          0000000180072674     service.obj
 0003:00001680       $pdata$SetFarDialogItem    0000000180072680     service.obj
 0003:0000168c       $pdata$SetKeyBar           000000018007268c     service.obj
 0003:00001698       $pdata$SetPanelBooleanProperty 0000000180072698     service.obj
 0003:000016a4       $pdata$SetPanelIntegerProperty 00000001800726a4     service.obj
 0003:000016b0       $pdata$TimerCallback       00000001800726b0     service.obj
 0003:000016bc       $pdata$_EditorGetString    00000001800726bc     service.obj
 0003:000016c8       $pdata$_EditorInsertText   00000001800726c8     service.obj
 0003:000016d4       $pdata$_EditorSetString    00000001800726d4     service.obj
 0003:000016e0       $pdata$_EditorTabConvert   00000001800726e0     service.obj
 0003:000016ec       $pdata$check_env_flag      00000001800726ec     service.obj
 0003:000016f8       $pdata$dir_exist           00000001800726f8     service.obj
 0003:00001704       $pdata$fprintf             0000000180072704     service.obj
 0003:00001710       $pdata$free_dialog         0000000180072710     service.obj
 0003:0000171c       $pdata$get_env_flag        000000018007271c     service.obj
 0003:00001728       $pdata$get_panel_item      0000000180072728     service.obj
 0003:00001734       $pdata$get_string_info     0000000180072734     service.obj
 0003:00001740       $pdata$luaopen_far         0000000180072740     service.obj
 0003:0000174c       $pdata$luaopen_luafar3     000000018007274c     service.obj
 0003:00001758       $pdata$plugin_load         0000000180072758     service.obj
 0003:00001764       $pdata$pushFileTime        0000000180072764     service.obj
 0003:00001770       $pdata$timer_Close         0000000180072770     service.obj
 0003:0000177c       $pdata$0$timer_Close       000000018007277c     service.obj
 0003:00001788       $pdata$1$timer_Close       0000000180072788     service.obj
 0003:00001794       $pdata$truncstring         0000000180072794     service.obj
 0003:000017a0       $pdata$str_rep             00000001800727a0     slnunico.obj
 0003:000017ac       $pdata$str_dump            00000001800727ac     slnunico.obj
 0003:000017b8       $pdata$str_format          00000001800727b8     slnunico.obj
 0003:000017c4       $pdata$utf8_valid          00000001800727c4     slnunico.obj
 0003:000017d0       $pdata$_snwprintf          00000001800727d0     slnunico.obj
 0003:000017dc       $pdata$luaopen_unicode     00000001800727dc     slnunico.obj
 0003:000017e8       $pdata$writer              00000001800727e8     slnunico.obj
 0003:000017f4       $pdata$Lutf8_byte          00000001800727f4     lutf8lib.obj
 0003:00001800       $pdata$Lutf8_char          0000000180072800     lutf8lib.obj
 0003:0000180c       $pdata$0$Lutf8_char        000000018007280c     lutf8lib.obj
 0003:00001818       $pdata$1$Lutf8_char        0000000180072818     lutf8lib.obj
 0003:00001824       $pdata$Lutf8_charpos       0000000180072824     lutf8lib.obj
 0003:00001830       $pdata$Lutf8_codepoint     0000000180072830     lutf8lib.obj
 0003:0000183c       $pdata$Lutf8_codes         000000018007283c     lutf8lib.obj
 0003:00001848       $pdata$Lutf8_escape        0000000180072848     lutf8lib.obj
 0003:00001854       $pdata$3$Lutf8_escape      0000000180072854     lutf8lib.obj
 0003:00001860       $pdata$4$Lutf8_escape      0000000180072860     lutf8lib.obj
 0003:0000186c       $pdata$Lutf8_gmatch        000000018007286c     lutf8lib.obj
 0003:00001878       $pdata$Lutf8_gsub          0000000180072878     lutf8lib.obj
 0003:00001884       $pdata$Lutf8_insert        0000000180072884     lutf8lib.obj
 0003:00001890       $pdata$Lutf8_len           0000000180072890     lutf8lib.obj
 0003:0000189c       $pdata$Lutf8_ncasecmp      000000018007289c     lutf8lib.obj
 0003:000018a8       $pdata$Lutf8_next          00000001800728a8     lutf8lib.obj
 0003:000018b4       $pdata$Lutf8_offset        00000001800728b4     lutf8lib.obj
 0003:000018c0       $pdata$Lutf8_remove        00000001800728c0     lutf8lib.obj
 0003:000018cc       $pdata$Lutf8_reverse       00000001800728cc     lutf8lib.obj
 0003:000018d8       $pdata$Lutf8_sub           00000001800728d8     lutf8lib.obj
 0003:000018e4       $pdata$Lutf8_width         00000001800728e4     lutf8lib.obj
 0003:000018f0       $pdata$0$Lutf8_width       00000001800728f0     lutf8lib.obj
 0003:000018fc       $pdata$1$Lutf8_width       00000001800728fc     lutf8lib.obj
 0003:00001908       $pdata$Lutf8_widthindex    0000000180072908     lutf8lib.obj
 0003:00001914       $pdata$add_utf8char        0000000180072914     lutf8lib.obj
 0003:00001920       $pdata$add_value           0000000180072920     lutf8lib.obj
 0003:0000192c       $pdata$1$add_value         000000018007292c     lutf8lib.obj
 0003:00001938       $pdata$2$add_value         0000000180072938     lutf8lib.obj
 0003:00001944       $pdata$3$add_value         0000000180072944     lutf8lib.obj
 0003:00001950       $pdata$4$add_value         0000000180072950     lutf8lib.obj
 0003:0000195c       $pdata$classend            000000018007295c     lutf8lib.obj
 0003:00001968       $pdata$convert             0000000180072968     lutf8lib.obj
 0003:00001974       $pdata$find_aux            0000000180072974     lutf8lib.obj
 0003:00001980       $pdata$gmatch_aux          0000000180072980     lutf8lib.obj
 0003:0000198c       $pdata$luaopen_utf8        000000018007298c     lutf8lib.obj
 0003:00001998       $pdata$match               0000000180072998     lutf8lib.obj
 0003:000019a4       $pdata$3$match             00000001800729a4     lutf8lib.obj
 0003:000019b0       $pdata$4$match             00000001800729b0     lutf8lib.obj
 0003:000019bc       $pdata$match_class         00000001800729bc     lutf8lib.obj
 0003:000019c8       $pdata$matchbalance        00000001800729c8     lutf8lib.obj
 0003:000019d4       $pdata$1$matchbalance      00000001800729d4     lutf8lib.obj
 0003:000019e0       $pdata$2$matchbalance      00000001800729e0     lutf8lib.obj
 0003:000019ec       $pdata$matchbracketclass   00000001800729ec     lutf8lib.obj
 0003:000019f8       $pdata$push_captures       00000001800729f8     lutf8lib.obj
 0003:00001a04       $pdata$2$push_captures     0000000180072a04     lutf8lib.obj
 0003:00001a10       $pdata$3$push_captures     0000000180072a10     lutf8lib.obj
 0003:00001a1c       $pdata$push_offset         0000000180072a1c     lutf8lib.obj
 0003:00001a28       $pdata$push_onecapture     0000000180072a28     lutf8lib.obj
 0003:00001a34       $pdata$3$push_onecapture   0000000180072a34     lutf8lib.obj
 0003:00001a40       $pdata$5$push_onecapture   0000000180072a40     lutf8lib.obj
 0003:00001a4c       $pdata$singlematch         0000000180072a4c     lutf8lib.obj
 0003:00001a58       $pdata$start_capture       0000000180072a58     lutf8lib.obj
 0003:00001a64       $pdata$utf8_index          0000000180072a64     lutf8lib.obj
 0003:00001a70       $pdata$utf8_isdigit        0000000180072a70     lutf8lib.obj
 0003:00001a7c       $pdata$utf8_isgraph        0000000180072a7c     lutf8lib.obj
 0003:00001a88       $pdata$utf8_islower        0000000180072a88     lutf8lib.obj
 0003:00001a94       $pdata$utf8_length         0000000180072a94     lutf8lib.obj
 0003:00001aa0       $pdata$utf8_width          0000000180072aa0     lutf8lib.obj
 0003:00001aac       $pdata$io_type             0000000180072aac     uliolib51.obj
 0003:00001ab8       $pdata$io_close            0000000180072ab8     uliolib51.obj
 0003:00001ac4       $pdata$io_gc               0000000180072ac4     uliolib51.obj
 0003:00001ad0       $pdata$io_tostring         0000000180072ad0     uliolib51.obj
 0003:00001adc       $pdata$io_open             0000000180072adc     uliolib51.obj
 0003:00001ae8       $pdata$io_popen            0000000180072ae8     uliolib51.obj
 0003:00001af4       $pdata$io_tmpfile          0000000180072af4     uliolib51.obj
 0003:00001b00       $pdata$f_lines             0000000180072b00     uliolib51.obj
 0003:00001b0c       $pdata$io_lines            0000000180072b0c     uliolib51.obj
 0003:00001b18       $pdata$1$io_lines          0000000180072b18     uliolib51.obj
 0003:00001b24       $pdata$2$io_lines          0000000180072b24     uliolib51.obj
 0003:00001b30       $pdata$io_read             0000000180072b30     uliolib51.obj
 0003:00001b3c       $pdata$f_read              0000000180072b3c     uliolib51.obj
 0003:00001b48       $pdata$io_write            0000000180072b48     uliolib51.obj
 0003:00001b54       $pdata$f_write             0000000180072b54     uliolib51.obj
 0003:00001b60       $pdata$f_seek              0000000180072b60     uliolib51.obj
 0003:00001b6c       $pdata$f_setvbuf           0000000180072b6c     uliolib51.obj
 0003:00001b78       $pdata$io_flush            0000000180072b78     uliolib51.obj
 0003:00001b84       $pdata$f_flush             0000000180072b84     uliolib51.obj
 0003:00001b90       $pdata$aux_close           0000000180072b90     uliolib51.obj
 0003:00001b9c       $pdata$fileerror           0000000180072b9c     uliolib51.obj
 0003:00001ba8       $pdata$fscanf              0000000180072ba8     uliolib51.obj
 0003:00001bb4       $pdata$g_iofile            0000000180072bb4     uliolib51.obj
 0003:00001bc0       $pdata$0$g_iofile          0000000180072bc0     uliolib51.obj
 0003:00001bcc       $pdata$1$g_iofile          0000000180072bcc     uliolib51.obj
 0003:00001bd8       $pdata$2$g_iofile          0000000180072bd8     uliolib51.obj
 0003:00001be4       $pdata$3$g_iofile          0000000180072be4     uliolib51.obj
 0003:00001bf0       $pdata$g_read              0000000180072bf0     uliolib51.obj
 0003:00001bfc       $pdata$g_write             0000000180072bfc     uliolib51.obj
 0003:00001c08       $pdata$io_fclose           0000000180072c08     uliolib51.obj
 0003:00001c14       $pdata$io_noclose          0000000180072c14     uliolib51.obj
 0003:00001c20       $pdata$io_pclose           0000000180072c20     uliolib51.obj
 0003:00001c2c       $pdata$io_readline         0000000180072c2c     uliolib51.obj
 0003:00001c38       $pdata$luaopen_uio         0000000180072c38     uliolib51.obj
 0003:00001c44       $pdata$newfile             0000000180072c44     uliolib51.obj
 0003:00001c50       $pdata$pushresult          0000000180072c50     uliolib51.obj
 0003:00001c5c       $pdata$read_chars          0000000180072c5c     uliolib51.obj
 0003:00001c68       $pdata$read_line           0000000180072c68     uliolib51.obj
 0003:00001c74       $pdata$ll_loadlib          0000000180072c74     uloadlib51.obj
 0003:00001c80       $pdata$loader_Lua          0000000180072c80     uloadlib51.obj
 0003:00001c8c       $pdata$loader_C            0000000180072c8c     uloadlib51.obj
 0003:00001c98       $pdata$loader_Croot        0000000180072c98     uloadlib51.obj
 0003:00001ca4       $pdata$loader_preload      0000000180072ca4     uloadlib51.obj
 0003:00001cb0       $pdata$ll_require          0000000180072cb0     uloadlib51.obj
 0003:00001cbc       $pdata$ll_module           0000000180072cbc     uloadlib51.obj
 0003:00001cc8       $pdata$0$ll_module         0000000180072cc8     uloadlib51.obj
 0003:00001cd4       $pdata$1$ll_module         0000000180072cd4     uloadlib51.obj
 0003:00001ce0       $pdata$ll_seeall           0000000180072ce0     uloadlib51.obj
 0003:00001cec       $pdata$findfile            0000000180072cec     uloadlib51.obj
 0003:00001cf8       $pdata$gctm                0000000180072cf8     uloadlib51.obj
 0003:00001d04       $pdata$ll_loadfunc         0000000180072d04     uloadlib51.obj
 0003:00001d10       $pdata$loaderror           0000000180072d10     uloadlib51.obj
 0003:00001d1c       $pdata$luaopen_upackage    0000000180072d1c     uloadlib51.obj
 0003:00001d28       $pdata$mkfuncname          0000000180072d28     uloadlib51.obj
 0003:00001d34       $pdata$setpath             0000000180072d34     uloadlib51.obj
 0003:00001d40       $pdata$ustring_WideCharToMultiByte 0000000180072d40     ustring.obj
 0003:00001d4c       $pdata$1$ustring_WideCharToMultiByte 0000000180072d4c     ustring.obj
 0003:00001d58       $pdata$2$ustring_WideCharToMultiByte 0000000180072d58     ustring.obj
 0003:00001d64       $pdata$ustring_MultiByteToWideChar 0000000180072d64     ustring.obj
 0003:00001d70       $pdata$ustring_OemToUtf8   0000000180072d70     ustring.obj
 0003:00001d7c       $pdata$1$ustring_OemToUtf8 0000000180072d7c     ustring.obj
 0003:00001d88       $pdata$2$ustring_OemToUtf8 0000000180072d88     ustring.obj
 0003:00001d94       $pdata$ustring_Utf8ToOem   0000000180072d94     ustring.obj
 0003:00001da0       $pdata$ustring_Utf16ToUtf8 0000000180072da0     ustring.obj
 0003:00001dac       $pdata$ustring_Utf8ToUtf16 0000000180072dac     ustring.obj
 0003:00001db8       $pdata$0$ustring_Utf8ToUtf16 0000000180072db8     ustring.obj
 0003:00001dc4       $pdata$1$ustring_Utf8ToUtf16 0000000180072dc4     ustring.obj
 0003:00001dd0       $pdata$ustring_GetACP      0000000180072dd0     ustring.obj
 0003:00001ddc       $pdata$ustring_GetOEMCP    0000000180072ddc     ustring.obj
 0003:00001de8       $pdata$ustring_GetConsoleCP 0000000180072de8     ustring.obj
 0003:00001df4       $pdata$ustring_SetConsoleCP 0000000180072df4     ustring.obj
 0003:00001e00       $pdata$ustring_GetConsoleOutputCP 0000000180072e00     ustring.obj
 0003:00001e0c       $pdata$ustring_SetConsoleOutputCP 0000000180072e0c     ustring.obj
 0003:00001e18       $pdata$ustring_EnumSystemCodePages 0000000180072e18     ustring.obj
 0003:00001e24       $pdata$ustring_GetCPInfo   0000000180072e24     ustring.obj
 0003:00001e30       $pdata$ustring_GetLogicalDriveStrings 0000000180072e30     ustring.obj
 0003:00001e3c       $pdata$0$ustring_GetLogicalDriveStrings 0000000180072e3c     ustring.obj
 0003:00001e48       $pdata$1$ustring_GetLogicalDriveStrings 0000000180072e48     ustring.obj
 0003:00001e54       $pdata$ustring_GetDriveType 0000000180072e54     ustring.obj
 0003:00001e60       $pdata$ustring_Uuid        0000000180072e60     ustring.obj
 0003:00001e6c       $pdata$ustring_SearchPath  0000000180072e6c     ustring.obj
 0003:00001e78       $pdata$ustring_GlobalMemoryStatus 0000000180072e78     ustring.obj
 0003:00001e84       $pdata$0$ustring_GlobalMemoryStatus 0000000180072e84     ustring.obj
 0003:00001e90       $pdata$2$ustring_GlobalMemoryStatus 0000000180072e90     ustring.obj
 0003:00001e9c       $pdata$ustring_Sleep       0000000180072e9c     ustring.obj
 0003:00001ea8       $pdata$ustring_SetFileAttr 0000000180072ea8     ustring.obj
 0003:00001eb4       $pdata$2$ustring_SetFileAttr 0000000180072eb4     ustring.obj
 0003:00001ec0       $pdata$3$ustring_SetFileAttr 0000000180072ec0     ustring.obj
 0003:00001ecc       $pdata$4$ustring_SetFileAttr 0000000180072ecc     ustring.obj
 0003:00001ed8       $pdata$5$ustring_SetFileAttr 0000000180072ed8     ustring.obj
 0003:00001ee4       $pdata$ustring_GetFileAttr 0000000180072ee4     ustring.obj
 0003:00001ef0       $pdata$2$ustring_GetFileAttr 0000000180072ef0     ustring.obj
 0003:00001efc       $pdata$3$ustring_GetFileAttr 0000000180072efc     ustring.obj
 0003:00001f08       $pdata$ustring_SHGetFolderPath 0000000180072f08     ustring.obj
 0003:00001f14       $pdata$1$ustring_SHGetFolderPath 0000000180072f14     ustring.obj
 0003:00001f20       $pdata$2$ustring_SHGetFolderPath 0000000180072f20     ustring.obj
 0003:00001f2c       $pdata$ustring_sub         0000000180072f2c     ustring.obj
 0003:00001f38       $pdata$ustring_len         0000000180072f38     ustring.obj
 0003:00001f44       $pdata$ustring_OutputDebugString 0000000180072f44     ustring.obj
 0003:00001f50       $pdata$0$ustring_OutputDebugString 0000000180072f50     ustring.obj
 0003:00001f5c       $pdata$1$ustring_OutputDebugString 0000000180072f5c     ustring.obj
 0003:00001f68       $pdata$ustring_system      0000000180072f68     ustring.obj
 0003:00001f74       $pdata$ustring_GetCurrentDir 0000000180072f74     ustring.obj
 0003:00001f80       $pdata$0$ustring_GetCurrentDir 0000000180072f80     ustring.obj
 0003:00001f8c       $pdata$1$ustring_GetCurrentDir 0000000180072f8c     ustring.obj
 0003:00001f98       $pdata$2$ustring_GetCurrentDir 0000000180072f98     ustring.obj
 0003:00001fa4       $pdata$3$ustring_GetCurrentDir 0000000180072fa4     ustring.obj
 0003:00001fb0       $pdata$ustring_SetCurrentDir 0000000180072fb0     ustring.obj
 0003:00001fbc       $pdata$2$ustring_SetCurrentDir 0000000180072fbc     ustring.obj
 0003:00001fc8       $pdata$3$ustring_SetCurrentDir 0000000180072fc8     ustring.obj
 0003:00001fd4       $pdata$ustring_GetKeyState 0000000180072fd4     ustring.obj
 0003:00001fe0       $pdata$EnumCodePagesProc   0000000180072fe0     ustring.obj
 0003:00001fec       $pdata$GetBoolFromTable    0000000180072fec     ustring.obj
 0003:00001ff8       $pdata$GetOptBoolFromTable 0000000180072ff8     ustring.obj
 0003:00002004       $pdata$GetOptIntFromArray  0000000180073004     ustring.obj
 0003:00002010       $pdata$GetOptIntFromTable  0000000180073010     ustring.obj
 0003:0000201c       $pdata$GetOptNumFromTable  000000018007301c     ustring.obj
 0003:00002028       $pdata$PushAttrString      0000000180073028     ustring.obj
 0003:00002034       $pdata$PutAttrToTable      0000000180073034     ustring.obj
 0003:00002040       $pdata$PutBoolToTable      0000000180073040     ustring.obj
 0003:0000204c       $pdata$PutIntToArray       000000018007304c     ustring.obj
 0003:00002058       $pdata$PutIntToTable       0000000180073058     ustring.obj
 0003:00002064       $pdata$PutLStrToTable      0000000180073064     ustring.obj
 0003:00002070       $pdata$PutNumToTable       0000000180073070     ustring.obj
 0003:0000207c       $pdata$PutStrToArray       000000018007307c     ustring.obj
 0003:00002088       $pdata$PutStrToTable       0000000180073088     ustring.obj
 0003:00002094       $pdata$PutWStrToArray      0000000180073094     ustring.obj
 0003:000020a0       $pdata$PutWStrToTable      00000001800730a0     ustring.obj
 0003:000020ac       $pdata$SysErrorReturn      00000001800730ac     ustring.obj
 0003:000020b8       $pdata$check_utf16_string  00000001800730b8     ustring.obj
 0003:000020c4       $pdata$check_utf8_string   00000001800730c4     ustring.obj
 0003:000020d0       $pdata$convert_multibyte_string 00000001800730d0     ustring.obj
 0003:000020dc       $pdata$luaopen_ustring     00000001800730dc     ustring.obj
 0003:000020e8       $pdata$opt_utf8_string     00000001800730e8     ustring.obj
 0003:000020f4       $pdata$push_multibyte_string 00000001800730f4     ustring.obj
 0003:00002100       $pdata$2$push_multibyte_string 0000000180073100     ustring.obj
 0003:0000210c       $pdata$3$push_multibyte_string 000000018007310c     ustring.obj
 0003:00002118       $pdata$push_utf8_string    0000000180073118     ustring.obj
 0003:00002124       $pdata$pusherror           0000000180073124     ustring.obj
 0003:00002130       $pdata$pusherrorcode       0000000180073130     ustring.obj
 0003:0000213c       $pdata$utf8_to_utf16       000000018007313c     ustring.obj
 0003:00002148       $pdata$GetAttrFromTable    0000000180073148     util.obj
 0003:00002154       $pdata$GetFileSizeFromTable 0000000180073154     util.obj
 0003:00002160       $pdata$GetFileTimeFromTable 0000000180073160     util.obj
 0003:0000216c       $pdata$GetIntFromArray     000000018007316c     util.obj
 0003:00002178       $pdata$PutFileTimeToTable  0000000180073178     util.obj
 0003:00002184       $pdata$luaLF_FieldError    0000000180073184     util.obj
 0003:00002190       $pdata$luaLF_SlotError     0000000180073190     util.obj
 0003:0000219c       $pdata$win_GetEnv          000000018007319c     win.obj
 0003:000021a8       $pdata$0$win_GetEnv        00000001800731a8     win.obj
 0003:000021b4       $pdata$1$win_GetEnv        00000001800731b4     win.obj
 0003:000021c0       $pdata$win_SetEnv          00000001800731c0     win.obj
 0003:000021cc       $pdata$win_SetRegKey       00000001800731cc     win.obj
 0003:000021d8       $pdata$win_GetRegKey       00000001800731d8     win.obj
 0003:000021e4       $pdata$win_DeleteRegKey    00000001800731e4     win.obj
 0003:000021f0       $pdata$win_DeleteRegValue  00000001800731f0     win.obj
 0003:000021fc       $pdata$win_EnumRegKey      00000001800731fc     win.obj
 0003:00002208       $pdata$win_EnumRegValue    0000000180073208     win.obj
 0003:00002214       $pdata$win_ExtractKey      0000000180073214     win.obj
 0003:00002220       $pdata$win_ExtractKeyEx    0000000180073220     win.obj
 0003:0000222c       $pdata$win_GetFileInfo     000000018007322c     win.obj
 0003:00002238       $pdata$win_GetSystemTimeAsFileTime 0000000180073238     win.obj
 0003:00002244       $pdata$win_FileTimeToSystemTime 0000000180073244     win.obj
 0003:00002250       $pdata$win_SystemTimeToFileTime 0000000180073250     win.obj
 0003:0000225c       $pdata$win_FileTimeToLocalFileTime 000000018007325c     win.obj
 0003:00002268       $pdata$win_CompareString   0000000180073268     win.obj
 0003:00002274       $pdata$win_wcscmp          0000000180073274     win.obj
 0003:00002280       $pdata$win_GetVirtualKeys  0000000180073280     win.obj
 0003:0000228c       $pdata$win_GetConsoleScreenBufferInfo 000000018007328c     win.obj
 0003:00002298       $pdata$win_CopyFile        0000000180073298     win.obj
 0003:000022a4       $pdata$win_MoveFile        00000001800732a4     win.obj
 0003:000022b0       $pdata$win_DeleteFile      00000001800732b0     win.obj
 0003:000022bc       $pdata$win_CreateDir       00000001800732bc     win.obj
 0003:000022c8       $pdata$win_RemoveDir       00000001800732c8     win.obj
 0003:000022d4       $pdata$win_ShellExecute    00000001800732d4     win.obj
 0003:000022e0       $pdata$win_IsProcess64bit  00000001800732e0     win.obj
 0003:000022ec       $pdata$win_WriteConsole    00000001800732ec     win.obj
 0003:000022f8       $pdata$win_IsWinVersion    00000001800732f8     win.obj
 0003:00002304       $pdata$1$win_IsWinVersion  0000000180073304     win.obj
 0003:00002310       $pdata$2$win_IsWinVersion  0000000180073310     win.obj
 0003:0000231c       $pdata$CheckHKey           000000018007331c     win.obj
 0003:00002328       $pdata$luaopen_win         0000000180073328     win.obj
 0003:00002334       $pdata$mkdir               0000000180073334     win.obj
 0003:00002340       $pdata$0$mkdir             0000000180073340     win.obj
 0003:0000234c       $pdata$?dllmain_crt_dispatch@@YAHQEAUHINSTANCE__@@KQEAX@Z 000000018007334c     LIBCMT:dll_dllmain.obj
 0003:00002358       $pdata$?dllmain_crt_process_attach@@YAHQEAUHINSTANCE__@@QEAX@Z 0000000180073358     LIBCMT:dll_dllmain.obj
 0003:00002364       $pdata$?dllmain_crt_process_detach@@YAH_N@Z 0000000180073364     LIBCMT:dll_dllmain.obj
 0003:00002370       $pdata$?dllmain_dispatch@@YAHQEAUHINSTANCE__@@KQEAX@Z 0000000180073370     LIBCMT:dll_dllmain.obj
 0003:0000237c       $pdata$_DllMainCRTStartup  000000018007337c     LIBCMT:dll_dllmain.obj
 0003:00002388       $pdata$__security_init_cookie 0000000180073388     LIBCMT:gs_support.obj
 0003:00002394       $pdata$__scrt_initialize_default_local_stdio_options 0000000180073394     LIBCMT:default_local_stdio_options.obj
 0003:000023a0       $pdata$__scrt_acquire_startup_lock 00000001800733a0     LIBCMT:utility.obj
 0003:000023ac       $pdata$__scrt_dllmain_after_initialize_c 00000001800733ac     LIBCMT:utility.obj
 0003:000023b8       $pdata$__scrt_dllmain_before_initialize_c 00000001800733b8     LIBCMT:utility.obj
 0003:000023c4       $pdata$__scrt_dllmain_crt_thread_attach 00000001800733c4     LIBCMT:utility.obj
 0003:000023d0       $pdata$__scrt_dllmain_crt_thread_detach 00000001800733d0     LIBCMT:utility.obj
 0003:000023dc       $pdata$__scrt_dllmain_exception_filter 00000001800733dc     LIBCMT:utility.obj
 0003:000023e8       $pdata$__scrt_dllmain_uninitialize_c 00000001800733e8     LIBCMT:utility.obj
 0003:000023f4       $pdata$__scrt_dllmain_uninitialize_critical 00000001800733f4     LIBCMT:utility.obj
 0003:00002400       $pdata$__scrt_initialize_crt 0000000180073400     LIBCMT:utility.obj
 0003:0000240c       $pdata$__scrt_initialize_onexit_tables 000000018007340c     LIBCMT:utility.obj
 0003:00002418       $pdata$__scrt_is_nonwritable_in_current_image 0000000180073418     LIBCMT:utility.obj
 0003:00002424       $pdata$__scrt_release_startup_lock 0000000180073424     LIBCMT:utility.obj
 0003:00002430       $pdata$__scrt_uninitialize_crt 0000000180073430     LIBCMT:utility.obj
 0003:0000243c       $pdata$__scrt_fastfail     000000018007343c     LIBCMT:utility_desktop.obj
 0003:00002448       $pdata$_RTC_Initialize     0000000180073448     LIBCMT:initsect.obj
 0003:00002454       $pdata$_RTC_Terminate      0000000180073454     LIBCMT:initsect.obj
 0003:00002460       $pdata$__isa_available_init 0000000180073460     LIBCMT:cpu_disp.obj
 0003:0000249c       $pdata$wcsstr              000000018007349c     libvcruntime:wcsstr.obj
 0003:000024a8       $pdata$strchr              00000001800734a8     libvcruntime:strchr.obj
 0003:000024b4       $pdata$wcschr              00000001800734b4     libvcruntime:wcschr.obj
 0003:000024d8       $pdata$strrchr             00000001800734d8     libvcruntime:strrchr.obj
 0003:000024e4       $pdata$__C_specific_handler 00000001800734e4     libvcruntime:riscchandler.obj
 0003:000024f0       $pdata$__std_type_info_destroy_list 00000001800734f0     libvcruntime:std_type_info.obj
 0003:000024fc       $pdata$__vcrt_initialize   00000001800734fc     libvcruntime:initialization.obj
 0003:00002508       $pdata$__vcrt_thread_attach 0000000180073508     libvcruntime:initialization.obj
 0003:00002514       $pdata$__vcrt_thread_detach 0000000180073514     libvcruntime:initialization.obj
 0003:00002520       $pdata$__vcrt_uninitialize 0000000180073520     libvcruntime:initialization.obj
 0003:0000252c       $pdata$__vcrt_uninitialize_critical 000000018007352c     libvcruntime:initialization.obj
 0003:0000255c       $pdata$__DestructExceptionObject 000000018007355c     libvcruntime:ehhelpers.obj
 0003:00002568       $pdata$__vcrt_freefls      0000000180073568     libvcruntime:per_thread_data.obj
 0003:00002574       $pdata$__vcrt_freeptd      0000000180073574     libvcruntime:per_thread_data.obj
 0003:00002580       $pdata$__vcrt_getptd_noexit 0000000180073580     libvcruntime:per_thread_data.obj
 0003:0000258c       $pdata$__vcrt_initialize_ptd 000000018007358c     libvcruntime:per_thread_data.obj
 0003:00002598       $pdata$__vcrt_uninitialize_ptd 0000000180073598     libvcruntime:per_thread_data.obj
 0003:000025a4       $pdata$__vcrt_initialize_locks 00000001800735a4     libvcruntime:locks.obj
 0003:000025b0       $pdata$__vcrt_uninitialize_locks 00000001800735b0     libvcruntime:locks.obj
 0003:000025bc       $pdata$?try_get_function@@YAPEAXW4function_id@?A0x14c33c87@@QEBDQEBW4module_id@2@2@Z 00000001800735bc     libvcruntime:winapi_downlevel.obj
 0003:000025c8       $pdata$__vcrt_FlsAlloc     00000001800735c8     libvcruntime:winapi_downlevel.obj
 0003:000025d4       $pdata$__vcrt_FlsFree      00000001800735d4     libvcruntime:winapi_downlevel.obj
 0003:000025e0       $pdata$__vcrt_FlsGetValue  00000001800735e0     libvcruntime:winapi_downlevel.obj
 0003:000025ec       $pdata$__vcrt_FlsSetValue  00000001800735ec     libvcruntime:winapi_downlevel.obj
 0003:000025f8       $pdata$__vcrt_InitializeCriticalSectionEx 00000001800735f8     libvcruntime:winapi_downlevel.obj
 0003:00002604       $pdata$__vcrt_initialize_winapi_thunks 0000000180073604     libvcruntime:winapi_downlevel.obj
 0003:00002610       $pdata$__vcrt_uninitialize_winapi_thunks 0000000180073610     libvcruntime:winapi_downlevel.obj
 0003:00002634       $pdata$??$?RV<lambda_a62c933ada0517137acf5807a1eeac1f>@@AEAV<lambda_a31071773b9a94e445cbd5d04ef99106>@@V<lambda_56065050dbf3ada7e59a83db45153de3>@@@?$__crt_seh_guarded_call@H@@QEAAH$$QEAV<lambda_a62c933ada0517137acf5807a1eeac1f>@@AEAV<lambda_a31071773b9a94e445cbd5d04ef99106>@@$$QEAV<lambda_56065050dbf3ada7e59a83db45153de3>@@@Z 0000000180073634     libucrt:output.obj
 0003:00002640       $pdata$??$common_vsprintf@Vstandard_base@__crt_stdio_output@@D@@YAH_KQEAD0QEBDQEAU__crt_locale_pointers@@1@Z 0000000180073640     libucrt:output.obj
 0003:0000264c       $pdata$??$common_vsprintf@Vstandard_base@__crt_stdio_output@@_W@@YAH_KQEA_W0QEB_WQEAU__crt_locale_pointers@@QEAD@Z 000000018007364c     libucrt:output.obj
 0003:00002658       $pdata$??$ensure_buffer_is_big_enough@D@formatting_buffer@__crt_stdio_output@@QEAA_N_K@Z 0000000180073658     libucrt:output.obj
 0003:00002664       $pdata$??$ensure_buffer_is_big_enough@_W@formatting_buffer@__crt_stdio_output@@QEAA_N_K@Z 0000000180073664     libucrt:output.obj
 0003:00002670       $pdata$??$type_case_integer_parse_into_buffer@I@?$output_processor@DV?$string_output_adapter@D@__crt_stdio_output@@V?$standard_base@DV?$string_output_adapter@D@__crt_stdio_output@@@2@@__crt_stdio_output@@AEAAXII_N@Z 0000000180073670     libucrt:output.obj
 0003:00002670       $pdata$??$type_case_integer_parse_into_buffer@I@?$output_processor@DV?$stream_output_adapter@D@__crt_stdio_output@@V?$standard_base@DV?$stream_output_adapter@D@__crt_stdio_output@@@2@@__crt_stdio_output@@AEAAXII_N@Z 0000000180073670     libucrt:output.obj
 0003:0000267c       $pdata$??$type_case_integer_parse_into_buffer@I@?$output_processor@_WV?$string_output_adapter@_W@__crt_stdio_output@@V?$standard_base@_WV?$string_output_adapter@_W@__crt_stdio_output@@@2@@__crt_stdio_output@@AEAAXII_N@Z 000000018007367c     libucrt:output.obj
 0003:00002688       $pdata$??$type_case_integer_parse_into_buffer@_K@?$output_processor@DV?$stream_output_adapter@D@__crt_stdio_output@@V?$standard_base@DV?$stream_output_adapter@D@__crt_stdio_output@@@2@@__crt_stdio_output@@AEAAX_KI_N@Z 0000000180073688     libucrt:output.obj
 0003:00002688       $pdata$??$type_case_integer_parse_into_buffer@_K@?$output_processor@DV?$string_output_adapter@D@__crt_stdio_output@@V?$standard_base@DV?$string_output_adapter@D@__crt_stdio_output@@@2@@__crt_stdio_output@@AEAAX_KI_N@Z 0000000180073688     libucrt:output.obj
 0003:00002694       $pdata$??$type_case_integer_parse_into_buffer@_K@?$output_processor@_WV?$string_output_adapter@_W@__crt_stdio_output@@V?$standard_base@_WV?$string_output_adapter@_W@__crt_stdio_output@@@2@@__crt_stdio_output@@AEAAX_KI_N@Z 0000000180073694     libucrt:output.obj
 0003:000026a0       $pdata$??$write_multiple_characters@V?$stream_output_adapter@D@__crt_stdio_output@@D@__crt_stdio_output@@YAXAEBV?$stream_output_adapter@D@0@DHQEAH@Z 00000001800736a0     libucrt:output.obj
 0003:000026ac       $pdata$??$write_multiple_characters@V?$string_output_adapter@D@__crt_stdio_output@@D@__crt_stdio_output@@YAXAEBV?$string_output_adapter@D@0@DHQEAH@Z 00000001800736ac     libucrt:output.obj
 0003:000026b8       $pdata$??$write_multiple_characters@V?$string_output_adapter@_W@__crt_stdio_output@@D@__crt_stdio_output@@YAXAEBV?$string_output_adapter@_W@0@DHQEAH@Z 00000001800736b8     libucrt:output.obj
 0003:000026c4       $pdata$??0_LocaleUpdate@@QEAA@QEAU__crt_locale_pointers@@@Z 00000001800736c4     libucrt:output.obj
 0003:000026d0       $pdata$??R<lambda_a31071773b9a94e445cbd5d04ef99106>@@QEBAHXZ 00000001800736d0     libucrt:output.obj
 0003:000026dc       $pdata$?force_decimal_point@__crt_stdio_output@@YAXPEADQEAU__crt_locale_pointers@@@Z 00000001800736dc     libucrt:output.obj
 0003:000026e8       $pdata$?parse_int_from_format_string@?$output_processor@DV?$string_output_adapter@D@__crt_stdio_output@@V?$standard_base@DV?$string_output_adapter@D@__crt_stdio_output@@@2@@__crt_stdio_output@@AEAA_NQEAH@Z 00000001800736e8     libucrt:output.obj
 0003:000026e8       $pdata$?parse_int_from_format_string@?$output_processor@DV?$stream_output_adapter@D@__crt_stdio_output@@V?$standard_base@DV?$stream_output_adapter@D@__crt_stdio_output@@@2@@__crt_stdio_output@@AEAA_NQEAH@Z 00000001800736e8     libucrt:output.obj
 0003:000026f4       $pdata$?parse_int_from_format_string@?$output_processor@_WV?$string_output_adapter@_W@__crt_stdio_output@@V?$standard_base@_WV?$string_output_adapter@_W@__crt_stdio_output@@@2@@__crt_stdio_output@@AEAA_NQEAH@Z 00000001800736f4     libucrt:output.obj
 0003:00002700       $pdata$?process@?$output_processor@DV?$stream_output_adapter@D@__crt_stdio_output@@V?$standard_base@DV?$stream_output_adapter@D@__crt_stdio_output@@@2@@__crt_stdio_output@@QEAAHXZ 0000000180073700     libucrt:output.obj
 0003:0000270c       $pdata$?process@?$output_processor@DV?$string_output_adapter@D@__crt_stdio_output@@V?$standard_base@DV?$string_output_adapter@D@__crt_stdio_output@@@2@@__crt_stdio_output@@QEAAHXZ 000000018007370c     libucrt:output.obj
 0003:00002718       $pdata$?process@?$output_processor@_WV?$string_output_adapter@_W@__crt_stdio_output@@V?$standard_base@_WV?$string_output_adapter@_W@__crt_stdio_output@@@2@@__crt_stdio_output@@QEAAHXZ 0000000180073718     libucrt:output.obj
 0003:00002724       $pdata$?state_case_normal@?$output_processor@DV?$stream_output_adapter@D@__crt_stdio_output@@V?$standard_base@DV?$stream_output_adapter@D@__crt_stdio_output@@@2@@__crt_stdio_output@@AEAA_NXZ 0000000180073724     libucrt:output.obj
 0003:00002730       $pdata$?state_case_normal@?$output_processor@DV?$string_output_adapter@D@__crt_stdio_output@@V?$standard_base@DV?$string_output_adapter@D@__crt_stdio_output@@@2@@__crt_stdio_output@@AEAA_NXZ 0000000180073730     libucrt:output.obj
 0003:0000273c       $pdata$?state_case_normal_tchar@?$output_processor@DV?$stream_output_adapter@D@__crt_stdio_output@@V?$standard_base@DV?$stream_output_adapter@D@__crt_stdio_output@@@2@@__crt_stdio_output@@AEAA_ND@Z 000000018007373c     libucrt:output.obj
 0003:00002748       $pdata$?state_case_normal_tchar@?$output_processor@DV?$string_output_adapter@D@__crt_stdio_output@@V?$standard_base@DV?$string_output_adapter@D@__crt_stdio_output@@@2@@__crt_stdio_output@@AEAA_ND@Z 0000000180073748     libucrt:output.obj
 0003:00002754       $pdata$?state_case_size@?$output_processor@DV?$stream_output_adapter@D@__crt_stdio_output@@V?$standard_base@DV?$stream_output_adapter@D@__crt_stdio_output@@@2@@__crt_stdio_output@@AEAA_NXZ 0000000180073754     libucrt:output.obj
 0003:00002760       $pdata$?state_case_size@?$output_processor@DV?$string_output_adapter@D@__crt_stdio_output@@V?$standard_base@DV?$string_output_adapter@D@__crt_stdio_output@@@2@@__crt_stdio_output@@AEAA_NXZ 0000000180073760     libucrt:output.obj
 0003:0000276c       $pdata$?state_case_size@?$output_processor@_WV?$string_output_adapter@_W@__crt_stdio_output@@V?$standard_base@_WV?$string_output_adapter@_W@__crt_stdio_output@@@2@@__crt_stdio_output@@AEAA_NXZ 000000018007376c     libucrt:output.obj
 0003:00002778       $pdata$?state_case_type@?$output_processor@DV?$stream_output_adapter@D@__crt_stdio_output@@V?$standard_base@DV?$stream_output_adapter@D@__crt_stdio_output@@@2@@__crt_stdio_output@@AEAA_NXZ 0000000180073778     libucrt:output.obj
 0003:00002784       $pdata$?state_case_type@?$output_processor@DV?$string_output_adapter@D@__crt_stdio_output@@V?$standard_base@DV?$string_output_adapter@D@__crt_stdio_output@@@2@@__crt_stdio_output@@AEAA_NXZ 0000000180073784     libucrt:output.obj
 0003:00002790       $pdata$?state_case_type@?$output_processor@_WV?$string_output_adapter@_W@__crt_stdio_output@@V?$standard_base@_WV?$string_output_adapter@_W@__crt_stdio_output@@@2@@__crt_stdio_output@@AEAA_NXZ 0000000180073790     libucrt:output.obj
 0003:0000279c       $pdata$?type_case_Z@?$output_processor@_WV?$string_output_adapter@_W@__crt_stdio_output@@V?$standard_base@_WV?$string_output_adapter@_W@__crt_stdio_output@@@2@@__crt_stdio_output@@AEAA_NXZ 000000018007379c     libucrt:output.obj
 0003:000027a8       $pdata$?type_case_a@?$output_processor@DV?$string_output_adapter@D@__crt_stdio_output@@V?$standard_base@DV?$string_output_adapter@D@__crt_stdio_output@@@2@@__crt_stdio_output@@AEAA_NXZ 00000001800737a8     libucrt:output.obj
 0003:000027a8       $pdata$?type_case_a@?$output_processor@DV?$stream_output_adapter@D@__crt_stdio_output@@V?$standard_base@DV?$stream_output_adapter@D@__crt_stdio_output@@@2@@__crt_stdio_output@@AEAA_NXZ 00000001800737a8     libucrt:output.obj
 0003:000027b4       $pdata$?type_case_a@?$output_processor@_WV?$string_output_adapter@_W@__crt_stdio_output@@V?$standard_base@_WV?$string_output_adapter@_W@__crt_stdio_output@@@2@@__crt_stdio_output@@AEAA_NXZ 00000001800737b4     libucrt:output.obj
 0003:000027c0       $pdata$?type_case_c_tchar@?$output_processor@DV?$string_output_adapter@D@__crt_stdio_output@@V?$standard_base@DV?$string_output_adapter@D@__crt_stdio_output@@@2@@__crt_stdio_output@@AEAA_ND@Z 00000001800737c0     libucrt:output.obj
 0003:000027c0       $pdata$?type_case_c_tchar@?$output_processor@DV?$stream_output_adapter@D@__crt_stdio_output@@V?$standard_base@DV?$stream_output_adapter@D@__crt_stdio_output@@@2@@__crt_stdio_output@@AEAA_ND@Z 00000001800737c0     libucrt:output.obj
 0003:000027cc       $pdata$?type_case_c_tchar@?$output_processor@_WV?$string_output_adapter@_W@__crt_stdio_output@@V?$standard_base@_WV?$string_output_adapter@_W@__crt_stdio_output@@@2@@__crt_stdio_output@@AEAA_N_W@Z 00000001800737cc     libucrt:output.obj
 0003:000027d8       $pdata$?type_case_integer@?$output_processor@DV?$string_output_adapter@D@__crt_stdio_output@@V?$standard_base@DV?$string_output_adapter@D@__crt_stdio_output@@@2@@__crt_stdio_output@@AEAA_NI_N@Z 00000001800737d8     libucrt:output.obj
 0003:000027d8       $pdata$?type_case_integer@?$output_processor@DV?$stream_output_adapter@D@__crt_stdio_output@@V?$standard_base@DV?$stream_output_adapter@D@__crt_stdio_output@@@2@@__crt_stdio_output@@AEAA_NI_N@Z 00000001800737d8     libucrt:output.obj
 0003:000027e4       $pdata$?type_case_integer@?$output_processor@_WV?$string_output_adapter@_W@__crt_stdio_output@@V?$standard_base@_WV?$string_output_adapter@_W@__crt_stdio_output@@@2@@__crt_stdio_output@@AEAA_NI_N@Z 00000001800737e4     libucrt:output.obj
 0003:000027f0       $pdata$?type_case_n@?$output_processor@_WV?$string_output_adapter@_W@__crt_stdio_output@@V?$standard_base@_WV?$string_output_adapter@_W@__crt_stdio_output@@@2@@__crt_stdio_output@@AEAA_NXZ 00000001800737f0     libucrt:output.obj
 0003:000027f0       $pdata$?type_case_n@?$output_processor@DV?$stream_output_adapter@D@__crt_stdio_output@@V?$standard_base@DV?$stream_output_adapter@D@__crt_stdio_output@@@2@@__crt_stdio_output@@AEAA_NXZ 00000001800737f0     libucrt:output.obj
 0003:000027f0       $pdata$?type_case_n@?$output_processor@DV?$string_output_adapter@D@__crt_stdio_output@@V?$standard_base@DV?$string_output_adapter@D@__crt_stdio_output@@@2@@__crt_stdio_output@@AEAA_NXZ 00000001800737f0     libucrt:output.obj
 0003:000027fc       $pdata$?type_case_s@?$output_processor@DV?$stream_output_adapter@D@__crt_stdio_output@@V?$standard_base@DV?$stream_output_adapter@D@__crt_stdio_output@@@2@@__crt_stdio_output@@AEAA_NXZ 00000001800737fc     libucrt:output.obj
 0003:000027fc       $pdata$?type_case_s@?$output_processor@DV?$string_output_adapter@D@__crt_stdio_output@@V?$standard_base@DV?$string_output_adapter@D@__crt_stdio_output@@@2@@__crt_stdio_output@@AEAA_NXZ 00000001800737fc     libucrt:output.obj
 0003:00002808       $pdata$?type_case_s@?$output_processor@_WV?$string_output_adapter@_W@__crt_stdio_output@@V?$standard_base@_WV?$string_output_adapter@_W@__crt_stdio_output@@@2@@__crt_stdio_output@@AEAA_NXZ 0000000180073808     libucrt:output.obj
 0003:00002814       $pdata$?validate_stream_is_ansi_if_required@?$__acrt_stdio_char_traits@D@@SA_NQEAU_iobuf@@@Z 0000000180073814     libucrt:output.obj
 0003:00002820       $pdata$?write_stored_string_tchar@?$output_processor@DV?$stream_output_adapter@D@__crt_stdio_output@@V?$standard_base@DV?$stream_output_adapter@D@__crt_stdio_output@@@2@@__crt_stdio_output@@AEAA_ND@Z 0000000180073820     libucrt:output.obj
 0003:0000282c       $pdata$?write_stored_string_tchar@?$output_processor@DV?$string_output_adapter@D@__crt_stdio_output@@V?$standard_base@DV?$string_output_adapter@D@__crt_stdio_output@@@2@@__crt_stdio_output@@AEAA_ND@Z 000000018007382c     libucrt:output.obj
 0003:00002838       $pdata$?write_stored_string_tchar@?$output_processor@_WV?$string_output_adapter@_W@__crt_stdio_output@@V?$standard_base@_WV?$string_output_adapter@_W@__crt_stdio_output@@@2@@__crt_stdio_output@@AEAA_N_W@Z 0000000180073838     libucrt:output.obj
 0003:00002844       $pdata$?write_string@?$string_output_adapter@D@__crt_stdio_output@@QEBAXQEBDHQEAHAEAV__crt_deferred_errno_cache@@@Z 0000000180073844     libucrt:output.obj
 0003:00002850       $pdata$?write_string@?$string_output_adapter@_W@__crt_stdio_output@@QEBAXQEB_WHQEAHAEAV__crt_deferred_errno_cache@@@Z 0000000180073850     libucrt:output.obj
 0003:0000285c       $pdata$?write_string_impl@?$output_adapter_common@DV?$stream_output_adapter@D@__crt_stdio_output@@@__crt_stdio_output@@IEBAXQEBDHQEAHAEAV__crt_deferred_errno_cache@@@Z 000000018007385c     libucrt:output.obj
 0003:00002868       $pdata$__stdio_common_vfprintf 0000000180073868     libucrt:output.obj
 0003:00002874       $pdata$_wcsdup             0000000180073874     libucrt:wcsdup.obj
 0003:00002880       $pdata$??$common_fsopen@_W@@YAPEAU_iobuf@@QEB_W0H@Z 0000000180073880     libucrt:fopen.obj
 0003:0000288c       $pdata$_fclose_nolock      000000018007388c     libucrt:fclose.obj
 0003:00002898       $pdata$fclose              0000000180073898     libucrt:fclose.obj
 0003:000028a4       $pdata$_clearfp            00000001800738a4     libucrt:ieee.obj
 0003:000028b0       $pdata$common_control87    00000001800738b0     libucrt:ieee.obj
 0003:000028bc       $pdata$__acrt_errno_map_os_error 00000001800738bc     libucrt:errno.obj
 0003:000028c8       $pdata$__doserrno          00000001800738c8     libucrt:errno.obj
 0003:000028d4       $pdata$_errno              00000001800738d4     libucrt:errno.obj
 0003:000028e0       $pdata$strerror            00000001800738e0     libucrt:strerror.obj
 0003:000028ec       $pdata$__acrt_initialize_stdio 00000001800738ec     libucrt:_file.obj
 0003:000028f8       $pdata$__acrt_uninitialize_stdio 00000001800738f8     libucrt:_file.obj
 0003:00002904       $pdata$??$common_freopen@_W@@YAHQEAPEAU_iobuf@@QEB_W1V__crt_stdio_stream@@H@Z 0000000180073904     libucrt:freopen.obj
 0003:00002910       $pdata$_wfreopen           0000000180073910     libucrt:freopen.obj
 0003:0000291c       $pdata$feof                000000018007391c     libucrt:feoferr.obj
 0003:00002928       $pdata$ferror              0000000180073928     libucrt:feoferr.obj
 0003:00002934       $pdata$_fread_nolock_s     0000000180073934     libucrt:fread.obj
 0003:00002940       $pdata$fread               0000000180073940     libucrt:fread.obj
 0003:0000294c       $pdata$fread_s             000000018007394c     libucrt:fread.obj
 0003:00002958       $pdata$_fgetc_nolock       0000000180073958     libucrt:fgetc.obj
 0003:00002964       $pdata$fgetc               0000000180073964     libucrt:fgetc.obj
 0003:00002970       $pdata$rewind              0000000180073970     libucrt:rewind.obj
 0003:0000297c       $pdata$_ungetc_nolock      000000018007397c     libucrt:ungetc.obj
 0003:00002988       $pdata$ungetc              0000000180073988     libucrt:ungetc.obj
 0003:000029a0       $pdata$iswctype            00000001800739a0     libucrt:iswctype.obj
 0003:000029ac       $pdata$isdigit             00000001800739ac     libucrt:_ctype.obj
 0003:000029b8       $pdata$isspace             00000001800739b8     libucrt:_ctype.obj
 0003:000029c4       $pdata$wcsncpy             00000001800739c4     libucrt:wcsncpy.obj
 0003:000029d0       $pdata$_wcsicmp            00000001800739d0     libucrt:wcsicmp.obj
 0003:000029dc       $pdata$_wcsicmp_l          00000001800739dc     libucrt:wcsicmp.obj
 0003:00002a00       $pdata$fallbackMethod      0000000180073a00     libucrt:strpbrk.obj
 0003:00002a0c       $pdata$strpbrk             0000000180073a0c     libucrt:strpbrk.obj
 0003:00002a18       $pdata$??$common_popen@_W@@YAPEAU_iobuf@@QEB_W0@Z 0000000180073a18     libucrt:popen.obj
 0003:00002a24       $pdata$??$common_popen_nolock@_W@@YAPEAU_iobuf@@QEB_W0HAEAY01H@Z 0000000180073a24     libucrt:popen.obj
 0003:00002a30       $pdata$??$get_executable_path@_W@@YAPEB_WQEB_W@Z 0000000180073a30     libucrt:popen.obj
 0003:00002a3c       $pdata$?idtab@@YAPEAUprocess_handle_pair@?A0xe43b7539@@QEAU_iobuf@@@Z 0000000180073a3c     libucrt:popen.obj
 0003:00002a48       $pdata$_pclose             0000000180073a48     libucrt:popen.obj
 0003:00002a54       $pdata$clearerr_s          0000000180073a54     libucrt:clearerr.obj
 0003:00002a60       $pdata$??$?RV<lambda_842d9ff0dc9ef11c61343bbaebe7f885>@@AEAV<lambda_c5860995281e5c4ce005b3de8f5874ee>@@V<lambda_d90129c13df834fdcbf8d2b88dafcf2d>@@@?$__crt_seh_guarded_call@X@@QEAAX$$QEAV<lambda_842d9ff0dc9ef11c61343bbaebe7f885>@@AEAV<lambda_c5860995281e5c4ce005b3de8f5874ee>@@$$QEAV<lambda_d90129c13df834fdcbf8d2b88dafcf2d>@@@Z 0000000180073a60     libucrt:fflush.obj
 0003:00002a6c       $pdata$??$?RV<lambda_886d6c58226a84441f68b9f2b8217b83>@@AEAV<lambda_ab61a845afdef5b7c387490eaf3616ee>@@V<lambda_f7f22ab5edc0698d5f6905b0d3f44752>@@@?$__crt_seh_guarded_call@X@@QEAAX$$QEAV<lambda_886d6c58226a84441f68b9f2b8217b83>@@AEAV<lambda_ab61a845afdef5b7c387490eaf3616ee>@@$$QEAV<lambda_f7f22ab5edc0698d5f6905b0d3f44752>@@@Z 0000000180073a6c     libucrt:fflush.obj
 0003:00002a78       $pdata$??$?RV<lambda_c376a267cfb53b6959b3b692ec76b120>@@AEAV<lambda_9a32fed5bf61b6b509b2d3f6003082a1>@@V<lambda_572fbb9fa0ab338edf41edfd4b5fcc8d>@@@?$__crt_seh_guarded_call@H@@QEAAH$$QEAV<lambda_c376a267cfb53b6959b3b692ec76b120>@@AEAV<lambda_9a32fed5bf61b6b509b2d3f6003082a1>@@$$QEAV<lambda_572fbb9fa0ab338edf41edfd4b5fcc8d>@@@Z 0000000180073a78     libucrt:fflush.obj
 0003:00002a84       $pdata$?common_flush_all@@YAH_N@Z 0000000180073a84     libucrt:fflush.obj
 0003:00002a90       $pdata$__acrt_stdio_flush_nolock 0000000180073a90     libucrt:fflush.obj
 0003:00002a9c       $pdata$_fflush_nolock      0000000180073a9c     libucrt:fflush.obj
 0003:00002aa8       $pdata$fflush              0000000180073aa8     libucrt:fflush.obj
 0003:00002ab4       $pdata$??$common_fgets@D@@YAPEADQEADHV__crt_stdio_stream@@@Z 0000000180073ab4     libucrt:fgets.obj
 0003:00002ac0       $pdata$?common_fseek@@YAHV__crt_stdio_stream@@_JH@Z 0000000180073ac0     libucrt:fseek.obj
 0003:00002acc       $pdata$?common_fseek_binary_mode_read_only_fast_track_nolock@@YA_NV__crt_stdio_stream@@_JH@Z 0000000180073acc     libucrt:fseek.obj
 0003:00002ad8       $pdata$?common_fseek_nolock@@YAHV__crt_stdio_stream@@_JH@Z 0000000180073ad8     libucrt:fseek.obj
 0003:00002ae4       $pdata$??$common_ftell@J@@YAJV__crt_stdio_stream@@@Z 0000000180073ae4     libucrt:ftell.obj
 0003:00002af0       $pdata$??$common_ftell_nolock@_J@@YA_JV__crt_stdio_stream@@@Z 0000000180073af0     libucrt:ftell.obj
 0003:00002afc       $pdata$?common_ftell_read_mode_nolock@@YA_JV__crt_stdio_stream@@_J1@Z 0000000180073afc     libucrt:ftell.obj
 0003:00002b08       $pdata$?common_ftell_translated_utf8_nolock@@YA_JV__crt_stdio_stream@@_J@Z 0000000180073b08     libucrt:ftell.obj
 0003:00002b14       $pdata$??$?RV<lambda_bdbcead8b570fa3d5ec6d9679862a6e5>@@AEAV<lambda_96f4279ff90247a4c5c5d9824f56f8c1>@@V<lambda_4606be27f17b5e5579e09050fab91818>@@@?$__crt_seh_guarded_call@_K@@QEAA_K$$QEAV<lambda_bdbcead8b570fa3d5ec6d9679862a6e5>@@AEAV<lambda_96f4279ff90247a4c5c5d9824f56f8c1>@@$$QEAV<lambda_4606be27f17b5e5579e09050fab91818>@@@Z 0000000180073b14     libucrt:fwrite.obj
 0003:00002b20       $pdata$??R<lambda_96f4279ff90247a4c5c5d9824f56f8c1>@@QEBA_KXZ 0000000180073b20     libucrt:fwrite.obj
 0003:00002b2c       $pdata$_fwrite_nolock      0000000180073b2c     libucrt:fwrite.obj
 0003:00002b38       $pdata$fwrite              0000000180073b38     libucrt:fwrite.obj
 0003:00002b44       $pdata$??$?RV<lambda_84ec643ea9557e2f7dc01bb0e9624395>@@AEAV<lambda_ca71763b3c0644891230e4f79ea54fa6>@@V<lambda_439a761618c59b0600e24586724d733b>@@@?$__crt_seh_guarded_call@H@@QEAAH$$QEAV<lambda_84ec643ea9557e2f7dc01bb0e9624395>@@AEAV<lambda_ca71763b3c0644891230e4f79ea54fa6>@@$$QEAV<lambda_439a761618c59b0600e24586724d733b>@@@Z 0000000180073b44     libucrt:setvbuf.obj
 0003:00002b50       $pdata$??R<lambda_ca71763b3c0644891230e4f79ea54fa6>@@QEBAHXZ 0000000180073b50     libucrt:setvbuf.obj
 0003:00002b5c       $pdata$setvbuf             0000000180073b5c     libucrt:setvbuf.obj
 0003:00002b68       $pdata$??$generate_tmpfile_file_name@D@@YA_NQEAD_K@Z 0000000180073b68     libucrt:tmpfile.obj
 0003:00002b74       $pdata$??$get_tmpfile_buffer_nolock@D@@YAPEADW4buffer_id@?A0x5b9a7937@@@Z 0000000180073b74     libucrt:tmpfile.obj
 0003:00002b80       $pdata$??$initialize_tmpfile_buffer_nolock@D@@YA_NW4buffer_id@?A0x5b9a7937@@@Z 0000000180073b80     libucrt:tmpfile.obj
 0003:00002b8c       $pdata$?common_tmpfile@@YAHQEAPEAU_iobuf@@H@Z 0000000180073b8c     libucrt:tmpfile.obj
 0003:00002b98       $pdata$?common_tmpfile_nolock@@YAHQEAPEAU_iobuf@@H@Z 0000000180073b98     libucrt:tmpfile.obj
 0003:00002ba4       $pdata$__acrt_stdio_free_tmpfile_name_buffers_nolock 0000000180073ba4     libucrt:tmpfile.obj
 0003:00002bb0       $pdata$tmpfile             0000000180073bb0     libucrt:tmpfile.obj
 0003:00002bbc       $pdata$??$?RV<lambda_082dd7c0feb7dbdaf245f261e54a6583>@@AEAV<lambda_f3caf1ecae5fe01a9a1a6239afa44510>@@V<lambda_c640b76c0755ae85b317b35c67c61e6b>@@@?$__crt_seh_guarded_call@H@@QEAAH$$QEAV<lambda_082dd7c0feb7dbdaf245f261e54a6583>@@AEAV<lambda_f3caf1ecae5fe01a9a1a6239afa44510>@@$$QEAV<lambda_c640b76c0755ae85b317b35c67c61e6b>@@@Z 0000000180073bbc     libucrt:input.obj
 0003:00002bc8       $pdata$??$parse_floating_point@V?$input_adapter_character_source@V?$stream_input_adapter@D@__crt_stdio_input@@@__crt_strtox@@M@__crt_strtox@@YA?AW4SLD_STATUS@@QEAU__crt_locale_pointers@@V?$input_adapter_character_source@V?$stream_input_adapter@D@__crt_stdio_input@@@0@QEAM@Z 0000000180073bc8     libucrt:input.obj
 0003:00002bd4       $pdata$??$parse_floating_point@V?$input_adapter_character_source@V?$stream_input_adapter@D@__crt_stdio_input@@@__crt_strtox@@N@__crt_strtox@@YA?AW4SLD_STATUS@@QEAU__crt_locale_pointers@@V?$input_adapter_character_source@V?$stream_input_adapter@D@__crt_stdio_input@@@0@QEAN@Z 0000000180073bd4     libucrt:input.obj
 0003:00002be0       $pdata$??$parse_floating_point_from_source@V?$input_adapter_character_source@V?$stream_input_adapter@D@__crt_stdio_input@@@__crt_strtox@@@__crt_strtox@@YA?AW4floating_point_parse_result@0@QEAU__crt_locale_pointers@@AEAV?$input_adapter_character_source@V?$stream_input_adapter@D@__crt_stdio_input@@@0@AEAUfloating_point_string@0@@Z 0000000180073be0     libucrt:input.obj
 0003:00002bec       $pdata$??$parse_floating_point_possible_infinity@DV?$input_adapter_character_source@V?$stream_input_adapter@D@__crt_stdio_input@@@__crt_strtox@@_K@__crt_strtox@@YA?AW4floating_point_parse_result@0@AEADAEAV?$input_adapter_character_source@V?$stream_input_adapter@D@__crt_stdio_input@@@0@_K@Z 0000000180073bec     libucrt:input.obj
 0003:00002bf8       $pdata$??$parse_floating_point_possible_nan@DV?$input_adapter_character_source@V?$stream_input_adapter@D@__crt_stdio_input@@@__crt_strtox@@_K@__crt_strtox@@YA?AW4floating_point_parse_result@0@AEADAEAV?$input_adapter_character_source@V?$stream_input_adapter@D@__crt_stdio_input@@@0@_K@Z 0000000180073bf8     libucrt:input.obj
 0003:00002c04       $pdata$??$parse_floating_point_possible_nan_is_ind@DV?$input_adapter_character_source@V?$stream_input_adapter@D@__crt_stdio_input@@@__crt_strtox@@@__crt_strtox@@YA_NAEADAEAV?$input_adapter_character_source@V?$stream_input_adapter@D@__crt_stdio_input@@@0@@Z 0000000180073c04     libucrt:input.obj
 0003:00002c10       $pdata$??$parse_floating_point_possible_nan_is_snan@DV?$input_adapter_character_source@V?$stream_input_adapter@D@__crt_stdio_input@@@__crt_strtox@@@__crt_strtox@@YA_NAEADAEAV?$input_adapter_character_source@V?$stream_input_adapter@D@__crt_stdio_input@@@0@@Z 0000000180073c10     libucrt:input.obj
 0003:00002c1c       $pdata$??$parse_floating_point_write_result@M@__crt_strtox@@YA?AW4SLD_STATUS@@W4floating_point_parse_result@0@AEBUfloating_point_string@0@QEAM@Z 0000000180073c1c     libucrt:input.obj
 0003:00002c28       $pdata$??$parse_floating_point_write_result@N@__crt_strtox@@YA?AW4SLD_STATUS@@W4floating_point_parse_result@0@AEBUfloating_point_string@0@QEAN@Z 0000000180073c28     libucrt:input.obj
 0003:00002c34       $pdata$??$parse_integer@_KV?$input_adapter_character_source@V?$stream_input_adapter@D@__crt_stdio_input@@@__crt_strtox@@@__crt_strtox@@YA_KQEAU__crt_locale_pointers@@V?$input_adapter_character_source@V?$stream_input_adapter@D@__crt_stdio_input@@@0@H_N@Z 0000000180073c34     libucrt:input.obj
 0003:00002c40       $pdata$??$process_floating_point_specifier_t@M@?$input_processor@DV?$stream_input_adapter@D@__crt_stdio_input@@@__crt_stdio_input@@AEAA_NXZ 0000000180073c40     libucrt:input.obj
 0003:00002c4c       $pdata$??$process_floating_point_specifier_t@N@?$input_processor@DV?$stream_input_adapter@D@__crt_stdio_input@@@__crt_stdio_input@@AEAA_NXZ 0000000180073c4c     libucrt:input.obj
 0003:00002c58       $pdata$??$process_string_specifier_tchar@D@?$input_processor@DV?$stream_input_adapter@D@__crt_stdio_input@@@__crt_stdio_input@@AEAA_NW4conversion_mode@1@D@Z 0000000180073c58     libucrt:input.obj
 0003:00002c64       $pdata$??$process_string_specifier_tchar@_W@?$input_processor@DV?$stream_input_adapter@D@__crt_stdio_input@@@__crt_stdio_input@@AEAA_NW4conversion_mode@1@_W@Z 0000000180073c64     libucrt:input.obj
 0003:00002c70       $pdata$??$skip_whitespace@Vstream_input_adapter@__crt_stdio_input@@D@__crt_stdio_input@@YAHAEAV?$stream_input_adapter@D@0@QEAU__crt_locale_pointers@@@Z 0000000180073c70     libucrt:input.obj
 0003:00002c7c       $pdata$??R<lambda_156378f40168adef48d7ddfcff3a1264>@@QEBA_NXZ 0000000180073c7c     libucrt:input.obj
 0003:00002c88       $pdata$??R<lambda_f3caf1ecae5fe01a9a1a6239afa44510>@@QEBAHXZ 0000000180073c88     libucrt:input.obj
 0003:00002c94       $pdata$?advance@?$format_string_parser@D@__crt_stdio_input@@QEAA_NXZ 0000000180073c94     libucrt:input.obj
 0003:00002ca0       $pdata$?as_double@floating_point_value@__crt_strtox@@QEBAAEANXZ 0000000180073ca0     libucrt:input.obj
 0003:00002cac       $pdata$?as_float@floating_point_value@__crt_strtox@@QEBAAEAMXZ 0000000180073cac     libucrt:input.obj
 0003:00002cb8       $pdata$?assemble_floating_point_value@__crt_strtox@@YA?AW4SLD_STATUS@@_KH_N1AEBVfloating_point_value@1@@Z 0000000180073cb8     libucrt:input.obj
 0003:00002cc4       $pdata$?assemble_floating_point_value_from_big_integer@__crt_strtox@@YA?AW4SLD_STATUS@@AEBUbig_integer@1@I_N1AEBVfloating_point_value@1@@Z 0000000180073cc4     libucrt:input.obj
 0003:00002cd0       $pdata$?convert_decimal_string_to_floating_type_common@__crt_strtox@@YA?AW4SLD_STATUS@@AEBUfloating_point_string@1@AEBVfloating_point_value@1@@Z 0000000180073cd0     libucrt:input.obj
 0003:00002cdc       $pdata$?convert_hexadecimal_string_to_floating_type_common@__crt_strtox@@YA?AW4SLD_STATUS@@AEBUfloating_point_string@1@AEBVfloating_point_value@1@@Z 0000000180073cdc     libucrt:input.obj
 0003:00002ce8       $pdata$?divide@__crt_strtox@@YA_KAEAUbig_integer@1@AEBU21@@Z 0000000180073ce8     libucrt:input.obj
 0003:00002cf4       $pdata$0$?divide@__crt_strtox@@YA_KAEAUbig_integer@1@AEBU21@@Z 0000000180073cf4     libucrt:input.obj
 0003:00002d00       $pdata$1$?divide@__crt_strtox@@YA_KAEAUbig_integer@1@AEBU21@@Z 0000000180073d00     libucrt:input.obj
 0003:00002d0c       $pdata$?process@?$input_processor@DV?$stream_input_adapter@D@__crt_stdio_input@@@__crt_stdio_input@@QEAAHXZ 0000000180073d0c     libucrt:input.obj
 0003:00002d18       $pdata$?process_conversion_specifier@?$input_processor@DV?$stream_input_adapter@D@__crt_stdio_input@@@__crt_stdio_input@@AEAA_NXZ 0000000180073d18     libucrt:input.obj
 0003:00002d24       $pdata$?process_floating_point_specifier@?$input_processor@DV?$stream_input_adapter@D@__crt_stdio_input@@@__crt_stdio_input@@AEAA_NXZ 0000000180073d24     libucrt:input.obj
 0003:00002d30       $pdata$?process_integer_specifier@?$input_processor@DV?$stream_input_adapter@D@__crt_stdio_input@@@__crt_stdio_input@@AEAA_NI_N@Z 0000000180073d30     libucrt:input.obj
 0003:00002d3c       $pdata$?process_literal_character_tchar@?$input_processor@DV?$stream_input_adapter@D@__crt_stdio_input@@@__crt_stdio_input@@AEAA_ND@Z 0000000180073d3c     libucrt:input.obj
 0003:00002d48       $pdata$?process_state@?$input_processor@DV?$stream_input_adapter@D@__crt_stdio_input@@@__crt_stdio_input@@AEAA_NXZ 0000000180073d48     libucrt:input.obj
 0003:00002d54       $pdata$?process_string_specifier@?$input_processor@DV?$stream_input_adapter@D@__crt_stdio_input@@@__crt_stdio_input@@AEAA_NW4conversion_mode@2@@Z 0000000180073d54     libucrt:input.obj
 0003:00002d60       $pdata$?scan_optional_field_width@?$format_string_parser@D@__crt_stdio_input@@AEAA_NXZ 0000000180073d60     libucrt:input.obj
 0003:00002d6c       $pdata$?scan_scanset_range@?$format_string_parser@D@__crt_stdio_input@@AEAA_NXZ 0000000180073d6c     libucrt:input.obj
 0003:00002d78       $pdata$?write_character@?$input_processor@DV?$stream_input_adapter@D@__crt_stdio_input@@@__crt_stdio_input@@AEAA_NQEFA_W_KAEAPEFA_WAEA_KD@Z 0000000180073d78     libucrt:input.obj
 0003:00002d84       $pdata$?write_integer@?$input_processor@DV?$stream_input_adapter@D@__crt_stdio_input@@@__crt_stdio_input@@AEAA_N_K@Z 0000000180073d84     libucrt:input.obj
 0003:00002d90       $pdata$__stdio_common_vfscanf 0000000180073d90     libucrt:input.obj
 0003:00002d9c       $pdata$memcpy_s            0000000180073d9c     libucrt:cfout.obj
 0003:00002d9c       $pdata$memcpy_s            0000000180073d9c     libucrt:input.obj
 0003:00002da8       $pdata$??$common_dupenv_s@_W@@YAHQEAPEA_WQEA_KQEB_WHQEBDH@Z 0000000180073da8     libucrt:getenv.obj
 0003:00002db4       $pdata$??$common_getenv@_W@@YAPEA_WQEB_W@Z 0000000180073db4     libucrt:getenv.obj
 0003:00002dc0       $pdata$??$common_getenv_nolock@_W@@YAPEA_WQEB_W@Z 0000000180073dc0     libucrt:getenv.obj
 0003:00002dcc       $pdata$_wdupenv_s          0000000180073dcc     libucrt:getenv.obj
 0003:00002dd8       $pdata$_wsystem            0000000180073dd8     libucrt:system.obj
 0003:00002de4       $pdata$_initterm           0000000180073de4     libucrt:initterm.obj
 0003:00002df0       $pdata$_initterm_e         0000000180073df0     libucrt:initterm.obj
 0003:00002dfc       $pdata$_seh_filter_exe     0000000180073dfc     libucrt:exception_filter.obj
 0003:00002e08       $pdata$??$?RV<lambda_d80eeec6fff315bfe5c115232f3240e3>@@AEAV<lambda_6e4b09c48022b2350581041d5f6b0c4c>@@V<lambda_2358e3775559c9db80273638284d5e45>@@@?$__crt_seh_guarded_call@X@@QEAAX$$QEAV<lambda_d80eeec6fff315bfe5c115232f3240e3>@@AEAV<lambda_6e4b09c48022b2350581041d5f6b0c4c>@@$$QEAV<lambda_2358e3775559c9db80273638284d5e45>@@@Z 0000000180073e08     libucrt:exit.obj
 0003:00002e14       $pdata$??R<lambda_6e4b09c48022b2350581041d5f6b0c4c>@@QEBA@XZ 0000000180073e14     libucrt:exit.obj
 0003:00002e20       $pdata$?common_exit@@YAXHW4_crt_exit_cleanup_mode@@W4_crt_exit_return_mode@@@Z 0000000180073e20     libucrt:exit.obj
 0003:00002e2c       $pdata$?exit_or_terminate_process@@YAXI@Z 0000000180073e2c     libucrt:exit.obj
 0003:00002e38       $pdata$?try_cor_exit_process@@YAXI@Z 0000000180073e38     libucrt:exit.obj
 0003:00002e44       $pdata$??$parse_command_line@D@@YAXPEADPEAPEAD0PEA_K2@Z 0000000180073e44     libucrt:argv_parsing.obj
 0003:00002e50       $pdata$__acrt_allocate_buffer_for_argv 0000000180073e50     libucrt:argv_parsing.obj
 0003:00002e5c       $pdata$_configure_narrow_argv 0000000180073e5c     libucrt:argv_parsing.obj
 0003:00002e68       $pdata$??$common_initialize_environment_nolock@D@@YAHXZ 0000000180073e68     libucrt:environment_initialization.obj
 0003:00002e74       $pdata$??$common_initialize_environment_nolock@_W@@YAHXZ 0000000180073e74     libucrt:environment_initialization.obj
 0003:00002e80       $pdata$??$create_environment@D@@YAQEAPEADQEAD@Z 0000000180073e80     libucrt:environment_initialization.obj
 0003:00002e8c       $pdata$??$create_environment@_W@@YAQEAPEA_WQEA_W@Z 0000000180073e8c     libucrt:environment_initialization.obj
 0003:00002e98       $pdata$??$free_environment@_W@@YAXQEAPEA_W@Z 0000000180073e98     libucrt:environment_initialization.obj
 0003:00002e98       $pdata$??$free_environment@D@@YAXQEAPEAD@Z 0000000180073e98     libucrt:environment_initialization.obj
 0003:00002ea4       $pdata$??$initialize_environment_by_cloning_nolock@_W@@YAHXZ 0000000180073ea4     libucrt:environment_initialization.obj
 0003:00002eb0       $pdata$??$uninitialize_environment_internal@D@@YAXAEAPEAPEAD@Z 0000000180073eb0     libucrt:environment_initialization.obj
 0003:00002ebc       $pdata$??$uninitialize_environment_internal@_W@@YAXAEAPEAPEA_W@Z 0000000180073ebc     libucrt:environment_initialization.obj
 0003:00002ec8       $pdata$__dcrt_get_or_create_wide_environment_nolock 0000000180073ec8     libucrt:environment_initialization.obj
 0003:00002ed4       $pdata$__dcrt_uninitialize_environments_nolock 0000000180073ed4     libucrt:environment_initialization.obj
 0003:00002ee0       $pdata$??$?RV<lambda_7777bce6b2f8c936911f934f8298dc43>@@AEAV<lambda_f03950bc5685219e0bcd2087efbe011e>@@V<lambda_3883c3dff614d5e0c5f61bb1ac94921c>@@@?$__crt_seh_guarded_call@H@@QEAAH$$QEAV<lambda_7777bce6b2f8c936911f934f8298dc43>@@AEAV<lambda_f03950bc5685219e0bcd2087efbe011e>@@$$QEAV<lambda_3883c3dff614d5e0c5f61bb1ac94921c>@@@Z 0000000180073ee0     libucrt:onexit.obj
 0003:00002eec       $pdata$??R<lambda_f03950bc5685219e0bcd2087efbe011e>@@QEBAHXZ 0000000180073eec     libucrt:onexit.obj
 0003:00002ef8       $pdata$_execute_onexit_table 0000000180073ef8     libucrt:onexit.obj
 0003:00002f04       $pdata$initialize_c        0000000180073f04     libucrt:initialization.obj
 0003:00002f10       $pdata$uninitialize_environment 0000000180073f10     libucrt:initialization.obj
 0003:00002f1c       $pdata$initialize_pointers 0000000180073f1c     libucrt:initialization.obj
 0003:00002f28       $pdata$uninitialize_allocated_memory 0000000180073f28     libucrt:initialization.obj
 0003:00002f34       $pdata$uninitialize_allocated_io_buffers 0000000180073f34     libucrt:initialization.obj
 0003:00002f40       $pdata$__acrt_thread_attach 0000000180073f40     libucrt:initialization.obj
 0003:00002f4c       $pdata$__acrt_thread_detach 0000000180073f4c     libucrt:initialization.obj
 0003:00002f58       $pdata$__acrt_uninitialize 0000000180073f58     libucrt:initialization.obj
 0003:00002f64       $pdata$__acrt_uninitialize_critical 0000000180073f64     libucrt:initialization.obj
 0003:00002f70       $pdata$terminate           0000000180073f70     libucrt:terminate.obj
 0003:00002f7c       $pdata$?_strupr_s_l_stat@@YAHQEAD_KQEAU__crt_locale_pointers@@@Z 0000000180073f7c     libucrt:strupr.obj
 0003:00002f88       $pdata$_strupr             0000000180073f88     libucrt:strupr.obj
 0003:00002f94       $pdata$_strupr_s_l         0000000180073f94     libucrt:strupr.obj
 0003:00002fa0       $pdata$_stricmp            0000000180073fa0     libucrt:stricmp.obj
 0003:00002fac       $pdata$_stricmp_l          0000000180073fac     libucrt:stricmp.obj
 0003:00002fb8       $pdata$strcpy_s            0000000180073fb8     libucrt:strcpy_s.obj
 0003:00002fc4       $pdata$??$parse_integer@KV?$c_string_character_source@D@__crt_strtox@@@__crt_strtox@@YAKQEAU__crt_locale_pointers@@V?$c_string_character_source@D@0@H_N@Z 0000000180073fc4     libucrt:atox.obj
 0003:00002fd0       $pdata$??$parse_integer@KV?$c_string_character_source@_W@__crt_strtox@@@__crt_strtox@@YAKQEAU__crt_locale_pointers@@V?$c_string_character_source@_W@0@H_N@Z 0000000180073fd0     libucrt:atox.obj
 0003:00002fdc       $pdata$??$parse_integer@_KV?$c_string_character_source@D@__crt_strtox@@@__crt_strtox@@YA_KQEAU__crt_locale_pointers@@V?$c_string_character_source@D@0@H_N@Z 0000000180073fdc     libucrt:atox.obj
 0003:00002fe8       $pdata$abort               0000000180073fe8     libucrt:abort.obj
 0003:00002ff4       $pdata$__acrt_call_reportfault 0000000180073ff4     libucrt:invalid_parameter.obj
 0003:00003000       $pdata$_invalid_parameter  0000000180074000     libucrt:invalid_parameter.obj
 0003:0000300c       $pdata$_invalid_parameter_noinfo 000000018007400c     libucrt:invalid_parameter.obj
 0003:00003018       $pdata$_invoke_watson      0000000180074018     libucrt:invalid_parameter.obj
 0003:00003024       $pdata$?internal_isupper_l@@YA_NHQEAU__crt_locale_pointers@@@Z 0000000180074024     libucrt:tolower_toupper.obj
 0003:00003030       $pdata$_tolower_l          0000000180074030     libucrt:tolower_toupper.obj
 0003:0000303c       $pdata$tolower             000000018007403c     libucrt:tolower_toupper.obj
 0003:00003048       $pdata$_free_base          0000000180074048     libucrt:free_base.obj
 0003:00003054       $pdata$_malloc_base        0000000180074054     libucrt:malloc_base.obj
 0003:00003060       $pdata$strtol              0000000180074060     libucrt:strtox.obj
 0003:0000306c       $pdata$strtoull            000000018007406c     libucrt:strtox.obj
 0003:00003078       $pdata$wcstol              0000000180074078     libucrt:strtox.obj
 0003:00003084       $pdata$_mbtowc_l           0000000180074084     libucrt:mbtowc.obj
 0003:00003090       $pdata$_wctomb_s_l         0000000180074090     libucrt:wctomb.obj
 0003:0000309c       $pdata$wctomb_s            000000018007409c     libucrt:wctomb.obj
 0003:000030a8       $pdata$??$?RV<lambda_0ae27a3a962d80f24befdcbee591983d>@@AEAV<lambda_8d0ee55de4b1038c4002e0adecdf1839>@@V<lambda_dc504788e8f1664fe9b84e20bfb512f2>@@@?$__crt_seh_guarded_call@X@@QEAAX$$QEAV<lambda_0ae27a3a962d80f24befdcbee591983d>@@AEAV<lambda_8d0ee55de4b1038c4002e0adecdf1839>@@$$QEAV<lambda_dc504788e8f1664fe9b84e20bfb512f2>@@@Z 00000001800740a8     libucrt:per_thread_data.obj
 0003:000030b4       $pdata$??$?RV<lambda_2d41944a1d46af3157314b8a01080d33>@@AEAV<lambda_8f455de75cd7d7f24b4096f044d8b9e6>@@V<lambda_aa500f224e6afead328df44964fe2772>@@@?$__crt_seh_guarded_call@X@@QEAAX$$QEAV<lambda_2d41944a1d46af3157314b8a01080d33>@@AEAV<lambda_8f455de75cd7d7f24b4096f044d8b9e6>@@$$QEAV<lambda_aa500f224e6afead328df44964fe2772>@@@Z 00000001800740b4     libucrt:per_thread_data.obj
 0003:000030c0       $pdata$??$?RV<lambda_aa87e3671a710a21b5dc78c0bdf72e11>@@AEAV<lambda_92619d2358a28f41a33ba319515a20b9>@@V<lambda_6992ecaafeb10aed2b74cb1fae11a551>@@@?$__crt_seh_guarded_call@X@@QEAAX$$QEAV<lambda_aa87e3671a710a21b5dc78c0bdf72e11>@@AEAV<lambda_92619d2358a28f41a33ba319515a20b9>@@$$QEAV<lambda_6992ecaafeb10aed2b74cb1fae11a551>@@@Z 00000001800740c0     libucrt:per_thread_data.obj
 0003:000030cc       $pdata$??$?RV<lambda_f2e299630e499de9f9a165e60fcd3db5>@@AEAV<lambda_2ae9d31cdba2644fcbeaf08da7c24588>@@V<lambda_40d01ff24d0e7b3814fdbdcee8eab3c7>@@@?$__crt_seh_guarded_call@X@@QEAAX$$QEAV<lambda_f2e299630e499de9f9a165e60fcd3db5>@@AEAV<lambda_2ae9d31cdba2644fcbeaf08da7c24588>@@$$QEAV<lambda_40d01ff24d0e7b3814fdbdcee8eab3c7>@@@Z 00000001800740cc     libucrt:per_thread_data.obj
 0003:000030d8       $pdata$?construct_ptd_array@@YAXQEAU__acrt_ptd@@@Z 00000001800740d8     libucrt:per_thread_data.obj
 0003:000030e4       $pdata$?destroy_fls@@YAXPEAX@Z 00000001800740e4     libucrt:per_thread_data.obj
 0003:000030f0       $pdata$?destroy_ptd_array@@YAXQEAU__acrt_ptd@@@Z 00000001800740f0     libucrt:per_thread_data.obj
 0003:000030fc       $pdata$?replace_current_thread_locale_nolock@@YAXQEAU__acrt_ptd@@QEAU__crt_locale_data@@@Z 00000001800740fc     libucrt:per_thread_data.obj
 0003:00003108       $pdata$__acrt_freeptd      0000000180074108     libucrt:per_thread_data.obj
 0003:00003114       $pdata$__acrt_getptd       0000000180074114     libucrt:per_thread_data.obj
 0003:00003120       $pdata$__acrt_getptd_head  0000000180074120     libucrt:per_thread_data.obj
 0003:0000312c       $pdata$__acrt_getptd_noexit 000000018007412c     libucrt:per_thread_data.obj
 0003:00003138       $pdata$__acrt_initialize_ptd 0000000180074138     libucrt:per_thread_data.obj
 0003:00003144       $pdata$__acrt_uninitialize_ptd 0000000180074144     libucrt:per_thread_data.obj
 0003:00003150       $pdata$__acrt_update_locale_info 0000000180074150     libucrt:locale_update.obj
 0003:0000315c       $pdata$__acrt_update_multibyte_info 000000018007415c     libucrt:locale_update.obj
 0003:00003168       $pdata$?fp_format_a@@YAHQEBNPEAD_KQEAD2H_NIQEAU__crt_locale_pointers@@@Z 0000000180074168     libucrt:cvt.obj
 0003:00003174       $pdata$?fp_format_e@@YAHQEBNQEAD_K12H_NIQEAU__crt_locale_pointers@@@Z 0000000180074174     libucrt:cvt.obj
 0003:00003180       $pdata$?fp_format_e_internal@@YAHQEAD_KH_NIQEAU_strflt@@2QEAU__crt_locale_pointers@@@Z 0000000180074180     libucrt:cvt.obj
 0003:0000318c       $pdata$?fp_format_f_internal@@YAHQEAD_KHQEAU_strflt@@_NQEAU__crt_locale_pointers@@@Z 000000018007418c     libucrt:cvt.obj
 0003:00003198       $pdata$?fp_format_g@@YAHQEBNQEAD_K12H_NIQEAU__crt_locale_pointers@@@Z 0000000180074198     libucrt:cvt.obj
 0003:000031a4       $pdata$?fp_format_nan_or_infinity@@YAHW4__acrt_fp_class@@_NPEAD_K1@Z 00000001800741a4     libucrt:cvt.obj
 0003:000031b0       $pdata$__acrt_fp_format    00000001800741b0     libucrt:cvt.obj
 0003:000031bc       $pdata$_fileno             00000001800741bc     libucrt:fileno.obj
 0003:000031c8       $pdata$__acrt_stdio_begin_temporary_buffering_nolock 00000001800741c8     libucrt:_sftbuf.obj
 0003:000031d4       $pdata$__acrt_stdio_end_temporary_buffering_nolock 00000001800741d4     libucrt:_sftbuf.obj
 0003:000031e0       $pdata$??$?RV<lambda_410d79af7f07d98d83a3f525b3859a53>@@AEAV<lambda_3e16ef9562a7dcce91392c22ab16ea36>@@V<lambda_38119f0e861e05405d8a144b9b982f0a>@@@?$__crt_seh_guarded_call@X@@QEAAX$$QEAV<lambda_410d79af7f07d98d83a3f525b3859a53>@@AEAV<lambda_3e16ef9562a7dcce91392c22ab16ea36>@@$$QEAV<lambda_38119f0e861e05405d8a144b9b982f0a>@@@Z 00000001800741e0     libucrt:wsetlocale.obj
 0003:000031ec       $pdata$__acrt_uninitialize_locale 00000001800741ec     libucrt:wsetlocale.obj
 0003:000031f8       $pdata$?initialize_inherited_file_handles_nolock@@YAXXZ 00000001800741f8     libucrt:ioinit.obj
 0003:00003204       $pdata$?initialize_stdio_handles_nolock@@YAXXZ 0000000180074204     libucrt:ioinit.obj
 0003:00003210       $pdata$__acrt_initialize_lowio 0000000180074210     libucrt:ioinit.obj
 0003:0000321c       $pdata$__acrt_uninitialize_lowio 000000018007421c     libucrt:ioinit.obj
 0003:00003228       $pdata$wcscpy_s            0000000180074228     libucrt:wcscpy_s.obj
 0003:00003234       $pdata$?__acrt_stdio_allocate_stream@@YA?AV__crt_stdio_stream@@XZ 0000000180074234     libucrt:stream.obj
 0003:00003240       $pdata$?find_or_allocate_unused_stream_nolock@@YA?AV__crt_stdio_stream@@XZ 0000000180074240     libucrt:stream.obj
 0003:0000324c       $pdata$??$__acrt_stdio_parse_mode@_W@@YA?AU__acrt_stdio_stream_mode@@QEB_W@Z 000000018007424c     libucrt:openfile.obj
 0003:00003258       $pdata$_wopenfile          0000000180074258     libucrt:openfile.obj
 0003:00003264       $pdata$??$?RV<lambda_751a882b2c74d4b022dec766aa51a29a>@@AEAV<lambda_628dfdc04ba53c8bfc02c9951375f3f5>@@V<lambda_f6c7be5f7998530c34de24c7437d6b54>@@@?$__crt_seh_guarded_call@H@@QEAAH$$QEAV<lambda_751a882b2c74d4b022dec766aa51a29a>@@AEAV<lambda_628dfdc04ba53c8bfc02c9951375f3f5>@@$$QEAV<lambda_f6c7be5f7998530c34de24c7437d6b54>@@@Z 0000000180074264     libucrt:close.obj
 0003:00003270       $pdata$_close              0000000180074270     libucrt:close.obj
 0003:0000327c       $pdata$_close_nolock       000000018007427c     libucrt:close.obj
 0003:00003288       $pdata$__acrt_stdio_free_buffer_nolock 0000000180074288     libucrt:_freebuf.obj
 0003:000032a0       $pdata$_calloc_base        00000001800742a0     libucrt:calloc_base.obj
 0003:000032ac       $pdata$strncpy_s           00000001800742ac     libucrt:strncpy_s.obj
 0003:000032b8       $pdata$?try_get_function@@YAPEAXW4function_id@?A0x391cf84c@@QEBDQEBW4module_id@2@2@Z 00000001800742b8     libucrt:winapi_thunks.obj
 0003:000032c4       $pdata$__acrt_AppPolicyGetProcessTerminationMethodInternal 00000001800742c4     libucrt:winapi_thunks.obj
 0003:000032d0       $pdata$__acrt_AreFileApisANSI 00000001800742d0     libucrt:winapi_thunks.obj
 0003:000032dc       $pdata$__acrt_CompareStringEx 00000001800742dc     libucrt:winapi_thunks.obj
 0003:000032e8       $pdata$__acrt_FlsAlloc     00000001800742e8     libucrt:winapi_thunks.obj
 0003:000032f4       $pdata$__acrt_FlsFree      00000001800742f4     libucrt:winapi_thunks.obj
 0003:00003300       $pdata$__acrt_FlsGetValue  0000000180074300     libucrt:winapi_thunks.obj
 0003:0000330c       $pdata$__acrt_FlsSetValue  000000018007430c     libucrt:winapi_thunks.obj
 0003:00003318       $pdata$__acrt_InitializeCriticalSectionEx 0000000180074318     libucrt:winapi_thunks.obj
 0003:00003324       $pdata$__acrt_LCMapStringEx 0000000180074324     libucrt:winapi_thunks.obj
 0003:00003330       $pdata$__acrt_LocaleNameToLCID 0000000180074330     libucrt:winapi_thunks.obj
 0003:0000333c       $pdata$__acrt_initialize_winapi_thunks 000000018007433c     libucrt:winapi_thunks.obj
 0003:00003348       $pdata$__acrt_uninitialize_winapi_thunks 0000000180074348     libucrt:winapi_thunks.obj
 0003:00003354       $pdata$_fcloseall          0000000180074354     libucrt:closeall.obj
 0003:00003360       $pdata$??$translate_text_mode_nolock@D@@YAHHQEAD_K@Z 0000000180074360     libucrt:read.obj
 0003:0000336c       $pdata$??$translate_text_mode_nolock@_W@@YAHHQEA_W_K@Z 000000018007436c     libucrt:read.obj
 0003:00003378       $pdata$?translate_ansi_or_utf8_nolock@@YAHHQEAD_KQEA_W1@Z 0000000180074378     libucrt:read.obj
 0003:00003384       $pdata$_read               0000000180074384     libucrt:read.obj
 0003:00003390       $pdata$_read_nolock        0000000180074390     libucrt:read.obj
 0003:0000339c       $pdata$__acrt_stdio_refill_and_read_narrow_nolock 000000018007439c     libucrt:_filbuf.obj
 0003:000033a8       $pdata$??$common_lseek@J@@YAJHJH@Z 00000001800743a8     libucrt:lseek.obj
 0003:000033b4       $pdata$??$common_lseek@_J@@YA_JH_JH@Z 00000001800743b4     libucrt:lseek.obj
 0003:000033c0       $pdata$??$common_lseek_nolock@J@@YAJHJH@Z 00000001800743c0     libucrt:lseek.obj
 0003:000033cc       $pdata$??$common_lseek_nolock@_J@@YA_JH_JH@Z 00000001800743cc     libucrt:lseek.obj
 0003:000033d8       $pdata$__acrt_stdio_allocate_buffer_nolock 00000001800743d8     libucrt:_getbuf.obj
 0003:000033e4       $pdata$__pctype_func       00000001800743e4     libucrt:ctype.obj
 0003:000033f0       $pdata$_isctype_l          00000001800743f0     libucrt:isctype.obj
 0003:000033fc       $pdata$_towlower_l         00000001800743fc     libucrt:towlower.obj
 0003:00003408       $pdata$_recalloc_base      0000000180074408     libucrt:recalloc.obj
 0003:00003414       $pdata$wcscat_s            0000000180074414     libucrt:wcscat_s.obj
 0003:00003420       $pdata$_cwait              0000000180074420     libucrt:wait.obj
 0003:0000342c       $pdata$__acrt_wgetpath     000000018007442c     libucrt:getpath.obj
 0003:00003438       $pdata$??$__acrt_mbs_to_wcs_cp@U__crt_win32_buffer_internal_dynamic_resizing@@@@YAHQEBDAEAV?$__crt_win32_buffer@_WU__crt_win32_buffer_internal_dynamic_resizing@@@@I@Z 0000000180074438     libucrt:createprocessa.obj
 0003:00003444       $pdata$__acrt_initialize_locks 0000000180074444     libucrt:locks.obj
 0003:00003450       $pdata$__acrt_uninitialize_locks 0000000180074450     libucrt:locks.obj
 0003:0000345c       $pdata$_waccess_s          000000018007445c     libucrt:waccess.obj
 0003:00003468       $pdata$_pipe               0000000180074468     libucrt:pipe.obj
 0003:00003474       $pdata$??$common_fdopen@_W@@YAPEAU_iobuf@@HQEB_W@Z 0000000180074474     libucrt:fdopen.obj
 0003:00003480       $pdata$??$?RV<lambda_a37b2b86f63e897a80ea819b0eb08c01>@@AEAV<lambda_38ce7e780aa69e748d6df282ebc68efe>@@V<lambda_99fb1378e971ab6e7edea83e3a7a83a2>@@@?$__crt_seh_guarded_call@H@@QEAAH$$QEAV<lambda_a37b2b86f63e897a80ea819b0eb08c01>@@AEAV<lambda_38ce7e780aa69e748d6df282ebc68efe>@@$$QEAV<lambda_99fb1378e971ab6e7edea83e3a7a83a2>@@@Z 0000000180074480     libucrt:commit.obj
 0003:0000348c       $pdata$_commit             000000018007448c     libucrt:commit.obj
 0003:00003498       $pdata$?write_double_translated_ansi_nolock@@YA?AUwrite_result@?A0x17268360@@HQEBDI@Z 0000000180074498     libucrt:write.obj
 0003:000034a4       $pdata$?write_text_ansi_nolock@@YA?AUwrite_result@?A0x17268360@@HQEBDI@Z 00000001800744a4     libucrt:write.obj
 0003:000034b0       $pdata$?write_text_utf16le_nolock@@YA?AUwrite_result@?A0x17268360@@HQEBDI@Z 00000001800744b0     libucrt:write.obj
 0003:000034bc       $pdata$?write_text_utf8_nolock@@YA?AUwrite_result@?A0x17268360@@HQEBDI@Z 00000001800744bc     libucrt:write.obj
 0003:000034c8       $pdata$_write              00000001800744c8     libucrt:write.obj
 0003:000034d4       $pdata$_write_nolock       00000001800744d4     libucrt:write.obj
 0003:000034e0       $pdata$??$write_buffer_nolock@D@@YA_NDV__crt_stdio_stream@@@Z 00000001800744e0     libucrt:_flsbuf.obj
 0003:000034ec       $pdata$?stream_is_at_end_of_file_nolock@@YA_NV__crt_stdio_stream@@@Z 00000001800744ec     libucrt:_flsbuf.obj
 0003:000034f8       $pdata$__acrt_stdio_flush_and_write_narrow_nolock 00000001800744f8     libucrt:_flsbuf.obj
 0003:00003504       $pdata$??$common_xtox@_KD@@YAH_KQEAD0I_N@Z 0000000180074504     libucrt:xtoa.obj
 0003:00003510       $pdata$??$common_xtox_s@_KD@@YAH_KQEAD0I_N@Z 0000000180074510     libucrt:xtoa.obj
 0003:0000351c       $pdata$_ui64toa_s          000000018007451c     libucrt:xtoa.obj
 0003:00003528       $pdata$_strdup             0000000180074528     libucrt:strdup.obj
 0003:00003534       $pdata$__acrt_GetTempPathA 0000000180074534     libucrt:gettemppath.obj
 0003:00003540       $pdata$??$common_sopen_dispatch@D@@YAHQEBDHHHQEAHH@Z 0000000180074540     libucrt:open.obj
 0003:0000354c       $pdata$??$common_sopen_dispatch@_W@@YAHQEB_WHHHQEAHH@Z 000000018007454c     libucrt:open.obj
 0003:00003558       $pdata$?configure_text_mode@@YAHHUfile_options@?A0xa9d50aae@@HAEAW4__crt_lowio_text_mode@@@Z 0000000180074558     libucrt:open.obj
 0003:00003564       $pdata$?decode_options@@YA?AUfile_options@?A0xa9d50aae@@HHH@Z 0000000180074564     libucrt:open.obj
 0003:00003570       $pdata$?truncate_ctrl_z_if_present@@YAHH@Z 0000000180074570     libucrt:open.obj
 0003:0000357c       $pdata$_sopen_nolock       000000018007457c     libucrt:open.obj
 0003:00003588       $pdata$_sopen_s            0000000180074588     libucrt:open.obj
 0003:00003594       $pdata$_wsopen_nolock      0000000180074594     libucrt:open.obj
 0003:000035a0       $pdata$_wsopen_s           00000001800745a0     libucrt:open.obj
 0003:000035ac       $pdata$__acrt_uninitialize_tmpfile 00000001800745ac     libucrt:rmtmp.obj
 0003:000035b8       $pdata$_rmtmp              00000001800745b8     libucrt:rmtmp.obj
 0003:000035c4       $pdata$fegetround          00000001800745c4     libucrt:fegetround.obj
 0003:000035d0       $pdata$_wcsnicoll          00000001800745d0     libucrt:wcsnicol.obj
 0003:000035dc       $pdata$_wcsnicoll_l        00000001800745dc     libucrt:wcsnicol.obj
 0003:000035e8       $pdata$??$?RV<lambda_a22f0c497e5168315e06dae667770027>@@AEAV<lambda_a094494068278ba5130ab06e1292f60a>@@V<lambda_24dc10c13f43218c635520766e23e324>@@@?$__crt_seh_guarded_call@_N@@QEAA_N$$QEAV<lambda_a22f0c497e5168315e06dae667770027>@@AEAV<lambda_a094494068278ba5130ab06e1292f60a>@@$$QEAV<lambda_24dc10c13f43218c635520766e23e324>@@@Z 00000001800745e8     libucrt:spawnv.obj
 0003:000035f4       $pdata$??$common_spawnv@_W@@YA_JHQEB_WQEBQEB_W1@Z 00000001800745f4     libucrt:spawnv.obj
 0003:00003600       $pdata$??$execute_command@_W@@YA_JHQEB_WQEBQEB_W1@Z 0000000180074600     libucrt:spawnv.obj
 0003:0000360c       $pdata$??R<lambda_a094494068278ba5130ab06e1292f60a>@@QEBA_NXZ 000000018007460c     libucrt:spawnv.obj
 0003:00003618       $pdata$?accumulate_inheritable_handles@@YA_NQEAPEAEQEA_K_N@Z 0000000180074618     libucrt:spawnv.obj
 0003:00003624       $pdata$??$common_spawnvp@_W@@YA_JHQEB_WQEBQEB_W1@Z 0000000180074624     libucrt:spawnvp.obj
 0003:00003630       $pdata$__acrt_get_process_end_policy 0000000180074630     libucrt:win_policies.obj
 0003:0000363c       $pdata$??$__acrt_wcs_to_mbs_cp@U__crt_win32_buffer_internal_dynamic_resizing@@@@YAHQEB_WAEAV?$__crt_win32_buffer@DU__crt_win32_buffer_internal_dynamic_resizing@@@@I@Z 000000018007463c     libucrt:argv_wildcards.obj
 0003:00003648       $pdata$??$common_expand_argv_wildcards@D@@YAHQEAPEADQEAPEAPEAD@Z 0000000180074648     libucrt:argv_wildcards.obj
 0003:00003654       $pdata$??$copy_and_add_argument_to_buffer@D@@YAHQEBD0_KAEAV?$argument_list@D@?A0x5f5c8891@@@Z 0000000180074654     libucrt:argv_wildcards.obj
 0003:00003660       $pdata$??$expand_argument_wildcards@D@@YAHQEAD0AEAV?$argument_list@D@?A0x5f5c8891@@@Z 0000000180074660     libucrt:argv_wildcards.obj
 0003:0000366c       $pdata$??$__acrt_wcs_to_mbs_cp@U__crt_win32_buffer_no_resizing@@@@YAHQEB_WAEAV?$__crt_win32_buffer@DU__crt_win32_buffer_no_resizing@@@@I@Z 000000018007466c     libucrt:getmodulefilenamea.obj
 0003:00003678       $pdata$__acrt_GetModuleFileNameA 0000000180074678     libucrt:getmodulefilenamea.obj
 0003:00003684       $pdata$??$?RV<lambda_efdfa57d1f175319df784efa44bb7b81>@@AEAV<lambda_5f0a4c1567f8adc6734073e5d1e1b35c>@@V<lambda_2e8a7d3640ea6ccb4c2413664c2db6fd>@@@?$__crt_seh_guarded_call@X@@QEAAX$$QEAV<lambda_efdfa57d1f175319df784efa44bb7b81>@@AEAV<lambda_5f0a4c1567f8adc6734073e5d1e1b35c>@@$$QEAV<lambda_2e8a7d3640ea6ccb4c2413664c2db6fd>@@@Z 0000000180074684     libucrt:mbctype.obj
 0003:00003690       $pdata$?getSystemCP@@YAHH@Z 0000000180074690     libucrt:mbctype.obj
 0003:0000369c       $pdata$?setSBCS@@YAXPEAU__crt_multibyte_data@@@Z 000000018007469c     libucrt:mbctype.obj
 0003:000036a8       $pdata$?setSBUpLow@@YAXPEAU__crt_multibyte_data@@@Z 00000001800746a8     libucrt:mbctype.obj
 0003:000036b4       $pdata$?setmbcp_internal@@YAHH_NQEAU__acrt_ptd@@QEAPEAU__crt_multibyte_data@@@Z 00000001800746b4     libucrt:mbctype.obj
 0003:000036c0       $pdata$?update_thread_multibyte_data_internal@@YAPEAU__crt_multibyte_data@@QEAU__acrt_ptd@@QEAPEAU1@@Z 00000001800746c0     libucrt:mbctype.obj
 0003:000036cc       $pdata$__acrt_initialize_multibyte 00000001800746cc     libucrt:mbctype.obj
 0003:000036d8       $pdata$__acrt_update_thread_multibyte_data 00000001800746d8     libucrt:mbctype.obj
 0003:000036e4       $pdata$_setmbcp_nolock     00000001800746e4     libucrt:mbctype.obj
 0003:000036f0       $pdata$?x_ismbbtype_l@@YAHPEAU__crt_locale_pointers@@IHH@Z 00000001800746f0     libucrt:ismbbyte.obj
 0003:000036fc       $pdata$__acrt_initialize_command_line 00000001800746fc     libucrt:argv_data.obj
 0003:00003708       $pdata$__acrt_WideCharToMultiByte 0000000180074708     libucrt:widechartomultibyte.obj
 0003:00003714       $pdata$__dcrt_get_narrow_environment_from_os 0000000180074714     libucrt:get_environment_from_os.obj
 0003:00003720       $pdata$__dcrt_get_wide_environment_from_os 0000000180074720     libucrt:get_environment_from_os.obj
 0003:0000372c       $pdata$??$common_set_variable_in_environment_nolock@_W@@YAHQEA_WH@Z 000000018007472c     libucrt:setenv.obj
 0003:00003738       $pdata$??$copy_environment@_W@@YAPEAPEA_WQEAPEA_W@Z 0000000180074738     libucrt:setenv.obj
 0003:00003744       $pdata$__acrt_initialize_heap 0000000180074744     libucrt:heap_handle.obj
 0003:00003750       $pdata$__acrt_execute_initializers 0000000180074750     libucrt:shared_initialization.obj
 0003:0000375c       $pdata$__acrt_execute_uninitializers 000000018007475c     libucrt:shared_initialization.obj
 0003:00003768       $pdata$_callnewh           0000000180074768     libucrt:new_handler.obj
 0003:00003774       $pdata$_query_new_handler  0000000180074774     libucrt:new_handler.obj
 0003:00003780       $pdata$??$?RV<lambda_450d765d439847d4c735a33c368b5fc0>@@AEAV<lambda_44731a7d0e6d81c3e6aa82d741081786>@@V<lambda_601a2a7da3b7a96e9554ac7215c4b07c>@@@?$__crt_seh_guarded_call@P6AXH@Z@@QEAAP6AXH@Z$$QEAV<lambda_450d765d439847d4c735a33c368b5fc0>@@AEAV<lambda_44731a7d0e6d81c3e6aa82d741081786>@@$$QEAV<lambda_601a2a7da3b7a96e9554ac7215c4b07c>@@@Z 0000000180074780     libucrt:signal.obj
 0003:0000378c       $pdata$__acrt_get_sigabrt_handler 000000018007478c     libucrt:signal.obj
 0003:00003798       $pdata$raise               0000000180074798     libucrt:signal.obj
 0003:000037a4       $pdata$?__acrt_LCMapStringA_stat@@YAHPEAU__crt_locale_pointers@@PEB_WKPEBDHPEADHHH@Z 00000001800747a4     libucrt:lcmapstringa.obj
 0003:000037b0       $pdata$__acrt_LCMapStringA 00000001800747b0     libucrt:lcmapstringa.obj
 0003:000037bc       $pdata$_isleadbyte_l       00000001800747bc     libucrt:_wctype.obj
 0003:000037c8       $pdata$?__mbrtowc_utf8@__crt_mbstring@@YA_KPEA_WPEBD_KPEAU_Mbstatet@@@Z 00000001800747c8     libucrt:mbrtowc.obj
 0003:000037d4       $pdata$?__mbsrtowcs_utf8@__crt_mbstring@@YA_KPEA_WPEAPEBD_KPEAU_Mbstatet@@@Z 00000001800747d4     libucrt:mbrtowc.obj
 0003:000037e0       $pdata$?__c32rtomb_utf8@__crt_mbstring@@YA_KPEAD_UPEAU_Mbstatet@@@Z 00000001800747e0     libucrt:c32rtomb.obj
 0003:000037ec       $pdata$__acrt_free_locale  00000001800747ec     libucrt:locale_refcounting.obj
 0003:000037f8       $pdata$__acrt_locale_free_lc_time_if_unreferenced 00000001800747f8     libucrt:locale_refcounting.obj
 0003:00003804       $pdata$__acrt_release_locale_ref 0000000180074804     libucrt:locale_refcounting.obj
 0003:00003810       $pdata$__acrt_update_thread_locale_data 0000000180074810     libucrt:locale_refcounting.obj
 0003:0000381c       $pdata$_updatetlocinfoEx_nolock 000000018007481c     libucrt:locale_refcounting.obj
 0003:00003828       $pdata$__acrt_fp_strflt_to_string 0000000180074828     libucrt:_fptostr.obj
 0003:00003834       $pdata$__acrt_fltout       0000000180074834     libucrt:cfout.obj
 0003:00003840       $pdata$_isatty             0000000180074840     libucrt:isatty.obj
 0003:0000384c       $pdata$__acrt_locale_free_monetary 000000018007484c     libucrt:initmon.obj
 0003:00003858       $pdata$__acrt_locale_free_numeric 0000000180074858     libucrt:initnum.obj
 0003:00003864       $pdata$?free_crt_array_internal@@YAXQEAPEBX_K@Z 0000000180074864     libucrt:inittime.obj
 0003:00003870       $pdata$__acrt_locale_free_time 0000000180074870     libucrt:inittime.obj
 0003:0000387c       $pdata$__acrt_GetStringTypeA 000000018007487c     libucrt:getstringtypea.obj
 0003:00003888       $pdata$__acrt_lowio_create_handle_array 0000000180074888     libucrt:osfinfo.obj
 0003:00003894       $pdata$__acrt_lowio_destroy_handle_array 0000000180074894     libucrt:osfinfo.obj
 0003:000038a0       $pdata$__acrt_lowio_ensure_fh_exists 00000001800748a0     libucrt:osfinfo.obj
 0003:000038ac       $pdata$__acrt_lowio_set_os_handle 00000001800748ac     libucrt:osfinfo.obj
 0003:000038b8       $pdata$_alloc_osfhnd       00000001800748b8     libucrt:osfinfo.obj
 0003:000038c4       $pdata$_free_osfhnd        00000001800748c4     libucrt:osfinfo.obj
 0003:000038d0       $pdata$_get_osfhandle      00000001800748d0     libucrt:osfinfo.obj
 0003:000038dc       $pdata$_wcsnicmp           00000001800748dc     libucrt:wcsnicmp.obj
 0003:000038e8       $pdata$_wcsnicmp_l         00000001800748e8     libucrt:wcsnicmp.obj
 0003:000038f4       $pdata$?GetTableIndexFromLocaleName@@YAHPEB_W@Z 00000001800748f4     libucrt:lcidtoname_downlevel.obj
 0003:00003900       $pdata$__acrt_DownlevelLocaleNameToLCID 0000000180074900     libucrt:lcidtoname_downlevel.obj
 0003:0000390c       $pdata$__acrt_LCMapStringW 000000018007490c     libucrt:lcmapstringw.obj
 0003:00003918       $pdata$_msize_base         0000000180074918     libucrt:msize.obj
 0003:00003924       $pdata$_realloc_base       0000000180074924     libucrt:realloc_base.obj
 0003:00003930       $pdata$_get_fmode          0000000180074930     libucrt:setmode.obj
 0003:0000393c       $pdata$_setmode_nolock     000000018007493c     libucrt:setmode.obj
 0003:00003948       $pdata$_putwch_nolock      0000000180074948     libucrt:putwch.obj
 0003:00003954       $pdata$_chsize_nolock      0000000180074954     libucrt:chsize.obj
 0003:00003960       $pdata$__acrt_fenv_set_control 0000000180074960     libucrt:_fenvutils.obj
 0003:0000396c       $pdata$__acrt_CompareStringW 000000018007496c     libucrt:comparestringw.obj
 0003:00003978       $pdata$??$construct_environment_block@_W@@YAHQEBQEB_WQEAPEA_W@Z 0000000180074978     libucrt:cenvarg.obj
 0003:00003984       $pdata$__acrt_pack_wide_command_line_and_environment 0000000180074984     libucrt:cenvarg.obj
 0003:00003990       $pdata$qsort               0000000180074990     libucrt:qsort.obj
 0003:0000399c       $pdata$4$qsort             000000018007499c     libucrt:qsort.obj
 0003:000039a8       $pdata$5$qsort             00000001800749a8     libucrt:qsort.obj
 0003:000039b4       $pdata$_mbsdec_l           00000001800749b4     libucrt:mbsdec.obj
 0003:000039c0       $pdata$?initialize_multibyte@@YAHXZ 00000001800749c0     libucrt:multibyte_initializer.obj
 0003:000039cc       $pdata$?__mbrtoc32_utf8@__crt_mbstring@@YA_KPEA_UPEBD_KPEAU_Mbstatet@@@Z 00000001800749cc     libucrt:mbrtoc32.obj
 0003:000039d8       $pdata$fegetenv            00000001800749d8     libucrt:fegetenv.obj
 0003:000039e4       $pdata$fesetenv            00000001800749e4     libucrt:fesetenv.obj
 0003:000039f0       $pdata$feholdexcept        00000001800749f0     libucrt:feholdexcept.obj
 0003:00003a08       $pdata$__dcrt_lowio_ensure_console_output_initialized 0000000180074a08     libucrt:initcon.obj
 0003:00003a14       $pdata$__dcrt_terminate_console_output 0000000180074a14     libucrt:initcon.obj
 0003:00003a20       $pdata$__dcrt_write_console 0000000180074a20     libucrt:initcon.obj
 0003:00003a2c       $pdata$_call_matherr       0000000180074a2c     libucrt:libm_error.obj
 0003:00003a38       $pdata$_exception_enabled  0000000180074a38     libucrt:libm_error.obj
 0003:00003a44       $pdata$_handle_error       0000000180074a44     libucrt:libm_error.obj
 0003:00003a50       $pdata$__acrt_initialize_fma3 0000000180074a50     libucrt:fma3_available.obj
 0003:00003a5c       $pdata$_log10_special      0000000180074a5c     libucrt:log_special.obj
 0003:00003a68       $pdata$_log_special_common 0000000180074a68     libucrt:log_special.obj
 0003:00003a74       $pdata$_raise_exc          0000000180074a74     libucrt:fpexcept.obj
 0003:00003a80       $pdata$_raise_exc_ex       0000000180074a80     libucrt:fpexcept.obj
 0003:00003a8c       $pdata$_set_errno_from_matherr 0000000180074a8c     libucrt:fpexcept.obj
 0003:00003a98       $pdata$_clrfp              0000000180074a98     libucrt:fpctrl.obj
 0003:00003aa4       $pdata$_ctrlfp             0000000180074aa4     libucrt:fpctrl.obj
 0003:00003ab0       $pdata$_set_statfp         0000000180074ab0     libucrt:fpctrl.obj
 0003:00003abc       $pdata$_statfp             0000000180074abc     libucrt:fpctrl.obj
 0003:00003ac8       $pdata$_IsNonwritableInCurrentImage 0000000180074ac8     LIBCMT:pesect.obj
 0003:00003ad4       $pdata$__GSHandlerCheck    0000000180074ad4     LIBCMT:gshandler.obj
 0003:00003ae0       $pdata$__GSHandlerCheckCommon 0000000180074ae0     LIBCMT:gshandler.obj
 0003:00003af8       $pdata$__GSHandlerCheck_SEH 0000000180074af8     LIBCMT:gshandlerseh.obj
 0003:00003b04       $pdata$__raise_securityfailure 0000000180074b04     LIBCMT:gs_report.obj
 0003:00003b10       $pdata$__report_gsfailure  0000000180074b10     LIBCMT:gs_report.obj
 0003:00003b1c       $pdata$__report_rangecheckfailure 0000000180074b1c     LIBCMT:gs_report.obj
 0003:00003b28       $pdata$__report_securityfailure 0000000180074b28     LIBCMT:gs_report.obj
 0003:00003b34       $pdata$capture_current_context 0000000180074b34     LIBCMT:gs_report.obj
 0003:00003b40       $pdata$capture_previous_context 0000000180074b40     LIBCMT:gs_report.obj
 0003:00003b4c       $pdata$_local_unwind       0000000180074b4c     libvcruntime:jmpuwind.obj
 0003:00003b64       $pdata$?fin$0@?0??dllmain_crt_process_attach@@YAHQEAUHINSTANCE__@@QEAX@Z@4HA 0000000180074b64     LIBCMT:dll_dllmain.obj
 0003:00003b70       $pdata$?fin$0@?0??dllmain_crt_process_detach@@YAH_N@Z@4HA 0000000180074b70     LIBCMT:dll_dllmain.obj
 0003:00003b7c       $pdata$?filt$0@?0??dllmain_dispatch@@YAHQEAUHINSTANCE__@@KQEAX@Z@4HA 0000000180074b7c     LIBCMT:dll_dllmain.obj
 0003:00003b88       $pdata$__scrt_is_nonwritable_in_current_image$filt$0 0000000180074b88     LIBCMT:utility.obj
 0003:00003b94       $pdata$__DestructExceptionObject$filt$0 0000000180074b94     libvcruntime:ehhelpers.obj
 0003:00003ba0       $pdata$?fin$0@?0???$?RV<lambda_c376a267cfb53b6959b3b692ec76b120>@@AEAV<lambda_9a32fed5bf61b6b509b2d3f6003082a1>@@V<lambda_572fbb9fa0ab338edf41edfd4b5fcc8d>@@@?$__crt_seh_guarded_call@H@@QEAAH$$QEAV<lambda_c376a267cfb53b6959b3b692ec76b120>@@AEAV<lambda_9a32fed5bf61b6b509b2d3f6003082a1>@@$$QEAV<lambda_572fbb9fa0ab338edf41edfd4b5fcc8d>@@@Z@4HA 0000000180074ba0     libucrt:fflush.obj
 0003:00003ba0       $pdata$?fin$0@?0???$?RV<lambda_bdbcead8b570fa3d5ec6d9679862a6e5>@@AEAV<lambda_96f4279ff90247a4c5c5d9824f56f8c1>@@V<lambda_4606be27f17b5e5579e09050fab91818>@@@?$__crt_seh_guarded_call@_K@@QEAA_K$$QEAV<lambda_bdbcead8b570fa3d5ec6d9679862a6e5>@@AEAV<lambda_96f4279ff90247a4c5c5d9824f56f8c1>@@$$QEAV<lambda_4606be27f17b5e5579e09050fab91818>@@@Z@4HA 0000000180074ba0     libucrt:fwrite.obj
 0003:00003ba0       $pdata$?fin$0@?0???$?RV<lambda_84ec643ea9557e2f7dc01bb0e9624395>@@AEAV<lambda_ca71763b3c0644891230e4f79ea54fa6>@@V<lambda_439a761618c59b0600e24586724d733b>@@@?$__crt_seh_guarded_call@H@@QEAAH$$QEAV<lambda_84ec643ea9557e2f7dc01bb0e9624395>@@AEAV<lambda_ca71763b3c0644891230e4f79ea54fa6>@@$$QEAV<lambda_439a761618c59b0600e24586724d733b>@@@Z@4HA 0000000180074ba0     libucrt:setvbuf.obj
 0003:00003ba0       $pdata$?fin$0@?0???$?RV<lambda_082dd7c0feb7dbdaf245f261e54a6583>@@AEAV<lambda_f3caf1ecae5fe01a9a1a6239afa44510>@@V<lambda_c640b76c0755ae85b317b35c67c61e6b>@@@?$__crt_seh_guarded_call@H@@QEAAH$$QEAV<lambda_082dd7c0feb7dbdaf245f261e54a6583>@@AEAV<lambda_f3caf1ecae5fe01a9a1a6239afa44510>@@$$QEAV<lambda_c640b76c0755ae85b317b35c67c61e6b>@@@Z@4HA 0000000180074ba0     libucrt:input.obj
 0003:00003ba0       $pdata$?fin$0@?0???$?RV<lambda_842d9ff0dc9ef11c61343bbaebe7f885>@@AEAV<lambda_c5860995281e5c4ce005b3de8f5874ee>@@V<lambda_d90129c13df834fdcbf8d2b88dafcf2d>@@@?$__crt_seh_guarded_call@X@@QEAAX$$QEAV<lambda_842d9ff0dc9ef11c61343bbaebe7f885>@@AEAV<lambda_c5860995281e5c4ce005b3de8f5874ee>@@$$QEAV<lambda_d90129c13df834fdcbf8d2b88dafcf2d>@@@Z@4HA 0000000180074ba0     libucrt:fflush.obj
 0003:00003ba0       $pdata$?fin$0@?0???$?RV<lambda_a62c933ada0517137acf5807a1eeac1f>@@AEAV<lambda_a31071773b9a94e445cbd5d04ef99106>@@V<lambda_56065050dbf3ada7e59a83db45153de3>@@@?$__crt_seh_guarded_call@H@@QEAAH$$QEAV<lambda_a62c933ada0517137acf5807a1eeac1f>@@AEAV<lambda_a31071773b9a94e445cbd5d04ef99106>@@$$QEAV<lambda_56065050dbf3ada7e59a83db45153de3>@@@Z@4HA 0000000180074ba0     libucrt:output.obj
 0003:00003bac       $pdata$?fin$0@?0???$common_fsopen@_W@@YAPEAU_iobuf@@QEB_W0H@Z@4HA 0000000180074bac     libucrt:fopen.obj
 0003:00003bb8       $pdata$fclose$fin$0        0000000180074bb8     libucrt:fclose.obj
 0003:00003bb8       $pdata$clearerr_s$fin$0    0000000180074bb8     libucrt:clearerr.obj
 0003:00003bb8       $pdata$rewind$fin$0        0000000180074bb8     libucrt:rewind.obj
 0003:00003bb8       $pdata$?fin$0@?0???$common_ftell@J@@YAJV__crt_stdio_stream@@@Z@4HA 0000000180074bb8     libucrt:ftell.obj
 0003:00003bb8       $pdata$?fin$0@?0??common_fseek@@YAHV__crt_stdio_stream@@_JH@Z@4HA 0000000180074bb8     libucrt:fseek.obj
 0003:00003bc4       $pdata$common_control87$filt$0 0000000180074bc4     libucrt:ieee.obj
 0003:00003bc4       $pdata$_ctrlfp$filt$0      0000000180074bc4     libucrt:fpctrl.obj
 0003:00003bd0       $pdata$?fin$0@?0???$common_freopen@_W@@YAHQEAPEAU_iobuf@@QEB_W1V__crt_stdio_stream@@H@Z@4HA 0000000180074bd0     libucrt:freopen.obj
 0003:00003bdc       $pdata$fread_s$fin$0       0000000180074bdc     libucrt:fread.obj
 0003:00003be8       $pdata$fgetc$fin$0         0000000180074be8     libucrt:fgetc.obj
 0003:00003bf4       $pdata$ungetc$fin$0        0000000180074bf4     libucrt:ungetc.obj
 0003:00003c00       $pdata$?fin$0@?0???$common_popen@_W@@YAPEAU_iobuf@@QEB_W0@Z@4HA 0000000180074c00     libucrt:popen.obj
 0003:00003c0c       $pdata$_pclose$fin$0       0000000180074c0c     libucrt:popen.obj
 0003:00003c18       $pdata$?fin$0@?0???$?RV<lambda_886d6c58226a84441f68b9f2b8217b83>@@AEAV<lambda_ab61a845afdef5b7c387490eaf3616ee>@@V<lambda_f7f22ab5edc0698d5f6905b0d3f44752>@@@?$__crt_seh_guarded_call@X@@QEAAX$$QEAV<lambda_886d6c58226a84441f68b9f2b8217b83>@@AEAV<lambda_ab61a845afdef5b7c387490eaf3616ee>@@$$QEAV<lambda_f7f22ab5edc0698d5f6905b0d3f44752>@@@Z@4HA 0000000180074c18     libucrt:fflush.obj
 0003:00003c24       $pdata$?fin$0@?0???$common_fgets@D@@YAPEADQEADHV__crt_stdio_stream@@@Z@4HA 0000000180074c24     libucrt:fgets.obj
 0003:00003c30       $pdata$?fin$0@?0??common_tmpfile@@YAHQEAPEAU_iobuf@@H@Z@4HA 0000000180074c30     libucrt:tmpfile.obj
 0003:00003c3c       $pdata$?fin$0@?0??common_tmpfile_nolock@@YAHQEAPEAU_iobuf@@H@Z@4HA 0000000180074c3c     libucrt:tmpfile.obj
 0003:00003c48       $pdata$?fin$0@?0???$common_dupenv_s@_W@@YAHQEAPEA_WQEA_KQEB_WHQEBDH@Z@4HA 0000000180074c48     libucrt:getenv.obj
 0003:00003c54       $pdata$?fin$0@?0???$common_getenv@_W@@YAPEA_WQEB_W@Z@4HA 0000000180074c54     libucrt:getenv.obj
 0003:00003c60       $pdata$?fin$0@?0???$?RV<lambda_7777bce6b2f8c936911f934f8298dc43>@@AEAV<lambda_f03950bc5685219e0bcd2087efbe011e>@@V<lambda_3883c3dff614d5e0c5f61bb1ac94921c>@@@?$__crt_seh_guarded_call@H@@QEAAH$$QEAV<lambda_7777bce6b2f8c936911f934f8298dc43>@@AEAV<lambda_f03950bc5685219e0bcd2087efbe011e>@@$$QEAV<lambda_3883c3dff614d5e0c5f61bb1ac94921c>@@@Z@4HA 0000000180074c60     libucrt:onexit.obj
 0003:00003c60       $pdata$?fin$0@?0???$?RV<lambda_f2e299630e499de9f9a165e60fcd3db5>@@AEAV<lambda_2ae9d31cdba2644fcbeaf08da7c24588>@@V<lambda_40d01ff24d0e7b3814fdbdcee8eab3c7>@@@?$__crt_seh_guarded_call@X@@QEAAX$$QEAV<lambda_f2e299630e499de9f9a165e60fcd3db5>@@AEAV<lambda_2ae9d31cdba2644fcbeaf08da7c24588>@@$$QEAV<lambda_40d01ff24d0e7b3814fdbdcee8eab3c7>@@@Z@4HA 0000000180074c60     libucrt:per_thread_data.obj
 0003:00003c60       $pdata$?fin$0@?0???$?RV<lambda_aa87e3671a710a21b5dc78c0bdf72e11>@@AEAV<lambda_92619d2358a28f41a33ba319515a20b9>@@V<lambda_6992ecaafeb10aed2b74cb1fae11a551>@@@?$__crt_seh_guarded_call@X@@QEAAX$$QEAV<lambda_aa87e3671a710a21b5dc78c0bdf72e11>@@AEAV<lambda_92619d2358a28f41a33ba319515a20b9>@@$$QEAV<lambda_6992ecaafeb10aed2b74cb1fae11a551>@@@Z@4HA 0000000180074c60     libucrt:per_thread_data.obj
 0003:00003c60       $pdata$?fin$0@?0???$?RV<lambda_0ae27a3a962d80f24befdcbee591983d>@@AEAV<lambda_8d0ee55de4b1038c4002e0adecdf1839>@@V<lambda_dc504788e8f1664fe9b84e20bfb512f2>@@@?$__crt_seh_guarded_call@X@@QEAAX$$QEAV<lambda_0ae27a3a962d80f24befdcbee591983d>@@AEAV<lambda_8d0ee55de4b1038c4002e0adecdf1839>@@$$QEAV<lambda_dc504788e8f1664fe9b84e20bfb512f2>@@@Z@4HA 0000000180074c60     libucrt:per_thread_data.obj
 0003:00003c60       $pdata$?fin$0@?0???$?RV<lambda_450d765d439847d4c735a33c368b5fc0>@@AEAV<lambda_44731a7d0e6d81c3e6aa82d741081786>@@V<lambda_601a2a7da3b7a96e9554ac7215c4b07c>@@@?$__crt_seh_guarded_call@P6AXH@Z@@QEAAP6AXH@Z$$QEAV<lambda_450d765d439847d4c735a33c368b5fc0>@@AEAV<lambda_44731a7d0e6d81c3e6aa82d741081786>@@$$QEAV<lambda_601a2a7da3b7a96e9554ac7215c4b07c>@@@Z@4HA 0000000180074c60     libucrt:signal.obj
 0003:00003c60       $pdata$?fin$0@?0???$?RV<lambda_2d41944a1d46af3157314b8a01080d33>@@AEAV<lambda_8f455de75cd7d7f24b4096f044d8b9e6>@@V<lambda_aa500f224e6afead328df44964fe2772>@@@?$__crt_seh_guarded_call@X@@QEAAX$$QEAV<lambda_2d41944a1d46af3157314b8a01080d33>@@AEAV<lambda_8f455de75cd7d7f24b4096f044d8b9e6>@@$$QEAV<lambda_aa500f224e6afead328df44964fe2772>@@@Z@4HA 0000000180074c60     libucrt:per_thread_data.obj
 0003:00003c60       $pdata$?fin$0@?0???$?RV<lambda_a22f0c497e5168315e06dae667770027>@@AEAV<lambda_a094494068278ba5130ab06e1292f60a>@@V<lambda_24dc10c13f43218c635520766e23e324>@@@?$__crt_seh_guarded_call@_N@@QEAA_N$$QEAV<lambda_a22f0c497e5168315e06dae667770027>@@AEAV<lambda_a094494068278ba5130ab06e1292f60a>@@$$QEAV<lambda_24dc10c13f43218c635520766e23e324>@@@Z@4HA 0000000180074c60     libucrt:spawnv.obj
 0003:00003c60       $pdata$?fin$0@?0???$?RV<lambda_d80eeec6fff315bfe5c115232f3240e3>@@AEAV<lambda_6e4b09c48022b2350581041d5f6b0c4c>@@V<lambda_2358e3775559c9db80273638284d5e45>@@@?$__crt_seh_guarded_call@X@@QEAAX$$QEAV<lambda_d80eeec6fff315bfe5c115232f3240e3>@@AEAV<lambda_6e4b09c48022b2350581041d5f6b0c4c>@@$$QEAV<lambda_2358e3775559c9db80273638284d5e45>@@@Z@4HA 0000000180074c60     libucrt:exit.obj
 0003:00003c60       $pdata$?fin$0@?0???$?RV<lambda_efdfa57d1f175319df784efa44bb7b81>@@AEAV<lambda_5f0a4c1567f8adc6734073e5d1e1b35c>@@V<lambda_2e8a7d3640ea6ccb4c2413664c2db6fd>@@@?$__crt_seh_guarded_call@X@@QEAAX$$QEAV<lambda_efdfa57d1f175319df784efa44bb7b81>@@AEAV<lambda_5f0a4c1567f8adc6734073e5d1e1b35c>@@$$QEAV<lambda_2e8a7d3640ea6ccb4c2413664c2db6fd>@@@Z@4HA 0000000180074c60     libucrt:mbctype.obj
 0003:00003c6c       $pdata$?filt$0@?0???R<lambda_6e4b09c48022b2350581041d5f6b0c4c>@@QEBA@XZ@4HA 0000000180074c6c     libucrt:exit.obj
 0003:00003c78       $pdata$?fin$0@?0???$?RV<lambda_410d79af7f07d98d83a3f525b3859a53>@@AEAV<lambda_3e16ef9562a7dcce91392c22ab16ea36>@@V<lambda_38119f0e861e05405d8a144b9b982f0a>@@@?$__crt_seh_guarded_call@X@@QEAAX$$QEAV<lambda_410d79af7f07d98d83a3f525b3859a53>@@AEAV<lambda_3e16ef9562a7dcce91392c22ab16ea36>@@$$QEAV<lambda_38119f0e861e05405d8a144b9b982f0a>@@@Z@4HA 0000000180074c78     libucrt:wsetlocale.obj
 0003:00003c84       $pdata$_alloc_osfhnd$fin$0 0000000180074c84     libucrt:osfinfo.obj
 0003:00003c84       $pdata$__acrt_initialize_lowio$fin$0 0000000180074c84     libucrt:ioinit.obj
 0003:00003c84       $pdata$__acrt_lowio_ensure_fh_exists$fin$0 0000000180074c84     libucrt:osfinfo.obj
 0003:00003c90       $pdata$_fcloseall$fin$0    0000000180074c90     libucrt:closeall.obj
 0003:00003c90       $pdata$?fin$0@?0??__acrt_stdio_allocate_stream@@YA?AV__crt_stdio_stream@@XZ@4HA 0000000180074c90     libucrt:stream.obj
 0003:00003c9c       $pdata$?fin$0@?0???$?RV<lambda_751a882b2c74d4b022dec766aa51a29a>@@AEAV<lambda_628dfdc04ba53c8bfc02c9951375f3f5>@@V<lambda_f6c7be5f7998530c34de24c7437d6b54>@@@?$__crt_seh_guarded_call@H@@QEAAH$$QEAV<lambda_751a882b2c74d4b022dec766aa51a29a>@@AEAV<lambda_628dfdc04ba53c8bfc02c9951375f3f5>@@$$QEAV<lambda_f6c7be5f7998530c34de24c7437d6b54>@@@Z@4HA 0000000180074c9c     libucrt:close.obj
 0003:00003c9c       $pdata$?fin$0@?0???$?RV<lambda_a37b2b86f63e897a80ea819b0eb08c01>@@AEAV<lambda_38ce7e780aa69e748d6df282ebc68efe>@@V<lambda_99fb1378e971ab6e7edea83e3a7a83a2>@@@?$__crt_seh_guarded_call@H@@QEAAH$$QEAV<lambda_a37b2b86f63e897a80ea819b0eb08c01>@@AEAV<lambda_38ce7e780aa69e748d6df282ebc68efe>@@$$QEAV<lambda_99fb1378e971ab6e7edea83e3a7a83a2>@@@Z@4HA 0000000180074c9c     libucrt:commit.obj
 0003:00003ca8       $pdata$_read$fin$0         0000000180074ca8     libucrt:read.obj
 0003:00003cb4       $pdata$_write$fin$0        0000000180074cb4     libucrt:write.obj
 0003:00003cb4       $pdata$?fin$0@?0???$common_lseek@J@@YAJHJH@Z@4HA 0000000180074cb4     libucrt:lseek.obj
 0003:00003cb4       $pdata$?fin$0@?0???$common_lseek@_J@@YA_JH_JH@Z@4HA 0000000180074cb4     libucrt:lseek.obj
 0003:00003cc0       $pdata$_pipe$fin$1         0000000180074cc0     libucrt:pipe.obj
 0003:00003ccc       $pdata$_pipe$fin$0         0000000180074ccc     libucrt:pipe.obj
 0003:00003cd8       $pdata$?fin$0@?0???$common_fdopen@_W@@YAPEAU_iobuf@@HQEB_W@Z@4HA 0000000180074cd8     libucrt:fdopen.obj
 0003:00003ce4       $pdata$?fin$0@?0???$common_sopen_dispatch@D@@YAHQEBDHHHQEAHH@Z@4HA 0000000180074ce4     libucrt:open.obj
 0003:00003ce4       $pdata$?fin$0@?0???$common_sopen_dispatch@_W@@YAHQEB_WHHHQEAHH@Z@4HA 0000000180074ce4     libucrt:open.obj
 0003:00003cf0       $pdata$_rmtmp$fin$0        0000000180074cf0     libucrt:rmtmp.obj
 0003:00003cfc       $pdata$_rmtmp$fin$1        0000000180074cfc     libucrt:rmtmp.obj
 0003:00003d08       $pdata$?fin$0@?0??update_thread_multibyte_data_internal@@YAPEAU__crt_multibyte_data@@QEAU__acrt_ptd@@QEAPEAU1@@Z@4HA 0000000180074d08     libucrt:mbctype.obj
 0003:00003d14       $pdata$_query_new_handler$fin$0 0000000180074d14     libucrt:new_handler.obj
 0003:00003d20       $pdata$raise$fin$0         0000000180074d20     libucrt:signal.obj
 0003:00003d2c       $pdata$__acrt_update_thread_locale_data$fin$0 0000000180074d2c     libucrt:locale_refcounting.obj
 0003:00003d38       $pdata$_IsNonwritableInCurrentImage$filt$0 0000000180074d38     LIBCMT:pesect.obj
 0004:0000131c       .idata$6                   000000018007631c     kernel32:KERNEL32.dll
 0004:00001338       .idata$6                   0000000180076338     user32:USER32.dll
 0004:000013dc       .idata$6                   00000001800763dc     advapi32:ADVAPI32.dll
 0004:0000140e       .idata$6                   000000018007640e     shell32:SHELL32.dll
 0004:000019b6       .idata$6                   00000001800769b6     lua51:lua51.dll
 0004:00001a02       .idata$6                   0000000180076a02     rpcrt4:RPCRT4.dll
 0005:00000060       $R000000                   0000000180077060     luafar3.res
